 CryLobby

 Timestamp is 5036e412 (Fri Aug 24 04:16:50 2012)

 Preferred load address is 0000000039a00000

 Start         Length     Name                   Class
 0001:00000000 000a2610H .text                   CODE
 0001:000a2610 00000092H .text$x                 CODE
 0001:000a26b0 0000034cH .text$yc                CODE
 0001:000a2a00 00000dcbH .text$yd                CODE
 0002:00000000 00000578H .idata$5                DATA
 0002:00000578 00000008H .CRT$XCA                DATA
 0002:00000580 00000178H .CRT$XCU                DATA
 0002:000006f8 00000008H .CRT$XCZ                DATA
 0002:00000700 00000008H .CRT$XIA                DATA
 0002:00000708 00000008H .CRT$XIAA               DATA
 0002:00000710 00000008H .CRT$XIZ                DATA
 0002:00000720 0000b770H .rdata                  DATA
 0002:0000be90 00000053H .rdata$debug            DATA
 0002:0000bee8 00000008H .rtc$IAA                DATA
 0002:0000bef0 00000008H .rtc$IZZ                DATA
 0002:0000bef8 00000008H .rtc$TAA                DATA
 0002:0000bf00 00000008H .rtc$TZZ                DATA
 0002:0000bf08 0000c86cH .xdata                  DATA
 0002:00018774 000000a0H .idata$2                DATA
 0002:00018814 00000014H .idata$3                DATA
 0002:00018828 00000578H .idata$4                DATA
 0002:00018da0 00000854H .idata$6                DATA
 0002:00019600 00000072H .edata                  DATA
 0003:00000000 00002410H .data                   DATA
 0003:00002420 000145b0H .bss                    DATA
 0004:00000000 0000c3ccH .pdata                  DATA
 0005:00000000 00000008H .tls$                   DATA
 0006:00000000 00000058H .rsrc$01                DATA
 0006:00000060 00000210H .rsrc$02                DATA

  Address         Publics by Value              Rva+Base               Lib:Object

 0000:00000000       ___safe_se_handler_table   0000000000000000     <absolute>
 0000:00000000       ___safe_se_handler_count   0000000000000000     <absolute>
 0000:00000000       __ImageBase                0000000039a00000     <linker-defined>
 0001:00000000       ?CryFatalError@@YAXPEBDZZ  0000000039a01000 f i CryDedicatedServer.obj
 0001:000000a0       ??_GIJob@CWorkQueue@@UEAAPEAXI@Z 0000000039a010a0 f i CryDLCStore.obj
 0001:000000a0       ??_EIJob@CWorkQueue@@UEAAPEAXI@Z 0000000039a010a0 f i CryDLCStore.obj
 0001:000000d0       ??_GCDummyMemReplay@@UEAAPEAXI@Z 0000000039a010d0 f i CryDLCStore.obj
 0001:000000d0       ??_ECDummyMemReplay@@UEAAPEAXI@Z 0000000039a010d0 f i CryDLCStore.obj
 0001:000000d0       ??_GIMemReplay@@UEAAPEAXI@Z 0000000039a010d0 f i CryDLCStore.obj
 0001:000000d0       ??_EIMemReplay@@UEAAPEAXI@Z 0000000039a010d0 f i CryDLCStore.obj
 0001:00000100       ?Initialise@CCryDLCStore@@UEAA?AW4ECryLobbyError@@XZ 0000000039a01100 f   CryDLCStore.obj
 0001:00000160       ?StartTask@CCryDLCStore@@AEAA?AW4ECryLobbyError@@IPEAI0IPEAX1@Z 0000000039a01160 f   CryDLCStore.obj
 0001:00000230       ?CreateTask@CCryDLCStore@@EEAAXPEAUSTask@1@IIIPEAX1@Z 0000000039a01230 f   CryDLCStore.obj
 0001:00000290       ?StartSubTask@CCryDLCStore@@IEAAXII@Z 0000000039a01290 f   CryDLCStore.obj
 0001:000002a0       ?StartSubTask@CCryDLCStore@@IEAAXIPEAUSTask@1@@Z 0000000039a012a0 f   CryDLCStore.obj
 0001:000002b0       ?FreeTask@CCryDLCStore@@MEAAXI@Z 0000000039a012b0 f   CryDLCStore.obj
 0001:00000350       ?ClearTask@CCryDLCStore@@MEAAXI@Z 0000000039a01350 f   CryDLCStore.obj
 0001:000003a0       ?CreateTaskParamMem@CCryDLCStore@@IEAA?AW4ECryLobbyError@@PEAUSTask@1@IPEBX_K@Z 0000000039a013a0 f   CryDLCStore.obj
 0001:00000430       ?UpdateTaskError@CCryDLCStore@@KAXPEAUSTask@1@W4ECryLobbyError@@@Z 0000000039a01430 f   CryDLCStore.obj
 0001:00000440       ?SetDownloadableVerifyCallback@CCryDLCStore@@UEAAXP6AXAEBUSCryDLCDownloadableInfo@@PEAV?$CryFixedStringT@$0BAE@@@PEA_N@Z@Z 0000000039a01440 f   CryDLCStore.obj
 0001:00000450       ?StartTaskRefreshingCatalog@CCryDLCStore@@IEAA_NI@Z 0000000039a01450 f   CryDLCStore.obj
 0001:00000480       ?StopTaskRefreshingCatalog@CCryDLCStore@@IEAA_NI@Z 0000000039a01480 f   CryDLCStore.obj
 0001:000004b0       ?StartTaskUsingCatalog@CCryDLCStore@@IEAA_NI@Z 0000000039a014b0 f   CryDLCStore.obj
 0001:000004f0       ?StopTaskUsingCatalog@CCryDLCStore@@IEAA_NI@Z 0000000039a014f0 f   CryDLCStore.obj
 0001:00000520       ?StartTaskReleasingCatalog@CCryDLCStore@@IEAA_NI@Z 0000000039a01520 f   CryDLCStore.obj
 0001:00000550       ?StopTaskReleasingCatalog@CCryDLCStore@@IEAA_NI@Z 0000000039a01550 f   CryDLCStore.obj
 0001:00000580       ?FreeOrderHandle@CCryDLCStore@@MEAAXI@Z 0000000039a01580 f   CryDLCStore.obj
 0001:00000590       ?CryLog@@YAXPEBDZZ         0000000039a01590 f i CryDLCStore.obj
 0001:000005f0       ?OnGameSpyObjectAvailable@CCryGameSpySBQR2Friends@@UEAAXW4EGameSpyObjectBit@ICryGameSpySBQR2LobbyComponent@@@Z 0000000039a015f0 f i CryGameSpySBQR2Friends.obj
 0001:000005f0       ?FBool@?$CGameSpySDKRef@VCGameSpySBQR2NATNegotiation@@@@AEAAXXZ 0000000039a015f0 f i GameSpySBQR2NatNegotiation.obj
 0001:000005f0       ?AddLabel@CDummyMemReplay@@UEAAXPEBD@Z 0000000039a015f0 f i CryDLCStore.obj
 0001:000005f0       ?UnMarkPool@CDummyMemReplay@@UEAAXHPEAX@Z 0000000039a015f0 f i CryDLCStore.obj
 0001:000005f0       ?AddHostMigrationEventListener@CCryLobby@@UEAAXPEAUIHostMigrationEventListener@@PEBDI@Z 0000000039a015f0 f i CryLobby.obj
 0001:000005f0       ?PushToTalkButtonUp@CCryVoice@@UEAAXI@Z 0000000039a015f0 f i CryVoice.obj
 0001:000005f0       ?AddTexturePoolContext@CDummyMemReplay@@UEAAXPEAXHHHPEBDI@Z 0000000039a015f0 f i CryDLCStore.obj
 0001:000005f0       ?LobbyAddrIDTick@ICryMatchMakingPrivate@@UEAAXXZ 0000000039a015f0 f i CryMatchMaking.obj
 0001:000005f0       ?OnGameSpyObjectAvailable@CCryGameSpySBQR2Voice@@UEAAXW4EGameSpyObjectBit@ICryGameSpySBQR2LobbyComponent@@@Z 0000000039a015f0 f i CryGameSpySBQR2Voice.obj
 0001:000005f0       gpiPeerPingReplyCallback   0000000039a015f0 f i GameSpy_2.11.00_VC10:gpiPeer.obj
 0001:000005f0       ?Tick@CCrySignIn@@UEAAXVCTimeValue@@@Z 0000000039a015f0 f i CrySignIn.obj
 0001:000005f0       ?OnGameSpyObjectAvailable@CCryGameSpySBQR2FriendsManagement@@UEAAXW4EGameSpyObjectBit@ICryGameSpySBQR2LobbyComponent@@@Z 0000000039a015f0 f i CryGameSpySBQR2FriendsManagement.obj
 0001:000005f0       ?OnGameSpyObjectUnavailable@CCryGameSpySBQR2Stats@@UEAAXW4EGameSpyObjectBit@ICryGameSpySBQR2LobbyComponent@@@Z 0000000039a015f0 f i CryGameSpySBQR2Stats.obj
 0001:000005f0       ?RegisterContainer@CDummyMemReplay@@UEAAXPEBXH@Z 0000000039a015f0 f i CryDLCStore.obj
 0001:000005f0       ?BanCmd@CCryMatchMaking@@UEAAXPEBDM@Z 0000000039a015f0 f i CryMatchMaking.obj
 0001:000005f0       ?AddAllocReference@CDummyMemReplay@@UEAAXPEAX0@Z 0000000039a015f0 f i CryDLCStore.obj
 0001:000005f0       ?RemoveContext@CDummyMemReplay@@UEAAXXZ 0000000039a015f0 f i CryDLCStore.obj
 0001:000005f0       ?UnregisterContainer@CDummyMemReplay@@UEAAXPEBX@Z 0000000039a015f0 f i CryDLCStore.obj
 0001:000005f0       ?SetVoicePlaybackVolume@CCryVoice@@UEAAXIM@Z 0000000039a015f0 f i CryVoice.obj
 0001:000005f0       ?RemoveAllocReference@CDummyMemReplay@@UEAAXPEAX@Z 0000000039a015f0 f i CryDLCStore.obj
 0001:000005f0       ?GetMemoryStatistics@?$VTableImpl@USNullAddr@@$0A@U?$IVisitor@V?$CNode@USNullAddr@@V?$CNode@GV?$CNode@USIPv4Addr@@V?$CNode@ULobbyIdAddr@@VCEnd@NTypelist@@@NTypelist@@@NTypelist@@@NTypelist@@@NTypelist@@@NConfigurableVariantHelpers@@U?$IMutatingVisitor@V?$CNode@USNullAddr@@V?$CNode@GV?$CNode@USIPv4Addr@@V?$CNode@ULobbyIdAddr@@VCEnd@NTypelist@@@NTypelist@@@NTypelist@@@NTypelist@@@NTypelist@@@3@@NConfigurableVariantHelpers@@SAXPEAVICrySizer@@PEBX@Z 0000000039a015f0 f i CryLobby.obj
 0001:000005f0       ?ExitScope_Alloc@CDummyMemReplay@@UEAAX_K00@Z 0000000039a015f0 f i CryDLCStore.obj
 0001:000005f0       ?MarkBucket@CDummyMemReplay@@UEAAXH_KPEAX0@Z 0000000039a015f0 f i CryDLCStore.obj
 0001:000005f0       ?Stop@CDummyMemReplay@@UEAAXXZ 0000000039a015f0 f i CryDLCStore.obj
 0001:000005f0       ?BindToContainer@CDummyMemReplay@@UEAAXPEBX0@Z 0000000039a015f0 f i CryDLCStore.obj
 0001:000005f0       ?LobbyAddrIDRecv@ICryMatchMakingPrivate@@UEAAXP6AXPEAXPEAEI_KAEAV?$CConfigurableVariant@V?$CNode@USNullAddr@@V?$CNode@GV?$CNode@USIPv4Addr@@V?$CNode@ULobbyIdAddr@@VCEnd@NTypelist@@@NTypelist@@@NTypelist@@@NTypelist@@@NTypelist@@$07VCDefaultVariantConversion@NConfigurableVariantHelpers@@VCDefaultVariantConstruction@4@@@@Z0@Z 0000000039a015f0 f i CryMatchMaking.obj
 0001:000005f0       ?Destruct@?$VTableImpl@G$0A@U?$IVisitor@V?$CNode@USNullAddr@@V?$CNode@GV?$CNode@USIPv4Addr@@V?$CNode@ULobbyIdAddr@@VCEnd@NTypelist@@@NTypelist@@@NTypelist@@@NTypelist@@@NTypelist@@@NConfigurableVariantHelpers@@U?$IMutatingVisitor@V?$CNode@USNullAddr@@V?$CNode@GV?$CNode@USIPv4Addr@@V?$CNode@ULobbyIdAddr@@VCEnd@NTypelist@@@NTypelist@@@NTypelist@@@NTypelist@@@NTypelist@@@2@@NConfigurableVariantHelpers@@SAXPEAX@Z 0000000039a015f0 f i CryGameSpySBQR2MatchMaking.obj
 0001:000005f0       ?GetInfo@CDummyMemReplay@@UEAAXAEAUCryReplayInfo@@@Z 0000000039a015f0 f i CryDLCStore.obj
 0001:000005f0       ?ConstructClone@?$VTableImpl@USNullAddr@@$0A@U?$IVisitor@V?$CNode@USNullAddr@@V?$CNode@GV?$CNode@USIPv4Addr@@V?$CNode@ULobbyIdAddr@@VCEnd@NTypelist@@@NTypelist@@@NTypelist@@@NTypelist@@@NTypelist@@@NConfigurableVariantHelpers@@U?$IMutatingVisitor@V?$CNode@USNullAddr@@V?$CNode@GV?$CNode@USIPv4Addr@@V?$CNode@ULobbyIdAddr@@VCEnd@NTypelist@@@NTypelist@@@NTypelist@@@NTypelist@@@NTypelist@@@3@@NConfigurableVariantHelpers@@SAXPEAXPEBX@Z 0000000039a015f0 f i CryLobby.obj
 0001:000005f0       ?OnBannedUserListChanged@CCryMatchMaking@@UEAAXXZ 0000000039a015f0 f i CryMatchMaking.obj
 0001:000005f0       ?OnGameSpyObjectAvailable@CCryGameSpySBQR2SignIn@@UEAAXW4EGameSpyObjectBit@ICryGameSpySBQR2LobbyComponent@@@Z 0000000039a015f0 f i CryGameSpySBQR2SignIn.obj
 0001:000005f0       ?Tick@CCryDLCStore@@UEAAXVCTimeValue@@@Z 0000000039a015f0 f i CryDLCStore.obj
 0001:000005f0       ?OnError@CCryGameSpySBQR2LobbyService@@UEAAXAEBV?$CConfigurableVariant@V?$CNode@USNullAddr@@V?$CNode@GV?$CNode@USIPv4Addr@@V?$CNode@ULobbyIdAddr@@VCEnd@NTypelist@@@NTypelist@@@NTypelist@@@NTypelist@@@NTypelist@@$07VCDefaultVariantConversion@NConfigurableVariantHelpers@@VCDefaultVariantConstruction@4@@@W4ESocketError@@@Z 0000000039a015f0 f i CryGameSpySBQR2Lobby.obj
 0001:000005f0       ?OnSystemEvent@CSystemEventListner_CryLobby@@UEAAXW4ESystemEvent@@_K1@Z 0000000039a015f0 f i CryLobbyDLL.obj
 0001:000005f0       ?Flush@CDummyMemReplay@@UEAAXXZ 0000000039a015f0 f i CryDLCStore.obj
 0001:000005f0       ?UnbanCmd@CCryMatchMaking@@UEAAX_K@Z 0000000039a015f0 f i CryMatchMaking.obj
 0001:000005f0       ?SetLeaderboardType@CCryStats@@UEAAXW4ECryLobbyLeaderboardType@@@Z 0000000039a015f0 f i CryStats.obj
 0001:000005f0       ?AllocUsage@CDummyMemReplay@@UEAAXW4Class@EMemReplayAllocClass@@_K1@Z 0000000039a015f0 f i CryDLCStore.obj
 0001:000005f0       ?OnGameSpyObjectCantMakeAvailable@CCryGameSpySBQR2SignIn@@UEAAXW4EGameSpyObjectBit@ICryGameSpySBQR2LobbyComponent@@@Z 0000000039a015f0 f i CryGameSpySBQR2SignIn.obj
 0001:000005f0       ?OnGameSpyObjectUnavailable@CCryGameSpySBQR2Friends@@UEAAXW4EGameSpyObjectBit@ICryGameSpySBQR2LobbyComponent@@@Z 0000000039a015f0 f i CryGameSpySBQR2Friends.obj
 0001:000005f0       ?EnablePushToTalk@CCryVoice@@UEAAXI_N@Z 0000000039a015f0 f i CryVoice.obj
 0001:000005f0       ?MapPage@CDummyMemReplay@@UEAAXPEAX_K@Z 0000000039a015f0 f i CryDLCStore.obj
 0001:000005f0       ?UnMarkBucket@CDummyMemReplay@@UEAAXHPEAX@Z 0000000039a015f0 f i CryDLCStore.obj
 0001:000005f0       ?OnGameSpyObjectCantMakeAvailable@CCryGameSpySBQR2Stats@@UEAAXW4EGameSpyObjectBit@ICryGameSpySBQR2LobbyComponent@@@Z 0000000039a015f0 f i CryGameSpySBQR2Stats.obj
 0001:000005f0       ?OnGameSpyObjectCantMakeAvailable@CCryGameSpySBQR2Friends@@UEAAXW4EGameSpyObjectBit@ICryGameSpySBQR2LobbyComponent@@@Z 0000000039a015f0 f i CryGameSpySBQR2Friends.obj
 0001:000005f0       ?UnMapPage@CDummyMemReplay@@UEAAXPEAX_K@Z 0000000039a015f0 f i CryDLCStore.obj
 0001:000005f0       ?ExitScope_Realloc@CDummyMemReplay@@UEAAX_K000@Z 0000000039a015f0 f i CryDLCStore.obj
 0001:000005f0       gviCodecsCleanup           0000000039a015f0 f i GameSpy_2.11.00_VC10:gvCodec.obj
 0001:000005f0       ?AddScreenshot@CDummyMemReplay@@UEAAXXZ 0000000039a015f0 f i CryDLCStore.obj
 0001:000005f0       ?OnGameSpyObjectUnavailable@CCryGameSpySBQR2FriendsManagement@@UEAAXW4EGameSpyObjectBit@ICryGameSpySBQR2LobbyComponent@@@Z 0000000039a015f0 f i CryGameSpySBQR2FriendsManagement.obj
 0001:000005f0       gsiExitThread              0000000039a015f0 f i GameSpy_2.11.00_VC10:gsPlatformThread.obj
 0001:000005f0       ?SwapContainers@CDummyMemReplay@@UEAAXPEBX0@Z 0000000039a015f0 f i CryDLCStore.obj
 0001:000005f0       ?RemoveHostMigrationEventListener@CCryLobby@@UEAAXPEAUIHostMigrationEventListener@@@Z 0000000039a015f0 f i CryLobby.obj
 0001:000005f0       ?BanCmd@CCryMatchMaking@@UEAAX_KM@Z 0000000039a015f0 f i CryMatchMaking.obj
 0001:000005f0       ?OnGameSpyObjectCantMakeAvailable@CCryGameSpySBQR2Voice@@UEAAXW4EGameSpyObjectBit@ICryGameSpySBQR2LobbyComponent@@@Z 0000000039a015f0 f i CryGameSpySBQR2Voice.obj
 0001:000005f0       ?RegisterFixedAddressRange@CDummyMemReplay@@UEAAXPEAX_KPEBD@Z 0000000039a015f0 f i CryDLCStore.obj
 0001:000005f0       ?DumpSymbols@CDummyMemReplay@@UEAAXXZ 0000000039a015f0 f i CryDLCStore.obj
 0001:000005f0       ?ExitScope_Free@CDummyMemReplay@@UEAAX_K@Z 0000000039a015f0 f i CryDLCStore.obj
 0001:000005f0       ?Destruct@?$VTableImpl@USNullAddr@@$0A@U?$IVisitor@V?$CNode@USNullAddr@@V?$CNode@GV?$CNode@USIPv4Addr@@V?$CNode@ULobbyIdAddr@@VCEnd@NTypelist@@@NTypelist@@@NTypelist@@@NTypelist@@@NTypelist@@@NConfigurableVariantHelpers@@U?$IMutatingVisitor@V?$CNode@USNullAddr@@V?$CNode@GV?$CNode@USIPv4Addr@@V?$CNode@ULobbyIdAddr@@VCEnd@NTypelist@@@NTypelist@@@NTypelist@@@NTypelist@@@NTypelist@@@3@@NConfigurableVariantHelpers@@SAXPEAX@Z 0000000039a015f0 f i CryLobby.obj
 0001:000005f0       ?GetMemoryStatistics@?$VTableImpl@G$0A@U?$IVisitor@V?$CNode@USNullAddr@@V?$CNode@GV?$CNode@USIPv4Addr@@V?$CNode@ULobbyIdAddr@@VCEnd@NTypelist@@@NTypelist@@@NTypelist@@@NTypelist@@@NTypelist@@@NConfigurableVariantHelpers@@U?$IMutatingVisitor@V?$CNode@USNullAddr@@V?$CNode@GV?$CNode@USIPv4Addr@@V?$CNode@ULobbyIdAddr@@VCEnd@NTypelist@@@NTypelist@@@NTypelist@@@NTypelist@@@NTypelist@@@2@@NConfigurableVariantHelpers@@SAXPEAVICrySizer@@PEBX@Z 0000000039a015f0 f i CryGameSpySBQR2MatchMaking.obj
 0001:000005f0       ?AddFrameStart@CDummyMemReplay@@UEAAXXZ 0000000039a015f0 f i CryDLCStore.obj
 0001:000005f0       ?FBool@?$CGameSpySDKRef@VCGameSpySBQR2GPConnection@@@@AEAAXXZ 0000000039a015f0 f i GameSpySBQR2AvailabilityCheck.obj
 0001:000005f0       ??1CCryRebroadcaster@@QEAA@XZ 0000000039a015f0 f i CryRebroadcaster.obj
 0001:000005f0       ?OnGameSpyObjectCantMakeAvailable@CCryGameSpySBQR2FriendsManagement@@UEAAXW4EGameSpyObjectBit@ICryGameSpySBQR2LobbyComponent@@@Z 0000000039a015f0 f i CryGameSpySBQR2FriendsManagement.obj
 0001:000005f0       ?TerminateHostMigration@CCryMatchMaking@@UEAAXI@Z 0000000039a015f0 f i CryMatchMaking.obj
 0001:000005f0       ?OnGameSpyObjectUnavailable@CCryGameSpySBQR2SignIn@@UEAAXW4EGameSpyObjectBit@ICryGameSpySBQR2LobbyComponent@@@Z 0000000039a015f0 f i CryGameSpySBQR2SignIn.obj
 0001:000005f0       ?GetMemoryStatistics@?$VTableImpl@USIPv4Addr@@$0A@U?$IVisitor@V?$CNode@USNullAddr@@V?$CNode@GV?$CNode@USIPv4Addr@@V?$CNode@ULobbyIdAddr@@VCEnd@NTypelist@@@NTypelist@@@NTypelist@@@NTypelist@@@NTypelist@@@NConfigurableVariantHelpers@@U?$IMutatingVisitor@V?$CNode@USNullAddr@@V?$CNode@GV?$CNode@USIPv4Addr@@V?$CNode@ULobbyIdAddr@@VCEnd@NTypelist@@@NTypelist@@@NTypelist@@@NTypelist@@@NTypelist@@@3@@NConfigurableVariantHelpers@@SAXPEAVICrySizer@@PEBX@Z 0000000039a015f0 f i CryLobby.obj
 0001:000005f0       ?Kick@CCryMatchMaking@@UEAAXPEBUCryUserID@@W4EDisconnectionCause@@@Z 0000000039a015f0 f i CryMatchMaking.obj
 0001:000005f0       ?Start@CDummyMemReplay@@UEAAX_NPEBD@Z 0000000039a015f0 f i CryDLCStore.obj
 0001:000005f0       ?UnbanCmd@CCryMatchMaking@@UEAAXPEBD@Z 0000000039a015f0 f i CryMatchMaking.obj
 0001:000005f0       ?AddContextV@CDummyMemReplay@@UEAAXHIPEBDPEAD@Z 0000000039a015f0 f i CryDLCStore.obj
 0001:000005f0       ?Ban@CCryMatchMaking@@UEAAXPEBUCryUserID@@M@Z 0000000039a015f0 f i CryMatchMaking.obj
 0001:000005f0       ?StartOnCommandLine@CDummyMemReplay@@UEAAXPEBD@Z 0000000039a015f0 f i CryDLCStore.obj
 0001:000005f0       ?Clone@?$VTableImpl@USNullAddr@@$0A@U?$IVisitor@V?$CNode@USNullAddr@@V?$CNode@GV?$CNode@USIPv4Addr@@V?$CNode@ULobbyIdAddr@@VCEnd@NTypelist@@@NTypelist@@@NTypelist@@@NTypelist@@@NTypelist@@@NConfigurableVariantHelpers@@U?$IMutatingVisitor@V?$CNode@USNullAddr@@V?$CNode@GV?$CNode@USIPv4Addr@@V?$CNode@ULobbyIdAddr@@VCEnd@NTypelist@@@NTypelist@@@NTypelist@@@NTypelist@@@NTypelist@@@3@@NConfigurableVariantHelpers@@SAXPEAXPEBX@Z 0000000039a015f0 f i CryLobby.obj
 0001:000005f0       ?OnGameSpyObjectAvailable@CCryGameSpySBQR2Stats@@UEAAXW4EGameSpyObjectBit@ICryGameSpySBQR2LobbyComponent@@@Z 0000000039a015f0 f i CryGameSpySBQR2Stats.obj
 0001:000005f0       ?AddContext@CDummyMemReplay@@UEAAXHIPEBD@Z 0000000039a015f0 f i CryDLCStore.obj
 0001:000005f0       ?DumpStats@CDummyMemReplay@@UEAAXXZ 0000000039a015f0 f i CryDLCStore.obj
 0001:000005f0       ?UnbindFromContainer@CDummyMemReplay@@UEAAXPEBX0@Z 0000000039a015f0 f i CryDLCStore.obj
 0001:000005f0       ?PostLocalizationChecks@CCryLobbyUI@@UEAAXXZ 0000000039a015f0 f i CryLobbyUI.obj
 0001:000005f0       ?BoolFunc@CryDLCPaymentMethodID@@AEBAXXZ 0000000039a015f0 f i CryGameSpySBQR2DLCStore.obj
 0001:000005f0       ?BanStatus@CCryMatchMaking@@UEAAXXZ 0000000039a015f0 f i CryMatchMaking.obj
 0001:000005f0       ?PushToTalkButtonDown@CCryVoice@@UEAAXI@Z 0000000039a015f0 f i CryVoice.obj
 0001:000005f0       ?AddSizerTree@CDummyMemReplay@@UEAAXPEBD@Z 0000000039a015f0 f i CryDLCStore.obj
 0001:000005f0       ?ExitScope@CDummyMemReplay@@UEAAXXZ 0000000039a015f0 f i CryDLCStore.obj
 0001:000005f0       ?BucketEnableCleanups@CDummyMemReplay@@UEAAXPEAX_N@Z 0000000039a015f0 f i CryDLCStore.obj
 0001:000005f0       gviResetEncoder            0000000039a015f0 f i GameSpy_2.11.00_VC10:gvCodec.obj
 0001:000005f0       ?Destruct@?$VTableImpl@USIPv4Addr@@$0A@U?$IVisitor@V?$CNode@USNullAddr@@V?$CNode@GV?$CNode@USIPv4Addr@@V?$CNode@ULobbyIdAddr@@VCEnd@NTypelist@@@NTypelist@@@NTypelist@@@NTypelist@@@NTypelist@@@NConfigurableVariantHelpers@@U?$IMutatingVisitor@V?$CNode@USNullAddr@@V?$CNode@GV?$CNode@USIPv4Addr@@V?$CNode@ULobbyIdAddr@@VCEnd@NTypelist@@@NTypelist@@@NTypelist@@@NTypelist@@@NTypelist@@@3@@NConfigurableVariantHelpers@@SAXPEAX@Z 0000000039a015f0 f i CryLobby.obj
 0001:000005f0       ?OnGameSpyObjectUnavailable@CCryGameSpySBQR2Voice@@UEAAXW4EGameSpyObjectBit@ICryGameSpySBQR2LobbyComponent@@@Z 0000000039a015f0 f i CryGameSpySBQR2Voice.obj
 0001:000005f0       ?MarkPool@CDummyMemReplay@@UEAAXH_KPEAX0PEBD@Z 0000000039a015f0 f i CryDLCStore.obj
 0001:00000600       ?AddLabelFmt@CDummyMemReplay@@UEAAXPEBDZZ 0000000039a01600 f i CryDLCStore.obj
 0001:00000610       ?StartTaskWithNoOrder@CCryDLCStore@@IEAA?AW4ECryLobbyError@@IPEAI0PEAX1@Z 0000000039a01610 f   CryDLCStore.obj
 0001:00000640       ?CreateTaskParamMem@CCryDLCStore@@IEAA?AW4ECryLobbyError@@IIPEBX_K@Z 0000000039a01640 f   CryDLCStore.obj
 0001:00000660       ?UpdateTaskError@CCryDLCStore@@IEAAXIW4ECryLobbyError@@@Z 0000000039a01660 f   CryDLCStore.obj
 0001:00000680       ?StartTaskRunning@CCryDLCStore@@MEAAXI@Z 0000000039a01680 f   CryDLCStore.obj
 0001:000006e0       ?EndTask@CCryDLCStore@@MEAAXI@Z 0000000039a016e0 f   CryDLCStore.obj
 0001:00000780       ?IsDownloading@CCryDLCStore@@UEAA_NXZ 0000000039a01780 f   CryDLCStore.obj
 0001:00000800       ?CryGetIMemReplay@@YAPEAUIMemReplay@@XZ 0000000039a01800 f i CryDLCStore.obj
 0001:00000880       ?StartTaskWithExistingOrder@CCryDLCStore@@IEAA?AW4ECryLobbyError@@IPEAI0IPEAX1@Z 0000000039a01880 f   CryDLCStore.obj
 0001:00000940       ?_Free@?$CryStringT@_W@@IEAAXXZ 0000000039a01940 f i CryDLCStore.obj
 0001:00000990       ??1SCryDLCDownloadableInfo@@QEAA@XZ 0000000039a01990 f i CryDLCStore.obj
 0001:00000a50       ?StartTaskWithNewOrder@CCryDLCStore@@IEAA?AW4ECryLobbyError@@IPEAI0UCryUserID@@0PEAX2@Z 0000000039a01a50 f   CryDLCStore.obj
 0001:00000ba0       ??4?$CryStringT@_W@@QEAAAEAV0@AEBV0@@Z 0000000039a01ba0 f i CryDLCStore.obj
 0001:00000c50       ??0SCryDLCDownloadableInfo@@QEAA@AEBU0@@Z 0000000039a01c50 f i CryDLCStore.obj
 0001:00000cd0       ?CreateOrderHandle@CCryDLCStore@@MEAA?AW4ECryLobbyError@@UCryUserID@@PEAI@Z 0000000039a01cd0 f   CryDLCStore.obj
 0001:00000df0       ??$__copy_ptrs@PEAUSItemQuantity@CCryDLCStore@@PEAU12@@priv@stlpmtx_std@@YAPEAUSItemQuantity@CCryDLCStore@@PEAU23@00AEBU__false_type@1@@Z 0000000039a01df0 f i CryDLCStore.obj
 0001:00000eb0       ?push_back@?$_Impl_vector@PEAXV?$STLGlobalAllocator@PEAX@stl@@@priv@stlpmtx_std@@QEAAXAEBQEAX@Z 0000000039a01eb0 f i CryDLCStore.obj
 0001:00000fd0       ??$__ucopy@PEAUSCryDLCDownloadableInfo@@PEAU1@_J@priv@stlpmtx_std@@YAPEAUSCryDLCDownloadableInfo@@PEAU2@00AEBUrandom_access_iterator_tag@1@PEA_J@Z 0000000039a01fd0 f i CryDLCStore.obj
 0001:000010a0       ?destroy@?$DynArray@V?$_smart_ptr@USCryDLCCategoryID@@@@HU?$SmallDynStorage@V?$_smart_ptr@USCryDLCCategoryID@@@@HUStandardAlloc@NAlloc@@@NArray@@@@IEAAXXZ 0000000039a020a0 f i CryDLCStore.obj
 0001:000010a0       ?destroy@?$DynArray@V?$_smart_ptr@USCryDLCImageID@@@@HU?$SmallDynStorage@V?$_smart_ptr@USCryDLCImageID@@@@HUStandardAlloc@NAlloc@@@NArray@@@@IEAAXXZ 0000000039a020a0 f i CryDLCStore.obj
 0001:00001130       ??$__destroy_range@PEAUSItemQuantity@CCryDLCStore@@U12@@stlpmtx_std@@YAXPEAUSItemQuantity@CCryDLCStore@@00@Z 0000000039a02130 f i CryDLCStore.obj
 0001:000011b0       ?Grab@?$CPolymorphicQueue@UIJob@CWorkQueue@@@@AEAAPEAX_KPEAX@Z 0000000039a021b0 f i CryDLCStore.obj
 0001:00001290       ??1SCryDLCItemInfo@@QEAA@XZ 0000000039a02290 f i CryDLCStore.obj
 0001:00001430       ?StopTaskRunning@CCryDLCStore@@MEAAXI@Z 0000000039a02430 f   CryDLCStore.obj
 0001:00001490       ?erase@?$_Impl_vector@USItemQuantity@CCryDLCStore@@V?$allocator@USItemQuantity@CCryDLCStore@@@stlpmtx_std@@@priv@stlpmtx_std@@QEAAPEAUSItemQuantity@CCryDLCStore@@PEAU45@0@Z 0000000039a02490 f i CryDLCStore.obj
 0001:00001520       ?ClearOrderHandle@CCryDLCStore@@MEAAXI@Z 0000000039a02520 f   CryDLCStore.obj
 0001:000015e0       ?UpdateDownloadable@CCryDLCStore@@IEAAXAEAUSCryDLCDownloadableInfo@@@Z 0000000039a025e0 f   CryDLCStore.obj
 0001:00001870       ??0CCryDLCStore@@QEAA@PEAVCCryLobby@@PEAVCCryLobbyService@@@Z 0000000039a02870 f   CryDLCStore.obj
 0001:000019c0       ??1CCryDLCStore@@UEAA@XZ   0000000039a029c0 f i CryDLCStore.obj
 0001:00001ac0       ??_ECCryDLCStore@@UEAAPEAXI@Z 0000000039a02ac0 f i CryDLCStore.obj
 0001:00001ac0       ??_GCCryDLCStore@@UEAAPEAXI@Z 0000000039a02ac0 f i CryDLCStore.obj
 0001:00001af0       ?Initialise@CCryFriends@@UEAA?AW4ECryLobbyError@@XZ 0000000039a02af0 f   CryFriends.obj
 0001:00001b10       ?Terminate@CCryFriends@@UEAA?AW4ECryLobbyError@@XZ 0000000039a02b10 f   CryFriends.obj
 0001:00001b70       ?StartTask@CCryFriends@@IEAA?AW4ECryLobbyError@@I_NPEAI1V?$CryLobbyID@USCryLobbySessionHandle@@$03@@PEAX3@Z 0000000039a02b70 f   CryFriends.obj
 0001:00001c60       ?FreeTask@CCryFriends@@MEAAXI@Z 0000000039a02c60 f   CryFriends.obj
 0001:00001ce0       ?CreateTaskParamMem@CCryFriends@@IEAA?AW4ECryLobbyError@@IIPEBX_K@Z 0000000039a02ce0 f   CryFriends.obj
 0001:00001d70       ??0CCryFriends@@QEAA@PEAVCCryLobby@@PEAVCCryLobbyService@@@Z 0000000039a02d70 f   CryFriends.obj
 0001:00001db0       ??_ECCryFriends@@WBA@EAAPEAXI@Z 0000000039a02db0 f i CryFriends.obj
 0001:00001dc0       ??_ECCryFriends@@UEAAPEAXI@Z 0000000039a02dc0 f i CryFriends.obj
 0001:00001dc0       ??_GCCryFriends@@UEAAPEAXI@Z 0000000039a02dc0 f i CryFriends.obj
 0001:00001e00       ??_GICryFriendsManagement@@UEAAPEAXI@Z 0000000039a02e00 f i CryFriendsManagement.obj
 0001:00001e00       ??_EICryFriendsManagement@@UEAAPEAXI@Z 0000000039a02e00 f i CryFriendsManagement.obj
 0001:00001e30       ?Initialise@CCryFriendsManagement@@QEAA?AW4ECryLobbyError@@XZ 0000000039a02e30 f   CryFriendsManagement.obj
 0001:00001e60       ?Terminate@CCryFriendsManagement@@QEAA?AW4ECryLobbyError@@XZ 0000000039a02e60 f   CryFriendsManagement.obj
 0001:00001ec0       ?StartTask@CCryFriendsManagement@@IEAA?AW4ECryLobbyError@@I_NPEAI1PEAX2@Z 0000000039a02ec0 f   CryFriendsManagement.obj
 0001:00001fa0       ?FreeTask@CCryFriendsManagement@@MEAAXI@Z 0000000039a02fa0 f   CryFriendsManagement.obj
 0001:00002020       ?CreateTaskParamMem@CCryFriendsManagement@@IEAA?AW4ECryLobbyError@@IIPEBX_K@Z 0000000039a03020 f   CryFriendsManagement.obj
 0001:000020b0       ??0CCryFriendsManagement@@QEAA@PEAVCCryLobby@@PEAVCCryLobbyService@@@Z 0000000039a030b0 f   CryFriendsManagement.obj
 0001:00002100       ??_ECCryFriendsManagement@@WBA@EAAPEAXI@Z 0000000039a03100 f i CryFriendsManagement.obj
 0001:00002110       ?CancelTask@CCryFriendsManagement@@UEAAXI@Z 0000000039a03110 f   CryFriendsManagement.obj
 0001:000021a0       ??_ECCryFriendsManagement@@UEAAPEAXI@Z 0000000039a031a0 f i CryFriendsManagement.obj
 0001:000021a0       ??_GCCryFriendsManagement@@UEAAPEAXI@Z 0000000039a031a0 f i CryFriendsManagement.obj
 0001:000021e0       ?ReadUINT16@CCryLobbyPacket@@QEAAGXZ 0000000039a031e0 f i CryLobby.obj
 0001:00002220       ?WriteUINT64@CCryLobbyPacket@@QEAAX_K@Z 0000000039a03220 f i CryLobby.obj
 0001:000022f0       ?ReadUINT64@CCryLobbyPacket@@QEAA_KXZ 0000000039a032f0 f i CryLobby.obj
 0001:000023b0       ?ReadBool@CCryLobbyPacket@@QEAA_NXZ 0000000039a033b0 f i CryLobby.obj
 0001:000023e0       ?ReadData@CCryLobbyPacket@@QEAAXPEAXI@Z 0000000039a033e0 f i CryLobby.obj
 0001:00002430       ?ReadPacketHeader@CCrySharedLobbyPacket@@QEAAXXZ 0000000039a03430 f i CryLobby.obj
 0001:00002540       ?WriteDataHeader@CCrySharedLobbyPacket@@QEAAXXZ 0000000039a03540 f i CryLobby.obj
 0001:000025b0       ?ReadDataHeader@CCrySharedLobbyPacket@@QEAAXXZ 0000000039a035b0 f i CryLobby.obj
 0001:00002620       ?ReleaseTask@CCryLobby@@QEAAXI@Z 0000000039a03620 f   CryLobby.obj
 0001:00002630       ?GetNextPacketFromBuffer@CCryLobby@@AEAA_NPEBEIAEAIPEAVCCryLobbyPacket@@@Z 0000000039a03630 f   CryLobby.obj
 0001:00002740       ?GetConfigurationInformation@CCryLobby@@QEAAXPEAUSConfigurationParams@@I@Z 0000000039a03740 f   CryLobby.obj
 0001:00002790       ?GetFlag@CCryLobbyService@@UEAA_NW4ECryLobbyServiceFlag@@@Z 0000000039a03790 f   CryLobby.obj
 0001:000027b0       ?UpdateTaskError@CCryLobbyService@@IEAAXIW4ECryLobbyError@@@Z 0000000039a037b0 f   CryLobby.obj
 0001:000027d0       ?GetSocketPorts@CCryLobbyService@@UEAAXAEAG0@Z 0000000039a037d0 f   CryLobby.obj
 0001:00002840       ?GetInternalSocketPort@CCryLobby@@QEAAGW4ECryLobbyService@@@Z 0000000039a03840 f   CryLobby.obj
 0001:00002860       ?GetLobbyParameters@CCryLobby@@UEBAAEBUSCryLobbyParameters@@XZ 0000000039a03860 f   CryLobby.obj
 0001:00002870       ?EncryptPacket@CCryLobby@@AEAAPEBEPEBEI@Z 0000000039a03870 f   CryLobby.obj
 0001:000028f0       ?DecodeAddress@CCryLobby@@SAXIGPEAD_N@Z 0000000039a038f0 f   CryLobby.obj
 0001:00002980       ?ConvertAddr@CCryLobby@@SA_NAEBV?$CConfigurableVariant@V?$CNode@USNullAddr@@V?$CNode@GV?$CNode@USIPv4Addr@@V?$CNode@ULobbyIdAddr@@VCEnd@NTypelist@@@NTypelist@@@NTypelist@@@NTypelist@@@NTypelist@@$07VCDefaultVariantConversion@NConfigurableVariantHelpers@@VCDefaultVariantConstruction@4@@@PEAUsockaddr_in@@@Z 0000000039a03980 f   CryLobby.obj
 0001:000029b0       ?ConvertAddr@CCryLobby@@SA_NAEBV?$CConfigurableVariant@V?$CNode@USNullAddr@@V?$CNode@GV?$CNode@USIPv4Addr@@V?$CNode@ULobbyIdAddr@@VCEnd@NTypelist@@@NTypelist@@@NTypelist@@@NTypelist@@@NTypelist@@$07VCDefaultVariantConversion@NConfigurableVariantHelpers@@VCDefaultVariantConstruction@4@@@PEAUsockaddr@@PEAH@Z 0000000039a039b0 f   CryLobby.obj
 0001:000029e0       ?GetResolver@CCryLobby@@SAPEAVCNetAddressResolver@@XZ 0000000039a039e0 f   CryLobby.obj
 0001:00002a00       ?MemAlloc@CCryLobby@@QEAAI_K@Z 0000000039a03a00 f   CryLobby.obj
 0001:00002a20       ?MemFree@CCryLobby@@QEAAXI@Z 0000000039a03a20 f   CryLobby.obj
 0001:00002a50       ?MemGetPtr@CCryLobby@@QEAAPEAXI@Z 0000000039a03a50 f   CryLobby.obj
 0001:00002a70       ?CryLogAlways@@YAXPEBDZZ   0000000039a03a70 f i CryLobby.obj
 0001:00002ad0       ??$__find@PEAUSEventCBData@CCryLobby@@U12@@priv@stlpmtx_std@@YAPEAUSEventCBData@CCryLobby@@PEAU23@0AEBU23@AEBUrandom_access_iterator_tag@1@@Z 0000000039a03ad0 f i CryLobby.obj
 0001:00002c50       ?MutatingVisit@?$VTableImpl@USNullAddr@@$0A@U?$IVisitor@V?$CNode@USNullAddr@@V?$CNode@GV?$CNode@USIPv4Addr@@V?$CNode@ULobbyIdAddr@@VCEnd@NTypelist@@@NTypelist@@@NTypelist@@@NTypelist@@@NTypelist@@@NConfigurableVariantHelpers@@U?$IMutatingVisitor@V?$CNode@USNullAddr@@V?$CNode@GV?$CNode@USIPv4Addr@@V?$CNode@ULobbyIdAddr@@VCEnd@NTypelist@@@NTypelist@@@NTypelist@@@NTypelist@@@NTypelist@@@3@@NConfigurableVariantHelpers@@SAXPEAU?$IMutatingVisitor@V?$CNode@USNullAddr@@V?$CNode@GV?$CNode@USIPv4Addr@@V?$CNode@ULobbyIdAddr@@VCEnd@NTypelist@@@NTypelist@@@NTypelist@@@NTypelist@@@NTypelist@@@2@PEAX1@Z 0000000039a03c50 f i CryLobby.obj
 0001:00002c50       ?Visit@?$VTableImpl@USNullAddr@@$0A@U?$IVisitor@V?$CNode@USNullAddr@@V?$CNode@GV?$CNode@USIPv4Addr@@V?$CNode@ULobbyIdAddr@@VCEnd@NTypelist@@@NTypelist@@@NTypelist@@@NTypelist@@@NTypelist@@@NConfigurableVariantHelpers@@U?$IMutatingVisitor@V?$CNode@USNullAddr@@V?$CNode@GV?$CNode@USIPv4Addr@@V?$CNode@ULobbyIdAddr@@VCEnd@NTypelist@@@NTypelist@@@NTypelist@@@NTypelist@@@NTypelist@@@3@@NConfigurableVariantHelpers@@SAXPEAU?$IVisitor@V?$CNode@USNullAddr@@V?$CNode@GV?$CNode@USIPv4Addr@@V?$CNode@ULobbyIdAddr@@VCEnd@NTypelist@@@NTypelist@@@NTypelist@@@NTypelist@@@NTypelist@@@2@PEBXPEAX@Z 0000000039a03c50 f i CryLobby.obj
 0001:00002c60       ?Clone@?$VTableImpl@USIPv4Addr@@$0A@U?$IVisitor@V?$CNode@USNullAddr@@V?$CNode@GV?$CNode@USIPv4Addr@@V?$CNode@ULobbyIdAddr@@VCEnd@NTypelist@@@NTypelist@@@NTypelist@@@NTypelist@@@NTypelist@@@NConfigurableVariantHelpers@@U?$IMutatingVisitor@V?$CNode@USNullAddr@@V?$CNode@GV?$CNode@USIPv4Addr@@V?$CNode@ULobbyIdAddr@@VCEnd@NTypelist@@@NTypelist@@@NTypelist@@@NTypelist@@@NTypelist@@@3@@NConfigurableVariantHelpers@@SAXPEAXPEBX@Z 0000000039a03c60 f i CryLobby.obj
 0001:00002c70       ?ConstructClone@?$VTableImpl@USIPv4Addr@@$0A@U?$IVisitor@V?$CNode@USNullAddr@@V?$CNode@GV?$CNode@USIPv4Addr@@V?$CNode@ULobbyIdAddr@@VCEnd@NTypelist@@@NTypelist@@@NTypelist@@@NTypelist@@@NTypelist@@@NConfigurableVariantHelpers@@U?$IMutatingVisitor@V?$CNode@USNullAddr@@V?$CNode@GV?$CNode@USIPv4Addr@@V?$CNode@ULobbyIdAddr@@VCEnd@NTypelist@@@NTypelist@@@NTypelist@@@NTypelist@@@NTypelist@@@3@@NConfigurableVariantHelpers@@SAXPEAXPEBX@Z 0000000039a03c70 f i CryLobby.obj
 0001:00002c80       ?Visit@?$VTableImpl@USIPv4Addr@@$0A@U?$IVisitor@V?$CNode@USNullAddr@@V?$CNode@GV?$CNode@USIPv4Addr@@V?$CNode@ULobbyIdAddr@@VCEnd@NTypelist@@@NTypelist@@@NTypelist@@@NTypelist@@@NTypelist@@@NConfigurableVariantHelpers@@U?$IMutatingVisitor@V?$CNode@USNullAddr@@V?$CNode@GV?$CNode@USIPv4Addr@@V?$CNode@ULobbyIdAddr@@VCEnd@NTypelist@@@NTypelist@@@NTypelist@@@NTypelist@@@NTypelist@@@3@@NConfigurableVariantHelpers@@SAXPEAU?$IVisitor@V?$CNode@USNullAddr@@V?$CNode@GV?$CNode@USIPv4Addr@@V?$CNode@ULobbyIdAddr@@VCEnd@NTypelist@@@NTypelist@@@NTypelist@@@NTypelist@@@NTypelist@@@2@PEBXPEAX@Z 0000000039a03c80 f i CryLobby.obj
 0001:00002c80       ?MutatingVisit@?$VTableImpl@USIPv4Addr@@$0A@U?$IVisitor@V?$CNode@USNullAddr@@V?$CNode@GV?$CNode@USIPv4Addr@@V?$CNode@ULobbyIdAddr@@VCEnd@NTypelist@@@NTypelist@@@NTypelist@@@NTypelist@@@NTypelist@@@NConfigurableVariantHelpers@@U?$IMutatingVisitor@V?$CNode@USNullAddr@@V?$CNode@GV?$CNode@USIPv4Addr@@V?$CNode@ULobbyIdAddr@@VCEnd@NTypelist@@@NTypelist@@@NTypelist@@@NTypelist@@@NTypelist@@@3@@NConfigurableVariantHelpers@@SAXPEAU?$IMutatingVisitor@V?$CNode@USNullAddr@@V?$CNode@GV?$CNode@USIPv4Addr@@V?$CNode@ULobbyIdAddr@@VCEnd@NTypelist@@@NTypelist@@@NTypelist@@@NTypelist@@@NTypelist@@@2@PEAX1@Z 0000000039a03c80 f i CryLobby.obj
 0001:00002ca0       ??_H@YAXPEAX_KHP6APEAX0@Z@Z 0000000039a03ca0 f i CryLobby.obj
 0001:00002cf0       ??_I@YAXPEAX_KHP6AX0@Z@Z   0000000039a03cf0 f i CryLobby.obj
 0001:00002d50       ??_GICryLobbyService@@UEAAPEAXI@Z 0000000039a03d50 f i CryLobby.obj
 0001:00002d50       ??_EICryLobbyService@@UEAAPEAXI@Z 0000000039a03d50 f i CryLobby.obj
 0001:00002d80       ??_EICryLobby@@UEAAPEAXI@Z 0000000039a03d80 f i CryLobby.obj
 0001:00002d80       ??_GICryLobby@@UEAAPEAXI@Z 0000000039a03d80 f i CryLobby.obj
 0001:00002db0       ?WritePacketHeader@CCrySharedLobbyPacket@@QEAAXXZ 0000000039a03db0 f i CryLobby.obj
 0001:00002ef0       ?SetLobbyService@CCryLobby@@UEAA?AW4ECryLobbyService@@W42@@Z 0000000039a03ef0 f   CryLobby.obj
 0001:00002f50       ?GetDisconnectTimeOut@CCryLobby@@AEAAIXZ 0000000039a03f50 f   CryLobby.obj
 0001:00002fd0       ?CreateTask@CCryLobby@@QEAAIXZ 0000000039a03fd0 f   CryLobby.obj
 0001:00003030       ?DebugGenerateError@CCryLobby@@QEAA_NIAEAW4ECryLobbyError@@@Z 0000000039a04030 f   CryLobby.obj
 0001:000030d0       ?DebugOKToStartTaskRunning@CCryLobby@@QEAA_NI@Z 0000000039a040d0 f   CryLobby.obj
 0001:00003190       ?DebugTickCallStartTaskRunning@CCryLobby@@QEAA_NI@Z 0000000039a04190 f   CryLobby.obj
 0001:000031e0       ?DebugOKToTickTask@CCryLobby@@QEAA_NI_N@Z 0000000039a041e0 f   CryLobby.obj
 0001:000032e0       ?CalculatePacketTypeEncoding@CCryLobby@@AEAAXXZ 0000000039a042e0 f   CryLobby.obj
 0001:000034d0       ?SendVoice@CCryLobby@@QEAA?AW4ESocketError@@PEAVCCryLobbyPacket@@AEBV?$CConfigurableVariant@V?$CNode@USNullAddr@@V?$CNode@GV?$CNode@USIPv4Addr@@V?$CNode@ULobbyIdAddr@@VCEnd@NTypelist@@@NTypelist@@@NTypelist@@@NTypelist@@@NTypelist@@$07VCDefaultVariantConversion@NConfigurableVariantHelpers@@VCDefaultVariantConstruction@4@@@@Z 0000000039a044d0 f   CryLobby.obj
 0001:000035b0       ?GetTCPService@CCryLobbyService@@UEAA?AV?$_smart_ptr@UICryTCPService@@@@PEBDG@Z 0000000039a045b0 f   CryLobby.obj
 0001:000035d0       ?GetLobbyServiceFlag@CCryLobby@@UEAA_NW4ECryLobbyService@@W4ECryLobbyServiceFlag@@@Z 0000000039a045d0 f   CryLobby.obj
 0001:000035f0       ??0CCryLobbyService@@QEAA@PEAVCCryLobby@@W4ECryLobbyService@@@Z 0000000039a045f0 f   CryLobby.obj
 0001:00003640       ?IsDead@CCryFriends@@UEBA_NXZ 0000000039a04640 f i CryFriends.obj
 0001:00003640       ?EnterScope@CDummyMemReplay@@UEAA_NW4Class@EMemReplayAllocClass@@GH@Z 0000000039a04640 f i CryDLCStore.obj
 0001:00003640       ?IsDead@CCryStats@@UEBA_NXZ 0000000039a04640 f i CryStats.obj
 0001:00003640       ?IsDead@CCryDLCStore@@UEBA_NXZ 0000000039a04640 f i CryDLCStore.obj
 0001:00003640       ?IsDead@CCryLobbyService@@UEBA_NXZ 0000000039a04640 f i CryLobby.obj
 0001:00003640       ?IsDead@CCryLobbyUI@@UEBA_NXZ 0000000039a04640 f i CryLobbyUI.obj
 0001:00003640       ?IsPushToTalkEnabled@CCryVoice@@UEAA_NI@Z 0000000039a04640 f i CryVoice.obj
 0001:00003640       ?IsDead@CCryGameSpySBQR2LobbyUI@@UEBA_NXZ 0000000039a04640 f i CryGameSpySBQR2LobbyUI.obj
 0001:00003640       ?IsDead@CCrySignIn@@UEBA_NXZ 0000000039a04640 f i CrySignIn.obj
 0001:00003640       ?IsDead@CCryMatchMaking@@UEBA_NXZ 0000000039a04640 f i CryMatchMaking.obj
 0001:00003640       ?IsDead@CCryFriendsManagement@@UEBA_NXZ 0000000039a04640 f i CryFriendsManagement.obj
 0001:00003640       ?LobbyAddrIDHasPendingData@ICryMatchMakingPrivate@@UEAA_NXZ 0000000039a04640 f i CryMatchMaking.obj
 0001:00003650       ??_ECCryLobbyService@@WBA@EAAPEAXI@Z 0000000039a04650 f i CryLobby.obj
 0001:00003660       ??1CCryLobbyService@@UEAA@XZ 0000000039a04660 f   CryLobby.obj
 0001:000036b0       ?Initialise@CCryLobbyService@@UEAA?AW4ECryLobbyError@@W4ECryLobbyServiceFeatures@@P6AXW42@PEAVCCryLobby@@W4ECryLobbyService@@@Z@Z 0000000039a046b0 f   CryLobby.obj
 0001:00003740       ?StartTask@CCryLobbyService@@IEAA?AW4ECryLobbyError@@II_NPEAI1PEAX2@Z 0000000039a04740 f   CryLobby.obj
 0001:00003870       ?FreeTask@CCryLobbyService@@IEAAXI@Z 0000000039a04870 f   CryLobby.obj
 0001:00003900       ?CancelTask@CCryLobbyService@@UEAAXI@Z 0000000039a04900 f   CryLobby.obj
 0001:00003990       ??4?$CConfigurableVariant@V?$CNode@USNullAddr@@V?$CNode@GV?$CNode@USIPv4Addr@@V?$CNode@ULobbyIdAddr@@VCEnd@NTypelist@@@NTypelist@@@NTypelist@@@NTypelist@@@NTypelist@@$07VCDefaultVariantConversion@NConfigurableVariantHelpers@@VCDefaultVariantConstruction@4@@@QEAAAEAV0@AEBV0@@Z 0000000039a04990 f i CryLobby.obj
 0001:00003a10       ?Execute@?$CClassJob@XVCCryGameSpySBQR2LobbyService@@@CWorkQueue@@UEAAXXZ 0000000039a04a10 f i CryGameSpySBQR2Lobby.obj
 0001:00003a10       ?Execute@?$CClassJob@XVCCryLobbyService@@@CWorkQueue@@UEAAXXZ 0000000039a04a10 f i CryLobby.obj
 0001:00003a40       ??_E?$SAbstractVisitDeclarator@AEBG@NConfigurableVariantHelpers@@UEAAPEAXI@Z 0000000039a04a40 f i CryLobby.obj
 0001:00003a40       ??_E?$SAbstractVisitDeclarator@AEBULobbyIdAddr@@@NConfigurableVariantHelpers@@UEAAPEAXI@Z 0000000039a04a40 f i CryLobby.obj
 0001:00003a40       ??_E?$SAbstractVisitDeclarator@AEBUSIPv4Addr@@@NConfigurableVariantHelpers@@UEAAPEAXI@Z 0000000039a04a40 f i CryLobby.obj
 0001:00003a40       ??_G?$SAbstractVisitDeclarator@AEBUSNullAddr@@@NConfigurableVariantHelpers@@UEAAPEAXI@Z 0000000039a04a40 f i CryLobby.obj
 0001:00003a40       ??_GISystemEventListener@@UEAAPEAXI@Z 0000000039a04a40 f i CryLobbyDLL.obj
 0001:00003a40       ??_EISystemEventListener@@UEAAPEAXI@Z 0000000039a04a40 f i CryLobbyDLL.obj
 0001:00003a40       ??_E?$SAbstractVisitDeclarator@AEBUSNullAddr@@@NConfigurableVariantHelpers@@UEAAPEAXI@Z 0000000039a04a40 f i CryLobby.obj
 0001:00003a40       ??_G?$SAbstractVisitDeclarator@AEBG@NConfigurableVariantHelpers@@UEAAPEAXI@Z 0000000039a04a40 f i CryLobby.obj
 0001:00003a40       ??_G?$SAbstractVisitDeclarator@AEBULobbyIdAddr@@@NConfigurableVariantHelpers@@UEAAPEAXI@Z 0000000039a04a40 f i CryLobby.obj
 0001:00003a40       ??_G?$SAbstractVisitDeclarator@AEBUSIPv4Addr@@@NConfigurableVariantHelpers@@UEAAPEAXI@Z 0000000039a04a40 f i CryLobby.obj
 0001:00003a70       ?OnInternalSocketChanged@CCryLobbyService@@UEAAXV?$_smart_ptr@UIDatagramSocket@@@@@Z 0000000039a04a70 f i CryLobby.obj
 0001:00003ac0       ?WritePacket@CCachedPacketBuffer@CCryLobby@@QEAA_NAEBV?$CConfigurableVariant@V?$CNode@USNullAddr@@V?$CNode@GV?$CNode@USIPv4Addr@@V?$CNode@ULobbyIdAddr@@VCEnd@NTypelist@@@NTypelist@@@NTypelist@@@NTypelist@@@NTypelist@@$07VCDefaultVariantConversion@NConfigurableVariantHelpers@@VCDefaultVariantConstruction@4@@@PEBEI@Z 0000000039a04ac0 f i CryLobby.obj
 0001:00003b90       ?InitialiseServiceCB@CCryLobby@@CAXW4ECryLobbyError@@PEAV1@W4ECryLobbyService@@@Z 0000000039a04b90 f   CryLobby.obj
 0001:00003c50       ?InternalSocketDie@CCryLobby@@AEAAXW4ECryLobbyService@@@Z 0000000039a04c50 f   CryLobby.obj
 0001:00003da0       ?ConnectionSetState@CCryLobby@@QEAAXV?$CryLobbyID@USCryLobbyConnectionID@@$0EA@@@W4ECryLobbyConnectionState@@@Z 0000000039a04da0 f   CryLobby.obj
 0001:00003e00       ?ConnectionGetState@CCryLobby@@QEAA?AW4ECryLobbyConnectionState@@V?$CryLobbyID@USCryLobbyConnectionID@@$0EA@@@@Z 0000000039a04e00 f   CryLobby.obj
 0001:00003e50       ?FreeConnection@CCryLobby@@QEAAXV?$CryLobbyID@USCryLobbyConnectionID@@$0EA@@@@Z 0000000039a04e50 f   CryLobby.obj
 0001:00003ef0       ?AddressFromConnection@CCryLobby@@QEAA_NAEAV?$CConfigurableVariant@V?$CNode@USNullAddr@@V?$CNode@GV?$CNode@USIPv4Addr@@V?$CNode@ULobbyIdAddr@@VCEnd@NTypelist@@@NTypelist@@@NTypelist@@@NTypelist@@@NTypelist@@$07VCDefaultVariantConversion@NConfigurableVariantHelpers@@VCDefaultVariantConstruction@4@@@V?$CryLobbyID@USCryLobbyConnectionID@@$0EA@@@@Z 0000000039a04ef0 f   CryLobby.obj
 0001:00003f30       ?UpdateConnectionPing@CCryLobby@@AEAAXV?$CryLobbyID@USCryLobbyConnectionID@@$0EA@@@G@Z 0000000039a04f30 f   CryLobby.obj
 0001:00004010       ?GetConnectionPing@CCryLobby@@UEAAGV?$CryLobbyID@USCryLobbyConnectionID@@$0EA@@@@Z 0000000039a05010 f   CryLobby.obj
 0001:00004030       ?DispatchEvent@CCryLobby@@QEAAXW4ECryLobbySystemEvent@@TUCryLobbyEventData@@@Z 0000000039a05030 f   CryLobby.obj
 0001:00004090       ??_ECCryLobbyService@@UEAAPEAXI@Z 0000000039a05090 f i CryLobby.obj
 0001:00004090       ??_GCCryLobbyService@@UEAAPEAXI@Z 0000000039a05090 f i CryLobby.obj
 0001:00004100       ?FreeSocketNT@CCryLobbyService@@QEAAXXZ 0000000039a05100 f   CryLobby.obj
 0001:00004130       ?GetInternalSocket@CCryLobby@@QEAA?AV?$_smart_ptr@UIDatagramSocket@@@@W4ECryLobbyService@@@Z 0000000039a05130 f   CryLobby.obj
 0001:00004170       ?TimeSincePacketInMS@CCryLobby@@QEBAIV?$CryLobbyID@USCryLobbyConnectionID@@$0EA@@@@Z 0000000039a05170 f   CryLobby.obj
 0001:000041e0       ?ForceTimeoutConnection@CCryLobby@@QEAAXV?$CryLobbyID@USCryLobbyConnectionID@@$0EA@@@@Z 0000000039a051e0 f   CryLobby.obj
 0001:00004250       ?GetNetAddress@CCryLobby@@QEBAPEBV?$CConfigurableVariant@V?$CNode@USNullAddr@@V?$CNode@GV?$CNode@USIPv4Addr@@V?$CNode@ULobbyIdAddr@@VCEnd@NTypelist@@@NTypelist@@@NTypelist@@@NTypelist@@@NTypelist@@$07VCDefaultVariantConversion@NConfigurableVariantHelpers@@VCDefaultVariantConstruction@4@@@V?$CryLobbyID@USCryLobbyConnectionID@@$0EA@@@@Z 0000000039a05250 f   CryLobby.obj
 0001:00004280       ?DecodeAddress@CCryLobby@@SAXAEBV?$CConfigurableVariant@V?$CNode@USNullAddr@@V?$CNode@GV?$CNode@USIPv4Addr@@V?$CNode@ULobbyIdAddr@@VCEnd@NTypelist@@@NTypelist@@@NTypelist@@@NTypelist@@@NTypelist@@$07VCDefaultVariantConversion@NConfigurableVariantHelpers@@VCDefaultVariantConstruction@4@@@PEAD_N@Z 0000000039a05280 f   CryLobby.obj
 0001:000042f0       ?Next@?$CPolymorphicQueue@UIJob@CWorkQueue@@@@AEAAPEAUIJob@CWorkQueue@@PEAU23@@Z 0000000039a052f0 f i CryLobby.obj
 0001:000043a0       ?_AllocData@?$CryStringT@D@@IEAAX_K@Z 0000000039a053a0 f i CryLobby.obj
 0001:00004410       ?InviteAccepted@CCryLobby@@QEAAXW4ECryLobbyService@@IV?$_smart_ptr@USCrySessionID@@@@W4ECryLobbyError@@@Z 0000000039a05410 f   CryLobby.obj
 0001:00004550       ?LogPacketsInBuffer@CCryLobby@@AEAAXPEBEI@Z 0000000039a05550 f   CryLobby.obj
 0001:00004610       ?CheckFreeGlobalResources@CCryLobby@@AEAAXXZ 0000000039a05610 f   CryLobby.obj
 0001:00004760       ?EndTask@CCryLobbyService@@IEAAXI@Z 0000000039a05760 f   CryLobby.obj
 0001:000048e0       ??0?$CryStringT@D@@QEAA@PEBD@Z 0000000039a058e0 f i CryLobby.obj
 0001:00004960       ?TerminateServiceCB@CCryLobby@@CAXW4ECryLobbyError@@PEAV1@W4ECryLobbyService@@@Z 0000000039a05960 f   CryLobby.obj
 0001:00004a20       ?FixPortBinding@@YAXAEAV?$CConfigurableVariant@V?$CNode@USNullAddr@@V?$CNode@GV?$CNode@USIPv4Addr@@V?$CNode@ULobbyIdAddr@@VCEnd@NTypelist@@@NTypelist@@@NTypelist@@@NTypelist@@@NTypelist@@$07VCDefaultVariantConversion@NConfigurableVariantHelpers@@VCDefaultVariantConstruction@4@@@H@Z 0000000039a05a20 f   CryLobby.obj
 0001:00004cc0       ?Terminate@CCryLobby@@UEAA?AW4ECryLobbyError@@W4ECryLobbyService@@W4ECryLobbyServiceFeatures@@P6AX0W42@PEAX@Z3@Z 0000000039a05cc0 f   CryLobby.obj
 0001:00004e10       ?CreateConnection@CCryLobby@@QEAA?AV?$CryLobbyID@USCryLobbyConnectionID@@$0EA@@@AEBV?$CConfigurableVariant@V?$CNode@USNullAddr@@V?$CNode@GV?$CNode@USIPv4Addr@@V?$CNode@ULobbyIdAddr@@VCEnd@NTypelist@@@NTypelist@@@NTypelist@@@NTypelist@@@NTypelist@@$07VCDefaultVariantConversion@NConfigurableVariantHelpers@@VCDefaultVariantConstruction@4@@@@Z 0000000039a05e10 f   CryLobby.obj
 0001:000050b0       ?ConnectionAddRef@CCryLobby@@QEAAXV?$CryLobbyID@USCryLobbyConnectionID@@$0EA@@@@Z 0000000039a060b0 f   CryLobby.obj
 0001:000051e0       ?AddReliablePacketToSendQueue@CCryLobby@@AEAA_NV?$CryLobbyID@USCryLobbyConnectionID@@$0EA@@@PEAVCCryLobbyPacket@@@Z 0000000039a061e0 f   CryLobby.obj
 0001:000053f0       ?AddPacketToReliableBuildPacket@CCryLobby@@AEAA_NV?$CryLobbyID@USCryLobbyConnectionID@@$0EA@@@PEAVCCryLobbyPacket@@@Z 0000000039a063f0 f   CryLobby.obj
 0001:000055b0       ?push_back@?$_Impl_vector@USEventCBData@CCryLobby@@V?$allocator@USEventCBData@CCryLobby@@@stlpmtx_std@@@priv@stlpmtx_std@@QEAAXAEBUSEventCBData@CCryLobby@@@Z 0000000039a065b0 f i CryLobby.obj
 0001:00005700       ?reserve@?$_Impl_vector@USEventCBData@CCryLobby@@V?$allocator@USEventCBData@CCryLobby@@@stlpmtx_std@@@priv@stlpmtx_std@@QEAAX_K@Z 0000000039a06700 f i CryLobby.obj
 0001:00005890       ?ConnectionRemoveRef@CCryLobby@@QEAAXV?$CryLobbyID@USCryLobbyConnectionID@@$0EA@@@@Z 0000000039a06890 f   CryLobby.obj
 0001:00005cd0       ?RegisterEventInterest@CCryLobby@@UEAAXW4ECryLobbySystemEvent@@P6AXTUCryLobbyEventData@@PEAX@Z2@Z 0000000039a06cd0 f   CryLobby.obj
 0001:00005d00       ?UnregisterEventInterest@CCryLobby@@UEAAXW4ECryLobbySystemEvent@@P6AXTUCryLobbyEventData@@PEAX@Z2@Z 0000000039a06d00 f   CryLobby.obj
 0001:00005d90       ??0?$CPolymorphicQueue@UIJob@CWorkQueue@@@@QEAA@XZ 0000000039a06d90 f i CryLobby.obj
 0001:00005e30       ?AbstractVisit@?$CVisitor@V?$CNode@ULobbyIdAddr@@VCEnd@NTypelist@@@NTypelist@@VCComparatorVisitor@?$less@V?$CConfigurableVariant@V?$CNode@USNullAddr@@V?$CNode@GV?$CNode@USIPv4Addr@@V?$CNode@ULobbyIdAddr@@VCEnd@NTypelist@@@NTypelist@@@NTypelist@@@NTypelist@@@NTypelist@@$07VCDefaultVariantConversion@NConfigurableVariantHelpers@@VCDefaultVariantConstruction@4@@@@stlpmtx_std@@U?$IVisitor@V?$CNode@USNullAddr@@V?$CNode@GV?$CNode@USIPv4Addr@@V?$CNode@ULobbyIdAddr@@VCEnd@NTypelist@@@NTypelist@@@NTypelist@@@NTypelist@@@NTypelist@@@NConfigurableVariantHelpers@@@NConfigurableVariantHelpers@@UEAAXAEBULobbyIdAddr@@PEAX@Z 0000000039a06e30 f i CryLobby.obj
 0001:00005e70       ?InternalSocketCreate@CCryLobby@@QEAAXW4ECryLobbyService@@@Z 0000000039a06e70 f   CryLobby.obj
 0001:000061e0       ?CreateSocketNT@CCryLobbyService@@QEAAXXZ 0000000039a071e0 f   CryLobby.obj
 0001:00006200       ?BeginFlush@?$CPolymorphicQueue@UIJob@CWorkQueue@@@@AEAA_NXZ 0000000039a07200 f i CryLobby.obj
 0001:000062c0       ?EndFlush@?$CPolymorphicQueue@UIJob@CWorkQueue@@@@AEAAXXZ 0000000039a072c0 f i CryLobby.obj
 0001:000063a0       ?AbstractVisit@?$CVisitor@V?$CNode@USIPv4Addr@@V?$CNode@ULobbyIdAddr@@VCEnd@NTypelist@@@NTypelist@@@NTypelist@@VCComparatorVisitor@?$less@V?$CConfigurableVariant@V?$CNode@USNullAddr@@V?$CNode@GV?$CNode@USIPv4Addr@@V?$CNode@ULobbyIdAddr@@VCEnd@NTypelist@@@NTypelist@@@NTypelist@@@NTypelist@@@NTypelist@@$07VCDefaultVariantConversion@NConfigurableVariantHelpers@@VCDefaultVariantConstruction@4@@@@stlpmtx_std@@U?$IVisitor@V?$CNode@USNullAddr@@V?$CNode@GV?$CNode@USIPv4Addr@@V?$CNode@ULobbyIdAddr@@VCEnd@NTypelist@@@NTypelist@@@NTypelist@@@NTypelist@@@NTypelist@@@NConfigurableVariantHelpers@@@NConfigurableVariantHelpers@@UEAAXAEBUSIPv4Addr@@PEAX@Z 0000000039a073a0 f i CryLobby.obj
 0001:000063e0       ??1?$CPolymorphicQueue@UIJob@CWorkQueue@@@@QEAA@XZ 0000000039a073e0 f i CryLobby.obj
 0001:00006570       ??$Add@VCCryLobbyService@@@CWorkQueue@@QEAAXP8CCryLobbyService@@EAAXXZPEAV1@@Z 0000000039a07570 f i CryLobby.obj
 0001:00006620       ??$Add@IVCCryGameSpySBQR2LobbyService@@@CWorkQueue@@QEAAXP8CCryGameSpySBQR2LobbyService@@EAAXI@ZPEAV1@I@Z 0000000039a07620 f i CryGameSpySBQR2Lobby.obj
 0001:00006620       ??$Add@IVCCryLobbyService@@@CWorkQueue@@QEAAXP8CCryLobbyService@@EAAXI@ZPEAV1@I@Z 0000000039a07620 f i CryLobby.obj
 0001:000066e0       ?AbstractVisit@?$CVisitor@V?$CNode@GV?$CNode@USIPv4Addr@@V?$CNode@ULobbyIdAddr@@VCEnd@NTypelist@@@NTypelist@@@NTypelist@@@NTypelist@@VCComparatorVisitor@?$less@V?$CConfigurableVariant@V?$CNode@USNullAddr@@V?$CNode@GV?$CNode@USIPv4Addr@@V?$CNode@ULobbyIdAddr@@VCEnd@NTypelist@@@NTypelist@@@NTypelist@@@NTypelist@@@NTypelist@@$07VCDefaultVariantConversion@NConfigurableVariantHelpers@@VCDefaultVariantConstruction@4@@@@stlpmtx_std@@U?$IVisitor@V?$CNode@USNullAddr@@V?$CNode@GV?$CNode@USIPv4Addr@@V?$CNode@ULobbyIdAddr@@VCEnd@NTypelist@@@NTypelist@@@NTypelist@@@NTypelist@@@NTypelist@@@NConfigurableVariantHelpers@@@NConfigurableVariantHelpers@@UEAAXAEBGPEAX@Z 0000000039a076e0 f i CryLobby.obj
 0001:00006720       ??1CCryLobby@@UEAA@XZ      0000000039a07720 f   CryLobby.obj
 0001:000069b0       ?GetCVars@CCryLobby@@UEAAAEAVCLobbyCVars@@XZ 0000000039a079b0 f i CryLobby.obj
 0001:000069c0       ?GetLobbyServiceType@CCryLobby@@UEAA?AW4ECryLobbyService@@XZ 0000000039a079c0 f i CryLobby.obj
 0001:000069d0       ?GetLobbyExtras@CCryLobby@@UEAAPEAVICryLobbyGFWLExtras@@XZ 0000000039a079d0 f i CryLobby.obj
 0001:000069e0       ?GetCryEngineLevelNameHint@CCryLobby@@UEAAPEBDXZ 0000000039a079e0 f i CryLobby.obj
 0001:000069f0       ?GetCryEngineRulesNameHint@CCryLobby@@UEAAPEBDXZ 0000000039a079f0 f i CryLobby.obj
 0001:00006a00       ??_ECCryLobby@@W7EAAPEAXI@Z 0000000039a07a00 f i CryLobby.obj
 0001:00006a10       ?GetLobbyService@CCryLobby@@UEAAPEAUICryLobbyService@@XZ 0000000039a07a10 f i CryLobby.obj
 0001:00006a30       ?GetMatchMaking@CCryLobby@@UEAAPEAUICryMatchMaking@@XZ 0000000039a07a30 f i CryLobby.obj
 0001:00006a60       ?GetVoice@CCryLobby@@UEAAPEAUICryVoice@@XZ 0000000039a07a60 f i CryLobby.obj
 0001:00006a90       ?GetReward@CCryLobby@@UEAAPEAUICryReward@@XZ 0000000039a07a90 f i CryLobby.obj
 0001:00006ac0       ?GetStats@CCryLobby@@UEAAPEAUICryStats@@XZ 0000000039a07ac0 f i CryLobby.obj
 0001:00006af0       ?GetOnlineStorage@CCryLobby@@UEAAPEAUICryOnlineStorage@@XZ 0000000039a07af0 f i CryLobby.obj
 0001:00006b20       ?GetLobbyUI@CCryLobby@@UEAAPEAUICryLobbyUI@@XZ 0000000039a07b20 f i CryLobby.obj
 0001:00006b50       ?GetFriends@CCryLobby@@UEAAPEAUICryFriends@@XZ 0000000039a07b50 f i CryLobby.obj
 0001:00006b80       ?GetFriendsManagement@CCryLobby@@UEAAPEAUICryFriendsManagement@@XZ 0000000039a07b80 f i CryLobby.obj
 0001:00006bb0       ?GetDLCStore@CCryLobby@@UEAAPEAUICryDLCStore@@XZ 0000000039a07bb0 f i CryLobby.obj
 0001:00006be0       ?GetLobbyService@CCryLobby@@UEAAPEAUICryLobbyService@@W4ECryLobbyService@@@Z 0000000039a07be0 f i CryLobby.obj
 0001:00006c00       ?SetCryEngineLoadHint@CCryLobby@@UEAAXPEBD0@Z 0000000039a07c00 f i CryLobby.obj
 0001:00006c50       ?SetUserPacketEnd@CCryLobby@@UEAAXI@Z 0000000039a07c50 f i CryLobby.obj
 0001:00006c60       ?Initialise@CCryLobby@@UEAA?AW4ECryLobbyError@@W4ECryLobbyService@@W4ECryLobbyServiceFeatures@@P6AX0PEAUSConfigurationParams@@I@ZP6AX0W42@PEAX@Z5@Z 0000000039a07c60 f   CryLobby.obj
 0001:00006eb0       ?ProcessEvents@CCryLobby@@UEAA?AW4ECryLobbyError@@XZ 0000000039a07eb0 f   CryLobby.obj
 0001:00006f60       ?Terminate@CCryLobbyService@@UEAA?AW4ECryLobbyError@@W4ECryLobbyServiceFeatures@@P6AXW42@PEAVCCryLobby@@W4ECryLobbyService@@@Z@Z 0000000039a07f60 f   CryLobby.obj
 0001:00006fe0       ??_E?$CVisitor@V?$CNode@USNullAddr@@V?$CNode@GV?$CNode@USIPv4Addr@@V?$CNode@ULobbyIdAddr@@VCEnd@NTypelist@@@NTypelist@@@NTypelist@@@NTypelist@@@NTypelist@@VCComparatorVisitor@?$less@V?$CConfigurableVariant@V?$CNode@USNullAddr@@V?$CNode@GV?$CNode@USIPv4Addr@@V?$CNode@ULobbyIdAddr@@VCEnd@NTypelist@@@NTypelist@@@NTypelist@@@NTypelist@@@NTypelist@@$07VCDefaultVariantConversion@NConfigurableVariantHelpers@@VCDefaultVariantConstruction@4@@@@stlpmtx_std@@U?$IVisitor@V?$CNode@USNullAddr@@V?$CNode@GV?$CNode@USIPv4Addr@@V?$CNode@ULobbyIdAddr@@VCEnd@NTypelist@@@NTypelist@@@NTypelist@@@NTypelist@@@NTypelist@@@NConfigurableVariantHelpers@@@NConfigurableVariantHelpers@@WBA@EAAPEAXI@Z 0000000039a07fe0 f i CryLobby.obj
 0001:00006ff0       ??_E?$CVisitor@V?$CNode@USNullAddr@@V?$CNode@GV?$CNode@USIPv4Addr@@V?$CNode@ULobbyIdAddr@@VCEnd@NTypelist@@@NTypelist@@@NTypelist@@@NTypelist@@@NTypelist@@VCComparatorVisitor@?$less@V?$CConfigurableVariant@V?$CNode@USNullAddr@@V?$CNode@GV?$CNode@USIPv4Addr@@V?$CNode@ULobbyIdAddr@@VCEnd@NTypelist@@@NTypelist@@@NTypelist@@@NTypelist@@@NTypelist@@$07VCDefaultVariantConversion@NConfigurableVariantHelpers@@VCDefaultVariantConstruction@4@@@@stlpmtx_std@@U?$IVisitor@V?$CNode@USNullAddr@@V?$CNode@GV?$CNode@USIPv4Addr@@V?$CNode@ULobbyIdAddr@@VCEnd@NTypelist@@@NTypelist@@@NTypelist@@@NTypelist@@@NTypelist@@@NConfigurableVariantHelpers@@@NConfigurableVariantHelpers@@WBI@EAAPEAXI@Z 0000000039a07ff0 f i CryLobby.obj
 0001:00007000       ??_E?$CVisitor@V?$CNode@USNullAddr@@V?$CNode@GV?$CNode@USIPv4Addr@@V?$CNode@ULobbyIdAddr@@VCEnd@NTypelist@@@NTypelist@@@NTypelist@@@NTypelist@@@NTypelist@@VCComparatorVisitor@?$less@V?$CConfigurableVariant@V?$CNode@USNullAddr@@V?$CNode@GV?$CNode@USIPv4Addr@@V?$CNode@ULobbyIdAddr@@VCEnd@NTypelist@@@NTypelist@@@NTypelist@@@NTypelist@@@NTypelist@@$07VCDefaultVariantConversion@NConfigurableVariantHelpers@@VCDefaultVariantConstruction@4@@@@stlpmtx_std@@U?$IVisitor@V?$CNode@USNullAddr@@V?$CNode@GV?$CNode@USIPv4Addr@@V?$CNode@ULobbyIdAddr@@VCEnd@NTypelist@@@NTypelist@@@NTypelist@@@NTypelist@@@NTypelist@@@NConfigurableVariantHelpers@@@NConfigurableVariantHelpers@@W7EAAPEAXI@Z 0000000039a08000 f i CryLobby.obj
 0001:00007010       ?AbstractVisit@?$CVisitor@V?$CNode@USNullAddr@@V?$CNode@GV?$CNode@USIPv4Addr@@V?$CNode@ULobbyIdAddr@@VCEnd@NTypelist@@@NTypelist@@@NTypelist@@@NTypelist@@@NTypelist@@VCComparatorVisitor@?$less@V?$CConfigurableVariant@V?$CNode@USNullAddr@@V?$CNode@GV?$CNode@USIPv4Addr@@V?$CNode@ULobbyIdAddr@@VCEnd@NTypelist@@@NTypelist@@@NTypelist@@@NTypelist@@@NTypelist@@$07VCDefaultVariantConversion@NConfigurableVariantHelpers@@VCDefaultVariantConstruction@4@@@@stlpmtx_std@@U?$IVisitor@V?$CNode@USNullAddr@@V?$CNode@GV?$CNode@USIPv4Addr@@V?$CNode@ULobbyIdAddr@@VCEnd@NTypelist@@@NTypelist@@@NTypelist@@@NTypelist@@@NTypelist@@@NConfigurableVariantHelpers@@@NConfigurableVariantHelpers@@UEAAXAEBUSNullAddr@@PEAX@Z 0000000039a08010 f i CryLobby.obj
 0001:00007020       ??_E?$CVisitor@V?$CNode@USNullAddr@@V?$CNode@GV?$CNode@USIPv4Addr@@V?$CNode@ULobbyIdAddr@@VCEnd@NTypelist@@@NTypelist@@@NTypelist@@@NTypelist@@@NTypelist@@VCComparatorVisitor@?$less@V?$CConfigurableVariant@V?$CNode@USNullAddr@@V?$CNode@GV?$CNode@USIPv4Addr@@V?$CNode@ULobbyIdAddr@@VCEnd@NTypelist@@@NTypelist@@@NTypelist@@@NTypelist@@@NTypelist@@$07VCDefaultVariantConversion@NConfigurableVariantHelpers@@VCDefaultVariantConstruction@4@@@@stlpmtx_std@@U?$IVisitor@V?$CNode@USNullAddr@@V?$CNode@GV?$CNode@USIPv4Addr@@V?$CNode@ULobbyIdAddr@@VCEnd@NTypelist@@@NTypelist@@@NTypelist@@@NTypelist@@@NTypelist@@@NConfigurableVariantHelpers@@@NConfigurableVariantHelpers@@UEAAPEAXI@Z 0000000039a08020 f i CryLobby.obj
 0001:00007020       ??_G?$CVisitor@V?$CNode@USNullAddr@@V?$CNode@GV?$CNode@USIPv4Addr@@V?$CNode@ULobbyIdAddr@@VCEnd@NTypelist@@@NTypelist@@@NTypelist@@@NTypelist@@@NTypelist@@VCComparatorVisitor@?$less@V?$CConfigurableVariant@V?$CNode@USNullAddr@@V?$CNode@GV?$CNode@USIPv4Addr@@V?$CNode@ULobbyIdAddr@@VCEnd@NTypelist@@@NTypelist@@@NTypelist@@@NTypelist@@@NTypelist@@$07VCDefaultVariantConversion@NConfigurableVariantHelpers@@VCDefaultVariantConstruction@4@@@@stlpmtx_std@@U?$IVisitor@V?$CNode@USNullAddr@@V?$CNode@GV?$CNode@USIPv4Addr@@V?$CNode@ULobbyIdAddr@@VCEnd@NTypelist@@@NTypelist@@@NTypelist@@@NTypelist@@@NTypelist@@@NConfigurableVariantHelpers@@@NConfigurableVariantHelpers@@UEAAPEAXI@Z 0000000039a08020 f i CryLobby.obj
 0001:00007070       ??0CCryLobby@@QEAA@XZ      0000000039a08070 f   CryLobby.obj
 0001:00007440       ??_ECCryLobby@@UEAAPEAXI@Z 0000000039a08440 f i CryLobby.obj
 0001:00007440       ??_GCCryLobby@@UEAAPEAXI@Z 0000000039a08440 f i CryLobby.obj
 0001:00007470       ?StartTaskRunning@CCryLobbyService@@IEAAXI@Z 0000000039a08470 f   CryLobby.obj
 0001:00007530       ?GetUserPrivileges@CCryLobbyService@@UEAA?AW4ECryLobbyError@@IPEAIP6AXIW42@IPEAX@Z2@Z 0000000039a08530 f   CryLobby.obj
 0001:00007610       ??8@YA_NAEBV?$CConfigurableVariant@V?$CNode@USNullAddr@@V?$CNode@GV?$CNode@USIPv4Addr@@V?$CNode@ULobbyIdAddr@@VCEnd@NTypelist@@@NTypelist@@@NTypelist@@@NTypelist@@@NTypelist@@$07VCDefaultVariantConversion@NConfigurableVariantHelpers@@VCDefaultVariantConstruction@4@@@0@Z 0000000039a08610 f i CryLobby.obj
 0001:00007710       ?FindConnection@CCryLobby@@QEAA?AV?$CryLobbyID@USCryLobbyConnectionID@@$0EA@@@AEBV?$CConfigurableVariant@V?$CNode@USNullAddr@@V?$CNode@GV?$CNode@USIPv4Addr@@V?$CNode@ULobbyIdAddr@@VCEnd@NTypelist@@@NTypelist@@@NTypelist@@@NTypelist@@@NTypelist@@$07VCDefaultVariantConversion@NConfigurableVariantHelpers@@VCDefaultVariantConstruction@4@@@@Z 0000000039a08710 f   CryLobby.obj
 0001:00007810       ?ConnectionFromAddress@CCryLobby@@QEAA_NPEAV?$CryLobbyID@USCryLobbyConnectionID@@$0EA@@@AEBV?$CConfigurableVariant@V?$CNode@USNullAddr@@V?$CNode@GV?$CNode@USIPv4Addr@@V?$CNode@ULobbyIdAddr@@VCEnd@NTypelist@@@NTypelist@@@NTypelist@@@NTypelist@@@NTypelist@@$07VCDefaultVariantConversion@NConfigurableVariantHelpers@@VCDefaultVariantConstruction@4@@@@Z 0000000039a08810 f   CryLobby.obj
 0001:00007840       ?Send@CCryLobby@@QEAA?AW4ESocketError@@PEAVCCryLobbyPacket@@AEBV?$CConfigurableVariant@V?$CNode@USNullAddr@@V?$CNode@GV?$CNode@USIPv4Addr@@V?$CNode@ULobbyIdAddr@@VCEnd@NTypelist@@@NTypelist@@@NTypelist@@@NTypelist@@@NTypelist@@$07VCDefaultVariantConversion@NConfigurableVariantHelpers@@VCDefaultVariantConstruction@4@@@V?$CryLobbyID@USCryLobbyConnectionID@@$0EA@@@PEAI@Z 0000000039a08840 f   CryLobby.obj
 0001:00007bc0       ?OnPacket@CCryLobby@@UEAAXAEBV?$CConfigurableVariant@V?$CNode@USNullAddr@@V?$CNode@GV?$CNode@USIPv4Addr@@V?$CNode@ULobbyIdAddr@@VCEnd@NTypelist@@@NTypelist@@@NTypelist@@@NTypelist@@@NTypelist@@$07VCDefaultVariantConversion@NConfigurableVariantHelpers@@VCDefaultVariantConstruction@4@@@PEBEI@Z 0000000039a08bc0 f   CryLobby.obj
 0001:00007d10       ?OnError@CCryLobby@@UEAAXAEBV?$CConfigurableVariant@V?$CNode@USNullAddr@@V?$CNode@GV?$CNode@USIPv4Addr@@V?$CNode@ULobbyIdAddr@@VCEnd@NTypelist@@@NTypelist@@@NTypelist@@@NTypelist@@@NTypelist@@$07VCDefaultVariantConversion@NConfigurableVariantHelpers@@VCDefaultVariantConstruction@4@@@W4ESocketError@@@Z 0000000039a08d10 f   CryLobby.obj
 0001:00007f10       ?OnSendComplete@CCryLobby@@QEAAXAEBV?$CConfigurableVariant@V?$CNode@USNullAddr@@V?$CNode@GV?$CNode@USIPv4Addr@@V?$CNode@ULobbyIdAddr@@VCEnd@NTypelist@@@NTypelist@@@NTypelist@@@NTypelist@@@NTypelist@@$07VCDefaultVariantConversion@NConfigurableVariantHelpers@@VCDefaultVariantConstruction@4@@@@Z 0000000039a08f10 f   CryLobby.obj
 0001:000080e0       ?ProcessPacket@CCryLobby@@QEAAXAEBV?$CConfigurableVariant@V?$CNode@USNullAddr@@V?$CNode@GV?$CNode@USIPv4Addr@@V?$CNode@ULobbyIdAddr@@VCEnd@NTypelist@@@NTypelist@@@NTypelist@@@NTypelist@@@NTypelist@@$07VCDefaultVariantConversion@NConfigurableVariantHelpers@@VCDefaultVariantConstruction@4@@@V?$CryLobbyID@USCryLobbyConnectionID@@$0EA@@@PEAVCCryLobbyPacket@@@Z 0000000039a090e0 f   CryLobby.obj
 0001:00008900       ?ProcessCachedPacketBuffer@CCryLobby@@QEAAXXZ 0000000039a09900 f   CryLobby.obj
 0001:00009270       ?Tick@CCryLobby@@UEAAX_N@Z 0000000039a0a270 f   CryLobby.obj
 0001:00009ee0       ??0CryLock_WinMutex@@QEAA@XZ 0000000039a0aee0 f   CryLobbyDLL.obj
 0001:00009f10       ??1CryLock_WinMutex@@QEAA@XZ 0000000039a0af10 f   CryLobbyDLL.obj
 0001:00009f20       ?Lock@CryLock_WinMutex@@QEAAXXZ 0000000039a0af20 f   CryLobbyDLL.obj
 0001:00009f30       ?Unlock@CryLock_WinMutex@@QEAAXXZ 0000000039a0af30 f   CryLobbyDLL.obj
 0001:00009f40       ?TryLock@CryLock_WinMutex@@QEAA_NXZ 0000000039a0af40 f   CryLobbyDLL.obj
 0001:00009f60       ??0CryLock_CritSection@@QEAA@XZ 0000000039a0af60 f   CryLobbyDLL.obj
 0001:00009f80       gsiDeleteCriticalSection   0000000039a0af80 f   GameSpy_2.11.00_VC10:gsPlatformThread.obj
 0001:00009f80       ??1CryLock_CritSection@@QEAA@XZ 0000000039a0af80 f   CryLobbyDLL.obj
 0001:00009f90       ?Lock@CryLock_CritSection@@QEAAXXZ 0000000039a0af90 f   CryLobbyDLL.obj
 0001:00009f90       gsiEnterCriticalSection    0000000039a0af90 f   GameSpy_2.11.00_VC10:gsPlatformThread.obj
 0001:00009fa0       ?Unlock@CryLock_CritSection@@QEAAXXZ 0000000039a0afa0 f   CryLobbyDLL.obj
 0001:00009fa0       gsiLeaveCriticalSection    0000000039a0afa0 f   GameSpy_2.11.00_VC10:gsPlatformThread.obj
 0001:00009fb0       ?TryLock@CryLock_CritSection@@QEAA_NXZ 0000000039a0afb0 f   CryLobbyDLL.obj
 0001:00009fd0       ?gen_state@CMTRand_int32@@AEAAXXZ 0000000039a0afd0 f   CryLobbyDLL.obj
 0001:0000a1a0       ?seed@CMTRand_int32@@QEAAXI@Z 0000000039a0b1a0 f   CryLobbyDLL.obj
 0001:0000a210       ?cry_rand@@YAIXZ           0000000039a0b210 f   CryLobbyDLL.obj
 0001:0000a240       ?Init@_CryMemoryManagerPoolHelper@@SAXXZ 0000000039a0b240 f i CryLobbyDLL.obj
 0001:0000a440       ?CryGetIMemoryManager@@YAPEAUIMemoryManager@@XZ 0000000039a0b440 f   CryLobbyDLL.obj
 0001:0000a490       ?CryInterlockedIncrement@@YAJPECH@Z 0000000039a0b490 f   CryLobbyDLL.obj
 0001:0000a4a0       ?CryInterlockedDecrement@@YAJPECH@Z 0000000039a0b4a0 f   CryLobbyDLL.obj
 0001:0000a4b0       ?CryGetCurrentThreadId@@YAIXZ 0000000039a0b4b0 f   CryLobbyDLL.obj
 0001:0000a4c0       ?CryPureCallHandler@@YAXXZ 0000000039a0b4c0 f   CryLobbyDLL.obj
 0001:0000a4d0       ?CryInvalidParameterHandler@@YAXPEB_W00I_K@Z 0000000039a0b4d0 f   CryLobbyDLL.obj
 0001:0000a4e0       ModuleInitISystem          0000000039a0b4e0 f   CryLobbyDLL.obj
 0001:0000a5b0       CryModuleGetMemoryInfo     0000000039a0b5b0 f   CryLobbyDLL.obj
 0001:0000a5f0       ?CryDeleteCriticalSectionInplace@@YAXPEAX@Z 0000000039a0b5f0 f   CryLobbyDLL.obj
 0001:0000a620       CryModuleMalloc            0000000039a0b620 f   CryLobbyDLL.obj
 0001:0000a6c0       CryModuleFree              0000000039a0b6c0 f   CryLobbyDLL.obj
 0001:0000a730       CryModuleMemalign          0000000039a0b730 f   CryLobbyDLL.obj
 0001:0000a7e0       ??2@YAPEAX_K@Z             0000000039a0b7e0 f   CryLobbyDLL.obj
 0001:0000a850       ??_U@YAPEAX_K@Z            0000000039a0b850 f   CryLobbyDLL.obj
 0001:0000a8c0       ??3@YAXPEAX@Z              0000000039a0b8c0 f   CryLobbyDLL.obj
 0001:0000a960       ??_V@YAXPEAX@Z             0000000039a0b960 f   CryLobbyDLL.obj
 0001:0000aa00       ??_GICryUnknown@@MEAAPEAXI@Z 0000000039a0ba00 f i CryLobbyDLL.obj
 0001:0000aa00       ??_ECEngineModule_CryLobby@@MEAAPEAXI@Z 0000000039a0ba00 f i CryLobbyDLL.obj
 0001:0000aa00       ??_GCEngineModule_CryLobby@@MEAAPEAXI@Z 0000000039a0ba00 f i CryLobbyDLL.obj
 0001:0000aa00       ??_EICryUnknown@@MEAAPEAXI@Z 0000000039a0ba00 f i CryLobbyDLL.obj
 0001:0000aa30       ??_GICryFactory@@MEAAPEAXI@Z 0000000039a0ba30 f i CryLobbyDLL.obj
 0001:0000aa30       ??_EICryFactory@@MEAAPEAXI@Z 0000000039a0ba30 f i CryLobbyDLL.obj
 0001:0000aa60       ??_GCSystemEventListner_CryLobby@@UEAAPEAXI@Z 0000000039a0ba60 f i CryLobbyDLL.obj
 0001:0000aa60       ??_ECSystemEventListner_CryLobby@@UEAAPEAXI@Z 0000000039a0ba60 f i CryLobbyDLL.obj
 0001:0000aa90       ?GetFactory@CEngineModule_CryLobby@@UEBAPEAUICryFactory@@XZ 0000000039a0ba90 f i CryLobbyDLL.obj
 0001:0000aaa0       ?GetName@CEngineModule_CryLobby@@MEAAPEBDXZ 0000000039a0baa0 f i CryLobbyDLL.obj
 0001:0000aab0       ?GetCategory@CEngineModule_CryLobby@@MEAAPEBDXZ 0000000039a0bab0 f i CryLobbyDLL.obj
 0001:0000aac0       ?Initialize@CEngineModule_CryLobby@@MEAA_NAEAUSSystemGlobalEnvironment@@AEBUSSystemInitParams@@@Z 0000000039a0bac0 f i CryLobbyDLL.obj
 0001:0000ab80       ?_AllocData@?$CryStringT@_W@@IEAAX_K@Z 0000000039a0bb80 f i CryLobbyDLL.obj
 0001:0000abf0       ?_AllocData@?$CryStackStringT@D$0BAA@@@QEAAX_K@Z 0000000039a0bbf0 f i CryLobbyDLL.obj
 0001:0000ac70       ?_Free@?$CryStringT@D@@IEAAXXZ 0000000039a0bc70 f i CryLobbyDLL.obj
 0001:0000acc0       ?_Assign@?$CryStringT@D@@IEAAXPEBD_K@Z 0000000039a0bcc0 f i CryLobbyDLL.obj
 0001:0000ada0       ?_MakeUnique@?$CryStringT@D@@IEAAXXZ 0000000039a0bda0 f i CryLobbyDLL.obj
 0001:0000ae60       ??0CFactory@CEngineModule_CryLobby@@AEAA@XZ 0000000039a0be60 f i CryLobbyDLL.obj
 0001:0000af00       ?GetClassNameA@CFactory@CEngineModule_CryLobby@@UEBAPEBDXZ 0000000039a0bf00 f i CryLobbyDLL.obj
 0001:0000af10       ?GetClassID@CFactory@CEngineModule_CryLobby@@UEBAAEBUCryGUID@@XZ 0000000039a0bf10 f i CryLobbyDLL.obj
 0001:0000af20       ?ClassSupports@CFactory@CEngineModule_CryLobby@@UEBA_NAEBUCryGUID@@@Z 0000000039a0bf20 f i CryLobbyDLL.obj
 0001:0000af60       ?ClassSupports@CFactory@CEngineModule_CryLobby@@UEBAXAEAPEBUCryGUID@@AEA_K@Z 0000000039a0bf60 f i CryLobbyDLL.obj
 0001:0000af70       ?destroy@sp_counted_base@detail@boost@@UEAAXXZ 0000000039a0bf70 f i CryLobbyDLL.obj
 0001:0000af90       ?sp_enable_shared_from_this@detail@boost@@YAXZZ 0000000039a0bf90 f i CryLobbyDLL.obj
 0001:0000afb0       ?dispose@?$sp_counted_impl_p@VCEngineModule_CryLobby@@@detail@boost@@UEAAXXZ 0000000039a0bfb0 f i CryLobbyDLL.obj
 0001:0000afd0       ??_GCFactory@CEngineModule_CryLobby@@UEAAPEAXI@Z 0000000039a0bfd0 f i CryLobbyDLL.obj
 0001:0000afd0       ??_ECFactory@CEngineModule_CryLobby@@UEAAPEAXI@Z 0000000039a0bfd0 f i CryLobbyDLL.obj
 0001:0000b010       ??$?0VCEngineModule_CryLobby@@@shared_count@detail@boost@@QEAA@PEAVCEngineModule_CryLobby@@@Z 0000000039a0c010 f i CryLobbyDLL.obj
 0001:0000b120       ??_G?$sp_counted_impl_p@VCEngineModule_CryLobby@@@detail@boost@@UEAAPEAXI@Z 0000000039a0c120 f i CryLobbyDLL.obj
 0001:0000b120       ??_Gsp_counted_base@detail@boost@@UEAAPEAXI@Z 0000000039a0c120 f i CryLobbyDLL.obj
 0001:0000b120       ??_Esp_counted_base@detail@boost@@UEAAPEAXI@Z 0000000039a0c120 f i CryLobbyDLL.obj
 0001:0000b120       ??_E?$sp_counted_impl_p@VCEngineModule_CryLobby@@@detail@boost@@UEAAPEAXI@Z 0000000039a0c120 f i CryLobbyDLL.obj
 0001:0000b150       ??_Gbad_alloc@std@@UEAAPEAXI@Z 0000000039a0c150 f i CryLobbyDLL.obj
 0001:0000b150       ??_Ebad_alloc@std@@UEAAPEAXI@Z 0000000039a0c150 f i CryLobbyDLL.obj
 0001:0000b190       ?QueryInterface@CEngineModule_CryLobby@@MEBAPEAXAEBUCryGUID@@@Z 0000000039a0c190 f i CryLobbyDLL.obj
 0001:0000b1e0       ?_Assign@?$CryStringT@_W@@IEAAXPEB_W_K@Z 0000000039a0c1e0 f i CryLobbyDLL.obj
 0001:0000b2d0       ?_Assign@?$CryStackStringT@D$0BAA@@@QEAAXPEBD_K@Z 0000000039a0c2d0 f i CryLobbyDLL.obj
 0001:0000b370       ??4?$CryStringT@D@@QEAAAEAV0@PEBD@Z 0000000039a0c370 f i CryLobbyDLL.obj
 0001:0000b3c0       ??4?$CryStringT@D@@QEAAAEAV0@AEBV0@@Z 0000000039a0c3c0 f i CryLobbyDLL.obj
 0001:0000b470       ?append@?$CryStringT@D@@QEAAAEAV1@_KD@Z 0000000039a0c470 f i CryLobbyDLL.obj
 0001:0000b560       ?CreateClassInstance@CFactory@CEngineModule_CryLobby@@UEBA?AV?$shared_ptr@UICryUnknown@@@boost@@XZ 0000000039a0c560 f i CryLobbyDLL.obj
 0001:0000b630       ?Initialise@CCryLobbyUI@@QEAA?AW4ECryLobbyError@@XZ 0000000039a0c630 f   CryLobbyUI.obj
 0001:0000b640       ?StartTask@CCryLobbyUI@@IEAA?AW4ECryLobbyError@@I_NPEAI1V?$CryLobbyID@USCryLobbySessionHandle@@$03@@PEAX3@Z 0000000039a0c640 f   CryLobbyUI.obj
 0001:0000b730       ?FreeTask@CCryLobbyUI@@IEAAXI@Z 0000000039a0c730 f   CryLobbyUI.obj
 0001:0000b7b0       ?CreateTaskParamMem@CCryLobbyUI@@IEAA?AW4ECryLobbyError@@IIPEBX_K@Z 0000000039a0c7b0 f   CryLobbyUI.obj
 0001:0000b840       ?UpdateTaskError@CCryFriends@@IEAAXIW4ECryLobbyError@@@Z 0000000039a0c840 f   CryFriends.obj
 0001:0000b840       ?UpdateTaskError@CCryLobbyUI@@IEAAXIW4ECryLobbyError@@@Z 0000000039a0c840 f   CryLobbyUI.obj
 0001:0000b840       ?UpdateTaskError@CCryStats@@IEAAXIW4ECryLobbyError@@@Z 0000000039a0c840 f   CryStats.obj
 0001:0000b840       ?UpdateTaskError@CCryFriendsManagement@@IEAAXIW4ECryLobbyError@@@Z 0000000039a0c840 f   CryFriendsManagement.obj
 0001:0000b860       ??0CCryLobbyUI@@QEAA@PEAVCCryLobby@@PEAVCCryLobbyService@@@Z 0000000039a0c860 f   CryLobbyUI.obj
 0001:0000b8a0       ?Terminate@CCryLobbyUI@@QEAA?AW4ECryLobbyError@@XZ 0000000039a0c8a0 f   CryLobbyUI.obj
 0001:0000b920       ?ReadUINT32@CCryLobbyPacket@@QEAAIXZ 0000000039a0c920 f i CryMatchMaking.obj
 0001:0000b980       ?GetChannelIDFromGameSessionHandle@CCryMatchMaking@@UEAAGI@Z 0000000039a0c980 f   CryMatchMaking.obj
 0001:0000b990       ?StartSubTask@CCryMatchMaking@@IEAAXII@Z 0000000039a0c990 f   CryMatchMaking.obj
 0001:0000b9a0       ?FreeTask@CCryMatchMaking@@IEAAXI@Z 0000000039a0c9a0 f   CryMatchMaking.obj
 0001:0000ba30       ?MatchmakingSessionJoinFromConsoleCallback@CCryMatchMaking@@KAXIW4ECryLobbyError@@IIGPEAX@Z 0000000039a0ca30 f   CryMatchMaking.obj
 0001:0000bae0       ?CreateTaskParam@CCryMatchMaking@@IEAA?AW4ECryLobbyError@@IIPEBXI_K@Z 0000000039a0cae0 f   CryMatchMaking.obj
 0001:0000bb80       ?FindTaskFromTaskTaskID@CCryMatchMaking@@IEAAIII@Z 0000000039a0cb80 f   CryMatchMaking.obj
 0001:0000bbb0       ?UpdateTaskError@CCryMatchMaking@@IEAAXIW4ECryLobbyError@@@Z 0000000039a0cbb0 f   CryMatchMaking.obj
 0001:0000bbd0       ?PacketToMemoryBlock@CCryMatchMaking@@IEAAIPEAVCCryLobbyPacket@@AEAI@Z 0000000039a0cbd0 f   CryMatchMaking.obj
 0001:0000bc80       ?MemoryBlockToPacket@CCryMatchMaking@@IEAAPEAVCCryLobbyPacket@@II@Z 0000000039a0cc80 f   CryMatchMaking.obj
 0001:0000bd00       ?OnError@CCryMatchMaking@@QEAAXAEBV?$CConfigurableVariant@V?$CNode@USNullAddr@@V?$CNode@GV?$CNode@USIPv4Addr@@V?$CNode@ULobbyIdAddr@@VCEnd@NTypelist@@@NTypelist@@@NTypelist@@@NTypelist@@@NTypelist@@$07VCDefaultVariantConversion@NConfigurableVariantHelpers@@VCDefaultVariantConstruction@4@@@W4ESocketError@@I@Z 0000000039a0cd00 f   CryMatchMaking.obj
 0001:0000bd50       ?OnSendComplete@CCryMatchMaking@@QEAAXAEBV?$CConfigurableVariant@V?$CNode@USNullAddr@@V?$CNode@GV?$CNode@USIPv4Addr@@V?$CNode@ULobbyIdAddr@@VCEnd@NTypelist@@@NTypelist@@@NTypelist@@@NTypelist@@@NTypelist@@$07VCDefaultVariantConversion@NConfigurableVariantHelpers@@VCDefaultVariantConstruction@4@@@I@Z 0000000039a0cd50 f   CryMatchMaking.obj
 0001:0000bda0       ?DispatchSessionEvent@CCryMatchMaking@@IEAAXIW4ECryLobbySystemEvent@@@Z 0000000039a0cda0 f   CryMatchMaking.obj
 0001:0000bdd0       ??_EICryMatchMaking@@UEAAPEAXI@Z 0000000039a0cdd0 f i CryMatchMaking.obj
 0001:0000bdd0       ??_GICryMatchMaking@@UEAAPEAXI@Z 0000000039a0cdd0 f i CryMatchMaking.obj
 0001:0000be00       ?ReadConnectionUID@CCryLobbyPacket@@QEAA?AUSCryMatchMakingConnectionUID@@XZ 0000000039a0ce00 f i CryMatchMaking.obj
 0001:0000be70       ?LobbyAddrIDSend@ICryMatchMakingPrivate@@UEAA?AW4ESocketError@@PEBEIAEBV?$CConfigurableVariant@V?$CNode@USNullAddr@@V?$CNode@GV?$CNode@USIPv4Addr@@V?$CNode@ULobbyIdAddr@@VCEnd@NTypelist@@@NTypelist@@@NTypelist@@@NTypelist@@@NTypelist@@$07VCDefaultVariantConversion@NConfigurableVariantHelpers@@VCDefaultVariantConstruction@4@@@@Z 0000000039a0ce70 f i CryMatchMaking.obj
 0001:0000be80       ?CreateGameSessionHandle@CCryMatchMaking@@QEAAIV?$CryLobbyID@USCryLobbySessionHandle@@$03@@USCryMatchMakingConnectionUID@@@Z 0000000039a0ce80 f   CryMatchMaking.obj
 0001:0000bea0       ?CreateConnectionUID@CCryMatchMaking@@QEAA?AUSCryMatchMakingConnectionUID@@V?$CryLobbyID@USCryLobbySessionHandle@@$03@@@Z 0000000039a0cea0 f   CryMatchMaking.obj
 0001:0000bf00       ?StartTask@CCryMatchMaking@@IEAA?AW4ECryLobbyError@@I_NPEAI1V?$CryLobbyID@USCryLobbySessionHandle@@$03@@PEAX3@Z 0000000039a0cf00 f   CryMatchMaking.obj
 0001:0000c060       ?FindTaskFromLobbyTaskID@CCryMatchMaking@@IEAAII@Z 0000000039a0d060 f   CryMatchMaking.obj
 0001:0000c0f0       ??A?$CryLobbyIDArray@PEAUSRConnection@SSession@CCryMatchMaking@@V?$CryLobbyID@USCryMatchMakingConnectionID@@$0EA@@@$0EA@@@QEAAAEAPEAUSRConnection@SSession@CCryMatchMaking@@AEBV?$CryLobbyID@USCryMatchMakingConnectionID@@$0EA@@@@Z 0000000039a0d0f0 f i CryMatchMaking.obj
 0001:0000c130       ??0?$CryLobbyID@USCryMatchMakingConnectionID@@$0EA@@@QEAA@I@Z 0000000039a0d130 f i CryMatchMaking.obj
 0001:0000c130       ??0?$CryLobbyID@USCryLobbyConnectionID@@$0EA@@@QEAA@I@Z 0000000039a0d130 f i CryLobby.obj
 0001:0000c180       ??0?$CryLobbyID@USCryLobbySessionHandle@@$03@@QEAA@I@Z 0000000039a0d180 f i CryMatchMaking.obj
 0001:0000c1d0       ?_M_advance@?$_Deque_iterator_base@USBannedUser@@@priv@stlpmtx_std@@QEAAX_J@Z 0000000039a0d1d0 f i CryMatchMaking.obj
 0001:0000c250       ?Draw2dLabel@IRenderer@@QEAAXMMMPEBM_NPEBDZZ 0000000039a0d250 f i CryMatchMaking.obj
 0001:0000c310       ?Reset@SSession@CCryMatchMaking@@UEAAXXZ 0000000039a0d310 f   CryMatchMaking.obj
 0001:0000c3c0       ?GetSessionHandleFromGameSessionHandle@CCryMatchMaking@@QEAA?AV?$CryLobbyID@USCryLobbySessionHandle@@$03@@I@Z 0000000039a0d3c0 f   CryMatchMaking.obj
 0001:0000c420       ?GetConnectionUIDFromGameSessionHandleAndChannelID@CCryMatchMaking@@UEAA?AUSCryMatchMakingConnectionUID@@IG@Z 0000000039a0d420 f   CryMatchMaking.obj
 0001:0000c4c0       ?GetConnectionUIDFromNubAndGameSessionHandle@CCryMatchMaking@@QEAA?AUSCryMatchMakingConnectionUID@@I@Z 0000000039a0d4c0 f   CryMatchMaking.obj
 0001:0000c5e0       ?DrawDebugText@CCryMatchMaking@@IEAAXXZ 0000000039a0d5e0 f   CryMatchMaking.obj
 0001:0000c720       ?EndTask@CCryMatchMaking@@IEAAXI@Z 0000000039a0d720 f   CryMatchMaking.obj
 0001:0000c840       ?GetCurrentNetNubSessionHandle@CCryMatchMaking@@QEBA?AV?$CryLobbyID@USCryLobbySessionHandle@@$03@@XZ 0000000039a0d840 f   CryMatchMaking.obj
 0001:0000c8e0       ?GetCurrentHostedNetNubSessionHandle@CCryMatchMaking@@QEBA?AV?$CryLobbyID@USCryLobbySessionHandle@@$03@@XZ 0000000039a0d8e0 f   CryMatchMaking.obj
 0001:0000c940       ?GetHostConnectionUID@CCryMatchMaking@@UEAA?AUSCryMatchMakingConnectionUID@@I@Z 0000000039a0d940 f   CryMatchMaking.obj
 0001:0000ca40       ?CancelTask@CCryMatchMaking@@UEAAXI@Z 0000000039a0da40 f   CryMatchMaking.obj
 0001:0000cad0       ?GetSessionIDFromConsole@CCryMatchMaking@@UEAA?AV?$_smart_ptr@USCrySessionID@@@@XZ 0000000039a0dad0 f   CryMatchMaking.obj
 0001:0000cb00       ?SessionJoinFromConsole@CCryMatchMaking@@UEAAXXZ 0000000039a0db00 f   CryMatchMaking.obj
 0001:0000cbd0       ?CreateSessionHandle@CCryMatchMaking@@IEAA?AW4ECryLobbyError@@PEAV?$CryLobbyID@USCryLobbySessionHandle@@$03@@_NIH@Z 0000000039a0dbd0 f   CryMatchMaking.obj
 0001:0000cd00       ?FreeSessionHandle@CCryMatchMaking@@MEAAXV?$CryLobbyID@USCryLobbySessionHandle@@$03@@@Z 0000000039a0dd00 f   CryMatchMaking.obj
 0001:0000cd90       ?FreeRemoteConnection@CCryMatchMaking@@MEAAXV?$CryLobbyID@USCryLobbySessionHandle@@$03@@V?$CryLobbyID@USCryMatchMakingConnectionID@@$0EA@@@@Z 0000000039a0dd90 f   CryMatchMaking.obj
 0001:0000ceb0       ?FindConnectionFromSessionUID@CCryMatchMaking@@IEAA_NV?$CryLobbyID@USCryLobbySessionHandle@@$03@@USCryMatchMakingConnectionUID@@PEAV?$CryLobbyID@USCryMatchMakingConnectionID@@$0EA@@@@Z 0000000039a0deb0 f   CryMatchMaking.obj
 0001:0000cf90       ?Initialise@CCryMatchMaking@@QEAA?AW4ECryLobbyError@@XZ 0000000039a0df90 f   CryMatchMaking.obj
 0001:0000d060       ?Send@CCryMatchMaking@@IEAA?AW4ESocketError@@IPEAVCCryLobbyPacket@@V?$CryLobbyID@USCryLobbySessionHandle@@$03@@AEBV?$CConfigurableVariant@V?$CNode@USNullAddr@@V?$CNode@GV?$CNode@USIPv4Addr@@V?$CNode@ULobbyIdAddr@@VCEnd@NTypelist@@@NTypelist@@@NTypelist@@@NTypelist@@@NTypelist@@$07VCDefaultVariantConversion@NConfigurableVariantHelpers@@VCDefaultVariantConstruction@4@@@@Z 0000000039a0e060 f   CryMatchMaking.obj
 0001:0000d100       ?SessionSendRequestInfo@CCryMatchMaking@@UEAA?AW4ECryLobbyError@@PEAVCCryLobbyPacket@@V?$_smart_ptr@USCrySessionID@@@@PEAIP6AXIW42@0PEAX@Z4@Z 0000000039a0e100 f   CryMatchMaking.obj
 0001:0000d160       ?DispatchUserPacket@CCryMatchMaking@@IEAAXIII@Z 0000000039a0e160 f   CryMatchMaking.obj
 0001:0000d1e0       ?StartSessionModifyLocalFlags@CCryMatchMaking@@IEAAXI@Z 0000000039a0e1e0 f   CryMatchMaking.obj
 0001:0000d260       ?GetSessionPlayerPing@CCryMatchMaking@@UEAA?AW4ECryLobbyError@@USCryMatchMakingConnectionUID@@QEAG@Z 0000000039a0e260 f   CryMatchMaking.obj
 0001:0000d420       ?GetTimeSincePacketFromServerMS@CCryMatchMaking@@UEAAII@Z 0000000039a0e420 f   CryMatchMaking.obj
 0001:0000d4f0       ?DisconnectFromServer@CCryMatchMaking@@UEAAXI@Z 0000000039a0e4f0 f   CryMatchMaking.obj
 0001:0000d5b0       ?StatusCmd@CCryMatchMaking@@UEAAXW4eStatusCmdMode@@@Z 0000000039a0e5b0 f   CryMatchMaking.obj
 0001:0000dcc0       ?KickCmd@CCryMatchMaking@@UEAAXI_KPEBDW4EDisconnectionCause@@@Z 0000000039a0ecc0 f   CryMatchMaking.obj
 0001:0000dcf0       ?Execute@?$CClassJob@XVCCryMatchMaking@@@CWorkQueue@@UEAAXXZ 0000000039a0ecf0 f i CryMatchMaking.obj
 0001:0000dd20       ?Execute@?$CClassJobNoRef4@IIV?$CryLobbyID@USCryLobbySessionHandle@@$03@@USCryMatchMakingConnectionUID@@VCCryMatchMaking@@@CWorkQueue@@UEAAXXZ 0000000039a0ed20 f i CryMatchMaking.obj
 0001:0000dd70       ?Execute@?$CClassJobNoRef2@IW4ECryLobbySystemEvent@@VCCryMatchMaking@@@CWorkQueue@@UEAAXXZ 0000000039a0ed70 f i CryMatchMaking.obj
 0001:0000dd70       ?Execute@?$CClassJobNoRef2@W4ECryLobbySystemEvent@@IVCCryMatchMaking@@@CWorkQueue@@UEAAXXZ 0000000039a0ed70 f i CryMatchMaking.obj
 0001:0000dda0       ?StartTaskRunning@CCryMatchMaking@@IEAAXI@Z 0000000039a0eda0 f   CryMatchMaking.obj
 0001:0000de10       ?FindConnectionFromUID@CCryMatchMaking@@IEAA_NUSCryMatchMakingConnectionUID@@PEAV?$CryLobbyID@USCryLobbySessionHandle@@$03@@PEAV?$CryLobbyID@USCryMatchMakingConnectionID@@$0EA@@@@Z 0000000039a0ee10 f   CryMatchMaking.obj
 0001:0000dec0       ?ProcessServerPing@CCryMatchMaking@@IEAAXAEBV?$CConfigurableVariant@V?$CNode@USNullAddr@@V?$CNode@GV?$CNode@USIPv4Addr@@V?$CNode@ULobbyIdAddr@@VCEnd@NTypelist@@@NTypelist@@@NTypelist@@@NTypelist@@@NTypelist@@$07VCDefaultVariantConversion@NConfigurableVariantHelpers@@VCDefaultVariantConstruction@4@@@PEAVCCrySharedLobbyPacket@@@Z 0000000039a0eec0 f   CryMatchMaking.obj
 0001:0000e220       ??4SCryUserInfoResult@@QEAAAEAU0@AEBU0@@Z 0000000039a0f220 f i CryMatchMaking.obj
 0001:0000e2c0       ??1SBannedUser@@QEAA@XZ    0000000039a0f2c0 f i CryMatchMaking.obj
 0001:0000e340       ??H?$_Deque_iterator@USBannedUser@@U?$_Nonconst_traits@USBannedUser@@@stlpmtx_std@@@priv@stlpmtx_std@@QEBA?AU012@_J@Z 0000000039a0f340 f i CryMatchMaking.obj
 0001:0000e3d0       ??G?$_Deque_iterator@USBannedUser@@U?$_Nonconst_traits@USBannedUser@@@stlpmtx_std@@@priv@stlpmtx_std@@QEBA?AU012@_J@Z 0000000039a0f3d0 f i CryMatchMaking.obj
 0001:0000e470       ??0SBannedUser@@QEAA@AEBU0@@Z 0000000039a0f470 f i CryMatchMaking.obj
 0001:0000e4e0       ??$__fill@U?$_Deque_iterator@USBannedUser@@U?$_Nonconst_traits@USBannedUser@@@stlpmtx_std@@@priv@stlpmtx_std@@USBannedUser@@_J@priv@stlpmtx_std@@YAXU?$_Deque_iterator@USBannedUser@@U?$_Nonconst_traits@USBannedUser@@@stlpmtx_std@@@01@0AEBUSBannedUser@@AEBUrandom_access_iterator_tag@1@PEA_J@Z 0000000039a0f4e0 f i CryMatchMaking.obj
 0001:0000e610       ??$__copy_backward@U?$_Deque_iterator@USBannedUser@@U?$_Nonconst_traits@USBannedUser@@@stlpmtx_std@@@priv@stlpmtx_std@@U123@_J@priv@stlpmtx_std@@YA?AU?$_Deque_iterator@USBannedUser@@U?$_Nonconst_traits@USBannedUser@@@stlpmtx_std@@@01@U201@00AEBUrandom_access_iterator_tag@1@PEA_J@Z 0000000039a0f610 f i CryMatchMaking.obj
 0001:0000e7b0       ??$__copy@U?$_Deque_iterator@USBannedUser@@U?$_Nonconst_traits@USBannedUser@@@stlpmtx_std@@@priv@stlpmtx_std@@U123@_J@priv@stlpmtx_std@@YA?AU?$_Deque_iterator@USBannedUser@@U?$_Nonconst_traits@USBannedUser@@@stlpmtx_std@@@01@U201@00AEBUrandom_access_iterator_tag@1@PEA_J@Z 0000000039a0f7b0 f i CryMatchMaking.obj
 0001:0000e960       ?DispatchSessionUserDataEvent@CCryMatchMaking@@IEAAXW4ECryLobbySystemEvent@@I@Z 0000000039a0f960 f   CryMatchMaking.obj
 0001:0000ea10       ?_M_initialize_map@?$_Deque_base@USBannedUser@@V?$allocator@USBannedUser@@@stlpmtx_std@@@priv@stlpmtx_std@@IEAAX_K@Z 0000000039a0fa10 f i CryMatchMaking.obj
 0001:0000eb30       ?_M_new_elements_at_front@?$_Impl_deque@USBannedUser@@V?$allocator@USBannedUser@@@stlpmtx_std@@@priv@stlpmtx_std@@IEAAX_K@Z 0000000039a0fb30 f i CryMatchMaking.obj
 0001:0000eba0       ?_M_new_elements_at_back@?$_Impl_deque@USBannedUser@@V?$allocator@USBannedUser@@@stlpmtx_std@@@priv@stlpmtx_std@@IEAAX_K@Z 0000000039a0fba0 f i CryMatchMaking.obj
 0001:0000ec20       ??$__ufill@U?$_Deque_iterator@USBannedUser@@U?$_Nonconst_traits@USBannedUser@@@stlpmtx_std@@@priv@stlpmtx_std@@USBannedUser@@_J@priv@stlpmtx_std@@YAXU?$_Deque_iterator@USBannedUser@@U?$_Nonconst_traits@USBannedUser@@@stlpmtx_std@@@01@0AEBUSBannedUser@@AEBUrandom_access_iterator_tag@1@PEA_J@Z 0000000039a0fc20 f i CryMatchMaking.obj
 0001:0000ed20       ??$__destroy_range_aux@U?$_Deque_iterator@USBannedUser@@U?$_Nonconst_traits@USBannedUser@@@stlpmtx_std@@@priv@stlpmtx_std@@USBannedUser@@@stlpmtx_std@@YAXU?$_Deque_iterator@USBannedUser@@U?$_Nonconst_traits@USBannedUser@@@stlpmtx_std@@@priv@0@0PEAUSBannedUser@@AEBU__false_type@0@@Z 0000000039a0fd20 f i CryMatchMaking.obj
 0001:0000ee10       ??$__ucopy@U?$_Deque_iterator@USBannedUser@@U?$_Nonconst_traits@USBannedUser@@@stlpmtx_std@@@priv@stlpmtx_std@@U123@_J@priv@stlpmtx_std@@YA?AU?$_Deque_iterator@USBannedUser@@U?$_Nonconst_traits@USBannedUser@@@stlpmtx_std@@@01@U201@00AEBUrandom_access_iterator_tag@1@PEA_J@Z 0000000039a0fe10 f i CryMatchMaking.obj
 0001:0000ef70       ??$uninitialized_fill@U?$_Deque_iterator@USBannedUser@@U?$_Nonconst_traits@USBannedUser@@@stlpmtx_std@@@priv@stlpmtx_std@@USBannedUser@@@stlpmtx_std@@YAXU?$_Deque_iterator@USBannedUser@@U?$_Nonconst_traits@USBannedUser@@@stlpmtx_std@@@priv@0@0AEBUSBannedUser@@@Z 0000000039a0ff70 f i CryMatchMaking.obj
 0001:0000efe0       ??$__destroy_range@PEAUSBannedUser@@U1@@stlpmtx_std@@YAXPEAUSBannedUser@@00@Z 0000000039a0ffe0 f i CryMatchMaking.obj
 0001:0000f080       ??$uninitialized_copy@U?$_Deque_iterator@USBannedUser@@U?$_Nonconst_traits@USBannedUser@@@stlpmtx_std@@@priv@stlpmtx_std@@U123@@stlpmtx_std@@YA?AU?$_Deque_iterator@USBannedUser@@U?$_Nonconst_traits@USBannedUser@@@stlpmtx_std@@@priv@0@U120@00@Z 0000000039a10080 f i CryMatchMaking.obj
 0001:0000f120       ?AddRemoteConnection@CCryMatchMaking@@IEAA?AV?$CryLobbyID@USCryMatchMakingConnectionID@@$0EA@@@V?$CryLobbyID@USCryLobbySessionHandle@@$03@@V?$CryLobbyID@USCryLobbyConnectionID@@$0EA@@@USCryMatchMakingConnectionUID@@I@Z 0000000039a10120 f   CryMatchMaking.obj
 0001:0000f360       ?Send@CCryMatchMaking@@IEAA?AW4ESocketError@@IPEAVCCryLobbyPacket@@V?$CryLobbyID@USCryLobbySessionHandle@@$03@@V?$CryLobbyID@USCryMatchMakingConnectionID@@$0EA@@@@Z 0000000039a10360 f   CryMatchMaking.obj
 0001:0000f510       ?SendToAll@CCryMatchMaking@@IEAAXIPEAVCCryLobbyPacket@@V?$CryLobbyID@USCryLobbySessionHandle@@$03@@V?$CryLobbyID@USCryMatchMakingConnectionID@@$0EA@@@@Z 0000000039a10510 f   CryMatchMaking.obj
 0001:0000f670       ?SendToServerNT@CCryMatchMaking@@IEAAXIIV?$CryLobbyID@USCryLobbySessionHandle@@$03@@@Z 0000000039a10670 f   CryMatchMaking.obj
 0001:0000f730       ?SendToAllClientsNT@CCryMatchMaking@@IEAAXIIV?$CryLobbyID@USCryLobbySessionHandle@@$03@@@Z 0000000039a10730 f   CryMatchMaking.obj
 0001:0000f7c0       ?SendToClientNT@CCryMatchMaking@@IEAAXIIV?$CryLobbyID@USCryLobbySessionHandle@@$03@@USCryMatchMakingConnectionUID@@@Z 0000000039a107c0 f   CryMatchMaking.obj
 0001:0000f920       ?SendServerPing@CCryMatchMaking@@IEAAXV?$CryLobbyID@USCryLobbySessionHandle@@$03@@@Z 0000000039a10920 f   CryMatchMaking.obj
 0001:0000fb60       ??$__uninitialized_copy_fill@U?$_Deque_iterator@USBannedUser@@U?$_Nonconst_traits@USBannedUser@@@stlpmtx_std@@@priv@stlpmtx_std@@USBannedUser@@@priv@stlpmtx_std@@YAXU?$_Deque_iterator@USBannedUser@@U?$_Nonconst_traits@USBannedUser@@@stlpmtx_std@@@01@000AEBUSBannedUser@@@Z 0000000039a10b60 f i CryMatchMaking.obj
 0001:0000fc70       ??$__uninitialized_fill_copy@U?$_Deque_iterator@USBannedUser@@U?$_Nonconst_traits@USBannedUser@@@stlpmtx_std@@@priv@stlpmtx_std@@USBannedUser@@U123@@priv@stlpmtx_std@@YA?AU?$_Deque_iterator@USBannedUser@@U?$_Nonconst_traits@USBannedUser@@@stlpmtx_std@@@01@U201@0AEBUSBannedUser@@00@Z 0000000039a10c70 f i CryMatchMaking.obj
 0001:0000fd80       ??1?$_Impl_deque@USBannedUser@@V?$allocator@USBannedUser@@@stlpmtx_std@@@priv@stlpmtx_std@@QEAA@XZ 0000000039a10d80 f i CryMatchMaking.obj
 0001:0000fdf0       ?_M_erase@?$_Impl_deque@USBannedUser@@V?$allocator@USBannedUser@@@stlpmtx_std@@@priv@stlpmtx_std@@IEAA?AU?$_Deque_iterator@USBannedUser@@U?$_Nonconst_traits@USBannedUser@@@stlpmtx_std@@@23@U423@0AEBU__false_type@3@@Z 0000000039a10df0 f i CryMatchMaking.obj
 0001:000101e0       ?clear@?$_Impl_deque@USBannedUser@@V?$allocator@USBannedUser@@@stlpmtx_std@@@priv@stlpmtx_std@@QEAAXXZ 0000000039a111e0 f i CryMatchMaking.obj
 0001:000102a0       ??$Add@IIV?$CryLobbyID@USCryLobbySessionHandle@@$03@@VCCryMatchMaking@@@CWorkQueue@@QEAAXP8CCryMatchMaking@@EAAXIIV?$CryLobbyID@USCryLobbySessionHandle@@$03@@@ZPEAV1@II0@Z 0000000039a112a0 f i CryMatchMaking.obj
 0001:00010370       ??$Add@IIIVCCryMatchMaking@@@CWorkQueue@@QEAAXP8CCryMatchMaking@@EAAXIII@ZPEAV1@III@Z 0000000039a11370 f i CryMatchMaking.obj
 0001:00010370       ??$Add@IIIVCCryGameSpySBQR2MatchMaking@@@CWorkQueue@@QEAAXP8CCryGameSpySBQR2MatchMaking@@EAAXIII@ZPEAV1@III@Z 0000000039a11370 f i CryGameSpySBQR2MatchMaking.obj
 0001:00010450       ??$Add@W4ECryLobbySystemEvent@@IVCCryMatchMaking@@@CWorkQueue@@QEAAXP8CCryMatchMaking@@EAAXW4ECryLobbySystemEvent@@I@ZPEAV1@0I@Z 0000000039a11450 f i CryMatchMaking.obj
 0001:00010450       ??$Add@IW4ECryLobbySystemEvent@@VCCryMatchMaking@@@CWorkQueue@@QEAAXP8CCryMatchMaking@@EAAXIW4ECryLobbySystemEvent@@@ZPEAV1@I0@Z 0000000039a11450 f i CryMatchMaking.obj
 0001:00010520       ?_M_fill_insert_aux@?$_Impl_deque@USBannedUser@@V?$allocator@USBannedUser@@@stlpmtx_std@@@priv@stlpmtx_std@@IEAA?AU?$_Deque_iterator@USBannedUser@@U?$_Nonconst_traits@USBannedUser@@@stlpmtx_std@@@23@U423@_KAEBUSBannedUser@@AEBU__false_type@3@@Z 0000000039a11520 f i CryMatchMaking.obj
 0001:00011080       ?SendToServer@CCryMatchMaking@@UEAA?AW4ECryLobbyError@@PEAVCCryLobbyPacket@@I@Z 0000000039a12080 f   CryMatchMaking.obj
 0001:000111d0       ?SendToAllClients@CCryMatchMaking@@UEAA?AW4ECryLobbyError@@PEAVCCryLobbyPacket@@I@Z 0000000039a121d0 f   CryMatchMaking.obj
 0001:00011320       ?SendToClient@CCryMatchMaking@@UEAA?AW4ECryLobbyError@@PEAVCCryLobbyPacket@@IUSCryMatchMakingConnectionUID@@@Z 0000000039a12320 f   CryMatchMaking.obj
 0001:000114d0       ?InitialDispatchUserPackets@CCryMatchMaking@@IEAAXV?$CryLobbyID@USCryLobbySessionHandle@@$03@@V?$CryLobbyID@USCryMatchMakingConnectionID@@$0EA@@@@Z 0000000039a124d0 f   CryMatchMaking.obj
 0001:00011690       ?SessionDisconnectRemoteConnection@CCryMatchMaking@@IEAAXV?$CryLobbyID@USCryLobbySessionHandle@@$03@@V?$CryLobbyID@USCryMatchMakingConnectionID@@$0EA@@@W4eDisconnectSource@1@1W4EDisconnectionCause@@@Z 0000000039a12690 f   CryMatchMaking.obj
 0001:00011bc0       ?SessionTerminateHostHintingForGroup@CCryMatchMaking@@UEAA?AW4ECryLobbyError@@IPEAUSCryMatchMakingConnectionUID@@IPEAIP6AXIW42@PEAX@Z3@Z 0000000039a12bc0 f   CryMatchMaking.obj
 0001:00011de0       ?SessionSetLocalFlags@CCryMatchMaking@@UEAA?AW4ECryLobbyError@@IIPEAIP6AXIW42@IIPEAX@Z2@Z 0000000039a12de0 f   CryMatchMaking.obj
 0001:00011f50       ?SessionClearLocalFlags@CCryMatchMaking@@UEAA?AW4ECryLobbyError@@IIPEAIP6AXIW42@IIPEAX@Z2@Z 0000000039a12f50 f   CryMatchMaking.obj
 0001:000120c0       ?SessionGetLocalFlags@CCryMatchMaking@@UEAA?AW4ECryLobbyError@@IPEAIP6AXIW42@IIPEAX@Z2@Z 0000000039a130c0 f   CryMatchMaking.obj
 0001:00012210       ?TickSessionPendingGroupDisconnect@CCryMatchMaking@@IEAAXI@Z 0000000039a13210 f   CryMatchMaking.obj
 0001:00012210       ?TickSessionModifyLocalFlags@CCryMatchMaking@@IEAAXI@Z 0000000039a13210 f   CryMatchMaking.obj
 0001:00012270       ?SessionUserDataEvent@CCryMatchMaking@@IEAAXW4ECryLobbySystemEvent@@V?$CryLobbyID@USCryLobbySessionHandle@@$03@@PEAUSCryUserInfoResult@@@Z 0000000039a13270 f   CryMatchMaking.obj
 0001:000124e0       ?erase@?$_Impl_deque@USBannedUser@@V?$allocator@USBannedUser@@@stlpmtx_std@@@priv@stlpmtx_std@@QEAA?AU?$_Deque_iterator@USBannedUser@@U?$_Nonconst_traits@USBannedUser@@@stlpmtx_std@@@23@U423@0@Z 0000000039a134e0 f i CryMatchMaking.obj
 0001:000125e0       ?_M_fill_insert@?$_Impl_deque@USBannedUser@@V?$allocator@USBannedUser@@@stlpmtx_std@@@priv@stlpmtx_std@@IEAAXU?$_Deque_iterator@USBannedUser@@U?$_Nonconst_traits@USBannedUser@@@stlpmtx_std@@@23@_KAEBUSBannedUser@@@Z 0000000039a135e0 f i CryMatchMaking.obj
 0001:00012850       ??0CCryMatchMaking@@QEAA@PEAVCCryLobby@@PEAVCCryLobbyService@@W4ECryLobbyService@@@Z 0000000039a13850 f   CryMatchMaking.obj
 0001:00012a00       ?SessionSetupDedicatedServer@CCryMatchMaking@@UEAA?AW4ECryLobbyError@@IPEAVCCryLobbyPacket@@PEAIP6AXIW42@IGPEAX@Z3@Z 0000000039a13a00 f i CryMatchMaking.obj
 0001:00012a00       ?CheckOnlineRetailStatus@CCryLobbyUI@@UEAA?AW4ECryLobbyError@@IPEAIP6AXIW42@PEAUSCryLobbyUIOnlineRetailCounts@@PEAX@Z3@Z 0000000039a13a00 f i CryLobbyUI.obj
 0001:00012a00       ?GetSessionIDFromSessionURL@CCryMatchMaking@@UEAA?AW4ECryLobbyError@@QEBDQEAV?$_smart_ptr@USCrySessionID@@@@@Z 0000000039a13a00 f i CryMatchMaking.obj
 0001:00012a00       ?SessionSendRequestInfoResponse@CCryMatchMaking@@UEAA?AW4ECryLobbyError@@PEAVCCryLobbyPacket@@PEAX@Z 0000000039a13a00 f i CryMatchMaking.obj
 0001:00012a00       ?ShowMessageList@CCryLobbyUI@@UEAA?AW4ECryLobbyError@@IPEAIP6AXIW42@PEAX@Z2@Z 0000000039a13a00 f i CryLobbyUI.obj
 0001:00012a00       ?ShowCommunitySessions@CCryLobbyUI@@UEAA?AW4ECryLobbyError@@IPEAIP6AXIW42@PEAX@Z2@Z 0000000039a13a00 f i CryLobbyUI.obj
 0001:00012a00       ?GetSessionIDFromIP@CCryMatchMaking@@UEAA?AW4ECryLobbyError@@QEBDQEAV?$_smart_ptr@USCrySessionID@@@@@Z 0000000039a13a00 f i CryMatchMaking.obj
 0001:00012a00       ?CheckProfanity@CCryLobbyService@@UEAA?AW4ECryLobbyError@@QEBDPEAIP6AXIW42@PEBD_NPEAX@Z5@Z 0000000039a13a00 f i CryLobby.obj
 0001:00012a00       ?ShowParty@CCryLobbyUI@@UEAA?AW4ECryLobbyError@@IPEAIP6AXIW42@PEAX@Z2@Z 0000000039a13a00 f i CryLobbyUI.obj
 0001:00012a00       ?ShowOnlineRetailBrowser@CCryLobbyUI@@UEAA?AW4ECryLobbyError@@IPEAIP6AXIW42@PEAX@Z2@Z 0000000039a13a00 f i CryLobbyUI.obj
 0001:00012a00       ?SessionReleaseDedicatedServer@CCryMatchMaking@@UEAA?AW4ECryLobbyError@@IPEAIP6AXIW42@PEAX@Z2@Z 0000000039a13a00 f i CryMatchMaking.obj
 0001:00012a10       ?GetNameFromGameSessionHandle@CCryMatchMaking@@UEAAPEBDI@Z 0000000039a13a10 f i CryMatchMaking.obj
 0001:00012a20       ??_ECCryMatchMaking@@WBA@EAAPEAXI@Z 0000000039a13a20 f i CryMatchMaking.obj
 0001:00012a30       ?GetSessionAddressFromSessionID@CCryMatchMaking@@UEAA?AW4ECryLobbyError@@V?$_smart_ptr@USCrySessionID@@@@AEAIAEAG@Z 0000000039a13a30 f i CryMatchMaking.obj
 0001:00012a90       ??_ECCryMatchMaking@@UEAAPEAXI@Z 0000000039a13a90 f i CryMatchMaking.obj
 0001:00012a90       ??_GCCryMatchMaking@@UEAAPEAXI@Z 0000000039a13a90 f i CryMatchMaking.obj
 0001:00012af0       ?TickBaseTask@CCryMatchMaking@@IEAAXI@Z 0000000039a13af0 f   CryMatchMaking.obj
 0001:00012b30       ?SessionDisconnectRemoteConnectionFromNub@CCryMatchMaking@@UEAAXIW4EDisconnectionCause@@@Z 0000000039a13b30 f   CryMatchMaking.obj
 0001:00012d20       ?SessionDisconnectRemoteConnectionViaNub@CCryMatchMaking@@IEAAXV?$CryLobbyID@USCryLobbySessionHandle@@$03@@V?$CryLobbyID@USCryMatchMakingConnectionID@@$0EA@@@W4eDisconnectSource@1@1W4EDisconnectionCause@@PEBD@Z 0000000039a13d20 f   CryMatchMaking.obj
 0001:00012e40       ?ProcessSessionDeleteRemoteConnection@CCryMatchMaking@@IEAAXAEBV?$CConfigurableVariant@V?$CNode@USNullAddr@@V?$CNode@GV?$CNode@USIPv4Addr@@V?$CNode@ULobbyIdAddr@@VCEnd@NTypelist@@@NTypelist@@@NTypelist@@@NTypelist@@@NTypelist@@$07VCDefaultVariantConversion@NConfigurableVariantHelpers@@VCDefaultVariantConstruction@4@@@PEAVCCrySharedLobbyPacket@@@Z 0000000039a13e40 f   CryMatchMaking.obj
 0001:00013240       ?OnPacket@CCryMatchMaking@@QEAAXAEBV?$CConfigurableVariant@V?$CNode@USNullAddr@@V?$CNode@GV?$CNode@USIPv4Addr@@V?$CNode@ULobbyIdAddr@@VCEnd@NTypelist@@@NTypelist@@@NTypelist@@@NTypelist@@@NTypelist@@$07VCDefaultVariantConversion@NConfigurableVariantHelpers@@VCDefaultVariantConstruction@4@@@PEAVCCryLobbyPacket@@@Z 0000000039a14240 f   CryMatchMaking.obj
 0001:00013520       ?KickCmd@CCryMatchMaking@@UEAAXV?$CryLobbyID@USCryLobbyConnectionID@@$0EA@@@_KPEBDW4EDisconnectionCause@@@Z 0000000039a14520 f   CryMatchMaking.obj
 0001:00013750       ?ResetConnection@CCryMatchMaking@@QEAAXV?$CryLobbyID@USCryLobbyConnectionID@@$0EA@@@@Z 0000000039a14750 f   CryMatchMaking.obj
 0001:00013920       ?resize@?$_Impl_deque@USBannedUser@@V?$allocator@USBannedUser@@@stlpmtx_std@@@priv@stlpmtx_std@@QEAAX_KAEBUSBannedUser@@@Z 0000000039a14920 f i CryMatchMaking.obj
 0001:000139e0       ?ExpireBans@CCryMatchMaking@@IEAA_NAEAV?$deque@USBannedUser@@V?$allocator@USBannedUser@@@stlpmtx_std@@@stlpmtx_std@@AEBVCTimeValue@@@Z 0000000039a149e0 f   CryMatchMaking.obj
 0001:00013cb0       ?Tick@CCryMatchMaking@@IEAAXVCTimeValue@@@Z 0000000039a14cb0 f   CryMatchMaking.obj
 0001:00013f80       ??_GICrySignIn@@UEAAPEAXI@Z 0000000039a14f80 f i CrySignIn.obj
 0001:00013f80       ??_EICrySignIn@@UEAAPEAXI@Z 0000000039a14f80 f i CrySignIn.obj
 0001:00013fb0       ??_9CCrySignIn@@$BDI@AA    0000000039a14fb0 f i CrySignIn.obj
 0001:00013fb0       ??_9CCryDLCStore@@$BDI@AA  0000000039a14fb0 f i CryDLCStore.obj
 0001:00013fc0       ??0CCrySignIn@@IEAA@PEAVCCryLobby@@PEAVCCryLobbyService@@@Z 0000000039a14fc0 f   CrySignIn.obj
 0001:00013ff0       ??_ECCrySignIn@@WBA@EAAPEAXI@Z 0000000039a14ff0 f i CrySignIn.obj
 0001:00014000       ??1CCrySignIn@@UEAA@XZ     0000000039a15000 f   CrySignIn.obj
 0001:00014020       ?EndTask@CCrySignIn@@MEAAXV?$CryLobbyID@USCrySignInTaskID@CCrySignIn@@$03@@@Z 0000000039a15020 f   CrySignIn.obj
 0001:00014070       ??_ECCrySignIn@@UEAAPEAXI@Z 0000000039a15070 f i CrySignIn.obj
 0001:00014070       ??_GCCrySignIn@@UEAAPEAXI@Z 0000000039a15070 f i CrySignIn.obj
 0001:000140b0       ?CancelTask@CCrySignIn@@UEAAXI@Z 0000000039a150b0 f   CrySignIn.obj
 0001:00014180       ?Initialise@CCrySignIn@@UEAA?AW4ECryLobbyError@@XZ 0000000039a15180 f   CrySignIn.obj
 0001:000141d0       ?Terminate@CCrySignIn@@UEAA?AW4ECryLobbyError@@XZ 0000000039a151d0 f   CrySignIn.obj
 0001:00014220       ?StartTaskRunning@CCrySignIn@@MEAAXV?$CryLobbyID@USCrySignInTaskID@CCrySignIn@@$03@@@Z 0000000039a15220 f   CrySignIn.obj
 0001:00014260       ?StartTask@CCrySignIn@@IEAA?AW4ECryLobbyError@@IPEAV?$CryLobbyID@USCrySignInTaskID@CCrySignIn@@$03@@PEAIPEAX2@Z 0000000039a15260 f   CrySignIn.obj
 0001:00014330       ?FreeTask@CCrySignIn@@MEAAXV?$CryLobbyID@USCrySignInTaskID@CCrySignIn@@$03@@@Z 0000000039a15330 f   CrySignIn.obj
 0001:000143d0       ?CreateTaskParamMem@CCrySignIn@@IEAA?AW4ECryLobbyError@@V?$CryLobbyID@USCrySignInTaskID@CCrySignIn@@$03@@IPEBX_K@Z 0000000039a153d0 f   CrySignIn.obj
 0001:00014480       ?UpdateTaskError@CCrySignIn@@IEAAXV?$CryLobbyID@USCrySignInTaskID@CCrySignIn@@$03@@W4ECryLobbyError@@@Z 0000000039a15480 f   CrySignIn.obj
 0001:000144d0       ?CreateTask@CCrySignIn@@MEAAXV?$CryLobbyID@USCrySignInTaskID@CCrySignIn@@$03@@IIPEAX1@Z 0000000039a154d0 f   CrySignIn.obj
 0001:00014570       ?ClearTask@CCrySignIn@@EEAAXV?$CryLobbyID@USCrySignInTaskID@CCrySignIn@@$03@@@Z 0000000039a15570 f   CrySignIn.obj
 0001:000145f0       ?Execute@?$CClassJobNoRef@IVCCryGameSpySBQR2FriendsManagement@@@CWorkQueue@@UEAAXXZ 0000000039a155f0 f i CryGameSpySBQR2FriendsManagement.obj
 0001:000145f0       ?Execute@?$CClassJobNoRef@V?$CryLobbyID@USCrySignInTaskID@CCrySignIn@@$03@@VCCrySignIn@@@CWorkQueue@@UEAAXXZ 0000000039a155f0 f i CrySignIn.obj
 0001:000145f0       ?Execute@?$CClassJobNoRef@V?$CryLobbyID@USCrySignInTaskID@CCrySignIn@@$03@@VCCryGameSpySBQR2SignIn@@@CWorkQueue@@UEAAXXZ 0000000039a155f0 f i CryGameSpySBQR2SignIn.obj
 0001:000145f0       ?Execute@?$CClassJobNoRef@IVCCryGameSpySBQR2Stats@@@CWorkQueue@@UEAAXXZ 0000000039a155f0 f i CryGameSpySBQR2Stats.obj
 0001:000145f0       ?Execute@?$CClassJobNoRef@IVCCryGameSpySBQR2LobbyUI@@@CWorkQueue@@UEAAXXZ 0000000039a155f0 f i CryGameSpySBQR2LobbyUI.obj
 0001:00014620       ??$Add@V?$CryLobbyID@USCrySignInTaskID@CCrySignIn@@$03@@VCCrySignIn@@@CWorkQueue@@QEAAXP8CCrySignIn@@EAAXV?$CryLobbyID@USCrySignInTaskID@CCrySignIn@@$03@@@ZPEAV1@0@Z 0000000039a15620 f i CrySignIn.obj
 0001:00014620       ??$Add@V?$CryLobbyID@USCrySignInTaskID@CCrySignIn@@$03@@VCCryGameSpySBQR2SignIn@@@CWorkQueue@@QEAAXP8CCryGameSpySBQR2SignIn@@EAAXV?$CryLobbyID@USCrySignInTaskID@CCrySignIn@@$03@@@ZPEAV1@0@Z 0000000039a15620 f i CryGameSpySBQR2SignIn.obj
 0001:000146e0       ?StopTaskRunning@CCrySignIn@@MEAAXV?$CryLobbyID@USCrySignInTaskID@CCrySignIn@@$03@@@Z 0000000039a156e0 f   CrySignIn.obj
 0001:00014760       ??_EICryStats@@UEAAPEAXI@Z 0000000039a15760 f i CryStats.obj
 0001:00014760       ??_GICryStats@@UEAAPEAXI@Z 0000000039a15760 f i CryStats.obj
 0001:00014790       ?Initialise@CCryStats@@QEAA?AW4ECryLobbyError@@XZ 0000000039a15790 f   CryStats.obj
 0001:000147c0       ?Terminate@CCryStats@@QEAA?AW4ECryLobbyError@@XZ 0000000039a157c0 f   CryStats.obj
 0001:00014820       ?StartTask@CCryStats@@IEAA?AW4ECryLobbyError@@I_NPEAI1V?$CryLobbyID@USCryLobbySessionHandle@@$03@@PEAX3@Z 0000000039a15820 f   CryStats.obj
 0001:00014910       ?FreeTask@CCryStats@@MEAAXI@Z 0000000039a15910 f   CryStats.obj
 0001:00014990       ?CreateTaskParamMem@CCryStats@@IEAA?AW4ECryLobbyError@@IIPEBX_K@Z 0000000039a15990 f   CryStats.obj
 0001:00014a20       ??0CCryStats@@QEAA@PEAVCCryLobby@@PEAVCCryLobbyService@@@Z 0000000039a15a20 f   CryStats.obj
 0001:00014a70       ?StatsVerifyString@CCryStats@@UEAA?AW4ECryLobbyError@@IPEAEIPEAIP6AXIW42@PEAX@Z3@Z 0000000039a15a70 f i CryStats.obj
 0001:00014a70       ?StatsWriteUserData@CCryStats@@UEAA?AW4ECryLobbyError@@PEAUCryUserID@@PEAPEAUSCryLobbyUserData@@PEAII2P6AXIW42@PEAX@Z4@Z 0000000039a15a70 f i CryStats.obj
 0001:00014a80       ??_ECCryStats@@WBA@EAAPEAXI@Z 0000000039a15a80 f i CryStats.obj
 0001:00014a90       ?CancelTask@CCryStats@@UEAAXI@Z 0000000039a15a90 f   CryStats.obj
 0001:00014b20       ?EncryptUserData@CCryStats@@IEAA?AW4ECryLobbyError@@IPEBEPEAE@Z 0000000039a15b20 f   CryStats.obj
 0001:00014c40       ?DecryptUserData@CCryStats@@IEAA?AW4ECryLobbyError@@IPEBEPEAE@Z 0000000039a15c40 f   CryStats.obj
 0001:00014d40       ??_GCCryStats@@UEAAPEAXI@Z 0000000039a15d40 f i CryStats.obj
 0001:00014d40       ??_ECCryStats@@UEAAPEAXI@Z 0000000039a15d40 f i CryStats.obj
 0001:00014d80       ?IsService@CCryTCPService@@UEAA_NPEBDG@Z 0000000039a15d80 f   CryTCPService.obj
 0001:00014dc0       ?HasResolved@CCryTCPService@@UEAA_NXZ 0000000039a15dc0 f   CryTCPService.obj
 0001:00014de0       ?IsResolving@CCryTCPService@@UEAA_NXZ 0000000039a15de0 f   CryTCPService.obj
 0001:00014e00       ?AddRef@CCryTCPService@@UEAAHXZ 0000000039a15e00 f   CryTCPService.obj
 0001:00014e10       ?GetConnectionStatus@CCryTCPService@@UEAA?AW4ECryTCPServiceConnectionStatus@@XZ 0000000039a15e10 f   CryTCPService.obj
 0001:00014e20       ?GetDataQueueLength@CCryTCPService@@UEAAIXZ 0000000039a15e20 f   CryTCPService.obj
 0001:00014e30       ?GetDataQueueSize@CCryTCPService@@UEAAIXZ 0000000039a15e30 f   CryTCPService.obj
 0001:00014e40       ??_EICryLobbyUI@@UEAAPEAXI@Z 0000000039a15e40 f i CryLobbyUI.obj
 0001:00014e40       ??_GICryTCPService@@UEAAPEAXI@Z 0000000039a15e40 f i CryTCPService.obj
 0001:00014e40       ??_GICryLobbyUI@@UEAAPEAXI@Z 0000000039a15e40 f i CryLobbyUI.obj
 0001:00014e40       ??_EICryTCPService@@UEAAPEAXI@Z 0000000039a15e40 f i CryTCPService.obj
 0001:00014e70       ?Connect@CCryTCPService@@MEAA?AW4ESocketError@@AEAH@Z 0000000039a15e70 f   CryTCPService.obj
 0001:00014ee0       ?CloseConnection@CCryTCPService@@MEAA?AW4ESocketError@@AEAH@Z 0000000039a15ee0 f   CryTCPService.obj
 0001:00014f00       ?Release@CCryTCPService@@UEAAHXZ 0000000039a15f00 f   CryTCPService.obj
 0001:00014f60       ?Send@CCryTCPService@@MEAA?AW4ESocketError@@V?$_smart_ptr@USTCPServiceData@@@@@Z 0000000039a15f60 f   CryTCPService.obj
 0001:00015010       ?Recv@CCryTCPService@@MEAA?AW4ESocketError@@V?$_smart_ptr@USTCPServiceData@@@@AEA_N@Z 0000000039a16010 f   CryTCPService.obj
 0001:00015140       ?ProcessTransaction@CCryTCPService@@AEAA?AV?$_smart_ptr@USTCPServiceData@@@@V2@@Z 0000000039a16140 f   CryTCPService.obj
 0001:000152d0       ?_M_initialize_map@?$_Deque_base@V?$_smart_ptr@USTCPServiceData@@@@V?$allocator@V?$_smart_ptr@USTCPServiceData@@@@@stlpmtx_std@@@priv@stlpmtx_std@@IEAAX_K@Z 0000000039a162d0 f i CryTCPService.obj
 0001:000153f0       ?_M_reallocate_map@?$_Impl_deque@USBannedUser@@V?$allocator@USBannedUser@@@stlpmtx_std@@@priv@stlpmtx_std@@IEAAX_K_N@Z 0000000039a163f0 f i CryMatchMaking.obj
 0001:000153f0       ?_M_reallocate_map@?$_Impl_deque@V?$_smart_ptr@USTCPServiceData@@@@V?$allocator@V?$_smart_ptr@USTCPServiceData@@@@@stlpmtx_std@@@priv@stlpmtx_std@@IEAAX_K_N@Z 0000000039a163f0 f i CryTCPService.obj
 0001:000153f0       ?_M_reallocate_map@?$_Impl_deque@HV?$allocator@H@stlpmtx_std@@@priv@stlpmtx_std@@IEAAX_K_N@Z 0000000039a163f0 f i CryGameSpySBQR2Friends.obj
 0001:00015590       ?Initialise@CCryTCPService@@UEAA?AW4ECryTCPServiceResult@@PEBDG@Z 0000000039a16590 f   CryTCPService.obj
 0001:00015770       ??$__destroy_range@U?$_Deque_iterator@V?$_smart_ptr@USTCPServiceData@@@@U?$_Nonconst_traits@V?$_smart_ptr@USTCPServiceData@@@@@stlpmtx_std@@@priv@stlpmtx_std@@V?$_smart_ptr@USTCPServiceData@@@@@stlpmtx_std@@YAXU?$_Deque_iterator@V?$_smart_ptr@USTCPServiceData@@@@U?$_Nonconst_traits@V?$_smart_ptr@USTCPServiceData@@@@@stlpmtx_std@@@priv@0@0PEAV?$_smart_ptr@USTCPServiceData@@@@@Z 0000000039a16770 f i CryTCPService.obj
 0001:00015840       ?pop_front@?$_Impl_deque@V?$_smart_ptr@USTCPServiceData@@@@V?$allocator@V?$_smart_ptr@USTCPServiceData@@@@@stlpmtx_std@@@priv@stlpmtx_std@@QEAAXXZ 0000000039a16840 f i CryTCPService.obj
 0001:000158f0       ?_M_push_back_aux_v@?$_Impl_deque@V?$_smart_ptr@USTCPServiceData@@@@V?$allocator@V?$_smart_ptr@USTCPServiceData@@@@@stlpmtx_std@@@priv@stlpmtx_std@@IEAAXAEBV?$_smart_ptr@USTCPServiceData@@@@@Z 0000000039a168f0 f i CryTCPService.obj
 0001:00015990       ??1?$_Impl_deque@V?$_smart_ptr@USTCPServiceData@@@@V?$allocator@V?$_smart_ptr@USTCPServiceData@@@@@stlpmtx_std@@@priv@stlpmtx_std@@QEAA@XZ 0000000039a16990 f i CryTCPService.obj
 0001:00015a00       ?GetAddress@CCryTCPService@@MEAA?AW4ENameRequestResult@@AEAUsockaddr_in@@@Z 0000000039a16a00 f   CryTCPService.obj
 0001:00015d30       ?DiscardQueueElement@CCryTCPService@@AEAAXXZ 0000000039a16d30 f   CryTCPService.obj
 0001:00015e20       ??0CCryTCPService@@QEAA@PEAVCCryTCPServiceFactory@@@Z 0000000039a16e20 f   CryTCPService.obj
 0001:00015ed0       ?Terminate@CCryTCPService@@UEAA?AW4ECryTCPServiceResult@@_N@Z 0000000039a16ed0 f   CryTCPService.obj
 0001:00015fe0       ?Tick@CCryTCPService@@UEAAXVCTimeValue@@@Z 0000000039a16fe0 f   CryTCPService.obj
 0001:00016450       ?UploadData@CCryTCPService@@UEAA_NV?$_smart_ptr@USTCPServiceData@@@@@Z 0000000039a17450 f   CryTCPService.obj
 0001:00016580       ??1CCryTCPService@@UEAA@XZ 0000000039a17580 f   CryTCPService.obj
 0001:00016650       ??_ECCryTCPService@@UEAAPEAXI@Z 0000000039a17650 f i CryTCPService.obj
 0001:00016650       ??_GCCryTCPService@@UEAAPEAXI@Z 0000000039a17650 f i CryTCPService.obj
 0001:00016680       ?Initialise@CCryTCPServiceFactory@@UEAA?AW4ECryLobbyError@@I@Z 0000000039a17680 f   CryTCPServiceFactory.obj
 0001:00016700       ?AddRef@CCryTCPServiceFactory@@UEAAHXZ 0000000039a17700 f   CryTCPServiceFactory.obj
 0001:00016710       ?NumFreeSockets@CCryTCPServiceFactory@@QEAAIXZ 0000000039a17710 f   CryTCPServiceFactory.obj
 0001:00016720       ?Connect@CCryTCPServiceFactory@@UEAA?AW4ESocketError@@AEAUsockaddr_in@@AEAH@Z 0000000039a17720 f   CryTCPServiceFactory.obj
 0001:00016870       ?Send@CCryTCPServiceFactory@@UEAA?AW4ESocketError@@HPEBD_KAEA_K@Z 0000000039a17870 f   CryTCPServiceFactory.obj
 0001:00016990       ?Recv@CCryTCPServiceFactory@@UEAA?AW4ESocketError@@HPEADAEA_KAEA_N@Z 0000000039a17990 f   CryTCPServiceFactory.obj
 0001:00016aa0       ?CloseConnection@CCryTCPServiceFactory@@UEAA?AW4ESocketError@@AEAH@Z 0000000039a17aa0 f   CryTCPServiceFactory.obj
 0001:00016af0       ?Release@CCryTCPServiceFactory@@UEAAHXZ 0000000039a17af0 f   CryTCPServiceFactory.obj
 0001:00016b50       ?CreateTCPService@CCryTCPServiceFactory@@MEAA?AV?$_smart_ptr@UICryTCPService@@@@PEBDG@Z 0000000039a17b50 f   CryTCPServiceFactory.obj
 0001:00016bf0       ?Tick@CCryTCPServiceFactory@@UEAAXVCTimeValue@@@Z 0000000039a17bf0 f   CryTCPServiceFactory.obj
 0001:00016cc0       ??$__uninitialized_fill_n@PEAV?$_smart_ptr@UICryTCPService@@@@_KV1@@priv@stlpmtx_std@@YAPEAV?$_smart_ptr@UICryTCPService@@@@PEAV2@_KAEBV2@@Z 0000000039a17cc0 f i CryTCPServiceFactory.obj
 0001:00016d30       ?_M_erase@?$_Impl_vector@V?$_smart_ptr@UICryTCPService@@@@V?$STLGlobalAllocator@V?$_smart_ptr@UICryTCPService@@@@@stl@@@priv@stlpmtx_std@@AEAAPEAV?$_smart_ptr@UICryTCPService@@@@PEAV4@0AEBU__false_type@3@@Z 0000000039a17d30 f i CryTCPServiceFactory.obj
 0001:00016e10       ??1?$_Impl_vector@V?$_smart_ptr@UICryTCPService@@@@V?$STLGlobalAllocator@V?$_smart_ptr@UICryTCPService@@@@@stl@@@priv@stlpmtx_std@@QEAA@XZ 0000000039a17e10 f i CryTCPServiceFactory.obj
 0001:00016e80       ?_M_insert_overflow_aux@?$_Impl_vector@V?$_smart_ptr@UICryTCPService@@@@V?$STLGlobalAllocator@V?$_smart_ptr@UICryTCPService@@@@@stl@@@priv@stlpmtx_std@@AEAAXPEAV?$_smart_ptr@UICryTCPService@@@@AEBV4@AEBU__false_type@3@_K_N@Z 0000000039a17e80 f i CryTCPServiceFactory.obj
 0001:00017040       ??0CCryTCPServiceFactory@@QEAA@XZ 0000000039a18040 f   CryTCPServiceFactory.obj
 0001:000170b0       ?Terminate@CCryTCPServiceFactory@@UEAA?AW4ECryLobbyError@@_N@Z 0000000039a180b0 f   CryTCPServiceFactory.obj
 0001:00017140       ?GetTCPService@CCryTCPServiceFactory@@UEAA?AV?$_smart_ptr@UICryTCPService@@@@PEBDG@Z 0000000039a18140 f   CryTCPServiceFactory.obj
 0001:00017340       ??_GCCryTCPServiceFactory@@UEAAPEAXI@Z 0000000039a18340 f i CryTCPServiceFactory.obj
 0001:00017340       ??_ECCryTCPServiceFactory@@UEAAPEAXI@Z 0000000039a18340 f i CryTCPServiceFactory.obj
 0001:000173b0       ??_GICryVoice@@UEAAPEAXI@Z 0000000039a183b0 f i CryVoice.obj
 0001:000173b0       ??_EICryVoice@@UEAAPEAXI@Z 0000000039a183b0 f i CryVoice.obj
 0001:000173e0       ??0CCryVoice@@QEAA@PEAVCCryLobby@@PEAVCCryLobbyService@@@Z 0000000039a183e0 f   CryVoice.obj
 0001:00017480       ?GetVoicePlaybackVolume@CCryVoice@@UEAAMI@Z 0000000039a18480 f i CryVoice.obj
 0001:00017490       ??_ECCryVoice@@WBA@EAAPEAXI@Z 0000000039a18490 f i CryVoice.obj
 0001:000174a0       ?Tick@CCryVoice@@IEAAXVCTimeValue@@@Z 0000000039a184a0 f   CryVoice.obj
 0001:00017560       ??_GCCryVoice@@UEAAPEAXI@Z 0000000039a18560 f i CryVoice.obj
 0001:00017560       ??_ECCryVoice@@UEAAPEAXI@Z 0000000039a18560 f i CryVoice.obj
 0001:000175a0       ?UnRegisterRemoteUser@CCryVoice@@IEAAXI@Z 0000000039a185a0 f   CryVoice.obj
 0001:00017630       ?GetRemoteUser@CCryVoice@@IEAAIUCryUserID@@@Z 0000000039a18630 f   CryVoice.obj
 0001:00017730       ?Mute@CCryVoice@@UEAAXIUCryUserID@@_N@Z 0000000039a18730 f   CryVoice.obj
 0001:000177f0       ?IsMuted@CCryVoice@@UEAA_NIUCryUserID@@@Z 0000000039a187f0 f   CryVoice.obj
 0001:00017910       ?MuteExternally@CCryVoice@@UEAAXIUCryUserID@@_N@Z 0000000039a18910 f   CryVoice.obj
 0001:00017960       ?IsMutedExternally@CCryVoice@@UEAA_NIUCryUserID@@@Z 0000000039a18960 f   CryVoice.obj
 0001:00017a80       ?IsSpeaking@CCryVoice@@UEAA_NIUCryUserID@@@Z 0000000039a18a80 f   CryVoice.obj
 0001:00017c70       ?IsMicrophoneConnected@CCryVoice@@UEAA_NUCryUserID@@@Z 0000000039a18c70 f   CryVoice.obj
 0001:00017d70       ?Initialise@CCryVoice@@IEAA?AW4ECryLobbyError@@XZ 0000000039a18d70 f   CryVoice.obj
 0001:00017e30       ?RegisterRemoteUser@CCryVoice@@IEAAIV?$CryLobbyID@USCryLobbyConnectionID@@$0EA@@@UCryUserID@@@Z 0000000039a18e30 f   CryVoice.obj
 0001:00017fa0       ??0CGameSpySBQR2AvailabilityCheck@@QEAA@PEAVCCryGameSpySBQR2LobbyService@@@Z 0000000039a18fa0 f   GameSpySBQR2AvailabilityCheck.obj
 0001:00017fd0       ?NeedThink@CGameSpySBQR2AvailabilityCheck@@MEBA_NXZ 0000000039a18fd0 f   GameSpySBQR2AvailabilityCheck.obj
 0001:00017ff0       SBServerGetPing            0000000039a18ff0 f   GameSpy_2.11.00_VC10:sb_server.obj
 0001:00017ff0       ?GetState@CGameSpySBQR2AvailabilityCheck@@QEAA?AW4EState@1@XZ 0000000039a18ff0 f   GameSpySBQR2AvailabilityCheck.obj
 0001:00018000       ??1?$CGameSpySDKRef@VCGameSpySBQR2GPConnection@@@@QEAA@XZ 0000000039a19000 f i GameSpySBQR2AvailabilityCheck.obj
 0001:00018000       ??1?$CGameSpySDKRef@VCGameSpySBQR2Sake@@@@QEAA@XZ 0000000039a19000 f i GameSpySBQR2Sake.obj
 0001:00018000       ??1?$CGameSpySDKRef@VCGameSpySBQR2NATNegotiation@@@@QEAA@XZ 0000000039a19000 f i GameSpySBQR2NatNegotiation.obj
 0001:00018000       ??1?$CGameSpySDKRef@VCGameSpySBQR2Core@@@@QEAA@XZ 0000000039a19000 f i GameSpySBQR2Core.obj
 0001:00018020       ??4?$CGameSpySDKRef@VCGameSpySBQR2NATNegotiation@@@@QEAAAEBV0@PEAVCGameSpySBQR2NATNegotiation@@@Z 0000000039a19020 f i GameSpySBQR2NatNegotiation.obj
 0001:00018020       ??4?$CGameSpySDKRef@VCGameSpySBQR2GPConnection@@@@QEAAAEBV0@PEAVCGameSpySBQR2GPConnection@@@Z 0000000039a19020 f i GameSpySBQR2AvailabilityCheck.obj
 0001:00018020       ??4?$CGameSpySDKRef@VCGameSpySBQR2Sake@@@@QEAAAEBV0@PEAVCGameSpySBQR2Sake@@@Z 0000000039a19020 f i GameSpySBQR2Sake.obj
 0001:00018020       ??4?$CGameSpySDKRef@VCGameSpySBQR2Core@@@@QEAAAEBV0@PEAVCGameSpySBQR2Core@@@Z 0000000039a19020 f i GameSpySBQR2Core.obj
 0001:00018060       ??_ECGameSpySBQR2AvailabilityCheck@@UEAAPEAXI@Z 0000000039a19060 f i GameSpySBQR2AvailabilityCheck.obj
 0001:00018060       ??_GCGameSpySBQR2AvailabilityCheck@@UEAAPEAXI@Z 0000000039a19060 f i GameSpySBQR2AvailabilityCheck.obj
 0001:000180a0       ?PerformThink@CGameSpySBQR2AvailabilityCheck@@MEAAXXZ 0000000039a190a0 f   GameSpySBQR2AvailabilityCheck.obj
 0001:000181f0       ??B?$CGameSpySDKRef@VCGameSpySBQR2NATNegotiation@@@@QEAAP80@EAAXXZXZ 0000000039a191f0 f i GameSpySBQR2NatNegotiation.obj
 0001:000181f0       ??B?$CGameSpySDKRef@VCGameSpySBQR2GPConnection@@@@QEAAP80@EAAXXZXZ 0000000039a191f0 f i GameSpySBQR2AvailabilityCheck.obj
 0001:00018210       ?NeedThink@CGameSpySBQR2Core@@MEBA_NXZ 0000000039a19210 f   GameSpySBQR2Core.obj
 0001:00018230       ??0?$CGameSpySDKRef@VCGameSpySBQR2Core@@@@QEAA@XZ 0000000039a19230 f i GameSpySBQR2Core.obj
 0001:00018230       ??0?$CGameSpySDKRef@VCGameSpySBQR2GPConnection@@@@QEAA@XZ 0000000039a19230 f i GameSpySBQR2AvailabilityCheck.obj
 0001:00018230       ??0?$CGameSpySDKRef@VCGameSpySBQR2NATNegotiation@@@@QEAA@XZ 0000000039a19230 f i GameSpySBQR2NatNegotiation.obj
 0001:00018230       ??0?$CGameSpySDKRef@VCGameSpySBQR2Sake@@@@QEAA@XZ 0000000039a19230 f i GameSpySBQR2Sake.obj
 0001:00018240       ?allocate@?$_STLP_alloc_proxy@PEAV?$_smart_ptr@USTask@CGameSpySBQR2Core@@@@V1@V?$allocator@V?$_smart_ptr@USTask@CGameSpySBQR2Core@@@@@stlpmtx_std@@@priv@stlpmtx_std@@QEAAPEAV?$_smart_ptr@USTask@CGameSpySBQR2Core@@@@_KAEA_K@Z 0000000039a19240 f i GameSpySBQR2Core.obj
 0001:000182b0       ??0STask@CGameSpySBQR2Core@@QEAA@PEAUIGameSpyLink@@@Z 0000000039a192b0 f   GameSpySBQR2Core.obj
 0001:00018300       ??1STask@CGameSpySBQR2Core@@UEAA@XZ 0000000039a19300 f   GameSpySBQR2Core.obj
 0001:00018380       ?CoreTaskFinished@STask@CGameSpySBQR2Core@@QEAAXXZ 0000000039a19380 f   GameSpySBQR2Core.obj
 0001:000184b0       ??_GSTask@CGameSpySBQR2Core@@UEAAPEAXI@Z 0000000039a194b0 f i GameSpySBQR2Core.obj
 0001:000184b0       ??_ESTask@CGameSpySBQR2Core@@UEAAPEAXI@Z 0000000039a194b0 f i GameSpySBQR2Core.obj
 0001:000184e0       ?_M_clear@?$_Impl_vector@V?$_smart_ptr@USTask@CGameSpySBQR2Core@@@@V?$allocator@V?$_smart_ptr@USTask@CGameSpySBQR2Core@@@@@stlpmtx_std@@@priv@stlpmtx_std@@AEAAXXZ 0000000039a194e0 f i GameSpySBQR2Core.obj
 0001:00018520       ??$_M_allocate_and_copy@PEAV?$_smart_ptr@USTask@CGameSpySBQR2Core@@@@@?$_Impl_vector@V?$_smart_ptr@USTask@CGameSpySBQR2Core@@@@V?$allocator@V?$_smart_ptr@USTask@CGameSpySBQR2Core@@@@@stlpmtx_std@@@priv@stlpmtx_std@@AEAAPEAV?$_smart_ptr@USTask@CGameSpySBQR2Core@@@@AEA_KPEAV3@1@Z 0000000039a19520 f i GameSpySBQR2Core.obj
 0001:000185f0       ??0CGameSpySBQR2Core@@QEAA@PEAVCCryGameSpySBQR2LobbyService@@@Z 0000000039a195f0 f   GameSpySBQR2Core.obj
 0001:000186e0       ?AddTask@CGameSpySBQR2Core@@QEAAXPEAUSTask@1@PEAVCGameSpySDK@@@Z 0000000039a196e0 f   GameSpySBQR2Core.obj
 0001:00018820       ?TearDown@CGameSpySBQR2Core@@AEAAXXZ 0000000039a19820 f   GameSpySBQR2Core.obj
 0001:000188b0       ??1CGameSpySBQR2Core@@UEAA@XZ 0000000039a198b0 f   GameSpySBQR2Core.obj
 0001:00018930       ?PerformThink@CGameSpySBQR2Core@@MEAAXXZ 0000000039a19930 f   GameSpySBQR2Core.obj
 0001:00018970       ??_GCGameSpySBQR2Core@@UEAAPEAXI@Z 0000000039a19970 f i GameSpySBQR2Core.obj
 0001:00018970       ??_ECGameSpySBQR2Core@@UEAAPEAXI@Z 0000000039a19970 f i GameSpySBQR2Core.obj
 0001:000189a0       ?NeedThink@CGameSpySBQR2NATNegotiation@@MEBA_NXZ 0000000039a199a0 f   GameSpySBQR2NatNegotiation.obj
 0001:000189c0       ?NegotiateProgress@CGameSpySBQR2NATNegotiation@@CAXW4NegotiateState@@PEAX@Z 0000000039a199c0 f   GameSpySBQR2NatNegotiation.obj
 0001:00018a00       ?NegotiateComplete@CGameSpySBQR2NATNegotiation@@CAXW4NegotiateResult@@_KPEAUsockaddr_in@@PEAX@Z 0000000039a19a00 f   GameSpySBQR2NatNegotiation.obj
 0001:00018ac0       ?DetectComplete@CGameSpySBQR2NATNegotiation@@CAXHU_NAT@@@Z 0000000039a19ac0 f   GameSpySBQR2NatNegotiation.obj
 0001:00018c80       ?ProcessTasks@CGameSpySBQR2NATNegotiation@@AEAAXI@Z 0000000039a19c80 f   GameSpySBQR2NatNegotiation.obj
 0001:00018d30       ??1SNegotiateTask@CGameSpySBQR2NATNegotiation@@UEAA@XZ 0000000039a19d30 f   GameSpySBQR2NatNegotiation.obj
 0001:00018db0       ?StartTask@SNegotiateTask@CGameSpySBQR2NATNegotiation@@UEAAXXZ 0000000039a19db0 f   GameSpySBQR2NatNegotiation.obj
 0001:00018e00       ?FailTask@SNegotiateTask@CGameSpySBQR2NATNegotiation@@UEAAXXZ 0000000039a19e00 f   GameSpySBQR2NatNegotiation.obj
 0001:00018ec0       ??1SDetectTask@CGameSpySBQR2NATNegotiation@@UEAA@XZ 0000000039a19ec0 f   GameSpySBQR2NatNegotiation.obj
 0001:00018f70       ?StartTask@SDetectTask@CGameSpySBQR2NATNegotiation@@UEAAXXZ 0000000039a19f70 f   GameSpySBQR2NatNegotiation.obj
 0001:00019070       ?FailTask@SDetectTask@CGameSpySBQR2NATNegotiation@@UEAAXXZ 0000000039a1a070 f   GameSpySBQR2NatNegotiation.obj
 0001:000191d0       ??_ESTaskBase@CGameSpySBQR2NATNegotiation@@UEAAPEAXI@Z 0000000039a1a1d0 f i GameSpySBQR2NatNegotiation.obj
 0001:000191d0       ??_GSTaskBase@CGameSpySBQR2NATNegotiation@@UEAAPEAXI@Z 0000000039a1a1d0 f i GameSpySBQR2NatNegotiation.obj
 0001:00019260       ??_GSNegotiateTask@CGameSpySBQR2NATNegotiation@@UEAAPEAXI@Z 0000000039a1a260 f i GameSpySBQR2NatNegotiation.obj
 0001:00019260       ??_ESNegotiateTask@CGameSpySBQR2NATNegotiation@@UEAAPEAXI@Z 0000000039a1a260 f i GameSpySBQR2NatNegotiation.obj
 0001:00019290       ??_GSDetectTask@CGameSpySBQR2NATNegotiation@@UEAAPEAXI@Z 0000000039a1a290 f i GameSpySBQR2NatNegotiation.obj
 0001:00019290       ??_ESDetectTask@CGameSpySBQR2NATNegotiation@@UEAAPEAXI@Z 0000000039a1a290 f i GameSpySBQR2NatNegotiation.obj
 0001:000192c0       ??$__destroy_range@V?$reverse_iterator@PEAV?$_smart_ptr@USTaskLink@CCryGameSpySBQR2DLCStore@@@@@stlpmtx_std@@V?$_smart_ptr@USTaskLink@CCryGameSpySBQR2DLCStore@@@@@stlpmtx_std@@YAXV?$reverse_iterator@PEAV?$_smart_ptr@USTaskLink@CCryGameSpySBQR2DLCStore@@@@@0@0PEAV?$_smart_ptr@USTaskLink@CCryGameSpySBQR2DLCStore@@@@@Z 0000000039a1a2c0 f i CryGameSpySBQR2DLCStore.obj
 0001:000192c0       ??$__destroy_mv_srcs@V?$reverse_iterator@PEAV?$_smart_ptr@USTaskLink@CCryGameSpySBQR2DLCStore@@@@@stlpmtx_std@@V?$_smart_ptr@USTaskLink@CCryGameSpySBQR2DLCStore@@@@@stlpmtx_std@@YAXV?$reverse_iterator@PEAV?$_smart_ptr@USTaskLink@CCryGameSpySBQR2DLCStore@@@@@0@0PEAV?$_smart_ptr@USTaskLink@CCryGameSpySBQR2DLCStore@@@@@Z 0000000039a1a2c0 f i CryGameSpySBQR2DLCStore.obj
 0001:000192c0       ??$__destroy_range@V?$reverse_iterator@PEAV?$_smart_ptr@USCallbackBase@CGameSpySBQR2GPConnection@@@@@stlpmtx_std@@V?$_smart_ptr@USCallbackBase@CGameSpySBQR2GPConnection@@@@@stlpmtx_std@@YAXV?$reverse_iterator@PEAV?$_smart_ptr@USCallbackBase@CGameSpySBQR2GPConnection@@@@@0@0PEAV?$_smart_ptr@USCallbackBase@CGameSpySBQR2GPConnection@@@@@Z 0000000039a1a2c0 f i GameSpySBQR2GPConnection.obj
 0001:000192c0       ??$__destroy_range@V?$reverse_iterator@PEAV?$_smart_ptr@USOrderLink@CCryGameSpySBQR2DLCStore@@@@@stlpmtx_std@@V?$_smart_ptr@USOrderLink@CCryGameSpySBQR2DLCStore@@@@@stlpmtx_std@@YAXV?$reverse_iterator@PEAV?$_smart_ptr@USOrderLink@CCryGameSpySBQR2DLCStore@@@@@0@0PEAV?$_smart_ptr@USOrderLink@CCryGameSpySBQR2DLCStore@@@@@Z 0000000039a1a2c0 f i CryGameSpySBQR2DLCStore.obj
 0001:000192c0       ??$__destroy_mv_srcs@V?$reverse_iterator@PEAV?$_smart_ptr@USTaskCallbackBase@CGameSpySBQR2GPConnection@@@@@stlpmtx_std@@V?$_smart_ptr@USTaskCallbackBase@CGameSpySBQR2GPConnection@@@@@stlpmtx_std@@YAXV?$reverse_iterator@PEAV?$_smart_ptr@USTaskCallbackBase@CGameSpySBQR2GPConnection@@@@@0@0PEAV?$_smart_ptr@USTaskCallbackBase@CGameSpySBQR2GPConnection@@@@@Z 0000000039a1a2c0 f i GameSpySBQR2GPConnection.obj
 0001:000192c0       ??$__destroy_mv_srcs@V?$reverse_iterator@PEAV?$_smart_ptr@USRegisteredLobbyData@CCryGameSpySBQR2MatchMaking@@@@@stlpmtx_std@@V?$_smart_ptr@USRegisteredLobbyData@CCryGameSpySBQR2MatchMaking@@@@@stlpmtx_std@@YAXV?$reverse_iterator@PEAV?$_smart_ptr@USRegisteredLobbyData@CCryGameSpySBQR2MatchMaking@@@@@0@0PEAV?$_smart_ptr@USRegisteredLobbyData@CCryGameSpySBQR2MatchMaking@@@@@Z 0000000039a1a2c0 f i CryGameSpySBQR2MatchMaking.obj
 0001:000192c0       ??$__destroy_range@V?$reverse_iterator@PEAV?$_smart_ptr@USTaskBase@CGameSpySBQR2NATNegotiation@@@@@stlpmtx_std@@V?$_smart_ptr@USTaskBase@CGameSpySBQR2NATNegotiation@@@@@stlpmtx_std@@YAXV?$reverse_iterator@PEAV?$_smart_ptr@USTaskBase@CGameSpySBQR2NATNegotiation@@@@@0@0PEAV?$_smart_ptr@USTaskBase@CGameSpySBQR2NATNegotiation@@@@@Z 0000000039a1a2c0 f i GameSpySBQR2NatNegotiation.obj
 0001:000192c0       ??$__destroy_range@V?$reverse_iterator@PEAV?$_smart_ptr@USTaskLink@CCryGameSpySBQR2Stats@@@@@stlpmtx_std@@V?$_smart_ptr@USTaskLink@CCryGameSpySBQR2Stats@@@@@stlpmtx_std@@YAXV?$reverse_iterator@PEAV?$_smart_ptr@USTaskLink@CCryGameSpySBQR2Stats@@@@@0@0PEAV?$_smart_ptr@USTaskLink@CCryGameSpySBQR2Stats@@@@@Z 0000000039a1a2c0 f i CryGameSpySBQR2Stats.obj
 0001:000192c0       ??$__destroy_range@V?$reverse_iterator@PEAV?$_smart_ptr@USTaskCallbackBase@CGameSpySBQR2GPConnection@@@@@stlpmtx_std@@V?$_smart_ptr@USTaskCallbackBase@CGameSpySBQR2GPConnection@@@@@stlpmtx_std@@YAXV?$reverse_iterator@PEAV?$_smart_ptr@USTaskCallbackBase@CGameSpySBQR2GPConnection@@@@@0@0PEAV?$_smart_ptr@USTaskCallbackBase@CGameSpySBQR2GPConnection@@@@@Z 0000000039a1a2c0 f i GameSpySBQR2GPConnection.obj
 0001:000192c0       ??$__destroy_mv_srcs@V?$reverse_iterator@PEAV?$_smart_ptr@USOrderLink@CCryGameSpySBQR2DLCStore@@@@@stlpmtx_std@@V?$_smart_ptr@USOrderLink@CCryGameSpySBQR2DLCStore@@@@@stlpmtx_std@@YAXV?$reverse_iterator@PEAV?$_smart_ptr@USOrderLink@CCryGameSpySBQR2DLCStore@@@@@0@0PEAV?$_smart_ptr@USOrderLink@CCryGameSpySBQR2DLCStore@@@@@Z 0000000039a1a2c0 f i CryGameSpySBQR2DLCStore.obj
 0001:000192c0       ??$__destroy_mv_srcs@V?$reverse_iterator@PEAV?$_smart_ptr@USTaskBase@CGameSpySBQR2Sake@@@@@stlpmtx_std@@V?$_smart_ptr@USTaskBase@CGameSpySBQR2Sake@@@@@stlpmtx_std@@YAXV?$reverse_iterator@PEAV?$_smart_ptr@USTaskBase@CGameSpySBQR2Sake@@@@@0@0PEAV?$_smart_ptr@USTaskBase@CGameSpySBQR2Sake@@@@@Z 0000000039a1a2c0 f i GameSpySBQR2Sake.obj
 0001:000192c0       ??$__destroy_range@V?$reverse_iterator@PEAV?$_smart_ptr@USTaskBase@CGameSpySBQR2Sake@@@@@stlpmtx_std@@V?$_smart_ptr@USTaskBase@CGameSpySBQR2Sake@@@@@stlpmtx_std@@YAXV?$reverse_iterator@PEAV?$_smart_ptr@USTaskBase@CGameSpySBQR2Sake@@@@@0@0PEAV?$_smart_ptr@USTaskBase@CGameSpySBQR2Sake@@@@@Z 0000000039a1a2c0 f i GameSpySBQR2Sake.obj
 0001:000192c0       ??$__destroy_range@V?$reverse_iterator@PEAV?$_smart_ptr@USRegisteredLobbyData@CCryGameSpySBQR2MatchMaking@@@@@stlpmtx_std@@V?$_smart_ptr@USRegisteredLobbyData@CCryGameSpySBQR2MatchMaking@@@@@stlpmtx_std@@YAXV?$reverse_iterator@PEAV?$_smart_ptr@USRegisteredLobbyData@CCryGameSpySBQR2MatchMaking@@@@@0@0PEAV?$_smart_ptr@USRegisteredLobbyData@CCryGameSpySBQR2MatchMaking@@@@@Z 0000000039a1a2c0 f i CryGameSpySBQR2MatchMaking.obj
 0001:000192c0       ??$__destroy_range@V?$reverse_iterator@PEAV?$_smart_ptr@USTask@CGameSpySBQR2Core@@@@@stlpmtx_std@@V?$_smart_ptr@USTask@CGameSpySBQR2Core@@@@@stlpmtx_std@@YAXV?$reverse_iterator@PEAV?$_smart_ptr@USTask@CGameSpySBQR2Core@@@@@0@0PEAV?$_smart_ptr@USTask@CGameSpySBQR2Core@@@@@Z 0000000039a1a2c0 f i GameSpySBQR2Core.obj
 0001:000192c0       ??$__destroy_mv_srcs@V?$reverse_iterator@PEAV?$_smart_ptr@USTaskBase@CGameSpySBQR2NATNegotiation@@@@@stlpmtx_std@@V?$_smart_ptr@USTaskBase@CGameSpySBQR2NATNegotiation@@@@@stlpmtx_std@@YAXV?$reverse_iterator@PEAV?$_smart_ptr@USTaskBase@CGameSpySBQR2NATNegotiation@@@@@0@0PEAV?$_smart_ptr@USTaskBase@CGameSpySBQR2NATNegotiation@@@@@Z 0000000039a1a2c0 f i GameSpySBQR2NatNegotiation.obj
 0001:000192c0       ??$__destroy_mv_srcs@V?$reverse_iterator@PEAV?$_smart_ptr@USCallbackBase@CGameSpySBQR2GPConnection@@@@@stlpmtx_std@@V?$_smart_ptr@USCallbackBase@CGameSpySBQR2GPConnection@@@@@stlpmtx_std@@YAXV?$reverse_iterator@PEAV?$_smart_ptr@USCallbackBase@CGameSpySBQR2GPConnection@@@@@0@0PEAV?$_smart_ptr@USCallbackBase@CGameSpySBQR2GPConnection@@@@@Z 0000000039a1a2c0 f i GameSpySBQR2GPConnection.obj
 0001:000192c0       ??$__destroy_mv_srcs@V?$reverse_iterator@PEAV?$_smart_ptr@USTask@CGameSpySBQR2Core@@@@@stlpmtx_std@@V?$_smart_ptr@USTask@CGameSpySBQR2Core@@@@@stlpmtx_std@@YAXV?$reverse_iterator@PEAV?$_smart_ptr@USTask@CGameSpySBQR2Core@@@@@0@0PEAV?$_smart_ptr@USTask@CGameSpySBQR2Core@@@@@Z 0000000039a1a2c0 f i GameSpySBQR2Core.obj
 0001:00019340       ??0CGameSpySBQR2NATNegotiation@@QEAA@PEAVCCryGameSpySBQR2LobbyService@@@Z 0000000039a1a340 f   GameSpySBQR2NatNegotiation.obj
 0001:000193b0       ?TearDown@CGameSpySBQR2NATNegotiation@@AEAAXXZ 0000000039a1a3b0 f   GameSpySBQR2NatNegotiation.obj
 0001:00019470       ?AddTask@CGameSpySBQR2NATNegotiation@@AEAAXPEAUSTaskBase@1@@Z 0000000039a1a470 f   GameSpySBQR2NatNegotiation.obj
 0001:00019620       ??0STaskBase@CGameSpySBQR2NATNegotiation@@QEAA@PEAV1@PEAUIGameSpyLink@@@Z 0000000039a1a620 f   GameSpySBQR2NatNegotiation.obj
 0001:000196a0       ??1CGameSpySBQR2NATNegotiation@@UEAA@XZ 0000000039a1a6a0 f   GameSpySBQR2NatNegotiation.obj
 0001:00019730       ?PerformThink@CGameSpySBQR2NATNegotiation@@MEAAXXZ 0000000039a1a730 f   GameSpySBQR2NatNegotiation.obj
 0001:00019800       ?BeginNegotiationWithSocket@CGameSpySBQR2NATNegotiation@@QEAAX_KHHP6AXUSResult@1@HPEAUIGameSpyLink@@@ZP6AX1H0PEAUsockaddr_in@@2@Z2@Z 0000000039a1a800 f   GameSpySBQR2NatNegotiation.obj
 0001:000198e0       ?StartNATDetection@CGameSpySBQR2NATNegotiation@@QEAAXP6AXUSResult@1@W4ENatType@@PEAUIGameSpyLink@@@Z2@Z 0000000039a1a8e0 f   GameSpySBQR2NatNegotiation.obj
 0001:00019990       ??_GCGameSpySBQR2NATNegotiation@@UEAAPEAXI@Z 0000000039a1a990 f i GameSpySBQR2NatNegotiation.obj
 0001:00019990       ??_ECGameSpySBQR2NATNegotiation@@UEAAPEAXI@Z 0000000039a1a990 f i GameSpySBQR2NatNegotiation.obj
 0001:000199c0       ?NeedThink@CGameSpySBQR2Sake@@MEBA_NXZ 0000000039a1a9c0 f   GameSpySBQR2Sake.obj
 0001:000199f0       ?CloneString@CGameSpySBQR2Sake@@CAXAEAPEADPEBDAEAPEAX@Z 0000000039a1a9f0 f   GameSpySBQR2Sake.obj
 0001:00019a80       ?CloneWString@CGameSpySBQR2Sake@@CAXAEAPEA_WPEB_WAEAPEAX@Z 0000000039a1aa80 f   GameSpySBQR2Sake.obj
 0001:00019b30       ?CloneSakeFieldNames@CGameSpySBQR2Sake@@CAXAEAPEAPEADAEAHPEBQEBDHAEAPEAX@Z 0000000039a1ab30 f   GameSpySBQR2Sake.obj
 0001:00019c50       ?FreeSakeFields@CGameSpySBQR2Sake@@CAXAEAPEAUSAKEField@@AEAH@Z 0000000039a1ac50 f   GameSpySBQR2Sake.obj
 0001:00019cd0       ?FreeInput@CGameSpySBQR2Sake@@CAXAEAPEAUSAKEGetMyRecordsInput@@@Z 0000000039a1acd0 f   GameSpySBQR2Sake.obj
 0001:00019d50       ?FreeInput@CGameSpySBQR2Sake@@CAXAEAPEAUSAKESearchForRecordsInput@@@Z 0000000039a1ad50 f   GameSpySBQR2Sake.obj
 0001:00019e10       ??$CloneArray@E@CGameSpySBQR2Sake@@CAXAEAPEAEAEAHPEBEHAEAPEAX@Z 0000000039a1ae10 f i GameSpySBQR2Sake.obj
 0001:00019e90       ?CloneSakeFields@CGameSpySBQR2Sake@@CAXAEAPEAUSAKEField@@AEAHPEBU2@HAEAPEAX@Z 0000000039a1ae90 f   GameSpySBQR2Sake.obj
 0001:0001a030       ?CloneInput@CGameSpySBQR2Sake@@CAPEAUSAKECreateRecordInput@@PEBU2@@Z 0000000039a1b030 f   GameSpySBQR2Sake.obj
 0001:0001a140       ?CloneInput@CGameSpySBQR2Sake@@CAPEAUSAKEGetMyRecordsInput@@PEBU2@@Z 0000000039a1b140 f   GameSpySBQR2Sake.obj
 0001:0001a280       ?CloneInput@CGameSpySBQR2Sake@@CAPEAUSAKEGetRecordCountInput@@PEBU2@@Z 0000000039a1b280 f   GameSpySBQR2Sake.obj
 0001:0001a3c0       ?CloneInput@CGameSpySBQR2Sake@@CAPEAUSAKESearchForRecordsInput@@PEBU2@@Z 0000000039a1b3c0 f   GameSpySBQR2Sake.obj
 0001:0001a620       ?CloneInput@CGameSpySBQR2Sake@@CAPEAUSAKEUpdateRecordInput@@PEBU2@@Z 0000000039a1b620 f   GameSpySBQR2Sake.obj
 0001:0001a730       ??_ESTaskBase@CGameSpySBQR2Sake@@UEAAPEAXI@Z 0000000039a1b730 f i GameSpySBQR2Sake.obj
 0001:0001a730       ??_GSTaskBase@CGameSpySBQR2Sake@@UEAAPEAXI@Z 0000000039a1b730 f i GameSpySBQR2Sake.obj
 0001:0001a770       ?StartTask@STaskBase@CGameSpySBQR2Sake@@UEAAXXZ 0000000039a1b770 f   GameSpySBQR2Sake.obj
 0001:0001a7e0       ?ProcessTasks@CGameSpySBQR2Sake@@AEAAXI@Z 0000000039a1b7e0 f   GameSpySBQR2Sake.obj
 0001:0001a870       ?SakeTaskFinished@STaskBase@CGameSpySBQR2Sake@@QEAAXXZ 0000000039a1b870 f   GameSpySBQR2Sake.obj
 0001:0001a990       ??$TaskFinished@USAKEUpdateRecordInput@@@CGameSpySBQR2Sake@@CAXPEAUSAKEInternal@@PEAUSAKERequestInternal@@W4SAKERequestResult@@PEAX33@Z 0000000039a1b990 f   GameSpySBQR2Sake.obj
 0001:0001aa00       ?_M_insert_overflow_aux@?$_Impl_vector@V?$_smart_ptr@USCallbackBase@CGameSpySBQR2GPConnection@@@@V?$allocator@V?$_smart_ptr@USCallbackBase@CGameSpySBQR2GPConnection@@@@@stlpmtx_std@@@priv@stlpmtx_std@@AEAAXPEAV?$_smart_ptr@USCallbackBase@CGameSpySBQR2GPConnection@@@@AEBV4@AEBU__false_type@3@_K_N@Z 0000000039a1ba00 f i GameSpySBQR2GPConnection.obj
 0001:0001aa00       ?_M_insert_overflow_aux@?$_Impl_vector@V?$_smart_ptr@USTask@CGameSpySBQR2Core@@@@V?$allocator@V?$_smart_ptr@USTask@CGameSpySBQR2Core@@@@@stlpmtx_std@@@priv@stlpmtx_std@@AEAAXPEAV?$_smart_ptr@USTask@CGameSpySBQR2Core@@@@AEBV4@AEBU__false_type@3@_K_N@Z 0000000039a1ba00 f i GameSpySBQR2Core.obj
 0001:0001aa00       ?_M_insert_overflow_aux@?$_Impl_vector@V?$_smart_ptr@USTaskBase@CGameSpySBQR2NATNegotiation@@@@V?$allocator@V?$_smart_ptr@USTaskBase@CGameSpySBQR2NATNegotiation@@@@@stlpmtx_std@@@priv@stlpmtx_std@@AEAAXPEAV?$_smart_ptr@USTaskBase@CGameSpySBQR2NATNegotiation@@@@AEBV4@AEBU__false_type@3@_K_N@Z 0000000039a1ba00 f i GameSpySBQR2NatNegotiation.obj
 0001:0001aa00       ?_M_insert_overflow_aux@?$_Impl_vector@V?$_smart_ptr@USRegisteredLobbyData@CCryGameSpySBQR2MatchMaking@@@@V?$allocator@V?$_smart_ptr@USRegisteredLobbyData@CCryGameSpySBQR2MatchMaking@@@@@stlpmtx_std@@@priv@stlpmtx_std@@AEAAXPEAV?$_smart_ptr@USRegisteredLobbyData@CCryGameSpySBQR2MatchMaking@@@@AEBV4@AEBU__false_type@3@_K_N@Z 0000000039a1ba00 f i CryGameSpySBQR2MatchMaking.obj
 0001:0001aa00       ?_M_insert_overflow_aux@?$_Impl_vector@V?$_smart_ptr@USTaskBase@CGameSpySBQR2Sake@@@@V?$allocator@V?$_smart_ptr@USTaskBase@CGameSpySBQR2Sake@@@@@stlpmtx_std@@@priv@stlpmtx_std@@AEAAXPEAV?$_smart_ptr@USTaskBase@CGameSpySBQR2Sake@@@@AEBV4@AEBU__false_type@3@_K_N@Z 0000000039a1ba00 f i GameSpySBQR2Sake.obj
 0001:0001aa00       ?_M_insert_overflow_aux@?$_Impl_vector@V?$_smart_ptr@USTaskCallbackBase@CGameSpySBQR2GPConnection@@@@V?$allocator@V?$_smart_ptr@USTaskCallbackBase@CGameSpySBQR2GPConnection@@@@@stlpmtx_std@@@priv@stlpmtx_std@@AEAAXPEAV?$_smart_ptr@USTaskCallbackBase@CGameSpySBQR2GPConnection@@@@AEBV4@AEBU__false_type@3@_K_N@Z 0000000039a1ba00 f i GameSpySBQR2GPConnection.obj
 0001:0001aa00       ?_M_insert_overflow_aux@?$_Impl_vector@V?$_smart_ptr@USTaskLink@CCryGameSpySBQR2DLCStore@@@@V?$allocator@V?$_smart_ptr@USTaskLink@CCryGameSpySBQR2DLCStore@@@@@stlpmtx_std@@@priv@stlpmtx_std@@AEAAXPEAV?$_smart_ptr@USTaskLink@CCryGameSpySBQR2DLCStore@@@@AEBV4@AEBU__false_type@3@_K_N@Z 0000000039a1ba00 f i CryGameSpySBQR2DLCStore.obj
 0001:0001aa00       ?_M_insert_overflow_aux@?$_Impl_vector@V?$_smart_ptr@USOrderLink@CCryGameSpySBQR2DLCStore@@@@V?$allocator@V?$_smart_ptr@USOrderLink@CCryGameSpySBQR2DLCStore@@@@@stlpmtx_std@@@priv@stlpmtx_std@@AEAAXPEAV?$_smart_ptr@USOrderLink@CCryGameSpySBQR2DLCStore@@@@AEBV4@AEBU__false_type@3@_K_N@Z 0000000039a1ba00 f i CryGameSpySBQR2DLCStore.obj
 0001:0001ac00       ??0CGameSpySBQR2Sake@@QEAA@PEAVCCryGameSpySBQR2LobbyService@@I@Z 0000000039a1bc00 f   GameSpySBQR2Sake.obj
 0001:0001acb0       ?AddTask@CGameSpySBQR2Sake@@AEAAXPEAUSTaskBase@1@@Z 0000000039a1bcb0 f   GameSpySBQR2Sake.obj
 0001:0001ae60       ??0STaskBase@CGameSpySBQR2Sake@@QEAA@PEAV1@PEAUIGameSpyLink@@HPEBD@Z 0000000039a1be60 f   GameSpySBQR2Sake.obj
 0001:0001aef0       ??0?$STask@USAKEUpdateRecordInput@@@CGameSpySBQR2Sake@@QEAA@PEAV1@PEAUIGameSpyLink@@PEAUSAKEUpdateRecordInput@@P6APEAUSAKERequestInternal@@PEAUSAKEInternal@@2P6AX3PEAU4@W4SAKERequestResult@@PEAX66@Z6@ZP6AX0USResult@1@21@Z@Z 0000000039a1bef0 f i GameSpySBQR2Sake.obj
 0001:0001afa0       ??1?$STask@USAKEUpdateRecordInput@@@CGameSpySBQR2Sake@@UEAA@XZ 0000000039a1bfa0 f i GameSpySBQR2Sake.obj
 0001:0001b010       ??_G?$STask@USAKEUpdateRecordInput@@@CGameSpySBQR2Sake@@UEAAPEAXI@Z 0000000039a1c010 f i GameSpySBQR2Sake.obj
 0001:0001b010       ??_E?$STask@USAKEUpdateRecordInput@@@CGameSpySBQR2Sake@@UEAAPEAXI@Z 0000000039a1c010 f i GameSpySBQR2Sake.obj
 0001:0001b040       ?FailTask@?$STask@USAKEUpdateRecordInput@@@CGameSpySBQR2Sake@@UEAAXXZ 0000000039a1c040 f i GameSpySBQR2Sake.obj
 0001:0001b0a0       ?CallStartTaskFunc@?$STask@USAKEUpdateRecordInput@@@CGameSpySBQR2Sake@@UEAAXXZ 0000000039a1c0a0 f i GameSpySBQR2Sake.obj
 0001:0001b0d0       ??0?$STask@USAKECreateRecordInput@@@CGameSpySBQR2Sake@@QEAA@PEAV1@PEAUIGameSpyLink@@PEAUSAKECreateRecordInput@@P6APEAUSAKERequestInternal@@PEAUSAKEInternal@@2P6AX3PEAU4@W4SAKERequestResult@@PEAX66@Z6@ZP6AX0USResult@1@2PEAUSAKECreateRecordOutput@@1@Z@Z 0000000039a1c0d0 f i GameSpySBQR2Sake.obj
 0001:0001b180       ??1?$STask@USAKECreateRecordInput@@@CGameSpySBQR2Sake@@UEAA@XZ 0000000039a1c180 f i GameSpySBQR2Sake.obj
 0001:0001b1f0       ??_G?$STask@USAKECreateRecordInput@@@CGameSpySBQR2Sake@@UEAAPEAXI@Z 0000000039a1c1f0 f i GameSpySBQR2Sake.obj
 0001:0001b1f0       ??_E?$STask@USAKECreateRecordInput@@@CGameSpySBQR2Sake@@UEAAPEAXI@Z 0000000039a1c1f0 f i GameSpySBQR2Sake.obj
 0001:0001b220       ??0?$STask@USAKEGetMyRecordsInput@@@CGameSpySBQR2Sake@@QEAA@PEAV1@PEAUIGameSpyLink@@PEAUSAKEGetMyRecordsInput@@P6APEAUSAKERequestInternal@@PEAUSAKEInternal@@2P6AX3PEAU4@W4SAKERequestResult@@PEAX66@Z6@ZP6AX0USResult@1@2PEAUSAKEGetMyRecordsOutput@@1@Z@Z 0000000039a1c220 f i GameSpySBQR2Sake.obj
 0001:0001b2d0       ??_E?$STask@USAKEGetMyRecordsInput@@@CGameSpySBQR2Sake@@UEAAPEAXI@Z 0000000039a1c2d0 f i GameSpySBQR2Sake.obj
 0001:0001b2d0       ??_G?$STask@USAKEGetMyRecordsInput@@@CGameSpySBQR2Sake@@UEAAPEAXI@Z 0000000039a1c2d0 f i GameSpySBQR2Sake.obj
 0001:0001b320       ?SakeTaskFailed@?$STask@USAKESearchForRecordsInput@@@CGameSpySBQR2Sake@@UEAAXXZ 0000000039a1c320 f i GameSpySBQR2Sake.obj
 0001:0001b320       ?SakeTaskFailed@?$STask@USAKECreateRecordInput@@@CGameSpySBQR2Sake@@UEAAXXZ 0000000039a1c320 f i GameSpySBQR2Sake.obj
 0001:0001b320       ?SakeTaskFailed@?$STask@USAKEGetRecordCountInput@@@CGameSpySBQR2Sake@@UEAAXXZ 0000000039a1c320 f i GameSpySBQR2Sake.obj
 0001:0001b320       ?SakeTaskFailed@?$STask@USAKEUpdateRecordInput@@@CGameSpySBQR2Sake@@UEAAXXZ 0000000039a1c320 f i GameSpySBQR2Sake.obj
 0001:0001b320       ?SakeTaskFailed@?$STask@USAKEGetMyRecordsInput@@@CGameSpySBQR2Sake@@UEAAXXZ 0000000039a1c320 f i GameSpySBQR2Sake.obj
 0001:0001b340       ??0?$STask@USAKEGetRecordCountInput@@@CGameSpySBQR2Sake@@QEAA@PEAV1@PEAUIGameSpyLink@@PEAUSAKEGetRecordCountInput@@P6APEAUSAKERequestInternal@@PEAUSAKEInternal@@2P6AX3PEAU4@W4SAKERequestResult@@PEAX66@Z6@ZP6AX0USResult@1@2PEAUSAKEGetRecordCountOutput@@1@Z@Z 0000000039a1c340 f i GameSpySBQR2Sake.obj
 0001:0001b3f0       ??1?$STask@USAKEGetRecordCountInput@@@CGameSpySBQR2Sake@@UEAA@XZ 0000000039a1c3f0 f i GameSpySBQR2Sake.obj
 0001:0001b460       ??_E?$STask@USAKEGetRecordCountInput@@@CGameSpySBQR2Sake@@UEAAPEAXI@Z 0000000039a1c460 f i GameSpySBQR2Sake.obj
 0001:0001b460       ??_G?$STask@USAKEGetRecordCountInput@@@CGameSpySBQR2Sake@@UEAAPEAXI@Z 0000000039a1c460 f i GameSpySBQR2Sake.obj
 0001:0001b490       ?FailTask@?$STask@USAKECreateRecordInput@@@CGameSpySBQR2Sake@@UEAAXXZ 0000000039a1c490 f i GameSpySBQR2Sake.obj
 0001:0001b490       ?FailTask@?$STask@USAKEGetMyRecordsInput@@@CGameSpySBQR2Sake@@UEAAXXZ 0000000039a1c490 f i GameSpySBQR2Sake.obj
 0001:0001b490       ?FailTask@?$STask@USAKEGetRecordCountInput@@@CGameSpySBQR2Sake@@UEAAXXZ 0000000039a1c490 f i GameSpySBQR2Sake.obj
 0001:0001b490       ?FailTask@?$STask@USAKESearchForRecordsInput@@@CGameSpySBQR2Sake@@UEAAXXZ 0000000039a1c490 f i GameSpySBQR2Sake.obj
 0001:0001b4f0       ??$TaskFinished@USAKEGetRecordCountInput@@@CGameSpySBQR2Sake@@CAXPEAUSAKEInternal@@PEAUSAKERequestInternal@@W4SAKERequestResult@@PEAX33@Z 0000000039a1c4f0 f i GameSpySBQR2Sake.obj
 0001:0001b4f0       ??$TaskFinished@USAKESearchForRecordsInput@@@CGameSpySBQR2Sake@@CAXPEAUSAKEInternal@@PEAUSAKERequestInternal@@W4SAKERequestResult@@PEAX33@Z 0000000039a1c4f0 f i GameSpySBQR2Sake.obj
 0001:0001b4f0       ??$TaskFinished@USAKEGetMyRecordsInput@@@CGameSpySBQR2Sake@@CAXPEAUSAKEInternal@@PEAUSAKERequestInternal@@W4SAKERequestResult@@PEAX33@Z 0000000039a1c4f0 f i GameSpySBQR2Sake.obj
 0001:0001b4f0       ??$TaskFinished@USAKECreateRecordInput@@@CGameSpySBQR2Sake@@CAXPEAUSAKEInternal@@PEAUSAKERequestInternal@@W4SAKERequestResult@@PEAX33@Z 0000000039a1c4f0 f i GameSpySBQR2Sake.obj
 0001:0001b560       ?CallStartTaskFunc@?$STask@USAKESearchForRecordsInput@@@CGameSpySBQR2Sake@@UEAAXXZ 0000000039a1c560 f i GameSpySBQR2Sake.obj
 0001:0001b560       ?CallStartTaskFunc@?$STask@USAKEGetMyRecordsInput@@@CGameSpySBQR2Sake@@UEAAXXZ 0000000039a1c560 f i GameSpySBQR2Sake.obj
 0001:0001b560       ?CallStartTaskFunc@?$STask@USAKECreateRecordInput@@@CGameSpySBQR2Sake@@UEAAXXZ 0000000039a1c560 f i GameSpySBQR2Sake.obj
 0001:0001b560       ?CallStartTaskFunc@?$STask@USAKEGetRecordCountInput@@@CGameSpySBQR2Sake@@UEAAXXZ 0000000039a1c560 f i GameSpySBQR2Sake.obj
 0001:0001b590       ??0?$STask@USAKESearchForRecordsInput@@@CGameSpySBQR2Sake@@QEAA@PEAV1@PEAUIGameSpyLink@@PEAUSAKESearchForRecordsInput@@P6APEAUSAKERequestInternal@@PEAUSAKEInternal@@2P6AX3PEAU4@W4SAKERequestResult@@PEAX66@Z6@ZP6AX0USResult@1@2PEAUSAKESearchForRecordsOutput@@1@Z@Z 0000000039a1c590 f i GameSpySBQR2Sake.obj
 0001:0001b640       ??_E?$STask@USAKESearchForRecordsInput@@@CGameSpySBQR2Sake@@UEAAPEAXI@Z 0000000039a1c640 f i GameSpySBQR2Sake.obj
 0001:0001b640       ??_G?$STask@USAKESearchForRecordsInput@@@CGameSpySBQR2Sake@@UEAAPEAXI@Z 0000000039a1c640 f i GameSpySBQR2Sake.obj
 0001:0001b690       ??1CGameSpySBQR2Sake@@UEAA@XZ 0000000039a1c690 f   GameSpySBQR2Sake.obj
 0001:0001b780       ?PerformThink@CGameSpySBQR2Sake@@MEAAXXZ 0000000039a1c780 f   GameSpySBQR2Sake.obj
 0001:0001b910       ?CreateRecord@CGameSpySBQR2Sake@@QEAAXPEAUSAKECreateRecordInput@@P6AXPEAV1@USResult@1@0PEAUSAKECreateRecordOutput@@PEAUIGameSpyLink@@@Z4@Z 0000000039a1c910 f   GameSpySBQR2Sake.obj
 0001:0001b9c0       ?GetMyRecords@CGameSpySBQR2Sake@@QEAAXPEAUSAKEGetMyRecordsInput@@P6AXPEAV1@USResult@1@0PEAUSAKEGetMyRecordsOutput@@PEAUIGameSpyLink@@@Z4@Z 0000000039a1c9c0 f   GameSpySBQR2Sake.obj
 0001:0001ba70       ?GetRecordCount@CGameSpySBQR2Sake@@QEAAXPEAUSAKEGetRecordCountInput@@P6AXPEAV1@USResult@1@0PEAUSAKEGetRecordCountOutput@@PEAUIGameSpyLink@@@Z4@Z 0000000039a1ca70 f   GameSpySBQR2Sake.obj
 0001:0001bb20       ?SearchForRecords@CGameSpySBQR2Sake@@QEAAXPEAUSAKESearchForRecordsInput@@P6AXPEAV1@USResult@1@0PEAUSAKESearchForRecordsOutput@@PEAUIGameSpyLink@@@Z4@Z 0000000039a1cb20 f   GameSpySBQR2Sake.obj
 0001:0001bbd0       ?UpdateRecord@CGameSpySBQR2Sake@@QEAAXPEAUSAKEUpdateRecordInput@@P6AXPEAV1@USResult@1@0PEAUIGameSpyLink@@@Z3@Z 0000000039a1cbd0 f   GameSpySBQR2Sake.obj
 0001:0001bc70       ??_ECGameSpySBQR2Sake@@UEAAPEAXI@Z 0000000039a1cc70 f i GameSpySBQR2Sake.obj
 0001:0001bc70       ??_GCGameSpySBQR2Sake@@UEAAPEAXI@Z 0000000039a1cc70 f i GameSpySBQR2Sake.obj
 0001:0001bca0       ?AddRef@CGameSpySDK@@QEAAXXZ 0000000039a1cca0 f   GameSpySDK.obj
 0001:0001bcb0       ?Release@CGameSpySDK@@QEAAXXZ 0000000039a1ccb0 f   GameSpySDK.obj
 0001:0001bcc0       ??0CGameSpyThinkerSDK@@IEAA@PEAVCCryGameSpySBQR2LobbyService@@@Z 0000000039a1ccc0 f   GameSpySDK.obj
 0001:0001bd10       ??1CGameSpyThinkerSDK@@UEAA@XZ 0000000039a1cd10 f   GameSpySDK.obj
 0001:0001bd20       ?DoThink@CGameSpyThinkerSDK@@QEAAXXZ 0000000039a1cd20 f   GameSpySDK.obj
 0001:0001bd40       ?GetThinker@CGameSpyThinkerSDK@@MEAAPEAV1@XZ 0000000039a1cd40 f   GameSpySDK.obj
 0001:0001bd40       ??0CCryRebroadcaster@@QEAA@PEAVCCryLobby@@@Z 0000000039a1cd40 f   CryRebroadcaster.obj
 0001:0001bd50       ?RequestThink@CGameSpySDK@@QEAAXXZ 0000000039a1cd50 f   GameSpySDK.obj
 0001:0001bd90       ??_ECGameSpySDK@@UEAAPEAXI@Z 0000000039a1cd90 f i GameSpySDK.obj
 0001:0001bd90       ??_GCGameSpySDK@@UEAAPEAXI@Z 0000000039a1cd90 f i GameSpySDK.obj
 0001:0001bd90       ??_ECGameSpyThinkerSDK@@UEAAPEAXI@Z 0000000039a1cd90 f i GameSpySDK.obj
 0001:0001bd90       ??_GCGameSpyThinkerSDK@@UEAAPEAXI@Z 0000000039a1cd90 f i GameSpySDK.obj
 0001:0001bdc0       ?Initialise@CCryGameSpySBQR2DLCStore@@UEAA?AW4ECryLobbyError@@XZ 0000000039a1cdc0 f   CryGameSpySBQR2DLCStore.obj
 0001:0001be00       ?Terminate@CCryGameSpySBQR2DLCStore@@UEAA?AW4ECryLobbyError@@XZ 0000000039a1ce00 f   CryGameSpySBQR2DLCStore.obj
 0001:0001be90       ?TickCheckAvailability@CCryGameSpySBQR2DLCStore@@IEAAXI@Z 0000000039a1ce90 f   CryGameSpySBQR2DLCStore.obj
 0001:0001bee0       ?TickCatalogListItems@CCryGameSpySBQR2DLCStore@@IEAAXI@Z 0000000039a1cee0 f   CryGameSpySBQR2DLCStore.obj
 0001:0001bee0       ?TickCatalogListCategories@CCryGameSpySBQR2DLCStore@@IEAAXI@Z 0000000039a1cee0 f   CryGameSpySBQR2DLCStore.obj
 0001:0001bf30       ?EndUserGetDownloadableAccess@CCryGameSpySBQR2DLCStore@@IEAAXI@Z 0000000039a1cf30 f   CryGameSpySBQR2DLCStore.obj
 0001:0001bfd0       ?CancelActiveDownloadInternal@CCryGameSpySBQR2DLCStore@@IEAAXXZ 0000000039a1cfd0 f   CryGameSpySBQR2DLCStore.obj
 0001:0001bfe0       ?EndUserListPaymentMethods@CCryGameSpySBQR2DLCStore@@IEAAXI@Z 0000000039a1cfe0 f   CryGameSpySBQR2DLCStore.obj
 0001:0001c0e0       ?StartOrderAdjustItemQuantity@CCryGameSpySBQR2DLCStore@@IEAAXI@Z 0000000039a1d0e0 f   CryGameSpySBQR2DLCStore.obj
 0001:0001c120       ?StartOrderCancel@CCryGameSpySBQR2DLCStore@@IEAAXI@Z 0000000039a1d120 f   CryGameSpySBQR2DLCStore.obj
 0001:0001c190       ?StartOrderFree@CCryGameSpySBQR2DLCStore@@IEAAXI@Z 0000000039a1d190 f   CryGameSpySBQR2DLCStore.obj
 0001:0001c210       ?CountItemsInOrderItemPurchase@CCryGameSpySBQR2DLCStore@@KAIPEAUD2GOrderItemPurchase@@@Z 0000000039a1d210 f   CryGameSpySBQR2DLCStore.obj
 0001:0001c270       ?OnGameSpyObjectAvailable@CCryGameSpySBQR2DLCStore@@UEAAXW4EGameSpyObjectBit@ICryGameSpySBQR2LobbyComponent@@@Z 0000000039a1d270 f   CryGameSpySBQR2DLCStore.obj
 0001:0001c2a0       ?OnGameSpyObjectUnavailable@CCryGameSpySBQR2DLCStore@@UEAAXW4EGameSpyObjectBit@ICryGameSpySBQR2LobbyComponent@@@Z 0000000039a1d2a0 f   CryGameSpySBQR2DLCStore.obj
 0001:0001c2d0       ?OnGameSpyObjectCantMakeAvailable@CCryGameSpySBQR2DLCStore@@UEAAXW4EGameSpyObjectBit@ICryGameSpySBQR2LobbyComponent@@@Z 0000000039a1d2d0 f   CryGameSpySBQR2DLCStore.obj
 0001:0001c340       ?CheckTaskGameSpyObjects@CCryGameSpySBQR2DLCStore@@IEAA?AW4ETaskGameSpyCheckResult@ICryGameSpySBQR2LobbyComponent@@I@Z 0000000039a1d340 f   CryGameSpySBQR2DLCStore.obj
 0001:0001c3d0       ?_AllocData@?$CryStackStringT@D$0BAE@@@QEAAX_K@Z 0000000039a1d3d0 f i CryGameSpySBQR2DLCStore.obj
 0001:0001c450       ??_9CCryGameSpySBQR2SignIn@@$BCI@AA 0000000039a1d450 f i CryGameSpySBQR2SignIn.obj
 0001:0001c450       ??_9CCryGameSpySBQR2DLCStore@@$BCI@AA 0000000039a1d450 f i CryGameSpySBQR2DLCStore.obj
 0001:0001c460       ?StartTaskRunning@CCryGameSpySBQR2DLCStore@@MEAAXI@Z 0000000039a1d460 f   CryGameSpySBQR2DLCStore.obj
 0001:0001c4b0       ?StartOrderSetPaymentMethod@CCryGameSpySBQR2DLCStore@@IEAAXI@Z 0000000039a1d4b0 f   CryGameSpySBQR2DLCStore.obj
 0001:0001c550       ?GetStoreAvailabilityCallback@CCryGameSpySBQR2DLCStore@@KAXHPEAUD2GGetStoreAvailabilityResponse@@PEAX@Z 0000000039a1d550 f   CryGameSpySBQR2DLCStore.obj
 0001:0001c630       ?CountItemsInOrderPurchase@CCryGameSpySBQR2DLCStore@@KAIPEAUD2GOrderPurchase@@@Z 0000000039a1d630 f   CryGameSpySBQR2DLCStore.obj
 0001:0001c6b0       ??4?$_smart_ptr@UIDatagramSocket@@@@QEAAAEAV0@AEBV0@@Z 0000000039a1d6b0 f i CryLobby.obj
 0001:0001c6b0       ??4?$_smart_ptr@VCNameRequest@@@@QEAAAEAV0@AEBV0@@Z 0000000039a1d6b0 f i CryTCPService.obj
 0001:0001c6b0       ??4?$_smart_ptr@VCCryGameSpySBQR2Friends@@@@QEAAAEAV0@AEBV0@@Z 0000000039a1d6b0 f i CryGameSpySBQR2FriendsManagement.obj
 0001:0001c6b0       ??4?$_smart_ptr@USTaskLink@CCryGameSpySBQR2DLCStore@@@@QEAAAEAV0@AEBV0@@Z 0000000039a1d6b0 f i CryGameSpySBQR2DLCStore.obj
 0001:0001c6b0       ??4?$_smart_ptr@USTaskBase@CGameSpySBQR2NATNegotiation@@@@QEAAAEAV0@AEBV0@@Z 0000000039a1d6b0 f i GameSpySBQR2NatNegotiation.obj
 0001:0001c6b0       ??4?$_smart_ptr@USTaskCallbackBase@CGameSpySBQR2GPConnection@@@@QEAAAEAV0@AEBV0@@Z 0000000039a1d6b0 f i GameSpySBQR2GPConnection.obj
 0001:0001c6b0       ??4?$_smart_ptr@USTaskBase@CGameSpySBQR2Sake@@@@QEAAAEAV0@AEBV0@@Z 0000000039a1d6b0 f i GameSpySBQR2Sake.obj
 0001:0001c6b0       ??4?$_smart_ptr@USCryDLCPaymentMethodID@@@@QEAAAEAV0@AEBV0@@Z 0000000039a1d6b0 f i CryDLCStore.obj
 0001:0001c6b0       ??4?$_smart_ptr@USTCPServiceData@@@@QEAAAEAV0@AEBV0@@Z 0000000039a1d6b0 f i CryTCPService.obj
 0001:0001c6b0       ??4?$_smart_ptr@USCrySessionID@@@@QEAAAEAV0@AEBV0@@Z 0000000039a1d6b0 f i CryLobby.obj
 0001:0001c6b0       ??4?$_smart_ptr@USGameSpyKey@CCryGameSpySBQR2MatchMaking@@@@QEAAAEAV0@AEBV0@@Z 0000000039a1d6b0 f i CryGameSpySBQR2MatchMaking.obj
 0001:0001c6b0       ??4?$_smart_ptr@USCryUserID@@@@QEAAAEAV0@AEBV0@@Z 0000000039a1d6b0 f i CryDLCStore.obj
 0001:0001c6b0       ??4?$_smart_ptr@USOrderLink@CCryGameSpySBQR2DLCStore@@@@QEAAAEAV0@AEBV0@@Z 0000000039a1d6b0 f i CryGameSpySBQR2DLCStore.obj
 0001:0001c6b0       ??4?$_smart_ptr@USCryDLCItemID@@@@QEAAAEAV0@AEBV0@@Z 0000000039a1d6b0 f i CryDLCStore.obj
 0001:0001c730       ??1?$CClassJobNoRef6@P6AXIW4ECryLobbyError@@V?$_smart_ptr@USCryDLCDownloadableID@@@@_NIIPEBDPEAX@ZIV2@IIPEAXVCCryGameSpySBQR2DLCStore@@@CWorkQueue@@UEAA@XZ 0000000039a1d730 f i CryGameSpySBQR2DLCStore.obj
 0001:0001c7d0       ??_E?$CClassJob@XVCCryGameSpySBQR2DLCStore@@@CWorkQueue@@UEAAPEAXI@Z 0000000039a1d7d0 f i CryGameSpySBQR2DLCStore.obj
 0001:0001c7d0       ??_E?$CClassJob@XVCCryMatchMaking@@@CWorkQueue@@UEAAPEAXI@Z 0000000039a1d7d0 f i CryMatchMaking.obj
 0001:0001c7d0       ??_G?$CClassJob@XVCCryLobbyService@@@CWorkQueue@@UEAAPEAXI@Z 0000000039a1d7d0 f i CryLobby.obj
 0001:0001c7d0       ??_G?$CClassJob@XVCCryGameSpySBQR2DLCStore@@@CWorkQueue@@UEAAPEAXI@Z 0000000039a1d7d0 f i CryGameSpySBQR2DLCStore.obj
 0001:0001c7d0       ??_G?$CClassJob@XVCCryMatchMaking@@@CWorkQueue@@UEAAPEAXI@Z 0000000039a1d7d0 f i CryMatchMaking.obj
 0001:0001c7d0       ??_E?$CClassJob@XVCCryGameSpySBQR2LobbyService@@@CWorkQueue@@UEAAPEAXI@Z 0000000039a1d7d0 f i CryGameSpySBQR2Lobby.obj
 0001:0001c7d0       ??_G?$CClassJob@XVCCryGameSpySBQR2LobbyService@@@CWorkQueue@@UEAAPEAXI@Z 0000000039a1d7d0 f i CryGameSpySBQR2Lobby.obj
 0001:0001c7d0       ??_E?$CClassJob@XVCCryLobbyService@@@CWorkQueue@@UEAAPEAXI@Z 0000000039a1d7d0 f i CryLobby.obj
 0001:0001c850       ??_G?$CClassJobNoRef6@P6AXIW4ECryLobbyError@@V?$_smart_ptr@USCryDLCDownloadableID@@@@_NIIPEBDPEAX@ZIV2@IIPEAXVCCryGameSpySBQR2DLCStore@@@CWorkQueue@@UEAAPEAXI@Z 0000000039a1d850 f i CryGameSpySBQR2DLCStore.obj
 0001:0001c850       ??_E?$CClassJobNoRef6@P6AXIW4ECryLobbyError@@V?$_smart_ptr@USCryDLCDownloadableID@@@@_NIIPEBDPEAX@ZIV2@IIPEAXVCCryGameSpySBQR2DLCStore@@@CWorkQueue@@UEAAPEAXI@Z 0000000039a1d850 f i CryGameSpySBQR2DLCStore.obj
 0001:0001c880       ?assign@?$Array@V?$_smart_ptr@USCryDLCImageID@@@@HU?$SmallDynStorage@V?$_smart_ptr@USCryDLCImageID@@@@HUStandardAlloc@NAlloc@@@NArray@@@@QEAAXU?$Array@$$CBV?$_smart_ptr@USCryDLCImageID@@@@HU?$ArrayStorage@$$CBV?$_smart_ptr@USCryDLCImageID@@@@H@NArray@@@@@Z 0000000039a1d880 f i CryGameSpySBQR2DLCStore.obj
 0001:0001c880       ?assign@?$Array@V?$_smart_ptr@USCryDLCCategoryID@@@@HU?$SmallDynStorage@V?$_smart_ptr@USCryDLCCategoryID@@@@HUStandardAlloc@NAlloc@@@NArray@@@@QEAAXU?$Array@$$CBV?$_smart_ptr@USCryDLCCategoryID@@@@HU?$ArrayStorage@$$CBV?$_smart_ptr@USCryDLCCategoryID@@@@H@NArray@@@@@Z 0000000039a1d880 f i CryGameSpySBQR2DLCStore.obj
 0001:0001c930       ?alloc@?$AllocPrefix@UStandardAlloc@NAlloc@@@NAlloc@@SAPEAXAEA_K_NHH@Z 0000000039a1d930 f i CryGameSpySBQR2DLCStore.obj
 0001:0001c9e0       ??8SCryGameSpySBQR2DLCPaymentMethodID@@UEAA_NAEBUSCryDLCPaymentMethodID@@@Z 0000000039a1d9e0 f i CryGameSpySBQR2DLCStore.obj
 0001:0001c9e0       ??8SCryGameSpySBQR2DLCDownloadableID@@UEAA_NAEBUSCryDLCDownloadableID@@@Z 0000000039a1d9e0 f i CryGameSpySBQR2DLCStore.obj
 0001:0001c9e0       ??8SCryGameSpySBQR2DLCItemID@@UEAA_NAEBUSCryDLCItemID@@@Z 0000000039a1d9e0 f i CryGameSpySBQR2DLCStore.obj
 0001:0001c9f0       ??0SOrderLink@CCryGameSpySBQR2DLCStore@@QEAA@PEAUSOrder@1@PEAV1@@Z 0000000039a1d9f0 f i CryGameSpySBQR2DLCStore.obj
 0001:0001ca50       ?ClearTask@CCryGameSpySBQR2DLCStore@@MEAAXI@Z 0000000039a1da50 f   CryGameSpySBQR2DLCStore.obj
 0001:0001caf0       ?CountItemsInPurchaseHistory@CCryGameSpySBQR2DLCStore@@KAIPEAUD2GPurchaseHistory@@@Z 0000000039a1daf0 f   CryGameSpySBQR2DLCStore.obj
 0001:0001cbb0       ?DispatchDownloadProgress@CCryGameSpySBQR2DLCStore@@IEAAXP6AXIW4ECryLobbyError@@V?$_smart_ptr@USCryDLCDownloadableID@@@@_NIIPEBDPEAX@ZI1II4@Z 0000000039a1dbb0 f   CryGameSpySBQR2DLCStore.obj
 0001:0001cc70       ?FreeTaskLinkFromCryNetwork@CCryGameSpySBQR2DLCStore@@KAXPEAUSTask@1@@Z 0000000039a1dc70 f   CryGameSpySBQR2DLCStore.obj
 0001:0001cd10       ?CreateOrderLink@CCryGameSpySBQR2DLCStore@@IEAA_NI@Z 0000000039a1dd10 f   CryGameSpySBQR2DLCStore.obj
 0001:0001cda0       ?FreeOrderLinkFromCryNetwork@CCryGameSpySBQR2DLCStore@@KAXPEAUSOrder@1@@Z 0000000039a1dda0 f   CryGameSpySBQR2DLCStore.obj
 0001:0001ce80       ?FreeOrderHandle@CCryGameSpySBQR2DLCStore@@MEAAXI@Z 0000000039a1de80 f   CryGameSpySBQR2DLCStore.obj
 0001:0001cef0       ?ClearOrderHandle@CCryGameSpySBQR2DLCStore@@MEAAXI@Z 0000000039a1def0 f   CryGameSpySBQR2DLCStore.obj
 0001:0001cfa0       ?GetRealDLCItemID@CCryGameSpySBQR2DLCStore@@UEAA?AW4ECryLobbyError@@V?$_smart_ptr@USCryDLCItemID@@@@PEAI@Z 0000000039a1dfa0 f   CryGameSpySBQR2DLCStore.obj
 0001:0001d050       ?set_size@?$SmallDynStorage@V?$_smart_ptr@USCryDLCImageID@@@@HUStandardAlloc@NAlloc@@@NArray@@QEAAXH@Z 0000000039a1e050 f i CryGameSpySBQR2DLCStore.obj
 0001:0001d050       ?set_size@?$SmallDynStorage@V?$_smart_ptr@USCryDLCCategoryID@@@@HUStandardAlloc@NAlloc@@@NArray@@QEAAXH@Z 0000000039a1e050 f i CryGameSpySBQR2DLCStore.obj
 0001:0001d0f0       ??$move_init@V?$_smart_ptr@USCryDLCCategoryID@@@@@NArray@@YAXPEAV?$_smart_ptr@USCryDLCCategoryID@@@@0_K@Z 0000000039a1e0f0 f i CryGameSpySBQR2DLCStore.obj
 0001:0001d0f0       ??$move_init@V?$_smart_ptr@USCryDLCImageID@@@@@NArray@@YAXPEAV?$_smart_ptr@USCryDLCImageID@@@@0_K@Z 0000000039a1e0f0 f i CryGameSpySBQR2DLCStore.obj
 0001:0001d1a0       ?_M_set@?$_Impl_vector@USCryDLCCategoryInfo@@V?$allocator@USCryDLCCategoryInfo@@@stlpmtx_std@@@priv@stlpmtx_std@@AEAAXPEAUSCryDLCCategoryInfo@@00@Z 0000000039a1e1a0 f i CryGameSpySBQR2DLCStore.obj
 0001:0001d1a0       ?_M_set@?$_Impl_vector@V?$_smart_ptr@USTask@CGameSpySBQR2Core@@@@V?$allocator@V?$_smart_ptr@USTask@CGameSpySBQR2Core@@@@@stlpmtx_std@@@priv@stlpmtx_std@@AEAAXPEAV?$_smart_ptr@USTask@CGameSpySBQR2Core@@@@00@Z 0000000039a1e1a0 f i GameSpySBQR2Core.obj
 0001:0001d1a0       ?_M_set@?$_Impl_vector@USCryDLCDownloadableInfo@@V?$allocator@USCryDLCDownloadableInfo@@@stlpmtx_std@@@priv@stlpmtx_std@@AEAAXPEAUSCryDLCDownloadableInfo@@00@Z 0000000039a1e1a0 f i CryDLCStore.obj
 0001:0001d1a0       ?_M_set@?$_Impl_vector@PEAXV?$STLGlobalAllocator@PEAX@stl@@@priv@stlpmtx_std@@AEAAXPEAPEAX00@Z 0000000039a1e1a0 f i CryDLCStore.obj
 0001:0001d1a0       ?_M_set@?$_Impl_vector@V?$_smart_ptr@USTaskLink@CCryGameSpySBQR2DLCStore@@@@V?$allocator@V?$_smart_ptr@USTaskLink@CCryGameSpySBQR2DLCStore@@@@@stlpmtx_std@@@priv@stlpmtx_std@@AEAAXPEAV?$_smart_ptr@USTaskLink@CCryGameSpySBQR2DLCStore@@@@00@Z 0000000039a1e1a0 f i CryGameSpySBQR2DLCStore.obj
 0001:0001d1a0       ?_M_set@?$_Impl_vector@V?$_smart_ptr@USRegisteredLobbyData@CCryGameSpySBQR2MatchMaking@@@@V?$allocator@V?$_smart_ptr@USRegisteredLobbyData@CCryGameSpySBQR2MatchMaking@@@@@stlpmtx_std@@@priv@stlpmtx_std@@AEAAXPEAV?$_smart_ptr@USRegisteredLobbyData@CCryGameSpySBQR2MatchMaking@@@@00@Z 0000000039a1e1a0 f i CryGameSpySBQR2MatchMaking.obj
 0001:0001d1a0       ?_M_set@?$_Impl_vector@USEventCBData@CCryLobby@@V?$allocator@USEventCBData@CCryLobby@@@stlpmtx_std@@@priv@stlpmtx_std@@AEAAXPEAUSEventCBData@CCryLobby@@00@Z 0000000039a1e1a0 f i CryLobby.obj
 0001:0001d1a0       ?_M_set@?$_Impl_vector@V?$_smart_ptr@UICryTCPService@@@@V?$STLGlobalAllocator@V?$_smart_ptr@UICryTCPService@@@@@stl@@@priv@stlpmtx_std@@AEAAXPEAV?$_smart_ptr@UICryTCPService@@@@00@Z 0000000039a1e1a0 f i CryTCPServiceFactory.obj
 0001:0001d1a0       ?_M_set@?$_Impl_vector@V?$_smart_ptr@USTaskBase@CGameSpySBQR2Sake@@@@V?$allocator@V?$_smart_ptr@USTaskBase@CGameSpySBQR2Sake@@@@@stlpmtx_std@@@priv@stlpmtx_std@@AEAAXPEAV?$_smart_ptr@USTaskBase@CGameSpySBQR2Sake@@@@00@Z 0000000039a1e1a0 f i GameSpySBQR2Sake.obj
 0001:0001d1a0       ?_M_set@?$_Impl_vector@USItemQuantity@CCryDLCStore@@V?$allocator@USItemQuantity@CCryDLCStore@@@stlpmtx_std@@@priv@stlpmtx_std@@AEAAXPEAUSItemQuantity@CCryDLCStore@@00@Z 0000000039a1e1a0 f i CryGameSpySBQR2DLCStore.obj
 0001:0001d1a0       ?_M_set@?$_Impl_vector@V?$_smart_ptr@USTaskCallbackBase@CGameSpySBQR2GPConnection@@@@V?$allocator@V?$_smart_ptr@USTaskCallbackBase@CGameSpySBQR2GPConnection@@@@@stlpmtx_std@@@priv@stlpmtx_std@@AEAAXPEAV?$_smart_ptr@USTaskCallbackBase@CGameSpySBQR2GPConnection@@@@00@Z 0000000039a1e1a0 f i GameSpySBQR2GPConnection.obj
 0001:0001d1a0       ?_M_set@?$_Impl_vector@V?$_smart_ptr@USOrderLink@CCryGameSpySBQR2DLCStore@@@@V?$allocator@V?$_smart_ptr@USOrderLink@CCryGameSpySBQR2DLCStore@@@@@stlpmtx_std@@@priv@stlpmtx_std@@AEAAXPEAV?$_smart_ptr@USOrderLink@CCryGameSpySBQR2DLCStore@@@@00@Z 0000000039a1e1a0 f i CryGameSpySBQR2DLCStore.obj
 0001:0001d1a0       ?_M_set@?$_Impl_vector@USCrySessionSearchData@@V?$allocator@USCrySessionSearchData@@@stlpmtx_std@@@priv@stlpmtx_std@@AEAAXPEAUSCrySessionSearchData@@00@Z 0000000039a1e1a0 f i CryGameSpySBQR2MatchMaking.obj
 0001:0001d1a0       ?_M_set@?$_Impl_vector@V?$_smart_ptr@USCallbackBase@CGameSpySBQR2GPConnection@@@@V?$allocator@V?$_smart_ptr@USCallbackBase@CGameSpySBQR2GPConnection@@@@@stlpmtx_std@@@priv@stlpmtx_std@@AEAAXPEAV?$_smart_ptr@USCallbackBase@CGameSpySBQR2GPConnection@@@@00@Z 0000000039a1e1a0 f i GameSpySBQR2GPConnection.obj
 0001:0001d1a0       ?_M_set@?$_Impl_vector@V?$_smart_ptr@USTaskBase@CGameSpySBQR2NATNegotiation@@@@V?$allocator@V?$_smart_ptr@USTaskBase@CGameSpySBQR2NATNegotiation@@@@@stlpmtx_std@@@priv@stlpmtx_std@@AEAAXPEAV?$_smart_ptr@USTaskBase@CGameSpySBQR2NATNegotiation@@@@00@Z 0000000039a1e1a0 f i GameSpySBQR2NatNegotiation.obj
 0001:0001d230       ?Execute@?$CClassJobNoRef@IVCCryGameSpySBQR2DLCStore@@@CWorkQueue@@UEAAXXZ 0000000039a1e230 f i CryGameSpySBQR2DLCStore.obj
 0001:0001d230       ?Execute@?$CClassJobNoRef@IVCCryDLCStore@@@CWorkQueue@@UEAAXXZ 0000000039a1e230 f i CryDLCStore.obj
 0001:0001d260       ?Execute@?$CClassJob@XVCCryGameSpySBQR2DLCStore@@@CWorkQueue@@UEAAXXZ 0000000039a1e260 f i CryGameSpySBQR2DLCStore.obj
 0001:0001d290       ?Execute@?$CClassJobNoRef6@P6AXIW4ECryLobbyError@@V?$_smart_ptr@USCryDLCDownloadableID@@@@_NIIPEBDPEAX@ZIV2@IIPEAXVCCryGameSpySBQR2DLCStore@@@CWorkQueue@@UEAAXXZ 0000000039a1e290 f i CryGameSpySBQR2DLCStore.obj
 0001:0001d300       ?Execute@?$CClassJobNoRef3@PEAUSTaskLink@CCryGameSpySBQR2DLCStore@@IIV2@@CWorkQueue@@UEAAXXZ 0000000039a1e300 f i CryGameSpySBQR2DLCStore.obj
 0001:0001d340       ?_Assign@?$CryStackStringT@D$0BAE@@@QEAAXPEBD_K@Z 0000000039a1e340 f i CryGameSpySBQR2DLCStore.obj
 0001:0001d3e0       ?pop_back@?$DynArray@V?$_smart_ptr@USCryDLCImageID@@@@HU?$SmallDynStorage@V?$_smart_ptr@USCryDLCImageID@@@@HUStandardAlloc@NAlloc@@@NArray@@@@QEAAXH@Z 0000000039a1e3e0 f i CryGameSpySBQR2DLCStore.obj
 0001:0001d3e0       ?pop_back@?$DynArray@V?$_smart_ptr@USCryDLCCategoryID@@@@HU?$SmallDynStorage@V?$_smart_ptr@USCryDLCCategoryID@@@@HUStandardAlloc@NAlloc@@@NArray@@@@QEAAXH@Z 0000000039a1e3e0 f i CryGameSpySBQR2DLCStore.obj
 0001:0001d4a0       ?append@?$CryStringT@_W@@QEAAAEAV1@_K_W@Z 0000000039a1e4a0 f i CryGameSpySBQR2DLCStore.obj
 0001:0001d5b0       ?_Concatenate@?$CryStringT@_W@@IEAAXPEB_W_K01@Z 0000000039a1e5b0 f i CryGameSpySBQR2DLCStore.obj
 0001:0001d670       ?_MakeUnique@?$CryStringT@_W@@IEAAXXZ 0000000039a1e670 f i CryGameSpySBQR2DLCStore.obj
 0001:0001d740       ??_GSOrderLink@CCryGameSpySBQR2DLCStore@@UEAAPEAXI@Z 0000000039a1e740 f i CryGameSpySBQR2DLCStore.obj
 0001:0001d740       ??_ESOrderLink@CCryGameSpySBQR2DLCStore@@UEAAPEAXI@Z 0000000039a1e740 f i CryGameSpySBQR2DLCStore.obj
 0001:0001d7c0       ?StopTaskRunning@CCryGameSpySBQR2DLCStore@@MEAAXI@Z 0000000039a1e7c0 f   CryGameSpySBQR2DLCStore.obj
 0001:0001d800       ?EndCatalogListCategories@CCryGameSpySBQR2DLCStore@@IEAAXI@Z 0000000039a1e800 f   CryGameSpySBQR2DLCStore.obj
 0001:0001d900       ?EndCatalogListItems@CCryGameSpySBQR2DLCStore@@IEAAXI@Z 0000000039a1e900 f   CryGameSpySBQR2DLCStore.obj
 0001:0001da10       ?TickCategoryGetInfo@CCryGameSpySBQR2DLCStore@@IEAAXI@Z 0000000039a1ea10 f   CryGameSpySBQR2DLCStore.obj
 0001:0001db10       ?EndCategoryGetInfo@CCryGameSpySBQR2DLCStore@@IEAAXI@Z 0000000039a1eb10 f   CryGameSpySBQR2DLCStore.obj
 0001:0001db80       ?EndCategoryListItems@CCryGameSpySBQR2DLCStore@@IEAAXI@Z 0000000039a1eb80 f   CryGameSpySBQR2DLCStore.obj
 0001:0001dc80       ?GetCategoryItems@CCryGameSpySBQR2DLCStore@@IEAA?AW4ECryLobbyError@@IPEA_WIIAEAPEAI@Z 0000000039a1ec80 f   CryGameSpySBQR2DLCStore.obj
 0001:0001de00       ?EndItemGetInfo@CCryGameSpySBQR2DLCStore@@IEAAXI@Z 0000000039a1ee00 f   CryGameSpySBQR2DLCStore.obj
 0001:0001de70       ??1SDispatchDownloadCompleteParam@CCryGameSpySBQR2DLCStore@@QEAA@XZ 0000000039a1ee70 f i CryGameSpySBQR2DLCStore.obj
 0001:0001def0       ??0SDispatchDownloadCompleteParam@CCryGameSpySBQR2DLCStore@@QEAA@AEBU01@@Z 0000000039a1eef0 f i CryGameSpySBQR2DLCStore.obj
 0001:0001df70       ?DispatchDownloadComplete@CCryGameSpySBQR2DLCStore@@IEAAXUSDispatchDownloadCompleteParam@1@@Z 0000000039a1ef70 f   CryGameSpySBQR2DLCStore.obj
 0001:0001dfe0       ??8SCryGameSpySBQR2DLCLicense@@UEAA_NAEBUSCryDLCLicense@@@Z 0000000039a1efe0 f i CryGameSpySBQR2DLCStore.obj
 0001:0001e040       ??1SCryGameSpySBQR2DLCLicense@@UEAA@XZ 0000000039a1f040 f i CryGameSpySBQR2DLCStore.obj
 0001:0001e0c0       ?EndOrderListItems@CCryGameSpySBQR2DLCStore@@IEAAXI@Z 0000000039a1f0c0 f   CryGameSpySBQR2DLCStore.obj
 0001:0001e260       ??1SCryDLCOrderInfo@@QEAA@XZ 0000000039a1f260 f i CryGameSpySBQR2DLCStore.obj
 0001:0001e360       ?TickOrderGetItemInfo@CCryGameSpySBQR2DLCStore@@IEAAXI@Z 0000000039a1f360 f   CryGameSpySBQR2DLCStore.obj
 0001:0001e360       ?TickItemGetInfo@CCryGameSpySBQR2DLCStore@@IEAAXI@Z 0000000039a1f360 f   CryGameSpySBQR2DLCStore.obj
 0001:0001e470       ?TickOrderSetPaymentMethod@CCryGameSpySBQR2DLCStore@@IEAAXI@Z 0000000039a1f470 f   CryGameSpySBQR2DLCStore.obj
 0001:0001e500       ??8SCryGameSpySBQR2DLCCategoryID@@UEAA_NAEBUSCryDLCCategoryID@@@Z 0000000039a1f500 f i CryGameSpySBQR2DLCStore.obj
 0001:0001e500       ??8SCryGameSpySBQR2DLCImageID@@UEAA_NAEBUSCryDLCImageID@@@Z 0000000039a1f500 f i CryGameSpySBQR2DLCStore.obj
 0001:0001e530       ?resize_raw@?$SmallDynStorage@V?$_smart_ptr@USCryDLCCategoryID@@@@HUStandardAlloc@NAlloc@@@NArray@@QEAAXHH_N@Z 0000000039a1f530 f i CryGameSpySBQR2DLCStore.obj
 0001:0001e6a0       ?resize_raw@?$SmallDynStorage@V?$_smart_ptr@USCryDLCImageID@@@@HUStandardAlloc@NAlloc@@@NArray@@QEAAXHH_N@Z 0000000039a1f6a0 f i CryGameSpySBQR2DLCStore.obj
 0001:0001e810       ??4?$CryStringT@_W@@QEAAAEAV0@PEB_W@Z 0000000039a1f810 f i CryGameSpySBQR2DLCStore.obj
 0001:0001e860       ??1?$CClassJobNoRef3@PEAUSTaskLink@CCryGameSpySBQR2DLCStore@@HV?$CryStringT@D@@V2@@CWorkQueue@@UEAA@XZ 0000000039a1f860 f i CryGameSpySBQR2DLCStore.obj
 0001:0001e8f0       ?Execute@?$CClassJobNoRef@USDispatchDownloadCompleteParam@CCryGameSpySBQR2DLCStore@@V2@@CWorkQueue@@UEAAXXZ 0000000039a1f8f0 f i CryGameSpySBQR2DLCStore.obj
 0001:0001e940       ?Execute@?$CClassJobNoRef3@PEAUSTaskLink@CCryGameSpySBQR2DLCStore@@HV?$CryStringT@D@@V2@@CWorkQueue@@UEAAXXZ 0000000039a1f940 f i CryGameSpySBQR2DLCStore.obj
 0001:0001e9a0       ??_E?$CClassJobNoRef@USDispatchDownloadCompleteParam@CCryGameSpySBQR2DLCStore@@V2@@CWorkQueue@@UEAAPEAXI@Z 0000000039a1f9a0 f i CryGameSpySBQR2DLCStore.obj
 0001:0001e9a0       ??_G?$CClassJobNoRef@USDispatchDownloadCompleteParam@CCryGameSpySBQR2DLCStore@@V2@@CWorkQueue@@UEAAPEAXI@Z 0000000039a1f9a0 f i CryGameSpySBQR2DLCStore.obj
 0001:0001ea20       ??_E?$CClassJobNoRef3@PEAUSTaskLink@CCryGameSpySBQR2DLCStore@@HV?$CryStringT@D@@V2@@CWorkQueue@@UEAAPEAXI@Z 0000000039a1fa20 f i CryGameSpySBQR2DLCStore.obj
 0001:0001ea20       ??_G?$CClassJobNoRef3@PEAUSTaskLink@CCryGameSpySBQR2DLCStore@@HV?$CryStringT@D@@V2@@CWorkQueue@@UEAAPEAXI@Z 0000000039a1fa20 f i CryGameSpySBQR2DLCStore.obj
 0001:0001ea50       ?_ConcatenateInPlace@?$CryStringT@_W@@IEAAXPEB_W_K@Z 0000000039a1fa50 f i CryGameSpySBQR2DLCStore.obj
 0001:0001eb20       ?erase@?$DynArray@V?$_smart_ptr@USCryDLCImageID@@@@HU?$SmallDynStorage@V?$_smart_ptr@USCryDLCImageID@@@@HUStandardAlloc@NAlloc@@@NArray@@@@QEAAPEAV?$_smart_ptr@USCryDLCImageID@@@@PEAV2@0@Z 0000000039a1fb20 f i CryGameSpySBQR2DLCStore.obj
 0001:0001eb20       ?erase@?$DynArray@V?$_smart_ptr@USCryDLCCategoryID@@@@HU?$SmallDynStorage@V?$_smart_ptr@USCryDLCCategoryID@@@@HUStandardAlloc@NAlloc@@@NArray@@@@QEAAPEAV?$_smart_ptr@USCryDLCCategoryID@@@@PEAV2@0@Z 0000000039a1fb20 f i CryGameSpySBQR2DLCStore.obj
 0001:0001ec00       ??$__copy_backward_ptrs@PEAUSItemQuantity@CCryDLCStore@@PEAU12@@priv@stlpmtx_std@@YAPEAUSItemQuantity@CCryDLCStore@@PEAU23@00AEBU__false_type@1@@Z 0000000039a1fc00 f i CryGameSpySBQR2DLCStore.obj
 0001:0001ecd0       ??$fill@PEAUSItemQuantity@CCryDLCStore@@U12@@stlpmtx_std@@YAXPEAUSItemQuantity@CCryDLCStore@@0AEBU12@@Z 0000000039a1fcd0 f i CryGameSpySBQR2DLCStore.obj
 0001:0001ed80       ??0STaskLink@CCryGameSpySBQR2DLCStore@@QEAA@PEAUSTask@1@PEAV1@PEAVCCryLobby@@@Z 0000000039a1fd80 f i CryGameSpySBQR2DLCStore.obj
 0001:0001ee10       ??1STaskLink@CCryGameSpySBQR2DLCStore@@UEAA@XZ 0000000039a1fe10 f i CryGameSpySBQR2DLCStore.obj
 0001:0001ee90       ??_GSTaskLink@CCryGameSpySBQR2DLCStore@@UEAAPEAXI@Z 0000000039a1fe90 f i CryGameSpySBQR2DLCStore.obj
 0001:0001ee90       ??_ESTaskLink@CCryGameSpySBQR2DLCStore@@UEAAPEAXI@Z 0000000039a1fe90 f i CryGameSpySBQR2DLCStore.obj
 0001:0001eec0       ?TickCategoryListItems@CCryGameSpySBQR2DLCStore@@IEAAXI@Z 0000000039a1fec0 f   CryGameSpySBQR2DLCStore.obj
 0001:0001ef60       ?StartDownloadableIsDownloaded@CCryGameSpySBQR2DLCStore@@IEAAXI@Z 0000000039a1ff60 f   CryGameSpySBQR2DLCStore.obj
 0001:0001f050       ?EndUserDownloadItem@CCryGameSpySBQR2DLCStore@@IEAAXI@Z 0000000039a20050 f   CryGameSpySBQR2DLCStore.obj
 0001:0001f250       ?EndUserRedownloadAllMissingItems@CCryGameSpySBQR2DLCStore@@IEAAXI@Z 0000000039a20250 f   CryGameSpySBQR2DLCStore.obj
 0001:0001f460       ?ReportPurchaseHistory@CCryGameSpySBQR2DLCStore@@IEAAXI@Z 0000000039a20460 f   CryGameSpySBQR2DLCStore.obj
 0001:0001f790       ??_GSCryGameSpySBQR2DLCLicense@@UEAAPEAXI@Z 0000000039a20790 f i CryGameSpySBQR2DLCStore.obj
 0001:0001f790       ??_ESCryGameSpySBQR2DLCLicense@@UEAAPEAXI@Z 0000000039a20790 f i CryGameSpySBQR2DLCStore.obj
 0001:0001f7c0       ??_GSCryGameSpySBQR2DLCImageID@@UEAAPEAXI@Z 0000000039a207c0 f i CryGameSpySBQR2DLCStore.obj
 0001:0001f7c0       ??_ESCryGameSpySBQR2DLCCategoryID@@UEAAPEAXI@Z 0000000039a207c0 f i CryGameSpySBQR2DLCStore.obj
 0001:0001f7c0       ??_GSCryGameSpySBQR2DLCCategoryID@@UEAAPEAXI@Z 0000000039a207c0 f i CryGameSpySBQR2DLCStore.obj
 0001:0001f7c0       ??_ESCryGameSpySBQR2DLCImageID@@UEAAPEAXI@Z 0000000039a207c0 f i CryGameSpySBQR2DLCStore.obj
 0001:0001f830       ?WriteItemsInOrderItemPurchase@CCryGameSpySBQR2DLCStore@@IEAAXPEAUSTask@1@PEAUD2GOrderItemPurchase@@AEAPEAUSPurchaseHistoryItem@1@@Z 0000000039a20830 f   CryGameSpySBQR2DLCStore.obj
 0001:0001fc20       ?CreateTaskLink@CCryGameSpySBQR2DLCStore@@IEAA_NI@Z 0000000039a20c20 f   CryGameSpySBQR2DLCStore.obj
 0001:0001fcd0       ?GetImageNameFromImageID@CCryGameSpySBQR2DLCStore@@UEAA?AW4ECryLobbyError@@V?$_smart_ptr@USCryDLCImageID@@@@PEAV?$CryStringT@_W@@@Z 0000000039a20cd0 f   CryGameSpySBQR2DLCStore.obj
 0001:0001fd50       ?pop_back@?$_Impl_vector@V?$_smart_ptr@USOrderLink@CCryGameSpySBQR2DLCStore@@@@V?$allocator@V?$_smart_ptr@USOrderLink@CCryGameSpySBQR2DLCStore@@@@@stlpmtx_std@@@priv@stlpmtx_std@@QEAAXXZ 0000000039a20d50 f i CryGameSpySBQR2DLCStore.obj
 0001:0001fd50       ?pop_back@?$_Impl_vector@V?$_smart_ptr@USTaskLink@CCryGameSpySBQR2DLCStore@@@@V?$allocator@V?$_smart_ptr@USTaskLink@CCryGameSpySBQR2DLCStore@@@@@stlpmtx_std@@@priv@stlpmtx_std@@QEAAXXZ 0000000039a20d50 f i CryGameSpySBQR2DLCStore.obj
 0001:0001fdd0       ?Format@?$CryStringT@_W@@QEAAAEAV1@PEB_WZZ 0000000039a20dd0 f i CryGameSpySBQR2DLCStore.obj
 0001:0001fe70       ??$__copy@PEAUSCryDLCDownloadableInfo@@PEAU1@_J@priv@stlpmtx_std@@YAPEAUSCryDLCDownloadableInfo@@PEAU2@00AEBUrandom_access_iterator_tag@1@PEA_J@Z 0000000039a20e70 f i CryGameSpySBQR2DLCStore.obj
 0001:0001ff60       ??4?$DynArray@V?$_smart_ptr@USCryDLCCategoryID@@@@HU?$SmallDynStorage@V?$_smart_ptr@USCryDLCCategoryID@@@@HUStandardAlloc@NAlloc@@@NArray@@@@QEAAAEAU0@U?$Array@$$CBV?$_smart_ptr@USCryDLCCategoryID@@@@HU?$ArrayStorage@$$CBV?$_smart_ptr@USCryDLCCategoryID@@@@H@NArray@@@@@Z 0000000039a20f60 f i CryGameSpySBQR2DLCStore.obj
 0001:00020070       ??4?$DynArray@V?$_smart_ptr@USCryDLCImageID@@@@HU?$SmallDynStorage@V?$_smart_ptr@USCryDLCImageID@@@@HUStandardAlloc@NAlloc@@@NArray@@@@QEAAAEAU0@U?$Array@$$CBV?$_smart_ptr@USCryDLCImageID@@@@HU?$ArrayStorage@$$CBV?$_smart_ptr@USCryDLCImageID@@@@H@NArray@@@@@Z 0000000039a21070 f i CryGameSpySBQR2DLCStore.obj
 0001:00020180       ?FreeTask@CCryGameSpySBQR2DLCStore@@MEAAXI@Z 0000000039a21180 f   CryGameSpySBQR2DLCStore.obj
 0001:00020350       ?EnsureD2GInitialised@CCryGameSpySBQR2DLCStore@@IEAA_NI@Z 0000000039a21350 f   CryGameSpySBQR2DLCStore.obj
 0001:000205a0       ?FixCurrencyString@CCryGameSpySBQR2DLCStore@@IEAAXPEA_WAEAV?$CryStringT@_W@@@Z 0000000039a215a0 f   CryGameSpySBQR2DLCStore.obj
 0001:00020760       ?append_raw@?$DynArray@V?$_smart_ptr@USCryDLCCategoryID@@@@HU?$SmallDynStorage@V?$_smart_ptr@USCryDLCCategoryID@@@@HUStandardAlloc@NAlloc@@@NArray@@@@QEAA?AU?$Array@V?$_smart_ptr@USCryDLCCategoryID@@@@HU?$ArrayStorage@V?$_smart_ptr@USCryDLCCategoryID@@@@H@NArray@@@@H@Z 0000000039a21760 f i CryGameSpySBQR2DLCStore.obj
 0001:00020820       ?append_raw@?$DynArray@V?$_smart_ptr@USCryDLCImageID@@@@HU?$SmallDynStorage@V?$_smart_ptr@USCryDLCImageID@@@@HUStandardAlloc@NAlloc@@@NArray@@@@QEAA?AU?$Array@V?$_smart_ptr@USCryDLCImageID@@@@HU?$ArrayStorage@V?$_smart_ptr@USCryDLCImageID@@@@H@NArray@@@@H@Z 0000000039a21820 f i CryGameSpySBQR2DLCStore.obj
 0001:000208e0       ??$__copy_ptrs@PEAUSCryDLCCategoryInfo@@PEAU1@@priv@stlpmtx_std@@YAPEAUSCryDLCCategoryInfo@@PEAU2@00AEBU__false_type@1@@Z 0000000039a218e0 f i CryGameSpySBQR2DLCStore.obj
 0001:000209b0       ??$__uninitialized_fill_n@PEAUSItemQuantity@CCryDLCStore@@_KU12@@priv@stlpmtx_std@@YAPEAUSItemQuantity@CCryDLCStore@@PEAU23@_KAEBU23@@Z 0000000039a219b0 f i CryGameSpySBQR2DLCStore.obj
 0001:00020a30       ??$__uninitialized_fill_n@PEAUSCryDLCCategoryInfo@@_KU1@@priv@stlpmtx_std@@YAPEAUSCryDLCCategoryInfo@@PEAU2@_KAEBU2@@Z 0000000039a21a30 f i CryGameSpySBQR2DLCStore.obj
 0001:00020ad0       ??$__destroy_mv_srcs@V?$reverse_iterator@PEAUSItemQuantity@CCryDLCStore@@@stlpmtx_std@@USItemQuantity@CCryDLCStore@@@stlpmtx_std@@YAXV?$reverse_iterator@PEAUSItemQuantity@CCryDLCStore@@@0@0PEAUSItemQuantity@CCryDLCStore@@@Z 0000000039a21ad0 f i CryGameSpySBQR2DLCStore.obj
 0001:00020ad0       ??$__destroy_range@V?$reverse_iterator@PEAUSItemQuantity@CCryDLCStore@@@stlpmtx_std@@USItemQuantity@CCryDLCStore@@@stlpmtx_std@@YAXV?$reverse_iterator@PEAUSItemQuantity@CCryDLCStore@@@0@0PEAUSItemQuantity@CCryDLCStore@@@Z 0000000039a21ad0 f i CryGameSpySBQR2DLCStore.obj
 0001:00020b50       ??$__ucopy_ptrs@PEAUSCryDLCCategoryInfo@@PEAU1@@priv@stlpmtx_std@@YAPEAUSCryDLCCategoryInfo@@PEAU2@00AEBU__false_type@1@@Z 0000000039a21b50 f i CryGameSpySBQR2DLCStore.obj
 0001:00020bf0       ?RemoveFromVector@SOrderLink@CCryGameSpySBQR2DLCStore@@QEAAXXZ 0000000039a21bf0 f i CryGameSpySBQR2DLCStore.obj
 0001:00020d00       ?RemoveFromVector@STaskLink@CCryGameSpySBQR2DLCStore@@QEAAXXZ 0000000039a21d00 f i CryGameSpySBQR2DLCStore.obj
 0001:00020e10       ?StartCheckAvailability@CCryGameSpySBQR2DLCStore@@IEAAXI@Z 0000000039a21e10 f   CryGameSpySBQR2DLCStore.obj
 0001:00020eb0       ?StartCategoryListItems@CCryGameSpySBQR2DLCStore@@IEAAXI@Z 0000000039a21eb0 f   CryGameSpySBQR2DLCStore.obj
 0001:00020ef0       ?StartUserRedownloadAllMissingItems@CCryGameSpySBQR2DLCStore@@IEAAXI@Z 0000000039a21ef0 f   CryGameSpySBQR2DLCStore.obj
 0001:00020ef0       ?StartUserGetDownloadableAccess@CCryGameSpySBQR2DLCStore@@IEAAXI@Z 0000000039a21ef0 f   CryGameSpySBQR2DLCStore.obj
 0001:00020f40       ?TickOrderFinalize@CCryGameSpySBQR2DLCStore@@IEAAXI@Z 0000000039a21f40 f   CryGameSpySBQR2DLCStore.obj
 0001:00021050       ?EndOrderGetInfo@CCryGameSpySBQR2DLCStore@@IEAAXI@Z 0000000039a22050 f   CryGameSpySBQR2DLCStore.obj
 0001:00021200       ?EndOrderGetItemInfo@CCryGameSpySBQR2DLCStore@@IEAAXI@Z 0000000039a22200 f   CryGameSpySBQR2DLCStore.obj
 0001:00021460       ?WriteItemsInPurchaseHistory@CCryGameSpySBQR2DLCStore@@IEAAXPEAUSTask@1@PEAUD2GPurchaseHistory@@AEAPEAUSPurchaseHistoryItem@1@@Z 0000000039a22460 f   CryGameSpySBQR2DLCStore.obj
 0001:000214f0       ?_M_fill_insert_aux@?$_Impl_vector@USItemQuantity@CCryDLCStore@@V?$allocator@USItemQuantity@CCryDLCStore@@@stlpmtx_std@@@priv@stlpmtx_std@@AEAAXPEAUSItemQuantity@CCryDLCStore@@_KAEBU45@AEBU__false_type@3@@Z 0000000039a224f0 f i CryGameSpySBQR2DLCStore.obj
 0001:00021730       ??$__destroy_range@PEAUSCryDLCCategoryInfo@@U1@@stlpmtx_std@@YAXPEAUSCryDLCCategoryInfo@@00@Z 0000000039a22730 f i CryGameSpySBQR2DLCStore.obj
 0001:000217d0       ??$_Destroy_Moved_Range@V?$reverse_iterator@PEAUSCryDLCCategoryInfo@@@stlpmtx_std@@@stlpmtx_std@@YAXV?$reverse_iterator@PEAUSCryDLCCategoryInfo@@@0@0@Z 0000000039a227d0 f i CryGameSpySBQR2DLCStore.obj
 0001:000217d0       ??$_Destroy_Range@V?$reverse_iterator@PEAUSCryDLCCategoryInfo@@@stlpmtx_std@@@stlpmtx_std@@YAXV?$reverse_iterator@PEAUSCryDLCCategoryInfo@@@0@0@Z 0000000039a227d0 f i CryDLCStore.obj
 0001:00021890       ??0?$DynArray@V?$_smart_ptr@USCryDLCCategoryID@@@@HU?$SmallDynStorage@V?$_smart_ptr@USCryDLCCategoryID@@@@HUStandardAlloc@NAlloc@@@NArray@@@@QEAA@AEBU0@@Z 0000000039a22890 f i CryGameSpySBQR2DLCStore.obj
 0001:00021970       ??0?$DynArray@V?$_smart_ptr@USCryDLCImageID@@@@HU?$SmallDynStorage@V?$_smart_ptr@USCryDLCImageID@@@@HUStandardAlloc@NAlloc@@@NArray@@@@QEAA@AEBU0@@Z 0000000039a22970 f i CryGameSpySBQR2DLCStore.obj
 0001:00021a50       ?EndTask@CCryGameSpySBQR2DLCStore@@MEAAXI@Z 0000000039a22a50 f   CryGameSpySBQR2DLCStore.obj
 0001:00021c90       ??0SCryDLCItemInfo@@QEAA@XZ 0000000039a22c90 f i CryGameSpySBQR2DLCStore.obj
 0001:00021d70       ?GetPurchaseHistoryCallback@CCryGameSpySBQR2DLCStore@@KAXHPEAUD2GGetPurchaseHistoryResponse@@PEAX@Z 0000000039a22d70 f   CryGameSpySBQR2DLCStore.obj
 0001:00021e70       ?GetUserCreditCardsCallback@CCryGameSpySBQR2DLCStore@@KAXHPEAUD2GGetUserCreditCardsResponse@@PEAX@Z 0000000039a22e70 f   CryGameSpySBQR2DLCStore.obj
 0001:00022190       ?GetOrderTotalCallback@CCryGameSpySBQR2DLCStore@@KAXHPEAUD2GGetOrderTotalResponse@@PEAX@Z 0000000039a23190 f   CryGameSpySBQR2DLCStore.obj
 0001:00022260       ?StartOrderCallback@CCryGameSpySBQR2DLCStore@@KAXHPEAUD2GStartOrderResponse@@PEAX@Z 0000000039a23260 f   CryGameSpySBQR2DLCStore.obj
 0001:00022390       ?OrderCompleteCallback@CCryGameSpySBQR2DLCStore@@KAXHPEAUD2GIsOrderCompleteResponse@@PEAX@Z 0000000039a23390 f   CryGameSpySBQR2DLCStore.obj
 0001:00022480       ?DownloadCompleteCallbackHandler@CCryGameSpySBQR2DLCStore@@IEAAXPEAUSTaskLink@1@HV?$CryStringT@D@@@Z 0000000039a23480 f   CryGameSpySBQR2DLCStore.obj
 0001:000225d0       ?_M_insert_overflow_aux@?$_Impl_vector@USItemQuantity@CCryDLCStore@@V?$allocator@USItemQuantity@CCryDLCStore@@@stlpmtx_std@@@priv@stlpmtx_std@@AEAAXPEAUSItemQuantity@CCryDLCStore@@AEBU45@AEBU__false_type@3@_K_N@Z 0000000039a235d0 f i CryGameSpySBQR2DLCStore.obj
 0001:000227f0       ??$__copy@PEAUSCryDLCItemInfo@@PEAU1@_J@priv@stlpmtx_std@@YAPEAUSCryDLCItemInfo@@PEAU2@00AEBUrandom_access_iterator_tag@1@PEA_J@Z 0000000039a237f0 f i CryGameSpySBQR2DLCStore.obj
 0001:00022960       ??0SCryDLCItemInfo@@QEAA@AEBU0@@Z 0000000039a23960 f i CryGameSpySBQR2DLCStore.obj
 0001:00022a30       ?_M_insert_overflow_aux@?$_Impl_vector@USCryDLCCategoryInfo@@V?$allocator@USCryDLCCategoryInfo@@@stlpmtx_std@@@priv@stlpmtx_std@@AEAAXPEAUSCryDLCCategoryInfo@@AEBU4@AEBU__false_type@3@_K_N@Z 0000000039a23a30 f i CryGameSpySBQR2DLCStore.obj
 0001:00022bf0       ??$Add@IVCCryDLCStore@@@CWorkQueue@@QEAAXP8CCryDLCStore@@EAAXI@ZPEAV1@I@Z 0000000039a23bf0 f i CryDLCStore.obj
 0001:00022bf0       ??$Add@IVCCryGameSpySBQR2DLCStore@@@CWorkQueue@@QEAAXP8CCryGameSpySBQR2DLCStore@@EAAXI@ZPEAV1@I@Z 0000000039a23bf0 f i CryGameSpySBQR2DLCStore.obj
 0001:00022cb0       ??$Add@VCCryGameSpySBQR2DLCStore@@@CWorkQueue@@QEAAXP8CCryGameSpySBQR2DLCStore@@EAAXXZPEAV1@@Z 0000000039a23cb0 f i CryGameSpySBQR2DLCStore.obj
 0001:00022d60       ??$Add@USDispatchDownloadCompleteParam@CCryGameSpySBQR2DLCStore@@V2@@CWorkQueue@@QEAAXP8CCryGameSpySBQR2DLCStore@@EAAXUSDispatchDownloadCompleteParam@1@@ZPEAV1@0@Z 0000000039a23d60 f i CryGameSpySBQR2DLCStore.obj
 0001:00022e90       ??$Add@P6AXIW4ECryLobbyError@@V?$_smart_ptr@USCryDLCDownloadableID@@@@_NIIPEBDPEAX@ZIV2@IIPEAXVCCryGameSpySBQR2DLCStore@@@CWorkQueue@@QEAAXP8CCryGameSpySBQR2DLCStore@@EAAXP6AXIW4ECryLobbyError@@V?$_smart_ptr@USCryDLCDownloadableID@@@@_NIIPEBDPEAX@ZI1II4@ZPEAV1@5I1II4@Z 0000000039a23e90 f i CryGameSpySBQR2DLCStore.obj
 0001:00023040       ??$Add@PEAUSTaskLink@CCryGameSpySBQR2DLCStore@@IIV2@@CWorkQueue@@QEAAXP8CCryGameSpySBQR2DLCStore@@EAAXPEAUSTaskLink@1@II@ZPEAV1@0II@Z 0000000039a24040 f i CryGameSpySBQR2DLCStore.obj
 0001:00023120       ??$Add@PEAUSTaskLink@CCryGameSpySBQR2DLCStore@@HV?$CryStringT@D@@V2@@CWorkQueue@@QEAAXP8CCryGameSpySBQR2DLCStore@@EAAXPEAUSTaskLink@1@HV?$CryStringT@D@@@ZPEAV1@0H1@Z 0000000039a24120 f i CryGameSpySBQR2DLCStore.obj
 0001:000232b0       ??1SOrder@CCryDLCStore@@QEAA@XZ 0000000039a242b0 f i CryGameSpySBQR2DLCStore.obj
 0001:00023380       ?CheckAvailability@CCryGameSpySBQR2DLCStore@@UEAA?AW4ECryLobbyError@@UCryUserID@@PEAIP6AXIW42@W4ECryDLCStoreStatus@@PEAX@Z4@Z 0000000039a24380 f   CryGameSpySBQR2DLCStore.obj
 0001:000234f0       ?CatalogListCategories@CCryGameSpySBQR2DLCStore@@UEAA?AW4ECryLobbyError@@PEAIP6AXIW42@PEAUSCryDLCCategoryInfo@@PEAX@Z3@Z 0000000039a244f0 f   CryGameSpySBQR2DLCStore.obj
 0001:00023610       ?CatalogListItems@CCryGameSpySBQR2DLCStore@@UEAA?AW4ECryLobbyError@@PEAIP6AXIW42@PEAUSCryDLCItemInfo@@PEAX@Z3@Z 0000000039a24610 f   CryGameSpySBQR2DLCStore.obj
 0001:00023730       ?CategoryGetInfo@CCryGameSpySBQR2DLCStore@@UEAA?AW4ECryLobbyError@@V?$_smart_ptr@USCryDLCCategoryID@@@@PEAIP6AXIW42@PEAUSCryDLCCategoryInfo@@PEAX@Z4@Z 0000000039a24730 f   CryGameSpySBQR2DLCStore.obj
 0001:00023920       ?CategoryListItems@CCryGameSpySBQR2DLCStore@@UEAA?AW4ECryLobbyError@@V?$_smart_ptr@USCryDLCCategoryID@@@@PEAIP6AXIW42@PEAUSCryDLCItemInfo@@PEAX@Z4@Z 0000000039a24920 f   CryGameSpySBQR2DLCStore.obj
 0001:00023ae0       ?ItemGetInfo@CCryGameSpySBQR2DLCStore@@UEAA?AW4ECryLobbyError@@V?$_smart_ptr@USCryDLCItemID@@@@PEAIP6AXIW42@PEAUSCryDLCItemInfo@@PEAX@Z4@Z 0000000039a24ae0 f   CryGameSpySBQR2DLCStore.obj
 0001:00023cb0       ?DownloadableIsDownloaded@CCryGameSpySBQR2DLCStore@@UEAA?AW4ECryLobbyError@@V?$_smart_ptr@USCryDLCDownloadableID@@@@PEBDPEAIP6AXIW42@_NPEAX@Z5@Z 0000000039a24cb0 f   CryGameSpySBQR2DLCStore.obj
 0001:00023de0       ?UserGetPurchaseHistory@CCryGameSpySBQR2DLCStore@@UEAA?AW4ECryLobbyError@@UCryUserID@@PEAIP6AXIW42@V?$_smart_ptr@USCryDLCItemID@@@@V?$_smart_ptr@USCryDLCDownloadableID@@@@V?$_smart_ptr@USCryDLCLicense@@@@PEAX@Z6@Z 0000000039a24de0 f   CryGameSpySBQR2DLCStore.obj
 0001:00023fb0       ?UserStartOrder@CCryGameSpySBQR2DLCStore@@UEAA?AW4ECryLobbyError@@UCryUserID@@PEAI1P6AXIW42@PEAX@Z3@Z 0000000039a24fb0 f   CryGameSpySBQR2DLCStore.obj
 0001:00024160       ?UserGetDownloadableAccess@CCryGameSpySBQR2DLCStore@@UEAA?AW4ECryLobbyError@@UCryUserID@@V?$_smart_ptr@USCryDLCDownloadableID@@@@PEAIP6AXIW42@W4EDownloadableAccess@@PEAX@Z5@Z 0000000039a25160 f   CryGameSpySBQR2DLCStore.obj
 0001:00024340       ?UserDownloadItem@CCryGameSpySBQR2DLCStore@@UEAA?AW4ECryLobbyError@@UCryUserID@@V?$_smart_ptr@USCryDLCDownloadableID@@@@PEAIP6AXIW42@1_NIIPEBDPEAX@Z6@Z 0000000039a25340 f   CryGameSpySBQR2DLCStore.obj
 0001:00024520       ?UserCancelActiveDownload@CCryGameSpySBQR2DLCStore@@UEAA?AW4ECryLobbyError@@UCryUserID@@@Z 0000000039a25520 f   CryGameSpySBQR2DLCStore.obj
 0001:000245d0       ?UserRedownloadAllMissingItems@CCryGameSpySBQR2DLCStore@@UEAA?AW4ECryLobbyError@@UCryUserID@@PEAIP6AXIW42@V?$_smart_ptr@USCryDLCDownloadableID@@@@_NIIPEBDPEAX@Z6@Z 0000000039a255d0 f   CryGameSpySBQR2DLCStore.obj
 0001:00024790       ?TickUserRedownloadAllMissingItems@CCryGameSpySBQR2DLCStore@@IEAAXI@Z 0000000039a25790 f   CryGameSpySBQR2DLCStore.obj
 0001:00024a80       ?UserListPaymentMethods@CCryGameSpySBQR2DLCStore@@UEAA?AW4ECryLobbyError@@UCryUserID@@PEAIP6AXIW42@PEAUSCryDLCPaymentMethodInfo@@PEAX@Z4@Z 0000000039a25a80 f   CryGameSpySBQR2DLCStore.obj
 0001:00024c00       ?OrderFinalize@CCryGameSpySBQR2DLCStore@@UEAA?AW4ECryLobbyError@@I_NPEAIP6AXIW42@V?$_smart_ptr@USCryDLCItemID@@@@V?$_smart_ptr@USCryDLCDownloadableID@@@@V?$_smart_ptr@USCryDLCLicense@@@@PEAX@Z6@Z 0000000039a25c00 f   CryGameSpySBQR2DLCStore.obj
 0001:00024d40       ?OrderAddItem@CCryGameSpySBQR2DLCStore@@UEAA?AW4ECryLobbyError@@IV?$_smart_ptr@USCryDLCItemID@@@@PEAIP6AXIW42@PEAX@Z3@Z 0000000039a25d40 f   CryGameSpySBQR2DLCStore.obj
 0001:00024ee0       ?OrderRemoveItem@CCryGameSpySBQR2DLCStore@@UEAA?AW4ECryLobbyError@@IV?$_smart_ptr@USCryDLCItemID@@@@PEAIP6AXIW42@PEAX@Z3@Z 0000000039a25ee0 f   CryGameSpySBQR2DLCStore.obj
 0001:00025080       ?OrderAddItemQuantity@CCryGameSpySBQR2DLCStore@@UEAA?AW4ECryLobbyError@@IV?$_smart_ptr@USCryDLCItemID@@@@IPEAIP6AXIW42@PEAX@Z3@Z 0000000039a26080 f   CryGameSpySBQR2DLCStore.obj
 0001:00025210       ?OrderRemoveItemQuantity@CCryGameSpySBQR2DLCStore@@UEAA?AW4ECryLobbyError@@IV?$_smart_ptr@USCryDLCItemID@@@@IPEAIP6AXIW42@PEAX@Z3@Z 0000000039a26210 f   CryGameSpySBQR2DLCStore.obj
 0001:000253a0       ?OrderListItems@CCryGameSpySBQR2DLCStore@@UEAA?AW4ECryLobbyError@@IPEAIP6AXIW42@V?$_smart_ptr@USCryDLCItemID@@@@IPEAX@Z3@Z 0000000039a263a0 f   CryGameSpySBQR2DLCStore.obj
 0001:00025480       ?OrderGetInfo@CCryGameSpySBQR2DLCStore@@UEAA?AW4ECryLobbyError@@IPEAIP6AXIW42@PEAUSCryDLCOrderInfo@@PEAX@Z3@Z 0000000039a26480 f   CryGameSpySBQR2DLCStore.obj
 0001:00025560       ?OrderGetItemInfo@CCryGameSpySBQR2DLCStore@@UEAA?AW4ECryLobbyError@@IV?$_smart_ptr@USCryDLCItemID@@@@PEAIP6AXIW42@PEAUSCryDLCItemInfo@@PEAUSCryDLCOrderItemInfo@@PEAX@Z5@Z 0000000039a26560 f   CryGameSpySBQR2DLCStore.obj
 0001:00025760       ?OrderSetPaymentMethod@CCryGameSpySBQR2DLCStore@@UEAA?AW4ECryLobbyError@@IVCryDLCPaymentMethodID@@PEAIP6AXIW42@PEAX@Z3@Z 0000000039a26760 f   CryGameSpySBQR2DLCStore.obj
 0001:00025920       ?OrderCancel@CCryGameSpySBQR2DLCStore@@UEAA?AW4ECryLobbyError@@IPEAIP6AXIW42@PEAX@Z2@Z 0000000039a26920 f   CryGameSpySBQR2DLCStore.obj
 0001:00025a00       ?OrderFree@CCryGameSpySBQR2DLCStore@@UEAA?AW4ECryLobbyError@@IPEAIP6AXIW42@PEAX@Z2@Z 0000000039a26a00 f   CryGameSpySBQR2DLCStore.obj
 0001:00025ae0       ?ReleaseCatalog@CCryGameSpySBQR2DLCStore@@UEAA?AW4ECryLobbyError@@PEAIP6AXIW42@PEAX@Z2@Z 0000000039a26ae0 f   CryGameSpySBQR2DLCStore.obj
 0001:00025c40       ?DownloadProgressCallbackHandler@CCryGameSpySBQR2DLCStore@@IEAAXPEAUSTaskLink@1@II@Z 0000000039a26c40 f   CryGameSpySBQR2DLCStore.obj
 0001:00025d50       ?DownloadProgressCallback@CCryGameSpySBQR2DLCStore@@KAXIIPEAX@Z 0000000039a26d50 f   CryGameSpySBQR2DLCStore.obj
 0001:00025e00       ?DownloadCompleteCallback@CCryGameSpySBQR2DLCStore@@KAXHPEAD0PEAX@Z 0000000039a26e00 f   CryGameSpySBQR2DLCStore.obj
 0001:00025eb0       ?erase@?$_Impl_vector@USCryDLCCategoryInfo@@V?$allocator@USCryDLCCategoryInfo@@@stlpmtx_std@@@priv@stlpmtx_std@@QEAAPEAUSCryDLCCategoryInfo@@PEAU4@0@Z 0000000039a26eb0 f i CryGameSpySBQR2DLCStore.obj
 0001:00025f40       ?erase@?$_Impl_vector@USCryDLCDownloadableInfo@@V?$allocator@USCryDLCDownloadableInfo@@@stlpmtx_std@@@priv@stlpmtx_std@@QEAAPEAUSCryDLCDownloadableInfo@@PEAU4@0@Z 0000000039a26f40 f i CryGameSpySBQR2DLCStore.obj
 0001:00025ff0       ?AddToVector@SOrderLink@CCryGameSpySBQR2DLCStore@@QEAAXAEAV?$vector@V?$_smart_ptr@USOrderLink@CCryGameSpySBQR2DLCStore@@@@V?$allocator@V?$_smart_ptr@USOrderLink@CCryGameSpySBQR2DLCStore@@@@@stlpmtx_std@@@stlpmtx_std@@@Z 0000000039a26ff0 f i CryGameSpySBQR2DLCStore.obj
 0001:000260c0       ?AddToVector@STaskLink@CCryGameSpySBQR2DLCStore@@QEAAXAEAV?$vector@V?$_smart_ptr@USTaskLink@CCryGameSpySBQR2DLCStore@@@@V?$allocator@V?$_smart_ptr@USTaskLink@CCryGameSpySBQR2DLCStore@@@@@stlpmtx_std@@@stlpmtx_std@@@Z 0000000039a270c0 f i CryGameSpySBQR2DLCStore.obj
 0001:000261a0       ?PassOrderLinkToGameSpy@CCryGameSpySBQR2DLCStore@@IEAAXI@Z 0000000039a271a0 f   CryGameSpySBQR2DLCStore.obj
 0001:000261d0       ?push_back@?$_Impl_vector@USCryDLCCategoryInfo@@V?$allocator@USCryDLCCategoryInfo@@@stlpmtx_std@@@priv@stlpmtx_std@@QEAAXAEBUSCryDLCCategoryInfo@@@Z 0000000039a271d0 f i CryGameSpySBQR2DLCStore.obj
 0001:00026290       ?TickUserGetPurchaseHistory@CCryGameSpySBQR2DLCStore@@IEAAXI@Z 0000000039a27290 f   CryGameSpySBQR2DLCStore.obj
 0001:00026360       ?TickUserDownloadItem@CCryGameSpySBQR2DLCStore@@IEAAXI@Z 0000000039a27360 f   CryGameSpySBQR2DLCStore.obj
 0001:00026520       ?StartUserListPaymentMethods@CCryGameSpySBQR2DLCStore@@IEAAXI@Z 0000000039a27520 f   CryGameSpySBQR2DLCStore.obj
 0001:000265e0       ?StartOrderFinalize@CCryGameSpySBQR2DLCStore@@IEAAXI@Z 0000000039a275e0 f   CryGameSpySBQR2DLCStore.obj
 0001:00026710       ?TickGetOrderTotal@CCryGameSpySBQR2DLCStore@@IEAAXI@Z 0000000039a27710 f   CryGameSpySBQR2DLCStore.obj
 0001:00026a10       ?TickOrderAdjustItemQuantity@CCryGameSpySBQR2DLCStore@@IEAAXI@Z 0000000039a27a10 f   CryGameSpySBQR2DLCStore.obj
 0001:00026da0       ?erase@?$_Impl_vector@USCryDLCItemInfo@@V?$allocator@USCryDLCItemInfo@@@stlpmtx_std@@@priv@stlpmtx_std@@QEAAPEAUSCryDLCItemInfo@@PEAU4@0@Z 0000000039a27da0 f i CryGameSpySBQR2DLCStore.obj
 0001:00026e50       ??0CCryGameSpySBQR2DLCStore@@QEAA@PEAVCCryLobby@@PEAVCCryLobbyService@@@Z 0000000039a27e50 f   CryGameSpySBQR2DLCStore.obj
 0001:000270f0       ??1CCryGameSpySBQR2DLCStore@@UEAA@XZ 0000000039a280f0 f i CryGameSpySBQR2DLCStore.obj
 0001:000272a0       ??_ECCryGameSpySBQR2DLCStore@@UEAAPEAXI@Z 0000000039a282a0 f i CryGameSpySBQR2DLCStore.obj
 0001:000272a0       ??_GCCryGameSpySBQR2DLCStore@@UEAAPEAXI@Z 0000000039a282a0 f i CryGameSpySBQR2DLCStore.obj
 0001:000272d0       ?TickReleaseCatalog@CCryGameSpySBQR2DLCStore@@IEAAXI@Z 0000000039a282d0 f   CryGameSpySBQR2DLCStore.obj
 0001:000273d0       ?LoadCatalogItemsCallback@CCryGameSpySBQR2DLCStore@@KAXHPEAUD2GLoadCatalogItemsResponse@@PEAX@Z 0000000039a283d0 f   CryGameSpySBQR2DLCStore.obj
 0001:00028380       ?TickRefreshCatalog@CCryGameSpySBQR2DLCStore@@IEAAXI@Z 0000000039a29380 f   CryGameSpySBQR2DLCStore.obj
 0001:000284a0       ?Tick@CCryGameSpySBQR2DLCStore@@UEAAXVCTimeValue@@@Z 0000000039a294a0 f   CryGameSpySBQR2DLCStore.obj
 0001:000289a0       ?_Rotate_left@?$_Rb_global@_N@priv@stlpmtx_std@@SAXPEAU_Rb_tree_node_base@23@AEAPEAU423@@Z 0000000039a299a0 f i CryGameSpySBQR2Friends.obj
 0001:00028a00       ?_Rotate_right@?$_Rb_global@_N@priv@stlpmtx_std@@SAXPEAU_Rb_tree_node_base@23@AEAPEAU423@@Z 0000000039a29a00 f i CryGameSpySBQR2Friends.obj
 0001:00028a60       ?Terminate@CCryGameSpySBQR2Friends@@UEAA?AW4ECryLobbyError@@XZ 0000000039a29a60 f   CryGameSpySBQR2Friends.obj
 0001:00028a80       ?StartTaskRunning@CCryGameSpySBQR2Friends@@AEAAXI@Z 0000000039a29a80 f   CryGameSpySBQR2Friends.obj
 0001:00028ae0       ?_Rebalance@?$_Rb_global@_N@priv@stlpmtx_std@@SAXPEAU_Rb_tree_node_base@23@AEAPEAU423@@Z 0000000039a29ae0 f i CryGameSpySBQR2Friends.obj
 0001:00028cd0       ?_AllocData@?$CryStackStringT@D$0CA@@@QEAAX_K@Z 0000000039a29cd0 f i CryGameSpySBQR2Friends.obj
 0001:00028d50       ?_Assign@?$CryStackStringT@D$0CA@@@QEAAXPEBD_K@Z 0000000039a29d50 f i CryGameSpySBQR2Friends.obj
 0001:00028df0       ?_AllocData@?$CryStackStringT@D$0CI@@@QEAAX_K@Z 0000000039a29df0 f i CryGameSpySBQR2Friends.obj
 0001:00028e70       ??1?$_Deque_base@V?$_smart_ptr@USTCPServiceData@@@@V?$allocator@V?$_smart_ptr@USTCPServiceData@@@@@stlpmtx_std@@@priv@stlpmtx_std@@QEAA@XZ 0000000039a29e70 f i CryTCPService.obj
 0001:00028e70       ??1?$_Deque_base@USBannedUser@@V?$allocator@USBannedUser@@@stlpmtx_std@@@priv@stlpmtx_std@@QEAA@XZ 0000000039a29e70 f i CryMatchMaking.obj
 0001:00028e70       ??1?$_Deque_base@HV?$allocator@H@stlpmtx_std@@@priv@stlpmtx_std@@QEAA@XZ 0000000039a29e70 f i CryGameSpySBQR2Friends.obj
 0001:00028ee0       ?Execute@?$CClassJobNoRef@IVCCryGameSpySBQR2Friends@@@CWorkQueue@@UEAAXXZ 0000000039a29ee0 f i CryGameSpySBQR2Friends.obj
 0001:00028f10       ?Execute@?$CClassJobNoRef2@HW4EOnlineState@@VCCryGameSpySBQR2Friends@@@CWorkQueue@@UEAAXXZ 0000000039a29f10 f i CryGameSpySBQR2Friends.obj
 0001:00028f10       ?Execute@?$CClassJobNoRef2@W4ECryLobbySystemEvent@@HVCCryGameSpySBQR2Friends@@@CWorkQueue@@UEAAXXZ 0000000039a29f10 f i CryGameSpySBQR2Friends.obj
 0001:00028f40       ??8SCryGameSpySBQR2UserID@@UEBA_NAEBUSCryUserID@@@Z 0000000039a29f40 f i CryGameSpySBQR2Friends.obj
 0001:00028f50       ??MSCryGameSpySBQR2UserID@@UEBA_NAEBUSCryUserID@@@Z 0000000039a29f50 f i CryGameSpySBQR2Friends.obj
 0001:00028f60       ??_ESCryLANSessionID@@UEAAPEAXI@Z 0000000039a29f60 f i CryLANMatchMaking.obj
 0001:00028f60       ??_GSCryGameSpySBQR2SessionID@@UEAAPEAXI@Z 0000000039a29f60 f i CryGameSpySBQR2FriendsManagement.obj
 0001:00028f60       ??_GSCryLANSessionID@@UEAAPEAXI@Z 0000000039a29f60 f i CryLANMatchMaking.obj
 0001:00028f60       ??_GSCryGameSpySBQR2UserID@@UEAAPEAXI@Z 0000000039a29f60 f i CryGameSpySBQR2Friends.obj
 0001:00028f60       ??_GSCryLANUserID@@UEAAPEAXI@Z 0000000039a29f60 f i CryLANMatchMaking.obj
 0001:00028f60       ??_ESCryGameSpySBQR2UserID@@UEAAPEAXI@Z 0000000039a29f60 f i CryGameSpySBQR2Friends.obj
 0001:00028f60       ??_ESCryLANUserID@@UEAAPEAXI@Z 0000000039a29f60 f i CryLANMatchMaking.obj
 0001:00028f60       ??_ESCryGameSpySBQR2SessionID@@UEAAPEAXI@Z 0000000039a29f60 f i CryGameSpySBQR2FriendsManagement.obj
 0001:00028fa0       ?CreateTaskLink@CCryGameSpySBQR2Friends@@AEAA?AW4ECryLobbyError@@I@Z 0000000039a29fa0 f   CryGameSpySBQR2Friends.obj
 0001:00029050       ?FreeTask@CCryGameSpySBQR2Friends@@MEAAXI@Z 0000000039a2a050 f   CryGameSpySBQR2Friends.obj
 0001:00029110       ?DispatchFriendIDEvent@CCryGameSpySBQR2Friends@@AEAAXW4ECryLobbySystemEvent@@H@Z 0000000039a2a110 f   CryGameSpySBQR2Friends.obj
 0001:00029270       ?GetFriendCountInSession@CCryGameSpySBQR2Friends@@QEAAIPEBD@Z 0000000039a2a270 f   CryGameSpySBQR2Friends.obj
 0001:00029340       ?Format@?$CryStackStringT@D$0BAA@@@QEAAAEAV1@PEBDZZ 0000000039a2a340 f i CryGameSpySBQR2Friends.obj
 0001:00029430       ?_M_initialize_map@?$_Deque_base@HV?$allocator@H@stlpmtx_std@@@priv@stlpmtx_std@@IEAAX_K@Z 0000000039a2a430 f i CryGameSpySBQR2Friends.obj
 0001:00029550       ?GetInviteSessionID@CCryGameSpySBQR2Friends@@QEAA_KH@Z 0000000039a2a550 f   CryGameSpySBQR2Friends.obj
 0001:000296b0       ??1SGameSpyProfile@CCryGameSpySBQR2Friends@@QEAA@XZ 0000000039a2a6b0 f i CryGameSpySBQR2Friends.obj
 0001:000297c0       ?StartFriendsSendGameInvite@CCryGameSpySBQR2Friends@@AEAAXI@Z 0000000039a2a7c0 f   CryGameSpySBQR2Friends.obj
 0001:00029970       ?GPGetInfoCallback@CCryGameSpySBQR2Friends@@CAXPEAVCGameSpySBQR2GPConnection@@USResult@2@PEAUGPGetInfoResponseArg@@PEAUIGameSpyLink@@@Z 0000000039a2a970 f   CryGameSpySBQR2Friends.obj
 0001:00029af0       ?GetFriendStatus@CCryGameSpySBQR2Friends@@QEAA?AW4ECryLobbyError@@HPEAUSFriendStatusInfo@@@Z 0000000039a2aaf0 f   CryGameSpySBQR2Friends.obj
 0001:00029d40       ??0SGameSpyProfile@CCryGameSpySBQR2Friends@@QEAA@AEBU01@@Z 0000000039a2ad40 f i CryGameSpySBQR2Friends.obj
 0001:00029eb0       ?EndFriendsGetFriendsList@CCryGameSpySBQR2Friends@@AEAAXI@Z 0000000039a2aeb0 f   CryGameSpySBQR2Friends.obj
 0001:0002a350       ?DispatchProfileOnlineStatus@CCryGameSpySBQR2Friends@@AEAAXHW4EOnlineState@@@Z 0000000039a2b350 f   CryGameSpySBQR2Friends.obj
 0001:0002a4d0       ?Format@?$CryStackStringT@D$0CI@@@QEAAAEAV1@PEBDZZ 0000000039a2b4d0 f i CryGameSpySBQR2Friends.obj
 0001:0002a5c0       ?_M_push_back_aux_v@?$_Impl_deque@HV?$allocator@H@stlpmtx_std@@@priv@stlpmtx_std@@IEAAXAEBH@Z 0000000039a2b5c0 f i CryGameSpySBQR2Friends.obj
 0001:0002a640       ?GetGUIDAsString@SCryGameSpySBQR2UserID@@UEBA?AV?$CryFixedStringT@$0CI@@@XZ 0000000039a2b640 f i CryGameSpySBQR2Friends.obj
 0001:0002a680       ?_M_erase@?$_Rb_tree@HU?$less@H@stlpmtx_std@@U?$pair@$$CBHUSGameSpyProfile@CCryGameSpySBQR2Friends@@@2@U?$_Select1st@U?$pair@$$CBHUSGameSpyProfile@CCryGameSpySBQR2Friends@@@stlpmtx_std@@@priv@2@U?$_MapTraitsT@U?$pair@$$CBHUSGameSpyProfile@CCryGameSpySBQR2Friends@@@stlpmtx_std@@@52@V?$allocator@U?$pair@$$CBHUSGameSpyProfile@CCryGameSpySBQR2Friends@@@stlpmtx_std@@@2@@priv@stlpmtx_std@@AEAAXPEAU_Rb_tree_node_base@23@@Z 0000000039a2b680 f i CryGameSpySBQR2Friends.obj
 0001:0002a6e0       ?_M_create_node@?$_Rb_tree@HU?$less@H@stlpmtx_std@@U?$pair@$$CBHUSGameSpyProfile@CCryGameSpySBQR2Friends@@@2@U?$_Select1st@U?$pair@$$CBHUSGameSpyProfile@CCryGameSpySBQR2Friends@@@stlpmtx_std@@@priv@2@U?$_MapTraitsT@U?$pair@$$CBHUSGameSpyProfile@CCryGameSpySBQR2Friends@@@stlpmtx_std@@@52@V?$allocator@U?$pair@$$CBHUSGameSpyProfile@CCryGameSpySBQR2Friends@@@stlpmtx_std@@@2@@priv@stlpmtx_std@@IEAAPEAU_Rb_tree_node_base@23@AEBU?$pair@$$CBHUSGameSpyProfile@CCryGameSpySBQR2Friends@@@3@@Z 0000000039a2b6e0 f i CryGameSpySBQR2Friends.obj
 0001:0002a760       ?clear@?$_Rb_tree@HU?$less@H@stlpmtx_std@@U?$pair@$$CBHUSGameSpyProfile@CCryGameSpySBQR2Friends@@@2@U?$_Select1st@U?$pair@$$CBHUSGameSpyProfile@CCryGameSpySBQR2Friends@@@stlpmtx_std@@@priv@2@U?$_MapTraitsT@U?$pair@$$CBHUSGameSpyProfile@CCryGameSpySBQR2Friends@@@stlpmtx_std@@@52@V?$allocator@U?$pair@$$CBHUSGameSpyProfile@CCryGameSpySBQR2Friends@@@stlpmtx_std@@@2@@priv@stlpmtx_std@@QEAAXXZ 0000000039a2b760 f i CryGameSpySBQR2Friends.obj
 0001:0002a7d0       ??$Add@IVCCryGameSpySBQR2Friends@@@CWorkQueue@@QEAAXP8CCryGameSpySBQR2Friends@@EAAXI@ZPEAV1@I@Z 0000000039a2b7d0 f i CryGameSpySBQR2Friends.obj
 0001:0002a890       ??$Add@HW4EOnlineState@@VCCryGameSpySBQR2Friends@@@CWorkQueue@@QEAAXP8CCryGameSpySBQR2Friends@@EAAXHW4EOnlineState@@@ZPEAV1@H0@Z 0000000039a2b890 f i CryGameSpySBQR2Friends.obj
 0001:0002a890       ??$Add@W4ECryLobbySystemEvent@@HVCCryGameSpySBQR2Friends@@@CWorkQueue@@QEAAXP8CCryGameSpySBQR2Friends@@EAAXW4ECryLobbySystemEvent@@H@ZPEAV1@0H@Z 0000000039a2b890 f i CryGameSpySBQR2Friends.obj
 0001:0002a960       ?_M_insert@?$_Rb_tree@HU?$less@H@stlpmtx_std@@U?$pair@$$CBHUSGameSpyProfile@CCryGameSpySBQR2Friends@@@2@U?$_Select1st@U?$pair@$$CBHUSGameSpyProfile@CCryGameSpySBQR2Friends@@@stlpmtx_std@@@priv@2@U?$_MapTraitsT@U?$pair@$$CBHUSGameSpyProfile@CCryGameSpySBQR2Friends@@@stlpmtx_std@@@52@V?$allocator@U?$pair@$$CBHUSGameSpyProfile@CCryGameSpySBQR2Friends@@@stlpmtx_std@@@2@@priv@stlpmtx_std@@AEAA?AU?$_Rb_tree_iterator@U?$pair@$$CBHUSGameSpyProfile@CCryGameSpySBQR2Friends@@@stlpmtx_std@@U?$_MapTraitsT@U?$pair@$$CBHUSGameSpyProfile@CCryGameSpySBQR2Friends@@@stlpmtx_std@@@priv@2@@23@PEAU_Rb_tree_node_base@23@AEBU?$pair@$$CBHUSGameSpyProfile@CCryGameSpySBQR2Friends@@@3@00@Z 0000000039a2b960 f i CryGameSpySBQR2Friends.obj
 0001:0002aa20       ?FriendsGetFriendsList@CCryGameSpySBQR2Friends@@UEAA?AW4ECryLobbyError@@IIIPEAIP6AXIW42@PEAUSFriendInfo@@IPEAX@Z3@Z 0000000039a2ba20 f   CryGameSpySBQR2Friends.obj
 0001:0002ab80       ?FriendsGetNamesList@CCryGameSpySBQR2Friends@@QEAA?AW4ECryLobbyError@@IPEAUCryUserID@@IPEAIP6AXIW42@PEAUSFriendInfo@@IPEAX@Z4@Z 0000000039a2bb80 f   CryGameSpySBQR2Friends.obj
 0001:0002ad90       ?FriendsSendGameInvite@CCryGameSpySBQR2Friends@@UEAA?AW4ECryLobbyError@@IIPEAUCryUserID@@IPEAIP6AXIW42@PEAX@Z3@Z 0000000039a2bd90 f   CryGameSpySBQR2Friends.obj
 0001:0002afb0       ?GPRecvBuddyRevokeCallback@CCryGameSpySBQR2Friends@@CAXPEAVCGameSpySBQR2GPConnection@@USResult@2@PEAUGPRecvBuddyRevokeArg@@PEAUIGameSpyLink@@@Z 0000000039a2bfb0 f   CryGameSpySBQR2Friends.obj
 0001:0002b140       ?insert_unique@?$_Rb_tree@HU?$less@H@stlpmtx_std@@U?$pair@$$CBHUSGameSpyProfile@CCryGameSpySBQR2Friends@@@2@U?$_Select1st@U?$pair@$$CBHUSGameSpyProfile@CCryGameSpySBQR2Friends@@@stlpmtx_std@@@priv@2@U?$_MapTraitsT@U?$pair@$$CBHUSGameSpyProfile@CCryGameSpySBQR2Friends@@@stlpmtx_std@@@52@V?$allocator@U?$pair@$$CBHUSGameSpyProfile@CCryGameSpySBQR2Friends@@@stlpmtx_std@@@2@@priv@stlpmtx_std@@QEAA?AU?$pair@U?$_Rb_tree_iterator@U?$pair@$$CBHUSGameSpyProfile@CCryGameSpySBQR2Friends@@@stlpmtx_std@@U?$_MapTraitsT@U?$pair@$$CBHUSGameSpyProfile@CCryGameSpySBQR2Friends@@@stlpmtx_std@@@priv@2@@priv@stlpmtx_std@@_N@3@AEBU?$pair@$$CBHUSGameSpyProfile@CCryGameSpySBQR2Friends@@@3@@Z 0000000039a2c140 f i CryGameSpySBQR2Friends.obj
 0001:0002b340       ?insert_unique@?$_Rb_tree@HU?$less@H@stlpmtx_std@@U?$pair@$$CBHUSGameSpyProfile@CCryGameSpySBQR2Friends@@@2@U?$_Select1st@U?$pair@$$CBHUSGameSpyProfile@CCryGameSpySBQR2Friends@@@stlpmtx_std@@@priv@2@U?$_MapTraitsT@U?$pair@$$CBHUSGameSpyProfile@CCryGameSpySBQR2Friends@@@stlpmtx_std@@@52@V?$allocator@U?$pair@$$CBHUSGameSpyProfile@CCryGameSpySBQR2Friends@@@stlpmtx_std@@@2@@priv@stlpmtx_std@@QEAA?AU?$_Rb_tree_iterator@U?$pair@$$CBHUSGameSpyProfile@CCryGameSpySBQR2Friends@@@stlpmtx_std@@U?$_MapTraitsT@U?$pair@$$CBHUSGameSpyProfile@CCryGameSpySBQR2Friends@@@stlpmtx_std@@@priv@2@@23@U423@AEBU?$pair@$$CBHUSGameSpyProfile@CCryGameSpySBQR2Friends@@@3@@Z 0000000039a2c340 f i CryGameSpySBQR2Friends.obj
 0001:0002b780       ??0CCryGameSpySBQR2Friends@@QEAA@PEAVCCryLobby@@PEAVCCryLobbyService@@@Z 0000000039a2c780 f   CryGameSpySBQR2Friends.obj
 0001:0002b880       ??_ECCryGameSpySBQR2Friends@@WBA@EAAPEAXI@Z 0000000039a2c880 f i CryGameSpySBQR2Friends.obj
 0001:0002b890       ??1CCryGameSpySBQR2Friends@@UEAA@XZ 0000000039a2c890 f i CryGameSpySBQR2Friends.obj
 0001:0002b980       ??_ECCryGameSpySBQR2Friends@@UEAAPEAXI@Z 0000000039a2c980 f i CryGameSpySBQR2Friends.obj
 0001:0002b980       ??_GCCryGameSpySBQR2Friends@@UEAAPEAXI@Z 0000000039a2c980 f i CryGameSpySBQR2Friends.obj
 0001:0002b9b0       ??$?AH@?$map@HUSGameSpyProfile@CCryGameSpySBQR2Friends@@U?$less@H@stlpmtx_std@@V?$allocator@U?$pair@$$CBHUSGameSpyProfile@CCryGameSpySBQR2Friends@@@stlpmtx_std@@@4@@stlpmtx_std@@QEAAAEAUSGameSpyProfile@CCryGameSpySBQR2Friends@@AEBH@Z 0000000039a2c9b0 f i CryGameSpySBQR2Friends.obj
 0001:0002bb60       ?ProcessActiveFriendStateChanges@CCryGameSpySBQR2Friends@@AEAAXXZ 0000000039a2cb60 f   CryGameSpySBQR2Friends.obj
 0001:0002bd40       ?EndFriendsGetNamesList@CCryGameSpySBQR2Friends@@AEAAXI@Z 0000000039a2cd40 f   CryGameSpySBQR2Friends.obj
 0001:0002c080       ?GPRecvBuddyStatusCallback@CCryGameSpySBQR2Friends@@CAXPEAVCGameSpySBQR2GPConnection@@USResult@2@PEAUGPRecvBuddyStatusArg@@PEAUIGameSpyLink@@@Z 0000000039a2d080 f   CryGameSpySBQR2Friends.obj
 0001:0002c470       ?GPGetReverseBuddiesCallback@CCryGameSpySBQR2Friends@@CAXPEAVCGameSpySBQR2GPConnection@@USResult@2@PEAUGPGetReverseBuddiesResponseArg@@PEAUIGameSpyLink@@@Z 0000000039a2d470 f   CryGameSpySBQR2Friends.obj
 0001:0002c600       ?FriendsSendFriendRequest@CCryGameSpySBQR2Friends@@QEAA?AW4ECryLobbyError@@HPEBD@Z 0000000039a2d600 f   CryGameSpySBQR2Friends.obj
 0001:0002c680       ?FriendsAcceptFriendRequest@CCryGameSpySBQR2Friends@@QEAA?AW4ECryLobbyError@@H@Z 0000000039a2d680 f   CryGameSpySBQR2Friends.obj
 0001:0002c760       ?FriendsDenyFriendRequest@CCryGameSpySBQR2Friends@@QEAA?AW4ECryLobbyError@@H@Z 0000000039a2d760 f   CryGameSpySBQR2Friends.obj
 0001:0002c7f0       ?FriendsRevokeFriendStatus@CCryGameSpySBQR2Friends@@QEAA?AW4ECryLobbyError@@H@Z 0000000039a2d7f0 f   CryGameSpySBQR2Friends.obj
 0001:0002c8d0       ?LateInitialise@CCryGameSpySBQR2Friends@@QEAAXPEAVCGameSpySBQR2GPConnection@@@Z 0000000039a2d8d0 f   CryGameSpySBQR2Friends.obj
 0001:0002ca90       ?EndTask@CCryGameSpySBQR2Friends@@AEAAXI@Z 0000000039a2da90 f   CryGameSpySBQR2Friends.obj
 0001:0002cb80       ?StopTaskRunning@CCryGameSpySBQR2Friends@@AEAAXI@Z 0000000039a2db80 f   CryGameSpySBQR2Friends.obj
 0001:0002cb80       ?TickFriendsSendGameInvite@CCryGameSpySBQR2Friends@@AEAAXI@Z 0000000039a2db80 f   CryGameSpySBQR2Friends.obj
 0001:0002cbf0       ?TickFriendsGetFriendsList@CCryGameSpySBQR2Friends@@AEAAXI@Z 0000000039a2dbf0 f   CryGameSpySBQR2Friends.obj
 0001:0002ccf0       ?TickFriendsGetNamesList@CCryGameSpySBQR2Friends@@AEAAXI@Z 0000000039a2dcf0 f   CryGameSpySBQR2Friends.obj
 0001:0002ce80       ?UpdateProfile@CCryGameSpySBQR2Friends@@AEAAXPEAVCGameSpySBQR2GPConnection@@HI@Z 0000000039a2de80 f   CryGameSpySBQR2Friends.obj
 0001:0002cf50       ?GPRecvBuddyRequestCallback@CCryGameSpySBQR2Friends@@CAXPEAVCGameSpySBQR2GPConnection@@USResult@2@PEAUGPRecvBuddyRequestArg@@PEAUIGameSpyLink@@@Z 0000000039a2df50 f   CryGameSpySBQR2Friends.obj
 0001:0002d090       ?GPRecvBuddyMessageCallback@CCryGameSpySBQR2Friends@@CAXPEAVCGameSpySBQR2GPConnection@@USResult@2@PEAUGPRecvBuddyMessageArg@@PEAUIGameSpyLink@@@Z 0000000039a2e090 f   CryGameSpySBQR2Friends.obj
 0001:0002d3c0       ?GPRecvGameInviteCallback@CCryGameSpySBQR2Friends@@CAXPEAVCGameSpySBQR2GPConnection@@USResult@2@PEAUGPRecvGameInviteArg@@PEAUIGameSpyLink@@@Z 0000000039a2e3c0 f   CryGameSpySBQR2Friends.obj
 0001:0002d6b0       ?GPRecvBuddyAuthCallback@CCryGameSpySBQR2Friends@@CAXPEAVCGameSpySBQR2GPConnection@@USResult@2@PEAUGPRecvBuddyAuthArg@@PEAUIGameSpyLink@@@Z 0000000039a2e6b0 f   CryGameSpySBQR2Friends.obj
 0001:0002d860       ?GPGetInfoTaskCallback@CCryGameSpySBQR2Friends@@CAXPEAVCGameSpySBQR2GPConnection@@USResult@2@PEAUGPGetInfoResponseArg@@PEAUIGameSpyLink@@@Z 0000000039a2e860 f   CryGameSpySBQR2Friends.obj
 0001:0002d9c0       ?InitialiseCallbacks@CCryGameSpySBQR2Friends@@QEAAXXZ 0000000039a2e9c0 f   CryGameSpySBQR2Friends.obj
 0001:0002daa0       ?StartFriendsGetFriendsList@CCryGameSpySBQR2Friends@@AEAAXI@Z 0000000039a2eaa0 f   CryGameSpySBQR2Friends.obj
 0001:0002dbc0       ?StartFriendsGetNamesList@CCryGameSpySBQR2Friends@@AEAAXI@Z 0000000039a2ebc0 f   CryGameSpySBQR2Friends.obj
 0001:0002de70       ?Initialise@CCryGameSpySBQR2Friends@@UEAA?AW4ECryLobbyError@@XZ 0000000039a2ee70 f   CryGameSpySBQR2Friends.obj
 0001:0002dee0       ?Tick@CCryGameSpySBQR2Friends@@QEAAXVCTimeValue@@@Z 0000000039a2eee0 f   CryGameSpySBQR2Friends.obj
 0001:0002e020       ??2SCrySharedUserID@@SAPEAX_K@Z 0000000039a2f020 f i CryGameSpySBQR2Friends.obj
 0001:0002e020       ??2SCrySharedSessionID@@SAPEAX_K@Z 0000000039a2f020 f i CryGameSpySBQR2FriendsManagement.obj
 0001:0002e070       ?FriendsManagementGetName@CCryGameSpySBQR2FriendsManagement@@UEAA?AW4ECryLobbyError@@IPEAUCryUserID@@IPEAIP6AXIW42@PEAUSFriendInfo@@IPEAX@Z4@Z 0000000039a2f070 f   CryGameSpySBQR2FriendsManagement.obj
 0001:0002e0e0       ?EndFriendsManagementFindUser@CCryGameSpySBQR2FriendsManagement@@AEAAXI@Z 0000000039a2f0e0 f   CryGameSpySBQR2FriendsManagement.obj
 0001:0002e160       ?EndFriendsManagementGetStatus@CCryGameSpySBQR2FriendsManagement@@AEAAXI@Z 0000000039a2f160 f   CryGameSpySBQR2FriendsManagement.obj
 0001:0002e1b0       ?StartTaskRunning@CCryGameSpySBQR2FriendsManagement@@AEAAXI@Z 0000000039a2f1b0 f   CryGameSpySBQR2FriendsManagement.obj
 0001:0002e210       ?Execute@?$CClassJobNoRef2@IV?$_smart_ptr@USCrySessionID@@@@VCCryGameSpySBQR2LobbyService@@@CWorkQueue@@UEAAXXZ 0000000039a2f210 f i CryGameSpySBQR2FriendsManagement.obj
 0001:0002e260       ??8SCryLANUserID@@UEBA_NAEBUSCryUserID@@@Z 0000000039a2f260 f i CryLANMatchMaking.obj
 0001:0002e260       ??8SCryGameSpySBQR2SessionID@@UEAA_NAEBUSCrySessionID@@@Z 0000000039a2f260 f i CryGameSpySBQR2FriendsManagement.obj
 0001:0002e270       ?AsCStr@SCryGameSpySBQR2SessionID@@UEBAXPEADH@Z 0000000039a2f270 f i CryGameSpySBQR2FriendsManagement.obj
 0001:0002e2b0       ?LateInitialise@CCryGameSpySBQR2FriendsManagement@@QEAAXV?$_smart_ptr@VCCryGameSpySBQR2Friends@@@@@Z 0000000039a2f2b0 f   CryGameSpySBQR2FriendsManagement.obj
 0001:0002e310       ??4SFriendInfo@@QEAAAEAU0@AEBU0@@Z 0000000039a2f310 f i CryGameSpySBQR2FriendsManagement.obj
 0001:0002e3b0       ?CreateTaskLink@CCryGameSpySBQR2FriendsManagement@@AEAA?AW4ECryLobbyError@@I@Z 0000000039a2f3b0 f   CryGameSpySBQR2FriendsManagement.obj
 0001:0002e460       ??1?$CClassJobNoRef2@IV?$_smart_ptr@USCrySessionID@@@@VCCryGameSpySBQR2LobbyService@@@CWorkQueue@@UEAA@XZ 0000000039a2f460 f i CryGameSpySBQR2FriendsManagement.obj
 0001:0002e500       ??_E?$CClassJobNoRef2@IV?$_smart_ptr@USCrySessionID@@@@VCCryGameSpySBQR2LobbyService@@@CWorkQueue@@UEAAPEAXI@Z 0000000039a2f500 f i CryGameSpySBQR2FriendsManagement.obj
 0001:0002e500       ??_G?$CClassJobNoRef2@IV?$_smart_ptr@USCrySessionID@@@@VCCryGameSpySBQR2LobbyService@@@CWorkQueue@@UEAAPEAXI@Z 0000000039a2f500 f i CryGameSpySBQR2FriendsManagement.obj
 0001:0002e530       ??0CCryGameSpySBQR2FriendsManagement@@QEAA@PEAVCCryLobby@@PEAVCCryLobbyService@@@Z 0000000039a2f530 f   CryGameSpySBQR2FriendsManagement.obj
 0001:0002e5d0       ??_ECCryGameSpySBQR2FriendsManagement@@WBA@EAAPEAXI@Z 0000000039a2f5d0 f i CryGameSpySBQR2FriendsManagement.obj
 0001:0002e5e0       ??1CCryGameSpySBQR2FriendsManagement@@UEAA@XZ 0000000039a2f5e0 f i CryGameSpySBQR2FriendsManagement.obj
 0001:0002e6b0       ??_ECCryGameSpySBQR2FriendsManagement@@UEAAPEAXI@Z 0000000039a2f6b0 f i CryGameSpySBQR2FriendsManagement.obj
 0001:0002e6b0       ??_GCCryGameSpySBQR2FriendsManagement@@UEAAPEAXI@Z 0000000039a2f6b0 f i CryGameSpySBQR2FriendsManagement.obj
 0001:0002e6e0       ?EndFriendsManagementTaskWithInfo@CCryGameSpySBQR2FriendsManagement@@AEAAXI@Z 0000000039a2f6e0 f   CryGameSpySBQR2FriendsManagement.obj
 0001:0002e930       ?FreeTask@CCryGameSpySBQR2FriendsManagement@@MEAAXI@Z 0000000039a2f930 f   CryGameSpySBQR2FriendsManagement.obj
 0001:0002ea50       ?EndTask@CCryGameSpySBQR2FriendsManagement@@AEAAXI@Z 0000000039a2fa50 f   CryGameSpySBQR2FriendsManagement.obj
 0001:0002eb70       ??$Add@IVCCryGameSpySBQR2LobbyUI@@@CWorkQueue@@QEAAXP8CCryGameSpySBQR2LobbyUI@@EAAXI@ZPEAV1@I@Z 0000000039a2fb70 f i CryGameSpySBQR2LobbyUI.obj
 0001:0002eb70       ??$Add@IVCCryGameSpySBQR2FriendsManagement@@@CWorkQueue@@QEAAXP8CCryGameSpySBQR2FriendsManagement@@EAAXI@ZPEAV1@I@Z 0000000039a2fb70 f i CryGameSpySBQR2FriendsManagement.obj
 0001:0002eb70       ??$Add@IVCCryGameSpySBQR2Stats@@@CWorkQueue@@QEAAXP8CCryGameSpySBQR2Stats@@EAAXI@ZPEAV1@I@Z 0000000039a2fb70 f i CryGameSpySBQR2Stats.obj
 0001:0002ec30       ??$Add@IV?$_smart_ptr@USCrySessionID@@@@VCCryGameSpySBQR2LobbyService@@@CWorkQueue@@QEAAXP8CCryGameSpySBQR2LobbyService@@EAAXIV?$_smart_ptr@USCrySessionID@@@@@ZPEAV1@I0@Z 0000000039a2fc30 f i CryGameSpySBQR2FriendsManagement.obj
 0001:0002edc0       ?FriendsManagementFindUser@CCryGameSpySBQR2FriendsManagement@@UEAA?AW4ECryLobbyError@@IPEAUSFriendManagementSearchInfo@@IPEAIP6AXIW42@PEAUSFriendInfo@@IPEAX@Z4@Z 0000000039a2fdc0 f   CryGameSpySBQR2FriendsManagement.obj
 0001:0002ef80       ?InitialiseTask@CCryGameSpySBQR2FriendsManagement@@AEAA?AW4ECryLobbyError@@W4ETask@1@IPEAUCryUserID@@IPEAIPEAX3@Z 0000000039a2ff80 f   CryGameSpySBQR2FriendsManagement.obj
 0001:0002f130       ?StopTaskRunning@CCryGameSpySBQR2FriendsManagement@@AEAAXI@Z 0000000039a30130 f   CryGameSpySBQR2FriendsManagement.obj
 0001:0002f1a0       ?StartFriendsManagementSendFriendRequest@CCryGameSpySBQR2FriendsManagement@@AEAAXI@Z 0000000039a301a0 f   CryGameSpySBQR2FriendsManagement.obj
 0001:0002f2f0       ?StartFriendsManagementAcceptFriendRequest@CCryGameSpySBQR2FriendsManagement@@AEAAXI@Z 0000000039a302f0 f   CryGameSpySBQR2FriendsManagement.obj
 0001:0002f440       ?StartFriendsManagementRejectFriendRequest@CCryGameSpySBQR2FriendsManagement@@AEAAXI@Z 0000000039a30440 f   CryGameSpySBQR2FriendsManagement.obj
 0001:0002f590       ?StartFriendsManagementRevokeFriendStatus@CCryGameSpySBQR2FriendsManagement@@AEAAXI@Z 0000000039a30590 f   CryGameSpySBQR2FriendsManagement.obj
 0001:0002f6e0       ?StartFriendsManagementIsUserFriend@CCryGameSpySBQR2FriendsManagement@@AEAAXI@Z 0000000039a306e0 f   CryGameSpySBQR2FriendsManagement.obj
 0001:0002f880       ?TickFriendsManagementFindUser@CCryGameSpySBQR2FriendsManagement@@AEAAXI@Z 0000000039a30880 f   CryGameSpySBQR2FriendsManagement.obj
 0001:0002f8f0       ?StartFriendsManagementBlockUser@CCryGameSpySBQR2FriendsManagement@@AEAAXI@Z 0000000039a308f0 f   CryGameSpySBQR2FriendsManagement.obj
 0001:0002fa50       ?StartFriendsManagementUnblockUser@CCryGameSpySBQR2FriendsManagement@@AEAAXI@Z 0000000039a30a50 f   CryGameSpySBQR2FriendsManagement.obj
 0001:0002fbb0       ?StartFriendsManagementIsUserBlocked@CCryGameSpySBQR2FriendsManagement@@AEAAXI@Z 0000000039a30bb0 f   CryGameSpySBQR2FriendsManagement.obj
 0001:0002fd50       ?StartFriendsManagementAcceptInvite@CCryGameSpySBQR2FriendsManagement@@AEAAXI@Z 0000000039a30d50 f   CryGameSpySBQR2FriendsManagement.obj
 0001:0002ff40       ?FindUserCallback@CCryGameSpySBQR2FriendsManagement@@CAXPEAVCGameSpySBQR2GPConnection@@USResult@2@PEAUGPProfileSearchResponseArg@@PEAUIGameSpyLink@@@Z 0000000039a30f40 f   CryGameSpySBQR2FriendsManagement.obj
 0001:000304c0       ?FriendsManagementGetStatus@CCryGameSpySBQR2FriendsManagement@@UEAA?AW4ECryLobbyError@@IPEAUCryUserID@@IPEAIP6AXIW42@PEAUSFriendStatusInfo@@IPEAX@Z4@Z 0000000039a314c0 f   CryGameSpySBQR2FriendsManagement.obj
 0001:00030700       ?StartFriendsManagementGetStatus@CCryGameSpySBQR2FriendsManagement@@AEAAXI@Z 0000000039a31700 f   CryGameSpySBQR2FriendsManagement.obj
 0001:00030850       ?FriendsManagementSendFriendRequest@CCryGameSpySBQR2FriendsManagement@@UEAA?AW4ECryLobbyError@@IPEAUCryUserID@@IPEAIP6AXIW42@PEAX@Z3@Z 0000000039a31850 f   CryGameSpySBQR2FriendsManagement.obj
 0001:000308b0       ?FriendsManagementAcceptFriendRequest@CCryGameSpySBQR2FriendsManagement@@UEAA?AW4ECryLobbyError@@IPEAUCryUserID@@IPEAIP6AXIW42@PEAX@Z3@Z 0000000039a318b0 f   CryGameSpySBQR2FriendsManagement.obj
 0001:00030910       ?FriendsManagementRejectFriendRequest@CCryGameSpySBQR2FriendsManagement@@UEAA?AW4ECryLobbyError@@IPEAUCryUserID@@IPEAIP6AXIW42@PEAX@Z3@Z 0000000039a31910 f   CryGameSpySBQR2FriendsManagement.obj
 0001:00030970       ?FriendsManagementRevokeFriendStatus@CCryGameSpySBQR2FriendsManagement@@UEAA?AW4ECryLobbyError@@IPEAUCryUserID@@IPEAIP6AXIW42@PEAX@Z3@Z 0000000039a31970 f   CryGameSpySBQR2FriendsManagement.obj
 0001:000309d0       ?FriendsManagementIsUserFriend@CCryGameSpySBQR2FriendsManagement@@UEAA?AW4ECryLobbyError@@IPEAUCryUserID@@IPEAIP6AXIW42@PEAUSFriendManagementInfo@@IPEAX@Z4@Z 0000000039a319d0 f   CryGameSpySBQR2FriendsManagement.obj
 0001:00030a30       ?FriendsManagementBlockUser@CCryGameSpySBQR2FriendsManagement@@UEAA?AW4ECryLobbyError@@IPEAUCryUserID@@IPEAIP6AXIW42@PEAX@Z3@Z 0000000039a31a30 f   CryGameSpySBQR2FriendsManagement.obj
 0001:00030a90       ?FriendsManagementUnblockUser@CCryGameSpySBQR2FriendsManagement@@UEAA?AW4ECryLobbyError@@IPEAUCryUserID@@IPEAIP6AXIW42@PEAX@Z3@Z 0000000039a31a90 f   CryGameSpySBQR2FriendsManagement.obj
 0001:00030af0       ?FriendsManagementIsUserBlocked@CCryGameSpySBQR2FriendsManagement@@UEAA?AW4ECryLobbyError@@IPEAUCryUserID@@IPEAIP6AXIW42@PEAUSFriendManagementInfo@@IPEAX@Z4@Z 0000000039a31af0 f   CryGameSpySBQR2FriendsManagement.obj
 0001:00030b50       ?FriendsManagementAcceptInvite@CCryGameSpySBQR2FriendsManagement@@UEAA?AW4ECryLobbyError@@IPEAUCryUserID@@PEAIP6AXIW42@PEAX@Z3@Z 0000000039a31b50 f   CryGameSpySBQR2FriendsManagement.obj
 0001:00030bb0       ?StartFriendsManagementFindUser@CCryGameSpySBQR2FriendsManagement@@AEAAXI@Z 0000000039a31bb0 f   CryGameSpySBQR2FriendsManagement.obj
 0001:00030c70       ?Tick@CCryGameSpySBQR2FriendsManagement@@QEAAXVCTimeValue@@@Z 0000000039a31c70 f   CryGameSpySBQR2FriendsManagement.obj
 0001:00030e10       ?SetNeedGameSpyObject@CCryGameSpySBQR2LobbyService@@QEAAXI_N@Z 0000000039a31e10 f   CryGameSpySBQR2Lobby.obj
 0001:00030e30       ?GetAnySignedInUser@CCryGameSpySBQR2LobbyService@@QEAA_NAEAI@Z 0000000039a31e30 f   CryGameSpySBQR2Lobby.obj
 0001:00030e60       ?GetSake@CCryGameSpySBQR2LobbyService@@QEAAPEAVCGameSpySBQR2Sake@@I@Z 0000000039a31e60 f   CryGameSpySBQR2Lobby.obj
 0001:00030ef0       ?SetGPProfile@CCryGameSpySBQR2LobbyService@@QEAAXIH@Z 0000000039a31ef0 f   CryGameSpySBQR2Lobby.obj
 0001:00030f10       ?GetGPProfile@CCryGameSpySBQR2LobbyService@@QEAAHI@Z 0000000039a31f10 f   CryGameSpySBQR2Lobby.obj
 0001:00030f30       ?SetGPLoginTicket@CCryGameSpySBQR2LobbyService@@QEAAXIQEAD@Z 0000000039a31f30 f   CryGameSpySBQR2Lobby.obj
 0001:00030f60       ?GetGPLoginTicket@CCryGameSpySBQR2LobbyService@@QEAAPEBDI@Z 0000000039a31f60 f   CryGameSpySBQR2Lobby.obj
 0001:00030f90       ?GetOnlineState@CCryGameSpySBQR2LobbyService@@QEAA?AW4EOnlineState@@I@Z 0000000039a31f90 f   CryGameSpySBQR2Lobby.obj
 0001:00030fb0       ?GetAvailabilityCheck@CCryGameSpySBQR2LobbyService@@QEAAPEAVCGameSpySBQR2AvailabilityCheck@@XZ 0000000039a31fb0 f   CryGameSpySBQR2Lobby.obj
 0001:00031010       ?GetCore@CCryGameSpySBQR2LobbyService@@QEAAPEAVCGameSpySBQR2Core@@XZ 0000000039a32010 f   CryGameSpySBQR2Lobby.obj
 0001:00031070       ?GetNATNegotiation@CCryGameSpySBQR2LobbyService@@QEAAPEAVCGameSpySBQR2NATNegotiation@@XZ 0000000039a32070 f   CryGameSpySBQR2Lobby.obj
 0001:000310d0       ?AddGameSpySDK@CCryGameSpySBQR2LobbyService@@QEAAXPEAVCGameSpySDK@@@Z 0000000039a320d0 f   CryGameSpySBQR2Lobby.obj
 0001:000310f0       ?QueueThink@CCryGameSpySBQR2LobbyService@@QEAAXPEAVCGameSpyThinkerSDK@@@Z 0000000039a320f0 f   CryGameSpySBQR2Lobby.obj
 0001:00031110       ?HasPublicAddress@CCryGameSpySBQR2LobbyService@@QEAA_NXZ 0000000039a32110 f   CryGameSpySBQR2Lobby.obj
 0001:00031120       ?GetPublicIP@CCryGameSpySBQR2LobbyService@@QEAAIXZ 0000000039a32120 f   CryGameSpySBQR2Lobby.obj
 0001:00031140       ?GetPublicPort@CCryGameSpySBQR2LobbyService@@QEAAGXZ 0000000039a32140 f   CryGameSpySBQR2Lobby.obj
 0001:00031160       ?GetPrivateIP@CCryGameSpySBQR2LobbyService@@QEAAIXZ 0000000039a32160 f   CryGameSpySBQR2Lobby.obj
 0001:000311f0       ?GetProductID@CCryGameSpySBQR2LobbyService@@QEAAHXZ 0000000039a321f0 f   CryGameSpySBQR2Lobby.obj
 0001:00031200       ?GetNameSpaceID@CCryGameSpySBQR2LobbyService@@QEAAHXZ 0000000039a32200 f   CryGameSpySBQR2Lobby.obj
 0001:00031210       ?GetPartnerID@CCryGameSpySBQR2LobbyService@@QEAAHXZ 0000000039a32210 f   CryGameSpySBQR2Lobby.obj
 0001:00031220       ?GetDistributionID@CCryGameSpySBQR2LobbyService@@QEAAIXZ 0000000039a32220 f   CryGameSpySBQR2Lobby.obj
 0001:00031230       ?GameDispatchOnlineStatus@CCryGameSpySBQR2LobbyService@@AEAAXW4ECryLobbySystemEvent@@IW4EOnlineState@@W4ECryLobbyError@@@Z 0000000039a32230 f   CryGameSpySBQR2Lobby.obj
 0001:00031270       ?QR2PublicAddressCallback@CCryGameSpySBQR2LobbyService@@CAXIGPEAX@Z 0000000039a32270 f   CryGameSpySBQR2Lobby.obj
 0001:000312b0       ?GetAvailableGameSpyObjects@CCryGameSpySBQR2LobbyService@@QEAAIXZ 0000000039a322b0 f   CryGameSpySBQR2Lobby.obj
 0001:000312f0       ?GetSocketPorts@CCryGameSpySBQR2LobbyService@@UEAAXAEAG0@Z 0000000039a322f0 f   CryGameSpySBQR2Lobby.obj
 0001:00031310       ?SetNeedAuthService@CCryGameSpySBQR2LobbyService@@QEAAX_N@Z 0000000039a32310 f   CryGameSpySBQR2Lobby.obj
 0001:00031330       ?AuthServiceGetCertificate@CCryGameSpySBQR2LobbyService@@QEAAPEAUGSLoginCertificate@@XZ 0000000039a32330 f   CryGameSpySBQR2Lobby.obj
 0001:00031350       ?AuthServiceGetPrivateData@CCryGameSpySBQR2LobbyService@@QEAAPEAUGSLoginCertificatePrivate@@XZ 0000000039a32350 f   CryGameSpySBQR2Lobby.obj
 0001:00031370       ?NATDetectionCallback@CCryGameSpySBQR2LobbyService@@CAXUSResult@CGameSpySBQR2NATNegotiation@@W4ENatType@@PEAUIGameSpyLink@@@Z 0000000039a32370 f   CryGameSpySBQR2Lobby.obj
 0001:000313b0       ?DispatchNATType@CCryGameSpySBQR2LobbyService@@AEAAXXZ 0000000039a323b0 f   CryGameSpySBQR2Lobby.obj
 0001:000313f0       ?LocalCDKeyReauthCallback@CCryGameSpySBQR2LobbyService@@SAXHHHPEADPEAX@Z 0000000039a323f0 f   CryGameSpySBQR2Lobby.obj
 0001:00031490       ?GetGameID@CCryGameSpySBQR2LobbyService@@QEBAIXZ 0000000039a32490 f   CryGameSpySBQR2Lobby.obj
 0001:000314a0       ?StopServerList@CCryGameSpySBQR2LobbyService@@QEAA?AW4ECryLobbyError@@XZ 0000000039a324a0 f   CryGameSpySBQR2Lobby.obj
 0001:00031500       ?ServerBrowserCallback@CCryGameSpySBQR2LobbyService@@CAXPEAU_ServerBrowser@@W4SBCallbackReason@@PEAU_SBServer@@PEAX@Z 0000000039a32500 f   CryGameSpySBQR2Lobby.obj
 0001:00031530       ?QR2HostRegisteredCallback@CCryGameSpySBQR2LobbyService@@CAXPEAX@Z 0000000039a32530 f   CryGameSpySBQR2Lobby.obj
 0001:00031540       ?GetMatchMaking@CCryGameSpySBQR2LobbyService@@UEAAPEAUICryMatchMaking@@XZ 0000000039a32540 f   CryGameSpySBQR2Lobby.obj
 0001:00031560       ?GetVoice@CCryGameSpySBQR2LobbyService@@UEAAPEAUICryVoice@@XZ 0000000039a32560 f   CryGameSpySBQR2Lobby.obj
 0001:00031580       ?GetStats@CCryGameSpySBQR2LobbyService@@UEAAPEAUICryStats@@XZ 0000000039a32580 f   CryGameSpySBQR2Lobby.obj
 0001:000315a0       ?GetLobbyUI@CCryGameSpySBQR2LobbyService@@UEAAPEAUICryLobbyUI@@XZ 0000000039a325a0 f   CryGameSpySBQR2Lobby.obj
 0001:000315c0       ?GetFriends@CCryGameSpySBQR2LobbyService@@UEAAPEAUICryFriends@@XZ 0000000039a325c0 f   CryGameSpySBQR2Lobby.obj
 0001:000315e0       ?GetFriendsManagement@CCryGameSpySBQR2LobbyService@@UEAAPEAUICryFriendsManagement@@XZ 0000000039a325e0 f   CryGameSpySBQR2Lobby.obj
 0001:00031600       ?GetDLCStore@CCryGameSpySBQR2LobbyService@@UEAAPEAUICryDLCStore@@XZ 0000000039a32600 f   CryGameSpySBQR2Lobby.obj
 0001:00031620       ?GetSignIn@CCryGameSpySBQR2LobbyService@@UEAAPEAUICrySignIn@@XZ 0000000039a32620 f   CryGameSpySBQR2Lobby.obj
 0001:00031640       ?GetName@CCryGameSpySBQR2LobbyService@@QEAAPEBDI@Z 0000000039a32640 f   CryGameSpySBQR2Lobby.obj
 0001:00031660       ?OnPacket@CCryGameSpySBQR2LobbyService@@UEAAXAEBV?$CConfigurableVariant@V?$CNode@USNullAddr@@V?$CNode@GV?$CNode@USIPv4Addr@@V?$CNode@ULobbyIdAddr@@VCEnd@NTypelist@@@NTypelist@@@NTypelist@@@NTypelist@@@NTypelist@@$07VCDefaultVariantConversion@NConfigurableVariantHelpers@@VCDefaultVariantConstruction@4@@@PEAVCCryLobbyPacket@@@Z 0000000039a32660 f   CryGameSpySBQR2Lobby.obj
 0001:000317a0       ?OnError@CCryGameSpySBQR2LobbyService@@UEAAXAEBV?$CConfigurableVariant@V?$CNode@USNullAddr@@V?$CNode@GV?$CNode@USIPv4Addr@@V?$CNode@ULobbyIdAddr@@VCEnd@NTypelist@@@NTypelist@@@NTypelist@@@NTypelist@@@NTypelist@@$07VCDefaultVariantConversion@NConfigurableVariantHelpers@@VCDefaultVariantConstruction@4@@@W4ESocketError@@I@Z 0000000039a327a0 f   CryGameSpySBQR2Lobby.obj
 0001:000317c0       ?OnSendComplete@CCryGameSpySBQR2LobbyService@@UEAAXAEBV?$CConfigurableVariant@V?$CNode@USNullAddr@@V?$CNode@GV?$CNode@USIPv4Addr@@V?$CNode@ULobbyIdAddr@@VCEnd@NTypelist@@@NTypelist@@@NTypelist@@@NTypelist@@@NTypelist@@$07VCDefaultVariantConversion@NConfigurableVariantHelpers@@VCDefaultVariantConstruction@4@@@I@Z 0000000039a327c0 f   CryGameSpySBQR2Lobby.obj
 0001:000317e0       ?QR2StateChanged@CCryGameSpySBQR2LobbyService@@QEAAXXZ 0000000039a327e0 f   CryGameSpySBQR2Lobby.obj
 0001:00031810       ?GetProfileNick@CCryGameSpySBQR2LobbyService@@QEAAPEBDXZ 0000000039a32810 f   CryGameSpySBQR2Lobby.obj
 0001:00031820       ?GetGameVersionString@CCryGameSpySBQR2LobbyService@@QEAAPEBDXZ 0000000039a32820 f   CryGameSpySBQR2Lobby.obj
 0001:00031830       ?GetGameSpyMatchMaking@CCryGameSpySBQR2LobbyService@@QEAAPEAVCCryGameSpySBQR2MatchMaking@@XZ 0000000039a32830 f   CryGameSpySBQR2Lobby.obj
 0001:00031840       ?QR2ServerKeyCallback@CCryGameSpySBQR2LobbyService@@CAXHPEAUqr2_buffer_s@@PEAX@Z 0000000039a32840 f   CryGameSpySBQR2Lobby.obj
 0001:00031870       ?QR2PlayerKeyCallback@CCryGameSpySBQR2LobbyService@@CAXHHPEAUqr2_buffer_s@@PEAX@Z 0000000039a32870 f   CryGameSpySBQR2Lobby.obj
 0001:000318a0       ?QR2TeamKeyCallback@CCryGameSpySBQR2LobbyService@@CAXHHPEAUqr2_buffer_s@@PEAX@Z 0000000039a328a0 f   CryGameSpySBQR2Lobby.obj
 0001:000318d0       ?QR2KeyListCallback@CCryGameSpySBQR2LobbyService@@CAXW4qr2_key_type@@PEAUqr2_keybuffer_s@@PEAX@Z 0000000039a328d0 f   CryGameSpySBQR2Lobby.obj
 0001:00031900       ?QR2PlayerTeamCountCallback@CCryGameSpySBQR2LobbyService@@CAHW4qr2_key_type@@PEAX@Z 0000000039a32900 f   CryGameSpySBQR2Lobby.obj
 0001:00031920       ?QR2AddErrorCallback@CCryGameSpySBQR2LobbyService@@CAXW4qr2_error_t@@PEADPEAX@Z 0000000039a32920 f   CryGameSpySBQR2Lobby.obj
 0001:00031950       ?NATNegotiateProgressCallback@CCryGameSpySBQR2LobbyService@@CAXUSResult@CGameSpySBQR2NATNegotiation@@HPEAUIGameSpyLink@@@Z 0000000039a32950 f   CryGameSpySBQR2Lobby.obj
 0001:000319c0       ?NATNegotiateCompletedCallback@CCryGameSpySBQR2LobbyService@@CAXUSResult@CGameSpySBQR2NATNegotiation@@H_KPEAUsockaddr_in@@PEAUIGameSpyLink@@@Z 0000000039a329c0 f   CryGameSpySBQR2Lobby.obj
 0001:00031a70       ?OnGameSpyObjectAvailable@CCryGameSpySBQR2LobbyService@@UEAAXW4EGameSpyObjectBit@ICryGameSpySBQR2LobbyComponent@@@Z 0000000039a32a70 f   CryGameSpySBQR2Lobby.obj
 0001:00031b20       ?OnGameSpyObjectUnavailable@CCryGameSpySBQR2LobbyService@@UEAAXW4EGameSpyObjectBit@ICryGameSpySBQR2LobbyComponent@@@Z 0000000039a32b20 f   CryGameSpySBQR2Lobby.obj
 0001:00031be0       ?OnGameSpyObjectCantMakeAvailable@CCryGameSpySBQR2LobbyService@@UEAAXW4EGameSpyObjectBit@ICryGameSpySBQR2LobbyComponent@@@Z 0000000039a32be0 f   CryGameSpySBQR2Lobby.obj
 0001:00031cd0       ?EndTask@CCryGameSpySBQR2LobbyService@@AEAAXI@Z 0000000039a32cd0 f   CryGameSpySBQR2Lobby.obj
 0001:00031d80       ?GetSystemTime@CCryGameSpySBQR2LobbyService@@UEAA?AW4ECryLobbyError@@IPEAUSCrySystemTime@@@Z 0000000039a32d80 f   CryGameSpySBQR2Lobby.obj
 0001:00031df0       ?AuthServiceWSLoginCallback@CCryGameSpySBQR2LobbyService@@CAXW4GHTTPResult@@PEAUWSLoginResponse@@PEAX@Z 0000000039a32df0 f   CryGameSpySBQR2Lobby.obj
 0001:00031ee0       ?AuthServiceInvalidateCertificate@CCryGameSpySBQR2LobbyService@@QEAAXXZ 0000000039a32ee0 f   CryGameSpySBQR2Lobby.obj
 0001:00031f40       ?ClearSignedInDetails@CCryGameSpySBQR2LobbyService@@AEAAXXZ 0000000039a32f40 f   CryGameSpySBQR2Lobby.obj
 0001:00031fb0       ?LocalCDKeyAuthCallback@CCryGameSpySBQR2LobbyService@@SAXHHHPEADPEAX@Z 0000000039a32fb0 f   CryGameSpySBQR2Lobby.obj
 0001:00032040       ?GetTitle@CCryGameSpySBQR2LobbyService@@QEBAPEBDXZ 0000000039a33040 f   CryGameSpySBQR2Lobby.obj
 0001:00032050       ?GetSecretKey@CCryGameSpySBQR2LobbyService@@QEBAPEBDXZ 0000000039a33050 f   CryGameSpySBQR2Lobby.obj
 0001:00032060       ?SendCookieToServer@CCryGameSpySBQR2LobbyService@@QEAA?AW4ECryLobbyError@@PEBDGI@Z 0000000039a33060 f   CryGameSpySBQR2Lobby.obj
 0001:00032100       ?StartServerList@CCryGameSpySBQR2LobbyService@@QEAA?AW4ECryLobbyError@@PEBEHPEBDP6AXW4SBCallbackReason@@PEAU_SBServer@@PEAX@Z4@Z 0000000039a33100 f   CryGameSpySBQR2Lobby.obj
 0001:000321d0       ?RequestServerUpdate@CCryGameSpySBQR2LobbyService@@QEAA?AW4ECryLobbyError@@PEAU_SBServer@@_N1@Z 0000000039a331d0 f   CryGameSpySBQR2Lobby.obj
 0001:00032240       ??4?$_smart_ptr@USTask@CGameSpySBQR2Core@@@@QEAAAEAV0@PEAUSTask@CGameSpySBQR2Core@@@Z 0000000039a33240 f i GameSpySBQR2Core.obj
 0001:00032240       ??4?$_smart_ptr@USThisLink@CCryGameSpySBQR2Friends@@@@QEAAAEAV0@PEAUSThisLink@CCryGameSpySBQR2Friends@@@Z 0000000039a33240 f i CryGameSpySBQR2Friends.obj
 0001:00032240       ??4?$_smart_ptr@USTaskLink@CCryGameSpySBQR2MatchMaking@@@@QEAAAEAV0@PEAUSTaskLink@CCryGameSpySBQR2MatchMaking@@@Z 0000000039a33240 f i CryGameSpySBQR2MatchMaking.obj
 0001:00032240       ??4?$_smart_ptr@USCrySessionID@@@@QEAAAEAV0@PEAUSCrySessionID@@@Z 0000000039a33240 f i CryGameSpySBQR2MatchMaking.obj
 0001:00032240       ??4?$_smart_ptr@USSessionLink@CCryGameSpySBQR2MatchMaking@@@@QEAAAEAV0@PEAUSSessionLink@CCryGameSpySBQR2MatchMaking@@@Z 0000000039a33240 f i CryGameSpySBQR2MatchMaking.obj
 0001:00032240       ??4?$_smart_ptr@USGameSpyKey@CCryGameSpySBQR2MatchMaking@@@@QEAAAEAV0@PEAUSGameSpyKey@CCryGameSpySBQR2MatchMaking@@@Z 0000000039a33240 f i CryGameSpySBQR2MatchMaking.obj
 0001:00032240       ??4?$_smart_ptr@VCCryGameSpySBQR2Stats@@@@QEAAAEAV0@PEAVCCryGameSpySBQR2Stats@@@Z 0000000039a33240 f i CryGameSpySBQR2Lobby.obj
 0001:00032240       ??4?$_smart_ptr@VCCryGameSpySBQR2SignIn@@@@QEAAAEAV0@PEAVCCryGameSpySBQR2SignIn@@@Z 0000000039a33240 f i CryGameSpySBQR2Lobby.obj
 0001:00032240       ??4?$_smart_ptr@USOrderLink@CCryGameSpySBQR2DLCStore@@@@QEAAAEAV0@PEAUSOrderLink@CCryGameSpySBQR2DLCStore@@@Z 0000000039a33240 f i CryGameSpySBQR2DLCStore.obj
 0001:00032240       ??4?$_smart_ptr@VCCryGameSpySBQR2MatchMaking@@@@QEAAAEAV0@PEAVCCryGameSpySBQR2MatchMaking@@@Z 0000000039a33240 f i CryGameSpySBQR2Lobby.obj
 0001:00032240       ??4?$_smart_ptr@UIGameSpyLink@@@@QEAAAEAV0@PEAUIGameSpyLink@@@Z 0000000039a33240 f i GameSpySBQR2Core.obj
 0001:00032240       ??4?$_smart_ptr@VCCryGameSpySBQR2LobbyUI@@@@QEAAAEAV0@PEAVCCryGameSpySBQR2LobbyUI@@@Z 0000000039a33240 f i CryGameSpySBQR2Lobby.obj
 0001:00032240       ??4?$_smart_ptr@VCCryLobbyService@@@@QEAAAEAV0@PEAVCCryLobbyService@@@Z 0000000039a33240 f i CryLobby.obj
 0001:00032240       ??4?$_smart_ptr@USTaskLink@CCryGameSpySBQR2SignIn@@@@QEAAAEAV0@PEAUSTaskLink@CCryGameSpySBQR2SignIn@@@Z 0000000039a33240 f i CryGameSpySBQR2SignIn.obj
 0001:00032240       ??4?$_smart_ptr@USTaskLink@CCryGameSpySBQR2Stats@@@@QEAAAEAV0@PEAUSTaskLink@CCryGameSpySBQR2Stats@@@Z 0000000039a33240 f i CryGameSpySBQR2Stats.obj
 0001:00032240       ??4?$_smart_ptr@VCCryGameSpySBQR2FriendsManagement@@@@QEAAAEAV0@PEAVCCryGameSpySBQR2FriendsManagement@@@Z 0000000039a33240 f i CryGameSpySBQR2Lobby.obj
 0001:00032240       ??4?$_smart_ptr@VCCryGameSpySBQR2DLCStore@@@@QEAAAEAV0@PEAVCCryGameSpySBQR2DLCStore@@@Z 0000000039a33240 f i CryGameSpySBQR2DLCStore.obj
 0001:00032240       ??4?$_smart_ptr@VCCryGameSpySBQR2Voice@@@@QEAAAEAV0@PEAVCCryGameSpySBQR2Voice@@@Z 0000000039a33240 f i CryGameSpySBQR2Lobby.obj
 0001:00032240       ??4?$_smart_ptr@USThisLink@CCryGameSpySBQR2LobbyService@@@@QEAAAEAV0@PEAUSThisLink@CCryGameSpySBQR2LobbyService@@@Z 0000000039a33240 f i CryGameSpySBQR2Lobby.obj
 0001:00032240       ??4?$_smart_ptr@USRegisteredLobbyData@CCryGameSpySBQR2MatchMaking@@@@QEAAAEAV0@PEAUSRegisteredLobbyData@CCryGameSpySBQR2MatchMaking@@@Z 0000000039a33240 f i CryGameSpySBQR2MatchMaking.obj
 0001:00032240       ??4?$_smart_ptr@USTaskLink@CCryGameSpySBQR2FriendsManagement@@@@QEAAAEAV0@PEAUSTaskLink@CCryGameSpySBQR2FriendsManagement@@@Z 0000000039a33240 f i CryGameSpySBQR2FriendsManagement.obj
 0001:00032240       ??4?$_smart_ptr@VCCryGameSpySBQR2Friends@@@@QEAAAEAV0@PEAVCCryGameSpySBQR2Friends@@@Z 0000000039a33240 f i CryGameSpySBQR2Lobby.obj
 0001:00032240       ??4?$_smart_ptr@VCCryLANMatchMaking@@@@QEAAAEAV0@PEAVCCryLANMatchMaking@@@Z 0000000039a33240 f i CryLANLobby.obj
 0001:00032240       ??4?$_smart_ptr@USTaskLink@CCryGameSpySBQR2Friends@@@@QEAAAEAV0@PEAUSTaskLink@CCryGameSpySBQR2Friends@@@Z 0000000039a33240 f i CryGameSpySBQR2Friends.obj
 0001:00032240       ??4?$_smart_ptr@USCallbackBase@CGameSpySBQR2GPConnection@@@@QEAAAEAV0@PEAUSCallbackBase@CGameSpySBQR2GPConnection@@@Z 0000000039a33240 f i GameSpySBQR2GPConnection.obj
 0001:00032240       ??4?$_smart_ptr@USTaskLink@CCryGameSpySBQR2DLCStore@@@@QEAAAEAV0@PEAUSTaskLink@CCryGameSpySBQR2DLCStore@@@Z 0000000039a33240 f i CryGameSpySBQR2DLCStore.obj
 0001:000322b0       ?_AllocData@?$CryStackStringT@D$0BF@@@QEAAX_K@Z 0000000039a332b0 f i CryGameSpySBQR2Lobby.obj
 0001:00032330       ?_Assign@?$CryStackStringT@D$0BF@@@QEAAXPEBD_K@Z 0000000039a33330 f i CryGameSpySBQR2Lobby.obj
 0001:000323d0       ?_AllocData@?$CryStackStringT@D$0BP@@@QEAAX_K@Z 0000000039a333d0 f i CryGameSpySBQR2Lobby.obj
 0001:00032450       ?_Assign@?$CryStackStringT@D$0BP@@@QEAAXPEBD_K@Z 0000000039a33450 f i CryGameSpySBQR2Lobby.obj
 0001:000324f0       ?_AllocData@?$CryStackStringT@D$0EA@@@QEAAX_K@Z 0000000039a334f0 f i CryGameSpySBQR2Lobby.obj
 0001:00032570       ??_GSTaskLink@CCryGameSpySBQR2SignIn@@UEAAPEAXI@Z 0000000039a33570 f i CryGameSpySBQR2SignIn.obj
 0001:00032570       ??_GSThisLink@CCryGameSpySBQR2Friends@@UEAAPEAXI@Z 0000000039a33570 f i CryGameSpySBQR2Friends.obj
 0001:00032570       ??_ESThisLink@CCryGameSpySBQR2LobbyService@@UEAAPEAXI@Z 0000000039a33570 f i CryGameSpySBQR2Lobby.obj
 0001:00032570       ??_ESTaskLink@CCryGameSpySBQR2SignIn@@UEAAPEAXI@Z 0000000039a33570 f i CryGameSpySBQR2SignIn.obj
 0001:00032570       ??_GSTaskLink@CCryGameSpySBQR2FriendsManagement@@UEAAPEAXI@Z 0000000039a33570 f i CryGameSpySBQR2FriendsManagement.obj
 0001:00032570       ??_ECMultiThreadRefCount@@UEAAPEAXI@Z 0000000039a33570 f i CryDLCStore.obj
 0001:00032570       ??_ESCryGameSpySBQR2DLCDownloadableID@@UEAAPEAXI@Z 0000000039a33570 f i CryGameSpySBQR2DLCStore.obj
 0001:00032570       ??_ESTaskLink@CCryGameSpySBQR2FriendsManagement@@UEAAPEAXI@Z 0000000039a33570 f i CryGameSpySBQR2FriendsManagement.obj
 0001:00032570       ??_ESTaskLink@CCryGameSpySBQR2MatchMaking@@UEAAPEAXI@Z 0000000039a33570 f i CryGameSpySBQR2MatchMaking.obj
 0001:00032570       ??_ESCryGameSpySBQR2DLCItemID@@UEAAPEAXI@Z 0000000039a33570 f i CryGameSpySBQR2DLCStore.obj
 0001:00032570       ??_ESSessionLink@CCryGameSpySBQR2MatchMaking@@UEAAPEAXI@Z 0000000039a33570 f i CryGameSpySBQR2MatchMaking.obj
 0001:00032570       ??_GSTaskLink@CCryGameSpySBQR2Friends@@UEAAPEAXI@Z 0000000039a33570 f i CryGameSpySBQR2Friends.obj
 0001:00032570       ??_GSTaskLink@CCryGameSpySBQR2MatchMaking@@UEAAPEAXI@Z 0000000039a33570 f i CryGameSpySBQR2MatchMaking.obj
 0001:00032570       ??_GSThisLink@CCryGameSpySBQR2LobbyService@@UEAAPEAXI@Z 0000000039a33570 f i CryGameSpySBQR2Lobby.obj
 0001:00032570       ??_ESTaskLink@CCryGameSpySBQR2Friends@@UEAAPEAXI@Z 0000000039a33570 f i CryGameSpySBQR2Friends.obj
 0001:00032570       ??_GSCryGameSpySBQR2DLCItemID@@UEAAPEAXI@Z 0000000039a33570 f i CryGameSpySBQR2DLCStore.obj
 0001:00032570       ??_GCMultiThreadRefCount@@UEAAPEAXI@Z 0000000039a33570 f i CryDLCStore.obj
 0001:00032570       ??_GSTaskLink@CCryGameSpySBQR2Stats@@UEAAPEAXI@Z 0000000039a33570 f i CryGameSpySBQR2Stats.obj
 0001:00032570       ??_ESThisLink@CCryGameSpySBQR2Friends@@UEAAPEAXI@Z 0000000039a33570 f i CryGameSpySBQR2Friends.obj
 0001:00032570       ??_GSSessionLink@CCryGameSpySBQR2MatchMaking@@UEAAPEAXI@Z 0000000039a33570 f i CryGameSpySBQR2MatchMaking.obj
 0001:00032570       ??_GSCryGameSpySBQR2DLCDownloadableID@@UEAAPEAXI@Z 0000000039a33570 f i CryGameSpySBQR2DLCStore.obj
 0001:00032570       ??_GSCryGameSpySBQR2DLCPaymentMethodID@@UEAAPEAXI@Z 0000000039a33570 f i CryGameSpySBQR2DLCStore.obj
 0001:00032570       ??_ESCryGameSpySBQR2DLCPaymentMethodID@@UEAAPEAXI@Z 0000000039a33570 f i CryGameSpySBQR2DLCStore.obj
 0001:00032570       ??_ESTaskLink@CCryGameSpySBQR2Stats@@UEAAPEAXI@Z 0000000039a33570 f i CryGameSpySBQR2Stats.obj
 0001:000325a0       ?GetPrivatePort@CCryGameSpySBQR2LobbyService@@QEAAGXZ 0000000039a335a0 f   CryGameSpySBQR2Lobby.obj
 0001:00032660       ?OnInternalSocketChanged@CCryGameSpySBQR2LobbyService@@UEAAXV?$_smart_ptr@UIDatagramSocket@@@@@Z 0000000039a33660 f   CryGameSpySBQR2Lobby.obj
 0001:000326b0       ?InviteAccepted@CCryGameSpySBQR2LobbyService@@QEAAXIV?$_smart_ptr@USCrySessionID@@@@@Z 0000000039a336b0 f   CryGameSpySBQR2Lobby.obj
 0001:00032760       ?QR2NatNegotiateCallback@CCryGameSpySBQR2LobbyService@@CAXHPEAX@Z 0000000039a33760 f   CryGameSpySBQR2Lobby.obj
 0001:00032890       ?AuthServiceStartLogin@CCryGameSpySBQR2LobbyService@@AEAAXXZ 0000000039a33890 f   CryGameSpySBQR2Lobby.obj
 0001:00032960       ?TickQR2@CCryGameSpySBQR2LobbyService@@QEAAXXZ 0000000039a33960 f   CryGameSpySBQR2Lobby.obj
 0001:00032cd0       ??0?$CryStackStringT@D$0BF@@@QEAA@PEBD@Z 0000000039a33cd0 f i CryGameSpySBQR2Lobby.obj
 0001:00032d60       ?clear@?$CryStackStringT@D$0BF@@@QEAAXXZ 0000000039a33d60 f i CryGameSpySBQR2Lobby.obj
 0001:00032dc0       ??0?$CryStackStringT@D$0BP@@@QEAA@PEBD@Z 0000000039a33dc0 f i CryGameSpySBQR2Lobby.obj
 0001:00032e50       ?clear@?$CryStackStringT@D$0BP@@@QEAAXXZ 0000000039a33e50 f i CryGameSpySBQR2Lobby.obj
 0001:00032eb0       ?clear@?$CryStackStringT@D$0DD@@@QEAAXXZ 0000000039a33eb0 f i CryGameSpySBQR2Lobby.obj
 0001:00032f10       ?Execute@?$CClassJobNoRef4@W4ECryLobbySystemEvent@@IW4EOnlineState@@W4ECryLobbyError@@VCCryGameSpySBQR2LobbyService@@@CWorkQueue@@UEAAXXZ 0000000039a33f10 f i CryGameSpySBQR2Lobby.obj
 0001:00032f50       ?Execute@?$CClassJobNoRef@IVCCryLobbyService@@@CWorkQueue@@UEAAXXZ 0000000039a33f50 f i CryLobby.obj
 0001:00032f50       ?Execute@?$CClassJobNoRef@IVCCryGameSpySBQR2LobbyService@@@CWorkQueue@@UEAAXXZ 0000000039a33f50 f i CryGameSpySBQR2Lobby.obj
 0001:00032f80       ?_Assign@?$CryStackStringT@D$0EA@@@QEAAXPEBD_K@Z 0000000039a33f80 f i CryGameSpySBQR2Lobby.obj
 0001:00033020       ?Terminate@CCryGameSpySBQR2LobbyService@@UEAA?AW4ECryLobbyError@@W4ECryLobbyServiceFeatures@@P6AXW42@PEAVCCryLobby@@W4ECryLobbyService@@@Z@Z 0000000039a34020 f   CryGameSpySBQR2Lobby.obj
 0001:00033450       ?InviteAcceptedAcknowledgement@CCryGameSpySBQR2LobbyService@@QEAAXH@Z 0000000039a34450 f   CryGameSpySBQR2Lobby.obj
 0001:00033460       ?SetName@CCryGameSpySBQR2LobbyService@@QEAAXIPEBD@Z 0000000039a34460 f   CryGameSpySBQR2Lobby.obj
 0001:00033570       ?GetUserID@CCryGameSpySBQR2LobbyService@@UEAA?AUCryUserID@@I@Z 0000000039a34570 f   CryGameSpySBQR2Lobby.obj
 0001:000336e0       ?GetProductCredentials@CCryGameSpySBQR2LobbyService@@AEAAXXZ 0000000039a346e0 f   CryGameSpySBQR2Lobby.obj
 0001:00033b30       ?Initialise@CCryGameSpySBQR2LobbyService@@UEAA?AW4ECryLobbyError@@W4ECryLobbyServiceFeatures@@P6AXW42@PEAVCCryLobby@@W4ECryLobbyService@@@Z@Z 0000000039a34b30 f   CryGameSpySBQR2Lobby.obj
 0001:00034050       ??$Add@W4ECryLobbySystemEvent@@IW4EOnlineState@@W4ECryLobbyError@@VCCryGameSpySBQR2LobbyService@@@CWorkQueue@@QEAAXP8CCryGameSpySBQR2LobbyService@@EAAXW4ECryLobbySystemEvent@@IW4EOnlineState@@W4ECryLobbyError@@@ZPEAV1@0I12@Z 0000000039a35050 f i CryGameSpySBQR2Lobby.obj
 0001:00034130       ??1CCryGameSpySBQR2LobbyService@@UEAA@XZ 0000000039a35130 f   CryGameSpySBQR2Lobby.obj
 0001:00034630       ??_ECCryGameSpySBQR2LobbyService@@WBA@EAAPEAXI@Z 0000000039a35630 f i CryGameSpySBQR2Lobby.obj
 0001:00034640       ?LobbyDispatchOnlineStatus@CCryGameSpySBQR2LobbyService@@AEAAXW4ECryLobbySystemEvent@@IW4EOnlineState@@W4ECryLobbyError@@@Z 0000000039a35640 f   CryGameSpySBQR2Lobby.obj
 0001:000346e0       ?StopTaskRunning@CCryGameSpySBQR2LobbyService@@AEAAXI@Z 0000000039a356e0 f   CryGameSpySBQR2Lobby.obj
 0001:00034740       ?StartGetUserPrivileges@CCryGameSpySBQR2LobbyService@@AEAAXI@Z 0000000039a35740 f   CryGameSpySBQR2Lobby.obj
 0001:00034880       ?TickGetUserPrivileges@CCryGameSpySBQR2LobbyService@@AEAAXI@Z 0000000039a35880 f   CryGameSpySBQR2Lobby.obj
 0001:00034a10       ??0CCryGameSpySBQR2LobbyService@@QEAA@PEAVCCryLobby@@W4ECryLobbyService@@@Z 0000000039a35a10 f   CryGameSpySBQR2Lobby.obj
 0001:00034f10       ??_ECCryGameSpySBQR2LobbyService@@UEAAPEAXI@Z 0000000039a35f10 f i CryGameSpySBQR2Lobby.obj
 0001:00034f10       ??_GCCryGameSpySBQR2LobbyService@@UEAAPEAXI@Z 0000000039a35f10 f i CryGameSpySBQR2Lobby.obj
 0001:00034f40       ?Tick@CCryGameSpySBQR2LobbyService@@UEAAXVCTimeValue@@@Z 0000000039a35f40 f   CryGameSpySBQR2Lobby.obj
 0001:000356c0       ?SetOnlineState@CCryGameSpySBQR2LobbyService@@QEAAXIW4EOnlineState@@W4ECryLobbyError@@@Z 0000000039a366c0 f   CryGameSpySBQR2Lobby.obj
 0001:00035790       ?GPErrorCallback@CCryGameSpySBQR2LobbyService@@CAXPEAVCGameSpySBQR2GPConnection@@USResult@2@PEAUGPErrorArg@@PEAUIGameSpyLink@@@Z 0000000039a36790 f   CryGameSpySBQR2Lobby.obj
 0001:000358e0       ?StartTaskRunning@CCryGameSpySBQR2LobbyService@@AEAAXI@Z 0000000039a368e0 f   CryGameSpySBQR2Lobby.obj
 0001:00035950       ?GetUserPrivileges@CCryGameSpySBQR2LobbyService@@UEAA?AW4ECryLobbyError@@IPEAIP6AXIW42@IPEAX@Z2@Z 0000000039a36950 f   CryGameSpySBQR2Lobby.obj
 0001:00035a40       ?GetGPConnection@CCryGameSpySBQR2LobbyService@@QEAAPEAVCGameSpySBQR2GPConnection@@I@Z 0000000039a36a40 f   CryGameSpySBQR2Lobby.obj
 0001:00035af0       ?Initialise@CCryGameSpySBQR2LobbyUI@@QEAA?AW4ECryLobbyError@@XZ 0000000039a36af0 f   CryGameSpySBQR2LobbyUI.obj
 0001:00035b00       ?Terminate@CCryGameSpySBQR2LobbyUI@@QEAA?AW4ECryLobbyError@@XZ 0000000039a36b00 f   CryGameSpySBQR2LobbyUI.obj
 0001:00035b10       ?EndTask@CCryGameSpySBQR2LobbyUI@@IEAAXI@Z 0000000039a36b10 f   CryGameSpySBQR2LobbyUI.obj
 0001:00035bc0       ?ShowFriends@CCryGameSpySBQR2LobbyUI@@UEAA?AW4ECryLobbyError@@IPEAIP6AXIW42@PEAX@Z2@Z 0000000039a36bc0 f   CryGameSpySBQR2LobbyUI.obj
 0001:00035bc0       ?ShowGameInvite@CCryGameSpySBQR2LobbyUI@@UEAA?AW4ECryLobbyError@@IIPEAUCryUserID@@IPEAIP6AXIW42@PEAX@Z3@Z 0000000039a36bc0 f   CryGameSpySBQR2LobbyUI.obj
 0001:00035bf0       ??0CCryGameSpySBQR2LobbyUI@@QEAA@PEAVCCryLobby@@PEAVCCryLobbyService@@@Z 0000000039a36bf0 f   CryGameSpySBQR2LobbyUI.obj
 0001:00035c30       ??_ECCryGameSpySBQR2LobbyUI@@WBA@EAAPEAXI@Z 0000000039a36c30 f i CryGameSpySBQR2LobbyUI.obj
 0001:00035c30       ??_ECCryLobbyUI@@WBA@EAAPEAXI@Z 0000000039a36c30 f i CryLobbyUI.obj
 0001:00035c40       ??_ECCryGameSpySBQR2LobbyUI@@UEAAPEAXI@Z 0000000039a36c40 f i CryGameSpySBQR2LobbyUI.obj
 0001:00035c40       ??_GCCryGameSpySBQR2LobbyUI@@UEAAPEAXI@Z 0000000039a36c40 f i CryGameSpySBQR2LobbyUI.obj
 0001:00035c40       ??_ECCryLobbyUI@@UEAAPEAXI@Z 0000000039a36c40 f i CryLobbyUI.obj
 0001:00035c40       ??_GCCryLobbyUI@@UEAAPEAXI@Z 0000000039a36c40 f i CryLobbyUI.obj
 0001:00035c80       ?ShowGamerCard@CCryGameSpySBQR2LobbyUI@@UEAA?AW4ECryLobbyError@@IUCryUserID@@PEAIP6AXIW42@PEAX@Z3@Z 0000000039a36c80 f   CryGameSpySBQR2LobbyUI.obj
 0001:00035c80       ?ShowFriendRequest@CCryGameSpySBQR2LobbyUI@@UEAA?AW4ECryLobbyError@@IUCryUserID@@PEAIP6AXIW42@PEAX@Z3@Z 0000000039a36c80 f   CryGameSpySBQR2LobbyUI.obj
 0001:00035d10       ?StartShowFriendRequest@CCryGameSpySBQR2LobbyUI@@IEAAXI@Z 0000000039a36d10 f   CryGameSpySBQR2LobbyUI.obj
 0001:00035d10       ?StartShowFriends@CCryGameSpySBQR2LobbyUI@@IEAAXI@Z 0000000039a36d10 f   CryGameSpySBQR2LobbyUI.obj
 0001:00035d10       ?StartShowGameInvite@CCryGameSpySBQR2LobbyUI@@IEAAXI@Z 0000000039a36d10 f   CryGameSpySBQR2LobbyUI.obj
 0001:00035d10       ?StartShowGamerCard@CCryGameSpySBQR2LobbyUI@@IEAAXI@Z 0000000039a36d10 f   CryGameSpySBQR2LobbyUI.obj
 0001:00035d90       ?StartSetRichPresence@CCryGameSpySBQR2LobbyUI@@IEAAXI@Z 0000000039a36d90 f   CryGameSpySBQR2LobbyUI.obj
 0001:00035e60       ?StartTaskRunning@CCryGameSpySBQR2LobbyUI@@IEAAXI@Z 0000000039a36e60 f   CryGameSpySBQR2LobbyUI.obj
 0001:00035f10       ?SetRichPresence@CCryGameSpySBQR2LobbyUI@@UEAA?AW4ECryLobbyError@@IPEAUSCryLobbyUserData@@IPEAIP6AXIW42@PEAX@Z3@Z 0000000039a36f10 f   CryGameSpySBQR2LobbyUI.obj
 0001:00036180       ?ReadString@CCryLobbyPacket@@QEAAXPEADI@Z 0000000039a37180 f i CryGameSpySBQR2MatchMaking.obj
 0001:000361f0       ?ReadCryLobbyUserData@CCryLobbyPacket@@QEAAXPEAUSCryLobbyUserData@@@Z 0000000039a371f0 f i CryGameSpySBQR2MatchMaking.obj
 0001:000362b0       ?WriteToPacket@SCryGameSpySBQR2SessionID@@QEBAXPEAVCCryLobbyPacket@@@Z 0000000039a372b0 f i CryGameSpySBQR2MatchMaking.obj
 0001:00036400       ?ReadFromPacket@SCryGameSpySBQR2SessionID@@QEAAXPEAVCCryLobbyPacket@@@Z 0000000039a37400 f i CryGameSpySBQR2MatchMaking.obj
 0001:00036570       ?ReadError@CCrySharedLobbyPacket@@QEAA?AW4ECryLobbyError@@XZ 0000000039a37570 f i CryGameSpySBQR2MatchMaking.obj
 0001:000365c0       ?OnChangedsv_password@@YAXPEAUICVar@@@Z 0000000039a375c0 f   CryGameSpySBQR2MatchMaking.obj
 0001:000366d0       ?Initialise@CCryGameSpySBQR2MatchMaking@@QEAA?AW4ECryLobbyError@@XZ 0000000039a376d0 f   CryGameSpySBQR2MatchMaking.obj
 0001:000366e0       ?Terminate@CCryGameSpySBQR2MatchMaking@@QEAA?AW4ECryLobbyError@@XZ 0000000039a376e0 f   CryGameSpySBQR2MatchMaking.obj
 0001:000366f0       ?GetSessionIDSizeInPacket@CCryGameSpySBQR2MatchMaking@@UEBAIXZ 0000000039a376f0 f   CryGameSpySBQR2MatchMaking.obj
 0001:00036700       ?ReturnSessionSearch@CCryGameSpySBQR2MatchMaking@@IEAAXP6AXIW4ECryLobbyError@@PEAUSCrySessionSearchResult@@PEAX@ZI012@Z 0000000039a37700 f   CryGameSpySBQR2MatchMaking.obj
 0001:00036720       ?GetLength@CCryFile@@QEAA_KXZ 0000000039a37720 f i CryGameSpySBQR2MatchMaking.obj
 0001:000367e0       ?GetLocalUserName@SSession@CCryGameSpySBQR2MatchMaking@@UEBAPEBDI@Z 0000000039a377e0 f   CryGameSpySBQR2MatchMaking.obj
 0001:00036800       ?GetConnectionName@CCryGameSpySBQR2MatchMaking@@MEBAPEBDPEAUSRConnection@SSession@CCryMatchMaking@@I@Z 0000000039a37800 f   CryGameSpySBQR2MatchMaking.obj
 0001:00036820       ?GetConnectionUserID@CCryGameSpySBQR2MatchMaking@@MEBA_KPEAUSRConnection@SSession@CCryMatchMaking@@I@Z 0000000039a37820 f   CryGameSpySBQR2MatchMaking.obj
 0001:00036840       ?OnGameSpyObjectAvailable@CCryGameSpySBQR2MatchMaking@@UEAAXW4EGameSpyObjectBit@ICryGameSpySBQR2LobbyComponent@@@Z 0000000039a37840 f   CryGameSpySBQR2MatchMaking.obj
 0001:00036870       ?OnGameSpyObjectUnavailable@CCryGameSpySBQR2MatchMaking@@UEAAXW4EGameSpyObjectBit@ICryGameSpySBQR2LobbyComponent@@@Z 0000000039a37870 f   CryGameSpySBQR2MatchMaking.obj
 0001:000368a0       ?OnGameSpyObjectCantMakeAvailable@CCryGameSpySBQR2MatchMaking@@UEAAXW4EGameSpyObjectBit@ICryGameSpySBQR2LobbyComponent@@@Z 0000000039a378a0 f   CryGameSpySBQR2MatchMaking.obj
 0001:00036910       ?CheckTaskGameSpyObjects@CCryGameSpySBQR2MatchMaking@@IEAA?AW4ETaskGameSpyCheckResult@ICryGameSpySBQR2LobbyComponent@@I@Z 0000000039a37910 f   CryGameSpySBQR2MatchMaking.obj
 0001:000369a0       ?EndSessionSendRequestInfo@CCryGameSpySBQR2MatchMaking@@IEAAXI@Z 0000000039a379a0 f   CryGameSpySBQR2MatchMaking.obj
 0001:00036a00       ?DispatchSessionRequestInfo@CCryGameSpySBQR2MatchMaking@@IEAAXIIII@Z 0000000039a37a00 f   CryGameSpySBQR2MatchMaking.obj
 0001:00036a90       ?CreateChallengeString@CCryGameSpySBQR2MatchMaking@@SAXPEAD@Z 0000000039a37a90 f   CryGameSpySBQR2MatchMaking.obj
 0001:00036b40       ?TranslateCDKeyError@CCryGameSpySBQR2MatchMaking@@SA?AW4ECryLobbyError@@PEAD@Z 0000000039a37b40 f   CryGameSpySBQR2MatchMaking.obj
 0001:00036c50       ?ImportHostName@CCryGameSpySBQR2MatchMaking@@IEAAXPEAUSServer@SSearch@1@PEAUSGameSpyKey@1@I@Z 0000000039a37c50 f   CryGameSpySBQR2MatchMaking.obj
 0001:00036c90       ?ExportGameTitle@CCryGameSpySBQR2MatchMaking@@IEAAXV?$CryLobbyID@USCryLobbySessionHandle@@$03@@PEAUSGameSpyKey@1@IPEAUqr2_buffer_s@@@Z 0000000039a37c90 f   CryGameSpySBQR2MatchMaking.obj
 0001:00036cc0       ?ImportNumPlayers@CCryGameSpySBQR2MatchMaking@@IEAAXPEAUSServer@SSearch@1@PEAUSGameSpyKey@1@I@Z 0000000039a37cc0 f   CryGameSpySBQR2MatchMaking.obj
 0001:00036cf0       ?ImportPasswordRequired@CCryGameSpySBQR2MatchMaking@@IEAAXPEAUSServer@SSearch@1@PEAUSGameSpyKey@1@I@Z 0000000039a37cf0 f   CryGameSpySBQR2MatchMaking.obj
 0001:00036d30       ?ExportPasswordRequired@CCryGameSpySBQR2MatchMaking@@IEAAXV?$CryLobbyID@USCryLobbySessionHandle@@$03@@PEAUSGameSpyKey@1@IPEAUqr2_buffer_s@@@Z 0000000039a37d30 f   CryGameSpySBQR2MatchMaking.obj
 0001:00036da0       ?ImportNumPublicSlots@CCryGameSpySBQR2MatchMaking@@IEAAXPEAUSServer@SSearch@1@PEAUSGameSpyKey@1@I@Z 0000000039a37da0 f   CryGameSpySBQR2MatchMaking.obj
 0001:00036dd0       ?ImportNumPrivateSlots@CCryGameSpySBQR2MatchMaking@@IEAAXPEAUSServer@SSearch@1@PEAUSGameSpyKey@1@I@Z 0000000039a37dd0 f   CryGameSpySBQR2MatchMaking.obj
 0001:00036e00       ?ImportRanked@CCryGameSpySBQR2MatchMaking@@IEAAXPEAUSServer@SSearch@1@PEAUSGameSpyKey@1@I@Z 0000000039a37e00 f   CryGameSpySBQR2MatchMaking.obj
 0001:00036e30       ?ImportCreateFlags@CCryGameSpySBQR2MatchMaking@@IEAAXPEAUSServer@SSearch@1@PEAUSGameSpyKey@1@I@Z 0000000039a37e30 f   CryGameSpySBQR2MatchMaking.obj
 0001:00036e60       ?ImportNumMigrations@CCryGameSpySBQR2MatchMaking@@IEAAXPEAUSServer@SSearch@1@PEAUSGameSpyKey@1@I@Z 0000000039a37e60 f   CryGameSpySBQR2MatchMaking.obj
 0001:00036e90       ?ImportDedicated@CCryGameSpySBQR2MatchMaking@@IEAAXPEAUSServer@SSearch@1@PEAUSGameSpyKey@1@I@Z 0000000039a37e90 f   CryGameSpySBQR2MatchMaking.obj
 0001:00036ec0       ?ExportDedicated@CCryGameSpySBQR2MatchMaking@@IEAAXV?$CryLobbyID@USCryLobbySessionHandle@@$03@@PEAUSGameSpyKey@1@IPEAUqr2_buffer_s@@@Z 0000000039a37ec0 f   CryGameSpySBQR2MatchMaking.obj
 0001:00036ef0       ?ExportHostUserID@CCryGameSpySBQR2MatchMaking@@IEAAXV?$CryLobbyID@USCryLobbySessionHandle@@$03@@PEAUSGameSpyKey@1@IPEAUqr2_buffer_s@@@Z 0000000039a37ef0 f   CryGameSpySBQR2MatchMaking.obj
 0001:00036f20       ??A?$CryLobbyIDArray@USRConnection@SSession@CCryGameSpySBQR2MatchMaking@@V?$CryLobbyID@USCryMatchMakingConnectionID@@$0EA@@@$0EA@@@QEAAAEAUSRConnection@SSession@CCryGameSpySBQR2MatchMaking@@AEBV?$CryLobbyID@USCryMatchMakingConnectionID@@$0EA@@@@Z 0000000039a37f20 f i CryGameSpySBQR2MatchMaking.obj
 0001:00036f60       ??A?$CryLobbyIDArray@USSession@CCryGameSpySBQR2MatchMaking@@V?$CryLobbyID@USCryLobbySessionHandle@@$03@@$03@@QEAAAEAUSSession@CCryGameSpySBQR2MatchMaking@@AEBV?$CryLobbyID@USCryLobbySessionHandle@@$03@@@Z 0000000039a37f60 f i CryGameSpySBQR2MatchMaking.obj
 0001:00036fa0       ?_AllocData@?$CryStackStringT@D$0EJ@@@QEAAX_K@Z 0000000039a37fa0 f i CryGameSpySBQR2MatchMaking.obj
 0001:00037020       ?Clone@?$VTableImpl@G$0A@U?$IVisitor@V?$CNode@USNullAddr@@V?$CNode@GV?$CNode@USIPv4Addr@@V?$CNode@ULobbyIdAddr@@VCEnd@NTypelist@@@NTypelist@@@NTypelist@@@NTypelist@@@NTypelist@@@NConfigurableVariantHelpers@@U?$IMutatingVisitor@V?$CNode@USNullAddr@@V?$CNode@GV?$CNode@USIPv4Addr@@V?$CNode@ULobbyIdAddr@@VCEnd@NTypelist@@@NTypelist@@@NTypelist@@@NTypelist@@@NTypelist@@@2@@NConfigurableVariantHelpers@@SAXPEAXPEBX@Z 0000000039a38020 f i CryGameSpySBQR2MatchMaking.obj
 0001:00037030       ?ConstructClone@?$VTableImpl@G$0A@U?$IVisitor@V?$CNode@USNullAddr@@V?$CNode@GV?$CNode@USIPv4Addr@@V?$CNode@ULobbyIdAddr@@VCEnd@NTypelist@@@NTypelist@@@NTypelist@@@NTypelist@@@NTypelist@@@NConfigurableVariantHelpers@@U?$IMutatingVisitor@V?$CNode@USNullAddr@@V?$CNode@GV?$CNode@USIPv4Addr@@V?$CNode@ULobbyIdAddr@@VCEnd@NTypelist@@@NTypelist@@@NTypelist@@@NTypelist@@@NTypelist@@@2@@NConfigurableVariantHelpers@@SAXPEAXPEBX@Z 0000000039a38030 f i CryGameSpySBQR2MatchMaking.obj
 0001:00037040       ?MutatingVisit@?$VTableImpl@G$0A@U?$IVisitor@V?$CNode@USNullAddr@@V?$CNode@GV?$CNode@USIPv4Addr@@V?$CNode@ULobbyIdAddr@@VCEnd@NTypelist@@@NTypelist@@@NTypelist@@@NTypelist@@@NTypelist@@@NConfigurableVariantHelpers@@U?$IMutatingVisitor@V?$CNode@USNullAddr@@V?$CNode@GV?$CNode@USIPv4Addr@@V?$CNode@ULobbyIdAddr@@VCEnd@NTypelist@@@NTypelist@@@NTypelist@@@NTypelist@@@NTypelist@@@2@@NConfigurableVariantHelpers@@SAXPEAU?$IMutatingVisitor@V?$CNode@USNullAddr@@V?$CNode@GV?$CNode@USIPv4Addr@@V?$CNode@ULobbyIdAddr@@VCEnd@NTypelist@@@NTypelist@@@NTypelist@@@NTypelist@@@NTypelist@@@2@PEAX1@Z 0000000039a38040 f i CryGameSpySBQR2MatchMaking.obj
 0001:00037040       ?Visit@?$VTableImpl@G$0A@U?$IVisitor@V?$CNode@USNullAddr@@V?$CNode@GV?$CNode@USIPv4Addr@@V?$CNode@ULobbyIdAddr@@VCEnd@NTypelist@@@NTypelist@@@NTypelist@@@NTypelist@@@NTypelist@@@NConfigurableVariantHelpers@@U?$IMutatingVisitor@V?$CNode@USNullAddr@@V?$CNode@GV?$CNode@USIPv4Addr@@V?$CNode@ULobbyIdAddr@@VCEnd@NTypelist@@@NTypelist@@@NTypelist@@@NTypelist@@@NTypelist@@@2@@NConfigurableVariantHelpers@@SAXPEAU?$IVisitor@V?$CNode@USNullAddr@@V?$CNode@GV?$CNode@USIPv4Addr@@V?$CNode@ULobbyIdAddr@@VCEnd@NTypelist@@@NTypelist@@@NTypelist@@@NTypelist@@@NTypelist@@@2@PEBXPEAX@Z 0000000039a38040 f i CryGameSpySBQR2MatchMaking.obj
 0001:00037060       ??4SCryLobbyUserData@@QEAAAEBU0@AEBU0@@Z 0000000039a38060 f i CryGameSpySBQR2MatchMaking.obj
 0001:00037110       ??_GSSession@CCryMatchMaking@@UEAAPEAXI@Z 0000000039a38110 f i CryGameSpySBQR2MatchMaking.obj
 0001:00037110       ??_GIDatagramListener@@UEAAPEAXI@Z 0000000039a38110 f i CryLobby.obj
 0001:00037110       ??_EICryFriends@@UEAAPEAXI@Z 0000000039a38110 f i CryFriends.obj
 0001:00037110       ??_GICryFriends@@UEAAPEAXI@Z 0000000039a38110 f i CryFriends.obj
 0001:00037110       ??_EIDatagramListener@@UEAAPEAXI@Z 0000000039a38110 f i CryLobby.obj
 0001:00037110       ??_ESSession@CCryMatchMaking@@UEAAPEAXI@Z 0000000039a38110 f i CryGameSpySBQR2MatchMaking.obj
 0001:00037140       ?ProcessPropagatePassword@CCryGameSpySBQR2MatchMaking@@QEAAXAEBV?$CConfigurableVariant@V?$CNode@USNullAddr@@V?$CNode@GV?$CNode@USIPv4Addr@@V?$CNode@ULobbyIdAddr@@VCEnd@NTypelist@@@NTypelist@@@NTypelist@@@NTypelist@@@NTypelist@@$07VCDefaultVariantConversion@NConfigurableVariantHelpers@@VCDefaultVariantConstruction@4@@@PEAVCCrySharedLobbyPacket@@@Z 0000000039a38140 f   CryGameSpySBQR2MatchMaking.obj
 0001:00037250       ?StartSessionCreate@CCryGameSpySBQR2MatchMaking@@IEAAXI@Z 0000000039a38250 f   CryGameSpySBQR2MatchMaking.obj
 0001:00037300       ?StartSessionUpdate@CCryGameSpySBQR2MatchMaking@@IEAAXI@Z 0000000039a38300 f   CryGameSpySBQR2MatchMaking.obj
 0001:00037390       ?ProcessServerData@CCryGameSpySBQR2MatchMaking@@IEAAXAEBV?$CConfigurableVariant@V?$CNode@USNullAddr@@V?$CNode@GV?$CNode@USIPv4Addr@@V?$CNode@ULobbyIdAddr@@VCEnd@NTypelist@@@NTypelist@@@NTypelist@@@NTypelist@@@NTypelist@@$07VCDefaultVariantConversion@NConfigurableVariantHelpers@@VCDefaultVariantConstruction@4@@@PEAVCCrySharedLobbyPacket@@@Z 0000000039a38390 f   CryGameSpySBQR2MatchMaking.obj
 0001:00037550       ?CalculateServerDataSize@CCryGameSpySBQR2MatchMaking@@IEAAIV?$CryLobbyID@USCryLobbySessionHandle@@$03@@@Z 0000000039a38550 f   CryGameSpySBQR2MatchMaking.obj
 0001:00037620       ?EndSessionCreate@CCryGameSpySBQR2MatchMaking@@IEAAXI@Z 0000000039a38620 f   CryGameSpySBQR2MatchMaking.obj
 0001:00037710       ?NATNegotiateProgressCallback@CCryGameSpySBQR2MatchMaking@@KAXUSResult@CGameSpySBQR2NATNegotiation@@HPEAUIGameSpyLink@@@Z 0000000039a38710 f   CryGameSpySBQR2MatchMaking.obj
 0001:00037780       ?CompleteNATNegotiation@CCryGameSpySBQR2MatchMaking@@KA_NW4NegotiateResult@@IPEAUSCryGameSpySBQR2RemoteConnectionID@@PEAUSRConnection@SSession@1@PEAUsockaddr_in@@@Z 0000000039a38780 f   CryGameSpySBQR2MatchMaking.obj
 0001:000378a0       ?CreateNATCookie@CCryGameSpySBQR2MatchMaking@@IEAAIPEAUSCryGameSpySBQR2RemoteConnectionID@@@Z 0000000039a388a0 f   CryGameSpySBQR2MatchMaking.obj
 0001:000378e0       ?FilterKey@CCryGameSpySBQR2MatchMaking@@KA_NPEAUSCryLobbyUserData@@PEAUSCrySessionSearchData@@@Z 0000000039a388e0 f   CryGameSpySBQR2MatchMaking.obj
 0001:00037bc0       ?Close@CCryFile@@QEAAXXZ   0000000039a38bc0 f i CryGameSpySBQR2MatchMaking.obj
 0001:00037c20       ?GetSIDFromSessionHandle@CCryGameSpySBQR2MatchMaking@@UEAA_KV?$CryLobbyID@USCryLobbySessionHandle@@$03@@@Z 0000000039a38c20 f   CryGameSpySBQR2MatchMaking.obj
 0001:00037c60       ?FindSessionFromSessionID@CCryGameSpySBQR2MatchMaking@@IEAA?AV?$CryLobbyID@USCryLobbySessionHandle@@$03@@_K@Z 0000000039a38c60 f   CryGameSpySBQR2MatchMaking.obj
 0001:00037d30       ?InformVoiceRemoteUsersLeft@CCryGameSpySBQR2MatchMaking@@IEAAXV?$CryLobbyID@USCryLobbySessionHandle@@$03@@V?$CryLobbyID@USCryMatchMakingConnectionID@@$0EA@@@@Z 0000000039a38d30 f   CryGameSpySBQR2MatchMaking.obj
 0001:00037dd0       ?GetCurrentInvitableSessionHandle@CCryGameSpySBQR2MatchMaking@@QEBA?AV?$CryLobbyID@USCryLobbySessionHandle@@$03@@XZ 0000000039a38dd0 f   CryGameSpySBQR2MatchMaking.obj
 0001:00037e70       ?SessionSendRequestInfoResponseNT@CCryGameSpySBQR2MatchMaking@@IEAAXIII@Z 0000000039a38e70 f   CryGameSpySBQR2MatchMaking.obj
 0001:00037f00       ?GetSessionIDFromSessionURL@CCryGameSpySBQR2MatchMaking@@UEAA?AW4ECryLobbyError@@QEBDQEAV?$_smart_ptr@USCrySessionID@@@@@Z 0000000039a38f00 f   CryGameSpySBQR2MatchMaking.obj
 0001:00037ff0       ?CDKeyAuthCallback@CCryGameSpySBQR2MatchMaking@@KAXHHHPEADPEAX@Z 0000000039a38ff0 f   CryGameSpySBQR2MatchMaking.obj
 0001:00038220       ?GetNameFromGameSessionHandle@CCryGameSpySBQR2MatchMaking@@UEAAPEBDI@Z 0000000039a39220 f   CryGameSpySBQR2MatchMaking.obj
 0001:00038310       ?ExportHostName@CCryGameSpySBQR2MatchMaking@@IEAAXV?$CryLobbyID@USCryLobbySessionHandle@@$03@@PEAUSGameSpyKey@1@IPEAUqr2_buffer_s@@@Z 0000000039a39310 f   CryGameSpySBQR2MatchMaking.obj
 0001:00038360       ?ExportNumPlayers@CCryGameSpySBQR2MatchMaking@@IEAAXV?$CryLobbyID@USCryLobbySessionHandle@@$03@@PEAUSGameSpyKey@1@IPEAUqr2_buffer_s@@@Z 0000000039a39360 f   CryGameSpySBQR2MatchMaking.obj
 0001:000383b0       ?ExportMaxPlayers@CCryGameSpySBQR2MatchMaking@@IEAAXV?$CryLobbyID@USCryLobbySessionHandle@@$03@@PEAUSGameSpyKey@1@IPEAUqr2_buffer_s@@@Z 0000000039a393b0 f   CryGameSpySBQR2MatchMaking.obj
 0001:00038420       ?ImportGameState@CCryGameSpySBQR2MatchMaking@@IEAAXPEAUSServer@SSearch@1@PEAUSGameSpyKey@1@I@Z 0000000039a39420 f   CryGameSpySBQR2MatchMaking.obj
 0001:00038670       ?ExportGameState@CCryGameSpySBQR2MatchMaking@@IEAAXV?$CryLobbyID@USCryLobbySessionHandle@@$03@@PEAUSGameSpyKey@1@IPEAUqr2_buffer_s@@@Z 0000000039a39670 f   CryGameSpySBQR2MatchMaking.obj
 0001:000387f0       ?ImportSessionID@CCryGameSpySBQR2MatchMaking@@IEAAXPEAUSServer@SSearch@1@PEAUSGameSpyKey@1@I@Z 0000000039a397f0 f   CryGameSpySBQR2MatchMaking.obj
 0001:00038860       ?ExportSessionID@CCryGameSpySBQR2MatchMaking@@IEAAXV?$CryLobbyID@USCryLobbySessionHandle@@$03@@PEAUSGameSpyKey@1@IPEAUqr2_buffer_s@@@Z 0000000039a39860 f   CryGameSpySBQR2MatchMaking.obj
 0001:000388c0       ?ExportNumPublicSlots@CCryGameSpySBQR2MatchMaking@@IEAAXV?$CryLobbyID@USCryLobbySessionHandle@@$03@@PEAUSGameSpyKey@1@IPEAUqr2_buffer_s@@@Z 0000000039a398c0 f   CryGameSpySBQR2MatchMaking.obj
 0001:00038910       ?ExportNumPrivateSlots@CCryGameSpySBQR2MatchMaking@@IEAAXV?$CryLobbyID@USCryLobbySessionHandle@@$03@@PEAUSGameSpyKey@1@IPEAUqr2_buffer_s@@@Z 0000000039a39910 f   CryGameSpySBQR2MatchMaking.obj
 0001:00038960       ?ExportRanked@CCryGameSpySBQR2MatchMaking@@IEAAXV?$CryLobbyID@USCryLobbySessionHandle@@$03@@PEAUSGameSpyKey@1@IPEAUqr2_buffer_s@@@Z 0000000039a39960 f   CryGameSpySBQR2MatchMaking.obj
 0001:000389b0       ?ExportCreateFlags@CCryGameSpySBQR2MatchMaking@@IEAAXV?$CryLobbyID@USCryLobbySessionHandle@@$03@@PEAUSGameSpyKey@1@IPEAUqr2_buffer_s@@@Z 0000000039a399b0 f   CryGameSpySBQR2MatchMaking.obj
 0001:00038a00       ?ExportNumMigrations@CCryGameSpySBQR2MatchMaking@@IEAAXV?$CryLobbyID@USCryLobbySessionHandle@@$03@@PEAUSGameSpyKey@1@IPEAUqr2_buffer_s@@@Z 0000000039a39a00 f   CryGameSpySBQR2MatchMaking.obj
 0001:00038a50       ?ImportServerInt8@CCryGameSpySBQR2MatchMaking@@IEAAXPEAUSServer@SSearch@1@PEAUSGameSpyKey@1@I@Z 0000000039a39a50 f   CryGameSpySBQR2MatchMaking.obj
 0001:00038a90       ?ExportServerInt8@CCryGameSpySBQR2MatchMaking@@IEAAXV?$CryLobbyID@USCryLobbySessionHandle@@$03@@PEAUSGameSpyKey@1@IPEAUqr2_buffer_s@@@Z 0000000039a39a90 f   CryGameSpySBQR2MatchMaking.obj
 0001:00038af0       ?ImportServerInt16@CCryGameSpySBQR2MatchMaking@@IEAAXPEAUSServer@SSearch@1@PEAUSGameSpyKey@1@I@Z 0000000039a39af0 f   CryGameSpySBQR2MatchMaking.obj
 0001:00038b40       ?ExportServerInt16@CCryGameSpySBQR2MatchMaking@@IEAAXV?$CryLobbyID@USCryLobbySessionHandle@@$03@@PEAUSGameSpyKey@1@IPEAUqr2_buffer_s@@@Z 0000000039a39b40 f   CryGameSpySBQR2MatchMaking.obj
 0001:00038ba0       ?ImportServerInt32@CCryGameSpySBQR2MatchMaking@@IEAAXPEAUSServer@SSearch@1@PEAUSGameSpyKey@1@I@Z 0000000039a39ba0 f   CryGameSpySBQR2MatchMaking.obj
 0001:00038ba0       ?ImportHostUserID@CCryGameSpySBQR2MatchMaking@@IEAAXPEAUSServer@SSearch@1@PEAUSGameSpyKey@1@I@Z 0000000039a39ba0 f   CryGameSpySBQR2MatchMaking.obj
 0001:00038be0       ?ExportServerInt32@CCryGameSpySBQR2MatchMaking@@IEAAXV?$CryLobbyID@USCryLobbySessionHandle@@$03@@PEAUSGameSpyKey@1@IPEAUqr2_buffer_s@@@Z 0000000039a39be0 f   CryGameSpySBQR2MatchMaking.obj
 0001:00038c40       ?ImportServerInt64@CCryGameSpySBQR2MatchMaking@@IEAAXPEAUSServer@SSearch@1@PEAUSGameSpyKey@1@I@Z 0000000039a39c40 f   CryGameSpySBQR2MatchMaking.obj
 0001:00038cd0       ?ExportServerInt64@CCryGameSpySBQR2MatchMaking@@IEAAXV?$CryLobbyID@USCryLobbySessionHandle@@$03@@PEAUSGameSpyKey@1@IPEAUqr2_buffer_s@@@Z 0000000039a39cd0 f   CryGameSpySBQR2MatchMaking.obj
 0001:00038d50       ?ImportServerFloat32@CCryGameSpySBQR2MatchMaking@@IEAAXPEAUSServer@SSearch@1@PEAUSGameSpyKey@1@I@Z 0000000039a39d50 f   CryGameSpySBQR2MatchMaking.obj
 0001:00038da0       ?ExportServerFloat32@CCryGameSpySBQR2MatchMaking@@IEAAXV?$CryLobbyID@USCryLobbySessionHandle@@$03@@PEAUSGameSpyKey@1@IPEAUqr2_buffer_s@@@Z 0000000039a39da0 f   CryGameSpySBQR2MatchMaking.obj
 0001:00038e20       ?ImportServerFloat64@CCryGameSpySBQR2MatchMaking@@IEAAXPEAUSServer@SSearch@1@PEAUSGameSpyKey@1@I@Z 0000000039a39e20 f   CryGameSpySBQR2MatchMaking.obj
 0001:00038e60       ?ExportServerFloat64@CCryGameSpySBQR2MatchMaking@@IEAAXV?$CryLobbyID@USCryLobbySessionHandle@@$03@@PEAUSGameSpyKey@1@IPEAUqr2_buffer_s@@@Z 0000000039a39e60 f   CryGameSpySBQR2MatchMaking.obj
 0001:00038ee0       ?ExportServerHash@CCryGameSpySBQR2MatchMaking@@IEAAXV?$CryLobbyID@USCryLobbySessionHandle@@$03@@PEAUSGameSpyKey@1@IPEAUqr2_buffer_s@@@Z 0000000039a39ee0 f   CryGameSpySBQR2MatchMaking.obj
 0001:00039020       ?ImportPlayerIndex@CCryGameSpySBQR2MatchMaking@@IEAAHV?$CryLobbyID@USCryLobbySessionHandle@@$03@@H@Z 0000000039a3a020 f   CryGameSpySBQR2MatchMaking.obj
 0001:00039120       ??A?$CryLobbyIDArray@USSearch@CCryGameSpySBQR2MatchMaking@@V?$CryLobbyID@USCryGSSearchHandle@CCryGameSpySBQR2MatchMaking@@$00@@$00@@QEAAAEAUSSearch@CCryGameSpySBQR2MatchMaking@@AEBV?$CryLobbyID@USCryGSSearchHandle@CCryGameSpySBQR2MatchMaking@@$00@@@Z 0000000039a3a120 f i CryGameSpySBQR2MatchMaking.obj
 0001:00039160       ?_Rebalance_for_erase@?$_Rb_global@_N@priv@stlpmtx_std@@SAPEAU_Rb_tree_node_base@23@PEAU423@AEAPEAU423@11@Z 0000000039a3a160 f i CryGameSpySBQR2MatchMaking.obj
 0001:000394b0       ?_AllocData@?$CryStackStringT@D$0BPP@@@QEAAX_K@Z 0000000039a3a4b0 f i CryGameSpySBQR2MatchMaking.obj
 0001:00039530       ??1SGameSpyKey@CCryGameSpySBQR2MatchMaking@@UEAA@XZ 0000000039a3a530 f i CryGameSpySBQR2MatchMaking.obj
 0001:000395f0       ??_GSGameSpyKey@CCryGameSpySBQR2MatchMaking@@UEAAPEAXI@Z 0000000039a3a5f0 f i CryGameSpySBQR2MatchMaking.obj
 0001:000395f0       ??_ESGameSpyKey@CCryGameSpySBQR2MatchMaking@@UEAAPEAXI@Z 0000000039a3a5f0 f i CryGameSpySBQR2MatchMaking.obj
 0001:00039620       ??1SRegisteredLobbyData@CCryGameSpySBQR2MatchMaking@@UEAA@XZ 0000000039a3a620 f i CryGameSpySBQR2MatchMaking.obj
 0001:000396c0       ?Kick@CCryGameSpySBQR2MatchMaking@@UEAAXPEBUCryUserID@@W4EDisconnectionCause@@@Z 0000000039a3a6c0 f   CryGameSpySBQR2MatchMaking.obj
 0001:000396f0       ?ResetTask@CCryGameSpySBQR2MatchMaking@@IEAAXI@Z 0000000039a3a6f0 f   CryGameSpySBQR2MatchMaking.obj
 0001:000397a0       ?SendServerData@CCryGameSpySBQR2MatchMaking@@IEAAXAEBV?$CConfigurableVariant@V?$CNode@USNullAddr@@V?$CNode@GV?$CNode@USIPv4Addr@@V?$CNode@ULobbyIdAddr@@VCEnd@NTypelist@@@NTypelist@@@NTypelist@@@NTypelist@@@NTypelist@@$07VCDefaultVariantConversion@NConfigurableVariantHelpers@@VCDefaultVariantConstruction@4@@@PEAVCCrySharedLobbyPacket@@@Z 0000000039a3a7a0 f   CryGameSpySBQR2MatchMaking.obj
 0001:00039d00       ?SessionJoinNNComplete@CCryGameSpySBQR2MatchMaking@@KAXUSResult@CGameSpySBQR2NATNegotiation@@H_KPEAUsockaddr_in@@PEAUIGameSpyLink@@@Z 0000000039a3ad00 f   CryGameSpySBQR2MatchMaking.obj
 0001:00039dc0       ?SessionSearchNNComplete@CCryGameSpySBQR2MatchMaking@@KAXUSResult@CGameSpySBQR2NATNegotiation@@H_KPEAUsockaddr_in@@PEAUIGameSpyLink@@@Z 0000000039a3adc0 f   CryGameSpySBQR2MatchMaking.obj
 0001:00039eb0       ?SessionSendRequestInfoNNComplete@CCryGameSpySBQR2MatchMaking@@KAXUSResult@CGameSpySBQR2NATNegotiation@@H_KPEAUsockaddr_in@@PEAUIGameSpyLink@@@Z 0000000039a3aeb0 f   CryGameSpySBQR2MatchMaking.obj
 0001:00039f40       ?StartFindUseAddress@CCryGameSpySBQR2MatchMaking@@IEAAXPEAUSCryGameSpySBQR2RemoteConnectionID@@IH_NP6AXUSResult@CGameSpySBQR2NATNegotiation@@H_KPEAUsockaddr_in@@PEAUIGameSpyLink@@@Z5@Z 0000000039a3af40 f   CryGameSpySBQR2MatchMaking.obj
 0001:0003a1e0       ?EndSessionSearch@CCryGameSpySBQR2MatchMaking@@IEAAXI@Z 0000000039a3b1e0 f   CryGameSpySBQR2MatchMaking.obj
 0001:0003a240       ?Ban@CCryGameSpySBQR2MatchMaking@@MEAAXPEBUCryUserID@@M@Z 0000000039a3b240 f   CryGameSpySBQR2MatchMaking.obj
 0001:0003a2c0       ?GetCurrentSessionPlayerCount@CCryGameSpySBQR2MatchMaking@@QEAAIXZ 0000000039a3b2c0 f   CryGameSpySBQR2MatchMaking.obj
 0001:0003a320       ?ClearSessionSearchServer@CCryGameSpySBQR2MatchMaking@@KAXPEAUSServer@SSearch@1@@Z 0000000039a3b320 f   CryGameSpySBQR2MatchMaking.obj
 0001:0003a3e0       ?MoveSessionSearchServer@CCryGameSpySBQR2MatchMaking@@KAXPEAUSServer@SSearch@1@0@Z 0000000039a3b3e0 f   CryGameSpySBQR2MatchMaking.obj
 0001:0003a500       ?ProcessSessionPing@CCryGameSpySBQR2MatchMaking@@IEAAXAEBV?$CConfigurableVariant@V?$CNode@USNullAddr@@V?$CNode@GV?$CNode@USIPv4Addr@@V?$CNode@ULobbyIdAddr@@VCEnd@NTypelist@@@NTypelist@@@NTypelist@@@NTypelist@@@NTypelist@@$07VCDefaultVariantConversion@NConfigurableVariantHelpers@@VCDefaultVariantConstruction@4@@@PEAVCCrySharedLobbyPacket@@@Z 0000000039a3b500 f   CryGameSpySBQR2MatchMaking.obj
 0001:0003a700       ?ProcessSessionPong@CCryGameSpySBQR2MatchMaking@@IEAAXAEBV?$CConfigurableVariant@V?$CNode@USNullAddr@@V?$CNode@GV?$CNode@USIPv4Addr@@V?$CNode@ULobbyIdAddr@@VCEnd@NTypelist@@@NTypelist@@@NTypelist@@@NTypelist@@@NTypelist@@$07VCDefaultVariantConversion@NConfigurableVariantHelpers@@VCDefaultVariantConstruction@4@@@PEAVCCrySharedLobbyPacket@@@Z 0000000039a3b700 f   CryGameSpySBQR2MatchMaking.obj
 0001:0003a850       ?AdjustSessionFriendCount@CCryGameSpySBQR2MatchMaking@@QEAAXPEBDH@Z 0000000039a3b850 f   CryGameSpySBQR2MatchMaking.obj
 0001:0003a9a0       ?StartSessionSendRequestInfo@CCryGameSpySBQR2MatchMaking@@IEAAXI@Z 0000000039a3b9a0 f   CryGameSpySBQR2MatchMaking.obj
 0001:0003aa40       ??4SCrySessionInfoRequester@@QEAAAEAU0@AEBU0@@Z 0000000039a3ba40 f i CryGameSpySBQR2MatchMaking.obj
 0001:0003aa80       ?GetSessionIDFromConsole@CCryGameSpySBQR2MatchMaking@@UEAA?AV?$_smart_ptr@USCrySessionID@@@@XZ 0000000039a3ba80 f   CryGameSpySBQR2MatchMaking.obj
 0001:0003ab10       ?GetSessionAddressFromSessionID@CCryGameSpySBQR2MatchMaking@@UEAA?AW4ECryLobbyError@@V?$_smart_ptr@USCrySessionID@@@@AEAIAEAG@Z 0000000039a3bb10 f   CryGameSpySBQR2MatchMaking.obj
 0001:0003abb0       ?ProcessCDKeyChallenge@CCryGameSpySBQR2MatchMaking@@IEAAXAEBV?$CConfigurableVariant@V?$CNode@USNullAddr@@V?$CNode@GV?$CNode@USIPv4Addr@@V?$CNode@ULobbyIdAddr@@VCEnd@NTypelist@@@NTypelist@@@NTypelist@@@NTypelist@@@NTypelist@@$07VCDefaultVariantConversion@NConfigurableVariantHelpers@@VCDefaultVariantConstruction@4@@@PEAVCCrySharedLobbyPacket@@@Z 0000000039a3bbb0 f   CryGameSpySBQR2MatchMaking.obj
 0001:0003ae90       ?SessionJoinFail@CCryGameSpySBQR2MatchMaking@@IEAAX_KW4ECryLobbyError@@IAEBV?$CConfigurableVariant@V?$CNode@USNullAddr@@V?$CNode@GV?$CNode@USIPv4Addr@@V?$CNode@ULobbyIdAddr@@VCEnd@NTypelist@@@NTypelist@@@NTypelist@@@NTypelist@@@NTypelist@@$07VCDefaultVariantConversion@NConfigurableVariantHelpers@@VCDefaultVariantConstruction@4@@@@Z 0000000039a3be90 f   CryGameSpySBQR2MatchMaking.obj
 0001:0003b020       ?ExportPlayerName@CCryGameSpySBQR2MatchMaking@@IEAAXV?$CryLobbyID@USCryLobbySessionHandle@@$03@@PEAUSGameSpyKey@1@IPEAUqr2_buffer_s@@@Z 0000000039a3c020 f   CryGameSpySBQR2MatchMaking.obj
 0001:0003b100       ?ExportPlayerID@CCryGameSpySBQR2MatchMaking@@IEAAXV?$CryLobbyID@USCryLobbySessionHandle@@$03@@PEAUSGameSpyKey@1@IPEAUqr2_buffer_s@@@Z 0000000039a3c100 f   CryGameSpySBQR2MatchMaking.obj
 0001:0003b1d0       ?FreeSessionHandle@CCryGameSpySBQR2MatchMaking@@MEAAXV?$CryLobbyID@USCryLobbySessionHandle@@$03@@@Z 0000000039a3c1d0 f   CryGameSpySBQR2MatchMaking.obj
 0001:0003b2a0       ?_M_compute_next_size@?$_Impl_vector@USCrySessionSearchData@@V?$allocator@USCrySessionSearchData@@@stlpmtx_std@@@priv@stlpmtx_std@@AEAA_K_K@Z 0000000039a3c2a0 f i CryGameSpySBQR2MatchMaking.obj
 0001:0003b2a0       ?_M_compute_next_size@?$_Impl_vector@USEventCBData@CCryLobby@@V?$allocator@USEventCBData@CCryLobby@@@stlpmtx_std@@@priv@stlpmtx_std@@AEAA_K_K@Z 0000000039a3c2a0 f i CryLobby.obj
 0001:0003b330       ?Execute@?$CClassJobNoRef5@P6AXIW4ECryLobbyError@@PEAUSCrySessionSearchResult@@PEAX@ZIW41@PEAU2@PEAXVCCryGameSpySBQR2MatchMaking@@@CWorkQueue@@UEAAXXZ 0000000039a3c330 f i CryGameSpySBQR2MatchMaking.obj
 0001:0003b380       ?Execute@?$CClassJobNoRef4@IIIIVCCryGameSpySBQR2MatchMaking@@@CWorkQueue@@UEAAXXZ 0000000039a3c380 f i CryGameSpySBQR2MatchMaking.obj
 0001:0003b3c0       ?Execute@?$CClassJobNoRef3@IIV?$CryLobbyID@USCryLobbySessionHandle@@$03@@VCCryMatchMaking@@@CWorkQueue@@UEAAXXZ 0000000039a3c3c0 f i CryMatchMaking.obj
 0001:0003b3c0       ?Execute@?$CClassJobNoRef3@IIIVCCryGameSpySBQR2MatchMaking@@@CWorkQueue@@UEAAXXZ 0000000039a3c3c0 f i CryGameSpySBQR2MatchMaking.obj
 0001:0003b3c0       ?Execute@?$CClassJobNoRef3@IIIVCCryMatchMaking@@@CWorkQueue@@UEAAXXZ 0000000039a3c3c0 f i CryMatchMaking.obj
 0001:0003b400       ??_E?$CClassJobNoRef4@IIV?$CryLobbyID@USCryLobbySessionHandle@@$03@@USCryMatchMakingConnectionUID@@VCCryMatchMaking@@@CWorkQueue@@UEAAPEAXI@Z 0000000039a3c400 f i CryMatchMaking.obj
 0001:0003b400       ??_G?$CClassJobNoRef4@IIV?$CryLobbyID@USCryLobbySessionHandle@@$03@@USCryMatchMakingConnectionUID@@VCCryMatchMaking@@@CWorkQueue@@UEAAPEAXI@Z 0000000039a3c400 f i CryMatchMaking.obj
 0001:0003b400       ??_G?$CClassJobNoRef5@P6AXIW4ECryLobbyError@@PEAUSCrySessionSearchResult@@PEAX@ZIW41@PEAU2@PEAXVCCryGameSpySBQR2MatchMaking@@@CWorkQueue@@UEAAPEAXI@Z 0000000039a3c400 f i CryGameSpySBQR2MatchMaking.obj
 0001:0003b400       ??_E?$CClassJobNoRef5@P6AXIW4ECryLobbyError@@PEAUSCrySessionSearchResult@@PEAX@ZIW41@PEAU2@PEAXVCCryGameSpySBQR2MatchMaking@@@CWorkQueue@@UEAAPEAXI@Z 0000000039a3c400 f i CryGameSpySBQR2MatchMaking.obj
 0001:0003b480       ??_E?$CClassJobNoRef3@IIIVCCryMatchMaking@@@CWorkQueue@@UEAAPEAXI@Z 0000000039a3c480 f i CryMatchMaking.obj
 0001:0003b480       ??_G?$CClassJobNoRef3@IIIVCCryMatchMaking@@@CWorkQueue@@UEAAPEAXI@Z 0000000039a3c480 f i CryMatchMaking.obj
 0001:0003b480       ??_G?$CClassJobNoRef3@IIV?$CryLobbyID@USCryLobbySessionHandle@@$03@@VCCryMatchMaking@@@CWorkQueue@@UEAAPEAXI@Z 0000000039a3c480 f i CryMatchMaking.obj
 0001:0003b480       ??_G?$CClassJobNoRef4@W4ECryLobbySystemEvent@@IW4EOnlineState@@W4ECryLobbyError@@VCCryGameSpySBQR2LobbyService@@@CWorkQueue@@UEAAPEAXI@Z 0000000039a3c480 f i CryGameSpySBQR2Lobby.obj
 0001:0003b480       ??_G?$CClassJobNoRef4@IIIIVCCryGameSpySBQR2MatchMaking@@@CWorkQueue@@UEAAPEAXI@Z 0000000039a3c480 f i CryGameSpySBQR2MatchMaking.obj
 0001:0003b480       ??_G?$CClassJobNoRef3@PEAUSTaskLink@CCryGameSpySBQR2DLCStore@@IIV2@@CWorkQueue@@UEAAPEAXI@Z 0000000039a3c480 f i CryGameSpySBQR2DLCStore.obj
 0001:0003b480       ??_G?$CClassJobNoRef3@IIIVCCryGameSpySBQR2MatchMaking@@@CWorkQueue@@UEAAPEAXI@Z 0000000039a3c480 f i CryGameSpySBQR2MatchMaking.obj
 0001:0003b480       ??_E?$CClassJobNoRef3@IIV?$CryLobbyID@USCryLobbySessionHandle@@$03@@VCCryMatchMaking@@@CWorkQueue@@UEAAPEAXI@Z 0000000039a3c480 f i CryMatchMaking.obj
 0001:0003b480       ??_E?$CClassJobNoRef3@PEAUSTaskLink@CCryGameSpySBQR2DLCStore@@IIV2@@CWorkQueue@@UEAAPEAXI@Z 0000000039a3c480 f i CryGameSpySBQR2DLCStore.obj
 0001:0003b480       ??_E?$CClassJobNoRef4@W4ECryLobbySystemEvent@@IW4EOnlineState@@W4ECryLobbyError@@VCCryGameSpySBQR2LobbyService@@@CWorkQueue@@UEAAPEAXI@Z 0000000039a3c480 f i CryGameSpySBQR2Lobby.obj
 0001:0003b480       ??_E?$CClassJobNoRef3@IIIVCCryGameSpySBQR2MatchMaking@@@CWorkQueue@@UEAAPEAXI@Z 0000000039a3c480 f i CryGameSpySBQR2MatchMaking.obj
 0001:0003b480       ??_E?$CClassJobNoRef4@IIIIVCCryGameSpySBQR2MatchMaking@@@CWorkQueue@@UEAAPEAXI@Z 0000000039a3c480 f i CryGameSpySBQR2MatchMaking.obj
 0001:0003b500       ??0SServer@SSearch@CCryGameSpySBQR2MatchMaking@@QEAA@XZ 0000000039a3c500 f i CryGameSpySBQR2MatchMaking.obj
 0001:0003b520       ??1SServer@SSearch@CCryGameSpySBQR2MatchMaking@@QEAA@XZ 0000000039a3c520 f i CryGameSpySBQR2MatchMaking.obj
 0001:0003b570       ??_ESRegisteredLobbyData@CCryGameSpySBQR2MatchMaking@@UEAAPEAXI@Z 0000000039a3c570 f i CryGameSpySBQR2MatchMaking.obj
 0001:0003b570       ??_GSRegisteredLobbyData@CCryGameSpySBQR2MatchMaking@@UEAAPEAXI@Z 0000000039a3c570 f i CryGameSpySBQR2MatchMaking.obj
 0001:0003b5a0       ?SessionGetCrySessionIDFromCrySessionHandle@CCryGameSpySBQR2MatchMaking@@UEAA?AV?$_smart_ptr@USCrySessionID@@@@I@Z 0000000039a3c5a0 f   CryGameSpySBQR2MatchMaking.obj
 0001:0003b710       ?WriteSessionIDToPacket@CCryGameSpySBQR2MatchMaking@@UEBA?AW4ECryLobbyError@@V?$_smart_ptr@USCrySessionID@@@@PEAVCCryLobbyPacket@@@Z 0000000039a3c710 f   CryGameSpySBQR2MatchMaking.obj
 0001:0003b7d0       ?ReadSessionIDFromPacket@CCryGameSpySBQR2MatchMaking@@UEBA?AV?$_smart_ptr@USCrySessionID@@@@PEAVCCryLobbyPacket@@@Z 0000000039a3c7d0 f   CryGameSpySBQR2MatchMaking.obj
 0001:0003b960       ?StartSessionJoin@CCryGameSpySBQR2MatchMaking@@IEAAXI@Z 0000000039a3c960 f   CryGameSpySBQR2MatchMaking.obj
 0001:0003ba50       ?CreateSessionHandle@CCryGameSpySBQR2MatchMaking@@IEAA?AW4ECryLobbyError@@PEAV?$CryLobbyID@USCryLobbySessionHandle@@$03@@_NIH@Z 0000000039a3ca50 f   CryGameSpySBQR2MatchMaking.obj
 0001:0003bbe0       ?AddServer@CCryGameSpySBQR2MatchMaking@@IEAAPEAUSServer@SSearch@1@PEAU31@PEAU_SBServer@@PEAUSTask@1@@Z 0000000039a3cbe0 f   CryGameSpySBQR2MatchMaking.obj
 0001:0003bdd0       ?ReadKeysFromSBServer@CCryGameSpySBQR2MatchMaking@@IEAAXPEAUSServer@SSearch@1@PEAU_SBServer@@@Z 0000000039a3cdd0 f   CryGameSpySBQR2MatchMaking.obj
 0001:0003beb0       ?SessionUserDataEvent@CCryGameSpySBQR2MatchMaking@@IEAAXW4ECryLobbySystemEvent@@V?$CryLobbyID@USCryLobbySessionHandle@@$03@@V?$CryLobbyID@USCryMatchMakingConnectionID@@$0EA@@@@Z 0000000039a3ceb0 f   CryGameSpySBQR2MatchMaking.obj
 0001:0003c170       ?InitialUserDataEvent@CCryGameSpySBQR2MatchMaking@@IEAAXV?$CryLobbyID@USCryLobbySessionHandle@@$03@@@Z 0000000039a3d170 f   CryGameSpySBQR2MatchMaking.obj
 0001:0003c260       ?FreeRemoteConnection@CCryGameSpySBQR2MatchMaking@@MEAAXV?$CryLobbyID@USCryLobbySessionHandle@@$03@@V?$CryLobbyID@USCryMatchMakingConnectionID@@$0EA@@@@Z 0000000039a3d260 f   CryGameSpySBQR2MatchMaking.obj
 0001:0003c380       ?InformVoiceRemoteUsersJoined@CCryGameSpySBQR2MatchMaking@@IEAAXV?$CryLobbyID@USCryLobbySessionHandle@@$03@@V?$CryLobbyID@USCryMatchMakingConnectionID@@$0EA@@@@Z 0000000039a3d380 f   CryGameSpySBQR2MatchMaking.obj
 0001:0003c510       ?ListKeys@CCryGameSpySBQR2MatchMaking@@QEAAXW4qr2_key_type@@PEAUqr2_keybuffer_s@@@Z 0000000039a3d510 f   CryGameSpySBQR2MatchMaking.obj
 0001:0003c5f0       ?ClearSessionSearch@CCryGameSpySBQR2MatchMaking@@IEAAXPEAUSSearch@1@@Z 0000000039a3d5f0 f   CryGameSpySBQR2MatchMaking.obj
 0001:0003c700       ?FreeSessionSearch@CCryGameSpySBQR2MatchMaking@@IEAAXPEAUSSearch@1@@Z 0000000039a3d700 f   CryGameSpySBQR2MatchMaking.obj
 0001:0003c7d0       ?GetSessionIDFromIP@CCryGameSpySBQR2MatchMaking@@UEAA?AW4ECryLobbyError@@QEBDQEAV?$_smart_ptr@USCrySessionID@@@@@Z 0000000039a3d7d0 f   CryGameSpySBQR2MatchMaking.obj
 0001:0003cad0       ?SessionJoinSuccess@CCryGameSpySBQR2MatchMaking@@IEAA?AW4ECryLobbyError@@PEAUSSession@1@V?$CryLobbyID@USCryMatchMakingConnectionID@@$0EA@@@IV?$CryLobbyID@USCryLobbySessionHandle@@$03@@@Z 0000000039a3dad0 f   CryGameSpySBQR2MatchMaking.obj
 0001:0003dd70       ?Format@?$CryStackStringT@D$0BPP@@@QEAAAEAV1@PEBDZZ 0000000039a3ed70 f i CryGameSpySBQR2MatchMaking.obj
 0001:0003de60       ??0?$_Vector_base@USCrySessionSearchData@@V?$allocator@USCrySessionSearchData@@@stlpmtx_std@@@priv@stlpmtx_std@@QEAA@_KAEBV?$allocator@USCrySessionSearchData@@@2@@Z 0000000039a3ee60 f i CryGameSpySBQR2MatchMaking.obj
 0001:0003df40       ??$__uninitialized_fill_n@PEAV?$_smart_ptr@USOrderLink@CCryGameSpySBQR2DLCStore@@@@_KV1@@priv@stlpmtx_std@@YAPEAV?$_smart_ptr@USOrderLink@CCryGameSpySBQR2DLCStore@@@@PEAV2@_KAEBV2@@Z 0000000039a3ef40 f i CryGameSpySBQR2DLCStore.obj
 0001:0003df40       ??$__uninitialized_fill_n@PEAV?$_smart_ptr@USTaskLink@CCryGameSpySBQR2DLCStore@@@@_KV1@@priv@stlpmtx_std@@YAPEAV?$_smart_ptr@USTaskLink@CCryGameSpySBQR2DLCStore@@@@PEAV2@_KAEBV2@@Z 0000000039a3ef40 f i CryGameSpySBQR2DLCStore.obj
 0001:0003df40       ??$__uninitialized_fill_n@PEAV?$_smart_ptr@USTaskCallbackBase@CGameSpySBQR2GPConnection@@@@_KV1@@priv@stlpmtx_std@@YAPEAV?$_smart_ptr@USTaskCallbackBase@CGameSpySBQR2GPConnection@@@@PEAV2@_KAEBV2@@Z 0000000039a3ef40 f i GameSpySBQR2GPConnection.obj
 0001:0003df40       ??$__uninitialized_fill_n@PEAV?$_smart_ptr@USRegisteredLobbyData@CCryGameSpySBQR2MatchMaking@@@@_KV1@@priv@stlpmtx_std@@YAPEAV?$_smart_ptr@USRegisteredLobbyData@CCryGameSpySBQR2MatchMaking@@@@PEAV2@_KAEBV2@@Z 0000000039a3ef40 f i CryGameSpySBQR2MatchMaking.obj
 0001:0003df40       ??$__uninitialized_fill_n@PEAV?$_smart_ptr@USTask@CGameSpySBQR2Core@@@@_KV1@@priv@stlpmtx_std@@YAPEAV?$_smart_ptr@USTask@CGameSpySBQR2Core@@@@PEAV2@_KAEBV2@@Z 0000000039a3ef40 f i GameSpySBQR2Core.obj
 0001:0003df40       ??$__uninitialized_fill_n@PEAV?$_smart_ptr@USCallbackBase@CGameSpySBQR2GPConnection@@@@_KV1@@priv@stlpmtx_std@@YAPEAV?$_smart_ptr@USCallbackBase@CGameSpySBQR2GPConnection@@@@PEAV2@_KAEBV2@@Z 0000000039a3ef40 f i GameSpySBQR2GPConnection.obj
 0001:0003df40       ??$__uninitialized_fill_n@PEAV?$_smart_ptr@USTaskBase@CGameSpySBQR2Sake@@@@_KV1@@priv@stlpmtx_std@@YAPEAV?$_smart_ptr@USTaskBase@CGameSpySBQR2Sake@@@@PEAV2@_KAEBV2@@Z 0000000039a3ef40 f i GameSpySBQR2Sake.obj
 0001:0003df40       ??$__uninitialized_fill_n@PEAV?$_smart_ptr@USTaskBase@CGameSpySBQR2NATNegotiation@@@@_KV1@@priv@stlpmtx_std@@YAPEAV?$_smart_ptr@USTaskBase@CGameSpySBQR2NATNegotiation@@@@PEAV2@_KAEBV2@@Z 0000000039a3ef40 f i GameSpySBQR2NatNegotiation.obj
 0001:0003dfb0       ?StartTask@CCryGameSpySBQR2MatchMaking@@IEAA?AW4ECryLobbyError@@W4ETask@1@PEAI1V?$CryLobbyID@USCryLobbySessionHandle@@$03@@PEAX3@Z 0000000039a3efb0 f   CryGameSpySBQR2MatchMaking.obj
 0001:0003e0a0       ?QueryKey@CCryGameSpySBQR2MatchMaking@@QEAAXW4qr2_key_type@@HHPEAUqr2_buffer_s@@@Z 0000000039a3f0a0 f   CryGameSpySBQR2MatchMaking.obj
 0001:0003e180       ?EndSessionGetUsers@CCryGameSpySBQR2MatchMaking@@IEAAXI@Z 0000000039a3f180 f   CryGameSpySBQR2MatchMaking.obj
 0001:0003e810       ?ProcessLocalUserData@CCryGameSpySBQR2MatchMaking@@IEAAXAEBV?$CConfigurableVariant@V?$CNode@USNullAddr@@V?$CNode@GV?$CNode@USIPv4Addr@@V?$CNode@ULobbyIdAddr@@VCEnd@NTypelist@@@NTypelist@@@NTypelist@@@NTypelist@@@NTypelist@@$07VCDefaultVariantConversion@NConfigurableVariantHelpers@@VCDefaultVariantConstruction@4@@@PEAVCCrySharedLobbyPacket@@@Z 0000000039a3f810 f   CryGameSpySBQR2MatchMaking.obj
 0001:0003e9c0       ?Open@CCryFile@@QEAA_NPEBD0H@Z 0000000039a3f9c0 f i CryGameSpySBQR2MatchMaking.obj
 0001:0003ec20       ?FindBannedUserByID@CCryGameSpySBQR2MatchMaking@@IEAAPEAUSBannedUser@@_K@Z 0000000039a3fc20 f   CryGameSpySBQR2MatchMaking.obj
 0001:0003eda0       ?FindBannedUserByName@CCryGameSpySBQR2MatchMaking@@IEAAPEAUSBannedUser@@PEBD@Z 0000000039a3fda0 f   CryGameSpySBQR2MatchMaking.obj
 0001:0003ef60       ?ReportBannedUsers@CCryGameSpySBQR2MatchMaking@@IEBAXAEBV?$deque@USBannedUser@@V?$allocator@USBannedUser@@@stlpmtx_std@@@stlpmtx_std@@@Z 0000000039a3ff60 f   CryGameSpySBQR2MatchMaking.obj
 0001:0003f170       ?ResolveBannedUser@CCryGameSpySBQR2MatchMaking@@IEAA_NHPEBD@Z 0000000039a40170 f   CryGameSpySBQR2MatchMaking.obj
 0001:0003f450       ?SaveBannedUsers@CCryGameSpySBQR2MatchMaking@@IEBAXAEAVXmlNodeRef@@AEBV?$deque@USBannedUser@@V?$allocator@USBannedUser@@@stlpmtx_std@@@stlpmtx_std@@@Z 0000000039a40450 f   CryGameSpySBQR2MatchMaking.obj
 0001:0003f620       ?back@?$deque@USBannedUser@@V?$allocator@USBannedUser@@@stlpmtx_std@@@stlpmtx_std@@QEAAAEAUSBannedUser@@XZ 0000000039a40620 f i CryGameSpySBQR2MatchMaking.obj
 0001:0003f660       ?_M_erase@?$_Rb_tree@EU?$less@E@stlpmtx_std@@U?$pair@$$CBEV?$_smart_ptr@USGameSpyKey@CCryGameSpySBQR2MatchMaking@@@@@2@U?$_Select1st@U?$pair@$$CBEV?$_smart_ptr@USGameSpyKey@CCryGameSpySBQR2MatchMaking@@@@@stlpmtx_std@@@priv@2@U?$_MapTraitsT@U?$pair@$$CBEV?$_smart_ptr@USGameSpyKey@CCryGameSpySBQR2MatchMaking@@@@@stlpmtx_std@@@52@V?$allocator@U?$pair@$$CBEV?$_smart_ptr@USGameSpyKey@CCryGameSpySBQR2MatchMaking@@@@@stlpmtx_std@@@2@@priv@stlpmtx_std@@AEAAXPEAU_Rb_tree_node_base@23@@Z 0000000039a40660 f i CryGameSpySBQR2MatchMaking.obj
 0001:0003f660       ?_M_erase@?$_Rb_tree@IU?$less@I@stlpmtx_std@@U?$pair@$$CBIV?$_smart_ptr@USRegisteredLobbyData@CCryGameSpySBQR2MatchMaking@@@@@2@U?$_Select1st@U?$pair@$$CBIV?$_smart_ptr@USRegisteredLobbyData@CCryGameSpySBQR2MatchMaking@@@@@stlpmtx_std@@@priv@2@U?$_MapTraitsT@U?$pair@$$CBIV?$_smart_ptr@USRegisteredLobbyData@CCryGameSpySBQR2MatchMaking@@@@@stlpmtx_std@@@52@V?$allocator@U?$pair@$$CBIV?$_smart_ptr@USRegisteredLobbyData@CCryGameSpySBQR2MatchMaking@@@@@stlpmtx_std@@@2@@priv@stlpmtx_std@@AEAAXPEAU_Rb_tree_node_base@23@@Z 0000000039a40660 f i CryGameSpySBQR2MatchMaking.obj
 0001:0003f660       ?_M_erase@?$_Rb_tree@IU?$less@I@stlpmtx_std@@U?$pair@$$CBIV?$_smart_ptr@USGameSpyKey@CCryGameSpySBQR2MatchMaking@@@@@2@U?$_Select1st@U?$pair@$$CBIV?$_smart_ptr@USGameSpyKey@CCryGameSpySBQR2MatchMaking@@@@@stlpmtx_std@@@priv@2@U?$_MapTraitsT@U?$pair@$$CBIV?$_smart_ptr@USGameSpyKey@CCryGameSpySBQR2MatchMaking@@@@@stlpmtx_std@@@52@V?$allocator@U?$pair@$$CBIV?$_smart_ptr@USGameSpyKey@CCryGameSpySBQR2MatchMaking@@@@@stlpmtx_std@@@2@@priv@stlpmtx_std@@AEAAXPEAU_Rb_tree_node_base@23@@Z 0000000039a40660 f i CryGameSpySBQR2MatchMaking.obj
 0001:0003f660       ?_M_erase@?$_Rb_tree@PEBDU?$less@PEBD@stlpmtx_std@@U?$pair@QEBDV?$_smart_ptr@USGameSpyKey@CCryGameSpySBQR2MatchMaking@@@@@2@U?$_Select1st@U?$pair@QEBDV?$_smart_ptr@USGameSpyKey@CCryGameSpySBQR2MatchMaking@@@@@stlpmtx_std@@@priv@2@U?$_MapTraitsT@U?$pair@QEBDV?$_smart_ptr@USGameSpyKey@CCryGameSpySBQR2MatchMaking@@@@@stlpmtx_std@@@52@V?$allocator@U?$pair@QEBDV?$_smart_ptr@USGameSpyKey@CCryGameSpySBQR2MatchMaking@@@@@stlpmtx_std@@@2@@priv@stlpmtx_std@@AEAAXPEAU_Rb_tree_node_base@23@@Z 0000000039a40660 f i CryGameSpySBQR2MatchMaking.obj
 0001:0003f700       ?Format@?$CryStackStringT@D$0EJ@@@QEAAAEAV1@PEBDZZ 0000000039a40700 f i CryGameSpySBQR2MatchMaking.obj
 0001:0003f7f0       ??0?$_Impl_vector@USCrySessionSearchData@@V?$allocator@USCrySessionSearchData@@@stlpmtx_std@@@priv@stlpmtx_std@@QEAA@AEBV012@@Z 0000000039a407f0 f i CryGameSpySBQR2MatchMaking.obj
 0001:0003f890       ?_M_create_node@?$_Rb_tree@EU?$less@E@stlpmtx_std@@U?$pair@$$CBEV?$_smart_ptr@USGameSpyKey@CCryGameSpySBQR2MatchMaking@@@@@2@U?$_Select1st@U?$pair@$$CBEV?$_smart_ptr@USGameSpyKey@CCryGameSpySBQR2MatchMaking@@@@@stlpmtx_std@@@priv@2@U?$_MapTraitsT@U?$pair@$$CBEV?$_smart_ptr@USGameSpyKey@CCryGameSpySBQR2MatchMaking@@@@@stlpmtx_std@@@52@V?$allocator@U?$pair@$$CBEV?$_smart_ptr@USGameSpyKey@CCryGameSpySBQR2MatchMaking@@@@@stlpmtx_std@@@2@@priv@stlpmtx_std@@IEAAPEAU_Rb_tree_node_base@23@AEBU?$pair@$$CBEV?$_smart_ptr@USGameSpyKey@CCryGameSpySBQR2MatchMaking@@@@@3@@Z 0000000039a40890 f i CryGameSpySBQR2MatchMaking.obj
 0001:0003f910       ?_M_create_node@?$_Rb_tree@PEBDU?$less@PEBD@stlpmtx_std@@U?$pair@QEBDV?$_smart_ptr@USGameSpyKey@CCryGameSpySBQR2MatchMaking@@@@@2@U?$_Select1st@U?$pair@QEBDV?$_smart_ptr@USGameSpyKey@CCryGameSpySBQR2MatchMaking@@@@@stlpmtx_std@@@priv@2@U?$_MapTraitsT@U?$pair@QEBDV?$_smart_ptr@USGameSpyKey@CCryGameSpySBQR2MatchMaking@@@@@stlpmtx_std@@@52@V?$allocator@U?$pair@QEBDV?$_smart_ptr@USGameSpyKey@CCryGameSpySBQR2MatchMaking@@@@@stlpmtx_std@@@2@@priv@stlpmtx_std@@IEAAPEAU_Rb_tree_node_base@23@AEBU?$pair@QEBDV?$_smart_ptr@USGameSpyKey@CCryGameSpySBQR2MatchMaking@@@@@3@@Z 0000000039a40910 f i CryGameSpySBQR2MatchMaking.obj
 0001:0003f990       ?_M_create_node@?$_Rb_tree@IU?$less@I@stlpmtx_std@@U?$pair@$$CBIV?$_smart_ptr@USRegisteredLobbyData@CCryGameSpySBQR2MatchMaking@@@@@2@U?$_Select1st@U?$pair@$$CBIV?$_smart_ptr@USRegisteredLobbyData@CCryGameSpySBQR2MatchMaking@@@@@stlpmtx_std@@@priv@2@U?$_MapTraitsT@U?$pair@$$CBIV?$_smart_ptr@USRegisteredLobbyData@CCryGameSpySBQR2MatchMaking@@@@@stlpmtx_std@@@52@V?$allocator@U?$pair@$$CBIV?$_smart_ptr@USRegisteredLobbyData@CCryGameSpySBQR2MatchMaking@@@@@stlpmtx_std@@@2@@priv@stlpmtx_std@@IEAAPEAU_Rb_tree_node_base@23@AEBU?$pair@$$CBIV?$_smart_ptr@USRegisteredLobbyData@CCryGameSpySBQR2MatchMaking@@@@@3@@Z 0000000039a40990 f i CryGameSpySBQR2MatchMaking.obj
 0001:0003f990       ?_M_create_node@?$_Rb_tree@IU?$less@I@stlpmtx_std@@U?$pair@$$CBIV?$_smart_ptr@USGameSpyKey@CCryGameSpySBQR2MatchMaking@@@@@2@U?$_Select1st@U?$pair@$$CBIV?$_smart_ptr@USGameSpyKey@CCryGameSpySBQR2MatchMaking@@@@@stlpmtx_std@@@priv@2@U?$_MapTraitsT@U?$pair@$$CBIV?$_smart_ptr@USGameSpyKey@CCryGameSpySBQR2MatchMaking@@@@@stlpmtx_std@@@52@V?$allocator@U?$pair@$$CBIV?$_smart_ptr@USGameSpyKey@CCryGameSpySBQR2MatchMaking@@@@@stlpmtx_std@@@2@@priv@stlpmtx_std@@IEAAPEAU_Rb_tree_node_base@23@AEBU?$pair@$$CBIV?$_smart_ptr@USGameSpyKey@CCryGameSpySBQR2MatchMaking@@@@@3@@Z 0000000039a40990 f i CryGameSpySBQR2MatchMaking.obj
 0001:0003fa10       ?UnbanCmd@CCryGameSpySBQR2MatchMaking@@MEAAX_K@Z 0000000039a40a10 f   CryGameSpySBQR2MatchMaking.obj
 0001:0003fab0       ?UnbanCmd@CCryGameSpySBQR2MatchMaking@@MEAAXPEBD@Z 0000000039a40ab0 f   CryGameSpySBQR2MatchMaking.obj
 0001:0003fb50       ?BanStatus@CCryGameSpySBQR2MatchMaking@@MEAAXXZ 0000000039a40b50 f   CryGameSpySBQR2MatchMaking.obj
 0001:0003fbe0       ?Format@?$CryStringT@D@@QEAAAEAV1@PEBDZZ 0000000039a40be0 f i CryGameSpySBQR2MatchMaking.obj
 0001:0003fc70       ?_M_insert@?$_Rb_tree@EU?$less@E@stlpmtx_std@@U?$pair@$$CBEV?$_smart_ptr@USGameSpyKey@CCryGameSpySBQR2MatchMaking@@@@@2@U?$_Select1st@U?$pair@$$CBEV?$_smart_ptr@USGameSpyKey@CCryGameSpySBQR2MatchMaking@@@@@stlpmtx_std@@@priv@2@U?$_MapTraitsT@U?$pair@$$CBEV?$_smart_ptr@USGameSpyKey@CCryGameSpySBQR2MatchMaking@@@@@stlpmtx_std@@@52@V?$allocator@U?$pair@$$CBEV?$_smart_ptr@USGameSpyKey@CCryGameSpySBQR2MatchMaking@@@@@stlpmtx_std@@@2@@priv@stlpmtx_std@@AEAA?AU?$_Rb_tree_iterator@U?$pair@$$CBEV?$_smart_ptr@USGameSpyKey@CCryGameSpySBQR2MatchMaking@@@@@stlpmtx_std@@U?$_MapTraitsT@U?$pair@$$CBEV?$_smart_ptr@USGameSpyKey@CCryGameSpySBQR2MatchMaking@@@@@stlpmtx_std@@@priv@2@@23@PEAU_Rb_tree_node_base@23@AEBU?$pair@$$CBEV?$_smart_ptr@USGameSpyKey@CCryGameSpySBQR2MatchMaking@@@@@3@00@Z 0000000039a40c70 f i CryGameSpySBQR2MatchMaking.obj
 0001:0003fd30       ?insert_unique@?$_Rb_tree@EU?$less@E@stlpmtx_std@@U?$pair@$$CBEV?$_smart_ptr@USGameSpyKey@CCryGameSpySBQR2MatchMaking@@@@@2@U?$_Select1st@U?$pair@$$CBEV?$_smart_ptr@USGameSpyKey@CCryGameSpySBQR2MatchMaking@@@@@stlpmtx_std@@@priv@2@U?$_MapTraitsT@U?$pair@$$CBEV?$_smart_ptr@USGameSpyKey@CCryGameSpySBQR2MatchMaking@@@@@stlpmtx_std@@@52@V?$allocator@U?$pair@$$CBEV?$_smart_ptr@USGameSpyKey@CCryGameSpySBQR2MatchMaking@@@@@stlpmtx_std@@@2@@priv@stlpmtx_std@@QEAA?AU?$pair@U?$_Rb_tree_iterator@U?$pair@$$CBEV?$_smart_ptr@USGameSpyKey@CCryGameSpySBQR2MatchMaking@@@@@stlpmtx_std@@U?$_MapTraitsT@U?$pair@$$CBEV?$_smart_ptr@USGameSpyKey@CCryGameSpySBQR2MatchMaking@@@@@stlpmtx_std@@@priv@2@@priv@stlpmtx_std@@_N@3@AEBU?$pair@$$CBEV?$_smart_ptr@USGameSpyKey@CCryGameSpySBQR2MatchMaking@@@@@3@@Z 0000000039a40d30 f i CryGameSpySBQR2MatchMaking.obj
 0001:0003ff30       ?_M_insert@?$_Rb_tree@PEBDU?$less@PEBD@stlpmtx_std@@U?$pair@QEBDV?$_smart_ptr@USGameSpyKey@CCryGameSpySBQR2MatchMaking@@@@@2@U?$_Select1st@U?$pair@QEBDV?$_smart_ptr@USGameSpyKey@CCryGameSpySBQR2MatchMaking@@@@@stlpmtx_std@@@priv@2@U?$_MapTraitsT@U?$pair@QEBDV?$_smart_ptr@USGameSpyKey@CCryGameSpySBQR2MatchMaking@@@@@stlpmtx_std@@@52@V?$allocator@U?$pair@QEBDV?$_smart_ptr@USGameSpyKey@CCryGameSpySBQR2MatchMaking@@@@@stlpmtx_std@@@2@@priv@stlpmtx_std@@AEAA?AU?$_Rb_tree_iterator@U?$pair@QEBDV?$_smart_ptr@USGameSpyKey@CCryGameSpySBQR2MatchMaking@@@@@stlpmtx_std@@U?$_MapTraitsT@U?$pair@QEBDV?$_smart_ptr@USGameSpyKey@CCryGameSpySBQR2MatchMaking@@@@@stlpmtx_std@@@priv@2@@23@PEAU_Rb_tree_node_base@23@AEBU?$pair@QEBDV?$_smart_ptr@USGameSpyKey@CCryGameSpySBQR2MatchMaking@@@@@3@00@Z 0000000039a40f30 f i CryGameSpySBQR2MatchMaking.obj
 0001:0003fff0       ?insert_unique@?$_Rb_tree@PEBDU?$less@PEBD@stlpmtx_std@@U?$pair@QEBDV?$_smart_ptr@USGameSpyKey@CCryGameSpySBQR2MatchMaking@@@@@2@U?$_Select1st@U?$pair@QEBDV?$_smart_ptr@USGameSpyKey@CCryGameSpySBQR2MatchMaking@@@@@stlpmtx_std@@@priv@2@U?$_MapTraitsT@U?$pair@QEBDV?$_smart_ptr@USGameSpyKey@CCryGameSpySBQR2MatchMaking@@@@@stlpmtx_std@@@52@V?$allocator@U?$pair@QEBDV?$_smart_ptr@USGameSpyKey@CCryGameSpySBQR2MatchMaking@@@@@stlpmtx_std@@@2@@priv@stlpmtx_std@@QEAA?AU?$pair@U?$_Rb_tree_iterator@U?$pair@QEBDV?$_smart_ptr@USGameSpyKey@CCryGameSpySBQR2MatchMaking@@@@@stlpmtx_std@@U?$_MapTraitsT@U?$pair@QEBDV?$_smart_ptr@USGameSpyKey@CCryGameSpySBQR2MatchMaking@@@@@stlpmtx_std@@@priv@2@@priv@stlpmtx_std@@_N@3@AEBU?$pair@QEBDV?$_smart_ptr@USGameSpyKey@CCryGameSpySBQR2MatchMaking@@@@@3@@Z 0000000039a40ff0 f i CryGameSpySBQR2MatchMaking.obj
 0001:000401f0       ?_M_insert@?$_Rb_tree@IU?$less@I@stlpmtx_std@@U?$pair@$$CBIV?$_smart_ptr@USGameSpyKey@CCryGameSpySBQR2MatchMaking@@@@@2@U?$_Select1st@U?$pair@$$CBIV?$_smart_ptr@USGameSpyKey@CCryGameSpySBQR2MatchMaking@@@@@stlpmtx_std@@@priv@2@U?$_MapTraitsT@U?$pair@$$CBIV?$_smart_ptr@USGameSpyKey@CCryGameSpySBQR2MatchMaking@@@@@stlpmtx_std@@@52@V?$allocator@U?$pair@$$CBIV?$_smart_ptr@USGameSpyKey@CCryGameSpySBQR2MatchMaking@@@@@stlpmtx_std@@@2@@priv@stlpmtx_std@@AEAA?AU?$_Rb_tree_iterator@U?$pair@$$CBIV?$_smart_ptr@USGameSpyKey@CCryGameSpySBQR2MatchMaking@@@@@stlpmtx_std@@U?$_MapTraitsT@U?$pair@$$CBIV?$_smart_ptr@USGameSpyKey@CCryGameSpySBQR2MatchMaking@@@@@stlpmtx_std@@@priv@2@@23@PEAU_Rb_tree_node_base@23@AEBU?$pair@$$CBIV?$_smart_ptr@USGameSpyKey@CCryGameSpySBQR2MatchMaking@@@@@3@00@Z 0000000039a411f0 f i CryGameSpySBQR2MatchMaking.obj
 0001:000401f0       ?_M_insert@?$_Rb_tree@IU?$less@I@stlpmtx_std@@U?$pair@$$CBIV?$_smart_ptr@USRegisteredLobbyData@CCryGameSpySBQR2MatchMaking@@@@@2@U?$_Select1st@U?$pair@$$CBIV?$_smart_ptr@USRegisteredLobbyData@CCryGameSpySBQR2MatchMaking@@@@@stlpmtx_std@@@priv@2@U?$_MapTraitsT@U?$pair@$$CBIV?$_smart_ptr@USRegisteredLobbyData@CCryGameSpySBQR2MatchMaking@@@@@stlpmtx_std@@@52@V?$allocator@U?$pair@$$CBIV?$_smart_ptr@USRegisteredLobbyData@CCryGameSpySBQR2MatchMaking@@@@@stlpmtx_std@@@2@@priv@stlpmtx_std@@AEAA?AU?$_Rb_tree_iterator@U?$pair@$$CBIV?$_smart_ptr@USRegisteredLobbyData@CCryGameSpySBQR2MatchMaking@@@@@stlpmtx_std@@U?$_MapTraitsT@U?$pair@$$CBIV?$_smart_ptr@USRegisteredLobbyData@CCryGameSpySBQR2MatchMaking@@@@@stlpmtx_std@@@priv@2@@23@PEAU_Rb_tree_node_base@23@AEBU?$pair@$$CBIV?$_smart_ptr@USRegisteredLobbyData@CCryGameSpySBQR2MatchMaking@@@@@3@00@Z 0000000039a411f0 f i CryGameSpySBQR2MatchMaking.obj
 0001:000402b0       ?insert_unique@?$_Rb_tree@IU?$less@I@stlpmtx_std@@U?$pair@$$CBIV?$_smart_ptr@USRegisteredLobbyData@CCryGameSpySBQR2MatchMaking@@@@@2@U?$_Select1st@U?$pair@$$CBIV?$_smart_ptr@USRegisteredLobbyData@CCryGameSpySBQR2MatchMaking@@@@@stlpmtx_std@@@priv@2@U?$_MapTraitsT@U?$pair@$$CBIV?$_smart_ptr@USRegisteredLobbyData@CCryGameSpySBQR2MatchMaking@@@@@stlpmtx_std@@@52@V?$allocator@U?$pair@$$CBIV?$_smart_ptr@USRegisteredLobbyData@CCryGameSpySBQR2MatchMaking@@@@@stlpmtx_std@@@2@@priv@stlpmtx_std@@QEAA?AU?$pair@U?$_Rb_tree_iterator@U?$pair@$$CBIV?$_smart_ptr@USRegisteredLobbyData@CCryGameSpySBQR2MatchMaking@@@@@stlpmtx_std@@U?$_MapTraitsT@U?$pair@$$CBIV?$_smart_ptr@USRegisteredLobbyData@CCryGameSpySBQR2MatchMaking@@@@@stlpmtx_std@@@priv@2@@priv@stlpmtx_std@@_N@3@AEBU?$pair@$$CBIV?$_smart_ptr@USRegisteredLobbyData@CCryGameSpySBQR2MatchMaking@@@@@3@@Z 0000000039a412b0 f i CryGameSpySBQR2MatchMaking.obj
 0001:000402b0       ?insert_unique@?$_Rb_tree@IU?$less@I@stlpmtx_std@@U?$pair@$$CBIV?$_smart_ptr@USGameSpyKey@CCryGameSpySBQR2MatchMaking@@@@@2@U?$_Select1st@U?$pair@$$CBIV?$_smart_ptr@USGameSpyKey@CCryGameSpySBQR2MatchMaking@@@@@stlpmtx_std@@@priv@2@U?$_MapTraitsT@U?$pair@$$CBIV?$_smart_ptr@USGameSpyKey@CCryGameSpySBQR2MatchMaking@@@@@stlpmtx_std@@@52@V?$allocator@U?$pair@$$CBIV?$_smart_ptr@USGameSpyKey@CCryGameSpySBQR2MatchMaking@@@@@stlpmtx_std@@@2@@priv@stlpmtx_std@@QEAA?AU?$pair@U?$_Rb_tree_iterator@U?$pair@$$CBIV?$_smart_ptr@USGameSpyKey@CCryGameSpySBQR2MatchMaking@@@@@stlpmtx_std@@U?$_MapTraitsT@U?$pair@$$CBIV?$_smart_ptr@USGameSpyKey@CCryGameSpySBQR2MatchMaking@@@@@stlpmtx_std@@@priv@2@@priv@stlpmtx_std@@_N@3@AEBU?$pair@$$CBIV?$_smart_ptr@USGameSpyKey@CCryGameSpySBQR2MatchMaking@@@@@3@@Z 0000000039a412b0 f i CryGameSpySBQR2MatchMaking.obj
 0001:000404b0       ?EndSessionQuery@CCryGameSpySBQR2MatchMaking@@IEAAXI@Z 0000000039a414b0 f   CryGameSpySBQR2MatchMaking.obj
 0001:00040840       ?CreateSessionAddress@CCryGameSpySBQR2MatchMaking@@IEAAXPEAU_SBServer@@PEAVCCryGameSpySBQR2LobbyService@@PEAUSCryGameSpySBQR2SessionID@@PEAUSServer@SSearch@1@@Z 0000000039a41840 f   CryGameSpySBQR2MatchMaking.obj
 0001:00040a50       ?SaveBannedUserList@CCryGameSpySBQR2MatchMaking@@IEBAXXZ 0000000039a41a50 f   CryGameSpySBQR2MatchMaking.obj
 0001:00040b50       ?push_back@?$_Impl_vector@USCrySessionSearchData@@V?$allocator@USCrySessionSearchData@@@stlpmtx_std@@@priv@stlpmtx_std@@QEAAXAEBUSCrySessionSearchData@@@Z 0000000039a41b50 f i CryGameSpySBQR2MatchMaking.obj
 0001:00040ca0       ?_M_push_back_aux_v@?$_Impl_deque@USBannedUser@@V?$allocator@USBannedUser@@@stlpmtx_std@@@priv@stlpmtx_std@@IEAAXAEBUSBannedUser@@@Z 0000000039a41ca0 f i CryGameSpySBQR2MatchMaking.obj
 0001:00040d30       ?insert_unique@?$_Rb_tree@EU?$less@E@stlpmtx_std@@U?$pair@$$CBEV?$_smart_ptr@USGameSpyKey@CCryGameSpySBQR2MatchMaking@@@@@2@U?$_Select1st@U?$pair@$$CBEV?$_smart_ptr@USGameSpyKey@CCryGameSpySBQR2MatchMaking@@@@@stlpmtx_std@@@priv@2@U?$_MapTraitsT@U?$pair@$$CBEV?$_smart_ptr@USGameSpyKey@CCryGameSpySBQR2MatchMaking@@@@@stlpmtx_std@@@52@V?$allocator@U?$pair@$$CBEV?$_smart_ptr@USGameSpyKey@CCryGameSpySBQR2MatchMaking@@@@@stlpmtx_std@@@2@@priv@stlpmtx_std@@QEAA?AU?$_Rb_tree_iterator@U?$pair@$$CBEV?$_smart_ptr@USGameSpyKey@CCryGameSpySBQR2MatchMaking@@@@@stlpmtx_std@@U?$_MapTraitsT@U?$pair@$$CBEV?$_smart_ptr@USGameSpyKey@CCryGameSpySBQR2MatchMaking@@@@@stlpmtx_std@@@priv@2@@23@U423@AEBU?$pair@$$CBEV?$_smart_ptr@USGameSpyKey@CCryGameSpySBQR2MatchMaking@@@@@3@@Z 0000000039a41d30 f i CryGameSpySBQR2MatchMaking.obj
 0001:00041180       ?insert_unique@?$_Rb_tree@PEBDU?$less@PEBD@stlpmtx_std@@U?$pair@QEBDV?$_smart_ptr@USGameSpyKey@CCryGameSpySBQR2MatchMaking@@@@@2@U?$_Select1st@U?$pair@QEBDV?$_smart_ptr@USGameSpyKey@CCryGameSpySBQR2MatchMaking@@@@@stlpmtx_std@@@priv@2@U?$_MapTraitsT@U?$pair@QEBDV?$_smart_ptr@USGameSpyKey@CCryGameSpySBQR2MatchMaking@@@@@stlpmtx_std@@@52@V?$allocator@U?$pair@QEBDV?$_smart_ptr@USGameSpyKey@CCryGameSpySBQR2MatchMaking@@@@@stlpmtx_std@@@2@@priv@stlpmtx_std@@QEAA?AU?$_Rb_tree_iterator@U?$pair@QEBDV?$_smart_ptr@USGameSpyKey@CCryGameSpySBQR2MatchMaking@@@@@stlpmtx_std@@U?$_MapTraitsT@U?$pair@QEBDV?$_smart_ptr@USGameSpyKey@CCryGameSpySBQR2MatchMaking@@@@@stlpmtx_std@@@priv@2@@23@U423@AEBU?$pair@QEBDV?$_smart_ptr@USGameSpyKey@CCryGameSpySBQR2MatchMaking@@@@@3@@Z 0000000039a42180 f i CryGameSpySBQR2MatchMaking.obj
 0001:000415d0       ?insert_unique@?$_Rb_tree@IU?$less@I@stlpmtx_std@@U?$pair@$$CBIV?$_smart_ptr@USGameSpyKey@CCryGameSpySBQR2MatchMaking@@@@@2@U?$_Select1st@U?$pair@$$CBIV?$_smart_ptr@USGameSpyKey@CCryGameSpySBQR2MatchMaking@@@@@stlpmtx_std@@@priv@2@U?$_MapTraitsT@U?$pair@$$CBIV?$_smart_ptr@USGameSpyKey@CCryGameSpySBQR2MatchMaking@@@@@stlpmtx_std@@@52@V?$allocator@U?$pair@$$CBIV?$_smart_ptr@USGameSpyKey@CCryGameSpySBQR2MatchMaking@@@@@stlpmtx_std@@@2@@priv@stlpmtx_std@@QEAA?AU?$_Rb_tree_iterator@U?$pair@$$CBIV?$_smart_ptr@USGameSpyKey@CCryGameSpySBQR2MatchMaking@@@@@stlpmtx_std@@U?$_MapTraitsT@U?$pair@$$CBIV?$_smart_ptr@USGameSpyKey@CCryGameSpySBQR2MatchMaking@@@@@stlpmtx_std@@@priv@2@@23@U423@AEBU?$pair@$$CBIV?$_smart_ptr@USGameSpyKey@CCryGameSpySBQR2MatchMaking@@@@@3@@Z 0000000039a425d0 f i CryGameSpySBQR2MatchMaking.obj
 0001:000415d0       ?insert_unique@?$_Rb_tree@IU?$less@I@stlpmtx_std@@U?$pair@$$CBIV?$_smart_ptr@USRegisteredLobbyData@CCryGameSpySBQR2MatchMaking@@@@@2@U?$_Select1st@U?$pair@$$CBIV?$_smart_ptr@USRegisteredLobbyData@CCryGameSpySBQR2MatchMaking@@@@@stlpmtx_std@@@priv@2@U?$_MapTraitsT@U?$pair@$$CBIV?$_smart_ptr@USRegisteredLobbyData@CCryGameSpySBQR2MatchMaking@@@@@stlpmtx_std@@@52@V?$allocator@U?$pair@$$CBIV?$_smart_ptr@USRegisteredLobbyData@CCryGameSpySBQR2MatchMaking@@@@@stlpmtx_std@@@2@@priv@stlpmtx_std@@QEAA?AU?$_Rb_tree_iterator@U?$pair@$$CBIV?$_smart_ptr@USRegisteredLobbyData@CCryGameSpySBQR2MatchMaking@@@@@stlpmtx_std@@U?$_MapTraitsT@U?$pair@$$CBIV?$_smart_ptr@USRegisteredLobbyData@CCryGameSpySBQR2MatchMaking@@@@@stlpmtx_std@@@priv@2@@23@U423@AEBU?$pair@$$CBIV?$_smart_ptr@USRegisteredLobbyData@CCryGameSpySBQR2MatchMaking@@@@@3@@Z 0000000039a425d0 f i CryGameSpySBQR2MatchMaking.obj
 0001:00041a10       ?EndTask@CCryGameSpySBQR2MatchMaking@@IEAAXI@Z 0000000039a42a10 f   CryGameSpySBQR2MatchMaking.obj
 0001:00041d50       ?StartSessionRequestJoin@CCryGameSpySBQR2MatchMaking@@IEAAXI@Z 0000000039a42d50 f   CryGameSpySBQR2MatchMaking.obj
 0001:00042330       ?GetLobbyConnectionFromRemoteConnectionID@CCryGameSpySBQR2MatchMaking@@IEAA?AV?$CryLobbyID@USCryLobbyConnectionID@@$0EA@@@AEAUSCryGameSpySBQR2RemoteConnectionID@@@Z 0000000039a43330 f   CryGameSpySBQR2MatchMaking.obj
 0001:00042450       ?OnBannedUserListChanged@CCryGameSpySBQR2MatchMaking@@MEAAXXZ 0000000039a43450 f   CryGameSpySBQR2MatchMaking.obj
 0001:00042460       ?SendCDKeyChallenge@CCryGameSpySBQR2MatchMaking@@IEAAXPEAUSRConnection@SSession@1@PEAD@Z 0000000039a43460 f   CryGameSpySBQR2MatchMaking.obj
 0001:000426b0       ?CDKeyReauthCallback@CCryGameSpySBQR2MatchMaking@@KAXHHHPEADPEAX@Z 0000000039a436b0 f   CryGameSpySBQR2MatchMaking.obj
 0001:00042790       ?RetryCDKeyTimeOuts@CCryGameSpySBQR2MatchMaking@@IEAAXVCTimeValue@@@Z 0000000039a43790 f   CryGameSpySBQR2MatchMaking.obj
 0001:00042a00       ?GetHostAddressFromSessionHandle@CCryGameSpySBQR2MatchMaking@@UEAA?AV?$CConfigurableVariant@V?$CNode@USNullAddr@@V?$CNode@GV?$CNode@USIPv4Addr@@V?$CNode@ULobbyIdAddr@@VCEnd@NTypelist@@@NTypelist@@@NTypelist@@@NTypelist@@@NTypelist@@$07VCDefaultVariantConversion@NConfigurableVariantHelpers@@VCDefaultVariantConstruction@4@@@I@Z 0000000039a43a00 f   CryGameSpySBQR2MatchMaking.obj
 0001:00042b60       ?pop_front@?$deque@USBannedUser@@V?$allocator@USBannedUser@@@stlpmtx_std@@@stlpmtx_std@@QEAAXXZ 0000000039a43b60 f i CryGameSpySBQR2MatchMaking.obj
 0001:00042bd0       ?_M_erase@?$_Rb_tree@EU?$less@E@stlpmtx_std@@U?$pair@$$CBEV?$CryStringT@D@@@2@U?$_Select1st@U?$pair@$$CBEV?$CryStringT@D@@@stlpmtx_std@@@priv@2@U?$_MapTraitsT@U?$pair@$$CBEV?$CryStringT@D@@@stlpmtx_std@@@52@V?$allocator@U?$pair@$$CBEV?$CryStringT@D@@@stlpmtx_std@@@2@@priv@stlpmtx_std@@AEAAXPEAU_Rb_tree_node_base@23@@Z 0000000039a43bd0 f i CryGameSpySBQR2MatchMaking.obj
 0001:00042c50       ?_M_erase@?$_Rb_tree@IU?$less@I@stlpmtx_std@@U?$pair@$$CBIV?$vector@USCrySessionSearchData@@V?$allocator@USCrySessionSearchData@@@stlpmtx_std@@@stlpmtx_std@@@2@U?$_Select1st@U?$pair@$$CBIV?$vector@USCrySessionSearchData@@V?$allocator@USCrySessionSearchData@@@stlpmtx_std@@@stlpmtx_std@@@stlpmtx_std@@@priv@2@U?$_MapTraitsT@U?$pair@$$CBIV?$vector@USCrySessionSearchData@@V?$allocator@USCrySessionSearchData@@@stlpmtx_std@@@stlpmtx_std@@@stlpmtx_std@@@52@V?$allocator@U?$pair@$$CBIV?$vector@USCrySessionSearchData@@V?$allocator@USCrySessionSearchData@@@stlpmtx_std@@@stlpmtx_std@@@stlpmtx_std@@@2@@priv@stlpmtx_std@@AEAAXPEAU_Rb_tree_node_base@23@@Z 0000000039a43c50 f i CryGameSpySBQR2MatchMaking.obj
 0001:00042d40       ?AddRemoteConnectionNNComplete@CCryGameSpySBQR2MatchMaking@@KAXUSResult@CGameSpySBQR2NATNegotiation@@H_KPEAUsockaddr_in@@PEAUIGameSpyLink@@@Z 0000000039a43d40 f   CryGameSpySBQR2MatchMaking.obj
 0001:00042f00       ?AddRemoteConnection@CCryGameSpySBQR2MatchMaking@@IEAA?AV?$CryLobbyID@USCryMatchMakingConnectionID@@$0EA@@@V?$CryLobbyID@USCryLobbySessionHandle@@$03@@V?$CryLobbyID@USCryLobbyConnectionID@@$0EA@@@USCryMatchMakingConnectionUID@@IGIGIGIPEBDQEAE_N@Z 0000000039a43f00 f   CryGameSpySBQR2MatchMaking.obj
 0001:000431e0       ?BannedUserGetInfoCallback@CCryGameSpySBQR2MatchMaking@@KAXPEAVCGameSpySBQR2GPConnection@@USResult@2@PEAUGPGetInfoResponseArg@@PEAUIGameSpyLink@@@Z 0000000039a441e0 f   CryGameSpySBQR2MatchMaking.obj
 0001:00043270       ?BannedUserProfileSearchCallback@CCryGameSpySBQR2MatchMaking@@KAXPEAVCGameSpySBQR2GPConnection@@USResult@2@PEAUGPProfileSearchResponseArg@@PEAUIGameSpyLink@@@Z 0000000039a44270 f   CryGameSpySBQR2MatchMaking.obj
 0001:00043310       ?ProcessCDKeyResponse@CCryGameSpySBQR2MatchMaking@@IEAAXAEBV?$CConfigurableVariant@V?$CNode@USNullAddr@@V?$CNode@GV?$CNode@USIPv4Addr@@V?$CNode@ULobbyIdAddr@@VCEnd@NTypelist@@@NTypelist@@@NTypelist@@@NTypelist@@@NTypelist@@$07VCDefaultVariantConversion@NConfigurableVariantHelpers@@VCDefaultVariantConstruction@4@@@PEAVCCrySharedLobbyPacket@@@Z 0000000039a44310 f   CryGameSpySBQR2MatchMaking.obj
 0001:000434d0       ??$?AE@?$map@EV?$_smart_ptr@USGameSpyKey@CCryGameSpySBQR2MatchMaking@@@@U?$less@E@stlpmtx_std@@V?$allocator@U?$pair@$$CBEV?$_smart_ptr@USGameSpyKey@CCryGameSpySBQR2MatchMaking@@@@@stlpmtx_std@@@3@@stlpmtx_std@@QEAAAEAV?$_smart_ptr@USGameSpyKey@CCryGameSpySBQR2MatchMaking@@@@AEBE@Z 0000000039a444d0 f i CryGameSpySBQR2MatchMaking.obj
 0001:00043550       ??$?APEBD@?$map@PEBDV?$_smart_ptr@USGameSpyKey@CCryGameSpySBQR2MatchMaking@@@@U?$less@PEBD@stlpmtx_std@@V?$allocator@U?$pair@QEBDV?$_smart_ptr@USGameSpyKey@CCryGameSpySBQR2MatchMaking@@@@@stlpmtx_std@@@3@@stlpmtx_std@@QEAAAEAV?$_smart_ptr@USGameSpyKey@CCryGameSpySBQR2MatchMaking@@@@AEBQEBD@Z 0000000039a44550 f i CryGameSpySBQR2MatchMaking.obj
 0001:000435d0       ??$?AI@?$map@IV?$_smart_ptr@USGameSpyKey@CCryGameSpySBQR2MatchMaking@@@@U?$less@I@stlpmtx_std@@V?$allocator@U?$pair@$$CBIV?$_smart_ptr@USGameSpyKey@CCryGameSpySBQR2MatchMaking@@@@@stlpmtx_std@@@3@@stlpmtx_std@@QEAAAEAV?$_smart_ptr@USGameSpyKey@CCryGameSpySBQR2MatchMaking@@@@AEBI@Z 0000000039a445d0 f i CryGameSpySBQR2MatchMaking.obj
 0001:000435d0       ??$?AI@?$map@IV?$_smart_ptr@USRegisteredLobbyData@CCryGameSpySBQR2MatchMaking@@@@U?$less@I@stlpmtx_std@@V?$allocator@U?$pair@$$CBIV?$_smart_ptr@USRegisteredLobbyData@CCryGameSpySBQR2MatchMaking@@@@@stlpmtx_std@@@3@@stlpmtx_std@@QEAAAEAV?$_smart_ptr@USRegisteredLobbyData@CCryGameSpySBQR2MatchMaking@@@@AEBI@Z 0000000039a445d0 f i CryGameSpySBQR2MatchMaking.obj
 0001:00043650       ??$Add@P6AXIW4ECryLobbyError@@PEAUSCrySessionSearchResult@@PEAX@ZIW41@PEAU2@PEAXVCCryGameSpySBQR2MatchMaking@@@CWorkQueue@@QEAAXP8CCryGameSpySBQR2MatchMaking@@EAAXP6AXIW4ECryLobbyError@@PEAUSCrySessionSearchResult@@PEAX@ZI012@ZPEAV1@3I012@Z 0000000039a44650 f i CryGameSpySBQR2MatchMaking.obj
 0001:00043740       ??$Add@IIIIVCCryGameSpySBQR2MatchMaking@@@CWorkQueue@@QEAAXP8CCryGameSpySBQR2MatchMaking@@EAAXIIII@ZPEAV1@IIII@Z 0000000039a44740 f i CryGameSpySBQR2MatchMaking.obj
 0001:00043820       ?_M_create_node@?$_Rb_tree@IU?$less@I@stlpmtx_std@@U?$pair@$$CBIV?$vector@USCrySessionSearchData@@V?$allocator@USCrySessionSearchData@@@stlpmtx_std@@@stlpmtx_std@@@2@U?$_Select1st@U?$pair@$$CBIV?$vector@USCrySessionSearchData@@V?$allocator@USCrySessionSearchData@@@stlpmtx_std@@@stlpmtx_std@@@stlpmtx_std@@@priv@2@U?$_MapTraitsT@U?$pair@$$CBIV?$vector@USCrySessionSearchData@@V?$allocator@USCrySessionSearchData@@@stlpmtx_std@@@stlpmtx_std@@@stlpmtx_std@@@52@V?$allocator@U?$pair@$$CBIV?$vector@USCrySessionSearchData@@V?$allocator@USCrySessionSearchData@@@stlpmtx_std@@@stlpmtx_std@@@stlpmtx_std@@@2@@priv@stlpmtx_std@@IEAAPEAU_Rb_tree_node_base@23@AEBU?$pair@$$CBIV?$vector@USCrySessionSearchData@@V?$allocator@USCrySessionSearchData@@@stlpmtx_std@@@stlpmtx_std@@@3@@Z 0000000039a44820 f i CryGameSpySBQR2MatchMaking.obj
 0001:000438a0       ?AddGameSpyKey@CCryGameSpySBQR2MatchMaking@@IEAAXW4qr2_key_type@@IIEPEBDP81@EAAXPEAUSServer@SSearch@1@PEAUSGameSpyKey@1@I@ZP81@EAAXV?$CryLobbyID@USCryLobbySessionHandle@@$03@@3IPEAUqr2_buffer_s@@@Z@Z 0000000039a448a0 f   CryGameSpySBQR2MatchMaking.obj
 0001:00043bb0       ?StartSessionEnd@CCryGameSpySBQR2MatchMaking@@IEAAXI@Z 0000000039a44bb0 f   CryGameSpySBQR2MatchMaking.obj
 0001:00043bb0       ?StartSessionStart@CCryGameSpySBQR2MatchMaking@@IEAAXI@Z 0000000039a44bb0 f   CryGameSpySBQR2MatchMaking.obj
 0001:00043bb0       ?StopTaskRunning@CCryGameSpySBQR2MatchMaking@@IEAAXI@Z 0000000039a44bb0 f   CryGameSpySBQR2MatchMaking.obj
 0001:00043c20       ?StartSessionQuery@CCryGameSpySBQR2MatchMaking@@IEAAXI@Z 0000000039a44c20 f   CryGameSpySBQR2MatchMaking.obj
 0001:00043d40       ?TickSessionQuery@CCryGameSpySBQR2MatchMaking@@IEAAXI@Z 0000000039a44d40 f   CryGameSpySBQR2MatchMaking.obj
 0001:00043ec0       ?TickSessionJoinFindUseAddress@CCryGameSpySBQR2MatchMaking@@IEAAXI@Z 0000000039a44ec0 f   CryGameSpySBQR2MatchMaking.obj
 0001:00043fe0       ?TickSessionJoin@CCryGameSpySBQR2MatchMaking@@IEAAXI@Z 0000000039a44fe0 f   CryGameSpySBQR2MatchMaking.obj
 0001:00044300       ?TickSessionSearchWaitStart@CCryGameSpySBQR2MatchMaking@@IEAAXI@Z 0000000039a45300 f   CryGameSpySBQR2MatchMaking.obj
 0001:00044420       ?FormatSearchTerm@CCryGameSpySBQR2MatchMaking@@IEAAXPEBDPEBUSCrySessionSearchData@@AEAV?$CryFixedStringT@$0BPP@@@@Z 0000000039a45420 f   CryGameSpySBQR2MatchMaking.obj
 0001:00044670       ?StartSessionDelete@CCryGameSpySBQR2MatchMaking@@IEAAXI@Z 0000000039a45670 f   CryGameSpySBQR2MatchMaking.obj
 0001:000448a0       ?StartSessionSetLocalUserData@CCryGameSpySBQR2MatchMaking@@IEAAXI@Z 0000000039a458a0 f   CryGameSpySBQR2MatchMaking.obj
 0001:00044ae0       ?SetSessionUserData@CCryGameSpySBQR2MatchMaking@@IEAA?AW4ECryLobbyError@@V?$CryLobbyID@USCryLobbySessionHandle@@$03@@PEAUSCryLobbyUserData@@I@Z 0000000039a45ae0 f   CryGameSpySBQR2MatchMaking.obj
 0001:00044ca0       ?FilterServerByKeys@CCryGameSpySBQR2MatchMaking@@IEAAXPEAUSServer@SSearch@1@PEAUSCrySessionSearchParam@@PEAUSCrySessionSearchData@@@Z 0000000039a45ca0 f   CryGameSpySBQR2MatchMaking.obj
 0001:00044e20       ?ProcessSessionRequestJoin@CCryGameSpySBQR2MatchMaking@@IEAAXAEBV?$CConfigurableVariant@V?$CNode@USNullAddr@@V?$CNode@GV?$CNode@USIPv4Addr@@V?$CNode@ULobbyIdAddr@@VCEnd@NTypelist@@@NTypelist@@@NTypelist@@@NTypelist@@@NTypelist@@$07VCDefaultVariantConversion@NConfigurableVariantHelpers@@VCDefaultVariantConstruction@4@@@PEAVCCrySharedLobbyPacket@@@Z 0000000039a45e20 f   CryGameSpySBQR2MatchMaking.obj
 0001:00045530       ?ProcessSessionAddRemoteConnections@CCryGameSpySBQR2MatchMaking@@IEAAXAEBV?$CConfigurableVariant@V?$CNode@USNullAddr@@V?$CNode@GV?$CNode@USIPv4Addr@@V?$CNode@ULobbyIdAddr@@VCEnd@NTypelist@@@NTypelist@@@NTypelist@@@NTypelist@@@NTypelist@@$07VCDefaultVariantConversion@NConfigurableVariantHelpers@@VCDefaultVariantConstruction@4@@@PEAVCCrySharedLobbyPacket@@@Z 0000000039a46530 f   CryGameSpySBQR2MatchMaking.obj
 0001:00045b80       ?ProcessSessionRequestJoinResult@CCryGameSpySBQR2MatchMaking@@IEAAXAEBV?$CConfigurableVariant@V?$CNode@USNullAddr@@V?$CNode@GV?$CNode@USIPv4Addr@@V?$CNode@ULobbyIdAddr@@VCEnd@NTypelist@@@NTypelist@@@NTypelist@@@NTypelist@@@NTypelist@@$07VCDefaultVariantConversion@NConfigurableVariantHelpers@@VCDefaultVariantConstruction@4@@@PEAVCCrySharedLobbyPacket@@@Z 0000000039a46b80 f   CryGameSpySBQR2MatchMaking.obj
 0001:00046110       ?BanCmd@CCryGameSpySBQR2MatchMaking@@MEAAX_KM@Z 0000000039a47110 f   CryGameSpySBQR2MatchMaking.obj
 0001:00046500       ?BanCmd@CCryGameSpySBQR2MatchMaking@@MEAAXPEBDM@Z 0000000039a47500 f   CryGameSpySBQR2MatchMaking.obj
 0001:00046880       ?LoadBannedUserList@CCryGameSpySBQR2MatchMaking@@IEAAXVCTimeValue@@@Z 0000000039a47880 f   CryGameSpySBQR2MatchMaking.obj
 0001:00046fa0       ?TickSessionSendRequestInfoNAT@CCryGameSpySBQR2MatchMaking@@IEAAXI@Z 0000000039a47fa0 f   CryGameSpySBQR2MatchMaking.obj
 0001:00047020       ?TickSessionSendRequestInfo@CCryGameSpySBQR2MatchMaking@@IEAAXI@Z 0000000039a48020 f   CryGameSpySBQR2MatchMaking.obj
 0001:00047200       ?ProcessSessionRequestInfo@CCryGameSpySBQR2MatchMaking@@IEAAXAEBV?$CConfigurableVariant@V?$CNode@USNullAddr@@V?$CNode@GV?$CNode@USIPv4Addr@@V?$CNode@ULobbyIdAddr@@VCEnd@NTypelist@@@NTypelist@@@NTypelist@@@NTypelist@@@NTypelist@@$07VCDefaultVariantConversion@NConfigurableVariantHelpers@@VCDefaultVariantConstruction@4@@@PEAVCCrySharedLobbyPacket@@@Z 0000000039a48200 f   CryGameSpySBQR2MatchMaking.obj
 0001:000474b0       ?SessionSendRequestInfoResponse@CCryGameSpySBQR2MatchMaking@@UEAA?AW4ECryLobbyError@@PEAVCCryLobbyPacket@@PEAX@Z 0000000039a484b0 f   CryGameSpySBQR2MatchMaking.obj
 0001:000477a0       ?ProcessSessionRequestInfoResponse@CCryGameSpySBQR2MatchMaking@@IEAAXAEBV?$CConfigurableVariant@V?$CNode@USNullAddr@@V?$CNode@GV?$CNode@USIPv4Addr@@V?$CNode@ULobbyIdAddr@@VCEnd@NTypelist@@@NTypelist@@@NTypelist@@@NTypelist@@@NTypelist@@$07VCDefaultVariantConversion@NConfigurableVariantHelpers@@VCDefaultVariantConstruction@4@@@PEAVCCrySharedLobbyPacket@@@Z 0000000039a487a0 f   CryGameSpySBQR2MatchMaking.obj
 0001:000479c0       ?_M_insert@?$_Rb_tree@IU?$less@I@stlpmtx_std@@U?$pair@$$CBIV?$vector@USCrySessionSearchData@@V?$allocator@USCrySessionSearchData@@@stlpmtx_std@@@stlpmtx_std@@@2@U?$_Select1st@U?$pair@$$CBIV?$vector@USCrySessionSearchData@@V?$allocator@USCrySessionSearchData@@@stlpmtx_std@@@stlpmtx_std@@@stlpmtx_std@@@priv@2@U?$_MapTraitsT@U?$pair@$$CBIV?$vector@USCrySessionSearchData@@V?$allocator@USCrySessionSearchData@@@stlpmtx_std@@@stlpmtx_std@@@stlpmtx_std@@@52@V?$allocator@U?$pair@$$CBIV?$vector@USCrySessionSearchData@@V?$allocator@USCrySessionSearchData@@@stlpmtx_std@@@stlpmtx_std@@@stlpmtx_std@@@2@@priv@stlpmtx_std@@AEAA?AU?$_Rb_tree_iterator@U?$pair@$$CBIV?$vector@USCrySessionSearchData@@V?$allocator@USCrySessionSearchData@@@stlpmtx_std@@@stlpmtx_std@@@stlpmtx_std@@U?$_MapTraitsT@U?$pair@$$CBIV?$vector@USCrySessionSearchData@@V?$allocator@USCrySessionSearchData@@@stlpmtx_std@@@stlpmtx_std@@@stlpmtx_std@@@priv@2@@23@PEAU_Rb_tree_node_base@23@AEBU?$pair@$$CBIV?$vector@USCrySessionSearchData@@V?$allocator@USCrySessionSearchData@@@stlpmtx_std@@@stlpmtx_std@@@3@00@Z 0000000039a489c0 f i CryGameSpySBQR2MatchMaking.obj
 0001:00047a80       ?insert_unique@?$_Rb_tree@IU?$less@I@stlpmtx_std@@U?$pair@$$CBIV?$vector@USCrySessionSearchData@@V?$allocator@USCrySessionSearchData@@@stlpmtx_std@@@stlpmtx_std@@@2@U?$_Select1st@U?$pair@$$CBIV?$vector@USCrySessionSearchData@@V?$allocator@USCrySessionSearchData@@@stlpmtx_std@@@stlpmtx_std@@@stlpmtx_std@@@priv@2@U?$_MapTraitsT@U?$pair@$$CBIV?$vector@USCrySessionSearchData@@V?$allocator@USCrySessionSearchData@@@stlpmtx_std@@@stlpmtx_std@@@stlpmtx_std@@@52@V?$allocator@U?$pair@$$CBIV?$vector@USCrySessionSearchData@@V?$allocator@USCrySessionSearchData@@@stlpmtx_std@@@stlpmtx_std@@@stlpmtx_std@@@2@@priv@stlpmtx_std@@QEAA?AU?$pair@U?$_Rb_tree_iterator@U?$pair@$$CBIV?$vector@USCrySessionSearchData@@V?$allocator@USCrySessionSearchData@@@stlpmtx_std@@@stlpmtx_std@@@stlpmtx_std@@U?$_MapTraitsT@U?$pair@$$CBIV?$vector@USCrySessionSearchData@@V?$allocator@USCrySessionSearchData@@@stlpmtx_std@@@stlpmtx_std@@@stlpmtx_std@@@priv@2@@priv@stlpmtx_std@@_N@3@AEBU?$pair@$$CBIV?$vector@USCrySessionSearchData@@V?$allocator@USCrySessionSearchData@@@stlpmtx_std@@@stlpmtx_std@@@3@@Z 0000000039a48a80 f i CryGameSpySBQR2MatchMaking.obj
 0001:00047c80       ?OnPacket@CCryGameSpySBQR2MatchMaking@@QEAAXAEBV?$CConfigurableVariant@V?$CNode@USNullAddr@@V?$CNode@GV?$CNode@USIPv4Addr@@V?$CNode@ULobbyIdAddr@@VCEnd@NTypelist@@@NTypelist@@@NTypelist@@@NTypelist@@@NTypelist@@$07VCDefaultVariantConversion@NConfigurableVariantHelpers@@VCDefaultVariantConstruction@4@@@PEAVCCryLobbyPacket@@@Z 0000000039a48c80 f   CryGameSpySBQR2MatchMaking.obj
 0001:00047d80       ?StartTaskRunning@CCryGameSpySBQR2MatchMaking@@IEAAXI@Z 0000000039a48d80 f   CryGameSpySBQR2MatchMaking.obj
 0001:00047f80       ?TickSessionUpdate@CCryGameSpySBQR2MatchMaking@@IEAAXI@Z 0000000039a48f80 f   CryGameSpySBQR2MatchMaking.obj
 0001:00048090       ?SetSessionData@CCryGameSpySBQR2MatchMaking@@IEAA?AW4ECryLobbyError@@V?$CryLobbyID@USCryLobbySessionHandle@@$03@@PEAUSCrySessionData@@@Z 0000000039a49090 f   CryGameSpySBQR2MatchMaking.obj
 0001:000481e0       ?SessionSearchServerBrowserCallback@CCryGameSpySBQR2MatchMaking@@KAXW4SBCallbackReason@@PEAU_SBServer@@PEAX@Z 0000000039a491e0 f   CryGameSpySBQR2MatchMaking.obj
 0001:000485e0       ?Reset@SSession@CCryGameSpySBQR2MatchMaking@@UEAAXXZ 0000000039a495e0 f   CryGameSpySBQR2MatchMaking.obj
 0001:00048670       ?ProcessBannedUserList@CCryGameSpySBQR2MatchMaking@@IEAAXVCTimeValue@@@Z 0000000039a49670 f   CryGameSpySBQR2MatchMaking.obj
 0001:00048960       ?SessionSendRequestInfo@CCryGameSpySBQR2MatchMaking@@UEAA?AW4ECryLobbyError@@PEAVCCryLobbyPacket@@V?$_smart_ptr@USCrySessionID@@@@PEAIP6AXIW42@0PEAX@Z4@Z 0000000039a49960 f   CryGameSpySBQR2MatchMaking.obj
 0001:00048d40       ?insert_unique@?$_Rb_tree@IU?$less@I@stlpmtx_std@@U?$pair@$$CBIV?$vector@USCrySessionSearchData@@V?$allocator@USCrySessionSearchData@@@stlpmtx_std@@@stlpmtx_std@@@2@U?$_Select1st@U?$pair@$$CBIV?$vector@USCrySessionSearchData@@V?$allocator@USCrySessionSearchData@@@stlpmtx_std@@@stlpmtx_std@@@stlpmtx_std@@@priv@2@U?$_MapTraitsT@U?$pair@$$CBIV?$vector@USCrySessionSearchData@@V?$allocator@USCrySessionSearchData@@@stlpmtx_std@@@stlpmtx_std@@@stlpmtx_std@@@52@V?$allocator@U?$pair@$$CBIV?$vector@USCrySessionSearchData@@V?$allocator@USCrySessionSearchData@@@stlpmtx_std@@@stlpmtx_std@@@stlpmtx_std@@@2@@priv@stlpmtx_std@@QEAA?AU?$_Rb_tree_iterator@U?$pair@$$CBIV?$vector@USCrySessionSearchData@@V?$allocator@USCrySessionSearchData@@@stlpmtx_std@@@stlpmtx_std@@@stlpmtx_std@@U?$_MapTraitsT@U?$pair@$$CBIV?$vector@USCrySessionSearchData@@V?$allocator@USCrySessionSearchData@@@stlpmtx_std@@@stlpmtx_std@@@stlpmtx_std@@@priv@2@@23@U423@AEBU?$pair@$$CBIV?$vector@USCrySessionSearchData@@V?$allocator@USCrySessionSearchData@@@stlpmtx_std@@@stlpmtx_std@@@3@@Z 0000000039a49d40 f i CryGameSpySBQR2MatchMaking.obj
 0001:00049180       ??0SSession@CCryGameSpySBQR2MatchMaking@@QEAA@XZ 0000000039a4a180 f i CryGameSpySBQR2MatchMaking.obj
 0001:000492e0       ??1SSession@CCryGameSpySBQR2MatchMaking@@UEAA@XZ 0000000039a4a2e0 f i CryGameSpySBQR2MatchMaking.obj
 0001:000493a0       ??_ESSession@CCryGameSpySBQR2MatchMaking@@UEAAPEAXI@Z 0000000039a4a3a0 f i CryGameSpySBQR2MatchMaking.obj
 0001:000493a0       ??_GSSession@CCryGameSpySBQR2MatchMaking@@UEAAPEAXI@Z 0000000039a4a3a0 f i CryGameSpySBQR2MatchMaking.obj
 0001:000493d0       ?SessionRegisterUserData@CCryGameSpySBQR2MatchMaking@@UEAA?AW4ECryLobbyError@@PEAUSCryLobbyUserData@@IPEAIP6AXIW42@PEAX@Z3@Z 0000000039a4a3d0 f   CryGameSpySBQR2MatchMaking.obj
 0001:0004a4c0       ?SessionCreate@CCryGameSpySBQR2MatchMaking@@UEAA?AW4ECryLobbyError@@PEAIHIPEAUSCrySessionData@@0P6AXIW42@IPEAX@Z3@Z 0000000039a4b4c0 f   CryGameSpySBQR2MatchMaking.obj
 0001:0004a750       ?SessionJoin@CCryGameSpySBQR2MatchMaking@@UEAA?AW4ECryLobbyError@@PEAIHIV?$_smart_ptr@USCrySessionID@@@@0P6AXIW42@IIGPEAX@Z3@Z 0000000039a4b750 f   CryGameSpySBQR2MatchMaking.obj
 0001:0004aa40       ?SessionSearch@CCryGameSpySBQR2MatchMaking@@UEAA?AW4ECryLobbyError@@IPEAUSCrySessionSearchParam@@PEAIP6AXIW42@PEAUSCrySessionSearchResult@@PEAX@Z4@Z 0000000039a4ba40 f   CryGameSpySBQR2MatchMaking.obj
 0001:0004ab90       ?SessionDelete@CCryGameSpySBQR2MatchMaking@@UEAA?AW4ECryLobbyError@@IPEAIP6AXIW42@PEAX@Z2@Z 0000000039a4bb90 f   CryGameSpySBQR2MatchMaking.obj
 0001:0004aca0       ?SessionMigrate@CCryGameSpySBQR2MatchMaking@@UEAA?AW4ECryLobbyError@@IPEAIHIPEAUSCrySessionData@@0P6AXIW42@IPEAX@Z3@Z 0000000039a4bca0 f   CryGameSpySBQR2MatchMaking.obj
 0001:0004adb0       ?SessionUpdate@CCryGameSpySBQR2MatchMaking@@UEAA?AW4ECryLobbyError@@IPEAUSCryLobbyUserData@@IPEAIP6AXIW42@PEAX@Z3@Z 0000000039a4bdb0 f   CryGameSpySBQR2MatchMaking.obj
 0001:0004af20       ?SessionUpdateSlots@CCryGameSpySBQR2MatchMaking@@UEAA?AW4ECryLobbyError@@IIIPEAIP6AXIW42@PEAX@Z2@Z 0000000039a4bf20 f   CryGameSpySBQR2MatchMaking.obj
 0001:0004b040       ?SessionQuery@CCryGameSpySBQR2MatchMaking@@UEAA?AW4ECryLobbyError@@IPEAIP6AXIW42@PEAUSCrySessionSearchResult@@PEAX@Z3@Z 0000000039a4c040 f   CryGameSpySBQR2MatchMaking.obj
 0001:0004b1a0       ?SessionGetUsers@CCryGameSpySBQR2MatchMaking@@UEAA?AW4ECryLobbyError@@IPEAIP6AXIW42@PEAUSCryUserInfoResult@@PEAX@Z3@Z 0000000039a4c1a0 f   CryGameSpySBQR2MatchMaking.obj
 0001:0004b2b0       ?SessionStart@CCryGameSpySBQR2MatchMaking@@UEAA?AW4ECryLobbyError@@IPEAIP6AXIW42@PEAX@Z2@Z 0000000039a4c2b0 f   CryGameSpySBQR2MatchMaking.obj
 0001:0004b3d0       ?SessionEnd@CCryGameSpySBQR2MatchMaking@@UEAA?AW4ECryLobbyError@@IPEAIP6AXIW42@PEAX@Z2@Z 0000000039a4c3d0 f   CryGameSpySBQR2MatchMaking.obj
 0001:0004b4f0       ?SessionSetLocalUserData@CCryGameSpySBQR2MatchMaking@@UEAA?AW4ECryLobbyError@@IPEAIIPEAEIP6AXIW42@PEAX@Z3@Z 0000000039a4c4f0 f   CryGameSpySBQR2MatchMaking.obj
 0001:0004b620       ?TickSessionCreate@CCryGameSpySBQR2MatchMaking@@IEAAXI@Z 0000000039a4c620 f   CryGameSpySBQR2MatchMaking.obj
 0001:0004b9c0       ??1CCryGameSpySBQR2MatchMaking@@UEAA@XZ 0000000039a4c9c0 f   CryGameSpySBQR2MatchMaking.obj
 0001:0004bd90       ??_ECCryGameSpySBQR2MatchMaking@@WBA@EAAPEAXI@Z 0000000039a4cd90 f i CryGameSpySBQR2MatchMaking.obj
 0001:0004bda0       ??$?AI@?$map@IV?$vector@USCrySessionSearchData@@V?$allocator@USCrySessionSearchData@@@stlpmtx_std@@@stlpmtx_std@@U?$less@I@2@V?$allocator@U?$pair@$$CBIV?$vector@USCrySessionSearchData@@V?$allocator@USCrySessionSearchData@@@stlpmtx_std@@@stlpmtx_std@@@stlpmtx_std@@@2@@stlpmtx_std@@QEAAAEAV?$vector@USCrySessionSearchData@@V?$allocator@USCrySessionSearchData@@@stlpmtx_std@@@1@AEBI@Z 0000000039a4cda0 f i CryGameSpySBQR2MatchMaking.obj
 0001:0004bf30       ??0CCryGameSpySBQR2MatchMaking@@QEAA@PEAVCCryLobby@@PEAVCCryLobbyService@@W4ECryLobbyService@@@Z 0000000039a4cf30 f   CryGameSpySBQR2MatchMaking.obj
 0001:0004e090       ??_ECCryGameSpySBQR2MatchMaking@@UEAAPEAXI@Z 0000000039a4f090 f i CryGameSpySBQR2MatchMaking.obj
 0001:0004e090       ??_GCCryGameSpySBQR2MatchMaking@@UEAAPEAXI@Z 0000000039a4f090 f i CryGameSpySBQR2MatchMaking.obj
 0001:0004e0c0       ?TickSessionSearch@CCryGameSpySBQR2MatchMaking@@IEAAXI@Z 0000000039a4f0c0 f   CryGameSpySBQR2MatchMaking.obj
 0001:0004f620       ?Tick@CCryGameSpySBQR2MatchMaking@@QEAAXVCTimeValue@@@Z 0000000039a50620 f   CryGameSpySBQR2MatchMaking.obj
 0001:0004f860       ?Terminate@CCryGameSpySBQR2SignIn@@UEAA?AW4ECryLobbyError@@XZ 0000000039a50860 f   CryGameSpySBQR2SignIn.obj
 0001:0004f870       ?StartTaskRunning@CCryGameSpySBQR2SignIn@@MEAAXV?$CryLobbyID@USCrySignInTaskID@CCrySignIn@@$03@@@Z 0000000039a50870 f   CryGameSpySBQR2SignIn.obj
 0001:0004f8c0       ?SignInUserConnectCallback@CCryGameSpySBQR2SignIn@@CAXPEAVCGameSpySBQR2GPConnection@@USResult@2@PEAUGPConnectResponseArg@@PEAUIGameSpyLink@@@Z 0000000039a508c0 f   CryGameSpySBQR2SignIn.obj
 0001:0004f9c0       ?StartSignInUser@CCryGameSpySBQR2SignIn@@AEAAXV?$CryLobbyID@USCrySignInTaskID@CCrySignIn@@$03@@@Z 0000000039a509c0 f   CryGameSpySBQR2SignIn.obj
 0001:0004fb20       ?StartSignOutUser@CCryGameSpySBQR2SignIn@@AEAAXV?$CryLobbyID@USCrySignInTaskID@CCrySignIn@@$03@@@Z 0000000039a50b20 f   CryGameSpySBQR2SignIn.obj
 0001:0004fbc0       ?EndSignOutUser@CCryGameSpySBQR2SignIn@@AEAAXV?$CryLobbyID@USCrySignInTaskID@CCrySignIn@@$03@@@Z 0000000039a50bc0 f   CryGameSpySBQR2SignIn.obj
 0001:0004fc20       ?EndCreateUser@CCryGameSpySBQR2SignIn@@AEAAXV?$CryLobbyID@USCrySignInTaskID@CCrySignIn@@$03@@@Z 0000000039a50c20 f   CryGameSpySBQR2SignIn.obj
 0001:0004fcb0       ?CreateUserNewUserCallback@CCryGameSpySBQR2SignIn@@CAXPEAVCGameSpySBQR2GPConnection@@USResult@2@PEAUGPNewUserResponseArg@@PEAUIGameSpyLink@@@Z 0000000039a50cb0 f   CryGameSpySBQR2SignIn.obj
 0001:0004fdd0       ?CreateUserProfileSearchCallback@CCryGameSpySBQR2SignIn@@CAXPEAVCGameSpySBQR2GPConnection@@USResult@2@PEAUGPProfileSearchResponseArg@@PEAUIGameSpyLink@@@Z 0000000039a50dd0 f   CryGameSpySBQR2SignIn.obj
 0001:00050180       ?CreateUserConnectAnyCallback@CCryGameSpySBQR2SignIn@@CAXPEAVCGameSpySBQR2GPConnection@@USResult@2@PEAUGPConnectResponseArg@@PEAUIGameSpyLink@@@Z 0000000039a51180 f   CryGameSpySBQR2SignIn.obj
 0001:00050250       ?CreateUserNewProfileCallback@CCryGameSpySBQR2SignIn@@CAXPEAVCGameSpySBQR2GPConnection@@USResult@2@PEAUGPNewProfileResponseArg@@PEAUIGameSpyLink@@@Z 0000000039a51250 f   CryGameSpySBQR2SignIn.obj
 0001:00050300       ?CreateUserConnectRequiredCallback@CCryGameSpySBQR2SignIn@@CAXPEAVCGameSpySBQR2GPConnection@@USResult@2@PEAUGPConnectResponseArg@@PEAUIGameSpyLink@@@Z 0000000039a51300 f   CryGameSpySBQR2SignIn.obj
 0001:00050490       ?CreateUserRegisterUniqueNickCallback@CCryGameSpySBQR2SignIn@@CAXPEAVCGameSpySBQR2GPConnection@@USResult@2@PEAUGPRegisterUniqueNickResponseArg@@PEAUIGameSpyLink@@@Z 0000000039a51490 f   CryGameSpySBQR2SignIn.obj
 0001:00050590       ?CreateUserCheckUserCallback@CCryGameSpySBQR2SignIn@@CAXPEAVCGameSpySBQR2GPConnection@@USResult@2@PEAUGPCheckResponseArg@@PEAUIGameSpyLink@@@Z 0000000039a51590 f   CryGameSpySBQR2SignIn.obj
 0001:00050650       ?TickGetUserCredentials@CCryGameSpySBQR2SignIn@@AEAAXV?$CryLobbyID@USCrySignInTaskID@CCrySignIn@@$03@@@Z 0000000039a51650 f   CryGameSpySBQR2SignIn.obj
 0001:000506a0       ?CreateTask@CCryGameSpySBQR2SignIn@@MEAAXV?$CryLobbyID@USCrySignInTaskID@CCrySignIn@@$03@@IIPEAX1@Z 0000000039a516a0 f   CryGameSpySBQR2SignIn.obj
 0001:00050720       ?set_size@?$SmallDynStorage@USUserCredential@@HUStandardAlloc@NAlloc@@@NArray@@QEAAXH@Z 0000000039a51720 f i CryGameSpySBQR2SignIn.obj
 0001:000507d0       ??_G?$CClassJobNoRef@IVCCryGameSpySBQR2LobbyUI@@@CWorkQueue@@UEAAPEAXI@Z 0000000039a517d0 f i CryGameSpySBQR2LobbyUI.obj
 0001:000507d0       ??_E?$CClassJobNoRef@IVCCryGameSpySBQR2DLCStore@@@CWorkQueue@@UEAAPEAXI@Z 0000000039a517d0 f i CryGameSpySBQR2DLCStore.obj
 0001:000507d0       ??_G?$CClassJobNoRef@IVCCryMatchMaking@@@CWorkQueue@@UEAAPEAXI@Z 0000000039a517d0 f i CryMatchMaking.obj
 0001:000507d0       ??_G?$CClassJobNoRef@V?$CryLobbyID@USCrySignInTaskID@CCrySignIn@@$03@@VCCrySignIn@@@CWorkQueue@@UEAAPEAXI@Z 0000000039a517d0 f i CrySignIn.obj
 0001:000507d0       ??_E?$CClassJobNoRef@IVCCryMatchMaking@@@CWorkQueue@@UEAAPEAXI@Z 0000000039a517d0 f i CryMatchMaking.obj
 0001:000507d0       ??_G?$CClassJobNoRef@IVCCryDLCStore@@@CWorkQueue@@UEAAPEAXI@Z 0000000039a517d0 f i CryDLCStore.obj
 0001:000507d0       ??_E?$CClassJobNoRef2@W4ECryLobbySystemEvent@@IVCCryMatchMaking@@@CWorkQueue@@UEAAPEAXI@Z 0000000039a517d0 f i CryMatchMaking.obj
 0001:000507d0       ??_E?$CClassJobNoRef@IVCCryLANMatchMaking@@@CWorkQueue@@UEAAPEAXI@Z 0000000039a517d0 f i CryLANMatchMaking.obj
 0001:000507d0       ??_G?$CClassJobNoRef2@IW4ECryLobbySystemEvent@@VCCryMatchMaking@@@CWorkQueue@@UEAAPEAXI@Z 0000000039a517d0 f i CryMatchMaking.obj
 0001:000507d0       ??_G?$CClassJobNoRef@IVCCryGameSpySBQR2MatchMaking@@@CWorkQueue@@UEAAPEAXI@Z 0000000039a517d0 f i CryGameSpySBQR2MatchMaking.obj
 0001:000507d0       ??_G?$CClassJobNoRef@IVCCryLANMatchMaking@@@CWorkQueue@@UEAAPEAXI@Z 0000000039a517d0 f i CryLANMatchMaking.obj
 0001:000507d0       ??_G?$CClassJobNoRef@IVCCryLobbyService@@@CWorkQueue@@UEAAPEAXI@Z 0000000039a517d0 f i CryLobby.obj
 0001:000507d0       ??_E?$CClassJobNoRef@V?$CryLobbyID@USCrySignInTaskID@CCrySignIn@@$03@@VCCrySignIn@@@CWorkQueue@@UEAAPEAXI@Z 0000000039a517d0 f i CrySignIn.obj
 0001:000507d0       ??_G?$CClassJobNoRef2@HW4EOnlineState@@VCCryGameSpySBQR2Friends@@@CWorkQueue@@UEAAPEAXI@Z 0000000039a517d0 f i CryGameSpySBQR2Friends.obj
 0001:000507d0       ??_G?$CClassJobNoRef@IVCCryGameSpySBQR2FriendsManagement@@@CWorkQueue@@UEAAPEAXI@Z 0000000039a517d0 f i CryGameSpySBQR2FriendsManagement.obj
 0001:000507d0       ??_E?$CClassJobNoRef@V?$CryLobbyID@USCrySignInTaskID@CCrySignIn@@$03@@VCCryGameSpySBQR2SignIn@@@CWorkQueue@@UEAAPEAXI@Z 0000000039a517d0 f i CryGameSpySBQR2SignIn.obj
 0001:000507d0       ??_E?$CClassJobNoRef@IVCCryGameSpySBQR2Stats@@@CWorkQueue@@UEAAPEAXI@Z 0000000039a517d0 f i CryGameSpySBQR2Stats.obj
 0001:000507d0       ??_E?$CClassJobNoRef@IVCCryGameSpySBQR2LobbyService@@@CWorkQueue@@UEAAPEAXI@Z 0000000039a517d0 f i CryGameSpySBQR2Lobby.obj
 0001:000507d0       ??_G?$CClassJobNoRef@IVCCryGameSpySBQR2Friends@@@CWorkQueue@@UEAAPEAXI@Z 0000000039a517d0 f i CryGameSpySBQR2Friends.obj
 0001:000507d0       ??_E?$CClassJobNoRef@IVCCryLobbyService@@@CWorkQueue@@UEAAPEAXI@Z 0000000039a517d0 f i CryLobby.obj
 0001:000507d0       ??_G?$CClassJobNoRef@IVCCryGameSpySBQR2Stats@@@CWorkQueue@@UEAAPEAXI@Z 0000000039a517d0 f i CryGameSpySBQR2Stats.obj
 0001:000507d0       ??_G?$CClassJobNoRef2@W4ECryLobbySystemEvent@@HVCCryGameSpySBQR2Friends@@@CWorkQueue@@UEAAPEAXI@Z 0000000039a517d0 f i CryGameSpySBQR2Friends.obj
 0001:000507d0       ??_E?$CClassJobNoRef@IVCCryGameSpySBQR2Friends@@@CWorkQueue@@UEAAPEAXI@Z 0000000039a517d0 f i CryGameSpySBQR2Friends.obj
 0001:000507d0       ??_G?$CClassJobNoRef@V?$CryLobbyID@USCrySignInTaskID@CCrySignIn@@$03@@VCCryGameSpySBQR2SignIn@@@CWorkQueue@@UEAAPEAXI@Z 0000000039a517d0 f i CryGameSpySBQR2SignIn.obj
 0001:000507d0       ??_E?$CClassJobNoRef@IVCCryGameSpySBQR2LobbyUI@@@CWorkQueue@@UEAAPEAXI@Z 0000000039a517d0 f i CryGameSpySBQR2LobbyUI.obj
 0001:000507d0       ??_G?$CClassJobNoRef2@W4ECryLobbySystemEvent@@IVCCryMatchMaking@@@CWorkQueue@@UEAAPEAXI@Z 0000000039a517d0 f i CryMatchMaking.obj
 0001:000507d0       ??_E?$CClassJobNoRef@IVCCryDLCStore@@@CWorkQueue@@UEAAPEAXI@Z 0000000039a517d0 f i CryDLCStore.obj
 0001:000507d0       ??_E?$CClassJobNoRef@IVCCryGameSpySBQR2MatchMaking@@@CWorkQueue@@UEAAPEAXI@Z 0000000039a517d0 f i CryGameSpySBQR2MatchMaking.obj
 0001:000507d0       ??_E?$CClassJobNoRef@IVCCryGameSpySBQR2FriendsManagement@@@CWorkQueue@@UEAAPEAXI@Z 0000000039a517d0 f i CryGameSpySBQR2FriendsManagement.obj
 0001:000507d0       ??_E?$CClassJobNoRef2@HW4EOnlineState@@VCCryGameSpySBQR2Friends@@@CWorkQueue@@UEAAPEAXI@Z 0000000039a517d0 f i CryGameSpySBQR2Friends.obj
 0001:000507d0       ??_E?$CClassJobNoRef2@IW4ECryLobbySystemEvent@@VCCryMatchMaking@@@CWorkQueue@@UEAAPEAXI@Z 0000000039a517d0 f i CryMatchMaking.obj
 0001:000507d0       ??_G?$CClassJobNoRef@IVCCryGameSpySBQR2DLCStore@@@CWorkQueue@@UEAAPEAXI@Z 0000000039a517d0 f i CryGameSpySBQR2DLCStore.obj
 0001:000507d0       ??_G?$CClassJobNoRef@IVCCryGameSpySBQR2LobbyService@@@CWorkQueue@@UEAAPEAXI@Z 0000000039a517d0 f i CryGameSpySBQR2Lobby.obj
 0001:000507d0       ??_E?$CClassJobNoRef2@W4ECryLobbySystemEvent@@HVCCryGameSpySBQR2Friends@@@CWorkQueue@@UEAAPEAXI@Z 0000000039a517d0 f i CryGameSpySBQR2Friends.obj
 0001:00050850       ??1SUser@CCryGameSpySBQR2SignIn@@QEAA@XZ 0000000039a51850 f i CryGameSpySBQR2SignIn.obj
 0001:00050900       ?StopTaskRunning@CCryGameSpySBQR2SignIn@@MEAAXV?$CryLobbyID@USCrySignInTaskID@CCrySignIn@@$03@@@Z 0000000039a51900 f   CryGameSpySBQR2SignIn.obj
 0001:000509d0       ?StartCreateUser@CCryGameSpySBQR2SignIn@@AEAAXV?$CryLobbyID@USCrySignInTaskID@CCrySignIn@@$03@@@Z 0000000039a519d0 f   CryGameSpySBQR2SignIn.obj
 0001:00050af0       ?TickCreateUser@CCryGameSpySBQR2SignIn@@AEAAXV?$CryLobbyID@USCrySignInTaskID@CCrySignIn@@$03@@@Z 0000000039a51af0 f   CryGameSpySBQR2SignIn.obj
 0001:00050df0       ?CreateTaskLink@CCryGameSpySBQR2SignIn@@AEAA?AW4ECryLobbyError@@V?$CryLobbyID@USCrySignInTaskID@CCrySignIn@@$03@@@Z 0000000039a51df0 f   CryGameSpySBQR2SignIn.obj
 0001:00050eb0       ?FreeTask@CCryGameSpySBQR2SignIn@@MEAAXV?$CryLobbyID@USCrySignInTaskID@CCrySignIn@@$03@@@Z 0000000039a51eb0 f   CryGameSpySBQR2SignIn.obj
 0001:00050f50       ??1?$CryLobbyIDArray@USTask@CCryGameSpySBQR2SignIn@@V?$CryLobbyID@USCrySignInTaskID@CCrySignIn@@$03@@$03@@QEAA@XZ 0000000039a51f50 f i CryGameSpySBQR2SignIn.obj
 0001:00050fd0       ??_ECCryGameSpySBQR2SignIn@@WBA@EAAPEAXI@Z 0000000039a51fd0 f i CryGameSpySBQR2SignIn.obj
 0001:00050fe0       ?Initialise@CCryGameSpySBQR2SignIn@@UEAA?AW4ECryLobbyError@@XZ 0000000039a51fe0 f   CryGameSpySBQR2SignIn.obj
 0001:00051050       ?GetUserCredentialsGetInfoCallback@CCryGameSpySBQR2SignIn@@CAXPEAVCGameSpySBQR2GPConnection@@USResult@2@PEAUGPGetInfoResponseArg@@PEAUIGameSpyLink@@@Z 0000000039a52050 f   CryGameSpySBQR2SignIn.obj
 0001:00051160       ??$move_init@USUserCredential@@@NArray@@YAXPEAUSUserCredential@@0_K@Z 0000000039a52160 f i CryGameSpySBQR2SignIn.obj
 0001:00051230       ??0CCryGameSpySBQR2SignIn@@QEAA@PEAVCCryLobby@@PEAVCCryGameSpySBQR2LobbyService@@@Z 0000000039a52230 f   CryGameSpySBQR2SignIn.obj
 0001:00051330       ??_GCCryGameSpySBQR2SignIn@@UEAAPEAXI@Z 0000000039a52330 f i CryGameSpySBQR2SignIn.obj
 0001:00051330       ??_ECCryGameSpySBQR2SignIn@@UEAAPEAXI@Z 0000000039a52330 f i CryGameSpySBQR2SignIn.obj
 0001:000513b0       ?StartGetUserCredentials@CCryGameSpySBQR2SignIn@@AEAAXV?$CryLobbyID@USCrySignInTaskID@CCrySignIn@@$03@@@Z 0000000039a523b0 f   CryGameSpySBQR2SignIn.obj
 0001:000514d0       ?resize_raw@?$SmallDynStorage@USUserCredential@@HUStandardAlloc@NAlloc@@@NArray@@QEAAXHH_N@Z 0000000039a524d0 f i CryGameSpySBQR2SignIn.obj
 0001:00051640       ?Tick@CCryGameSpySBQR2SignIn@@UEAAXVCTimeValue@@@Z 0000000039a52640 f   CryGameSpySBQR2SignIn.obj
 0001:00051770       ?SignInUser@CCryGameSpySBQR2SignIn@@UEAA?AW4ECryLobbyError@@IAEBU?$DynArray@USUserCredential@@HU?$SmallDynStorage@USUserCredential@@HUStandardAlloc@NAlloc@@@NArray@@@@PEAIP6AXIW42@IPEAX@Z3@Z 0000000039a52770 f   CryGameSpySBQR2SignIn.obj
 0001:000519e0       ?SignOutUser@CCryGameSpySBQR2SignIn@@UEAA?AW4ECryLobbyError@@IPEAIP6AXIW42@IPEAX@Z2@Z 0000000039a529e0 f   CryGameSpySBQR2SignIn.obj
 0001:00051b20       ?CreateUser@CCryGameSpySBQR2SignIn@@AEAA?AW4ECryLobbyError@@W4ETask@CCrySignIn@@IAEBU?$DynArray@USUserCredential@@HU?$SmallDynStorage@USUserCredential@@HUStandardAlloc@NAlloc@@@NArray@@@@PEAIP6AXIW42@IPEBDPEAX@Z5@Z 0000000039a52b20 f   CryGameSpySBQR2SignIn.obj
 0001:00051dc0       ?GetUserCredentials@CCryGameSpySBQR2SignIn@@UEAA?AW4ECryLobbyError@@IPEAIP6AXIW42@IPEAU?$DynArray@USUserCredential@@HU?$SmallDynStorage@USUserCredential@@HUStandardAlloc@NAlloc@@@NArray@@@@PEAX@Z3@Z 0000000039a52dc0 f   CryGameSpySBQR2SignIn.obj
 0001:00051f30       ?CreateUser@CCryGameSpySBQR2SignIn@@UEAA?AW4ECryLobbyError@@IAEBU?$DynArray@USUserCredential@@HU?$SmallDynStorage@USUserCredential@@HUStandardAlloc@NAlloc@@@NArray@@@@PEAIP6AXIW42@IPEBDPEAX@Z4@Z 0000000039a52f30 f   CryGameSpySBQR2SignIn.obj
 0001:00051f70       ?CreateAndSignInUser@CCryGameSpySBQR2SignIn@@UEAA?AW4ECryLobbyError@@IAEBU?$DynArray@USUserCredential@@HU?$SmallDynStorage@USUserCredential@@HUStandardAlloc@NAlloc@@@NArray@@@@PEAIP6AXIW42@IPEBDPEAX@Z4@Z 0000000039a52f70 f   CryGameSpySBQR2SignIn.obj
 0001:00051fb0       ?EndGetUserCredentials@CCryGameSpySBQR2SignIn@@AEAAXV?$CryLobbyID@USCrySignInTaskID@CCrySignIn@@$03@@@Z 0000000039a52fb0 f   CryGameSpySBQR2SignIn.obj
 0001:00052470       ?EndTask@CCryGameSpySBQR2SignIn@@MEAAXV?$CryLobbyID@USCrySignInTaskID@CCrySignIn@@$03@@@Z 0000000039a53470 f   CryGameSpySBQR2SignIn.obj
 0001:00052570       ?Initialise@CCryGameSpySBQR2Stats@@QEAA?AW4ECryLobbyError@@XZ 0000000039a53570 f   CryGameSpySBQR2Stats.obj
 0001:000525d0       ?FindFieldFromName@CCryGameSpySBQR2Stats@@AEAAPEAUSAKEField@@PEAU2@HPEBD@Z 0000000039a535d0 f   CryGameSpySBQR2Stats.obj
 0001:00052670       ?EndStatsReadLeaderBoard@CCryGameSpySBQR2Stats@@AEAAXI@Z 0000000039a53670 f   CryGameSpySBQR2Stats.obj
 0001:000526c0       ?PopulateUserDataWriteFields@CCryGameSpySBQR2Stats@@AEAAXIPEAUSCryGameSpyOneUserDataWrite@1@PEAH@Z 0000000039a536c0 f   CryGameSpySBQR2Stats.obj
 0001:00052790       ?EndStatsReadUserData@CCryGameSpySBQR2Stats@@AEAAXI@Z 0000000039a53790 f   CryGameSpySBQR2Stats.obj
 0001:000527f0       ?SetLeaderboardType@CCryGameSpySBQR2Stats@@UEAAXW4ECryLobbyLeaderboardType@@@Z 0000000039a537f0 f   CryGameSpySBQR2Stats.obj
 0001:00052800       ?GetLeaderboardType@CCryGameSpySBQR2Stats@@UEAA?AW4ECryLobbyLeaderboardType@@XZ 0000000039a53800 f   CryGameSpySBQR2Stats.obj
 0001:00052810       ?_AllocData@?$CryStackStringT@D$07@@QEAAX_K@Z 0000000039a53810 f i CryGameSpySBQR2Stats.obj
 0001:00052890       ?EndTask@CCryGameSpySBQR2Stats@@AEAAXI@Z 0000000039a53890 f   CryGameSpySBQR2Stats.obj
 0001:00052960       ?FindRegisteredBoardInfo@CCryGameSpySBQR2Stats@@AEAAPEAUSRegisterLeaderBoardData@1@IW4ECryLobbyLeaderboardType@@@Z 0000000039a53960 f   CryGameSpySBQR2Stats.obj
 0001:000529b0       ?FindRegisteredBoardInfo@CCryGameSpySBQR2Stats@@AEAAPEAUSRegisterLeaderBoardData@1@PEBD@Z 0000000039a539b0 f   CryGameSpySBQR2Stats.obj
 0001:00052a60       ?BuildStatsWriteArray@CCryGameSpySBQR2Stats@@AEAA?AW4ECryLobbyError@@IIIPEAPEAUSCryLobbyUserData@@PEAIPEAPEAUSCryGameSpyOneUserDataWrite@1@PEAPEAEI@Z 0000000039a53a60 f   CryGameSpySBQR2Stats.obj
 0001:00052e90       ?CreateTaskLink@CCryGameSpySBQR2Stats@@AEAA?AW4ECryLobbyError@@PEAUSTask@1@@Z 0000000039a53e90 f   CryGameSpySBQR2Stats.obj
 0001:00052f30       ?FreeTask@CCryGameSpySBQR2Stats@@EEAAXI@Z 0000000039a53f30 f   CryGameSpySBQR2Stats.obj
 0001:00052fd0       ?resize_raw@?$SmallDynStorage@USRegisterUserData@CCryGameSpySBQR2Stats@@HUStandardAlloc@NAlloc@@@NArray@@QEAAXHH_N@Z 0000000039a53fd0 f i CryGameSpySBQR2Stats.obj
 0001:00053160       ?_M_erase@?$_Rb_tree@HU?$less@H@stlpmtx_std@@U?$pair@$$CBHH@2@U?$_Select1st@U?$pair@$$CBHH@stlpmtx_std@@@priv@2@U?$_MapTraitsT@U?$pair@$$CBHH@stlpmtx_std@@@52@V?$allocator@U?$pair@$$CBHH@stlpmtx_std@@@2@@priv@stlpmtx_std@@AEAAXPEAU_Rb_tree_node_base@23@@Z 0000000039a54160 f i CryGameSpySBQR2Stats.obj
 0001:000531c0       ?StartTask@CCryGameSpySBQR2Stats@@AEAA?AW4ECryLobbyError@@W4ETask@1@_N1IPEAI2V?$CryLobbyID@USCryLobbySessionHandle@@$03@@PEAX4@Z 0000000039a541c0 f   CryGameSpySBQR2Stats.obj
 0001:000532b0       ?BuildLeaderBoardWriteArray@CCryGameSpySBQR2Stats@@AEAA?AW4ECryLobbyError@@IIIPEAPEAUSCryStatsLeaderBoardWrite@@PEAIIPEAPEAUSCryGameSpyOneLeaderBoardWrite@1@1@Z 0000000039a542b0 f   CryGameSpySBQR2Stats.obj
 0001:00053630       ?InitialiseLeaderBoardReadTask@CCryGameSpySBQR2Stats@@AEAA?AW4ECryLobbyError@@IAEAIPEAPEAUSRegisterLeaderBoardData@1@PEAPEAUSCryGameSpyStatsBoardReadInfo@1@IPEAIP6AXIW42@PEAUSCryStatsLeaderBoardReadResult@@PEAX@Z6@Z 0000000039a54630 f   CryGameSpySBQR2Stats.obj
 0001:00053990       ?set_size@?$SmallDynStorage@USRegisterLeaderBoardDataGroup@CCryGameSpySBQR2Stats@@HUStandardAlloc@NAlloc@@@NArray@@QEAAXH@Z 0000000039a54990 f i CryGameSpySBQR2Stats.obj
 0001:00053a50       ?set_size@?$SmallDynStorage@USRegisterUserData@CCryGameSpySBQR2Stats@@HUStandardAlloc@NAlloc@@@NArray@@QEAAXH@Z 0000000039a54a50 f i CryGameSpySBQR2Stats.obj
 0001:00053af0       ?_M_create_node@?$_Rb_tree@HU?$less@H@stlpmtx_std@@U?$pair@$$CBHH@2@U?$_Select1st@U?$pair@$$CBHH@stlpmtx_std@@@priv@2@U?$_MapTraitsT@U?$pair@$$CBHH@stlpmtx_std@@@52@V?$allocator@U?$pair@$$CBHH@stlpmtx_std@@@2@@priv@stlpmtx_std@@IEAAPEAU_Rb_tree_node_base@23@AEBU?$pair@$$CBHH@3@@Z 0000000039a54af0 f i CryGameSpySBQR2Stats.obj
 0001:00053b60       ?append_raw@?$DynArray@USRegisterUserData@CCryGameSpySBQR2Stats@@HU?$SmallDynStorage@USRegisterUserData@CCryGameSpySBQR2Stats@@HUStandardAlloc@NAlloc@@@NArray@@@@QEAA?AU?$Array@USRegisterUserData@CCryGameSpySBQR2Stats@@HU?$ArrayStorage@USRegisterUserData@CCryGameSpySBQR2Stats@@H@NArray@@@@H@Z 0000000039a54b60 f i CryGameSpySBQR2Stats.obj
 0001:00053c20       ?Format@?$CryStackStringT@D$07@@QEAAAEAV1@PEBDZZ 0000000039a54c20 f i CryGameSpySBQR2Stats.obj
 0001:00053d10       ?_M_insert@?$_Rb_tree@HU?$less@H@stlpmtx_std@@U?$pair@$$CBHH@2@U?$_Select1st@U?$pair@$$CBHH@stlpmtx_std@@@priv@2@U?$_MapTraitsT@U?$pair@$$CBHH@stlpmtx_std@@@52@V?$allocator@U?$pair@$$CBHH@stlpmtx_std@@@2@@priv@stlpmtx_std@@AEAA?AU?$_Rb_tree_iterator@U?$pair@$$CBHH@stlpmtx_std@@U?$_MapTraitsT@U?$pair@$$CBHH@stlpmtx_std@@@priv@2@@23@PEAU_Rb_tree_node_base@23@AEBU?$pair@$$CBHH@3@00@Z 0000000039a54d10 f i CryGameSpySBQR2Stats.obj
 0001:00053dd0       ?_M_copy@?$_Rb_tree@HU?$less@H@stlpmtx_std@@U?$pair@$$CBHH@2@U?$_Select1st@U?$pair@$$CBHH@stlpmtx_std@@@priv@2@U?$_MapTraitsT@U?$pair@$$CBHH@stlpmtx_std@@@52@V?$allocator@U?$pair@$$CBHH@stlpmtx_std@@@2@@priv@stlpmtx_std@@AEAAPEAU_Rb_tree_node_base@23@PEAU423@0@Z 0000000039a54dd0 f i CryGameSpySBQR2Stats.obj
 0001:00053f40       ?insert_unique@?$_Rb_tree@HU?$less@H@stlpmtx_std@@U?$pair@$$CBHH@2@U?$_Select1st@U?$pair@$$CBHH@stlpmtx_std@@@priv@2@U?$_MapTraitsT@U?$pair@$$CBHH@stlpmtx_std@@@52@V?$allocator@U?$pair@$$CBHH@stlpmtx_std@@@2@@priv@stlpmtx_std@@QEAA?AU?$pair@U?$_Rb_tree_iterator@U?$pair@$$CBHH@stlpmtx_std@@U?$_MapTraitsT@U?$pair@$$CBHH@stlpmtx_std@@@priv@2@@priv@stlpmtx_std@@_N@3@AEBU?$pair@$$CBHH@3@@Z 0000000039a54f40 f i CryGameSpySBQR2Stats.obj
 0001:00054140       ?insert_unique@?$_Rb_tree@HU?$less@H@stlpmtx_std@@U?$pair@$$CBHH@2@U?$_Select1st@U?$pair@$$CBHH@stlpmtx_std@@@priv@2@U?$_MapTraitsT@U?$pair@$$CBHH@stlpmtx_std@@@52@V?$allocator@U?$pair@$$CBHH@stlpmtx_std@@@2@@priv@stlpmtx_std@@QEAA?AU?$_Rb_tree_iterator@U?$pair@$$CBHH@stlpmtx_std@@U?$_MapTraitsT@U?$pair@$$CBHH@stlpmtx_std@@@priv@2@@23@U423@AEBU?$pair@$$CBHH@3@@Z 0000000039a55140 f i CryGameSpySBQR2Stats.obj
 0001:00054580       ??0?$_Rb_tree@HU?$less@H@stlpmtx_std@@U?$pair@$$CBHH@2@U?$_Select1st@U?$pair@$$CBHH@stlpmtx_std@@@priv@2@U?$_MapTraitsT@U?$pair@$$CBHH@stlpmtx_std@@@52@V?$allocator@U?$pair@$$CBHH@stlpmtx_std@@@2@@priv@stlpmtx_std@@QEAA@AEBV012@@Z 0000000039a55580 f i CryGameSpySBQR2Stats.obj
 0001:00054640       ?Terminate@CCryGameSpySBQR2Stats@@QEAA?AW4ECryLobbyError@@XZ 0000000039a55640 f   CryGameSpySBQR2Stats.obj
 0001:00054740       ??1SRegisterLeaderBoardDataGroup@CCryGameSpySBQR2Stats@@QEAA@XZ 0000000039a55740 f i CryGameSpySBQR2Stats.obj
 0001:00054880       ?init@?$DynArray@USRegisterLeaderBoardDataGroup@CCryGameSpySBQR2Stats@@HU?$SmallDynStorage@USRegisterLeaderBoardDataGroup@CCryGameSpySBQR2Stats@@HUStandardAlloc@NAlloc@@@NArray@@@@KAPEAUSRegisterLeaderBoardDataGroup@CCryGameSpySBQR2Stats@@U?$Array@USRegisterLeaderBoardDataGroup@CCryGameSpySBQR2Stats@@HU?$ArrayStorage@USRegisterLeaderBoardDataGroup@CCryGameSpySBQR2Stats@@H@NArray@@@@@Z 0000000039a55880 f i CryGameSpySBQR2Stats.obj
 0001:00054a00       ??$?AH@?$map@HHU?$less@H@stlpmtx_std@@V?$allocator@U?$pair@$$CBHH@stlpmtx_std@@@2@@stlpmtx_std@@QEAAAEAHAEBH@Z 0000000039a55a00 f i CryGameSpySBQR2Stats.obj
 0001:00054a80       ?ReadUserDataCallback@CCryGameSpySBQR2Stats@@CAXPEAUSAKEField@@PEAV1@PEAUSTask@1@PEAUSCryGameSpyStatsUserReadInfo@1@0IPEAUSCryLobbyUserData@@@Z 0000000039a55a80 f   CryGameSpySBQR2Stats.obj
 0001:00054c20       ??0SRegisterLeaderBoardDataGroup@CCryGameSpySBQR2Stats@@QEAA@AEBU01@@Z 0000000039a55c20 f i CryGameSpySBQR2Stats.obj
 0001:00054d50       ?StopTaskRunning@CCryGameSpySBQR2Stats@@AEAAXI@Z 0000000039a55d50 f   CryGameSpySBQR2Stats.obj
 0001:00054dc0       ?GetRecordCountCallback@CCryGameSpySBQR2Stats@@CAXPEAVCGameSpySBQR2Sake@@USResult@2@PEAUSAKEGetRecordCountInput@@PEAUSAKEGetRecordCountOutput@@PEAUIGameSpyLink@@@Z 0000000039a55dc0 f   CryGameSpySBQR2Stats.obj
 0001:00054eb0       ?SearchForRecordsCallback@CCryGameSpySBQR2Stats@@CAXPEAVCGameSpySBQR2Sake@@USResult@2@PEAUSAKESearchForRecordsInput@@PEAUSAKESearchForRecordsOutput@@PEAUIGameSpyLink@@@Z 0000000039a55eb0 f   CryGameSpySBQR2Stats.obj
 0001:00055540       ?ReadUserDataGetMyRecordsCallback@CCryGameSpySBQR2Stats@@CAXPEAVCGameSpySBQR2Sake@@USResult@2@PEAUSAKEGetMyRecordsInput@@PEAUSAKEGetMyRecordsOutput@@PEAUIGameSpyLink@@@Z 0000000039a56540 f   CryGameSpySBQR2Stats.obj
 0001:00055540       ?ReadUserDataSearchForRecordsCallback@CCryGameSpySBQR2Stats@@CAXPEAVCGameSpySBQR2Sake@@USResult@2@PEAUSAKESearchForRecordsInput@@PEAUSAKESearchForRecordsOutput@@PEAUIGameSpyLink@@@Z 0000000039a56540 f   CryGameSpySBQR2Stats.obj
 0001:000556f0       ?StartStatsReadLeaderBoard@CCryGameSpySBQR2Stats@@AEAAXI@Z 0000000039a566f0 f   CryGameSpySBQR2Stats.obj
 0001:00055840       ?StartNextStatsWrite@CCryGameSpySBQR2Stats@@AEAAXIPEAUSTask@1@PEAUSCryGameSpyStatsUserDataWriteInfo@1@@Z 0000000039a56840 f   CryGameSpySBQR2Stats.obj
 0001:000558c0       ?LeaderBoardUpdateCallback@CCryGameSpySBQR2Stats@@CAXPEAVCGameSpySBQR2Sake@@USResult@2@PEAUSAKEUpdateRecordInput@@PEAUIGameSpyLink@@@Z 0000000039a568c0 f   CryGameSpySBQR2Stats.obj
 0001:000559e0       ?UpdateLeaderBoardRecord@CCryGameSpySBQR2Stats@@AEAAXPEAUSTask@1@PEAUSCryGameSpyStatsBoardWriteInfo@1@@Z 0000000039a569e0 f   CryGameSpySBQR2Stats.obj
 0001:00055a90       ?StartStatsReadUserData@CCryGameSpySBQR2Stats@@AEAAXI@Z 0000000039a56a90 f   CryGameSpySBQR2Stats.obj
 0001:00055c80       ?pop_back@?$DynArray@USRegisterLeaderBoardDataGroup@CCryGameSpySBQR2Stats@@HU?$SmallDynStorage@USRegisterLeaderBoardDataGroup@CCryGameSpySBQR2Stats@@HUStandardAlloc@NAlloc@@@NArray@@@@QEAAXH@Z 0000000039a56c80 f i CryGameSpySBQR2Stats.obj
 0001:00055d10       ?StartTaskRunning@CCryGameSpySBQR2Stats@@AEAAXI@Z 0000000039a56d10 f   CryGameSpySBQR2Stats.obj
 0001:00055dc0       ?StatsWriteLeaderBoards@CCryGameSpySBQR2Stats@@AEAA?AW4ECryLobbyError@@IPEAPEAUSCryStatsLeaderBoardWrite@@PEAII@Z 0000000039a56dc0 f   CryGameSpySBQR2Stats.obj
 0001:00055f10       ?StatsReadLeaderBoardByUserID@CCryGameSpySBQR2Stats@@UEAA?AW4ECryLobbyError@@IPEAUCryUserID@@IPEAIP6AXIW42@PEAUSCryStatsLeaderBoardReadResult@@PEAX@Z4@Z 0000000039a56f10 f   CryGameSpySBQR2Stats.obj
 0001:00056160       ?StatsReadLeaderBoardByRankForRange@CCryGameSpySBQR2Stats@@UEAA?AW4ECryLobbyError@@IIIPEAIP6AXIW42@PEAUSCryStatsLeaderBoardReadResult@@PEAX@Z3@Z 0000000039a57160 f   CryGameSpySBQR2Stats.obj
 0001:00056280       ?StatsReadLeaderBoardByRankForUser@CCryGameSpySBQR2Stats@@UEAA?AW4ECryLobbyError@@IIIPEAIP6AXIW42@PEAUSCryStatsLeaderBoardReadResult@@PEAX@Z3@Z 0000000039a57280 f   CryGameSpySBQR2Stats.obj
 0001:000563b0       ?StatsRegisterUserData@CCryGameSpySBQR2Stats@@UEAA?AW4ECryLobbyError@@PEAUSCryLobbyUserData@@IPEAIP6AXIW42@PEAX@Z3@Z 0000000039a573b0 f   CryGameSpySBQR2Stats.obj
 0001:00056850       ?StatsWriteUserData@CCryGameSpySBQR2Stats@@AEAA?AW4ECryLobbyError@@IPEAPEAUSCryLobbyUserData@@PEAII@Z 0000000039a57850 f   CryGameSpySBQR2Stats.obj
 0001:000569c0       ?StatsCreateCallback@CCryGameSpySBQR2Stats@@CAXPEAVCGameSpySBQR2Sake@@USResult@2@PEAUSAKECreateRecordInput@@PEAUSAKECreateRecordOutput@@PEAUIGameSpyLink@@@Z 0000000039a579c0 f   CryGameSpySBQR2Stats.obj
 0001:00056ae0       ?StatsUpdateCallback@CCryGameSpySBQR2Stats@@CAXPEAVCGameSpySBQR2Sake@@USResult@2@PEAUSAKEUpdateRecordInput@@PEAUIGameSpyLink@@@Z 0000000039a57ae0 f   CryGameSpySBQR2Stats.obj
 0001:00056ba0       ?StatsWriteLeaderBoardGetCallback@CCryGameSpySBQR2Stats@@CAXPEAV1@PEAUSTask@1@PEAUSAKEField@@I@Z 0000000039a57ba0 f   CryGameSpySBQR2Stats.obj
 0001:00056c90       ?UpdateStatsRecord@CCryGameSpySBQR2Stats@@AEAAXIPEAUSCryGameSpyOneUserDataWrite@1@@Z 0000000039a57c90 f   CryGameSpySBQR2Stats.obj
 0001:00056d80       ?CreateStatsRecord@CCryGameSpySBQR2Stats@@AEAAXIPEAUSCryGameSpyOneUserDataWrite@1@@Z 0000000039a57d80 f   CryGameSpySBQR2Stats.obj
 0001:00056e10       ?StatsReadUserData@CCryGameSpySBQR2Stats@@AEAA?AW4ECryLobbyError@@IPEAUSUser@1@PEAIP6AXIW42@PEAUSCryLobbyUserData@@IPEAX@Z4@Z 0000000039a57e10 f   CryGameSpySBQR2Stats.obj
 0001:00057100       ??1?$DynArray@USRegisterLeaderBoardDataGroup@CCryGameSpySBQR2Stats@@HU?$SmallDynStorage@USRegisterLeaderBoardDataGroup@CCryGameSpySBQR2Stats@@HUStandardAlloc@NAlloc@@@NArray@@@@QEAA@XZ 0000000039a58100 f i CryGameSpySBQR2Stats.obj
 0001:00057180       ??$move_init@USRegisterLeaderBoardDataGroup@CCryGameSpySBQR2Stats@@@NArray@@YAXPEAUSRegisterLeaderBoardDataGroup@CCryGameSpySBQR2Stats@@0_K@Z 0000000039a58180 f i CryGameSpySBQR2Stats.obj
 0001:000571f0       ??0CCryGameSpySBQR2Stats@@QEAA@PEAVCCryLobby@@PEAVCCryLobbyService@@@Z 0000000039a581f0 f   CryGameSpySBQR2Stats.obj
 0001:00057480       ??_ECCryGameSpySBQR2Stats@@WBA@EAAPEAXI@Z 0000000039a58480 f i CryGameSpySBQR2Stats.obj
 0001:00057490       ??1CCryGameSpySBQR2Stats@@UEAA@XZ 0000000039a58490 f i CryGameSpySBQR2Stats.obj
 0001:000576b0       ?StatsWriteLeaderBoards@CCryGameSpySBQR2Stats@@UEAA?AW4ECryLobbyError@@IIPEAUSCryStatsLeaderBoardWrite@@IPEAIP6AXIW42@PEAX@Z3@Z 0000000039a586b0 f   CryGameSpySBQR2Stats.obj
 0001:000577e0       ?StatsWriteLeaderBoards@CCryGameSpySBQR2Stats@@UEAA?AW4ECryLobbyError@@IPEAUCryUserID@@PEAPEAUSCryStatsLeaderBoardWrite@@PEAII2P6AXIW42@PEAX@Z4@Z 0000000039a587e0 f   CryGameSpySBQR2Stats.obj
 0001:000579d0       ?StatsWriteUserData@CCryGameSpySBQR2Stats@@UEAA?AW4ECryLobbyError@@IPEAUSCryLobbyUserData@@IPEAIP6AXIW42@PEAX@Z3@Z 0000000039a589d0 f   CryGameSpySBQR2Stats.obj
 0001:00057b60       ?StatsWriteUserData@CCryGameSpySBQR2Stats@@UEAA?AW4ECryLobbyError@@PEAUCryUserID@@PEAPEAUSCryLobbyUserData@@PEAII2P6AXIW42@PEAX@Z4@Z 0000000039a58b60 f   CryGameSpySBQR2Stats.obj
 0001:00057d60       ?StatsWriteUserDataGetCallback@CCryGameSpySBQR2Stats@@CAXPEAV1@PEAUSTask@1@PEAUSAKEField@@I@Z 0000000039a58d60 f   CryGameSpySBQR2Stats.obj
 0001:00057e70       ?StatsWriteLeaderBoardSearchForRecordsCallback@CCryGameSpySBQR2Stats@@CAXPEAVCGameSpySBQR2Sake@@USResult@2@PEAUSAKESearchForRecordsInput@@PEAUSAKESearchForRecordsOutput@@PEAUIGameSpyLink@@@Z 0000000039a58e70 f   CryGameSpySBQR2Stats.obj
 0001:00057e70       ?StatsWriteLeaderBoardGetMyRecordsCallback@CCryGameSpySBQR2Stats@@CAXPEAVCGameSpySBQR2Sake@@USResult@2@PEAUSAKEGetMyRecordsInput@@PEAUSAKEGetMyRecordsOutput@@PEAUIGameSpyLink@@@Z 0000000039a58e70 f   CryGameSpySBQR2Stats.obj
 0001:00057f40       ?FindLeaderBoardRecord@CCryGameSpySBQR2Stats@@AEAAXIPEAUSCryGameSpyStatsBoardWriteInfo@1@@Z 0000000039a58f40 f   CryGameSpySBQR2Stats.obj
 0001:000580a0       ?StatsReadUserData@CCryGameSpySBQR2Stats@@UEAA?AW4ECryLobbyError@@IPEAIP6AXIW42@PEAUSCryLobbyUserData@@IPEAX@Z3@Z 0000000039a590a0 f   CryGameSpySBQR2Stats.obj
 0001:000580e0       ?StatsReadUserData@CCryGameSpySBQR2Stats@@UEAA?AW4ECryLobbyError@@IUCryUserID@@PEAIP6AXIW42@PEAUSCryLobbyUserData@@IPEAX@Z4@Z 0000000039a590e0 f   CryGameSpySBQR2Stats.obj
 0001:00058180       ?resize_raw@?$SmallDynStorage@USRegisterLeaderBoardDataGroup@CCryGameSpySBQR2Stats@@HUStandardAlloc@NAlloc@@@NArray@@QEAAXHH_N@Z 0000000039a59180 f i CryGameSpySBQR2Stats.obj
 0001:00058310       ??_GCCryGameSpySBQR2Stats@@UEAAPEAXI@Z 0000000039a59310 f i CryGameSpySBQR2Stats.obj
 0001:00058310       ??_ECCryGameSpySBQR2Stats@@UEAAPEAXI@Z 0000000039a59310 f i CryGameSpySBQR2Stats.obj
 0001:00058340       ?QueueNextLeaderBoardSake@CCryGameSpySBQR2Stats@@AEAAXIPEAUSCryGameSpyStatsBoardWriteInfo@1@@Z 0000000039a59340 f   CryGameSpySBQR2Stats.obj
 0001:00058460       ?GetInfoCallback@CCryGameSpySBQR2Stats@@CAXPEAVCGameSpySBQR2GPConnection@@USResult@2@PEAUGPGetInfoResponseArg@@PEAUIGameSpyLink@@@Z 0000000039a59460 f   CryGameSpySBQR2Stats.obj
 0001:00058590       ?StatsWriteUserDataGetMyRecordsCallback@CCryGameSpySBQR2Stats@@CAXPEAVCGameSpySBQR2Sake@@USResult@2@PEAUSAKEGetMyRecordsInput@@PEAUSAKEGetMyRecordsOutput@@PEAUIGameSpyLink@@@Z 0000000039a59590 f   CryGameSpySBQR2Stats.obj
 0001:00058590       ?StatsWriteUserDataSearchForRecordsCallback@CCryGameSpySBQR2Stats@@CAXPEAVCGameSpySBQR2Sake@@USResult@2@PEAUSAKESearchForRecordsInput@@PEAUSAKESearchForRecordsOutput@@PEAUIGameSpyLink@@@Z 0000000039a59590 f   CryGameSpySBQR2Stats.obj
 0001:00058660       ?FindOwnStatsRecord@CCryGameSpySBQR2Stats@@AEAAXPEAUSTask@1@PEAUSCryGameSpyOneUserDataWrite@1@@Z 0000000039a59660 f   CryGameSpySBQR2Stats.obj
 0001:000586e0       ?FindOthersStatsRecord@CCryGameSpySBQR2Stats@@AEAAXPEAUSTask@1@PEAUSCryGameSpyOneUserDataWrite@1@@Z 0000000039a596e0 f   CryGameSpySBQR2Stats.obj
 0001:000587e0       ?StartCurrentStatsWrite@CCryGameSpySBQR2Stats@@AEAAXIPEAUSTask@1@@Z 0000000039a597e0 f   CryGameSpySBQR2Stats.obj
 0001:00058a00       ?expand_raw@?$DynArray@USRegisterLeaderBoardDataGroup@CCryGameSpySBQR2Stats@@HU?$SmallDynStorage@USRegisterLeaderBoardDataGroup@CCryGameSpySBQR2Stats@@HUStandardAlloc@NAlloc@@@NArray@@@@IEAAPEAUSRegisterLeaderBoardDataGroup@CCryGameSpySBQR2Stats@@PEAU23@H@Z 0000000039a59a00 f i CryGameSpySBQR2Stats.obj
 0001:00058ac0       ?QueueNextLeaderBoard@CCryGameSpySBQR2Stats@@AEAA_NIPEAUSCryGameSpyStatsBoardWriteInfo@1@@Z 0000000039a59ac0 f   CryGameSpySBQR2Stats.obj
 0001:00058c60       ?StartStatsWriteLeaderBoard@CCryGameSpySBQR2Stats@@AEAAXI@Z 0000000039a59c60 f   CryGameSpySBQR2Stats.obj
 0001:00058d70       ?LeaderBoardCreateCallback@CCryGameSpySBQR2Stats@@CAXPEAVCGameSpySBQR2Sake@@USResult@2@PEAUSAKECreateRecordInput@@PEAUSAKECreateRecordOutput@@PEAUIGameSpyLink@@@Z 0000000039a59d70 f   CryGameSpySBQR2Stats.obj
 0001:00058eb0       ?Tick@CCryGameSpySBQR2Stats@@QEAAXVCTimeValue@@@Z 0000000039a59eb0 f   CryGameSpySBQR2Stats.obj
 0001:00058fb0       ?StatsRegisterLeaderBoards@CCryGameSpySBQR2Stats@@UEAA?AW4ECryLobbyError@@PEAUSCryStatsLeaderBoardWrite@@IPEAIP6AXIW42@PEAX@Z3@Z 0000000039a59fb0 f   CryGameSpySBQR2Stats.obj
 0001:00059470       ?IsSpeaking@CCryGameSpySBQR2Voice@@UEAA_NI@Z 0000000039a5a470 f   CryGameSpySBQR2Voice.obj
 0001:000594a0       ?VOIPPushToTalkChanged@CCryGameSpySBQR2Voice@@KAXPEAUICVar@@@Z 0000000039a5a4a0 f   CryGameSpySBQR2Voice.obj
 0001:00059510       ?VOIPPlaybackVolumeChanged@CCryGameSpySBQR2Voice@@KAXPEAUICVar@@@Z 0000000039a5a510 f   CryGameSpySBQR2Voice.obj
 0001:00059560       ?EnablePushToTalk@CCryGameSpySBQR2Voice@@UEAAXI_N@Z 0000000039a5a560 f   CryGameSpySBQR2Voice.obj
 0001:00059570       ?IsPushToTalkEnabled@CCryGameSpySBQR2Voice@@UEAA_NI@Z 0000000039a5a570 f   CryGameSpySBQR2Voice.obj
 0001:00059580       ?PushToTalkButtonDown@CCryGameSpySBQR2Voice@@UEAAXI@Z 0000000039a5a580 f   CryGameSpySBQR2Voice.obj
 0001:00059590       ?PushToTalkButtonUp@CCryGameSpySBQR2Voice@@UEAAXI@Z 0000000039a5a590 f   CryGameSpySBQR2Voice.obj
 0001:000595a0       ?SetVoicePlaybackVolume@CCryGameSpySBQR2Voice@@UEAAXIM@Z 0000000039a5a5a0 f   CryGameSpySBQR2Voice.obj
 0001:000595f0       ?GetVoicePlaybackVolume@CCryGameSpySBQR2Voice@@UEAAMI@Z 0000000039a5a5f0 f   CryGameSpySBQR2Voice.obj
 0001:00059600       ?Terminate@CCryGameSpySBQR2Voice@@QEAA?AW4ECryLobbyError@@XZ 0000000039a5a600 f   CryGameSpySBQR2Voice.obj
 0001:000596c0       ?UnRegisterRemoteUser@CCryGameSpySBQR2Voice@@QEAAXV?$CryLobbyID@USCryLobbyConnectionID@@$0EA@@@@Z 0000000039a5a6c0 f   CryGameSpySBQR2Voice.obj
 0001:00059730       ?CreateDevice@CCryGameSpySBQR2Voice@@IEAA_NAEAPEAUGVIDevice@@HI@Z 0000000039a5a730 f   CryGameSpySBQR2Voice.obj
 0001:00059810       ?CaptureVoiceData@CCryGameSpySBQR2Voice@@IEAAIXZ 0000000039a5a810 f   CryGameSpySBQR2Voice.obj
 0001:00059920       ?ProcessMicrophoneNotification@CCryGameSpySBQR2Voice@@IEAAXAEBV?$CConfigurableVariant@V?$CNode@USNullAddr@@V?$CNode@GV?$CNode@USIPv4Addr@@V?$CNode@ULobbyIdAddr@@VCEnd@NTypelist@@@NTypelist@@@NTypelist@@@NTypelist@@@NTypelist@@$07VCDefaultVariantConversion@NConfigurableVariantHelpers@@VCDefaultVariantConstruction@4@@@PEAVCCryLobbyPacket@@@Z 0000000039a5a920 f   CryGameSpySBQR2Voice.obj
 0001:00059a20       ?ProcessMicrophoneRequest@CCryGameSpySBQR2Voice@@IEAAXAEBV?$CConfigurableVariant@V?$CNode@USNullAddr@@V?$CNode@GV?$CNode@USIPv4Addr@@V?$CNode@ULobbyIdAddr@@VCEnd@NTypelist@@@NTypelist@@@NTypelist@@@NTypelist@@@NTypelist@@$07VCDefaultVariantConversion@NConfigurableVariantHelpers@@VCDefaultVariantConstruction@4@@@PEAVCCryLobbyPacket@@@Z 0000000039a5aa20 f   CryGameSpySBQR2Voice.obj
 0001:00059ab0       ?InitDevices@CCryGameSpySBQR2Voice@@IEAA?AW4ECryLobbyError@@XZ 0000000039a5aab0 f   CryGameSpySBQR2Voice.obj
 0001:00059c70       ?ProcessVoiceData@CCryGameSpySBQR2Voice@@IEAAXAEBV?$CConfigurableVariant@V?$CNode@USNullAddr@@V?$CNode@GV?$CNode@USIPv4Addr@@V?$CNode@ULobbyIdAddr@@VCEnd@NTypelist@@@NTypelist@@@NTypelist@@@NTypelist@@@NTypelist@@$07VCDefaultVariantConversion@NConfigurableVariantHelpers@@VCDefaultVariantConstruction@4@@@PEAVCCrySharedLobbyPacket@@@Z 0000000039a5ac70 f   CryGameSpySBQR2Voice.obj
 0001:00059ea0       ?VOIPEnabledChanged@CCryGameSpySBQR2Voice@@KAXPEAUICVar@@@Z 0000000039a5aea0 f   CryGameSpySBQR2Voice.obj
 0001:00059f00       ?Initialise@CCryGameSpySBQR2Voice@@QEAA?AW4ECryLobbyError@@XZ 0000000039a5af00 f   CryGameSpySBQR2Voice.obj
 0001:0005a050       ?OnPacket@CCryGameSpySBQR2Voice@@QEAAXAEBV?$CConfigurableVariant@V?$CNode@USNullAddr@@V?$CNode@GV?$CNode@USIPv4Addr@@V?$CNode@ULobbyIdAddr@@VCEnd@NTypelist@@@NTypelist@@@NTypelist@@@NTypelist@@@NTypelist@@$07VCDefaultVariantConversion@NConfigurableVariantHelpers@@VCDefaultVariantConstruction@4@@@PEAVCCryLobbyPacket@@@Z 0000000039a5b050 f   CryGameSpySBQR2Voice.obj
 0001:0005a0a0       ?RegisterRemoteUser@CCryGameSpySBQR2Voice@@QEAAIV?$CryLobbyID@USCryLobbyConnectionID@@$0EA@@@UCryUserID@@@Z 0000000039a5b0a0 f   CryGameSpySBQR2Voice.obj
 0001:0005a140       ?LateSetUserLobbyConnection@CCryGameSpySBQR2Voice@@QEAAXV?$CryLobbyID@USCryLobbyConnectionID@@$0EA@@@UCryUserID@@@Z 0000000039a5b140 f   CryGameSpySBQR2Voice.obj
 0001:0005a1f0       ?IsMicrophoneConnected@CCryGameSpySBQR2Voice@@UEAA_NUCryUserID@@@Z 0000000039a5b1f0 f   CryGameSpySBQR2Voice.obj
 0001:0005a3b0       ??0CCryGameSpySBQR2Voice@@QEAA@PEAVCCryLobby@@PEAVCCryLobbyService@@@Z 0000000039a5b3b0 f   CryGameSpySBQR2Voice.obj
 0001:0005a560       ??_ECCryGameSpySBQR2Voice@@WBA@EAAPEAXI@Z 0000000039a5b560 f i CryGameSpySBQR2Voice.obj
 0001:0005a570       ??1CCryGameSpySBQR2Voice@@UEAA@XZ 0000000039a5b570 f i CryGameSpySBQR2Voice.obj
 0001:0005a600       ??_ECCryGameSpySBQR2Voice@@UEAAPEAXI@Z 0000000039a5b600 f i CryGameSpySBQR2Voice.obj
 0001:0005a600       ??_GCCryGameSpySBQR2Voice@@UEAAPEAXI@Z 0000000039a5b600 f i CryGameSpySBQR2Voice.obj
 0001:0005a630       ?SendVoiceData@CCryGameSpySBQR2Voice@@IEAAXXZ 0000000039a5b630 f   CryGameSpySBQR2Voice.obj
 0001:0005a880       ?SendMicrophoneNotification@CCryGameSpySBQR2Voice@@MEAAXI@Z 0000000039a5b880 f   CryGameSpySBQR2Voice.obj
 0001:0005a990       ?SendMicrophoneRequest@CCryGameSpySBQR2Voice@@MEAAXI@Z 0000000039a5b990 f   CryGameSpySBQR2Voice.obj
 0001:0005aa80       ?Tick@CCryGameSpySBQR2Voice@@QEAAXVCTimeValue@@@Z 0000000039a5ba80 f   CryGameSpySBQR2Voice.obj
 0001:0005abb0       ?NeedThink@CGameSpySBQR2GPConnection@@MEBA_NXZ 0000000039a5bbb0 f   GameSpySBQR2GPConnection.obj
 0001:0005abd0       ?GetUserIndex@CGameSpySBQR2GPConnection@@QEAAIXZ 0000000039a5bbd0 f   GameSpySBQR2GPConnection.obj
 0001:0005abe0       ?Disconnect@CGameSpySBQR2GPConnection@@QEAAXXZ 0000000039a5bbe0 f   GameSpySBQR2GPConnection.obj
 0001:0005abf0       ?IsBlocked@CGameSpySBQR2GPConnection@@QEAA_NH@Z 0000000039a5bbf0 f   GameSpySBQR2GPConnection.obj
 0001:0005ac10       ?IsBuddy@CGameSpySBQR2GPConnection@@QEAA_NH@Z 0000000039a5bc10 f   GameSpySBQR2GPConnection.obj
 0001:0005ac30       ?SetStatus@CGameSpySBQR2GPConnection@@QEAAXW4GPEnum@@@Z 0000000039a5bc30 f   GameSpySBQR2GPConnection.obj
 0001:0005ac50       ?IsConnected@CGameSpySBQR2GPConnection@@QEAA_NXZ 0000000039a5bc50 f   GameSpySBQR2GPConnection.obj
 0001:0005ac80       ??$SynthesizeTaskFailure@UGPNewProfileResponseArg@@@CGameSpySBQR2GPConnection@@AEAAXW4GPResult@@P6AXPEAV0@USResult@0@PEAUGPNewProfileResponseArg@@PEAUIGameSpyLink@@@Z4@Z 0000000039a5bc80 f i GameSpySBQR2GPConnection.obj
 0001:0005ac80       ??$SynthesizeTaskFailure@UGPProfileSearchResponseArg@@@CGameSpySBQR2GPConnection@@AEAAXW4GPResult@@P6AXPEAV0@USResult@0@PEAUGPProfileSearchResponseArg@@PEAUIGameSpyLink@@@Z4@Z 0000000039a5bc80 f i GameSpySBQR2GPConnection.obj
 0001:0005ac80       ??$SynthesizeTaskFailure@UGPCheckResponseArg@@@CGameSpySBQR2GPConnection@@AEAAXW4GPResult@@P6AXPEAV0@USResult@0@PEAUGPCheckResponseArg@@PEAUIGameSpyLink@@@Z4@Z 0000000039a5bc80 f i GameSpySBQR2GPConnection.obj
 0001:0005ac80       ??$SynthesizeTaskFailure@UGPNewUserResponseArg@@@CGameSpySBQR2GPConnection@@AEAAXW4GPResult@@P6AXPEAV0@USResult@0@PEAUGPNewUserResponseArg@@PEAUIGameSpyLink@@@Z4@Z 0000000039a5bc80 f i GameSpySBQR2GPConnection.obj
 0001:0005ac80       ??$SynthesizeTaskFailure@UGPConnectResponseArg@@@CGameSpySBQR2GPConnection@@AEAAXW4GPResult@@P6AXPEAV0@USResult@0@PEAUGPConnectResponseArg@@PEAUIGameSpyLink@@@Z4@Z 0000000039a5bc80 f i GameSpySBQR2GPConnection.obj
 0001:0005ac80       ??$SynthesizeTaskFailure@UGPGetReverseBuddiesResponseArg@@@CGameSpySBQR2GPConnection@@AEAAXW4GPResult@@P6AXPEAV0@USResult@0@PEAUGPGetReverseBuddiesResponseArg@@PEAUIGameSpyLink@@@Z4@Z 0000000039a5bc80 f i GameSpySBQR2GPConnection.obj
 0001:0005ac80       ??$SynthesizeTaskFailure@UGPRegisterUniqueNickResponseArg@@@CGameSpySBQR2GPConnection@@AEAAXW4GPResult@@P6AXPEAV0@USResult@0@PEAUGPRegisterUniqueNickResponseArg@@PEAUIGameSpyLink@@@Z4@Z 0000000039a5bc80 f i GameSpySBQR2GPConnection.obj
 0001:0005ac80       ??$SynthesizeTaskFailure@UGPGetInfoResponseArg@@@CGameSpySBQR2GPConnection@@AEAAXW4GPResult@@P6AXPEAV0@USResult@0@PEAUGPGetInfoResponseArg@@PEAUIGameSpyLink@@@Z4@Z 0000000039a5bc80 f i GameSpySBQR2GPConnection.obj
 0001:0005acf0       ?GetImmediateResult@CGameSpySBQR2GPConnection@@AEAA?AUSResult@1@W4GPResult@@@Z 0000000039a5bcf0 f   GameSpySBQR2GPConnection.obj
 0001:0005adf0       ?_AllocData@?$CryStackStringT@D$0DD@@@QEAAX_K@Z 0000000039a5bdf0 f i GameSpySBQR2GPConnection.obj
 0001:0005ae70       ??$TaskFinished@UGPRecvBuddyStatusArg@@@CGameSpySBQR2GPConnection@@CAXPEAPEAXPEAX1@Z 0000000039a5be70 f i GameSpySBQR2GPConnection.obj
 0001:0005ae70       ??$TaskFinished@UGPConnectResponseArg@@@CGameSpySBQR2GPConnection@@CAXPEAPEAXPEAX1@Z 0000000039a5be70 f i GameSpySBQR2GPConnection.obj
 0001:0005ae70       ??$TaskFinished@UGPErrorArg@@@CGameSpySBQR2GPConnection@@CAXPEAPEAXPEAX1@Z 0000000039a5be70 f i GameSpySBQR2GPConnection.obj
 0001:0005ae70       ??$TaskFinished@UGPNewProfileResponseArg@@@CGameSpySBQR2GPConnection@@CAXPEAPEAXPEAX1@Z 0000000039a5be70 f i GameSpySBQR2GPConnection.obj
 0001:0005ae70       ??$TaskFinished@UGPCheckResponseArg@@@CGameSpySBQR2GPConnection@@CAXPEAPEAXPEAX1@Z 0000000039a5be70 f i GameSpySBQR2GPConnection.obj
 0001:0005ae70       ??$TaskFinished@UGPRecvBuddyMessageArg@@@CGameSpySBQR2GPConnection@@CAXPEAPEAXPEAX1@Z 0000000039a5be70 f i GameSpySBQR2GPConnection.obj
 0001:0005ae70       ??$TaskFinished@UGPRecvGameInviteArg@@@CGameSpySBQR2GPConnection@@CAXPEAPEAXPEAX1@Z 0000000039a5be70 f i GameSpySBQR2GPConnection.obj
 0001:0005ae70       ??$TaskFinished@UGPNewUserResponseArg@@@CGameSpySBQR2GPConnection@@CAXPEAPEAXPEAX1@Z 0000000039a5be70 f i GameSpySBQR2GPConnection.obj
 0001:0005ae70       ??$TaskFinished@UGPRecvBuddyRequestArg@@@CGameSpySBQR2GPConnection@@CAXPEAPEAXPEAX1@Z 0000000039a5be70 f i GameSpySBQR2GPConnection.obj
 0001:0005ae70       ??$TaskFinished@UGPRegisterUniqueNickResponseArg@@@CGameSpySBQR2GPConnection@@CAXPEAPEAXPEAX1@Z 0000000039a5be70 f i GameSpySBQR2GPConnection.obj
 0001:0005ae70       ??$TaskFinished@UGPGetInfoResponseArg@@@CGameSpySBQR2GPConnection@@CAXPEAPEAXPEAX1@Z 0000000039a5be70 f i GameSpySBQR2GPConnection.obj
 0001:0005ae70       ??$TaskFinished@UGPRecvBuddyAuthArg@@@CGameSpySBQR2GPConnection@@CAXPEAPEAXPEAX1@Z 0000000039a5be70 f i GameSpySBQR2GPConnection.obj
 0001:0005ae70       ??$TaskFinished@UGPGetReverseBuddiesResponseArg@@@CGameSpySBQR2GPConnection@@CAXPEAPEAXPEAX1@Z 0000000039a5be70 f i GameSpySBQR2GPConnection.obj
 0001:0005ae70       ??$TaskFinished@UGPRecvBuddyRevokeArg@@@CGameSpySBQR2GPConnection@@CAXPEAPEAXPEAX1@Z 0000000039a5be70 f i GameSpySBQR2GPConnection.obj
 0001:0005af60       ?AddToBlockedList@CGameSpySBQR2GPConnection@@QEAA?AUSResult@1@H@Z 0000000039a5bf60 f   GameSpySBQR2GPConnection.obj
 0001:0005afa0       ?AuthBuddyRequest@CGameSpySBQR2GPConnection@@QEAA?AUSResult@1@H@Z 0000000039a5bfa0 f   GameSpySBQR2GPConnection.obj
 0001:0005afe0       ?DeleteBuddy@CGameSpySBQR2GPConnection@@QEAA?AUSResult@1@H@Z 0000000039a5bfe0 f   GameSpySBQR2GPConnection.obj
 0001:0005b020       ?DenyBuddyRequest@CGameSpySBQR2GPConnection@@QEAA?AUSResult@1@H@Z 0000000039a5c020 f   GameSpySBQR2GPConnection.obj
 0001:0005b060       ?GetBuddyIndex@CGameSpySBQR2GPConnection@@QEAA?AUSResult@1@HPEAH@Z 0000000039a5c060 f   GameSpySBQR2GPConnection.obj
 0001:0005b0a0       ?GetBuddyStatus@CGameSpySBQR2GPConnection@@QEAA?AUSResult@1@HPEAUGPBuddyStatus@@@Z 0000000039a5c0a0 f   GameSpySBQR2GPConnection.obj
 0001:0005b0e0       ?GetLoginTicket@CGameSpySBQR2GPConnection@@QEAA?AUSResult@1@QEAD@Z 0000000039a5c0e0 f   GameSpySBQR2GPConnection.obj
 0001:0005b120       ?InvitePlayer@CGameSpySBQR2GPConnection@@QEAA?AUSResult@1@HQEBD@Z 0000000039a5c120 f   GameSpySBQR2GPConnection.obj
 0001:0005b190       ?RemoveFromBlockedList@CGameSpySBQR2GPConnection@@QEAA?AUSResult@1@H@Z 0000000039a5c190 f   GameSpySBQR2GPConnection.obj
 0001:0005b1d0       ?RevokeBuddyAuthorization@CGameSpySBQR2GPConnection@@QEAA?AUSResult@1@H@Z 0000000039a5c1d0 f   GameSpySBQR2GPConnection.obj
 0001:0005b210       ?SendBuddyMessage@CGameSpySBQR2GPConnection@@QEAA?AUSResult@1@HPEBD@Z 0000000039a5c210 f   GameSpySBQR2GPConnection.obj
 0001:0005b250       ?SendBuddyRequest@CGameSpySBQR2GPConnection@@QEAA?AUSResult@1@HQEBD@Z 0000000039a5c250 f   GameSpySBQR2GPConnection.obj
 0001:0005b290       ??0?$CryStackStringT@D$0DD@@@QEAA@PEBD@Z 0000000039a5c290 f i GameSpySBQR2GPConnection.obj
 0001:0005b320       ??$EventReceived@UGPRecvBuddyAuthArg@@@CGameSpySBQR2GPConnection@@CAXPEAPEAXPEAX1@Z 0000000039a5c320 f i GameSpySBQR2GPConnection.obj
 0001:0005b3d0       ??$EventReceived@UGPRecvBuddyMessageArg@@@CGameSpySBQR2GPConnection@@CAXPEAPEAXPEAX1@Z 0000000039a5c3d0 f i GameSpySBQR2GPConnection.obj
 0001:0005b480       ??$EventReceived@UGPRecvBuddyRequestArg@@@CGameSpySBQR2GPConnection@@CAXPEAPEAXPEAX1@Z 0000000039a5c480 f i GameSpySBQR2GPConnection.obj
 0001:0005b530       ??$EventReceived@UGPRecvBuddyRevokeArg@@@CGameSpySBQR2GPConnection@@CAXPEAPEAXPEAX1@Z 0000000039a5c530 f i GameSpySBQR2GPConnection.obj
 0001:0005b5e0       ??$EventReceived@UGPRecvBuddyStatusArg@@@CGameSpySBQR2GPConnection@@CAXPEAPEAXPEAX1@Z 0000000039a5c5e0 f i GameSpySBQR2GPConnection.obj
 0001:0005b690       ??$EventReceived@UGPRecvGameInviteArg@@@CGameSpySBQR2GPConnection@@CAXPEAPEAXPEAX1@Z 0000000039a5c690 f i GameSpySBQR2GPConnection.obj
 0001:0005b740       ??$EventReceived@UGPErrorArg@@@CGameSpySBQR2GPConnection@@CAXPEAPEAXPEAX1@Z 0000000039a5c740 f i GameSpySBQR2GPConnection.obj
 0001:0005b7f0       ?_Assign@?$CryStackStringT@D$0DD@@@QEAAXPEBD_K@Z 0000000039a5c7f0 f i GameSpySBQR2GPConnection.obj
 0001:0005b890       ??$TaskFinished@UGPProfileSearchResponseArg@@@CGameSpySBQR2GPConnection@@CAXPEAPEAXPEAX1@Z 0000000039a5c890 f i GameSpySBQR2GPConnection.obj
 0001:0005b990       ?ProcessTasks@CGameSpySBQR2GPConnection@@AEAAXI@Z 0000000039a5c990 f   GameSpySBQR2GPConnection.obj
 0001:0005ba40       ?ErrorReceived@CGameSpySBQR2GPConnection@@CAXPEAPEAXPEAX1@Z 0000000039a5ca40 f   GameSpySBQR2GPConnection.obj
 0001:0005ba70       ??$__copy_backward_ptrs@PEAV?$_smart_ptr@USCallbackBase@CGameSpySBQR2GPConnection@@@@PEAV1@@priv@stlpmtx_std@@YAPEAV?$_smart_ptr@USCallbackBase@CGameSpySBQR2GPConnection@@@@PEAV2@00AEBU__false_type@1@@Z 0000000039a5ca70 f i GameSpySBQR2GPConnection.obj
 0001:0005bb20       ??$fill@PEAV?$_smart_ptr@USCallbackBase@CGameSpySBQR2GPConnection@@@@V1@@stlpmtx_std@@YAXPEAV?$_smart_ptr@USCallbackBase@CGameSpySBQR2GPConnection@@@@0AEBV1@@Z 0000000039a5cb20 f i GameSpySBQR2GPConnection.obj
 0001:0005bbd0       ?SetStatusString@CGameSpySBQR2GPConnection@@QEAAXPEBD@Z 0000000039a5cbd0 f   GameSpySBQR2GPConnection.obj
 0001:0005bd10       ?SetLocationString@CGameSpySBQR2GPConnection@@QEAAXPEBD@Z 0000000039a5cd10 f   GameSpySBQR2GPConnection.obj
 0001:0005be50       ?_M_fill_insert_aux@?$_Impl_vector@V?$_smart_ptr@USCallbackBase@CGameSpySBQR2GPConnection@@@@V?$allocator@V?$_smart_ptr@USCallbackBase@CGameSpySBQR2GPConnection@@@@@stlpmtx_std@@@priv@stlpmtx_std@@AEAAXPEAV?$_smart_ptr@USCallbackBase@CGameSpySBQR2GPConnection@@@@_KAEBV4@AEBU__false_type@3@@Z 0000000039a5ce50 f i GameSpySBQR2GPConnection.obj
 0001:0005c070       ??$__destroy_range@PEAV?$_smart_ptr@USTaskBase@CGameSpySBQR2NATNegotiation@@@@V1@@stlpmtx_std@@YAXPEAV?$_smart_ptr@USTaskBase@CGameSpySBQR2NATNegotiation@@@@00@Z 0000000039a5d070 f i GameSpySBQR2NatNegotiation.obj
 0001:0005c070       ??$__destroy_range@PEAV?$_smart_ptr@USTask@CGameSpySBQR2Core@@@@V1@@stlpmtx_std@@YAXPEAV?$_smart_ptr@USTask@CGameSpySBQR2Core@@@@00@Z 0000000039a5d070 f i GameSpySBQR2Core.obj
 0001:0005c070       ??$__destroy_range@PEAV?$_smart_ptr@USTaskCallbackBase@CGameSpySBQR2GPConnection@@@@V1@@stlpmtx_std@@YAXPEAV?$_smart_ptr@USTaskCallbackBase@CGameSpySBQR2GPConnection@@@@00@Z 0000000039a5d070 f i GameSpySBQR2GPConnection.obj
 0001:0005c070       ??$__destroy_range@PEAV?$_smart_ptr@USTaskBase@CGameSpySBQR2Sake@@@@V1@@stlpmtx_std@@YAXPEAV?$_smart_ptr@USTaskBase@CGameSpySBQR2Sake@@@@00@Z 0000000039a5d070 f i GameSpySBQR2Sake.obj
 0001:0005c0f0       ?_M_erase@?$_Impl_vector@V?$_smart_ptr@USTaskCallbackBase@CGameSpySBQR2GPConnection@@@@V?$allocator@V?$_smart_ptr@USTaskCallbackBase@CGameSpySBQR2GPConnection@@@@@stlpmtx_std@@@priv@stlpmtx_std@@AEAAPEAV?$_smart_ptr@USTaskCallbackBase@CGameSpySBQR2GPConnection@@@@PEAV4@0AEBU__false_type@3@@Z 0000000039a5d0f0 f i GameSpySBQR2GPConnection.obj
 0001:0005c0f0       ?_M_erase@?$_Impl_vector@V?$_smart_ptr@USTask@CGameSpySBQR2Core@@@@V?$allocator@V?$_smart_ptr@USTask@CGameSpySBQR2Core@@@@@stlpmtx_std@@@priv@stlpmtx_std@@AEAAPEAV?$_smart_ptr@USTask@CGameSpySBQR2Core@@@@PEAV4@0AEBU__false_type@3@@Z 0000000039a5d0f0 f i GameSpySBQR2Core.obj
 0001:0005c0f0       ?_M_erase@?$_Impl_vector@V?$_smart_ptr@USTaskBase@CGameSpySBQR2NATNegotiation@@@@V?$allocator@V?$_smart_ptr@USTaskBase@CGameSpySBQR2NATNegotiation@@@@@stlpmtx_std@@@priv@stlpmtx_std@@AEAAPEAV?$_smart_ptr@USTaskBase@CGameSpySBQR2NATNegotiation@@@@PEAV4@0AEBU__false_type@3@@Z 0000000039a5d0f0 f i GameSpySBQR2NatNegotiation.obj
 0001:0005c0f0       ?_M_erase@?$_Impl_vector@V?$_smart_ptr@USTaskBase@CGameSpySBQR2Sake@@@@V?$allocator@V?$_smart_ptr@USTaskBase@CGameSpySBQR2Sake@@@@@stlpmtx_std@@@priv@stlpmtx_std@@AEAAPEAV?$_smart_ptr@USTaskBase@CGameSpySBQR2Sake@@@@PEAV4@0AEBU__false_type@3@@Z 0000000039a5d0f0 f i GameSpySBQR2Sake.obj
 0001:0005c1d0       ??0CGameSpySBQR2GPConnection@@QEAA@PEAVCCryGameSpySBQR2LobbyService@@I@Z 0000000039a5d1d0 f   GameSpySBQR2GPConnection.obj
 0001:0005c4a0       ?AddTaskCallback@CGameSpySBQR2GPConnection@@AEAAXPEAUSTaskCallbackBase@1@@Z 0000000039a5d4a0 f   GameSpySBQR2GPConnection.obj
 0001:0005c640       ?TearDown@CGameSpySBQR2GPConnection@@AEAAXXZ 0000000039a5d640 f   GameSpySBQR2GPConnection.obj
 0001:0005c6c0       ??$AddEventCallback@UGPErrorArg@@@CGameSpySBQR2GPConnection@@QEAAXP6AXPEAV0@USResult@0@PEAUGPErrorArg@@PEAUIGameSpyLink@@@Z3@Z 0000000039a5d6c0 f i GameSpySBQR2GPConnection.obj
 0001:0005c8a0       ??$AddEventCallback@UGPRecvBuddyAuthArg@@@CGameSpySBQR2GPConnection@@QEAAXP6AXPEAV0@USResult@0@PEAUGPRecvBuddyAuthArg@@PEAUIGameSpyLink@@@Z3@Z 0000000039a5d8a0 f i GameSpySBQR2GPConnection.obj
 0001:0005ca80       ??$AddEventCallback@UGPRecvBuddyMessageArg@@@CGameSpySBQR2GPConnection@@QEAAXP6AXPEAV0@USResult@0@PEAUGPRecvBuddyMessageArg@@PEAUIGameSpyLink@@@Z3@Z 0000000039a5da80 f i GameSpySBQR2GPConnection.obj
 0001:0005cc70       ??$AddEventCallback@UGPRecvBuddyRequestArg@@@CGameSpySBQR2GPConnection@@QEAAXP6AXPEAV0@USResult@0@PEAUGPRecvBuddyRequestArg@@PEAUIGameSpyLink@@@Z3@Z 0000000039a5dc70 f i GameSpySBQR2GPConnection.obj
 0001:0005ce50       ??$AddEventCallback@UGPRecvBuddyRevokeArg@@@CGameSpySBQR2GPConnection@@QEAAXP6AXPEAV0@USResult@0@PEAUGPRecvBuddyRevokeArg@@PEAUIGameSpyLink@@@Z3@Z 0000000039a5de50 f i GameSpySBQR2GPConnection.obj
 0001:0005d030       ??$AddEventCallback@UGPRecvBuddyStatusArg@@@CGameSpySBQR2GPConnection@@QEAAXP6AXPEAV0@USResult@0@PEAUGPRecvBuddyStatusArg@@PEAUIGameSpyLink@@@Z3@Z 0000000039a5e030 f i GameSpySBQR2GPConnection.obj
 0001:0005d220       ??$AddEventCallback@UGPRecvGameInviteArg@@@CGameSpySBQR2GPConnection@@QEAAXP6AXPEAV0@USResult@0@PEAUGPRecvGameInviteArg@@PEAUIGameSpyLink@@@Z3@Z 0000000039a5e220 f i GameSpySBQR2GPConnection.obj
 0001:0005d410       ?FailTask@?$STaskCallbackMid@UGPCheckResponseArg@@@CGameSpySBQR2GPConnection@@UEAAXAEAV?$_smart_ptr@USTaskCallbackBase@CGameSpySBQR2GPConnection@@@@W4GPResult@@@Z 0000000039a5e410 f i GameSpySBQR2GPConnection.obj
 0001:0005d410       ?FailTask@?$STaskCallbackMid@UGPGetInfoResponseArg@@@CGameSpySBQR2GPConnection@@UEAAXAEAV?$_smart_ptr@USTaskCallbackBase@CGameSpySBQR2GPConnection@@@@W4GPResult@@@Z 0000000039a5e410 f i GameSpySBQR2GPConnection.obj
 0001:0005d410       ?FailTask@?$STaskCallbackMid@UGPRegisterUniqueNickResponseArg@@@CGameSpySBQR2GPConnection@@UEAAXAEAV?$_smart_ptr@USTaskCallbackBase@CGameSpySBQR2GPConnection@@@@W4GPResult@@@Z 0000000039a5e410 f i GameSpySBQR2GPConnection.obj
 0001:0005d410       ?FailTask@?$STaskCallbackMid@UGPProfileSearchResponseArg@@@CGameSpySBQR2GPConnection@@UEAAXAEAV?$_smart_ptr@USTaskCallbackBase@CGameSpySBQR2GPConnection@@@@W4GPResult@@@Z 0000000039a5e410 f i GameSpySBQR2GPConnection.obj
 0001:0005d410       ?FailTask@?$STaskCallbackMid@UGPConnectResponseArg@@@CGameSpySBQR2GPConnection@@UEAAXAEAV?$_smart_ptr@USTaskCallbackBase@CGameSpySBQR2GPConnection@@@@W4GPResult@@@Z 0000000039a5e410 f i GameSpySBQR2GPConnection.obj
 0001:0005d410       ?FailTask@?$STaskCallbackMid@UGPNewUserResponseArg@@@CGameSpySBQR2GPConnection@@UEAAXAEAV?$_smart_ptr@USTaskCallbackBase@CGameSpySBQR2GPConnection@@@@W4GPResult@@@Z 0000000039a5e410 f i GameSpySBQR2GPConnection.obj
 0001:0005d410       ?FailTask@?$STaskCallbackMid@UGPNewProfileResponseArg@@@CGameSpySBQR2GPConnection@@UEAAXAEAV?$_smart_ptr@USTaskCallbackBase@CGameSpySBQR2GPConnection@@@@W4GPResult@@@Z 0000000039a5e410 f i GameSpySBQR2GPConnection.obj
 0001:0005d410       ?FailTask@?$STaskCallbackMid@UGPGetReverseBuddiesResponseArg@@@CGameSpySBQR2GPConnection@@UEAAXAEAV?$_smart_ptr@USTaskCallbackBase@CGameSpySBQR2GPConnection@@@@W4GPResult@@@Z 0000000039a5e410 f i GameSpySBQR2GPConnection.obj
 0001:0005d460       ??0?$STaskCallbackMid@UGPConnectResponseArg@@@CGameSpySBQR2GPConnection@@QEAA@PEAV1@PEAUIGameSpyLink@@P6AX0USResult@1@PEAUGPConnectResponseArg@@1@Z@Z 0000000039a5e460 f i GameSpySBQR2GPConnection.obj
 0001:0005d460       ??0?$STaskCallbackMid@UGPNewUserResponseArg@@@CGameSpySBQR2GPConnection@@QEAA@PEAV1@PEAUIGameSpyLink@@P6AX0USResult@1@PEAUGPNewUserResponseArg@@1@Z@Z 0000000039a5e460 f i GameSpySBQR2GPConnection.obj
 0001:0005d460       ??0?$STaskCallbackMid@UGPNewProfileResponseArg@@@CGameSpySBQR2GPConnection@@QEAA@PEAV1@PEAUIGameSpyLink@@P6AX0USResult@1@PEAUGPNewProfileResponseArg@@1@Z@Z 0000000039a5e460 f i GameSpySBQR2GPConnection.obj
 0001:0005d460       ??0?$STaskCallbackMid@UGPGetReverseBuddiesResponseArg@@@CGameSpySBQR2GPConnection@@QEAA@PEAV1@PEAUIGameSpyLink@@P6AX0USResult@1@PEAUGPGetReverseBuddiesResponseArg@@1@Z@Z 0000000039a5e460 f i GameSpySBQR2GPConnection.obj
 0001:0005d460       ??0?$STaskCallbackMid@UGPCheckResponseArg@@@CGameSpySBQR2GPConnection@@QEAA@PEAV1@PEAUIGameSpyLink@@P6AX0USResult@1@PEAUGPCheckResponseArg@@1@Z@Z 0000000039a5e460 f i GameSpySBQR2GPConnection.obj
 0001:0005d460       ??0?$STaskCallbackMid@UGPGetInfoResponseArg@@@CGameSpySBQR2GPConnection@@QEAA@PEAV1@PEAUIGameSpyLink@@P6AX0USResult@1@PEAUGPGetInfoResponseArg@@1@Z@Z 0000000039a5e460 f i GameSpySBQR2GPConnection.obj
 0001:0005d460       ??0?$STaskCallbackMid@UGPRegisterUniqueNickResponseArg@@@CGameSpySBQR2GPConnection@@QEAA@PEAV1@PEAUIGameSpyLink@@P6AX0USResult@1@PEAUGPRegisterUniqueNickResponseArg@@1@Z@Z 0000000039a5e460 f i GameSpySBQR2GPConnection.obj
 0001:0005d4f0       ??_GSCallbackBase@CGameSpySBQR2GPConnection@@UEAAPEAXI@Z 0000000039a5e4f0 f i GameSpySBQR2GPConnection.obj
 0001:0005d4f0       ??_ESCallbackBase@CGameSpySBQR2GPConnection@@UEAAPEAXI@Z 0000000039a5e4f0 f i GameSpySBQR2GPConnection.obj
 0001:0005d4f0       ??_G?$SEventCallback@UGPRecvBuddyMessageArg@@@CGameSpySBQR2GPConnection@@UEAAPEAXI@Z 0000000039a5e4f0 f i GameSpySBQR2GPConnection.obj
 0001:0005d4f0       ??_G?$STaskCallback0@UGPGetReverseBuddiesResponseArg@@@CGameSpySBQR2GPConnection@@UEAAPEAXI@Z 0000000039a5e4f0 f i GameSpySBQR2GPConnection.obj
 0001:0005d4f0       ??_E?$STaskCallbackMid@UGPGetInfoResponseArg@@@CGameSpySBQR2GPConnection@@UEAAPEAXI@Z 0000000039a5e4f0 f i GameSpySBQR2GPConnection.obj
 0001:0005d4f0       ??_G?$STaskCallbackMid@UGPGetInfoResponseArg@@@CGameSpySBQR2GPConnection@@UEAAPEAXI@Z 0000000039a5e4f0 f i GameSpySBQR2GPConnection.obj
 0001:0005d4f0       ??_GSTaskCallbackBase@CGameSpySBQR2GPConnection@@UEAAPEAXI@Z 0000000039a5e4f0 f i GameSpySBQR2GPConnection.obj
 0001:0005d4f0       ??_E?$STaskCallbackMid@UGPCheckResponseArg@@@CGameSpySBQR2GPConnection@@UEAAPEAXI@Z 0000000039a5e4f0 f i GameSpySBQR2GPConnection.obj
 0001:0005d4f0       ??_E?$STaskCallback0@UGPGetReverseBuddiesResponseArg@@@CGameSpySBQR2GPConnection@@UEAAPEAXI@Z 0000000039a5e4f0 f i GameSpySBQR2GPConnection.obj
 0001:0005d4f0       ??_G?$STaskCallbackMid@UGPRegisterUniqueNickResponseArg@@@CGameSpySBQR2GPConnection@@UEAAPEAXI@Z 0000000039a5e4f0 f i GameSpySBQR2GPConnection.obj
 0001:0005d4f0       ??_ESTaskCallbackBase@CGameSpySBQR2GPConnection@@UEAAPEAXI@Z 0000000039a5e4f0 f i GameSpySBQR2GPConnection.obj
 0001:0005d4f0       ??_E?$STaskCallbackMid@UGPNewProfileResponseArg@@@CGameSpySBQR2GPConnection@@UEAAPEAXI@Z 0000000039a5e4f0 f i GameSpySBQR2GPConnection.obj
 0001:0005d4f0       ??_E?$STaskCallbackMid@UGPProfileSearchResponseArg@@@CGameSpySBQR2GPConnection@@UEAAPEAXI@Z 0000000039a5e4f0 f i GameSpySBQR2GPConnection.obj
 0001:0005d4f0       ??_G?$SEventCallback@UGPRecvBuddyAuthArg@@@CGameSpySBQR2GPConnection@@UEAAPEAXI@Z 0000000039a5e4f0 f i GameSpySBQR2GPConnection.obj
 0001:0005d4f0       ??_E?$SEventCallback@UGPRecvBuddyRequestArg@@@CGameSpySBQR2GPConnection@@UEAAPEAXI@Z 0000000039a5e4f0 f i GameSpySBQR2GPConnection.obj
 0001:0005d4f0       ??_E?$SEventCallback@UGPErrorArg@@@CGameSpySBQR2GPConnection@@UEAAPEAXI@Z 0000000039a5e4f0 f i GameSpySBQR2GPConnection.obj
 0001:0005d4f0       ??_G?$SEventCallback@UGPErrorArg@@@CGameSpySBQR2GPConnection@@UEAAPEAXI@Z 0000000039a5e4f0 f i GameSpySBQR2GPConnection.obj
 0001:0005d4f0       ??_G?$STaskCallbackMid@UGPGetReverseBuddiesResponseArg@@@CGameSpySBQR2GPConnection@@UEAAPEAXI@Z 0000000039a5e4f0 f i GameSpySBQR2GPConnection.obj
 0001:0005d4f0       ??_G?$STaskCallbackMid@UGPCheckResponseArg@@@CGameSpySBQR2GPConnection@@UEAAPEAXI@Z 0000000039a5e4f0 f i GameSpySBQR2GPConnection.obj
 0001:0005d4f0       ??_G?$STaskCallbackMid@UGPConnectResponseArg@@@CGameSpySBQR2GPConnection@@UEAAPEAXI@Z 0000000039a5e4f0 f i GameSpySBQR2GPConnection.obj
 0001:0005d4f0       ??_E?$SEventCallback@UGPRecvBuddyRevokeArg@@@CGameSpySBQR2GPConnection@@UEAAPEAXI@Z 0000000039a5e4f0 f i GameSpySBQR2GPConnection.obj
 0001:0005d4f0       ??_E?$STaskCallbackMid@UGPRegisterUniqueNickResponseArg@@@CGameSpySBQR2GPConnection@@UEAAPEAXI@Z 0000000039a5e4f0 f i GameSpySBQR2GPConnection.obj
 0001:0005d4f0       ??_G?$SEventCallback@UGPRecvBuddyRevokeArg@@@CGameSpySBQR2GPConnection@@UEAAPEAXI@Z 0000000039a5e4f0 f i GameSpySBQR2GPConnection.obj
 0001:0005d4f0       ??_E?$STaskCallbackMid@UGPConnectResponseArg@@@CGameSpySBQR2GPConnection@@UEAAPEAXI@Z 0000000039a5e4f0 f i GameSpySBQR2GPConnection.obj
 0001:0005d4f0       ??_E?$STaskCallbackMid@UGPNewUserResponseArg@@@CGameSpySBQR2GPConnection@@UEAAPEAXI@Z 0000000039a5e4f0 f i GameSpySBQR2GPConnection.obj
 0001:0005d4f0       ??_G?$SEventCallback@UGPRecvGameInviteArg@@@CGameSpySBQR2GPConnection@@UEAAPEAXI@Z 0000000039a5e4f0 f i GameSpySBQR2GPConnection.obj
 0001:0005d4f0       ??_G?$STaskCallbackMid@UGPNewProfileResponseArg@@@CGameSpySBQR2GPConnection@@UEAAPEAXI@Z 0000000039a5e4f0 f i GameSpySBQR2GPConnection.obj
 0001:0005d4f0       ??_E?$STaskCallback2@UGPGetInfoResponseArg@@HW4GPEnum@@@CGameSpySBQR2GPConnection@@UEAAPEAXI@Z 0000000039a5e4f0 f i GameSpySBQR2GPConnection.obj
 0001:0005d4f0       ??_G?$STaskCallbackMid@UGPProfileSearchResponseArg@@@CGameSpySBQR2GPConnection@@UEAAPEAXI@Z 0000000039a5e4f0 f i GameSpySBQR2GPConnection.obj
 0001:0005d4f0       ??_E?$SEventCallback@UGPRecvBuddyStatusArg@@@CGameSpySBQR2GPConnection@@UEAAPEAXI@Z 0000000039a5e4f0 f i GameSpySBQR2GPConnection.obj
 0001:0005d4f0       ??_E?$STaskCallbackMid@UGPGetReverseBuddiesResponseArg@@@CGameSpySBQR2GPConnection@@UEAAPEAXI@Z 0000000039a5e4f0 f i GameSpySBQR2GPConnection.obj
 0001:0005d4f0       ??_E?$SEventCallback@UGPRecvBuddyMessageArg@@@CGameSpySBQR2GPConnection@@UEAAPEAXI@Z 0000000039a5e4f0 f i GameSpySBQR2GPConnection.obj
 0001:0005d4f0       ??_E?$SEventCallback@UGPRecvGameInviteArg@@@CGameSpySBQR2GPConnection@@UEAAPEAXI@Z 0000000039a5e4f0 f i GameSpySBQR2GPConnection.obj
 0001:0005d4f0       ??_E?$SEventCallback@UGPRecvBuddyAuthArg@@@CGameSpySBQR2GPConnection@@UEAAPEAXI@Z 0000000039a5e4f0 f i GameSpySBQR2GPConnection.obj
 0001:0005d4f0       ??_G?$STaskCallbackMid@UGPNewUserResponseArg@@@CGameSpySBQR2GPConnection@@UEAAPEAXI@Z 0000000039a5e4f0 f i GameSpySBQR2GPConnection.obj
 0001:0005d4f0       ??_G?$SEventCallback@UGPRecvBuddyRequestArg@@@CGameSpySBQR2GPConnection@@UEAAPEAXI@Z 0000000039a5e4f0 f i GameSpySBQR2GPConnection.obj
 0001:0005d4f0       ??_G?$STaskCallback2@UGPGetInfoResponseArg@@HW4GPEnum@@@CGameSpySBQR2GPConnection@@UEAAPEAXI@Z 0000000039a5e4f0 f i GameSpySBQR2GPConnection.obj
 0001:0005d4f0       ??_G?$SEventCallback@UGPRecvBuddyStatusArg@@@CGameSpySBQR2GPConnection@@UEAAPEAXI@Z 0000000039a5e4f0 f i GameSpySBQR2GPConnection.obj
 0001:0005d580       ??0?$STaskCallbackMid@UGPProfileSearchResponseArg@@@CGameSpySBQR2GPConnection@@QEAA@PEAV1@PEAUIGameSpyLink@@P6AX0USResult@1@PEAUGPProfileSearchResponseArg@@1@Z@Z 0000000039a5e580 f i GameSpySBQR2GPConnection.obj
 0001:0005d610       ??1CGameSpySBQR2GPConnection@@UEAA@XZ 0000000039a5e610 f   GameSpySBQR2GPConnection.obj
 0001:0005d9a0       ?PerformThink@CGameSpySBQR2GPConnection@@MEAAXXZ 0000000039a5e9a0 f   GameSpySBQR2GPConnection.obj
 0001:0005dc50       ??0?$STaskCallback3@UGPCheckResponseArg@@V?$CryFixedStringT@$0BP@@@V?$CryFixedStringT@$0DD@@@V2@@CGameSpySBQR2GPConnection@@QEAA@PEAV1@PEAUIGameSpyLink@@P6AX0USResult@1@PEAUGPCheckResponseArg@@1@ZP6A?AW4GPResult@@PEAPEAXPEBD66W4GPEnum@@P6AX5PEAX8@Z8@ZV?$CryFixedStringT@$0BP@@@V?$CryFixedStringT@$0DD@@@V7@@Z 0000000039a5ec50 f i GameSpySBQR2GPConnection.obj
 0001:0005dd90       ?StartTask@?$STaskCallback3@UGPCheckResponseArg@@V?$CryFixedStringT@$0BP@@@V?$CryFixedStringT@$0DD@@@V2@@CGameSpySBQR2GPConnection@@UEAA?AW4GPResult@@XZ 0000000039a5ed90 f i GameSpySBQR2GPConnection.obj
 0001:0005dde0       ??1?$STaskCallback3@UGPCheckResponseArg@@V?$CryFixedStringT@$0BP@@@V?$CryFixedStringT@$0DD@@@V2@@CGameSpySBQR2GPConnection@@UEAA@XZ 0000000039a5ede0 f i GameSpySBQR2GPConnection.obj
 0001:0005ded0       ??_G?$STaskCallback3@UGPCheckResponseArg@@V?$CryFixedStringT@$0BP@@@V?$CryFixedStringT@$0DD@@@V2@@CGameSpySBQR2GPConnection@@UEAAPEAXI@Z 0000000039a5eed0 f i GameSpySBQR2GPConnection.obj
 0001:0005ded0       ??_E?$STaskCallback3@UGPCheckResponseArg@@V?$CryFixedStringT@$0BP@@@V?$CryFixedStringT@$0DD@@@V2@@CGameSpySBQR2GPConnection@@UEAAPEAXI@Z 0000000039a5eed0 f i GameSpySBQR2GPConnection.obj
 0001:0005df00       ??0?$STaskCallback4@UGPConnectResponseArg@@V?$CryFixedStringT@$0BP@@@V?$CryFixedStringT@$0DD@@@V2@W4GPEnum@@@CGameSpySBQR2GPConnection@@QEAA@PEAV1@PEAUIGameSpyLink@@P6AX0USResult@1@PEAUGPConnectResponseArg@@1@ZP6A?AW4GPResult@@PEAPEAXPEBD66W4GPEnum@@7P6AX5PEAX8@Z8@ZV?$CryFixedStringT@$0BP@@@V?$CryFixedStringT@$0DD@@@V7@7@Z 0000000039a5ef00 f i GameSpySBQR2GPConnection.obj
 0001:0005e050       ?StartTask@?$STaskCallback4@UGPConnectResponseArg@@V?$CryFixedStringT@$0BP@@@V?$CryFixedStringT@$0DD@@@V2@W4GPEnum@@@CGameSpySBQR2GPConnection@@UEAA?AW4GPResult@@XZ 0000000039a5f050 f i GameSpySBQR2GPConnection.obj
 0001:0005e0a0       ??1?$STaskCallback4@UGPConnectResponseArg@@V?$CryFixedStringT@$0BP@@@V?$CryFixedStringT@$0DD@@@V2@W4GPEnum@@@CGameSpySBQR2GPConnection@@UEAA@XZ 0000000039a5f0a0 f i GameSpySBQR2GPConnection.obj
 0001:0005e190       ??_G?$STaskCallback4@UGPConnectResponseArg@@V?$CryFixedStringT@$0BP@@@V?$CryFixedStringT@$0DD@@@V2@W4GPEnum@@@CGameSpySBQR2GPConnection@@UEAAPEAXI@Z 0000000039a5f190 f i GameSpySBQR2GPConnection.obj
 0001:0005e190       ??_E?$STaskCallback4@UGPConnectResponseArg@@V?$CryFixedStringT@$0BP@@@V?$CryFixedStringT@$0DD@@@V2@W4GPEnum@@@CGameSpySBQR2GPConnection@@UEAAPEAXI@Z 0000000039a5f190 f i GameSpySBQR2GPConnection.obj
 0001:0005e1c0       ??0?$STaskCallback3@UGPConnectResponseArg@@V?$CryFixedStringT@$0BF@@@V?$CryFixedStringT@$0BP@@@W4GPEnum@@@CGameSpySBQR2GPConnection@@QEAA@PEAV1@PEAUIGameSpyLink@@P6AX0USResult@1@PEAUGPConnectResponseArg@@1@ZP6A?AW4GPResult@@PEAPEAXPEBD6W4GPEnum@@7P6AX5PEAX8@Z8@ZV?$CryFixedStringT@$0BF@@@V?$CryFixedStringT@$0BP@@@7@Z 0000000039a5f1c0 f i GameSpySBQR2GPConnection.obj
 0001:0005e2b0       ?StartTask@?$STaskCallback3@UGPConnectResponseArg@@V?$CryFixedStringT@$0BF@@@V?$CryFixedStringT@$0BP@@@W4GPEnum@@@CGameSpySBQR2GPConnection@@UEAA?AW4GPResult@@XZ 0000000039a5f2b0 f i GameSpySBQR2GPConnection.obj
 0001:0005e300       ??1?$STaskCallback3@UGPConnectResponseArg@@V?$CryFixedStringT@$0BF@@@V?$CryFixedStringT@$0BP@@@W4GPEnum@@@CGameSpySBQR2GPConnection@@UEAA@XZ 0000000039a5f300 f i GameSpySBQR2GPConnection.obj
 0001:0005e3c0       ??_E?$STaskCallback3@UGPConnectResponseArg@@V?$CryFixedStringT@$0BF@@@V?$CryFixedStringT@$0BP@@@W4GPEnum@@@CGameSpySBQR2GPConnection@@UEAAPEAXI@Z 0000000039a5f3c0 f i GameSpySBQR2GPConnection.obj
 0001:0005e3c0       ??_G?$STaskCallback3@UGPConnectResponseArg@@V?$CryFixedStringT@$0BF@@@V?$CryFixedStringT@$0BP@@@W4GPEnum@@@CGameSpySBQR2GPConnection@@UEAAPEAXI@Z 0000000039a5f3c0 f i GameSpySBQR2GPConnection.obj
 0001:0005e3f0       ?StartTask@?$STaskCallback2@UGPGetInfoResponseArg@@HW4GPEnum@@@CGameSpySBQR2GPConnection@@UEAA?AW4GPResult@@XZ 0000000039a5f3f0 f i GameSpySBQR2GPConnection.obj
 0001:0005e430       ?StartTask@?$STaskCallback0@UGPGetReverseBuddiesResponseArg@@@CGameSpySBQR2GPConnection@@UEAA?AW4GPResult@@XZ 0000000039a5f430 f i GameSpySBQR2GPConnection.obj
 0001:0005e450       ?StartTask@?$STaskCallback2@UGPNewProfileResponseArg@@V?$CryFixedStringT@$0BP@@@W4GPEnum@@@CGameSpySBQR2GPConnection@@UEAA?AW4GPResult@@XZ 0000000039a5f450 f i GameSpySBQR2GPConnection.obj
 0001:0005e490       ??1?$STaskCallback2@UGPNewProfileResponseArg@@V?$CryFixedStringT@$0BP@@@W4GPEnum@@@CGameSpySBQR2GPConnection@@UEAA@XZ 0000000039a5f490 f i GameSpySBQR2GPConnection.obj
 0001:0005e520       ??_E?$STaskCallback2@UGPNewProfileResponseArg@@V?$CryFixedStringT@$0BP@@@W4GPEnum@@@CGameSpySBQR2GPConnection@@UEAAPEAXI@Z 0000000039a5f520 f i GameSpySBQR2GPConnection.obj
 0001:0005e520       ??_G?$STaskCallback2@UGPNewProfileResponseArg@@V?$CryFixedStringT@$0BP@@@W4GPEnum@@@CGameSpySBQR2GPConnection@@UEAAPEAXI@Z 0000000039a5f520 f i GameSpySBQR2GPConnection.obj
 0001:0005e550       ??0?$STaskCallback5@UGPNewUserResponseArg@@V?$CryFixedStringT@$0BP@@@V?$CryFixedStringT@$0BF@@@V?$CryFixedStringT@$0DD@@@V2@PEBD@CGameSpySBQR2GPConnection@@QEAA@PEAV1@PEAUIGameSpyLink@@P6AX0USResult@1@PEAUGPNewUserResponseArg@@1@ZP6A?AW4GPResult@@PEAPEAXPEBD6666W4GPEnum@@P6AX5PEAX8@Z8@ZV?$CryFixedStringT@$0BP@@@V?$CryFixedStringT@$0BF@@@V?$CryFixedStringT@$0DD@@@V7@6@Z 0000000039a5f550 f i GameSpySBQR2GPConnection.obj
 0001:0005e6f0       ?StartTask@?$STaskCallback5@UGPNewUserResponseArg@@V?$CryFixedStringT@$0BP@@@V?$CryFixedStringT@$0BF@@@V?$CryFixedStringT@$0DD@@@V2@PEBD@CGameSpySBQR2GPConnection@@UEAA?AW4GPResult@@XZ 0000000039a5f6f0 f i GameSpySBQR2GPConnection.obj
 0001:0005e750       ??1?$STaskCallback5@UGPNewUserResponseArg@@V?$CryFixedStringT@$0BP@@@V?$CryFixedStringT@$0BF@@@V?$CryFixedStringT@$0DD@@@V2@PEBD@CGameSpySBQR2GPConnection@@UEAA@XZ 0000000039a5f750 f i GameSpySBQR2GPConnection.obj
 0001:0005e860       ??_E?$STaskCallback5@UGPNewUserResponseArg@@V?$CryFixedStringT@$0BP@@@V?$CryFixedStringT@$0BF@@@V?$CryFixedStringT@$0DD@@@V2@PEBD@CGameSpySBQR2GPConnection@@UEAAPEAXI@Z 0000000039a5f860 f i GameSpySBQR2GPConnection.obj
 0001:0005e860       ??_G?$STaskCallback5@UGPNewUserResponseArg@@V?$CryFixedStringT@$0BP@@@V?$CryFixedStringT@$0BF@@@V?$CryFixedStringT@$0DD@@@V2@PEBD@CGameSpySBQR2GPConnection@@UEAAPEAXI@Z 0000000039a5f860 f i GameSpySBQR2GPConnection.obj
 0001:0005e890       ??0?$STaskCallback6@UGPProfileSearchResponseArg@@V?$CryFixedStringT@$0BP@@@V?$CryFixedStringT@$0BF@@@V?$CryFixedStringT@$0DD@@@PEBDPEBDH@CGameSpySBQR2GPConnection@@QEAA@PEAV1@PEAUIGameSpyLink@@P6AX0USResult@1@PEAUGPProfileSearchResponseArg@@1@ZP6A?AW4GPResult@@PEAPEAXPEBD6666HW4GPEnum@@P6AX5PEAX8@Z8@ZV?$CryFixedStringT@$0BP@@@V?$CryFixedStringT@$0BF@@@V?$CryFixedStringT@$0DD@@@66H@Z 0000000039a5f890 f i GameSpySBQR2GPConnection.obj
 0001:0005ea00       ?StartTask@?$STaskCallback6@UGPProfileSearchResponseArg@@V?$CryFixedStringT@$0BP@@@V?$CryFixedStringT@$0BF@@@V?$CryFixedStringT@$0DD@@@PEBDPEBDH@CGameSpySBQR2GPConnection@@UEAA?AW4GPResult@@XZ 0000000039a5fa00 f i GameSpySBQR2GPConnection.obj
 0001:0005ea70       ??1?$STaskCallback6@UGPProfileSearchResponseArg@@V?$CryFixedStringT@$0BP@@@V?$CryFixedStringT@$0BF@@@V?$CryFixedStringT@$0DD@@@PEBDPEBDH@CGameSpySBQR2GPConnection@@UEAA@XZ 0000000039a5fa70 f i GameSpySBQR2GPConnection.obj
 0001:0005eb60       ??_E?$STaskCallback6@UGPProfileSearchResponseArg@@V?$CryFixedStringT@$0BP@@@V?$CryFixedStringT@$0BF@@@V?$CryFixedStringT@$0DD@@@PEBDPEBDH@CGameSpySBQR2GPConnection@@UEAAPEAXI@Z 0000000039a5fb60 f i GameSpySBQR2GPConnection.obj
 0001:0005eb60       ??_G?$STaskCallback6@UGPProfileSearchResponseArg@@V?$CryFixedStringT@$0BP@@@V?$CryFixedStringT@$0BF@@@V?$CryFixedStringT@$0DD@@@PEBDPEBDH@CGameSpySBQR2GPConnection@@UEAAPEAXI@Z 0000000039a5fb60 f i GameSpySBQR2GPConnection.obj
 0001:0005eb90       ?StartTask@?$STaskCallback3@UGPProfileSearchResponseArg@@V?$CryFixedStringT@$0BF@@@USIntPtrArg@CGameSpySBQR2GPConnection@@H@CGameSpySBQR2GPConnection@@UEAA?AW4GPResult@@XZ 0000000039a5fb90 f i GameSpySBQR2GPConnection.obj
 0001:0005ebd0       ??1?$STaskCallback3@UGPProfileSearchResponseArg@@V?$CryFixedStringT@$0BF@@@USIntPtrArg@CGameSpySBQR2GPConnection@@H@CGameSpySBQR2GPConnection@@UEAA@XZ 0000000039a5fbd0 f i GameSpySBQR2GPConnection.obj
 0001:0005ec60       ??_G?$STaskCallback3@UGPProfileSearchResponseArg@@V?$CryFixedStringT@$0BF@@@USIntPtrArg@CGameSpySBQR2GPConnection@@H@CGameSpySBQR2GPConnection@@UEAAPEAXI@Z 0000000039a5fc60 f i GameSpySBQR2GPConnection.obj
 0001:0005ec60       ??_E?$STaskCallback3@UGPProfileSearchResponseArg@@V?$CryFixedStringT@$0BF@@@USIntPtrArg@CGameSpySBQR2GPConnection@@H@CGameSpySBQR2GPConnection@@UEAAPEAXI@Z 0000000039a5fc60 f i GameSpySBQR2GPConnection.obj
 0001:0005ec90       ?StartTask@?$STaskCallback2@UGPRegisterUniqueNickResponseArg@@V?$CryFixedStringT@$0BF@@@PEBD@CGameSpySBQR2GPConnection@@UEAA?AW4GPResult@@XZ 0000000039a5fc90 f i GameSpySBQR2GPConnection.obj
 0001:0005ecd0       ??1?$STaskCallback2@UGPRegisterUniqueNickResponseArg@@V?$CryFixedStringT@$0BF@@@PEBD@CGameSpySBQR2GPConnection@@UEAA@XZ 0000000039a5fcd0 f i GameSpySBQR2GPConnection.obj
 0001:0005ed60       ??_E?$STaskCallback2@UGPRegisterUniqueNickResponseArg@@V?$CryFixedStringT@$0BF@@@PEBD@CGameSpySBQR2GPConnection@@UEAAPEAXI@Z 0000000039a5fd60 f i GameSpySBQR2GPConnection.obj
 0001:0005ed60       ??_G?$STaskCallback2@UGPRegisterUniqueNickResponseArg@@V?$CryFixedStringT@$0BF@@@PEBD@CGameSpySBQR2GPConnection@@UEAAPEAXI@Z 0000000039a5fd60 f i GameSpySBQR2GPConnection.obj
 0001:0005ed90       ??_GCGameSpySBQR2GPConnection@@UEAAPEAXI@Z 0000000039a5fd90 f i GameSpySBQR2GPConnection.obj
 0001:0005ed90       ??_ECGameSpySBQR2GPConnection@@UEAAPEAXI@Z 0000000039a5fd90 f i GameSpySBQR2GPConnection.obj
 0001:0005edc0       ?CheckUser@CGameSpySBQR2GPConnection@@QEAAXQEBD00P6AXPEAV1@USResult@1@PEAUGPCheckResponseArg@@PEAUIGameSpyLink@@@Z4@Z 0000000039a5fdc0 f   GameSpySBQR2GPConnection.obj
 0001:0005eef0       ?Connect@CGameSpySBQR2GPConnection@@QEAAXQEBD00P6AXPEAV1@USResult@1@PEAUGPConnectResponseArg@@PEAUIGameSpyLink@@@Z4@Z 0000000039a5fef0 f   GameSpySBQR2GPConnection.obj
 0001:0005f020       ?ConnectUniqueNick@CGameSpySBQR2GPConnection@@QEAAXQEBD0P6AXPEAV1@USResult@1@PEAUGPConnectResponseArg@@PEAUIGameSpyLink@@@Z4@Z 0000000039a60020 f   GameSpySBQR2GPConnection.obj
 0001:0005f130       ?GetInfo@CGameSpySBQR2GPConnection@@QEAAXHP6AXPEAV1@USResult@1@PEAUGPGetInfoResponseArg@@PEAUIGameSpyLink@@@Z3@Z 0000000039a60130 f   GameSpySBQR2GPConnection.obj
 0001:0005f200       ?GetReverseBuddies@CGameSpySBQR2GPConnection@@QEAAXP6AXPEAV1@USResult@1@PEAUGPGetReverseBuddiesResponseArg@@PEAUIGameSpyLink@@@Z3@Z 0000000039a60200 f   GameSpySBQR2GPConnection.obj
 0001:0005f2b0       ?NewProfile@CGameSpySBQR2GPConnection@@QEAAXQEBDP6AXPEAV1@USResult@1@PEAUGPNewProfileResponseArg@@PEAUIGameSpyLink@@@Z4@Z 0000000039a602b0 f   GameSpySBQR2GPConnection.obj
 0001:0005f3e0       ?NewUser@CGameSpySBQR2GPConnection@@QEAAXQEBD000P6AXPEAV1@USResult@1@PEAUGPNewUserResponseArg@@PEAUIGameSpyLink@@@Z4@Z 0000000039a603e0 f   GameSpySBQR2GPConnection.obj
 0001:0005f540       ?ProfileSearch@CGameSpySBQR2GPConnection@@QEAAXQEBD00P6AXPEAV1@USResult@1@PEAUGPProfileSearchResponseArg@@PEAUIGameSpyLink@@@Z4@Z 0000000039a60540 f   GameSpySBQR2GPConnection.obj
 0001:0005f680       ?ProfileSearchUniqueNick@CGameSpySBQR2GPConnection@@QEAAXQEBDP6AXPEAV1@USResult@1@PEAUGPProfileSearchResponseArg@@PEAUIGameSpyLink@@@Z4@Z 0000000039a60680 f   GameSpySBQR2GPConnection.obj
 0001:0005f7c0       ?RegisterUniqueNick@CGameSpySBQR2GPConnection@@QEAAXQEBDP6AXPEAV1@USResult@1@PEAUGPRegisterUniqueNickResponseArg@@PEAUIGameSpyLink@@@Z4@Z 0000000039a607c0 f   GameSpySBQR2GPConnection.obj
 0001:0005f8f0       ?GetSocketPorts@CCryLANLobbyService@@UEAAXAEAG0@Z 0000000039a608f0 f   CryLANLobby.obj
 0001:0005f900       ?Tick@CCryLANLobbyService@@UEAAXVCTimeValue@@@Z 0000000039a60900 f   CryLANLobby.obj
 0001:0005f990       ?GetSystemTime@CCryLANLobbyService@@UEAA?AW4ECryLobbyError@@IPEAUSCrySystemTime@@@Z 0000000039a60990 f   CryLANLobby.obj
 0001:0005fa00       ?OnPacket@CCryLANLobbyService@@UEAAXAEBV?$CConfigurableVariant@V?$CNode@USNullAddr@@V?$CNode@GV?$CNode@USIPv4Addr@@V?$CNode@ULobbyIdAddr@@VCEnd@NTypelist@@@NTypelist@@@NTypelist@@@NTypelist@@@NTypelist@@$07VCDefaultVariantConversion@NConfigurableVariantHelpers@@VCDefaultVariantConstruction@4@@@PEAVCCryLobbyPacket@@@Z 0000000039a60a00 f   CryLANLobby.obj
 0001:0005fa20       ?OnError@CCryLANLobbyService@@UEAAXAEBV?$CConfigurableVariant@V?$CNode@USNullAddr@@V?$CNode@GV?$CNode@USIPv4Addr@@V?$CNode@ULobbyIdAddr@@VCEnd@NTypelist@@@NTypelist@@@NTypelist@@@NTypelist@@@NTypelist@@$07VCDefaultVariantConversion@NConfigurableVariantHelpers@@VCDefaultVariantConstruction@4@@@W4ESocketError@@I@Z 0000000039a60a20 f   CryLANLobby.obj
 0001:0005fa40       ?OnSendComplete@CCryLANLobbyService@@UEAAXAEBV?$CConfigurableVariant@V?$CNode@USNullAddr@@V?$CNode@GV?$CNode@USIPv4Addr@@V?$CNode@ULobbyIdAddr@@VCEnd@NTypelist@@@NTypelist@@@NTypelist@@@NTypelist@@@NTypelist@@$07VCDefaultVariantConversion@NConfigurableVariantHelpers@@VCDefaultVariantConstruction@4@@@I@Z 0000000039a60a40 f   CryLANLobby.obj
 0001:0005fa60       ??0CCryLANLobbyService@@QEAA@PEAVCCryLobby@@W4ECryLobbyService@@@Z 0000000039a60a60 f   CryLANLobby.obj
 0001:0005faa0       ??_ECCryLANLobbyService@@WBA@EAAPEAXI@Z 0000000039a60aa0 f i CryLANLobby.obj
 0001:0005fab0       ?GetMatchMaking@CCryLANLobbyService@@UEAAPEAUICryMatchMaking@@XZ 0000000039a60ab0 f i CryLANLobby.obj
 0001:0005fad0       ?GetUserID@CCryLANLobbyService@@UEAA?AUCryUserID@@I@Z 0000000039a60ad0 f i CryLANLobby.obj
 0001:0005fb00       ??1CCryLANLobbyService@@UEAA@XZ 0000000039a60b00 f i CryLANLobby.obj
 0001:0005fb70       ?Initialise@CCryLANLobbyService@@UEAA?AW4ECryLobbyError@@W4ECryLobbyServiceFeatures@@P6AXW42@PEAVCCryLobby@@W4ECryLobbyService@@@Z@Z 0000000039a60b70 f   CryLANLobby.obj
 0001:0005fcf0       ?Terminate@CCryLANLobbyService@@UEAA?AW4ECryLobbyError@@W4ECryLobbyServiceFeatures@@P6AXW42@PEAVCCryLobby@@W4ECryLobbyService@@@Z@Z 0000000039a60cf0 f   CryLANLobby.obj
 0001:0005fe20       ??_GCCryLANLobbyService@@UEAAPEAXI@Z 0000000039a60e20 f i CryLANLobby.obj
 0001:0005fe20       ??_ECCryLANLobbyService@@UEAAPEAXI@Z 0000000039a60e20 f i CryLANLobby.obj
 0001:0005fe50       ?GetLocalUserName@SSession@CCryLANMatchMaking@@UEBAPEBDI@Z 0000000039a60e50 f   CryLANMatchMaking.obj
 0001:0005fe70       ?GetConnectionName@CCryLANMatchMaking@@EEBAPEBDPEAUSRConnection@SSession@CCryMatchMaking@@I@Z 0000000039a60e70 f   CryLANMatchMaking.obj
 0001:0005fea0       ?GetSessionIDSizeInPacket@CCryLANMatchMaking@@UEBAIXZ 0000000039a60ea0 f   CryLANMatchMaking.obj
 0001:0005feb0       ?ParamFilter@CCryLANMatchMaking@@AEAA_NIPEBUSCrySessionSearchData@@PEBUSCrySessionSearchResult@@@Z 0000000039a60eb0 f   CryLANMatchMaking.obj
 0001:00060380       ?get_deleter@?$sp_counted_impl_p@VCEngineModule_CryLobby@@@detail@boost@@UEAAPEAXAEBVsp_typeinfo@23@@Z 0000000039a61380 f   CryLobbyDLL.obj
 0001:00060380       gpiSendOrBufferChar        0000000039a61380 f   GameSpy_2.11.00_VC10:gpiBuffer.obj
 0001:00060380       ?GetLeaderboardType@CCryStats@@UEAA?AW4ECryLobbyLeaderboardType@@XZ 0000000039a61380 f   CryStats.obj
 0001:00060380       ?GetOnlineStorage@CCryGameSpySBQR2LobbyService@@UEAAPEAUICryOnlineStorage@@XZ 0000000039a61380 f   CryGameSpySBQR2Lobby.obj
 0001:00060380       ?GetLobbyUI@CCryLANLobbyService@@UEAAPEAUICryLobbyUI@@XZ 0000000039a61380 f   CryLANLobby.obj
 0001:00060380       ?QueryComposite@CEngineModule_CryLobby@@MEBAPEAXPEBD@Z 0000000039a61380 f   CryLobbyDLL.obj
 0001:00060380       ?GetDLCStore@CCryLobbyService@@UEAAPEAUICryDLCStore@@XZ 0000000039a61380 f   CryLobby.obj
 0001:00060380       ?GetVoice@CCryLANLobbyService@@UEAAPEAUICryVoice@@XZ 0000000039a61380 f   CryLANLobby.obj
 0001:00060380       ?GetReward@CCryLANLobbyService@@UEAAPEAUICryReward@@XZ 0000000039a61380 f   CryLANLobby.obj
 0001:00060380       ?SessionEnsureBestHost@CCryGameSpySBQR2MatchMaking@@UEAA?AW4ECryLobbyError@@IPEAIP6AXIW42@PEAX@Z2@Z 0000000039a61380 f   CryGameSpySBQR2MatchMaking.obj
 0001:00060380       ?GetMemorySize@?$VTableImpl@USNullAddr@@$0A@U?$IVisitor@V?$CNode@USNullAddr@@V?$CNode@GV?$CNode@USIPv4Addr@@V?$CNode@ULobbyIdAddr@@VCEnd@NTypelist@@@NTypelist@@@NTypelist@@@NTypelist@@@NTypelist@@@NConfigurableVariantHelpers@@U?$IMutatingVisitor@V?$CNode@USNullAddr@@V?$CNode@GV?$CNode@USIPv4Addr@@V?$CNode@ULobbyIdAddr@@VCEnd@NTypelist@@@NTypelist@@@NTypelist@@@NTypelist@@@NTypelist@@@3@@NConfigurableVariantHelpers@@SAHPEBX@Z 0000000039a61380 f   CryLobby.obj
 0001:00060380       ?GetCrysis3Lobby@CCryLobbyService@@UEAAPEAUICrysis3Lobby@@XZ 0000000039a61380 f   CryLobby.obj
 0001:00060380       ?GetConnectionUserID@CCryMatchMaking@@MEBA_KPEAUSRConnection@SSession@1@I@Z 0000000039a61380 f   CryMatchMaking.obj
 0001:00060380       ?GetMemorySize@?$VTableImpl@G$0A@U?$IVisitor@V?$CNode@USNullAddr@@V?$CNode@GV?$CNode@USIPv4Addr@@V?$CNode@ULobbyIdAddr@@VCEnd@NTypelist@@@NTypelist@@@NTypelist@@@NTypelist@@@NTypelist@@@NConfigurableVariantHelpers@@U?$IMutatingVisitor@V?$CNode@USNullAddr@@V?$CNode@GV?$CNode@USIPv4Addr@@V?$CNode@ULobbyIdAddr@@VCEnd@NTypelist@@@NTypelist@@@NTypelist@@@NTypelist@@@NTypelist@@@2@@NConfigurableVariantHelpers@@SAHPEBX@Z 0000000039a61380 f   CryGameSpySBQR2MatchMaking.obj
 0001:00060380       ?GetReward@CCryGameSpySBQR2LobbyService@@UEAAPEAUICryReward@@XZ 0000000039a61380 f   CryGameSpySBQR2Lobby.obj
 0001:00060380       ?Terminate@CCryDLCStore@@UEAA?AW4ECryLobbyError@@XZ 0000000039a61380 f   CryDLCStore.obj
 0001:00060380       ?GetSignIn@CCryLobbyService@@UEAAPEAUICrySignIn@@XZ 0000000039a61380 f   CryLobby.obj
 0001:00060380       ?SessionEnsureBestHost@CCryLANMatchMaking@@UEAA?AW4ECryLobbyError@@IPEAIP6AXIW42@PEAX@Z2@Z 0000000039a61380 f   CryLANMatchMaking.obj
 0001:00060380       ?GetStats@CCryLANLobbyService@@UEAAPEAUICryStats@@XZ 0000000039a61380 f   CryLANLobby.obj
 0001:00060380       ?GetSessionHostMigrationState@CCryMatchMaking@@UEAA?AW4eHostMigrationState@@I@Z 0000000039a61380 f   CryMatchMaking.obj
 0001:00060380       ?GetFriends@CCryLANLobbyService@@UEAAPEAUICryFriends@@XZ 0000000039a61380 f   CryLANLobby.obj
 0001:00060380       ?GetMemorySize@?$VTableImpl@USIPv4Addr@@$0A@U?$IVisitor@V?$CNode@USNullAddr@@V?$CNode@GV?$CNode@USIPv4Addr@@V?$CNode@ULobbyIdAddr@@VCEnd@NTypelist@@@NTypelist@@@NTypelist@@@NTypelist@@@NTypelist@@@NConfigurableVariantHelpers@@U?$IMutatingVisitor@V?$CNode@USNullAddr@@V?$CNode@GV?$CNode@USIPv4Addr@@V?$CNode@ULobbyIdAddr@@VCEnd@NTypelist@@@NTypelist@@@NTypelist@@@NTypelist@@@NTypelist@@@3@@NConfigurableVariantHelpers@@SAHPEBX@Z 0000000039a61380 f   CryLobby.obj
 0001:00060380       ?GetOnlineStorage@CCryLANLobbyService@@UEAAPEAUICryOnlineStorage@@XZ 0000000039a61380 f   CryLANLobby.obj
 0001:00060380       ?Terminate@CCryMatchMaking@@QEAA?AW4ECryLobbyError@@XZ 0000000039a61380 f   CryMatchMaking.obj
 0001:00060380       ?GetFriendsManagement@CCryLANLobbyService@@UEAAPEAUICryFriendsManagement@@XZ 0000000039a61380 f   CryLANLobby.obj
 0001:00060380       ?GetConnectionName@CCryMatchMaking@@MEBAPEBDPEAUSRConnection@SSession@1@I@Z 0000000039a61380 f   CryMatchMaking.obj
 0001:00060390       ?GetConnectionUserID@CCryLANMatchMaking@@EEBA_KPEAUSRConnection@SSession@CCryMatchMaking@@I@Z 0000000039a61390 f   CryLANMatchMaking.obj
 0001:000603c0       ?WriteToPacket@SCryLANSessionID@@QEBAXPEAVCCryLobbyPacket@@@Z 0000000039a613c0 f i CryLANMatchMaking.obj
 0001:00060490       ?Reset@SSession@CCryLANMatchMaking@@UEAAXXZ 0000000039a61490 f   CryLANMatchMaking.obj
 0001:000604f0       ??A?$CryLobbyIDArray@USSearch@CCryLANMatchMaking@@V?$CryLobbyID@USCryLANSearchHandle@CCryLANMatchMaking@@$01@@$01@@QEAAAEAUSSearch@CCryLANMatchMaking@@AEBV?$CryLobbyID@USCryLANSearchHandle@CCryLANMatchMaking@@$01@@@Z 0000000039a614f0 f i CryLANMatchMaking.obj
 0001:00060530       ??A?$CryLobbyIDArray@USSession@CCryLANMatchMaking@@V?$CryLobbyID@USCryLobbySessionHandle@@$03@@$03@@QEAAAEAUSSession@CCryLANMatchMaking@@AEBV?$CryLobbyID@USCryLobbySessionHandle@@$03@@@Z 0000000039a61530 f i CryLANMatchMaking.obj
 0001:00060570       ?ReadFromPacket@SCryLANSessionID@@QEAAXPEAVCCryLobbyPacket@@@Z 0000000039a61570 f i CryLANMatchMaking.obj
 0001:00060680       ??1SCryLANSessionID@@UEAA@XZ 0000000039a61680 f i CryLANMatchMaking.obj
 0001:00060690       ?CreateSessionHandle@CCryLANMatchMaking@@AEAA?AW4ECryLobbyError@@PEAV?$CryLobbyID@USCryLobbySessionHandle@@$03@@_NIH@Z 0000000039a61690 f   CryLANMatchMaking.obj
 0001:00060760       ?GetSIDFromSessionHandle@CCryLANMatchMaking@@EEAA_KV?$CryLobbyID@USCryLobbySessionHandle@@$03@@@Z 0000000039a61760 f   CryLANMatchMaking.obj
 0001:000607a0       ?FindSessionFromServerID@CCryLANMatchMaking@@AEAA?AV?$CryLobbyID@USCryLobbySessionHandle@@$03@@V2@@Z 0000000039a617a0 f   CryLANMatchMaking.obj
 0001:00060880       ?CreateSessionSearchHandle@CCryLANMatchMaking@@AEAA?AW4ECryLobbyError@@PEAV?$CryLobbyID@USCryLANSearchHandle@CCryLANMatchMaking@@$01@@@Z 0000000039a61880 f   CryLANMatchMaking.obj
 0001:000609a0       ?SetSessionUserData@CCryLANMatchMaking@@AEAA?AW4ECryLobbyError@@V?$CryLobbyID@USCryLobbySessionHandle@@$03@@PEAUSCryLobbyUserData@@I@Z 0000000039a619a0 f   CryLANMatchMaking.obj
 0001:00060ae0       ?SetSessionData@CCryLANMatchMaking@@AEAA?AW4ECryLobbyError@@V?$CryLobbyID@USCryLobbySessionHandle@@$03@@PEAUSCrySessionData@@@Z 0000000039a61ae0 f   CryLANMatchMaking.obj
 0001:00060c30       ?Initialise@CCryLANMatchMaking@@QEAA?AW4ECryLobbyError@@XZ 0000000039a61c30 f   CryLANMatchMaking.obj
 0001:00060cb0       ?SetLocalUserName@CCryLANMatchMaking@@AEAAXV?$CryLobbyID@USCryLobbySessionHandle@@$03@@I@Z 0000000039a61cb0 f   CryLANMatchMaking.obj
 0001:00060d40       ?CalculateServerDataSize@CCryLANMatchMaking@@AEAA_KV?$CryLobbyID@USCryLobbySessionHandle@@$03@@@Z 0000000039a61d40 f   CryLANMatchMaking.obj
 0001:00060e40       ?SendServerData@CCryLANMatchMaking@@AEAAXAEBV?$CConfigurableVariant@V?$CNode@USNullAddr@@V?$CNode@GV?$CNode@USIPv4Addr@@V?$CNode@ULobbyIdAddr@@VCEnd@NTypelist@@@NTypelist@@@NTypelist@@@NTypelist@@@NTypelist@@$07VCDefaultVariantConversion@NConfigurableVariantHelpers@@VCDefaultVariantConstruction@4@@@PEAVCCrySharedLobbyPacket@@@Z 0000000039a61e40 f   CryLANMatchMaking.obj
 0001:00061370       ?SessionGetCrySessionIDFromCrySessionHandle@CCryLANMatchMaking@@UEAA?AV?$_smart_ptr@USCrySessionID@@@@I@Z 0000000039a62370 f   CryLANMatchMaking.obj
 0001:00061380       ?Kick@CCryLANMatchMaking@@UEAAXPEBUCryUserID@@W4EDisconnectionCause@@@Z 0000000039a62380 f   CryLANMatchMaking.obj
 0001:000613b0       ?Execute@?$CClassJobNoRef@IVCCryLANMatchMaking@@@CWorkQueue@@UEAAXXZ 0000000039a623b0 f i CryLANMatchMaking.obj
 0001:000613b0       ?Execute@?$CClassJobNoRef@IVCCryGameSpySBQR2MatchMaking@@@CWorkQueue@@UEAAXXZ 0000000039a623b0 f i CryGameSpySBQR2MatchMaking.obj
 0001:000613b0       ?Execute@?$CClassJobNoRef@IVCCryMatchMaking@@@CWorkQueue@@UEAAXXZ 0000000039a623b0 f i CryMatchMaking.obj
 0001:000613e0       ?Execute@?$CClassJobNoRef5@IIGIIVCCryLANMatchMaking@@@CWorkQueue@@UEAAXXZ 0000000039a623e0 f i CryLANMatchMaking.obj
 0001:00061430       ??_G?$CClassJobNoRef5@IIGIIVCCryLANMatchMaking@@@CWorkQueue@@UEAAPEAXI@Z 0000000039a62430 f i CryLANMatchMaking.obj
 0001:00061430       ??_E?$CClassJobNoRef5@IIGIIVCCryLANMatchMaking@@@CWorkQueue@@UEAAPEAXI@Z 0000000039a62430 f i CryLANMatchMaking.obj
 0001:000614b0       ??0SCryLANSessionID@@QEAA@XZ 0000000039a624b0 f i CryLANMatchMaking.obj
 0001:000614e0       ?IsFromInvite@SCryGameSpySBQR2SessionID@@UEBA_NXZ 0000000039a624e0 f i CryGameSpySBQR2FriendsManagement.obj
 0001:000614e0       ?IsFromInvite@SCryLANSessionID@@UEBA_NXZ 0000000039a624e0 f i CryLANMatchMaking.obj
 0001:000614f0       ?snprintf@@YAHPEADHPEBDZZ  0000000039a624f0 f i CryLANMatchMaking.obj
 0001:00061520       ??8SCryLANSessionID@@UEAA_NAEBUSCrySessionID@@@Z 0000000039a62520 f i CryLANMatchMaking.obj
 0001:00061540       ??MSCryLANSessionID@@UEAA_NAEBUSCrySessionID@@@Z 0000000039a62540 f i CryLANMatchMaking.obj
 0001:00061580       ?AsCStr@SCryLANSessionID@@UEBAXPEADH@Z 0000000039a62580 f i CryLANMatchMaking.obj
 0001:000615c0       ?WriteSessionIDToPacket@CCryLANMatchMaking@@UEBA?AW4ECryLobbyError@@V?$_smart_ptr@USCrySessionID@@@@PEAVCCryLobbyPacket@@@Z 0000000039a625c0 f   CryLANMatchMaking.obj
 0001:000616b0       ?ReadSessionIDFromPacket@CCryLANMatchMaking@@UEBA?AV?$_smart_ptr@USCrySessionID@@@@PEAVCCryLobbyPacket@@@Z 0000000039a626b0 f   CryLANMatchMaking.obj
 0001:00061820       ?ServerDataToGame@CCryLANMatchMaking@@AEAAXIIGII@Z 0000000039a62820 f   CryLANMatchMaking.obj
 0001:00061e20       ??MSCryGameSpySBQR2SessionID@@UEAA_NAEBUSCrySessionID@@@Z 0000000039a62e20 f i CryGameSpySBQR2FriendsManagement.obj
 0001:00061e20       ??MSCryLANUserID@@UEBA_NAEBUSCryUserID@@@Z 0000000039a62e20 f i CryLANMatchMaking.obj
 0001:00061e30       ?SessionUserDataEvent@CCryLANMatchMaking@@AEAAXW4ECryLobbySystemEvent@@V?$CryLobbyID@USCryLobbySessionHandle@@$03@@V?$CryLobbyID@USCryMatchMakingConnectionID@@$0EA@@@@Z 0000000039a62e30 f   CryLANMatchMaking.obj
 0001:00062240       ?InitialUserDataEvent@CCryLANMatchMaking@@AEAAXV?$CryLobbyID@USCryLobbySessionHandle@@$03@@@Z 0000000039a63240 f   CryLANMatchMaking.obj
 0001:00062320       ??0SSession@CCryLANMatchMaking@@QEAA@XZ 0000000039a63320 f i CryLANMatchMaking.obj
 0001:000623c0       ??_ESSession@CCryLANMatchMaking@@UEAAPEAXI@Z 0000000039a633c0 f i CryLANMatchMaking.obj
 0001:000623c0       ??_GSSession@CCryLANMatchMaking@@UEAAPEAXI@Z 0000000039a633c0 f i CryLANMatchMaking.obj
 0001:00062400       ?FreeRemoteConnection@CCryLANMatchMaking@@EEAAXV?$CryLobbyID@USCryLobbySessionHandle@@$03@@V?$CryLobbyID@USCryMatchMakingConnectionID@@$0EA@@@@Z 0000000039a63400 f   CryLANMatchMaking.obj
 0001:000624d0       ?ProcessLocalUserData@CCryLANMatchMaking@@AEAAXAEBV?$CConfigurableVariant@V?$CNode@USNullAddr@@V?$CNode@GV?$CNode@USIPv4Addr@@V?$CNode@ULobbyIdAddr@@VCEnd@NTypelist@@@NTypelist@@@NTypelist@@@NTypelist@@@NTypelist@@$07VCDefaultVariantConversion@NConfigurableVariantHelpers@@VCDefaultVariantConstruction@4@@@PEAVCCrySharedLobbyPacket@@@Z 0000000039a634d0 f   CryLANMatchMaking.obj
 0001:00062680       ?GetSessionIDFromConsole@CCryLANMatchMaking@@UEAA?AV?$_smart_ptr@USCrySessionID@@@@XZ 0000000039a63680 f   CryLANMatchMaking.obj
 0001:00062bb0       ?EndSessionGetUsers@CCryLANMatchMaking@@AEAAXI@Z 0000000039a63bb0 f   CryLANMatchMaking.obj
 0001:00063270       ?EndTask@CCryLANMatchMaking@@AEAAXI@Z 0000000039a64270 f   CryLANMatchMaking.obj
 0001:00063560       ?GetGUIDAsString@SCryLANUserID@@UEBA?AV?$CryFixedStringT@$0CI@@@XZ 0000000039a64560 f i CryLANMatchMaking.obj
 0001:000635a0       ?AddRemoteConnection@CCryLANMatchMaking@@AEAA?AV?$CryLobbyID@USCryMatchMakingConnectionID@@$0EA@@@V?$CryLobbyID@USCryLobbySessionHandle@@$03@@V?$CryLobbyID@USCryLobbyConnectionID@@$0EA@@@USCryMatchMakingConnectionUID@@IGIPEBDQEAE_N@Z 0000000039a645a0 f   CryLANMatchMaking.obj
 0001:000637a0       ?ProcessSessionRequestJoin@CCryLANMatchMaking@@AEAAXAEBV?$CConfigurableVariant@V?$CNode@USNullAddr@@V?$CNode@GV?$CNode@USIPv4Addr@@V?$CNode@ULobbyIdAddr@@VCEnd@NTypelist@@@NTypelist@@@NTypelist@@@NTypelist@@@NTypelist@@$07VCDefaultVariantConversion@NConfigurableVariantHelpers@@VCDefaultVariantConstruction@4@@@PEAVCCrySharedLobbyPacket@@@Z 0000000039a647a0 f   CryLANMatchMaking.obj
 0001:000645f0       ?ProcessSessionAddRemoteConnections@CCryLANMatchMaking@@AEAAXAEBV?$CConfigurableVariant@V?$CNode@USNullAddr@@V?$CNode@GV?$CNode@USIPv4Addr@@V?$CNode@ULobbyIdAddr@@VCEnd@NTypelist@@@NTypelist@@@NTypelist@@@NTypelist@@@NTypelist@@$07VCDefaultVariantConversion@NConfigurableVariantHelpers@@VCDefaultVariantConstruction@4@@@PEAVCCrySharedLobbyPacket@@@Z 0000000039a655f0 f   CryLANMatchMaking.obj
 0001:00064a00       ?GetHostAddressFromSessionHandle@CCryLANMatchMaking@@EEAA?AV?$CConfigurableVariant@V?$CNode@USNullAddr@@V?$CNode@GV?$CNode@USIPv4Addr@@V?$CNode@ULobbyIdAddr@@VCEnd@NTypelist@@@NTypelist@@@NTypelist@@@NTypelist@@@NTypelist@@$07VCDefaultVariantConversion@NConfigurableVariantHelpers@@VCDefaultVariantConstruction@4@@@I@Z 0000000039a65a00 f   CryLANMatchMaking.obj
 0001:00064b50       ??$Add@IVCCryGameSpySBQR2MatchMaking@@@CWorkQueue@@QEAAXP8CCryGameSpySBQR2MatchMaking@@EAAXI@ZPEAV1@I@Z 0000000039a65b50 f i CryGameSpySBQR2MatchMaking.obj
 0001:00064b50       ??$Add@IVCCryLANMatchMaking@@@CWorkQueue@@QEAAXP8CCryLANMatchMaking@@EAAXI@ZPEAV1@I@Z 0000000039a65b50 f i CryLANMatchMaking.obj
 0001:00064b50       ??$Add@IVCCryMatchMaking@@@CWorkQueue@@QEAAXP8CCryMatchMaking@@EAAXI@ZPEAV1@I@Z 0000000039a65b50 f i CryMatchMaking.obj
 0001:00064c10       ??$Add@IIGIIVCCryLANMatchMaking@@@CWorkQueue@@QEAAXP8CCryLANMatchMaking@@EAAXIIGII@ZPEAV1@IIGII@Z 0000000039a65c10 f i CryLANMatchMaking.obj
 0001:00064d00       ?StopTaskRunning@CCryLANMatchMaking@@AEAAXI@Z 0000000039a65d00 f   CryLANMatchMaking.obj
 0001:00064d60       ?SendSessionQuery@CCryLANMatchMaking@@AEAAXVCTimeValue@@I_N@Z 0000000039a65d60 f   CryLANMatchMaking.obj
 0001:000650a0       ?StartSessionSetLocalUserData@CCryLANMatchMaking@@AEAAXI@Z 0000000039a660a0 f   CryLANMatchMaking.obj
 0001:000652e0       ?StartSessionDelete@CCryLANMatchMaking@@AEAAXI@Z 0000000039a662e0 f   CryLANMatchMaking.obj
 0001:000654d0       ?StartSessionJoin@CCryLANMatchMaking@@AEAAXI@Z 0000000039a664d0 f   CryLANMatchMaking.obj
 0001:000657b0       ?TickSessionJoin@CCryLANMatchMaking@@AEAAXI@Z 0000000039a667b0 f   CryLANMatchMaking.obj
 0001:000658e0       ?ProcessSessionRequestJoinResult@CCryLANMatchMaking@@AEAAXAEBV?$CConfigurableVariant@V?$CNode@USNullAddr@@V?$CNode@GV?$CNode@USIPv4Addr@@V?$CNode@ULobbyIdAddr@@VCEnd@NTypelist@@@NTypelist@@@NTypelist@@@NTypelist@@@NTypelist@@$07VCDefaultVariantConversion@NConfigurableVariantHelpers@@VCDefaultVariantConstruction@4@@@PEAVCCrySharedLobbyPacket@@@Z 0000000039a668e0 f   CryLANMatchMaking.obj
 0001:00065d50       ?ProcessServerData@CCryLANMatchMaking@@AEAAXAEBV?$CConfigurableVariant@V?$CNode@USNullAddr@@V?$CNode@GV?$CNode@USIPv4Addr@@V?$CNode@ULobbyIdAddr@@VCEnd@NTypelist@@@NTypelist@@@NTypelist@@@NTypelist@@@NTypelist@@$07VCDefaultVariantConversion@NConfigurableVariantHelpers@@VCDefaultVariantConstruction@4@@@PEAVCCrySharedLobbyPacket@@@Z 0000000039a66d50 f   CryLANMatchMaking.obj
 0001:00065fd0       ?OnPacket@CCryLANMatchMaking@@QEAAXAEBV?$CConfigurableVariant@V?$CNode@USNullAddr@@V?$CNode@GV?$CNode@USIPv4Addr@@V?$CNode@ULobbyIdAddr@@VCEnd@NTypelist@@@NTypelist@@@NTypelist@@@NTypelist@@@NTypelist@@$07VCDefaultVariantConversion@NConfigurableVariantHelpers@@VCDefaultVariantConstruction@4@@@PEAVCCryLobbyPacket@@@Z 0000000039a66fd0 f   CryLANMatchMaking.obj
 0001:000660b0       ?StartTaskRunning@CCryLANMatchMaking@@AEAAXI@Z 0000000039a670b0 f   CryLANMatchMaking.obj
 0001:00066240       ?Tick@CCryLANMatchMaking@@QEAAXVCTimeValue@@@Z 0000000039a67240 f   CryLANMatchMaking.obj
 0001:00066320       ?SessionRegisterUserData@CCryLANMatchMaking@@UEAA?AW4ECryLobbyError@@PEAUSCryLobbyUserData@@IPEAIP6AXIW42@PEAX@Z3@Z 0000000039a67320 f   CryLANMatchMaking.obj
 0001:00066460       ?SessionCreate@CCryLANMatchMaking@@UEAA?AW4ECryLobbyError@@PEAIHIPEAUSCrySessionData@@0P6AXIW42@IPEAX@Z3@Z 0000000039a67460 f   CryLANMatchMaking.obj
 0001:00066690       ?SessionMigrate@CCryLANMatchMaking@@UEAA?AW4ECryLobbyError@@IPEAIHIPEAUSCrySessionData@@0P6AXIW42@IPEAX@Z3@Z 0000000039a67690 f   CryLANMatchMaking.obj
 0001:00066820       ?SessionQuery@CCryLANMatchMaking@@UEAA?AW4ECryLobbyError@@IPEAIP6AXIW42@PEAUSCrySessionSearchResult@@PEAX@Z3@Z 0000000039a67820 f   CryLANMatchMaking.obj
 0001:00066970       ?SessionGetUsers@CCryLANMatchMaking@@UEAA?AW4ECryLobbyError@@IPEAIP6AXIW42@PEAUSCryUserInfoResult@@PEAX@Z3@Z 0000000039a67970 f   CryLANMatchMaking.obj
 0001:00066ac0       ?SessionSetLocalUserData@CCryLANMatchMaking@@UEAA?AW4ECryLobbyError@@IPEAIIPEAEIP6AXIW42@PEAX@Z3@Z 0000000039a67ac0 f   CryLANMatchMaking.obj
 0001:00066c20       ?SessionUpdate@CCryLANMatchMaking@@UEAA?AW4ECryLobbyError@@IPEAUSCryLobbyUserData@@IPEAIP6AXIW42@PEAX@Z3@Z 0000000039a67c20 f   CryLANMatchMaking.obj
 0001:00066da0       ?SessionUpdateSlots@CCryLANMatchMaking@@UEAA?AW4ECryLobbyError@@IIIPEAIP6AXIW42@PEAX@Z2@Z 0000000039a67da0 f   CryLANMatchMaking.obj
 0001:00066ee0       ?SessionStart@CCryLANMatchMaking@@UEAA?AW4ECryLobbyError@@IPEAIP6AXIW42@PEAX@Z2@Z 0000000039a67ee0 f   CryLANMatchMaking.obj
 0001:00067030       ?SessionEnd@CCryLANMatchMaking@@UEAA?AW4ECryLobbyError@@IPEAIP6AXIW42@PEAX@Z2@Z 0000000039a68030 f   CryLANMatchMaking.obj
 0001:00067180       ?SessionDelete@CCryLANMatchMaking@@UEAA?AW4ECryLobbyError@@IPEAIP6AXIW42@PEAX@Z2@Z 0000000039a68180 f   CryLANMatchMaking.obj
 0001:000672d0       ?SessionSearch@CCryLANMatchMaking@@UEAA?AW4ECryLobbyError@@IPEAUSCrySessionSearchParam@@PEAIP6AXIW42@PEAUSCrySessionSearchResult@@PEAX@Z4@Z 0000000039a682d0 f   CryLANMatchMaking.obj
 0001:000674c0       ?SessionJoin@CCryLANMatchMaking@@UEAA?AW4ECryLobbyError@@PEAIHIV?$_smart_ptr@USCrySessionID@@@@0P6AXIW42@IIGPEAX@Z3@Z 0000000039a684c0 f   CryLANMatchMaking.obj
 0001:000676d0       ??0CCryLANMatchMaking@@QEAA@PEAVCCryLobby@@PEAVCCryLobbyService@@W4ECryLobbyService@@@Z 0000000039a686d0 f   CryLANMatchMaking.obj
 0001:00067a90       ??_ECCryLANMatchMaking@@WBA@EAAPEAXI@Z 0000000039a68a90 f i CryLANMatchMaking.obj
 0001:00067aa0       ??1CCryLANMatchMaking@@UEAA@XZ 0000000039a68aa0 f i CryLANMatchMaking.obj
 0001:00067b50       ??_GCCryLANMatchMaking@@UEAAPEAXI@Z 0000000039a68b50 f i CryLANMatchMaking.obj
 0001:00067b50       ??_ECCryLANMatchMaking@@UEAAPEAXI@Z 0000000039a68b50 f i CryLANMatchMaking.obj
 0001:00067b80       ??1CLobbyCVars@@QEAA@XZ    0000000039a68b80 f   LobbyCVars.obj
 0001:00067b90       ?GameSpyLogInvitesCallback@CLobbyCVars@@CAXTUCryLobbyEventData@@PEAX@Z 0000000039a68b90 f   LobbyCVars.obj
 0001:00067be0       ?GameSpyListFriendsCallback@CLobbyCVars@@CAXIW4ECryLobbyError@@PEAUSFriendInfo@@IPEAX@Z 0000000039a68be0 f   LobbyCVars.obj
 0001:00067c40       ?GameSpyLogFriendEventCallback@CLobbyCVars@@CAXTUCryLobbyEventData@@PEAX@Z 0000000039a68c40 f   LobbyCVars.obj
 0001:00067c60       ?GameSpyIsProfileBlockedCallback@CLobbyCVars@@CAXIW4ECryLobbyError@@PEAUSFriendManagementInfo@@IPEAX@Z 0000000039a68c60 f   LobbyCVars.obj
 0001:00067cc0       ?GameSpyIsUserFriendCallback@CLobbyCVars@@CAXIW4ECryLobbyError@@PEAUSFriendManagementInfo@@IPEAX@Z 0000000039a68cc0 f   LobbyCVars.obj
 0001:00067d20       ?GameSpyGetNameCallback@CLobbyCVars@@CAXIW4ECryLobbyError@@PEAUSFriendInfo@@IPEAX@Z 0000000039a68d20 f   LobbyCVars.obj
 0001:00067d80       ?GameSpyFindUserCallback@CLobbyCVars@@CAXIW4ECryLobbyError@@PEAUSFriendInfo@@IPEAX@Z 0000000039a68d80 f   LobbyCVars.obj
 0001:00067de0       ?GameSpyGetProfileIDCmd@CLobbyCVars@@CAXPEAUIConsoleCmdArgs@@@Z 0000000039a68de0 f   LobbyCVars.obj
 0001:00067e80       ?GameSpyAcceptInviteCmd@CLobbyCVars@@CAXPEAUIConsoleCmdArgs@@@Z 0000000039a68e80 f   LobbyCVars.obj
 0001:00068060       ?GameSpySendInviteCmd@CLobbyCVars@@CAXPEAUIConsoleCmdArgs@@@Z 0000000039a69060 f   LobbyCVars.obj
 0001:000682e0       ?GameSpyLogInvitesCmd@CLobbyCVars@@CAXPEAUIConsoleCmdArgs@@@Z 0000000039a692e0 f   LobbyCVars.obj
 0001:00068330       ?GameSpyListFriendsCmd@CLobbyCVars@@CAXPEAUIConsoleCmdArgs@@@Z 0000000039a69330 f   LobbyCVars.obj
 0001:000683c0       ?GameSpySendFriendRequestCmd@CLobbyCVars@@CAXPEAUIConsoleCmdArgs@@@Z 0000000039a693c0 f   LobbyCVars.obj
 0001:000685a0       ?GameSpyAcceptFriendRequestCmd@CLobbyCVars@@CAXPEAUIConsoleCmdArgs@@@Z 0000000039a695a0 f   LobbyCVars.obj
 0001:00068780       ?GameSpyRevokeFriendStatusCmd@CLobbyCVars@@CAXPEAUIConsoleCmdArgs@@@Z 0000000039a69780 f   LobbyCVars.obj
 0001:00068960       ?GameSpyLogFriendEventsCmd@CLobbyCVars@@CAXPEAUIConsoleCmdArgs@@@Z 0000000039a69960 f   LobbyCVars.obj
 0001:00068a10       ?GameSpyBlockProfile@CLobbyCVars@@CAXPEAUIConsoleCmdArgs@@@Z 0000000039a69a10 f   LobbyCVars.obj
 0001:00068be0       ?GameSpyUnblockProfile@CLobbyCVars@@CAXPEAUIConsoleCmdArgs@@@Z 0000000039a69be0 f   LobbyCVars.obj
 0001:00068db0       ?GameSpyIsProfileBlocked@CLobbyCVars@@CAXPEAUIConsoleCmdArgs@@@Z 0000000039a69db0 f   LobbyCVars.obj
 0001:00068f80       ?GameSpyIsUserFriend@CLobbyCVars@@CAXPEAUIConsoleCmdArgs@@@Z 0000000039a69f80 f   LobbyCVars.obj
 0001:00069150       ?GameSpyGetName@CLobbyCVars@@CAXPEAUIConsoleCmdArgs@@@Z 0000000039a6a150 f   LobbyCVars.obj
 0001:00069320       ?GameSpyFindUser@CLobbyCVars@@CAXPEAUIConsoleCmdArgs@@@Z 0000000039a6a320 f   LobbyCVars.obj
 0001:00069480       ??0CLobbyCVars@@QEAA@XZ    0000000039a6a480 f   LobbyCVars.obj
 0001:00069f40       ?DeInitialize@?$Node_Alloc_Lock@$00$00@@SAXXZ 0000000039a6af40 f i StdAfx.obj
 0001:00069fa8       connect                    0000000039a6afa8 f   Wsock32:WSOCK32.dll
 0001:00069fae       ioctlsocket                0000000039a6afae f   Wsock32:WSOCK32.dll
 0001:00069fb4       closesocket                0000000039a6afb4 f   Wsock32:WSOCK32.dll
 0001:00069fba       setsockopt                 0000000039a6afba f   Wsock32:WSOCK32.dll
 0001:00069fc0       socket                     0000000039a6afc0 f   Wsock32:WSOCK32.dll
 0001:00069fc6       send                       0000000039a6afc6 f   Wsock32:WSOCK32.dll
 0001:00069fcc       __WSAFDIsSet               0000000039a6afcc f   Wsock32:WSOCK32.dll
 0001:00069fd2       select                     0000000039a6afd2 f   Wsock32:WSOCK32.dll
 0001:00069fd8       recv                       0000000039a6afd8 f   Wsock32:WSOCK32.dll
 0001:00069fde       htons                      0000000039a6afde f   Wsock32:WSOCK32.dll
 0001:00069fe4       inet_ntoa                  0000000039a6afe4 f   Wsock32:WSOCK32.dll
 0001:00069fea       ntohs                      0000000039a6afea f   Wsock32:WSOCK32.dll
 0001:00069ff0       getsockname                0000000039a6aff0 f   Wsock32:WSOCK32.dll
 0001:00069ff6       ntohl                      0000000039a6aff6 f   Wsock32:WSOCK32.dll
 0001:00069ffc       htonl                      0000000039a6affc f   Wsock32:WSOCK32.dll
 0001:0006a020       __chkstk                   0000000039a6b020 f   MSVCRT:chkstk.obj
 0001:0006a020       _alloca_probe              0000000039a6b020     MSVCRT:chkstk.obj
 0001:0006a070       _onexit                    0000000039a6b070 f   MSVCRT:atonexit.obj
 0001:0006a120       atexit                     0000000039a6b120 f   MSVCRT:atonexit.obj
 0001:0006a138       _purecall                  0000000039a6b138 f   MSVCRT:MSVCR100.dll
 0001:0006a13e       memcpy                     0000000039a6b13e f   MSVCRT:MSVCR100.dll
 0001:0006a144       memset                     0000000039a6b144 f   MSVCRT:MSVCR100.dll
 0001:0006a14a       ?what@exception@std@@UEBAPEBDXZ 0000000039a6b14a f   MSVCRT:MSVCR100.dll
 0001:0006a1b0       _CRT_INIT                  0000000039a6b1b0 f   MSVCRT:crtdll.obj
 0001:0006a548       _DllMainCRTStartup         0000000039a6b548 f   MSVCRT:crtdll.obj
 0001:0006a586       __C_specific_handler       0000000039a6b586 f   MSVCRT:MSVCR100.dll
 0001:0006a58c       _unlock                    0000000039a6b58c f   MSVCRT:MSVCR100.dll
 0001:0006a592       __dllonexit                0000000039a6b592 f   MSVCRT:MSVCR100.dll
 0001:0006a598       _lock                      0000000039a6b598 f   MSVCRT:MSVCR100.dll
 0001:0006a5a0       __clean_type_info_names    0000000039a6b5a0 f   MSVCRT:tncleanup.obj
 0001:0006a5ac       _RTC_Initialize            0000000039a6b5ac f   MSVCRT:_initsect_.obj
 0001:0006a5e4       _RTC_Terminate             0000000039a6b5e4 f   MSVCRT:_initsect_.obj
 0001:0006a620       _ValidateImageBase         0000000039a6b620 f   MSVCRT:pesect.obj
 0001:0006a650       _FindPESection             0000000039a6b650 f   MSVCRT:pesect.obj
 0001:0006a6a0       _IsNonwritableInCurrentImage 0000000039a6b6a0 f   MSVCRT:pesect.obj
 0001:0006a6e2       _initterm                  0000000039a6b6e2 f   MSVCRT:MSVCR100.dll
 0001:0006a6e8       _initterm_e                0000000039a6b6e8 f   MSVCRT:MSVCR100.dll
 0001:0006a6ee       _amsg_exit                 0000000039a6b6ee f   MSVCRT:MSVCR100.dll
 0001:0006a6f4       __CppXcptFilter            0000000039a6b6f4 f   MSVCRT:MSVCR100.dll
 0001:0006a6fc       DllMain                    0000000039a6b6fc f   MSVCRT:dllmain.obj
 0001:0006a720       __security_init_cookie     0000000039a6b720 f   MSVCRT:gs_support.obj
 0001:0006a7d4       __clean_type_info_names_internal 0000000039a6b7d4 f   MSVCRT:MSVCR100.dll
 0001:0006a950       NNFreeNegotiateList        0000000039a6b950 f   GameSpy_2.11.00_VC10:natneg.obj
 0001:0006b2a0       NNStartNatDetection        0000000039a6c2a0 f   GameSpy_2.11.00_VC10:natneg.obj
 0001:0006b4a0       NNInternalBeginNegotiationWithSocket 0000000039a6c4a0 f   GameSpy_2.11.00_VC10:natneg.obj
 0001:0006b5e0       NNCancel                   0000000039a6c5e0 f   GameSpy_2.11.00_VC10:natneg.obj
 0001:0006b8f0       NNBeginNegotiationWithSocket 0000000039a6c8f0 f   GameSpy_2.11.00_VC10:natneg.obj
 0001:0006baf0       NNProcessData              0000000039a6caf0 f   GameSpy_2.11.00_VC10:natneg.obj
 0001:0006bf90       NNThink                    0000000039a6cf90 f   GameSpy_2.11.00_VC10:natneg.obj
 0001:0006c070       GSIStartAvailableCheckA    0000000039a6d070 f   GameSpy_2.11.00_VC10:gsAvailable.obj
 0001:0006c200       GSIAvailableCheckThink     0000000039a6d200 f   GameSpy_2.11.00_VC10:gsAvailable.obj
 0001:0006c3d0       GSIGetAvailable            0000000039a6d3d0 f   GameSpy_2.11.00_VC10:gsAvailable.obj
 0001:0006c3e0       ptTrackUsageA              0000000039a6d3e0 f   GameSpy_2.11.00_VC10:ptMain.obj
 0001:0006c4e0       gsCoreInitialize           0000000039a6d4e0 f   GameSpy_2.11.00_VC10:gsCore.obj
 0001:0006c610       gsCoreIsShutdown           0000000039a6d610 f   GameSpy_2.11.00_VC10:gsCore.obj
 0001:0006c640       gsiCoreExecuteTask         0000000039a6d640 f   GameSpy_2.11.00_VC10:gsCore.obj
 0001:0006c6c0       gsiCoreCreateTask          0000000039a6d6c0 f   GameSpy_2.11.00_VC10:gsCore.obj
 0001:0006c700       gsCoreThink                0000000039a6d700 f   GameSpy_2.11.00_VC10:gsCore.obj
 0001:0006c970       gsCoreShutdown             0000000039a6d970 f   GameSpy_2.11.00_VC10:gsCore.obj
 0001:0006ca60       sakeStartup                0000000039a6da60 f   GameSpy_2.11.00_VC10:sakeMain.obj
 0001:0006cae0       sakeiFreeRequest           0000000039a6dae0 f   GameSpy_2.11.00_VC10:sakeRequest.obj
 0001:0006cae0       sakeShutdown               0000000039a6dae0 f   GameSpy_2.11.00_VC10:sakeMain.obj
 0001:0006caf0       sakeSetGame                0000000039a6daf0 f   GameSpy_2.11.00_VC10:sakeMain.obj
 0001:0006cb40       sakeSetProfile             0000000039a6db40 f   GameSpy_2.11.00_VC10:sakeMain.obj
 0001:0006cb70       sakeGetStartRequestResult  0000000039a6db70 f   GameSpy_2.11.00_VC10:sakeMain.obj
 0001:0006cb80       sakeCreateRecord           0000000039a6db80 f   GameSpy_2.11.00_VC10:sakeMain.obj
 0001:0006cbe0       sakeUpdateRecord           0000000039a6dbe0 f   GameSpy_2.11.00_VC10:sakeMain.obj
 0001:0006cc40       sakeSearchForRecords       0000000039a6dc40 f   GameSpy_2.11.00_VC10:sakeMain.obj
 0001:0006cca0       sakeGetMyRecords           0000000039a6dca0 f   GameSpy_2.11.00_VC10:sakeMain.obj
 0001:0006cd00       sakeGetRecordCount         0000000039a6dd00 f   GameSpy_2.11.00_VC10:sakeMain.obj
 0001:0006cd60       d2gCreateInstance          0000000039a6dd60 f   GameSpy_2.11.00_VC10:d2gMain.obj
 0001:0006cda0       d2gInitialize              0000000039a6dda0 f   GameSpy_2.11.00_VC10:d2gMain.obj
 0001:0006ce60       d2gCleanup                 0000000039a6de60 f   GameSpy_2.11.00_VC10:d2gMain.obj
 0001:0006cf10       d2gCreateCatalog           0000000039a6df10 f   GameSpy_2.11.00_VC10:d2gMain.obj
 0001:0006d000       d2gCleanupCatalog          0000000039a6e000 f   GameSpy_2.11.00_VC10:d2gMain.obj
 0001:0006d050       d2gGetStoreAvailability    0000000039a6e050 f   GameSpy_2.11.00_VC10:d2gMain.obj
 0001:0006d0d0       d2gLoadCatalogItems        0000000039a6e0d0 f   GameSpy_2.11.00_VC10:d2gMain.obj
 0001:0006d170       d2gGetUserCreditCards      0000000039a6e170 f   GameSpy_2.11.00_VC10:d2gMain.obj
 0001:0006d1f0       d2gGetOrderTotal           0000000039a6e1f0 f   GameSpy_2.11.00_VC10:d2gMain.obj
 0001:0006d2f0       d2gStartOrder              0000000039a6e2f0 f   GameSpy_2.11.00_VC10:d2gMain.obj
 0001:0006d380       d2gIsOrderComplete         0000000039a6e380 f   GameSpy_2.11.00_VC10:d2gMain.obj
 0001:0006d410       d2gGetPurchaseHistory      0000000039a6e410 f   GameSpy_2.11.00_VC10:d2gMain.obj
 0001:0006d490       d2gStartDownloadFileById   0000000039a6e490 f   GameSpy_2.11.00_VC10:d2gMain.obj
 0001:0006d550       d2gFreeCatalogItemList     0000000039a6e550 f   GameSpy_2.11.00_VC10:d2gMain.obj
 0001:0006d570       d2gFreeOrderTotal          0000000039a6e570 f   GameSpy_2.11.00_VC10:d2gMain.obj
 0001:0006d580       d2gFreeOrderPurchase       0000000039a6e580 f   GameSpy_2.11.00_VC10:d2gMain.obj
 0001:0006d590       d2gFreeCreditCardInfoList  0000000039a6e590 f   GameSpy_2.11.00_VC10:d2gMain.obj
 0001:0006d5a0       d2gGetCategories           0000000039a6e5a0 f   GameSpy_2.11.00_VC10:d2gMain.obj
 0001:0006d610       d2gCancelDownload          0000000039a6e610 f   GameSpy_2.11.00_VC10:d2gMain.obj
 0001:0006d660       gsimalloc                  0000000039a6e660 f   GameSpy_2.11.00_VC10:gsMemory.obj
 0001:0006d670       gsirealloc                 0000000039a6e670 f   GameSpy_2.11.00_VC10:gsMemory.obj
 0001:0006d680       gsifree                    0000000039a6e680 f   GameSpy_2.11.00_VC10:gsMemory.obj
 0001:0006e3c0       gcd_init                   0000000039a6f3c0 f   GameSpy_2.11.00_VC10:gcdkeys.obj
 0001:0006e5b0       gcd_authenticate_user      0000000039a6f5b0 f   GameSpy_2.11.00_VC10:gcdkeys.obj
 0001:0006e7d0       gcd_process_reauth         0000000039a6f7d0 f   GameSpy_2.11.00_VC10:gcdkeys.obj
 0001:0006e8c0       gcd_disconnect_user        0000000039a6f8c0 f   GameSpy_2.11.00_VC10:gcdkeys.obj
 0001:0006eb50       gcd_think                  0000000039a6fb50 f   GameSpy_2.11.00_VC10:gcdkeys.obj
 0001:0006ef30       gcd_compute_response       0000000039a6ff30 f   GameSpy_2.11.00_VC10:gcdkeyc.obj
 0001:0006f340       ServerBrowserNewA          0000000039a70340 f   GameSpy_2.11.00_VC10:sb_serverbrowsing.obj
 0001:0006f440       ServerBrowserSendNatNegotiateCookieToServerA 0000000039a70440 f   GameSpy_2.11.00_VC10:sb_serverbrowsing.obj
 0001:0006f4a0       ServerBrowserThink         0000000039a704a0 f   GameSpy_2.11.00_VC10:sb_serverbrowsing.obj
 0001:0006f4d0       ServerBrowserHalt          0000000039a704d0 f   GameSpy_2.11.00_VC10:sb_serverbrowsing.obj
 0001:0006f500       ServerBrowserClear         0000000039a70500 f   GameSpy_2.11.00_VC10:sb_serverbrowsing.obj
 0001:0006f540       ServerBrowserBeginUpdate2  0000000039a70540 f   GameSpy_2.11.00_VC10:sb_serverbrowsing.obj
 0001:0006f6d0       ServerBrowserUpdateA       0000000039a706d0 f   GameSpy_2.11.00_VC10:sb_serverbrowsing.obj
 0001:0006f770       ServerBrowserAuxUpdateServer 0000000039a70770 f   GameSpy_2.11.00_VC10:sb_serverbrowsing.obj
 0001:0006f860       qr2_register_natneg_callback 0000000039a70860 f   GameSpy_2.11.00_VC10:qr2.obj
 0001:0006f880       qr2_register_publicaddress_callback 0000000039a70880 f   GameSpy_2.11.00_VC10:qr2.obj
 0001:0006f8a0       qr2_register_hostregistered_callback 0000000039a708a0 f   GameSpy_2.11.00_VC10:qr2.obj
 0001:0006f8c0       qr2_keybuffer_add          0000000039a708c0 f   GameSpy_2.11.00_VC10:qr2.obj
 0001:0006f8f0       qr2_buffer_addA            0000000039a708f0 f   GameSpy_2.11.00_VC10:qr2.obj
 0001:00070780       qr2_init_socketA           0000000039a71780 f   GameSpy_2.11.00_VC10:qr2.obj
 0001:00070ac0       qr2_buffer_add_int         0000000039a71ac0 f   GameSpy_2.11.00_VC10:qr2.obj
 0001:00070c80       qr2_parse_queryA           0000000039a71c80 f   GameSpy_2.11.00_VC10:qr2.obj
 0001:00071910       qr2_send_statechanged      0000000039a72910 f   GameSpy_2.11.00_VC10:qr2.obj
 0001:00071970       qr2_shutdown               0000000039a72970 f   GameSpy_2.11.00_VC10:qr2.obj
 0001:00071a00       qr2_think                  0000000039a72a00 f   GameSpy_2.11.00_VC10:qr2.obj
 0001:00071a70       gpInitialize               0000000039a72a70 f   GameSpy_2.11.00_VC10:gp.obj
 0001:00071a90       gpDestroy                  0000000039a72a90 f   GameSpy_2.11.00_VC10:gp.obj
 0001:00071ab0       gpProcess                  0000000039a72ab0 f   GameSpy_2.11.00_VC10:gp.obj
 0001:00071ae0       gpSetCallback              0000000039a72ae0 f   GameSpy_2.11.00_VC10:gp.obj
 0001:00071b40       gpConnectA                 0000000039a72b40 f   GameSpy_2.11.00_VC10:gp.obj
 0001:00071c80       gpConnectUniqueNickA       0000000039a72c80 f   GameSpy_2.11.00_VC10:gp.obj
 0001:00071db0       gpDisconnect               0000000039a72db0 f   GameSpy_2.11.00_VC10:gp.obj
 0001:00071e10       gpIsConnected              0000000039a72e10 f   GameSpy_2.11.00_VC10:gp.obj
 0001:00071e40       gpCheckUserA               0000000039a72e40 f   GameSpy_2.11.00_VC10:gp.obj
 0001:00071f60       gpNewUserA                 0000000039a72f60 f   GameSpy_2.11.00_VC10:gp.obj
 0001:00072120       gpRegisterUniqueNickA      0000000039a73120 f   GameSpy_2.11.00_VC10:gp.obj
 0001:000721d0       gpGetErrorCode             0000000039a731d0 f   GameSpy_2.11.00_VC10:gp.obj
 0001:00072210       gpGetErrorStringA          0000000039a73210 f   GameSpy_2.11.00_VC10:gp.obj
 0001:00072260       gpNewProfileA              0000000039a73260 f   GameSpy_2.11.00_VC10:gp.obj
 0001:00072320       gpProfileSearchA           0000000039a73320 f   GameSpy_2.11.00_VC10:gp.obj
 0001:000723f0       gpProfileSearchUniquenickA 0000000039a733f0 f   GameSpy_2.11.00_VC10:gp.obj
 0001:000724a0       gpGetInfo                  0000000039a734a0 f   GameSpy_2.11.00_VC10:gp.obj
 0001:00072570       gpSendBuddyRequestA        0000000039a73570 f   GameSpy_2.11.00_VC10:gp.obj
 0001:00072660       gpAuthBuddyRequest         0000000039a73660 f   GameSpy_2.11.00_VC10:gp.obj
 0001:000726b0       gpDenyBuddyRequest         0000000039a736b0 f   GameSpy_2.11.00_VC10:gp.obj
 0001:00072770       gpGetBuddyStatus           0000000039a73770 f   GameSpy_2.11.00_VC10:gp.obj
 0001:000728d0       gpGetBuddyIndex            0000000039a738d0 f   GameSpy_2.11.00_VC10:gp.obj
 0001:000729c0       gpIsBuddy                  0000000039a739c0 f   GameSpy_2.11.00_VC10:gp.obj
 0001:00072a40       gpDeleteBuddy              0000000039a73a40 f   GameSpy_2.11.00_VC10:gp.obj
 0001:00072a90       gpAddToBlockedList         0000000039a73a90 f   GameSpy_2.11.00_VC10:gp.obj
 0001:00072ae0       gpRemoveFromBlockedList    0000000039a73ae0 f   GameSpy_2.11.00_VC10:gp.obj
 0001:00072b30       gpIsBlocked                0000000039a73b30 f   GameSpy_2.11.00_VC10:gp.obj
 0001:00072b80       gpSetStatusA               0000000039a73b80 f   GameSpy_2.11.00_VC10:gp.obj
 0001:00072e10       gpSendBuddyMessageA        0000000039a73e10 f   GameSpy_2.11.00_VC10:gp.obj
 0001:00072e90       gpInvitePlayerA            0000000039a73e90 f   GameSpy_2.11.00_VC10:gp.obj
 0001:00072fe0       gpGetReverseBuddies        0000000039a73fe0 f   GameSpy_2.11.00_VC10:gp.obj
 0001:00073060       gpRevokeBuddyAuthorization 0000000039a74060 f   GameSpy_2.11.00_VC10:gp.obj
 0001:000730b0       gpGetLoginTicket           0000000039a740b0 f   GameSpy_2.11.00_VC10:gp.obj
 0001:000731a0       wsLoginCertIsValid         0000000039a741a0 f   GameSpy_2.11.00_VC10:AuthService.obj
 0001:000733c0       wsLoginCertWriteXML        0000000039a743c0 f   GameSpy_2.11.00_VC10:AuthService.obj
 0001:000735b0       wsLoginCertReadXML         0000000039a745b0 f   GameSpy_2.11.00_VC10:AuthService.obj
 0001:000739a0       wsLoginUnique              0000000039a749a0 f   GameSpy_2.11.00_VC10:AuthService.obj
 0001:00073c90       SBServerFree               0000000039a74c90 f   GameSpy_2.11.00_VC10:sb_server.obj
 0001:00073cc0       SBServerAddKeyValue        0000000039a74cc0 f   GameSpy_2.11.00_VC10:sb_server.obj
 0001:00073d10       SBServerAddIntKeyValue     0000000039a74d10 f   GameSpy_2.11.00_VC10:sb_server.obj
 0001:00073d90       SBServerGetStringValueA    0000000039a74d90 f   GameSpy_2.11.00_VC10:sb_server.obj
 0001:00073df0       SBServerGetFloatValueA     0000000039a74df0 f   GameSpy_2.11.00_VC10:sb_server.obj
 0001:00073e70       SBServerGetBoolValueA      0000000039a74e70 f   GameSpy_2.11.00_VC10:sb_server.obj
 0001:00073f00       SBServerHasFullKeys        0000000039a74f00 f   GameSpy_2.11.00_VC10:sb_server.obj
 0001:00073f10       SBServerHasValidPing       0000000039a74f10 f   GameSpy_2.11.00_VC10:sb_server.obj
 0001:00073f20       gt2GetRemoteIP             0000000039a74f20 f   GameSpy_2.11.00_VC10:gt2Main.obj
 0001:00073f20       SBServerGetPublicInetAddress 0000000039a74f20 f   GameSpy_2.11.00_VC10:sb_server.obj
 0001:00073f20       ArrayLength                0000000039a74f20 f   GameSpy_2.11.00_VC10:darray.obj
 0001:00073f30       SBServerGetPublicQueryPort 0000000039a74f30 f   GameSpy_2.11.00_VC10:sb_server.obj
 0001:00073f40       gt2GetRemotePort           0000000039a74f40 f   GameSpy_2.11.00_VC10:gt2Main.obj
 0001:00073f40       SBServerGetPublicQueryPortNBO 0000000039a74f40 f   GameSpy_2.11.00_VC10:sb_server.obj
 0001:00073f50       SBServerHasPrivateAddress  0000000039a74f50 f   GameSpy_2.11.00_VC10:sb_server.obj
 0001:00073f60       SBServerDirectConnect      0000000039a74f60 f   GameSpy_2.11.00_VC10:sb_server.obj
 0001:00073f70       SBServerGetPrivateInetAddress 0000000039a74f70 f   GameSpy_2.11.00_VC10:sb_server.obj
 0001:00073f70       gsXmlWriterGetDataLength   0000000039a74f70 f   GameSpy_2.11.00_VC10:gsXML.obj
 0001:00073f70       gt2GetLocalIP              0000000039a74f70 f   GameSpy_2.11.00_VC10:gt2Main.obj
 0001:00073f80       SBServerGetPrivateQueryPort 0000000039a74f80 f   GameSpy_2.11.00_VC10:sb_server.obj
 0001:00073f90       SBServerSetNext            0000000039a74f90 f   GameSpy_2.11.00_VC10:sb_server.obj
 0001:00073fa0       SBServerGetNext            0000000039a74fa0 f   GameSpy_2.11.00_VC10:sb_server.obj
 0001:00073fb0       SBServerParseKeyVals       0000000039a74fb0 f   GameSpy_2.11.00_VC10:sb_server.obj
 0001:00074150       SBServerParseQR2FullKeysSingle 0000000039a75150 f   GameSpy_2.11.00_VC10:sb_server.obj
 0001:00074380       SBServerParseQR2FullKeysSplit 0000000039a75380 f   GameSpy_2.11.00_VC10:sb_server.obj
 0001:00074630       SBAllocServer              0000000039a75630 f   GameSpy_2.11.00_VC10:sb_server.obj
 0001:000746e0       SBServerSetFlags           0000000039a756e0 f   GameSpy_2.11.00_VC10:sb_server.obj
 0001:000746f0       SBServerSetPrivateAddr     0000000039a756f0 f   GameSpy_2.11.00_VC10:sb_server.obj
 0001:00074700       SBServerSetICMPIP          0000000039a75700 f   GameSpy_2.11.00_VC10:sb_server.obj
 0001:00074710       SBServerSetState           0000000039a75710 f   GameSpy_2.11.00_VC10:sb_server.obj
 0001:00074720       SBServerGetState           0000000039a75720 f   GameSpy_2.11.00_VC10:sb_server.obj
 0001:00074730       SBIsNullServer             0000000039a75730 f   GameSpy_2.11.00_VC10:sb_server.obj
 0001:000747a0       SBRefStrHash               0000000039a757a0 f   GameSpy_2.11.00_VC10:sb_server.obj
 0001:000747f0       SBServerGetIntValueA       0000000039a757f0 f   GameSpy_2.11.00_VC10:sb_server.obj
 0001:000748c0       qr2_internal_is_master_only_key 0000000039a758c0 f   GameSpy_2.11.00_VC10:qr2regkeys.obj
 0001:00074920       qr2_register_keyA          0000000039a75920 f   GameSpy_2.11.00_VC10:qr2regkeys.obj
 0001:00074940       gvStartup                  0000000039a75940 f   GameSpy_2.11.00_VC10:gvMain.obj
 0001:00074980       gvCleanup                  0000000039a75980 f   GameSpy_2.11.00_VC10:gvMain.obj
 0001:000749a0       gvThink                    0000000039a759a0 f   GameSpy_2.11.00_VC10:gvMain.obj
 0001:000749b0       gvSetCustomCodec           0000000039a759b0 f   GameSpy_2.11.00_VC10:gvMain.obj
 0001:000749c0       gvListDevices              0000000039a759c0 f   GameSpy_2.11.00_VC10:gvMain.obj
 0001:000749d0       gvNewDevice                0000000039a759d0 f   GameSpy_2.11.00_VC10:gvMain.obj
 0001:000749f0       gvFreeDevice               0000000039a759f0 f   GameSpy_2.11.00_VC10:gvMain.obj
 0001:00074a00       gvStartDevice              0000000039a75a00 f   GameSpy_2.11.00_VC10:gvMain.obj
 0001:00074a10       gvStopDevice               0000000039a75a10 f   GameSpy_2.11.00_VC10:gvMain.obj
 0001:00074a20       gvSetDeviceVolume          0000000039a75a20 f   GameSpy_2.11.00_VC10:gvMain.obj
 0001:00074a50       gvCapturePacket            0000000039a75a50 f   GameSpy_2.11.00_VC10:gvMain.obj
 0001:00074a70       gvGetAvailableCaptureBytes 0000000039a75a70 f   GameSpy_2.11.00_VC10:gvMain.obj
 0001:00074a80       gvPlayPacket               0000000039a75a80 f   GameSpy_2.11.00_VC10:gvMain.obj
 0001:00074ab0       gsiStringToInt64           0000000039a75ab0 f   GameSpy_2.11.00_VC10:gsPlatformUtil.obj
 0001:00074ac0       gsiInt64ToString           0000000039a75ac0 f   GameSpy_2.11.00_VC10:gsPlatformUtil.obj
 0001:00074ae0       gsiCancelResolvingHostname 0000000039a75ae0 f   GameSpy_2.11.00_VC10:gsPlatformUtil.obj
 0001:00074b20       gsiGetResolvedIP           0000000039a75b20 f   GameSpy_2.11.00_VC10:gsPlatformUtil.obj
 0001:00074b70       goastrdup                  0000000039a75b70 f   GameSpy_2.11.00_VC10:gsPlatformUtil.obj
 0001:00074bd0       goawstrdup                 0000000039a75bd0 f   GameSpy_2.11.00_VC10:gsPlatformUtil.obj
 0001:00074c30       SocketStartUp              0000000039a75c30 f   GameSpy_2.11.00_VC10:gsPlatformUtil.obj
 0001:00074c70       SocketShutDown             0000000039a75c70 f   GameSpy_2.11.00_VC10:gsPlatformUtil.obj
 0001:00074c80       current_time               0000000039a75c80 f   GameSpy_2.11.00_VC10:gsPlatformUtil.obj
 0001:00074c90       current_time_hires         0000000039a75c90 f   GameSpy_2.11.00_VC10:gsPlatformUtil.obj
 0001:00074d10       msleep                     0000000039a75d10 f   GameSpy_2.11.00_VC10:gsPlatformUtil.obj
 0001:00074d20       gsiSecondsToDate           0000000039a75d20 f   GameSpy_2.11.00_VC10:gsPlatformUtil.obj
 0001:00074d30       gsiDateToSeconds           0000000039a75d30 f   GameSpy_2.11.00_VC10:gsPlatformUtil.obj
 0001:00074d40       Util_RandSeed              0000000039a75d40 f   GameSpy_2.11.00_VC10:gsPlatformUtil.obj
 0001:00074d60       Util_RandInt               0000000039a75d60 f   GameSpy_2.11.00_VC10:gsPlatformUtil.obj
 0001:00074e60       B64Decode                  0000000039a75e60 f   GameSpy_2.11.00_VC10:gsPlatformUtil.obj
 0001:000750d0       B64Encode                  0000000039a760d0 f   GameSpy_2.11.00_VC10:gsPlatformUtil.obj
 0001:00075260       B64DecodeLen               0000000039a76260 f   GameSpy_2.11.00_VC10:gsPlatformUtil.obj
 0001:000752f0       B64InitEncodeStream        0000000039a762f0 f   GameSpy_2.11.00_VC10:gsPlatformUtil.obj
 0001:00075300       B64EncodeStream            0000000039a76300 f   GameSpy_2.11.00_VC10:gsPlatformUtil.obj
 0001:00075580       GOAGetUniqueID_Internal    0000000039a76580 f   GameSpy_2.11.00_VC10:gsPlatformUtil.obj
 0001:00075720       gsifopen                   0000000039a76720 f   GameSpy_2.11.00_VC10:gsPlatformUtil.obj
 0001:00075730       gsiResolveHostnameThread   0000000039a76730 f   GameSpy_2.11.00_VC10:gsPlatformUtil.obj
 0001:000757b0       gsiStartResolvingHostname  0000000039a767b0 f   GameSpy_2.11.00_VC10:gsPlatformUtil.obj
 0001:000758a0       ArrayNew                   0000000039a768a0 f   GameSpy_2.11.00_VC10:darray.obj
 0001:00075920       ArrayNth                   0000000039a76920 f   GameSpy_2.11.00_VC10:darray.obj
 0001:00075940       ArrayRemoveAt              0000000039a76940 f   GameSpy_2.11.00_VC10:darray.obj
 0001:000759c0       ArrayMapBackwards          0000000039a769c0 f   GameSpy_2.11.00_VC10:darray.obj
 0001:00075a20       ArrayMapBackwards2         0000000039a76a20 f   GameSpy_2.11.00_VC10:darray.obj
 0001:00075bd0       ArrayFree                  0000000039a76bd0 f   GameSpy_2.11.00_VC10:darray.obj
 0001:00075c30       ArrayInsertAt              0000000039a76c30 f   GameSpy_2.11.00_VC10:darray.obj
 0001:00075d10       ArrayInsertSorted          0000000039a76d10 f   GameSpy_2.11.00_VC10:darray.obj
 0001:00075dc0       ArrayDeleteAt              0000000039a76dc0 f   GameSpy_2.11.00_VC10:darray.obj
 0001:00075e60       ArrayReplaceAt             0000000039a76e60 f   GameSpy_2.11.00_VC10:darray.obj
 0001:00075ee0       ArraySearch                0000000039a76ee0 f   GameSpy_2.11.00_VC10:darray.obj
 0001:00075fc0       ArrayClear                 0000000039a76fc0 f   GameSpy_2.11.00_VC10:darray.obj
 0001:00076070       ArrayAppend                0000000039a77070 f   GameSpy_2.11.00_VC10:darray.obj
 0001:00076090       SetSockBlocking            0000000039a77090 f   GameSpy_2.11.00_VC10:gsPlatformSocket.obj
 0001:000760c0       SetReceiveBufferSize       0000000039a770c0 f   GameSpy_2.11.00_VC10:gsPlatformSocket.obj
 0001:00076100       GSISocketSelect            0000000039a77100 f   GameSpy_2.11.00_VC10:gsPlatformSocket.obj
 0001:00076260       CanReceiveOnSocket         0000000039a77260 f   GameSpy_2.11.00_VC10:gsPlatformSocket.obj
 0001:00076290       CanSendOnSocket            0000000039a77290 f   GameSpy_2.11.00_VC10:gsPlatformSocket.obj
 0001:000762c0       getlocalhost               0000000039a772c0 f   GameSpy_2.11.00_VC10:gsPlatformSocket.obj
 0001:00076330       IsPrivateIP                0000000039a77330 f   GameSpy_2.11.00_VC10:gsPlatformSocket.obj
 0001:00076380       AddressToString            0000000039a77380 f   GameSpy_2.11.00_VC10:NATify.obj
 0001:000764e0       DiscoverReachability       0000000039a774e0 f   GameSpy_2.11.00_VC10:NATify.obj
 0001:000765c0       DiscoverMapping            0000000039a775c0 f   GameSpy_2.11.00_VC10:NATify.obj
 0001:000769f0       NatifyThink                0000000039a779f0 f   GameSpy_2.11.00_VC10:NATify.obj
 0001:00076a00       DetermineNatType           0000000039a77a00 f   GameSpy_2.11.00_VC10:NATify.obj
 0001:00076cb0       UCS2CharToUTF8String       0000000039a77cb0 f   GameSpy_2.11.00_VC10:gsStringUtil.obj
 0001:00076d10       _UTF8ToUCS2ConversionLengthOnly 0000000039a77d10 f   GameSpy_2.11.00_VC10:gsStringUtil.obj
 0001:00076d90       UTF8ToUCS2StringLen2       0000000039a77d90 f   GameSpy_2.11.00_VC10:gsStringUtil.obj
 0001:00076f10       gsiSafeStrcpyA             0000000039a77f10 f   GameSpy_2.11.00_VC10:gsStringUtil.obj
 0001:00076f60       gsiSafeStrcatA             0000000039a77f60 f   GameSpy_2.11.00_VC10:gsStringUtil.obj
 0001:00076fe0       UTF8ToUCS2StringAllocLen   0000000039a77fe0 f   GameSpy_2.11.00_VC10:gsStringUtil.obj
 0001:00077050       UTF8ToUCS2StringAlloc      0000000039a78050 f   GameSpy_2.11.00_VC10:gsStringUtil.obj
 0001:00077280       ghttpStartup               0000000039a78280 f   GameSpy_2.11.00_VC10:ghttpMain.obj
 0001:000772d0       ghttpCleanup               0000000039a782d0 f   GameSpy_2.11.00_VC10:ghttpMain.obj
 0001:00077320       ghttpGetExA                0000000039a78320 f   GameSpy_2.11.00_VC10:ghttpMain.obj
 0001:00077690       ghttpSaveExA               0000000039a78690 f   GameSpy_2.11.00_VC10:ghttpMain.obj
 0001:000776e0       ghttpRequestThink          0000000039a786e0 f   GameSpy_2.11.00_VC10:ghttpMain.obj
 0001:00077710       ghttpCancelRequest         0000000039a78710 f   GameSpy_2.11.00_VC10:ghttpMain.obj
 0001:00077730       ghttpCloseRequest          0000000039a78730 f   GameSpy_2.11.00_VC10:ghttpMain.obj
 0001:00077770       ghttpNewPost               0000000039a78770 f   GameSpy_2.11.00_VC10:ghttpMain.obj
 0001:00077780       ghttpPostSetAutoFree       0000000039a78780 f   GameSpy_2.11.00_VC10:ghttpMain.obj
 0001:000777a0       ghttpFreePost              0000000039a787a0 f   GameSpy_2.11.00_VC10:ghttpMain.obj
 0001:000777c0       ghttpPostAddXml            0000000039a787c0 f   GameSpy_2.11.00_VC10:ghttpMain.obj
 0001:000777d0       ghttpGetA                  0000000039a787d0 f   GameSpy_2.11.00_VC10:ghttpMain.obj
 0001:00077900       gsiInitializeCriticalSection 0000000039a78900 f   GameSpy_2.11.00_VC10:gsPlatformThread.obj
 0001:00077900       ?CryCreateCriticalSectionInplace@@YAXPEAX@Z 0000000039a78900 f   CryLobbyDLL.obj
 0001:00077910       gsiStartThread             0000000039a78910 f   GameSpy_2.11.00_VC10:gsPlatformThread.obj
 0001:00077960       gsiCancelThread            0000000039a78960 f   GameSpy_2.11.00_VC10:gsPlatformThread.obj
 0001:00077970       gsiCleanupThread           0000000039a78970 f   GameSpy_2.11.00_VC10:gsPlatformThread.obj
 0001:00077980       sakeiInitRequest           0000000039a78980 f   GameSpy_2.11.00_VC10:sakeRequest.obj
 0001:00077f60       sakeiStartRequest          0000000039a78f60 f   GameSpy_2.11.00_VC10:sakeRequest.obj
 0001:000784d0       sakeiStartCreateRecordRequest 0000000039a794d0 f   GameSpy_2.11.00_VC10:sakeRequestModify.obj
 0001:00078580       sakeiStartUpdateRecordRequest 0000000039a79580 f   GameSpy_2.11.00_VC10:sakeRequestModify.obj
 0001:00078f90       sakeiStartSearchForRecordsRequest 0000000039a79f90 f   GameSpy_2.11.00_VC10:sakeRequestRead.obj
 0001:00079020       sakeiStartGetMyRecordsRequest 0000000039a7a020 f   GameSpy_2.11.00_VC10:sakeRequestRead.obj
 0001:00079590       sakeiStartGetRecordCountRequest 0000000039a7a590 f   GameSpy_2.11.00_VC10:sakeRequestMisc.obj
 0001:000795a0       d2giResultFromStoreAvailabilityCode 0000000039a7a5a0 f   GameSpy_2.11.00_VC10:d2gUtil.obj
 0001:000795f0       d2giSetServiceUrl          0000000039a7a5f0 f   GameSpy_2.11.00_VC10:d2gUtil.obj
 0001:000796b0       d2giResultFromStatusCode   0000000039a7a6b0 f   GameSpy_2.11.00_VC10:d2gUtil.obj
 0001:00079850       d2giResultFromHttpResult   0000000039a7a850 f   GameSpy_2.11.00_VC10:d2gUtil.obj
 0001:000798f0       d2giResultFromHttpRequest  0000000039a7a8f0 f   GameSpy_2.11.00_VC10:d2gUtil.obj
 0001:00079970       d2giOrderValidationResultFromCode 0000000039a7a970 f   GameSpy_2.11.00_VC10:d2gUtil.obj
 0001:00079aa0       d2giResultFromDownloadStatusCode 0000000039a7aaa0 f   GameSpy_2.11.00_VC10:d2gUtil.obj
 0001:00079ae0       d2giWriteOrderTotalToXml   0000000039a7aae0 f   GameSpy_2.11.00_VC10:d2gUtil.obj
 0001:00079e10       d2giNewCatalogItem         0000000039a7ae10 f   GameSpy_2.11.00_VC10:d2gUtil.obj
 0001:00079e90       d2giGetCatalogItem         0000000039a7ae90 f   GameSpy_2.11.00_VC10:d2gUtil.obj
 0001:00079ef0       d2giResetCatalogItem       0000000039a7aef0 f   GameSpy_2.11.00_VC10:d2gUtil.obj
 0001:0007a070       d2giFreeCatalogItems       0000000039a7b070 f   GameSpy_2.11.00_VC10:d2gUtil.obj
 0001:0007a180       d2giFreeCreditCardInfoList 0000000039a7b180 f   GameSpy_2.11.00_VC10:d2gUtil.obj
 0001:0007a1f0       d2giFreeOrder              0000000039a7b1f0 f   GameSpy_2.11.00_VC10:d2gUtil.obj
 0001:0007a270       d2giFreeOrderItem          0000000039a7b270 f   GameSpy_2.11.00_VC10:d2gUtil.obj
 0001:0007a300       d2giFreeOrderItemPurchases 0000000039a7b300 f   GameSpy_2.11.00_VC10:d2gUtil.obj
 0001:0007a470       d2giFreeOrderTotal         0000000039a7b470 f   GameSpy_2.11.00_VC10:d2gUtil.obj
 0001:0007a4f0       d2giFreeOrderPurchase      0000000039a7b4f0 f   GameSpy_2.11.00_VC10:d2gUtil.obj
 0001:0007a530       d2giFreePurchaseHistory    0000000039a7b530 f   GameSpy_2.11.00_VC10:d2gUtil.obj
 0001:0007a5d0       d2giGetAllItemsFromCache   0000000039a7b5d0 f   GameSpy_2.11.00_VC10:d2gUtil.obj
 0001:0007a720       d2giGetCategoriesFromCache 0000000039a7b720 f   GameSpy_2.11.00_VC10:d2gUtil.obj
 0001:0007a8c0       d2giCheckItemsQuantities   0000000039a7b8c0 f   GameSpy_2.11.00_VC10:d2gUtil.obj
 0001:0007a8e0       d2giNewExtraInfo           0000000039a7b8e0 f   GameSpy_2.11.00_VC10:d2gUtil.obj
 0001:0007a930       d2giGetExtraInfo           0000000039a7b930 f   GameSpy_2.11.00_VC10:d2gUtil.obj
 0001:0007a9b0       d2giResetExtraInfo         0000000039a7b9b0 f   GameSpy_2.11.00_VC10:d2gUtil.obj
 0001:0007a9f0       d2giCreateManifestXmlStr   0000000039a7b9f0 f   GameSpy_2.11.00_VC10:d2gUtil.obj
 0001:0007ab20       d2giWriteCachedItemsToXml  0000000039a7bb20 f   GameSpy_2.11.00_VC10:d2gUtil.obj
 0001:0007ae90       d2giUpdateManifestRecord   0000000039a7be90 f   GameSpy_2.11.00_VC10:d2gUtil.obj
 0001:0007b340       d2giServiceGetStoreAvail   0000000039a7c340 f   GameSpy_2.11.00_VC10:d2gServices.obj
 0001:0007b5c0       d2giServiceLoadCatalogItems 0000000039a7c5c0 f   GameSpy_2.11.00_VC10:d2gServices.obj
 0001:0007b830       d2giServiceGetUserCreditCards 0000000039a7c830 f   GameSpy_2.11.00_VC10:d2gServices.obj
 0001:0007bae0       d2giServiceGetOrderTotal   0000000039a7cae0 f   GameSpy_2.11.00_VC10:d2gServices.obj
 0001:0007bd80       d2giServicePurchaseItemsCallback 0000000039a7cd80 f   GameSpy_2.11.00_VC10:d2gServices.obj
 0001:0007bde0       d2giServicePurchaseItems   0000000039a7cde0 f   GameSpy_2.11.00_VC10:d2gServices.obj
 0001:0007c010       d2giServiceIsOrderCompleteCallback 0000000039a7d010 f   GameSpy_2.11.00_VC10:d2gServices.obj
 0001:0007c070       d2giServiceIsOrderComplete 0000000039a7d070 f   GameSpy_2.11.00_VC10:d2gServices.obj
 0001:0007c430       d2giServiceGetDownloadInfo 0000000039a7d430 f   GameSpy_2.11.00_VC10:d2gServices.obj
 0001:0007c740       d2giServiceGetPurchaseHistory 0000000039a7d740 f   GameSpy_2.11.00_VC10:d2gServices.obj
 0001:0007c970       d2giCancelDownload         0000000039a7d970 f   GameSpy_2.11.00_VC10:d2gServices.obj
 0001:0007c980       GSMD5Init                  0000000039a7d980 f   GameSpy_2.11.00_VC10:md5c.obj
 0001:0007c9b0       GSMD5Print                 0000000039a7d9b0 f   GameSpy_2.11.00_VC10:md5c.obj
 0001:0007d300       GSMD5Update                0000000039a7e300 f   GameSpy_2.11.00_VC10:md5c.obj
 0001:0007d3d0       GSMD5Final                 0000000039a7e3d0 f   GameSpy_2.11.00_VC10:md5c.obj
 0001:0007d4f0       GSMD5Digest                0000000039a7e4f0 f   GameSpy_2.11.00_VC10:md5c.obj
 0001:0007d8a0       SBQueryEngineInit          0000000039a7e8a0 f   GameSpy_2.11.00_VC10:sb_queryengine.obj
 0001:0007d940       SBQueryEngineSetPublicIP   0000000039a7e940 f   GameSpy_2.11.00_VC10:sb_queryengine.obj
 0001:0007d950       SBEngineHaltUpdates        0000000039a7e950 f   GameSpy_2.11.00_VC10:sb_queryengine.obj
 0001:0007d970       SBQueryEngineUpdateServer  0000000039a7e970 f   GameSpy_2.11.00_VC10:sb_queryengine.obj
 0001:0007dd90       SBQueryEngineThink         0000000039a7ed90 f   GameSpy_2.11.00_VC10:sb_queryengine.obj
 0001:0007e060       SBQueryEngineAddQueryKey   0000000039a7f060 f   GameSpy_2.11.00_VC10:sb_queryengine.obj
 0001:0007e080       SBQueryEngineRemoveServerFromFIFOs 0000000039a7f080 f   GameSpy_2.11.00_VC10:sb_queryengine.obj
 0001:0007e130       SBServerListAppendServer   0000000039a7f130 f   GameSpy_2.11.00_VC10:sb_serverlist.obj
 0001:0007e170       SBServerListFindServerByIP 0000000039a7f170 f   GameSpy_2.11.00_VC10:sb_serverlist.obj
 0001:0007e200       SBServerListRemoveAt       0000000039a7f200 f   GameSpy_2.11.00_VC10:sb_serverlist.obj
 0001:0007e270       SBServerListClear          0000000039a7f270 f   GameSpy_2.11.00_VC10:sb_serverlist.obj
 0001:0007e330       SBRefStr                   0000000039a7f330 f   GameSpy_2.11.00_VC10:sb_serverlist.obj
 0001:0007e3b0       SBReleaseStr               0000000039a7f3b0 f   GameSpy_2.11.00_VC10:sb_serverlist.obj
 0001:0007e400       NTSLengthSB                0000000039a7f400 f   GameSpy_2.11.00_VC10:sb_serverlist.obj
 0001:0007e820       SBServerListDisconnect     0000000039a7f820 f   GameSpy_2.11.00_VC10:sb_serverlist.obj
 0001:0007f960       SBServerListInit           0000000039a80960 f   GameSpy_2.11.00_VC10:sb_serverlist.obj
 0001:0007fb80       SBServerListConnectAndQuery 0000000039a80b80 f   GameSpy_2.11.00_VC10:sb_serverlist.obj
 0001:00080100       SBListThink                0000000039a81100 f   GameSpy_2.11.00_VC10:sb_serverlist.obj
 0001:000802a0       SBGetServerRulesFromMaster 0000000039a812a0 f   GameSpy_2.11.00_VC10:sb_serverlist.obj
 0001:00080330       SBSendMessageToServer      0000000039a81330 f   GameSpy_2.11.00_VC10:sb_serverlist.obj
 0001:00080400       SBSendNatNegotiateCookieToServer 0000000039a81400 f   GameSpy_2.11.00_VC10:sb_serverlist.obj
 0001:00080470       gpiDestroy                 0000000039a81470 f   GameSpy_2.11.00_VC10:gpi.obj
 0001:000804f0       gpiReset                   0000000039a814f0 f   GameSpy_2.11.00_VC10:gpi.obj
 0001:000807c0       gpiProcessConnectionManager 0000000039a817c0 f   GameSpy_2.11.00_VC10:gpi.obj
 0001:00080c40       gpiProcess                 0000000039a81c40 f   GameSpy_2.11.00_VC10:gpi.obj
 0001:00080d80       gpiInitialize              0000000039a81d80 f   GameSpy_2.11.00_VC10:gpi.obj
 0001:00080fa0       strzcpy                    0000000039a81fa0 f   GameSpy_2.11.00_VC10:gpiUtility.obj
 0001:00080fd0       gpiValueForKeyWithIndex    0000000039a81fd0 f   GameSpy_2.11.00_VC10:gpiUtility.obj
 0001:000810a0       gpiValueForKey             0000000039a820a0 f   GameSpy_2.11.00_VC10:gpiUtility.obj
 0001:00081140       gpiSetError                0000000039a82140 f   GameSpy_2.11.00_VC10:gpiUtility.obj
 0001:00081180       gpiSetErrorString          0000000039a82180 f   GameSpy_2.11.00_VC10:gpiUtility.obj
 0001:000811b0       gpiEncodeString            0000000039a821b0 f   GameSpy_2.11.00_VC10:gpiUtility.obj
 0001:00081260       gpiCheckForError           0000000039a82260 f   GameSpy_2.11.00_VC10:gpiUtility.obj
 0001:000813a0       gpiCheckSocketConnect      0000000039a823a0 f   GameSpy_2.11.00_VC10:gpiUtility.obj
 0001:00081480       gpiReadKeyAndValue         0000000039a82480 f   GameSpy_2.11.00_VC10:gpiUtility.obj
 0001:00082140       gpiProcessConnect          0000000039a83140 f   GameSpy_2.11.00_VC10:gpiConnect.obj
 0001:000826c0       gpiCheckConnect            0000000039a836c0 f   GameSpy_2.11.00_VC10:gpiConnect.obj
 0001:00082890       gpiDisconnect              0000000039a83890 f   GameSpy_2.11.00_VC10:gpiConnect.obj
 0001:00082aa0       gpiProcessRemoteAuthResponse 0000000039a83aa0 f   GameSpy_2.11.00_VC10:gpiConnect.obj
 0001:00082ba0       gpiConnect                 0000000039a83ba0 f   GameSpy_2.11.00_VC10:gpiConnect.obj
 0001:000830e0       gpiProfileSearch           0000000039a840e0 f   GameSpy_2.11.00_VC10:gpiSearch.obj
 0001:00083300       gpiProfileSearchUniquenick 0000000039a84300 f   GameSpy_2.11.00_VC10:gpiSearch.obj
 0001:000833f0       gpiCheckUser               0000000039a843f0 f   GameSpy_2.11.00_VC10:gpiSearch.obj
 0001:00083520       gpiNewUser                 0000000039a84520 f   GameSpy_2.11.00_VC10:gpiSearch.obj
 0001:00083670       gpiOthersBuddy             0000000039a84670 f   GameSpy_2.11.00_VC10:gpiSearch.obj
 0001:000855f0       gpiProcessSearches         0000000039a865f0 f   GameSpy_2.11.00_VC10:gpiSearch.obj
 0001:00085870       gpiRegisterUniqueNick      0000000039a86870 f   GameSpy_2.11.00_VC10:gpiUnique.obj
 0001:00085920       gpiProcessRegisterUniqueNick 0000000039a86920 f   GameSpy_2.11.00_VC10:gpiUnique.obj
 0001:00085a40       gpiProcessRegisterCdKey    0000000039a86a40 f   GameSpy_2.11.00_VC10:gpiUnique.obj
 0001:00085c80       gpiInitProfiles            0000000039a86c80 f   GameSpy_2.11.00_VC10:gpiProfile.obj
 0001:00085ce0       gpiProcessNewProfile       0000000039a86ce0 f   GameSpy_2.11.00_VC10:gpiProfile.obj
 0001:00085e20       gpiGetProfile              0000000039a86e20 f   GameSpy_2.11.00_VC10:gpiProfile.obj
 0001:00085e60       gpiNewProfile              0000000039a86e60 f   GameSpy_2.11.00_VC10:gpiProfile.obj
 0001:00086080       gpiProcessDeleteProfle     0000000039a87080 f   GameSpy_2.11.00_VC10:gpiProfile.obj
 0001:000861a0       gpiRemoveProfileByID       0000000039a871a0 f   GameSpy_2.11.00_VC10:gpiProfile.obj
 0001:000861e0       gpiRemoveProfile           0000000039a871e0 f   GameSpy_2.11.00_VC10:gpiProfile.obj
 0001:000862a0       gpiProfileMap              0000000039a872a0 f   GameSpy_2.11.00_VC10:gpiProfile.obj
 0001:00086310       gpiFindBuddy               0000000039a87310 f   GameSpy_2.11.00_VC10:gpiProfile.obj
 0001:00086370       gpiRemoveBuddyStatus       0000000039a87370 f   GameSpy_2.11.00_VC10:gpiProfile.obj
 0001:000863b0       gpiRemoveBuddyStatusInfo   0000000039a873b0 f   GameSpy_2.11.00_VC10:gpiProfile.obj
 0001:00086420       gpiCanFreeProfile          0000000039a87420 f   GameSpy_2.11.00_VC10:gpiProfile.obj
 0001:00086480       gpiRemoveFromBlockedList   0000000039a87480 f   GameSpy_2.11.00_VC10:gpiProfile.obj
 0001:00086590       gpiProfileListAdd          0000000039a87590 f   GameSpy_2.11.00_VC10:gpiProfile.obj
 0001:00086660       gpiFindProfileByUser       0000000039a87660 f   GameSpy_2.11.00_VC10:gpiProfile.obj
 0001:000866d0       gpiAddToBlockedList        0000000039a876d0 f   GameSpy_2.11.00_VC10:gpiProfile.obj
 0001:00086940       gpiProcessRecvBlockedList  0000000039a87940 f   GameSpy_2.11.00_VC10:gpiProfile.obj
 0001:00086cc0       gpiInfoCacheToArg          0000000039a87cc0 f   GameSpy_2.11.00_VC10:gpiInfo.obj
 0001:00086f30       gpiAddLocalInfo            0000000039a87f30 f   GameSpy_2.11.00_VC10:gpiInfo.obj
 0001:00087030       gpiSendGetInfo             0000000039a88030 f   GameSpy_2.11.00_VC10:gpiInfo.obj
 0001:00087110       gpiGetInfo                 0000000039a88110 f   GameSpy_2.11.00_VC10:gpiInfo.obj
 0001:000872d0       gpiFreeInfoCache           0000000039a882d0 f   GameSpy_2.11.00_VC10:gpiInfo.obj
 0001:000873a0       gpiSetInfoCache            0000000039a883a0 f   GameSpy_2.11.00_VC10:gpiInfo.obj
 0001:00087490       gpiProcessGetInfo          0000000039a88490 f   GameSpy_2.11.00_VC10:gpiInfo.obj
 0001:00087c60       gpiSendAuthBuddyRequest    0000000039a88c60 f   GameSpy_2.11.00_VC10:gpiBuddy.obj
 0001:00087d90       gpiSendAddBuddyRequest     0000000039a88d90 f   GameSpy_2.11.00_VC10:gpiBuddy.obj
 0001:00087f40       gpiProcessRecvBuddyStatusInfo 0000000039a88f40 f   GameSpy_2.11.00_VC10:gpiBuddy.obj
 0001:00088490       gpiProcessRecvAddBuddyResponse 0000000039a89490 f   GameSpy_2.11.00_VC10:gpiBuddy.obj
 0001:00088620       gpiSendServerBuddyMessage  0000000039a89620 f   GameSpy_2.11.00_VC10:gpiBuddy.obj
 0001:00088740       gpiSendBuddyMessage        0000000039a89740 f   GameSpy_2.11.00_VC10:gpiBuddy.obj
 0001:00088890       gpiBuddyHandleKeyRequest   0000000039a89890 f   GameSpy_2.11.00_VC10:gpiBuddy.obj
 0001:00088a10       gpiBuddyHandleKeyReply     0000000039a89a10 f   GameSpy_2.11.00_VC10:gpiBuddy.obj
 0001:00088e50       gpiAuthBuddyRequest        0000000039a89e50 f   GameSpy_2.11.00_VC10:gpiBuddy.obj
 0001:00088f00       gpiFixBuddyIndices         0000000039a89f00 f   GameSpy_2.11.00_VC10:gpiBuddy.obj
 0001:00088f30       gpiBuddyDeletedLocally     0000000039a89f30 f   GameSpy_2.11.00_VC10:gpiBuddy.obj
 0001:00088f80       gpiRevokeBuddyAuthorization 0000000039a89f80 f   GameSpy_2.11.00_VC10:gpiBuddy.obj
 0001:00089040       gpiProcessRecvBuddyMessage 0000000039a8a040 f   GameSpy_2.11.00_VC10:gpiBuddy.obj
 0001:00089a50       gpiProcessRecvBuddyList    0000000039a8aa50 f   GameSpy_2.11.00_VC10:gpiBuddy.obj
 0001:00089d20       gpiDeleteBuddy             0000000039a8ad20 f   GameSpy_2.11.00_VC10:gpiBuddy.obj
 0001:0008a1c0       gpiPeerSendMessages        0000000039a8b1c0 f   GameSpy_2.11.00_VC10:gpiPeer.obj
 0001:0008a690       gpiDestroyPeer             0000000039a8b690 f   GameSpy_2.11.00_VC10:gpiPeer.obj
 0001:0008a6e0       gpiRemovePeer              0000000039a8b6e0 f   GameSpy_2.11.00_VC10:gpiPeer.obj
 0001:0008a7e0       gpiGetPeerByProfile        0000000039a8b7e0 f   GameSpy_2.11.00_VC10:gpiPeer.obj
 0001:0008a830       gpiAddPeer                 0000000039a8b830 f   GameSpy_2.11.00_VC10:gpiPeer.obj
 0001:0008a8e0       gpiPeerGetSig              0000000039a8b8e0 f   GameSpy_2.11.00_VC10:gpiPeer.obj
 0001:0008a940       gpiPeerStartConnect        0000000039a8b940 f   GameSpy_2.11.00_VC10:gpiPeer.obj
 0001:0008aa50       gpiPeerAddMessage          0000000039a8ba50 f   GameSpy_2.11.00_VC10:gpiPeer.obj
 0001:0008abb0       gpiPeerStartTransferMessage 0000000039a8bbb0 f   GameSpy_2.11.00_VC10:gpiPeer.obj
 0001:0008ac20       gpiPeerFinishTransferMessage 0000000039a8bc20 f   GameSpy_2.11.00_VC10:gpiPeer.obj
 0001:0008ad00       gpiPeerLeftCallback        0000000039a8bd00 f   GameSpy_2.11.00_VC10:gpiPeer.obj
 0001:0008ad50       gpiPeerMessageCallback     0000000039a8bd50 f   GameSpy_2.11.00_VC10:gpiPeer.obj
 0001:0008aea0       gpiPeerAcceptedCallback    0000000039a8bea0 f   GameSpy_2.11.00_VC10:gpiPeer.obj
 0001:0008af00       gpiPeerAddOp               0000000039a8bf00 f   GameSpy_2.11.00_VC10:gpiPeer.obj
 0001:0008af40       gpiPeerRemoveOp            0000000039a8bf40 f   GameSpy_2.11.00_VC10:gpiPeer.obj
 0001:0008b290       gpiCheckTimedOutPeerOperations 0000000039a8c290 f   GameSpy_2.11.00_VC10:gpiPeer.obj
 0001:0008b360       gpiProcessPeers            0000000039a8c360 f   GameSpy_2.11.00_VC10:gpiPeer.obj
 0001:0008b430       gpiAppendCharToBuffer      0000000039a8c430 f   GameSpy_2.11.00_VC10:gpiBuffer.obj
 0001:0008b4c0       gpiAppendStringToBufferLen 0000000039a8c4c0 f   GameSpy_2.11.00_VC10:gpiBuffer.obj
 0001:0008b590       gpiAppendStringToBuffer    0000000039a8c590 f   GameSpy_2.11.00_VC10:gpiBuffer.obj
 0001:0008b5c0       gpiAppendIntToBuffer       0000000039a8c5c0 f   GameSpy_2.11.00_VC10:gpiBuffer.obj
 0001:0008b630       gpiSendOrBufferStringLenToPeer 0000000039a8c630 f   GameSpy_2.11.00_VC10:gpiBuffer.obj
 0001:0008b720       gpiSendOrBufferString      0000000039a8c720 f   GameSpy_2.11.00_VC10:gpiBuffer.obj
 0001:0008b750       gpiRecvToBuffer            0000000039a8c750 f   GameSpy_2.11.00_VC10:gpiBuffer.obj
 0001:0008b890       gpiSendFromBuffer          0000000039a8c890 f   GameSpy_2.11.00_VC10:gpiBuffer.obj
 0001:0008b9d0       gpiSendBufferToPeer        0000000039a8c9d0 f   GameSpy_2.11.00_VC10:gpiBuffer.obj
 0001:0008bb30       gpiReadMessageFromBuffer   0000000039a8cb30 f   GameSpy_2.11.00_VC10:gpiBuffer.obj
 0001:0008bc60       gpiClipBufferToPosition    0000000039a8cc60 f   GameSpy_2.11.00_VC10:gpiBuffer.obj
 0001:0008bcb0       gsXmlCreateStreamWriterNoNamespace 0000000039a8ccb0 f   GameSpy_2.11.00_VC10:gsXML.obj
 0001:0008bd00       gsXmlFreeWriter            0000000039a8cd00 f   GameSpy_2.11.00_VC10:gsXML.obj
 0001:0008bd20       gsXmlFreeReader            0000000039a8cd20 f   GameSpy_2.11.00_VC10:gsXML.obj
 0001:0008bd50       gsXmlCloseWriterNoNamespace 0000000039a8cd50 f   GameSpy_2.11.00_VC10:gsXML.obj
 0001:0008bd60       gsXmlWriterGetData         0000000039a8cd60 f   GameSpy_2.11.00_VC10:gsXML.obj
 0001:0008bd60       ??C?$CGameSpySDKRef@VCGameSpySBQR2Sake@@@@QEAAPEAVCGameSpySBQR2Sake@@XZ 0000000039a8cd60 f   GameSpySBQR2Sake.obj
 0001:0008bd60       ??C?$CGameSpySDKRef@VCGameSpySBQR2NATNegotiation@@@@QEAAPEAVCGameSpySBQR2NATNegotiation@@XZ 0000000039a8cd60 f   GameSpySBQR2NatNegotiation.obj
 0001:0008bd60       ??C?$CGameSpySDKRef@VCGameSpySBQR2GPConnection@@@@QEAAPEAVCGameSpySBQR2GPConnection@@XZ 0000000039a8cd60 f   GameSpySBQR2AvailabilityCheck.obj
 0001:0008c1b0       gsXmlMoveToStart           0000000039a8d1b0 f   GameSpy_2.11.00_VC10:gsXML.obj
 0001:0008c1d0       gsXmlMoveToParent          0000000039a8d1d0 f   GameSpy_2.11.00_VC10:gsXML.obj
 0001:0008c330       gsXmlCountChildren         0000000039a8d330 f   GameSpy_2.11.00_VC10:gsXML.obj
 0001:0008c480       gsXmlCreateStreamReader    0000000039a8d480 f   GameSpy_2.11.00_VC10:gsXML.obj
 0001:0008c840       gsXmlMoveToNext            0000000039a8d840 f   GameSpy_2.11.00_VC10:gsXML.obj
 0001:0008c960       gsXmlMoveToSibling         0000000039a8d960 f   GameSpy_2.11.00_VC10:gsXML.obj
 0001:0008cad0       gsXmlMoveToChild           0000000039a8dad0 f   GameSpy_2.11.00_VC10:gsXML.obj
 0001:0008cc00       gsXmlReadChildAsString     0000000039a8dc00 f   GameSpy_2.11.00_VC10:gsXML.obj
 0001:0008cd60       gsXmlReadChildAsStringNT   0000000039a8dd60 f   GameSpy_2.11.00_VC10:gsXML.obj
 0001:0008cdf0       gsXmlReadChildAsHexBinary  0000000039a8ddf0 f   GameSpy_2.11.00_VC10:gsXML.obj
 0001:0008cf90       gsXmlReadChildAsBase64Binary 0000000039a8df90 f   GameSpy_2.11.00_VC10:gsXML.obj
 0001:0008d130       gsXmlReadChildAsInt        0000000039a8e130 f   GameSpy_2.11.00_VC10:gsXML.obj
 0001:0008d290       gsXmlReadChildAsInt64      0000000039a8e290 f   GameSpy_2.11.00_VC10:gsXML.obj
 0001:0008d3f0       gsXmlReadChildAsDateTimeElement 0000000039a8e3f0 f   GameSpy_2.11.00_VC10:gsXML.obj
 0001:0008d600       gsXmlReadChildAsFloat      0000000039a8e600 f   GameSpy_2.11.00_VC10:gsXML.obj
 0001:0008d770       gsXmlReadChildAsLargeInt   0000000039a8e770 f   GameSpy_2.11.00_VC10:gsXML.obj
 0001:0008d810       gsXmlCreateStreamWriter    0000000039a8e810 f   GameSpy_2.11.00_VC10:gsXML.obj
 0001:0008dc00       gsXmlCloseWriter           0000000039a8ec00 f   GameSpy_2.11.00_VC10:gsXML.obj
 0001:0008e0b0       gsXmlWriteOpenTag          0000000039a8f0b0 f   GameSpy_2.11.00_VC10:gsXML.obj
 0001:0008e140       gsXmlWriteCloseTag         0000000039a8f140 f   GameSpy_2.11.00_VC10:gsXML.obj
 0001:0008e1e0       gsXmlWriteOpenTagNoNamespace 0000000039a8f1e0 f   GameSpy_2.11.00_VC10:gsXML.obj
 0001:0008e240       gsXmlWriteCloseTagNoNamespace 0000000039a8f240 f   GameSpy_2.11.00_VC10:gsXML.obj
 0001:0008e2b0       gsXmlWriteAsciiStringElement 0000000039a8f2b0 f   GameSpy_2.11.00_VC10:gsXML.obj
 0001:0008e2b0       gsXmlWriteStringElement    0000000039a8f2b0 f   GameSpy_2.11.00_VC10:gsXML.obj
 0001:0008e410       gsXmlWriteIntElement       0000000039a8f410 f   GameSpy_2.11.00_VC10:gsXML.obj
 0001:0008e4a0       gsXmlWriteIntElementNoNamespace 0000000039a8f4a0 f   GameSpy_2.11.00_VC10:gsXML.obj
 0001:0008e540       gsXmlWriteInt64Element     0000000039a8f540 f   GameSpy_2.11.00_VC10:gsXML.obj
 0001:0008e5c0       gsXmlWriteFloatElement     0000000039a8f5c0 f   GameSpy_2.11.00_VC10:gsXML.obj
 0001:0008e650       gsXmlWriteFloatElementNoNamespace 0000000039a8f650 f   GameSpy_2.11.00_VC10:gsXML.obj
 0001:0008e700       gsXmlWriteHexBinaryElement 0000000039a8f700 f   GameSpy_2.11.00_VC10:gsXML.obj
 0001:0008e850       gsXmlWriteBase64BinaryElement 0000000039a8f850 f   GameSpy_2.11.00_VC10:gsXML.obj
 0001:0008e990       gsXmlWriteDateTimeElement  0000000039a8f990 f   GameSpy_2.11.00_VC10:gsXML.obj
 0001:0008ea60       gsXmlWriteLargeIntElement  0000000039a8fa60 f   GameSpy_2.11.00_VC10:gsXML.obj
 0001:0008ecd0       gsXmlParseBuffer           0000000039a8fcd0 f   GameSpy_2.11.00_VC10:gsXML.obj
 0001:0008ed70       gsXmlWriteUnicodeStringElement 0000000039a8fd70 f   GameSpy_2.11.00_VC10:gsXML.obj
 0001:0008f100       gsiExecuteSoapWithTimeout  0000000039a90100 f   GameSpy_2.11.00_VC10:gsSoap.obj
 0001:0008f1f0       gsiExecuteSoap             0000000039a901f0 f   GameSpy_2.11.00_VC10:gsSoap.obj
 0001:0008f360       gsCryptRSAVerifySignedHash 0000000039a90360 f   GameSpy_2.11.00_VC10:gsCrypt.obj
 0001:0008f590       gsCryptRSAEncryptBuffer    0000000039a90590 f   GameSpy_2.11.00_VC10:gsCrypt.obj
 0001:0008fc90       gsiLargeIntMultM           0000000039a90c90 f   GameSpy_2.11.00_VC10:gsLargeInt.obj
 0001:0008fee0       gsLargeIntSetFromHexString 0000000039a90ee0 f   GameSpy_2.11.00_VC10:gsLargeInt.obj
 0001:0008ffe0       gsLargeIntReverseBytes     0000000039a90fe0 f   GameSpy_2.11.00_VC10:gsLargeInt.obj
 0001:00090020       gsLargeIntSetFromMemoryStream 0000000039a91020 f   GameSpy_2.11.00_VC10:gsLargeInt.obj
 0001:000900a0       gsLargeIntWriteToMemoryStream 0000000039a910a0 f   GameSpy_2.11.00_VC10:gsLargeInt.obj
 0001:000904e0       gsLargeIntSquareMod        0000000039a914e0 f   GameSpy_2.11.00_VC10:gsLargeInt.obj
 0001:000907f0       gsLargeIntAddToMD5         0000000039a917f0 f   GameSpy_2.11.00_VC10:gsLargeInt.obj
 0001:00090960       gsLargeIntPowerMod         0000000039a91960 f   GameSpy_2.11.00_VC10:gsLargeInt.obj
 0001:00090e50       TableNew2                  0000000039a91e50 f   GameSpy_2.11.00_VC10:hashtable.obj
 0001:00090f00       TableFree                  0000000039a91f00 f   GameSpy_2.11.00_VC10:hashtable.obj
 0001:00090f60       TableEnter                 0000000039a91f60 f   GameSpy_2.11.00_VC10:hashtable.obj
 0001:00090fe0       TableRemove                0000000039a91fe0 f   GameSpy_2.11.00_VC10:hashtable.obj
 0001:00091070       TableLookup                0000000039a92070 f   GameSpy_2.11.00_VC10:hashtable.obj
 0001:00091100       TableMapSafe               0000000039a92100 f   GameSpy_2.11.00_VC10:hashtable.obj
 0001:00091170       TableMapSafe2              0000000039a92170 f   GameSpy_2.11.00_VC10:hashtable.obj
 0001:000911e0       TableNew                   0000000039a921e0 f   GameSpy_2.11.00_VC10:hashtable.obj
 0001:000912a0       gviHardwareStartup         0000000039a922a0 f   GameSpy_2.11.00_VC10:gvDirectSound.obj
 0001:00091310       gviHardwareCleanup         0000000039a92310 f   GameSpy_2.11.00_VC10:gvDirectSound.obj
 0001:00091350       gviHardwareThink           0000000039a92350 f   GameSpy_2.11.00_VC10:gvDirectSound.obj
 0001:00091780       gviHardwareListDevices     0000000039a92780 f   GameSpy_2.11.00_VC10:gvDirectSound.obj
 0001:00092150       gviHardwareNewDevice       0000000039a93150 f   GameSpy_2.11.00_VC10:gvDirectSound.obj
 0001:00092390       gviNewSourceList           0000000039a93390 f   GameSpy_2.11.00_VC10:gvSource.obj
 0001:000923f0       gviClearSourceList         0000000039a933f0 f   GameSpy_2.11.00_VC10:gvSource.obj
 0001:00092460       gviIsSourceTalking         0000000039a93460 f   GameSpy_2.11.00_VC10:gvSource.obj
 0001:00092480       gviListTalkingSources      0000000039a93480 f   GameSpy_2.11.00_VC10:gvSource.obj
 0001:000926b0       gviAddPacketToSourceList   0000000039a936b0 f   GameSpy_2.11.00_VC10:gvSource.obj
 0001:00092890       gviWriteSourcesToBuffer    0000000039a93890 f   GameSpy_2.11.00_VC10:gvSource.obj
 0001:000929d0       gviFreeSourceList          0000000039a939d0 f   GameSpy_2.11.00_VC10:gvSource.obj
 0001:000929f0       gviSetCustomCodec          0000000039a939f0 f   GameSpy_2.11.00_VC10:gvCodec.obj
 0001:00092a60       gviNewDecoder              0000000039a93a60 f   GameSpy_2.11.00_VC10:gvCodec.obj
 0001:00092a80       gviFreeDecoder             0000000039a93a80 f   GameSpy_2.11.00_VC10:gvCodec.obj
 0001:00092aa0       gviEncode                  0000000039a93aa0 f   GameSpy_2.11.00_VC10:gvCodec.obj
 0001:00092ab0       gviDecodeAdd               0000000039a93ab0 f   GameSpy_2.11.00_VC10:gvCodec.obj
 0001:00092ac0       gviCodecsInitialize        0000000039a93ac0 f   GameSpy_2.11.00_VC10:gvCodec.obj
 0001:00092ae0       gviIsFrameStampGT          0000000039a93ae0 f   GameSpy_2.11.00_VC10:gvFrame.obj
 0001:00092b00       gviIsFrameStampGTE         0000000039a93b00 f   GameSpy_2.11.00_VC10:gvFrame.obj
 0001:00092b20       gviPutPendingFrame         0000000039a93b20 f   GameSpy_2.11.00_VC10:gvFrame.obj
 0001:00092b40       gviGetPendingFrame         0000000039a93b40 f   GameSpy_2.11.00_VC10:gvFrame.obj
 0001:00092b70       gviFramesCleanup           0000000039a93b70 f   GameSpy_2.11.00_VC10:gvFrame.obj
 0001:00092bc0       gviFramesStartup           0000000039a93bc0 f   GameSpy_2.11.00_VC10:gvFrame.obj
 0001:00092d60       ghiFreeConnection          0000000039a93d60 f   GameSpy_2.11.00_VC10:ghttpConnection.obj
 0001:00092ee0       ghiRequestToConnection     0000000039a93ee0 f   GameSpy_2.11.00_VC10:ghttpConnection.obj
 0001:00092f30       ghiRedirectConnection      0000000039a93f30 f   GameSpy_2.11.00_VC10:ghttpConnection.obj
 0001:00093080       ghiCleanupConnections      0000000039a94080 f   GameSpy_2.11.00_VC10:ghttpConnection.obj
 0001:00093160       ghiNewConnection           0000000039a94160 f   GameSpy_2.11.00_VC10:ghttpConnection.obj
 0001:00093330       ghiCallCompletedCallback   0000000039a94330 f   GameSpy_2.11.00_VC10:ghttpCallbacks.obj
 0001:000933a0       ghiCallProgressCallback    0000000039a943a0 f   GameSpy_2.11.00_VC10:ghttpCallbacks.obj
 0001:000933f0       ghiCallPostCallback        0000000039a943f0 f   GameSpy_2.11.00_VC10:ghttpCallbacks.obj
 0001:000935d0       ghiDoSocketInit            0000000039a945d0 f   GameSpy_2.11.00_VC10:ghttpProcess.obj
 0001:00093690       ghiDoHostLookup            0000000039a94690 f   GameSpy_2.11.00_VC10:ghttpProcess.obj
 0001:00093770       ghiDoLookupPending         0000000039a94770 f   GameSpy_2.11.00_VC10:ghttpProcess.obj
 0001:000937f0       ghiDoConnecting            0000000039a947f0 f   GameSpy_2.11.00_VC10:ghttpProcess.obj
 0001:000939e0       ghiDoSecuringSession       0000000039a949e0 f   GameSpy_2.11.00_VC10:ghttpProcess.obj
 0001:00093b30       ghiDoSendingRequest        0000000039a94b30 f   GameSpy_2.11.00_VC10:ghttpProcess.obj
 0001:00093df0       ghiDoPosting               0000000039a94df0 f   GameSpy_2.11.00_VC10:ghttpProcess.obj
 0001:00093eb0       ghiDoWaiting               0000000039a94eb0 f   GameSpy_2.11.00_VC10:ghttpProcess.obj
 0001:00094030       ghiDoReceivingStatus       0000000039a95030 f   GameSpy_2.11.00_VC10:ghttpProcess.obj
 0001:00094520       ghiDoReceivingHeaders      0000000039a95520 f   GameSpy_2.11.00_VC10:ghttpProcess.obj
 0001:00094a30       ghiDoReceivingFile         0000000039a95a30 f   GameSpy_2.11.00_VC10:ghttpProcess.obj
 0001:00094ba0       ghiCreateLock              0000000039a95ba0 f   GameSpy_2.11.00_VC10:ghttpCommon.obj
 0001:00094be0       ghiFreeLock                0000000039a95be0 f   GameSpy_2.11.00_VC10:ghttpCommon.obj
 0001:00094c20       ghiLock                    0000000039a95c20 f   GameSpy_2.11.00_VC10:ghttpCommon.obj
 0001:00094c40       ghiUnlock                  0000000039a95c40 f   GameSpy_2.11.00_VC10:ghttpCommon.obj
 0001:00094c60       ghiDecryptReceivedData     0000000039a95c60 f   GameSpy_2.11.00_VC10:ghttpCommon.obj
 0001:00094db0       ghiDoReceive               0000000039a95db0 f   GameSpy_2.11.00_VC10:ghttpCommon.obj
 0001:00094f30       ghiDoSend                  0000000039a95f30 f   GameSpy_2.11.00_VC10:ghttpCommon.obj
 0001:00095040       ghiTrySendThenBuffer       0000000039a96040 f   GameSpy_2.11.00_VC10:ghttpCommon.obj
 0001:000951f0       ghiNewPost                 0000000039a961f0 f   GameSpy_2.11.00_VC10:ghttpPost.obj
 0001:00095260       ghiPostSetAutoFree         0000000039a96260 f   GameSpy_2.11.00_VC10:ghttpPost.obj
 0001:00095270       ghiIsPostAutoFree          0000000039a96270 f   GameSpy_2.11.00_VC10:ghttpPost.obj
 0001:00095280       ghiFreePost                0000000039a96280 f   GameSpy_2.11.00_VC10:ghttpPost.obj
 0001:000952a0       ghiPostAddXml              0000000039a962a0 f   GameSpy_2.11.00_VC10:ghttpPost.obj
 0001:000952e0       ghiPostGetContentType      0000000039a962e0 f   GameSpy_2.11.00_VC10:ghttpPost.obj
 0001:000956d0       ghiPostInitState           0000000039a966d0 f   GameSpy_2.11.00_VC10:ghttpPost.obj
 0001:000958b0       ghiPostCleanupState        0000000039a968b0 f   GameSpy_2.11.00_VC10:ghttpPost.obj
 0001:000963f0       ghiPostDoPosting           0000000039a973f0 f   GameSpy_2.11.00_VC10:ghttpPost.obj
 0001:00096640       ghiResizeBuffer            0000000039a97640 f   GameSpy_2.11.00_VC10:ghttpBuffer.obj
 0001:000966a0       ghiInitBuffer              0000000039a976a0 f   GameSpy_2.11.00_VC10:ghttpBuffer.obj
 0001:00096710       ghiInitFixedBuffer         0000000039a97710 f   GameSpy_2.11.00_VC10:ghttpBuffer.obj
 0001:00096760       ghiInitReadOnlyBuffer      0000000039a97760 f   GameSpy_2.11.00_VC10:ghttpBuffer.obj
 0001:000967b0       ghiFreeBuffer              0000000039a977b0 f   GameSpy_2.11.00_VC10:ghttpBuffer.obj
 0001:00096800       ghiAppendDataToBuffer      0000000039a97800 f   GameSpy_2.11.00_VC10:ghttpBuffer.obj
 0001:00096920       ghiEncryptDataToBuffer     0000000039a97920 f   GameSpy_2.11.00_VC10:ghttpBuffer.obj
 0001:00096a60       ghiAppendHeaderToBuffer    0000000039a97a60 f   GameSpy_2.11.00_VC10:ghttpBuffer.obj
 0001:00096ae0       ghiAppendCharToBuffer      0000000039a97ae0 f   GameSpy_2.11.00_VC10:ghttpBuffer.obj
 0001:00096b90       ghiAppendIntToBuffer       0000000039a97b90 f   GameSpy_2.11.00_VC10:ghttpBuffer.obj
 0001:00096be0       ghiResetBuffer             0000000039a97be0 f   GameSpy_2.11.00_VC10:ghttpBuffer.obj
 0001:00096c00       ghiSendBufferedData        0000000039a97c00 f   GameSpy_2.11.00_VC10:ghttpBuffer.obj
 0001:00096ce0       ghiReadDataFromBufferFixed 0000000039a97ce0 f   GameSpy_2.11.00_VC10:ghttpBuffer.obj
 0001:00096d30       d2giParseResponseHeader    0000000039a97d30 f   GameSpy_2.11.00_VC10:d2gDeserialize.obj
 0001:00096d90       d2giParseItemInfoFromResponse 0000000039a97d90 f   GameSpy_2.11.00_VC10:d2gDeserialize.obj
 0001:00096f20       d2giParseProductInfoFromResponse 0000000039a97f20 f   GameSpy_2.11.00_VC10:d2gDeserialize.obj
 0001:00097090       d2giParseGeoInfoFromResponse 0000000039a98090 f   GameSpy_2.11.00_VC10:d2gDeserialize.obj
 0001:00097170       d2giParseImageListFromResponse 0000000039a98170 f   GameSpy_2.11.00_VC10:d2gDeserialize.obj
 0001:000972c0       d2giParseCategoryListFromResponse 0000000039a982c0 f   GameSpy_2.11.00_VC10:d2gDeserialize.obj
 0001:00097410       d2giParseItemTotalFromResponse 0000000039a98410 f   GameSpy_2.11.00_VC10:d2gDeserialize.obj
 0001:000974e0       d2giParseOrderItemValidationFromResponse 0000000039a984e0 f   GameSpy_2.11.00_VC10:d2gDeserialize.obj
 0001:00097600       d2giParseOrderItemFromResponse 0000000039a98600 f   GameSpy_2.11.00_VC10:d2gDeserialize.obj
 0001:000976a0       d2giParseOrderItemLicensesFromResponse 0000000039a986a0 f   GameSpy_2.11.00_VC10:d2gDeserialize.obj
 0001:00097820       d2giParseOrderItemDownloadsFromResponse 0000000039a98820 f   GameSpy_2.11.00_VC10:d2gDeserialize.obj
 0001:00097a10       d2giParseOrderItemPurchaseFromResponse 0000000039a98a10 f   GameSpy_2.11.00_VC10:d2gDeserialize.obj
 0001:00097c20       d2giParseOrderValidationFromResponse 0000000039a98c20 f   GameSpy_2.11.00_VC10:d2gDeserialize.obj
 0001:00097d30       d2giParseOrderFromResponse 0000000039a98d30 f   GameSpy_2.11.00_VC10:d2gDeserialize.obj
 0001:00097f00       d2giParseOrderTotalFromResponse 0000000039a98f00 f   GameSpy_2.11.00_VC10:d2gDeserialize.obj
 0001:00098070       d2giParseOrderPurchaseFromResponse 0000000039a99070 f   GameSpy_2.11.00_VC10:d2gDeserialize.obj
 0001:00098240       d2giParseDownloadHeaderFromResponse 0000000039a99240 f   GameSpy_2.11.00_VC10:d2gDeserialize.obj
 0001:00098320       d2giParseDownloadUserHeadersFromResponse 0000000039a99320 f   GameSpy_2.11.00_VC10:d2gDeserialize.obj
 0001:00098420       d2giParseExtraInfo         0000000039a99420 f   GameSpy_2.11.00_VC10:d2gDeserialize.obj
 0001:00098520       d2giParseExtraInfoList     0000000039a99520 f   GameSpy_2.11.00_VC10:d2gDeserialize.obj
 0001:00098630       d2giParseDownload          0000000039a99630 f   GameSpy_2.11.00_VC10:d2gDeserialize.obj
 0001:000986a0       d2giParseGetResponse       0000000039a996a0 f   GameSpy_2.11.00_VC10:d2gDeserialize.obj
 0001:000986f0       d2giParseItemFromResponse  0000000039a996f0 f   GameSpy_2.11.00_VC10:d2gDeserialize.obj
 0001:00098830       d2giParseGetStoreAvailResponse 0000000039a99830 f   GameSpy_2.11.00_VC10:d2gDeserialize.obj
 0001:000988d0       d2giParseCreditCardInfoList 0000000039a998d0 f   GameSpy_2.11.00_VC10:d2gDeserialize.obj
 0001:00098b80       d2giParseItemsFromResponse 0000000039a99b80 f   GameSpy_2.11.00_VC10:d2gDeserialize.obj
 0001:00098d70       d2giParseLoadCatalogItemsFromResponse 0000000039a99d70 f   GameSpy_2.11.00_VC10:d2gDeserialize.obj
 0001:00098e30       d2giParseGetOrderTotalResponse 0000000039a99e30 f   GameSpy_2.11.00_VC10:d2gDeserialize.obj
 0001:00098f10       d2giParseStartOrderResponse 0000000039a99f10 f   GameSpy_2.11.00_VC10:d2gDeserialize.obj
 0001:00099000       d2giParseIsOrderCompleteResponse 0000000039a9a000 f   GameSpy_2.11.00_VC10:d2gDeserialize.obj
 0001:000990f0       d2giParseGetPurchaseHistoryResponse 0000000039a9a0f0 f   GameSpy_2.11.00_VC10:d2gDeserialize.obj
 0001:00099280       d2giParseManifestRecord    0000000039a9a280 f   GameSpy_2.11.00_VC10:d2gDeserialize.obj
 0001:00099350       d2giParseAndDecodeManifestRecord 0000000039a9a350 f   GameSpy_2.11.00_VC10:d2gDeserialize.obj
 0001:00099410       d2giDownloadHttpProgressCallback 0000000039a9a410 f   GameSpy_2.11.00_VC10:d2gDownloads.obj
 0001:00099460       d2giDownloadHttpCompletedCallback 0000000039a9a460 f   GameSpy_2.11.00_VC10:d2gDownloads.obj
 0001:00099520       d2giDownloadThreadFunc     0000000039a9a520 f   GameSpy_2.11.00_VC10:d2gDownloads.obj
 0001:000995c0       d2giStartDownloadThread    0000000039a9a5c0 f   GameSpy_2.11.00_VC10:d2gDownloads.obj
 0001:000997c0       GOACryptInit               0000000039a9a7c0 f   GameSpy_2.11.00_VC10:sb_crypt.obj
 0001:00099920       GOADecrypt                 0000000039a9a920 f   GameSpy_2.11.00_VC10:sb_crypt.obj
 0001:00099a50       gpiStatusInfoKeyFree       0000000039a9aa50 f   GameSpy_2.11.00_VC10:gpiKeys.obj
 0001:00099a80       gpiStatusInfoKeysInit      0000000039a9aa80 f   GameSpy_2.11.00_VC10:gpiKeys.obj
 0001:00099ae0       gpiStatusInfoKeysDestroy   0000000039a9aae0 f   GameSpy_2.11.00_VC10:gpiKeys.obj
 0001:00099b10       gpiStatusInfoKeyCompFunc   0000000039a9ab10 f   GameSpy_2.11.00_VC10:gpiKeys.obj
 0001:00099b40       gpiStatusInfoAddKey        0000000039a9ab40 f   GameSpy_2.11.00_VC10:gpiKeys.obj
 0001:00099bd0       gpiStatusInfoSetKey        0000000039a9abd0 f   GameSpy_2.11.00_VC10:gpiKeys.obj
 0001:00099c70       gpiStatusInfoCheckKey      0000000039a9ac70 f   GameSpy_2.11.00_VC10:gpiKeys.obj
 0001:00099d00       gpiSaveKeysToBuffer        0000000039a9ad00 f   GameSpy_2.11.00_VC10:gpiKeys.obj
 0001:0009a120       gpiFailedOpCallback        0000000039a9b120 f   GameSpy_2.11.00_VC10:gpiOperation.obj
 0001:0009a340       gpiAddOperation            0000000039a9b340 f   GameSpy_2.11.00_VC10:gpiOperation.obj
 0001:0009a430       gpiDestroyOperation        0000000039a9b430 f   GameSpy_2.11.00_VC10:gpiOperation.obj
 0001:0009a4b0       gpiRemoveOperation         0000000039a9b4b0 f   GameSpy_2.11.00_VC10:gpiOperation.obj
 0001:0009a510       gpiFindOperationByID       0000000039a9b510 f   GameSpy_2.11.00_VC10:gpiOperation.obj
 0001:0009a550       gpiOperationsAreBlocking   0000000039a9b550 f   GameSpy_2.11.00_VC10:gpiOperation.obj
 0001:0009a580       gpiProcessOperation        0000000039a9b580 f   GameSpy_2.11.00_VC10:gpiOperation.obj
 0001:0009a620       gpiAddCallback             0000000039a9b620 f   GameSpy_2.11.00_VC10:gpiCallback.obj
 0001:0009a920       gpiProcessCallbacks        0000000039a9b920 f   GameSpy_2.11.00_VC10:gpiCallback.obj
 0001:0009ac90       gpiCallErrorCallback       0000000039a9bc90 f   GameSpy_2.11.00_VC10:gpiCallback.obj
 0001:0009ad90       gsUdpMsgHandlerFree        0000000039a9bd90 f   GameSpy_2.11.00_VC10:gsUdpEngine.obj
 0001:0009ada0       gsUdpMsgHandlerCompare     0000000039a9bda0 f   GameSpy_2.11.00_VC10:gsUdpEngine.obj
 0001:0009adb0       gsUdpMsgHandlerCompare2    0000000039a9bdb0 f   GameSpy_2.11.00_VC10:gsUdpEngine.obj
 0001:0009add0       gsUdpRemotePeerCompare     0000000039a9bdd0 f   GameSpy_2.11.00_VC10:gsUdpEngine.obj
 0001:0009adf0       gsUdpRemotePeerCompare2    0000000039a9bdf0 f   GameSpy_2.11.00_VC10:gsUdpEngine.obj
 0001:0009ae00       gsUdpSocketError           0000000039a9be00 f   GameSpy_2.11.00_VC10:gsUdpEngine.obj
 0001:0009ae80       gsUdpClosedRoutingCB       0000000039a9be80 f   GameSpy_2.11.00_VC10:gsUdpEngine.obj
 0001:0009b000       gsUdpConnectedRoutingCB    0000000039a9c000 f   GameSpy_2.11.00_VC10:gsUdpEngine.obj
 0001:0009b210       gsUdpPingRoutingCB         0000000039a9c210 f   GameSpy_2.11.00_VC10:gsUdpEngine.obj
 0001:0009b310       gsUdpReceivedRoutingCB     0000000039a9c310 f   GameSpy_2.11.00_VC10:gsUdpEngine.obj
 0001:0009b450       gsUdpUnrecognizedMsgCB     0000000039a9c450 f   GameSpy_2.11.00_VC10:gsUdpEngine.obj
 0001:0009b4d0       gsUdpConnAttemptCB         0000000039a9c4d0 f   GameSpy_2.11.00_VC10:gsUdpEngine.obj
 0001:0009b650       gsUdpEngineIsInitialized   0000000039a9c650 f   GameSpy_2.11.00_VC10:gsUdpEngine.obj
 0001:0009b660       gsUdpEngineInitialize      0000000039a9c660 f   GameSpy_2.11.00_VC10:gsUdpEngine.obj
 0001:0009b810       gsUdpEngineGetPeerState    0000000039a9c810 f   GameSpy_2.11.00_VC10:gsUdpEngine.obj
 0001:0009b8a0       gsUdpEngineStartTalkingToPeer 0000000039a9c8a0 f   GameSpy_2.11.00_VC10:gsUdpEngine.obj
 0001:0009baf0       gsUdpEngineSendMessage     0000000039a9caf0 f   GameSpy_2.11.00_VC10:gsUdpEngine.obj
 0001:0009bc40       gsUdpEngineThink           0000000039a9cc40 f   GameSpy_2.11.00_VC10:gsUdpEngine.obj
 0001:0009bc70       gsUdpEngineShutdown        0000000039a9cc70 f   GameSpy_2.11.00_VC10:gsUdpEngine.obj
 0001:0009bcc0       gsUdpEngineGetLocalPort    0000000039a9ccc0 f   GameSpy_2.11.00_VC10:gsUdpEngine.obj
 0001:0009bce0       gsUdpEngineAddMsgHandler   0000000039a9cce0 f   GameSpy_2.11.00_VC10:gsUdpEngine.obj
 0001:0009bdc0       gsUdpEngineRemoveMsgHandler 0000000039a9cdc0 f   GameSpy_2.11.00_VC10:gsUdpEngine.obj
 0001:0009be80       gsUdpEngineNoMoreMsgHandlers 0000000039a9ce80 f   GameSpy_2.11.00_VC10:gsUdpEngine.obj
 0001:0009bec0       gsUdpEngineNoApp           0000000039a9cec0 f   GameSpy_2.11.00_VC10:gsUdpEngine.obj
 0001:0009bf20       gsUdpEngineGetPeerOutBufferFreeSpace 0000000039a9cf20 f   GameSpy_2.11.00_VC10:gsUdpEngine.obj
 0001:0009bf90       gpiHandleTransferMessage   0000000039a9cf90 f   GameSpy_2.11.00_VC10:gpiTransfer.obj
 0001:0009c090       gviNewDevice               0000000039a9d090 f   GameSpy_2.11.00_VC10:gvDevice.obj
 0001:0009c140       gviFreeDevice              0000000039a9d140 f   GameSpy_2.11.00_VC10:gvDevice.obj
 0001:0009c170       gviDeviceUnplugged         0000000039a9d170 f   GameSpy_2.11.00_VC10:gvDevice.obj
 0001:0009c1a0       gviNewDeviceList           0000000039a9d1a0 f   GameSpy_2.11.00_VC10:gvDevice.obj
 0001:0009c1b0       gviFreeDeviceList          0000000039a9d1b0 f   GameSpy_2.11.00_VC10:gvDevice.obj
 0001:0009c1c0       gviAppendDeviceToList      0000000039a9d1c0 f   GameSpy_2.11.00_VC10:gvDevice.obj
 0001:0009c1e0       gviGetNumDevices           0000000039a9d1e0 f   GameSpy_2.11.00_VC10:gvDevice.obj
 0001:0009c1f0       gviGetDevice               0000000039a9d1f0 f   GameSpy_2.11.00_VC10:gvDevice.obj
 0001:0009c210       gviDeleteDeviceFromList    0000000039a9d210 f   GameSpy_2.11.00_VC10:gvDevice.obj
 0001:0009c280       gviGetSamplesVolume        0000000039a9d280 f   GameSpy_2.11.00_VC10:gvUtil.obj
 0001:0009c2d0       gviIsOverThreshold         0000000039a9d2d0 f   GameSpy_2.11.00_VC10:gvUtil.obj
 0001:0009c330       gviRoundUpToNearestMultiple 0000000039a9d330 f   GameSpy_2.11.00_VC10:gvUtil.obj
 0001:0009c350       gviRoundDownToNearestMultiple 0000000039a9d350 f   GameSpy_2.11.00_VC10:gvUtil.obj
 0001:0009c360       gviRoundToNearestMultiple  0000000039a9d360 f   GameSpy_2.11.00_VC10:gvUtil.obj
 0001:0009c390       gviMultiplyByBytesPerMillisecond 0000000039a9d390 f   GameSpy_2.11.00_VC10:gvUtil.obj
 0001:0009c3c0       gviDivideByBytesPerMillisecond 0000000039a9d3c0 f   GameSpy_2.11.00_VC10:gvUtil.obj
 0001:0009caa0       ghiEncryptorSslInitFunc    0000000039a9daa0 f   GameSpy_2.11.00_VC10:ghttpEncryption.obj
 0001:0009cb40       ghiEncryptorSslCleanupFunc 0000000039a9db40 f   GameSpy_2.11.00_VC10:ghttpEncryption.obj
 0001:0009cb80       ghiEncryptorSslStartFunc   0000000039a9db80 f   GameSpy_2.11.00_VC10:ghttpEncryption.obj
 0001:0009cd00       ghiEncryptorSslEncryptFunc 0000000039a9dd00 f   GameSpy_2.11.00_VC10:ghttpEncryption.obj
 0001:0009dce0       ghiEncryptorSslDecryptRecv 0000000039a9ece0 f   GameSpy_2.11.00_VC10:ghttpEncryption.obj
 0001:0009dce0       ghiEncryptorSslEncryptSend 0000000039a9ece0 f   GameSpy_2.11.00_VC10:ghttpEncryption.obj
 0001:0009dcf0       ghiEncryptorSslDecryptFunc 0000000039a9ecf0 f   GameSpy_2.11.00_VC10:ghttpEncryption.obj
 0001:0009df10       ghttpSetRequestEncryptionEngine 0000000039a9ef10 f   GameSpy_2.11.00_VC10:ghttpEncryption.obj
 0001:0009e010       gt2AddressToString         0000000039a9f010 f   GameSpy_2.11.00_VC10:gt2Utility.obj
 0001:0009e0d0       gt2StringToAddress         0000000039a9f0d0 f   GameSpy_2.11.00_VC10:gt2Utility.obj
 0001:0009e200       gti2MessageCheck           0000000039a9f200 f   GameSpy_2.11.00_VC10:gt2Utility.obj
 0001:0009e240       gt2CreateSocket            0000000039a9f240 f   GameSpy_2.11.00_VC10:gt2Main.obj
 0001:0009e260       gt2Think                   0000000039a9f260 f   GameSpy_2.11.00_VC10:gt2Main.obj
 0001:0009e290       gt2Listen                  0000000039a9f290 f   GameSpy_2.11.00_VC10:gt2Main.obj
 0001:0009e2a0       gt2Accept                  0000000039a9f2a0 f   GameSpy_2.11.00_VC10:gt2Main.obj
 0001:0009e2b0       gt2Reject                  0000000039a9f2b0 f   GameSpy_2.11.00_VC10:gt2Main.obj
 0001:0009e2c0       gt2Connect                 0000000039a9f2c0 f   GameSpy_2.11.00_VC10:gt2Main.obj
 0001:0009e430       gt2Send                    0000000039a9f430 f   GameSpy_2.11.00_VC10:gt2Main.obj
 0001:0009e510       gt2CloseAllConnectionsHard 0000000039a9f510 f   GameSpy_2.11.00_VC10:gt2Main.obj
 0001:0009e530       gt2GetConnectionState      0000000039a9f530 f   GameSpy_2.11.00_VC10:gt2Main.obj
 0001:0009e550       gt2GetLocalPort            0000000039a9f550 f   GameSpy_2.11.00_VC10:gt2Main.obj
 0001:0009e560       gt2GetOutgoingBufferSize   0000000039a9f560 f   GameSpy_2.11.00_VC10:gt2Main.obj
 0001:0009e570       gt2GetOutgoingBufferFreeSpace 0000000039a9f570 f   GameSpy_2.11.00_VC10:gt2Main.obj
 0001:0009e580       gt2SetUnrecognizedMessageCallback 0000000039a9f580 f   GameSpy_2.11.00_VC10:gt2Main.obj
 0001:0009e590       gt2CloseSocket             0000000039a9f590 f   GameSpy_2.11.00_VC10:gt2Main.obj
 0001:0009e5c0       RC4Init                    0000000039a9f5c0 f   GameSpy_2.11.00_VC10:gsRC4.obj
 0001:0009e660       RC4Encrypt                 0000000039a9f660 f   GameSpy_2.11.00_VC10:gsRC4.obj
 0001:0009e6e0       GSSHA1Reset                0000000039a9f6e0 f   GameSpy_2.11.00_VC10:gsSHA1.obj
 0001:0009e720       SHA1ProcessMessageBlock    0000000039a9f720 f   GameSpy_2.11.00_VC10:gsSHA1.obj
 0001:0009ebd0       SHA1PadMessage             0000000039a9fbd0 f   GameSpy_2.11.00_VC10:gsSHA1.obj
 0001:0009ecd0       GSSHA1Result               0000000039a9fcd0 f   GameSpy_2.11.00_VC10:gsSHA1.obj
 0001:0009ed90       GSSHA1Input                0000000039a9fd90 f   GameSpy_2.11.00_VC10:gsSHA1.obj
 0001:0009eea0       gti2SocketFindConnection   0000000039a9fea0 f   GameSpy_2.11.00_VC10:gt2Socket.obj
 0001:0009ef20       gti2CreateSocket           0000000039a9ff20 f   GameSpy_2.11.00_VC10:gt2Socket.obj
 0001:0009f130       gti2CloseSocket            0000000039aa0130 f   GameSpy_2.11.00_VC10:gt2Socket.obj
 0001:0009f180       gti2Listen                 0000000039aa0180 f   GameSpy_2.11.00_VC10:gt2Socket.obj
 0001:0009f190       gti2NewSocketConnection    0000000039aa0190 f   GameSpy_2.11.00_VC10:gt2Socket.obj
 0001:0009f3f0       gti2FreeSocketConnection   0000000039aa03f0 f   GameSpy_2.11.00_VC10:gt2Socket.obj
 0001:0009f4e0       gti2SocketConnectionsThink 0000000039aa04e0 f   GameSpy_2.11.00_VC10:gt2Socket.obj
 0001:0009f520       gti2FreeClosedConnections  0000000039aa0520 f   GameSpy_2.11.00_VC10:gt2Socket.obj
 0001:0009f5f0       gti2SocketError            0000000039aa05f0 f   GameSpy_2.11.00_VC10:gt2Socket.obj
 0001:0009f660       gti2SocketSend             0000000039aa0660 f   GameSpy_2.11.00_VC10:gt2Socket.obj
 0001:0009fbb0       gti2HandleConnectionReset  0000000039aa0bb0 f   GameSpy_2.11.00_VC10:gt2Message.obj
 0001:0009fc70       gti2HandleHostUnreachable  0000000039aa0c70 f   GameSpy_2.11.00_VC10:gt2Message.obj
 0001:0009fe10       gti2SendAppUnreliable      0000000039aa0e10 f   GameSpy_2.11.00_VC10:gt2Message.obj
 0001:0009ff20       gti2SendAck                0000000039aa0f20 f   GameSpy_2.11.00_VC10:gt2Message.obj
 0001:0009ffe0       gti2SendNack               0000000039aa0fe0 f   GameSpy_2.11.00_VC10:gt2Message.obj
 0001:000a00a0       gti2SendClosedOnSocket     0000000039aa10a0 f   GameSpy_2.11.00_VC10:gt2Message.obj
 0001:000a0120       gti2ResendMessage          0000000039aa1120 f   GameSpy_2.11.00_VC10:gt2Message.obj
 0001:000a0570       gti2SendClosed             0000000039aa1570 f   GameSpy_2.11.00_VC10:gt2Message.obj
 0001:000a0870       gti2SendAppReliable        0000000039aa1870 f   GameSpy_2.11.00_VC10:gt2Message.obj
 0001:000a0900       gti2SendClientChallenge    0000000039aa1900 f   GameSpy_2.11.00_VC10:gt2Message.obj
 0001:000a0980       gti2SendClientResponse     0000000039aa1980 f   GameSpy_2.11.00_VC10:gt2Message.obj
 0001:000a0a30       gti2SendAccept             0000000039aa1a30 f   GameSpy_2.11.00_VC10:gt2Message.obj
 0001:000a0a90       gti2SendReject             0000000039aa1a90 f   GameSpy_2.11.00_VC10:gt2Message.obj
 0001:000a0b30       gti2SendClose              0000000039aa1b30 f   GameSpy_2.11.00_VC10:gt2Message.obj
 0001:000a0b90       gti2SendKeepAlive          0000000039aa1b90 f   GameSpy_2.11.00_VC10:gt2Message.obj
 0001:000a0bf0       gti2Send                   0000000039aa1bf0 f   GameSpy_2.11.00_VC10:gt2Message.obj
 0001:000a13b0       gti2ReceiveMessages        0000000039aa23b0 f   GameSpy_2.11.00_VC10:gt2Message.obj
 0001:000a14e0       gti2NewOutgoingConnection  0000000039aa24e0 f   GameSpy_2.11.00_VC10:gt2Connection.obj
 0001:000a1510       gti2NewIncomingConnection  0000000039aa2510 f   GameSpy_2.11.00_VC10:gt2Connection.obj
 0001:000a1540       gti2StartConnectionAttempt 0000000039aa2540 f   GameSpy_2.11.00_VC10:gt2Connection.obj
 0001:000a1630       gti2AcceptConnection       0000000039aa2630 f   GameSpy_2.11.00_VC10:gt2Connection.obj
 0001:000a16a0       gti2RejectConnection       0000000039aa26a0 f   GameSpy_2.11.00_VC10:gt2Connection.obj
 0001:000a16f0       gti2ConnectionSendData     0000000039aa26f0 f   GameSpy_2.11.00_VC10:gt2Connection.obj
 0001:000a17c0       gti2ConnectionClosed       0000000039aa27c0 f   GameSpy_2.11.00_VC10:gt2Connection.obj
 0001:000a1810       gti2ConnectionCleanup      0000000039aa2810 f   GameSpy_2.11.00_VC10:gt2Connection.obj
 0001:000a1950       gti2ConnectionThink        0000000039aa2950 f   GameSpy_2.11.00_VC10:gt2Connection.obj
 0001:000a19d0       gti2CloseConnection        0000000039aa29d0 f   GameSpy_2.11.00_VC10:gt2Connection.obj
 0001:000a1a60       gti2SocketErrorCallback    0000000039aa2a60 f   GameSpy_2.11.00_VC10:gt2Callback.obj
 0001:000a1ab0       gti2ConnectAttemptCallback 0000000039aa2ab0 f   GameSpy_2.11.00_VC10:gt2Callback.obj
 0001:000a1b40       gti2ConnectedCallback      0000000039aa2b40 f   GameSpy_2.11.00_VC10:gt2Callback.obj
 0001:000a1bb0       gti2ReceivedCallback       0000000039aa2bb0 f   GameSpy_2.11.00_VC10:gt2Callback.obj
 0001:000a1c20       gti2ClosedCallback         0000000039aa2c20 f   GameSpy_2.11.00_VC10:gt2Callback.obj
 0001:000a1c80       gti2PingCallback           0000000039aa2c80 f   GameSpy_2.11.00_VC10:gt2Callback.obj
 0001:000a1ce0       gti2SendFilterCallback     0000000039aa2ce0 f   GameSpy_2.11.00_VC10:gt2Callback.obj
 0001:000a1d90       gti2ReceiveFilterCallback  0000000039aa2d90 f   GameSpy_2.11.00_VC10:gt2Callback.obj
 0001:000a1e40       gti2DumpCallback           0000000039aa2e40 f   GameSpy_2.11.00_VC10:gt2Callback.obj
 0001:000a1ef0       gti2UnrecognizedMessageCallback 0000000039aa2ef0 f   GameSpy_2.11.00_VC10:gt2Callback.obj
 0001:000a1f70       gti2AllocateBuffer         0000000039aa2f70 f   GameSpy_2.11.00_VC10:gt2Buffer.obj
 0001:000a1fb0       gti2GetBufferFreeSpace     0000000039aa2fb0 f   GameSpy_2.11.00_VC10:gt2Buffer.obj
 0001:000a1fc0       gti2BufferWriteByte        0000000039aa2fc0 f   GameSpy_2.11.00_VC10:gt2Buffer.obj
 0001:000a1fd0       gti2BufferWriteUShort      0000000039aa2fd0 f   GameSpy_2.11.00_VC10:gt2Buffer.obj
 0001:000a2000       gti2BufferWriteData        0000000039aa3000 f   GameSpy_2.11.00_VC10:gt2Buffer.obj
 0001:000a2050       gti2BufferShorten          0000000039aa3050 f   GameSpy_2.11.00_VC10:gt2Buffer.obj
 0001:000a20a0       gti2GetChallenge           0000000039aa30a0 f   GameSpy_2.11.00_VC10:gt2Auth.obj
 0001:000a2190       gti2GetResponse            0000000039aa3190 f   GameSpy_2.11.00_VC10:gt2Auth.obj
 0001:000a2350       gti2CheckResponse          0000000039aa3350 f   GameSpy_2.11.00_VC10:gt2Auth.obj
 0001:000a238c       GetDeviceID                0000000039aa338c f   dsound:DSOUND.dll
 0001:000a2392       DirectSoundEnumerateA      0000000039aa3392 f   dsound:DSOUND.dll
 0001:000a2398       DirectSoundCaptureEnumerateA 0000000039aa3398 f   dsound:DSOUND.dll
 0001:000a239e       DirectSoundCaptureCreate   0000000039aa339e f   dsound:DSOUND.dll
 0001:000a23a4       DirectSoundCreate          0000000039aa33a4 f   dsound:DSOUND.dll
 0001:000a23aa       sendto                     0000000039aa33aa f   Wsock32:WSOCK32.dll
 0001:000a23b0       gethostbyname              0000000039aa33b0 f   Wsock32:WSOCK32.dll
 0001:000a23b6       inet_addr                  0000000039aa33b6 f   Wsock32:WSOCK32.dll
 0001:000a23bc       bind                       0000000039aa33bc f   Wsock32:WSOCK32.dll
 0001:000a23c2       WSAGetLastError            0000000039aa33c2 f   Wsock32:WSOCK32.dll
 0001:000a23c8       recvfrom                   0000000039aa33c8 f   Wsock32:WSOCK32.dll
 0001:000a23ce       WSAStartup                 0000000039aa33ce f   Wsock32:WSOCK32.dll
 0001:000a23d4       WSACleanup                 0000000039aa33d4 f   Wsock32:WSOCK32.dll
 0001:000a23da       gethostname                0000000039aa33da f   Wsock32:WSOCK32.dll
 0001:000a23e0       shutdown                   0000000039aa33e0 f   Wsock32:WSOCK32.dll
 0001:000a23e8       __GSHandlerCheckCommon     0000000039aa33e8 f   MSVCRT:gshandler.obj
 0001:000a244c       __GSHandlerCheck           0000000039aa344c f   MSVCRT:gshandler.obj
 0001:000a2480       __security_check_cookie    0000000039aa3480 f   MSVCRT:amdsecgs.obj
 0001:000a24a0       memcmp                     0000000039aa34a0 f   MSVCRT:MSVCR100.dll
 0001:000a24a6       log                        0000000039aa34a6 f   MSVCRT:MSVCR100.dll
 0001:000a24ac       exp                        0000000039aa34ac f   MSVCRT:MSVCR100.dll
 0001:000a24b4       __report_gsfailure         0000000039aa34b4 f   MSVCRT:gs_report.obj
 0001:000a25fe       __crt_debugger_hook        0000000039aa35fe f   MSVCRT:MSVCR100.dll
 0001:000a2604       RtlVirtualUnwind           0000000039aa3604 f   kernel32:KERNEL32.dll
 0001:000a260a       RtlLookupFunctionEntry     0000000039aa360a f   kernel32:KERNEL32.dll
 0001:000a2aa0       ??__Fs_dummyMemReplay@?1??CryGetIMemReplay@@YAPEAUIMemReplay@@XZ@YAXXZ 0000000039aa3aa0 f i CryDLCStore.obj
 0001:000a2c40       ??__Fp@?1??CreateClassInstance@CFactory@CEngineModule_CryLobby@@UEBA?AV?$shared_ptr@UICryUnknown@@@boost@@XZ@YAXXZ 0000000039aa3c40 f i CryLobbyDLL.obj
 0002:00000000       __imp_RegQueryValueExA     0000000039aa5000     advapi32:ADVAPI32.dll
 0002:00000008       __imp_RegCreateKeyExA      0000000039aa5008     advapi32:ADVAPI32.dll
 0002:00000010       __imp_RegSetValueExA       0000000039aa5010     advapi32:ADVAPI32.dll
 0002:00000018       __imp_RegCloseKey          0000000039aa5018     advapi32:ADVAPI32.dll
 0002:00000020       __imp_RegOpenKeyExA        0000000039aa5020     advapi32:ADVAPI32.dll
 0002:00000028       \177ADVAPI32_NULL_THUNK_DATA 0000000039aa5028     advapi32:ADVAPI32.dll
 0002:00000030       __imp_GetDeviceID          0000000039aa5030     dsound:DSOUND.dll
 0002:00000038       __imp_DirectSoundCaptureEnumerateA 0000000039aa5038     dsound:DSOUND.dll
 0002:00000040       __imp_DirectSoundCaptureCreate 0000000039aa5040     dsound:DSOUND.dll
 0002:00000048       __imp_DirectSoundCreate    0000000039aa5048     dsound:DSOUND.dll
 0002:00000050       __imp_DirectSoundEnumerateA 0000000039aa5050     dsound:DSOUND.dll
 0002:00000058       \177DSOUND_NULL_THUNK_DATA 0000000039aa5058     dsound:DSOUND.dll
 0002:00000060       __imp_CreateThread         0000000039aa5060     kernel32:KERNEL32.dll
 0002:00000068       __imp_QueryPerformanceFrequency 0000000039aa5068     kernel32:KERNEL32.dll
 0002:00000070       __imp_GetSystemTimeAsFileTime 0000000039aa5070     kernel32:KERNEL32.dll
 0002:00000078       __imp_GetCurrentProcessId  0000000039aa5078     kernel32:KERNEL32.dll
 0002:00000080       __imp_GetTickCount         0000000039aa5080     kernel32:KERNEL32.dll
 0002:00000088       __imp_QueryPerformanceCounter 0000000039aa5088     kernel32:KERNEL32.dll
 0002:00000090       __imp_DisableThreadLibraryCalls 0000000039aa5090     kernel32:KERNEL32.dll
 0002:00000098       __imp_CloseHandle          0000000039aa5098     kernel32:KERNEL32.dll
 0002:000000a0       __imp_WaitForSingleObject  0000000039aa50a0     kernel32:KERNEL32.dll
 0002:000000a8       __imp_CreateMutexA         0000000039aa50a8     kernel32:KERNEL32.dll
 0002:000000b0       __imp_ReleaseMutex         0000000039aa50b0     kernel32:KERNEL32.dll
 0002:000000b8       __imp_InitializeCriticalSection 0000000039aa50b8     kernel32:KERNEL32.dll
 0002:000000c0       __imp_DeleteCriticalSection 0000000039aa50c0     kernel32:KERNEL32.dll
 0002:000000c8       __imp_EnterCriticalSection 0000000039aa50c8     kernel32:KERNEL32.dll
 0002:000000d0       __imp_LeaveCriticalSection 0000000039aa50d0     kernel32:KERNEL32.dll
 0002:000000d8       __imp_TryEnterCriticalSection 0000000039aa50d8     kernel32:KERNEL32.dll
 0002:000000e0       __imp_TerminateThread      0000000039aa50e0     kernel32:KERNEL32.dll
 0002:000000e8       __imp_GetCurrentThreadId   0000000039aa50e8     kernel32:KERNEL32.dll
 0002:000000f0       __imp_LoadLibraryA         0000000039aa50f0     kernel32:KERNEL32.dll
 0002:000000f8       __imp_GetProcAddress       0000000039aa50f8     kernel32:KERNEL32.dll
 0002:00000100       __imp_GetModuleHandleA     0000000039aa5100     kernel32:KERNEL32.dll
 0002:00000108       __imp_IsDebuggerPresent    0000000039aa5108     kernel32:KERNEL32.dll
 0002:00000110       __imp_Sleep                0000000039aa5110     kernel32:KERNEL32.dll
 0002:00000118       __imp_DecodePointer        0000000039aa5118     kernel32:KERNEL32.dll
 0002:00000120       __imp_EncodePointer        0000000039aa5120     kernel32:KERNEL32.dll
 0002:00000128       __imp_SetUnhandledExceptionFilter 0000000039aa5128     kernel32:KERNEL32.dll
 0002:00000130       __imp_RtlVirtualUnwind     0000000039aa5130     kernel32:KERNEL32.dll
 0002:00000138       __imp_RtlLookupFunctionEntry 0000000039aa5138     kernel32:KERNEL32.dll
 0002:00000140       __imp_TerminateProcess     0000000039aa5140     kernel32:KERNEL32.dll
 0002:00000148       __imp_GetCurrentProcess    0000000039aa5148     kernel32:KERNEL32.dll
 0002:00000150       __imp_RtlCaptureContext    0000000039aa5150     kernel32:KERNEL32.dll
 0002:00000158       __imp_UnhandledExceptionFilter 0000000039aa5158     kernel32:KERNEL32.dll
 0002:00000160       \177KERNEL32_NULL_THUNK_DATA 0000000039aa5160     kernel32:KERNEL32.dll
 0002:00000168       __imp_strcpy_s             0000000039aa5168     MSVCRT:MSVCR100.dll
 0002:00000170       __imp_memset               0000000039aa5170     MSVCRT:MSVCR100.dll
 0002:00000178       __imp_sscanf_s             0000000039aa5178     MSVCRT:MSVCR100.dll
 0002:00000180       __imp_strcspn              0000000039aa5180     MSVCRT:MSVCR100.dll
 0002:00000188       __imp_strchr               0000000039aa5188     MSVCRT:MSVCR100.dll
 0002:00000190       __imp_atof                 0000000039aa5190     MSVCRT:MSVCR100.dll
 0002:00000198       __imp_strrchr              0000000039aa5198     MSVCRT:MSVCR100.dll
 0002:000001a0       __imp__set_invalid_parameter_handler 0000000039aa51a0     MSVCRT:MSVCR100.dll
 0002:000001a8       __imp__set_purecall_handler 0000000039aa51a8     MSVCRT:MSVCR100.dll
 0002:000001b0       __imp_??0exception@std@@QEAA@AEBQEBDH@Z 0000000039aa51b0     MSVCRT:MSVCR100.dll
 0002:000001b8       __imp_?what@exception@std@@UEBAPEBDXZ 0000000039aa51b8     MSVCRT:MSVCR100.dll
 0002:000001c0       __imp_??1exception@std@@UEAA@XZ 0000000039aa51c0     MSVCRT:MSVCR100.dll
 0002:000001c8       __imp__snprintf            0000000039aa51c8     MSVCRT:MSVCR100.dll
 0002:000001d0       __imp_sprintf              0000000039aa51d0     MSVCRT:MSVCR100.dll
 0002:000001d8       __imp__time64              0000000039aa51d8     MSVCRT:MSVCR100.dll
 0002:000001e0       __imp_exit                 0000000039aa51e0     MSVCRT:MSVCR100.dll
 0002:000001e8       __imp_strncpy              0000000039aa51e8     MSVCRT:MSVCR100.dll
 0002:000001f0       __imp_wcsrchr              0000000039aa51f0     MSVCRT:MSVCR100.dll
 0002:000001f8       __imp__vscwprintf          0000000039aa51f8     MSVCRT:MSVCR100.dll
 0002:00000200       __imp__vsnwprintf          0000000039aa5200     MSVCRT:MSVCR100.dll
 0002:00000208       __imp_strstr               0000000039aa5208     MSVCRT:MSVCR100.dll
 0002:00000210       __imp_strpbrk              0000000039aa5210     MSVCRT:MSVCR100.dll
 0002:00000218       __imp_atol                 0000000039aa5218     MSVCRT:MSVCR100.dll
 0002:00000220       __imp__localtime64         0000000039aa5220     MSVCRT:MSVCR100.dll
 0002:00000228       __imp__localtime64_s       0000000039aa5228     MSVCRT:MSVCR100.dll
 0002:00000230       __imp__mktime64            0000000039aa5230     MSVCRT:MSVCR100.dll
 0002:00000238       __imp__vscprintf           0000000039aa5238     MSVCRT:MSVCR100.dll
 0002:00000240       __imp_vsnprintf            0000000039aa5240     MSVCRT:MSVCR100.dll
 0002:00000240       __imp__vsnprintf           0000000039aa5240     MSVCRT:MSVCR100.dll
 0002:00000248       __imp_fread                0000000039aa5248     MSVCRT:MSVCR100.dll
 0002:00000250       __imp_fseek                0000000039aa5250     MSVCRT:MSVCR100.dll
 0002:00000258       __imp_ftell                0000000039aa5258     MSVCRT:MSVCR100.dll
 0002:00000260       __imp_rand_s               0000000039aa5260     MSVCRT:MSVCR100.dll
 0002:00000268       __imp_strncpy_s            0000000039aa5268     MSVCRT:MSVCR100.dll
 0002:00000270       __imp_fclose               0000000039aa5270     MSVCRT:MSVCR100.dll
 0002:00000278       __imp_sscanf               0000000039aa5278     MSVCRT:MSVCR100.dll
 0002:00000280       __imp__strtoui64           0000000039aa5280     MSVCRT:MSVCR100.dll
 0002:00000288       __imp__i64toa_s            0000000039aa5288     MSVCRT:MSVCR100.dll
 0002:00000290       __imp__timezone            0000000039aa5290     MSVCRT:MSVCR100.dll
 0002:00000290       __imp_timezone             0000000039aa5290     MSVCRT:MSVCR100.dll
 0002:00000298       __imp__gcvt_s              0000000039aa5298     MSVCRT:MSVCR100.dll
 0002:000002a0       __imp_fopen                0000000039aa52a0     MSVCRT:MSVCR100.dll
 0002:000002a8       __imp_sprintf_s            0000000039aa52a8     MSVCRT:MSVCR100.dll
 0002:000002b0       __imp_strftime             0000000039aa52b0     MSVCRT:MSVCR100.dll
 0002:000002b8       __imp__itoa_s              0000000039aa52b8     MSVCRT:MSVCR100.dll
 0002:000002c0       __imp_strtoul              0000000039aa52c0     MSVCRT:MSVCR100.dll
 0002:000002c8       __imp___C_specific_handler 0000000039aa52c8     MSVCRT:MSVCR100.dll
 0002:000002d0       __imp__unlock              0000000039aa52d0     MSVCRT:MSVCR100.dll
 0002:000002d8       __imp___dllonexit          0000000039aa52d8     MSVCRT:MSVCR100.dll
 0002:000002e0       __imp__lock                0000000039aa52e0     MSVCRT:MSVCR100.dll
 0002:000002e8       __imp__onexit              0000000039aa52e8     MSVCRT:MSVCR100.dll
 0002:000002f0       __imp_vsnprintf_s          0000000039aa52f0     MSVCRT:MSVCR100.dll
 0002:000002f0       __imp__vsnprintf_s         0000000039aa52f0     MSVCRT:MSVCR100.dll
 0002:000002f8       __imp__malloc_crt          0000000039aa52f8     MSVCRT:MSVCR100.dll
 0002:00000300       __imp__initterm            0000000039aa5300     MSVCRT:MSVCR100.dll
 0002:00000308       __imp__initterm_e          0000000039aa5308     MSVCRT:MSVCR100.dll
 0002:00000310       __imp_free                 0000000039aa5310     MSVCRT:MSVCR100.dll
 0002:00000318       __imp__encoded_null        0000000039aa5318     MSVCRT:MSVCR100.dll
 0002:00000320       __imp__amsg_exit           0000000039aa5320     MSVCRT:MSVCR100.dll
 0002:00000328       __imp___CppXcptFilter      0000000039aa5328     MSVCRT:MSVCR100.dll
 0002:00000330       __imp___clean_type_info_names_internal 0000000039aa5330     MSVCRT:MSVCR100.dll
 0002:00000338       __imp_puts                 0000000039aa5338     MSVCRT:MSVCR100.dll
 0002:00000340       __imp_abort                0000000039aa5340     MSVCRT:MSVCR100.dll
 0002:00000348       __imp_memcpy               0000000039aa5348     MSVCRT:MSVCR100.dll
 0002:00000350       __imp_memmove              0000000039aa5350     MSVCRT:MSVCR100.dll
 0002:00000358       __imp__purecall            0000000039aa5358     MSVCRT:MSVCR100.dll
 0002:00000360       __imp_fputs                0000000039aa5360     MSVCRT:MSVCR100.dll
 0002:00000368       __imp_remove               0000000039aa5368     MSVCRT:MSVCR100.dll
 0002:00000370       __imp_clock                0000000039aa5370     MSVCRT:MSVCR100.dll
 0002:00000378       __imp__atoi64              0000000039aa5378     MSVCRT:MSVCR100.dll
 0002:00000380       __imp__gmtime64            0000000039aa5380     MSVCRT:MSVCR100.dll
 0002:00000388       __imp_isdigit              0000000039aa5388     MSVCRT:MSVCR100.dll
 0002:00000390       __imp_tolower              0000000039aa5390     MSVCRT:MSVCR100.dll
 0002:00000398       __imp_rand                 0000000039aa5398     MSVCRT:MSVCR100.dll
 0002:000003a0       __imp_srand                0000000039aa53a0     MSVCRT:MSVCR100.dll
 0002:000003a8       __imp__aligned_malloc      0000000039aa53a8     MSVCRT:MSVCR100.dll
 0002:000003b0       __imp_rename               0000000039aa53b0     MSVCRT:MSVCR100.dll
 0002:000003b8       __imp_memcmp               0000000039aa53b8     MSVCRT:MSVCR100.dll
 0002:000003c0       __imp__strlwr              0000000039aa53c0     MSVCRT:MSVCR100.dll
 0002:000003c8       __imp_isalnum              0000000039aa53c8     MSVCRT:MSVCR100.dll
 0002:000003d0       __imp_log                  0000000039aa53d0     MSVCRT:MSVCR100.dll
 0002:000003d8       __imp_exp                  0000000039aa53d8     MSVCRT:MSVCR100.dll
 0002:000003e0       __imp_fwrite               0000000039aa53e0     MSVCRT:MSVCR100.dll
 0002:000003e8       __imp_malloc               0000000039aa53e8     MSVCRT:MSVCR100.dll
 0002:000003f0       __imp_feof                 0000000039aa53f0     MSVCRT:MSVCR100.dll
 0002:000003f8       __imp_rewind               0000000039aa53f8     MSVCRT:MSVCR100.dll
 0002:00000400       __imp_strncat              0000000039aa5400     MSVCRT:MSVCR100.dll
 0002:00000408       __imp___crt_debugger_hook  0000000039aa5408     MSVCRT:MSVCR100.dll
 0002:00000410       __imp_strncmp              0000000039aa5410     MSVCRT:MSVCR100.dll
 0002:00000418       __imp_strcmpi              0000000039aa5418     MSVCRT:MSVCR100.dll
 0002:00000418       __imp__stricmp             0000000039aa5418     MSVCRT:MSVCR100.dll
 0002:00000420       __imp__strtoi64            0000000039aa5420     MSVCRT:MSVCR100.dll
 0002:00000428       __imp_fgets                0000000039aa5428     MSVCRT:MSVCR100.dll
 0002:00000430       __imp__strnicmp            0000000039aa5430     MSVCRT:MSVCR100.dll
 0002:00000430       __imp_strnicmp             0000000039aa5430     MSVCRT:MSVCR100.dll
 0002:00000438       __imp_isspace              0000000039aa5438     MSVCRT:MSVCR100.dll
 0002:00000440       __imp_atoi                 0000000039aa5440     MSVCRT:MSVCR100.dll
 0002:00000448       __imp_realloc              0000000039aa5448     MSVCRT:MSVCR100.dll
 0002:00000450       \177MSVCR100_NULL_THUNK_DATA 0000000039aa5450     MSVCRT:MSVCR100.dll
 0002:00000458       __imp_GetForegroundWindow  0000000039aa5458     user32:USER32.dll
 0002:00000460       __imp_GetDesktopWindow     0000000039aa5460     user32:USER32.dll
 0002:00000468       __imp_MessageBoxA          0000000039aa5468     user32:USER32.dll
 0002:00000470       \177USER32_NULL_THUNK_DATA 0000000039aa5470     user32:USER32.dll
 0002:00000478       __imp_getaddrinfo          0000000039aa5478     Ws2_32:WS2_32.dll
 0002:00000480       __imp_freeaddrinfo         0000000039aa5480     Ws2_32:WS2_32.dll
 0002:00000488       \177WS2_32_NULL_THUNK_DATA 0000000039aa5488     Ws2_32:WS2_32.dll
 0002:00000490       __imp_WSACleanup           0000000039aa5490     Wsock32:WSOCK32.dll
 0002:00000498       __imp_WSAStartup           0000000039aa5498     Wsock32:WSOCK32.dll
 0002:000004a0       __imp_gethostname          0000000039aa54a0     Wsock32:WSOCK32.dll
 0002:000004a8       __imp_WSAGetLastError      0000000039aa54a8     Wsock32:WSOCK32.dll
 0002:000004b0       __imp_bind                 0000000039aa54b0     Wsock32:WSOCK32.dll
 0002:000004b8       __imp_inet_addr            0000000039aa54b8     Wsock32:WSOCK32.dll
 0002:000004c0       __imp_gethostbyname        0000000039aa54c0     Wsock32:WSOCK32.dll
 0002:000004c8       __imp_sendto               0000000039aa54c8     Wsock32:WSOCK32.dll
 0002:000004d0       __imp_shutdown             0000000039aa54d0     Wsock32:WSOCK32.dll
 0002:000004d8       __imp_connect              0000000039aa54d8     Wsock32:WSOCK32.dll
 0002:000004e0       __imp_closesocket          0000000039aa54e0     Wsock32:WSOCK32.dll
 0002:000004e8       __imp_ioctlsocket          0000000039aa54e8     Wsock32:WSOCK32.dll
 0002:000004f0       __imp_recvfrom             0000000039aa54f0     Wsock32:WSOCK32.dll
 0002:000004f8       __imp_htonl                0000000039aa54f8     Wsock32:WSOCK32.dll
 0002:00000500       __imp_ntohl                0000000039aa5500     Wsock32:WSOCK32.dll
 0002:00000508       __imp_getsockname          0000000039aa5508     Wsock32:WSOCK32.dll
 0002:00000510       __imp_ntohs                0000000039aa5510     Wsock32:WSOCK32.dll
 0002:00000518       __imp_inet_ntoa            0000000039aa5518     Wsock32:WSOCK32.dll
 0002:00000520       __imp_htons                0000000039aa5520     Wsock32:WSOCK32.dll
 0002:00000528       __imp_recv                 0000000039aa5528     Wsock32:WSOCK32.dll
 0002:00000530       __imp_select               0000000039aa5530     Wsock32:WSOCK32.dll
 0002:00000538       __imp___WSAFDIsSet         0000000039aa5538     Wsock32:WSOCK32.dll
 0002:00000540       __imp_send                 0000000039aa5540     Wsock32:WSOCK32.dll
 0002:00000548       __imp_socket               0000000039aa5548     Wsock32:WSOCK32.dll
 0002:00000550       __imp_setsockopt           0000000039aa5550     Wsock32:WSOCK32.dll
 0002:00000558       \177WSOCK32_NULL_THUNK_DATA 0000000039aa5558     Wsock32:WSOCK32.dll
 0002:00000560       __imp_CoUninitialize       0000000039aa5560     ole32:ole32.dll
 0002:00000568       __imp_CoInitialize         0000000039aa5568     ole32:ole32.dll
 0002:00000570       \177ole32_NULL_THUNK_DATA  0000000039aa5570     ole32:ole32.dll
 0002:00000578       __xc_a                     0000000039aa5578     MSVCRT:cinitexe.obj
 0002:000006f8       __xc_z                     0000000039aa56f8     MSVCRT:cinitexe.obj
 0002:00000700       __xi_a                     0000000039aa5700     MSVCRT:cinitexe.obj
 0002:00000710       __xi_z                     0000000039aa5710     MSVCRT:cinitexe.obj
 0002:0000073c       ??_C@_02DKCKIIND@?$CFs?$AA@ 0000000039aa573c     CryDedicatedServer.obj
 0002:00000740       ??_C@_0CI@IOKCCNHB@Deleting?5Reference?5Counted?5Objec@ 0000000039aa5740     CryDedicatedServer.obj
 0002:00000768       ??_7IJob@CWorkQueue@@6B@   0000000039aa5768     CryDLCStore.obj
 0002:00000780       ??_7IMemReplay@@6B@        0000000039aa5780     CryDLCStore.obj
 0002:000008b0       ??_C@_0P@PCJPAHLM@out?5of?5memory?6?$AA@ 0000000039aa58b0     CryDLCStore.obj
 0002:000008c0       ??_C@_06NBFPPGEG@vector?$AA@ 0000000039aa58c0     CryDLCStore.obj
 0002:000008d0       ??_7CDummyMemReplay@@6B@   0000000039aa58d0     CryDLCStore.obj
 0002:00000a00       ??_C@_0BK@KIDLLGKF@?$FLLobby?$FNTry?5cancel?5task?5?$CFd?$AA@ 0000000039aa5a00     CryDLCStore.obj
 0002:00000a20       ??_7CCryDLCStore@@6BICryDLCStore@@@ 0000000039aa5a20     CryDLCStore.obj
 0002:00000b10       ??_7CCryDLCStore@@6BCMultiThreadRefCount@@@ 0000000039aa5b10     CryDLCStore.obj
 0002:00000b80       ??_7CCryFriends@@6BICryFriends@@@ 0000000039aa5b80     CryFriends.obj
 0002:00000b98       ??_7CCryFriends@@6BCMultiThreadRefCount@@@ 0000000039aa5b98     CryFriends.obj
 0002:00000bc0       ??_C@_0BJ@ENIGCEJG@?$FLLobby?$FN?5Task?5?$CFd?5canceled?$AA@ 0000000039aa5bc0     CryFriends.obj
 0002:00000be0       ??_7ICryFriendsManagement@@6B@ 0000000039aa5be0     CryFriendsManagement.obj
 0002:00000c50       ??_7CCryFriendsManagement@@6BICryFriendsManagement@@@ 0000000039aa5c50     CryFriendsManagement.obj
 0002:00000cc0       ??_7CCryFriendsManagement@@6BCMultiThreadRefCount@@@ 0000000039aa5cc0     CryFriendsManagement.obj
 0002:00000cd8       ??_C@_0CC@OJJLEFLK@gSPyI9?$CC?B?$KD$h83H8Uasd73nn?$CI?$CJu12gh?$FL?$FL@ 0000000039aa5cd8     CryLobby.obj
 0002:00000d00       ??_7ICryLobby@@6B@         0000000039aa5d00     CryLobby.obj
 0002:00000de0       ??_7ICryLobbyService@@6B@  0000000039aa5de0     CryLobby.obj
 0002:00000e70       ??_C@_0BH@NJHHGFMG@net_lobby_default_port?$AA@ 0000000039aa5e70     CryLobby.obj
 0002:00000e88       ??_C@_0P@EMMOIPDD@?$CFi?4?$CFi?4?$CFi?4?$CFi?3?$CFi?$AA@ 0000000039aa5e88     CryLobby.obj
 0002:00000e98       ??_C@_0M@OPOCDNEK@?$CFi?4?$CFi?4?$CFi?4?$CFi?$AA@ 0000000039aa5e98     CryLobby.obj
 0002:00000eb0       ??_C@_0ED@CJJCEIAN@CryLobbyID?5is?5being?5constructed?5@ 0000000039aa5eb0     CryLobby.obj
 0002:00000ef8       ??_7?$SAbstractVisitDeclarator@AEBG@NConfigurableVariantHelpers@@6B@ 0000000039aa5ef8     CryLobby.obj
 0002:00000ef8       ??_7?$SAbstractVisitDeclarator@AEBUSIPv4Addr@@@NConfigurableVariantHelpers@@6B@ 0000000039aa5ef8     CryLobby.obj
 0002:00000ef8       ??_7?$SAbstractVisitDeclarator@AEBUSNullAddr@@@NConfigurableVariantHelpers@@6B@ 0000000039aa5ef8     CryLobby.obj
 0002:00000ef8       ??_7ISystemEventListener@@6B@ 0000000039aa5ef8     CryLobbyDLL.obj
 0002:00000ef8       ??_7?$SAbstractVisitDeclarator@AEBULobbyIdAddr@@@NConfigurableVariantHelpers@@6B@ 0000000039aa5ef8     CryLobby.obj
 0002:00000f08       ??_C@_0DH@NHMABMAP@CLobby?3?3CCachedPacketBuffer?5high@ 0000000039aa5f08     CryLobby.obj
 0002:00000f40       __real@447a0000            0000000039aa5f40     CryLobby.obj
 0002:00000f44       __real@00000000            0000000039aa5f44     CryLobby.obj
 0002:00000f48       ??_C@_0DC@LKPPOAEB@?$FLLobby?$FN?5Generating?5random?5eCLE_T@ 0000000039aa5f48     CryLobby.obj
 0002:00000f80       ??_C@_0CA@MEGFFFAJ@?$FLLobby?$FN?5Delayed?5task?5?$CFd?5started?$AA@ 0000000039aa5f80     CryLobby.obj
 0002:00000fa0       ??_C@_0DC@OGGBLKAN@?$FLLobby?$FN?5Delay?5start?5task?5?$CFd?5for?5@ 0000000039aa5fa0     CryLobby.obj
 0002:00000fd8       ??_C@_0CA@GNJKMGIG@?$FLLobby?$FN?5Delayed?5task?5?$CFd?5ticking?$AA@ 0000000039aa5fd8     CryLobby.obj
 0002:00000ff8       ??_C@_0DK@OGCKFJGH@?$FLLobby?$FN?5Delay?5start?5ticking?5task@ 0000000039aa5ff8     CryLobby.obj
 0002:00001040       ??_7CCryLobbyService@@6BICryLobbyService@@@ 0000000039aa6040     CryLobby.obj
 0002:000010d0       ??_7CCryLobbyService@@6BCMultiThreadRefCount@@@ 0000000039aa60d0     CryLobby.obj
 0002:00001128       ??_C@_0DP@LDPNJJIE@CryLobbyIDArray?5is?5being?5indexed@ 0000000039aa6128     CryLobby.obj
 0002:00001168       ??_7?$CClassJobNoRef@IVCCryLobbyService@@@CWorkQueue@@6B@ 0000000039aa6168     CryLobby.obj
 0002:00001168       ??_7?$CClassJobNoRef@IVCCryGameSpySBQR2LobbyService@@@CWorkQueue@@6B@ 0000000039aa6168     CryGameSpySBQR2Lobby.obj
 0002:00001180       ??_C@_0GJ@NMNAMLII@CCachedPacketBuffer?3?3WritePacket@ 0000000039aa6180     CryLobby.obj
 0002:000011f0       ??_C@_09KOIOCIHC@?$DMUNKNOWN?$DO?$AA@ 0000000039aa61f0     CryLobby.obj
 0002:00001200       ??_C@_0BL@PPGFBDEF@?5?5?5?5packet?5?$CFd?5?$CI?$CFd?$CJ?5size?5?$CFd?$AA@ 0000000039aa6200     CryLobby.obj
 0002:00001220       ??_C@_0CL@NOIFNGBK@?$FLLobby?$FN?5Lobby?5Service?5EndTask?5?$CFd@ 0000000039aa6220     CryLobby.obj
 0002:00001250       ??_C@_0DF@NFKCPHPH@Name?5resolution?5for?5?8?$CFs?8?5failed?5@ 0000000039aa6250     CryLobby.obj
 0002:00001288       ??_C@_0DJ@HPNHKBLE@Address?5to?5bind?5?8?$CFs?8?5does?5not?5ap@ 0000000039aa6288     CryLobby.obj
 0002:000012c4       ??_C@_05HKPGCKL@?$CFs?3?$CFd?$AA@ 0000000039aa62c4     CryLobby.obj
 0002:000012d0       ??_C@_07CMGGDNPL@sv_bind?$AA@ 0000000039aa62d0     CryLobby.obj
 0002:000012d8       ??_C@_0L@LLCOMNCF@0?40?40?40?3?$CFd?$AA@ 0000000039aa62d8     CryLobby.obj
 0002:000012e8       ??_C@_0CH@FCPHILED@?$FLLobby?$FN?5Terminate?5service?5?$CFd?5err@ 0000000039aa62e8     CryLobby.obj
 0002:00001310       ??_C@_0DD@FBEPBICC@?$FLlobby?$FN?5Create?5reliable?5connecti@ 0000000039aa6310     CryLobby.obj
 0002:00001350       ??_C@_0EL@DNHJGLKG@RefCount?5of?5connection?5lcid?5?$CFd?5a@ 0000000039aa6350     CryLobby.obj
 0002:000013a0       ??_C@_0BD@MGAOJKCH@counter?5?$CFd?5size?5?$CFd?$AA@ 0000000039aa63a0     CryLobby.obj
 0002:000013c0       ??_C@_0FA@KAEEEGCI@?$FLLobby?$FN?5Trying?5to?5send?5to?5connec@ 0000000039aa63c0     CryLobby.obj
 0002:00001410       ??_C@_0EO@LHJCBDII@RefCount?5of?5connection?5lcid?5?$CFd?5a@ 0000000039aa6410     CryLobby.obj
 0002:00001460       ??_C@_0CL@OFPOKMKP@?$FLlobby?$FN?5Release?5connection?5lcid?5@ 0000000039aa6460     CryLobby.obj
 0002:00001490       ??_C@_0CE@JJJLEFDC@?$FLLobby?$FN?5Keep?5packet?5?$CFd?5?$CI?$CFd?$CJ?5Size@ 0000000039aa6490     CryLobby.obj
 0002:000014b8       ??_C@_0CB@HFDFNKLG@?$FLLobby?$FN?5Remove?5packet?5?$CFd?5Size?5?$CFd@ 0000000039aa64b8     CryLobby.obj
 0002:000014e0       ??_C@_0CB@FINBGIDI@?$FLLobby?$FN?5?$CFd?5packets?5in?5send?5queue@ 0000000039aa64e0     CryLobby.obj
 0002:00001510       ??_C@_0EL@JGKPAFKL@RefCount?5of?5connection?5lcid?5?$CFd?5a@ 0000000039aa6510     CryLobby.obj
 0002:00001560       ??_C@_0CC@OPBFEGDI@?$FLLobby?$FN?5Created?5socket?5on?5port?5?$CF@ 0000000039aa6560     CryLobby.obj
 0002:00001588       ??_C@_0CD@KACCGBIE@?$FLLobby?$FN?5Creating?5socket?5on?5port?5@ 0000000039aa6588     CryLobby.obj
 0002:000015b0       ??_C@_0CL@FNOOPFJL@?$FLLobby?$FN?5Failed?5to?5create?5socket?5@ 0000000039aa65b0     CryLobby.obj
 0002:000015e0       ??_C@_0EH@OEGCKMND@?$FLLobby?$FN?5Creating?5socket?5on?5port?5@ 0000000039aa65e0     CryLobby.obj
 0002:00001628       ??_C@_03BANLECBK@LAN?$AA@  0000000039aa6628     CryLobby.obj
 0002:0000162c       ??_C@_06KCABBADG@Online?$AA@ 0000000039aa662c     CryLobby.obj
 0002:00001638       ??_7CCryLobby@@6BIDatagramListener@@@ 0000000039aa6638     CryLobby.obj
 0002:00001650       ??_7CCryLobby@@6BICryLobby@@@ 0000000039aa6650     CryLobby.obj
 0002:00001748       ??_C@_0CI@EIILMEMD@?$FLLobby?$FN?5Initialise?5service?5?$CFd?5er@ 0000000039aa6748     CryLobby.obj
 0002:00001770       ??_7?$CVisitor@V?$CNode@USNullAddr@@V?$CNode@GV?$CNode@USIPv4Addr@@V?$CNode@ULobbyIdAddr@@VCEnd@NTypelist@@@NTypelist@@@NTypelist@@@NTypelist@@@NTypelist@@VCComparatorVisitor@?$less@V?$CConfigurableVariant@V?$CNode@USNullAddr@@V?$CNode@GV?$CNode@USIPv4Addr@@V?$CNode@ULobbyIdAddr@@VCEnd@NTypelist@@@NTypelist@@@NTypelist@@@NTypelist@@@NTypelist@@$07VCDefaultVariantConversion@NConfigurableVariantHelpers@@VCDefaultVariantConstruction@4@@@@stlpmtx_std@@U?$IVisitor@V?$CNode@USNullAddr@@V?$CNode@GV?$CNode@USIPv4Addr@@V?$CNode@ULobbyIdAddr@@VCEnd@NTypelist@@@NTypelist@@@NTypelist@@@NTypelist@@@NTypelist@@@NConfigurableVariantHelpers@@@NConfigurableVariantHelpers@@6B?$IVisitor@V?$CNode@ULobbyIdAddr@@VCEnd@NTypelist@@@NTypelist@@@1@@ 0000000039aa6770     CryLobby.obj
 0002:00001780       ??_7?$CVisitor@V?$CNode@USNullAddr@@V?$CNode@GV?$CNode@USIPv4Addr@@V?$CNode@ULobbyIdAddr@@VCEnd@NTypelist@@@NTypelist@@@NTypelist@@@NTypelist@@@NTypelist@@VCComparatorVisitor@?$less@V?$CConfigurableVariant@V?$CNode@USNullAddr@@V?$CNode@GV?$CNode@USIPv4Addr@@V?$CNode@ULobbyIdAddr@@VCEnd@NTypelist@@@NTypelist@@@NTypelist@@@NTypelist@@@NTypelist@@$07VCDefaultVariantConversion@NConfigurableVariantHelpers@@VCDefaultVariantConstruction@4@@@@stlpmtx_std@@U?$IVisitor@V?$CNode@USNullAddr@@V?$CNode@GV?$CNode@USIPv4Addr@@V?$CNode@ULobbyIdAddr@@VCEnd@NTypelist@@@NTypelist@@@NTypelist@@@NTypelist@@@NTypelist@@@NConfigurableVariantHelpers@@@NConfigurableVariantHelpers@@6B?$SAbstractVisitDeclarator@AEBUSIPv4Addr@@@1@@ 0000000039aa6780     CryLobby.obj
 0002:00001790       ??_7?$CVisitor@V?$CNode@USNullAddr@@V?$CNode@GV?$CNode@USIPv4Addr@@V?$CNode@ULobbyIdAddr@@VCEnd@NTypelist@@@NTypelist@@@NTypelist@@@NTypelist@@@NTypelist@@VCComparatorVisitor@?$less@V?$CConfigurableVariant@V?$CNode@USNullAddr@@V?$CNode@GV?$CNode@USIPv4Addr@@V?$CNode@ULobbyIdAddr@@VCEnd@NTypelist@@@NTypelist@@@NTypelist@@@NTypelist@@@NTypelist@@$07VCDefaultVariantConversion@NConfigurableVariantHelpers@@VCDefaultVariantConstruction@4@@@@stlpmtx_std@@U?$IVisitor@V?$CNode@USNullAddr@@V?$CNode@GV?$CNode@USIPv4Addr@@V?$CNode@ULobbyIdAddr@@VCEnd@NTypelist@@@NTypelist@@@NTypelist@@@NTypelist@@@NTypelist@@@NConfigurableVariantHelpers@@@NConfigurableVariantHelpers@@6B?$IVisitor@V?$CNode@GV?$CNode@USIPv4Addr@@V?$CNode@ULobbyIdAddr@@VCEnd@NTypelist@@@NTypelist@@@NTypelist@@@NTypelist@@@1@@ 0000000039aa6790     CryLobby.obj
 0002:000017a0       ??_7?$CVisitor@V?$CNode@USNullAddr@@V?$CNode@GV?$CNode@USIPv4Addr@@V?$CNode@ULobbyIdAddr@@VCEnd@NTypelist@@@NTypelist@@@NTypelist@@@NTypelist@@@NTypelist@@VCComparatorVisitor@?$less@V?$CConfigurableVariant@V?$CNode@USNullAddr@@V?$CNode@GV?$CNode@USIPv4Addr@@V?$CNode@ULobbyIdAddr@@VCEnd@NTypelist@@@NTypelist@@@NTypelist@@@NTypelist@@@NTypelist@@$07VCDefaultVariantConversion@NConfigurableVariantHelpers@@VCDefaultVariantConstruction@4@@@@stlpmtx_std@@U?$IVisitor@V?$CNode@USNullAddr@@V?$CNode@GV?$CNode@USIPv4Addr@@V?$CNode@ULobbyIdAddr@@VCEnd@NTypelist@@@NTypelist@@@NTypelist@@@NTypelist@@@NTypelist@@@NConfigurableVariantHelpers@@@NConfigurableVariantHelpers@@6B?$SAbstractVisitDeclarator@AEBUSNullAddr@@@1@@ 0000000039aa67a0     CryLobby.obj
 0002:000017b0       ??_C@_0EK@KEBLADP@Trying?5to?5create?5a?5lobby?5when?5we@ 0000000039aa67b0     CryLobby.obj
 0002:00001800       ??_C@_0FA@GBLNPGEL@?$FLLobby?$FN?5Failed?5to?5send?5setting?5c@ 0000000039aa6800     CryLobby.obj
 0002:00001850       ??_C@_0EE@GLMKIOI@?$FLlobby?$FN?5Send?5reliable?5connection@ 0000000039aa6850     CryLobby.obj
 0002:000018a0       ??_C@_0FA@JLPNKEIB@?$FLlobby?$FN?5Socket?5error?5?$CFd?5on?5conne@ 0000000039aa68a0     CryLobby.obj
 0002:000018f0       ??_C@_0EO@BGMNJBFK@?$FLlobby?$FN?5Send?5complete?5on?5connect@ 0000000039aa68f0     CryLobby.obj
 0002:00001940       ??_C@_0DP@MDBHJNGH@?$FLLobby?$FN?5Setting?5recvCookie?5?$CFllx?5@ 0000000039aa6940     CryLobby.obj
 0002:00001980       ??_C@_0DM@FFCFBEAE@?$FLLobby?$FN?5Sending?5cookie?5?$CFllx?5with@ 0000000039aa6980     CryLobby.obj
 0002:000019c0       ??_C@_0DM@FJGMAHHD@?$FLLobby?$FN?5setting?5refCount?5back?5to@ 0000000039aa69c0     CryLobby.obj
 0002:00001a00       ??_C@_0IE@JKIMNNDO@?$FLLobby?$FN?5Connection?5Request?5on?5ex@ 0000000039aa6a00     CryLobby.obj
 0002:00001a90       ??_C@_0EK@LMFDBLMK@?$FLLobby?$FN?5Connection?5Request?5on?5ex@ 0000000039aa6a90     CryLobby.obj
 0002:00001ae0       ??_C@_0EM@EHOAOJDL@?$FLlobby?$FN?5Got?5ack?5on?5connection?5lc@ 0000000039aa6ae0     CryLobby.obj
 0002:00001b30       ??_C@_0DL@LFMHMANL@?$FLlobby?$FN?5Send?5ack?5for?5non?5connect@ 0000000039aa6b30     CryLobby.obj
 0002:00001b70       ??_C@_0DE@CLCDKCCL@?5?5?5?5Ignoring?5packet?5?$CFd?5?$CI?$CFd?$CJ?5size@ 0000000039aa6b70     CryLobby.obj
 0002:00001ba8       ??_C@_0DF@OLMNCCIN@?5?5?5?5Ignoring?5packet?5?$CFd?5?$CI?$CFd?$CJ?5size@ 0000000039aa6ba8     CryLobby.obj
 0002:00001be0       ??_C@_0FP@LGODLNLE@?$FLlobby?$FN?5OnPacket?5reliable?5packet@ 0000000039aa6be0     CryLobby.obj
 0002:00001c40       ??_C@_0CD@DIOLLNFJ@?5?5?5?5Process?5packet?5?$CFd?5?$CI?$CFd?$CJ?5size?5@ 0000000039aa6c40     CryLobby.obj
 0002:00001c68       ??_C@_0BO@LAIJDFBG@?$FLlobby?$FN?5Send?5ack?5?$CIcounter?$DN?$CFu?$CJ?$AA@ 0000000039aa6c68     CryLobby.obj
 0002:00001c88       ??_C@_0CB@CDILAOAC@?$FLlobby?$FN?5Repeat?5packet?5counter?5?$CFd@ 0000000039aa6c88     CryLobby.obj
 0002:00001cb0       ??_C@_0FD@BFEEGKKG@?$FLlobby?$FN?5Got?5ack?$CIfirst?$CJ?5on?5connec@ 0000000039aa6cb0     CryLobby.obj
 0002:00001d08       ??_C@_0BO@DAEDKAEA@?$FLlobby?$FN?5New?5packet?5counter?5?$CFd?$AA@ 0000000039aa6d08     CryLobby.obj
 0002:00001d28       ??_C@_0DN@JMCPDJKE@?$FLlobby?$FN?5OnPacket?5reliable?5connec@ 0000000039aa6d28     CryLobby.obj
 0002:00001d70       ??_C@_0EJ@MBJMMNBM@?$FLLobby?$FN?5Setting?5freeing?5connecti@ 0000000039aa6d70     CryLobby.obj
 0002:00001dc0       ??_C@_0FJ@DCLHJKAC@?$FLlobby?$FN?5Send?5reliable?5connection@ 0000000039aa6dc0     CryLobby.obj
 0002:00001e20       ??_C@_0HK@CPAFIMLJ@?$FLLobby?$FN?5Connection?5to?5lcid?5?$CFd?5ad@ 0000000039aa6e20     CryLobby.obj
 0002:00001ea0       ??_C@_0FI@CDGDHOP@?$FLLobby?$FN?5Failed?5to?5send?5setting?5p@ 0000000039aa6ea0     CryLobby.obj
 0002:00001f00       ??_C@_0EP@OOBHODCP@?$FLLobby?$FN?5Sending?5connection?5reque@ 0000000039aa6f00     CryLobby.obj
 0002:00001f50       ??_C@_0GH@HJNEAHNC@?$FLLobby?$FN?5No?5references?5to?5connect@ 0000000039aa6f50     CryLobby.obj
 0002:00001fc0       ??_C@_0FK@HNJPBJJC@?$FLLobby?$FN?5Failed?5to?5send?5setting?5c@ 0000000039aa6fc0     CryLobby.obj
 0002:00002020       ??_C@_0EB@LEFNIPPJ@CCryLobby?3?3TimerCallback?$CI?$CJ?5long?5@ 0000000039aa7020     CryLobby.obj
 0002:00002061       ??_C@_00CNPNBAHC@?$AA@     0000000039aa7061     CryLobbyDLL.obj
 0002:00002064       ??_C@_04LOAJBDKD@true?$AA@ 0000000039aa7064     CryLobbyDLL.obj
 0002:0000206c       ??_C@_01HIHLOKLC@1?$AA@    0000000039aa706c     CryLobbyDLL.obj
 0002:00002070       ??_C@_05LAPONLG@false?$AA@ 0000000039aa7070     CryLobbyDLL.obj
 0002:00002078       ??_C@_01GBGANLPD@0?$AA@    0000000039aa7078     CryLobbyDLL.obj
 0002:0000207c       __real@41200000            0000000039aa707c     CryLobbyDLL.obj
 0002:00002080       ??_C@_0DJ@DLJMMMP@Could?5not?5access?5CrySystem?4dll?5?$CI@ 0000000039aa7080     CryLobbyDLL.obj
 0002:000020c0       ??_C@_0P@NHEMOHAI@Memory?5Manager?$AA@ 0000000039aa70c0     CryLobbyDLL.obj
 0002:000020d0       ??_C@_0O@FFDHMLKN@CrySystem?4dll?$AA@ 0000000039aa70d0     CryLobbyDLL.obj
 0002:000020e0       ??_C@_0BO@JDKBDPNB@CryGetIMemoryManagerInterface?$AA@ 0000000039aa70e0     CryLobbyDLL.obj
 0002:00002100       ??_C@_0BB@PNKHDABP@CrySystemCrtFree?$AA@ 0000000039aa7100     CryLobbyDLL.obj
 0002:00002118       ??_C@_0BB@MFMFBMDO@CrySystemCrtSize?$AA@ 0000000039aa7118     CryLobbyDLL.obj
 0002:00002130       ??_C@_0BD@BBIFHONI@CrySystemCrtMalloc?$AA@ 0000000039aa7130     CryLobbyDLL.obj
 0002:00002148       ??_C@_0O@LCCIKADF@CryGetMemSize?$AA@ 0000000039aa7148     CryLobbyDLL.obj
 0002:00002158       ??_C@_07CKAGCLEE@CryFree?$AA@ 0000000039aa7158     CryLobbyDLL.obj
 0002:00002160       ??_C@_0L@FICCDMFO@CryRealloc?$AA@ 0000000039aa7160     CryLobbyDLL.obj
 0002:00002170       ??_C@_09MCKPOEAK@CryMalloc?$AA@ 0000000039aa7170     CryLobbyDLL.obj
 0002:00002180       ??_7ICryUnknown@@6B@       0000000039aa7180     CryLobbyDLL.obj
 0002:000021a0       ?iid@?1??IID@ICryUnknown@@CAAEBUCryGUID@@XZ@4U3@B 0000000039aa71a0     CryLobbyDLL.obj
 0002:000021b0       ?iid@?1??IID@IEngineModule@@CAAEBUCryGUID@@XZ@4U3@B 0000000039aa71b0     CryLobbyDLL.obj
 0002:000021c0       ??_7ICryFactory@@6B@       0000000039aa71c0     CryLobbyDLL.obj
 0002:000021f0       ??_C@_0BD@PJOKHJBB@Pure?5function?5call?$AA@ 0000000039aa71f0     CryLobbyDLL.obj
 0002:00002208       ??_C@_0CL@LKHBOBAH@Invalid?5parameter?5detected?5in?5CR@ 0000000039aa7208     CryLobbyDLL.obj
 0002:00002238       ??_C@_0BO@HAMEIFMK@Critical?5Section?5hanging?5lock?$AA@ 0000000039aa7238     CryLobbyDLL.obj
 0002:00002258       ??_7CSystemEventListner_CryLobby@@6B@ 0000000039aa7258     CryLobbyDLL.obj
 0002:00002268       ??_7CEngineModule_CryLobby@@6B@ 0000000039aa7268     CryLobbyDLL.obj
 0002:000022a0       ??_C@_08COBFBPHE@CryLobby?$AA@ 0000000039aa72a0     CryLobbyDLL.obj
 0002:000022b0       ??_C@_09BHIABECK@CryEngine?$AA@ 0000000039aa72b0     CryLobbyDLL.obj
 0002:000022bc       ??_C@_06ICGJLFIM@string?$AA@ 0000000039aa72bc     CryLobbyDLL.obj
 0002:000022c8       ??_7CFactory@CEngineModule_CryLobby@@6B@ 0000000039aa72c8     CryLobbyDLL.obj
 0002:000022f8       ??_7bad_alloc@std@@6B@     0000000039aa72f8     CryLobbyDLL.obj
 0002:00002308       ??_C@_0P@GHFPNOJB@bad?5allocation?$AA@ 0000000039aa7308     CryLobbyDLL.obj
 0002:00002318       ??_C@_0BG@BENKABNO@EngineModule_CryLobby?$AA@ 0000000039aa7318     CryLobbyDLL.obj
 0002:00002330       ?cid@?1??GetClassID@CFactory@CEngineModule_CryLobby@@UEBAAEBUCryGUID@@XZ@4U4@B 0000000039aa7330     CryLobbyDLL.obj
 0002:00002340       ??_7sp_counted_base@detail@boost@@6B@ 0000000039aa7340     CryLobbyDLL.obj
 0002:00002360       ??_7?$sp_counted_impl_p@VCEngineModule_CryLobby@@@detail@boost@@6B@ 0000000039aa7360     CryLobbyDLL.obj
 0002:00002380       ??_C@_0BN@FOKPCDPC@Boost?5threw?5an?5exception?3?5?$CFs?$AA@ 0000000039aa7380     CryLobbyDLL.obj
 0002:000023a0       ??_C@_03JBIPMCLC@int?$AA@  0000000039aa73a0     CryLobbyDLL.obj
 0002:000023a4       ??_C@_01PKGAHCOL@?$CJ?$AA@ 0000000039aa73a4     CryLobbyDLL.obj
 0002:000023a8       ??_C@_01ODHLEDKK@?$CI?$AA@ 0000000039aa73a8     CryLobbyDLL.obj
 0002:000023ac       ??_C@_01IHBHIGKO@?0?$AA@   0000000039aa73ac     CryLobbyDLL.obj
 0002:000023b0       ??_C@_01FHEEJDEE@A?$AA@    0000000039aa73b0     CryLobbyDLL.obj
 0002:000023c0       ??_7CCryLobbyUI@@6BICryLobbyUI@@@ 0000000039aa73c0     CryLobbyUI.obj
 0002:00002420       ??_7CCryLobbyUI@@6BCMultiThreadRefCount@@@ 0000000039aa7420     CryLobbyUI.obj
 0002:00002420       ??_7CCryGameSpySBQR2LobbyUI@@6BCMultiThreadRefCount@@@ 0000000039aa7420     CryGameSpySBQR2LobbyUI.obj
 0002:00002430       ??_7ICryMatchMaking@@6B@   0000000039aa7430     CryMatchMaking.obj
 0002:000025d8       ??_C@_0CD@IBAPCJKA@connect?5?$DMsession?$DO?$CFd?0?$CFd?4?$CFd?4?$CFd?4?$CFd?3@ 0000000039aa75d8     CryMatchMaking.obj
 0002:00002600       ??_C@_0M@PCENNPGA@?$CFd?4?$CFd?4?$CFd?4?$CFd?$AA@ 0000000039aa7600     CryMatchMaking.obj
 0002:0000260c       __real@3727c5ac            0000000039aa760c     CryMatchMaking.obj
 0002:00002610       ??_C@_0CA@CNBPBDJK@?$FLLobby?$FN?5?$CFs?5ERROR?5invalid?5packet?$AA@ 0000000039aa7610     CryMatchMaking.obj
 0002:00002630       ??_C@_0CB@JPHEDBC@?$FLMatchmaking?$FN?3?5Too?5many?5tasks?4?4?4@ 0000000039aa7630     CryMatchMaking.obj
 0002:00002658       ??_C@_0CP@MMMFEPOD@?$FLMatchmaking?$FN?3?5task?5?$FL?$CFi?$FN?0?5starte@ 0000000039aa7658     CryMatchMaking.obj
 0002:00002688       ??_C@_0CJ@DMMIMJKJ@?$FLMatchmaking?$FN?3?5Trying?5to?5start?5t@ 0000000039aa7688     CryMatchMaking.obj
 0002:000026b8       ??_7?$CClassJobNoRef3@IIIVCCryGameSpySBQR2MatchMaking@@@CWorkQueue@@6B@ 0000000039aa76b8     CryGameSpySBQR2MatchMaking.obj
 0002:000026b8       ??_7?$CClassJobNoRef3@IIIVCCryMatchMaking@@@CWorkQueue@@6B@ 0000000039aa76b8     CryMatchMaking.obj
 0002:000026b8       ??_7?$CClassJobNoRef3@IIV?$CryLobbyID@USCryLobbySessionHandle@@$03@@VCCryMatchMaking@@@CWorkQueue@@6B@ 0000000039aa76b8     CryMatchMaking.obj
 0002:000026c8       ??_7?$CClassJobNoRef4@IIV?$CryLobbyID@USCryLobbySessionHandle@@$03@@USCryMatchMakingConnectionUID@@VCCryMatchMaking@@@CWorkQueue@@6B@ 0000000039aa76c8     CryMatchMaking.obj
 0002:000026d8       ??_7?$CClassJobNoRef2@W4ECryLobbySystemEvent@@IVCCryMatchMaking@@@CWorkQueue@@6B@ 0000000039aa76d8     CryMatchMaking.obj
 0002:000026d8       ??_7?$CClassJobNoRef2@IW4ECryLobbySystemEvent@@VCCryMatchMaking@@@CWorkQueue@@6B@ 0000000039aa76d8     CryMatchMaking.obj
 0002:000026e8       ??_7?$CClassJob@XVCCryMatchMaking@@@CWorkQueue@@6B@ 0000000039aa76e8     CryMatchMaking.obj
 0002:000026f8       __real@3f000000            0000000039aa76f8     CryMatchMaking.obj
 0002:000026fc       __real@3f800000            0000000039aa76fc     CryMatchMaking.obj
 0002:00002700       __real@41700000            0000000039aa7700     CryMatchMaking.obj
 0002:00002704       __real@43960000            0000000039aa7704     CryMatchMaking.obj
 0002:00002708       __real@3fc00000            0000000039aa7708     CryMatchMaking.obj
 0002:0000270c       __real@43af0000            0000000039aa770c     CryMatchMaking.obj
 0002:00002710       ??_C@_0CB@GINNBEOB@?$FLLobby?$FN?5EndTask?5?$CFd?5?$CI?$CFd?$CJ?5error?5?$CFd@ 0000000039aa7710     CryMatchMaking.obj
 0002:00002740       ??_C@_0EG@GFNNDIBN@?$FLLobby?$FN?5Free?5connection?5called?5w@ 0000000039aa7740     CryMatchMaking.obj
 0002:00002790       ??_C@_0EE@BPNDELBK@?$FLLobby?$FN?5Free?5connection?5session?5@ 0000000039aa7790     CryMatchMaking.obj
 0002:000027e0       ??_C@_0EC@MLOLGIHB@?$FLMatchMaking?$FN?3?5Setting?5local?5fla@ 0000000039aa77e0     CryMatchMaking.obj
 0002:00002828       ??_C@_0BH@BOBLBNH@?5?$CFc?5?5?5?$CF02i?5?5?$CF?916lld?5?$CFs?$AA@ 0000000039aa7828     CryMatchMaking.obj
 0002:00002840       ??_C@_0BP@LKBJCAKN@?5?5?5LCxID?5UserID?5?5?5?5?5?5?5?5?5?5?5Name?$AA@ 0000000039aa7840     CryMatchMaking.obj
 0002:00002860       ??_C@_0BC@OOICEFOP@?5Session?3?5?$CFi?5?$CI?$CFs?$CJ?$AA@ 0000000039aa7860     CryMatchMaking.obj
 0002:00002874       ??_C@_06DCBACPNP@CLIENT?$AA@ 0000000039aa7874     CryMatchMaking.obj
 0002:00002880       ??_C@_0DN@GJNGJFP@?9?9?9?9?9?9?9?9?9?9?9?9?9?9?9?9?9?9?9?9?9?9?9?9?9?9?9?9?9?9?9?9@ 0000000039aa7880     CryMatchMaking.obj
 0002:000028c0       ??_C@_06HNFCPEFM@SERVER?$AA@ 0000000039aa78c0     CryMatchMaking.obj
 0002:000028c8       ??_C@_0DM@NDNFFNFH@name?3?5?$CFs?5?5id?3?5?$CFd?5?5ip?3?5?$CFs?5?5ping?3?5@ 0000000039aa78c8     CryMatchMaking.obj
 0002:00002908       ??_C@_0BD@BCNEODCB@Connection?5Status?3?$AA@ 0000000039aa7908     CryMatchMaking.obj
 0002:00002920       ??_C@_0CL@CADKIPPD@?6?9?9?9?9?9?9?9?9?9?9?9?9?9?9?9?9?9?9?9?9?9?9?9?9?9?9?9?9?9?9?9@ 0000000039aa7920     CryMatchMaking.obj
 0002:00002950       ??_C@_0BF@PJHOOCJF@time?5remaining?3?50?300?$AA@ 0000000039aa7950     CryMatchMaking.obj
 0002:00002968       ??_C@_0P@LENIEGOL@players?3?5?$CFi?116?$AA@ 0000000039aa7968     CryMatchMaking.obj
 0002:00002978       ??_C@_0BD@OCFMNGID@gamerules?3?5unknown?$AA@ 0000000039aa7978     CryMatchMaking.obj
 0002:00002990       ??_C@_0N@NEFIFPBJ@level?3?5lobby?$AA@ 0000000039aa7990     CryMatchMaking.obj
 0002:000029a0       ??_C@_0M@KENPMFNK@version?3?5?$CFs?$AA@ 0000000039aa79a0     CryMatchMaking.obj
 0002:000029ac       ??_C@_06GKIIFFB@ip?3?5?$CFs?$AA@ 0000000039aa79ac     CryMatchMaking.obj
 0002:000029b8       ??_C@_08FCHJADKJ@name?3?5?$CFs?$AA@ 0000000039aa79b8     CryMatchMaking.obj
 0002:000029c8       ??_C@_0L@NPLHBDIN@?$CFs?5Status?3?$AA@ 0000000039aa79c8     CryMatchMaking.obj
 0002:000029d8       ??_C@_0CK@OHPHFMNE@?9?9?9?9?9?9?9?9?9?9?9?9?9?9?9?9?9?9?9?9?9?9?9?9?9?9?9?9?9?9?9?9@ 0000000039aa79d8     CryMatchMaking.obj
 0002:00002a04       ??_C@_06PJIGMIJB@Client?$AA@ 0000000039aa7a04     CryMatchMaking.obj
 0002:00002a0c       ??_C@_06LGMEBDBC@Server?$AA@ 0000000039aa7a0c     CryMatchMaking.obj
 0002:00002a18       ??_C@_0DJ@CBBGAKCH@?$FLServer?5Ping?$FN?3?5ping?5received?5for@ 0000000039aa7a18     CryMatchMaking.obj
 0002:00002a60       ??_C@_0EL@BHLPLAC@New?5remote?5connection?5addr?5?$CFs?0?5s@ 0000000039aa7a60     CryMatchMaking.obj
 0002:00002ab0       ??_C@_0FL@CPNNBBDL@Failed?5to?5send?5packet?5to?5connect@ 0000000039aa7ab0     CryMatchMaking.obj
 0002:00002b10       ??_C@_0N@NMLGHBBA@SendToServer?$AA@ 0000000039aa7b10     CryMatchMaking.obj
 0002:00002b20       ??_C@_0BB@LKDIHFDM@SendToAllClients?$AA@ 0000000039aa7b20     CryMatchMaking.obj
 0002:00002b38       ??_C@_0N@JDPEKKJD@SendToClient?$AA@ 0000000039aa7b38     CryMatchMaking.obj
 0002:00002b50       ??_C@_0GJ@PIPDLNEO@CCryMatchMaking?3?3SessionDisconne@ 0000000039aa7b50     CryMatchMaking.obj
 0002:00002bc0       ??_C@_0GJ@JBDPEBED@CCryMatchMaking?3?3SessionDisconne@ 0000000039aa7bc0     CryMatchMaking.obj
 0002:00002c30       ??_C@_0GJ@ECKGLJFJ@CCryMatchMaking?3?3SessionDisconne@ 0000000039aa7c30     CryMatchMaking.obj
 0002:00002ca0       ??_C@_0GJ@NOMEDGPK@CCryMatchMaking?3?3SessionDisconne@ 0000000039aa7ca0     CryMatchMaking.obj
 0002:00002d10       ??_C@_0EB@FDJDDKMA@?$FLMatchMaking?$FN?5Start?5SessionTermi@ 0000000039aa7d10     CryMatchMaking.obj
 0002:00002d58       ??_C@_0DC@CCLDPKAP@?$FLMatchMaking?$FN?5Start?5SessionSetLo@ 0000000039aa7d58     CryMatchMaking.obj
 0002:00002d90       ??_C@_0DE@JPEDGOFA@?$FLMatchMaking?$FN?5Start?5SessionClear@ 0000000039aa7d90     CryMatchMaking.obj
 0002:00002dc8       ??_C@_0DC@CDJNNNNA@?$FLMatchMaking?$FN?5Start?5SessionGetLo@ 0000000039aa7dc8     CryMatchMaking.obj
 0002:00002e00       ??_C@_0BH@LMIOEFH@net_fullStatusOnClient?$AA@ 0000000039aa7e00     CryMatchMaking.obj
 0002:00002e18       ??_C@_0CC@IMDCFFNE@Maximum?5number?5of?5rooms?5per?5worl@ 0000000039aa7e18     CryMatchMaking.obj
 0002:00002e40       ??_7CCryMatchMaking@@6BICryMatchMakingPrivate@@@ 0000000039aa7e40     CryMatchMaking.obj
 0002:00003010       ??_7CCryMatchMaking@@6BCMultiThreadRefCount@@@ 0000000039aa8010     CryMatchMaking.obj
 0002:00003070       ??_C@_0EL@BCBHKCBF@SessionDisconnectRemoteConnectio@ 0000000039aa8070     CryMatchMaking.obj
 0002:000030c0       ??_C@_0BA@CBEPFNDL@Session?5deleted?$AA@ 0000000039aa80c0     CryMatchMaking.obj
 0002:000030d0       ??_C@_0EM@NGECCPNO@?$FLLobby?$FN?5session?5?$CFd?5mmcid?5?$CFd?5lcid@ 0000000039aa80d0     CryMatchMaking.obj
 0002:00003120       ??_C@_0EG@DBDLICGO@?$FLLobby?$FN?5session?5?$CFd?5mmcid?5?$CFd?5lcid@ 0000000039aa8120     CryMatchMaking.obj
 0002:00003168       ??_C@_0BD@MHOOPILL@Kicked?5from?5server?$AA@ 0000000039aa8168     CryMatchMaking.obj
 0002:00003180       ??_C@_0BK@MMMIGBMF@Kicked?5?$CFs?5?$CIcx?3?$CFi?5id?3?$CFllx?$CJ?$AA@ 0000000039aa8180     CryMatchMaking.obj
 0002:000031a0       ??_C@_0DM@GIPEJAEI@Unable?5to?5find?5player?5with?5name?5@ 0000000039aa81a0     CryMatchMaking.obj
 0002:000031e0       ??_C@_0EP@KPAALHLM@?$FLMatchmaking?$FN?5FreeRemoteConnecti@ 0000000039aa81e0     CryMatchMaking.obj
 0002:00003230       ??_C@_0BB@KFNOPBGD@reset?5connection?$AA@ 0000000039aa8230     CryMatchMaking.obj
 0002:00003248       ??_C@_0BO@NOJLAGDJ@?$FLMatchmaking?$FN?5ResetConnection?$AA@ 0000000039aa8248     CryMatchMaking.obj
 0002:00003268       ??_C@_0BA@DADPBCNM@Connection?5lost?$AA@ 0000000039aa8268     CryMatchMaking.obj
 0002:00003278       ??_7ICrySignIn@@6B@        0000000039aa8278     CrySignIn.obj
 0002:000032b0       ??_7CCrySignIn@@6BICrySignIn@@@ 0000000039aa82b0     CrySignIn.obj
 0002:000032f0       ??_7CCrySignIn@@6BCMultiThreadRefCount@@@ 0000000039aa82f0     CrySignIn.obj
 0002:00003350       ??_C@_0EF@BMDHCBBG@CryLobbyID?5is?5being?5pre?9incremen@ 0000000039aa8350     CrySignIn.obj
 0002:00003398       ??_C@_0CB@ECAHCMKM@?$FLLobby?$FN?5SignIn?5task?5?$CFd?5cancelled@ 0000000039aa8398     CrySignIn.obj
 0002:000033c0       ??_7?$CClassJobNoRef@IVCCryGameSpySBQR2FriendsManagement@@@CWorkQueue@@6B@ 0000000039aa83c0     CryGameSpySBQR2FriendsManagement.obj
 0002:000033c0       ??_7?$CClassJobNoRef@IVCCryGameSpySBQR2LobbyUI@@@CWorkQueue@@6B@ 0000000039aa83c0     CryGameSpySBQR2LobbyUI.obj
 0002:000033c0       ??_7?$CClassJobNoRef@IVCCryGameSpySBQR2Stats@@@CWorkQueue@@6B@ 0000000039aa83c0     CryGameSpySBQR2Stats.obj
 0002:000033c0       ??_7?$CClassJobNoRef@V?$CryLobbyID@USCrySignInTaskID@CCrySignIn@@$03@@VCCryGameSpySBQR2SignIn@@@CWorkQueue@@6B@ 0000000039aa83c0     CryGameSpySBQR2SignIn.obj
 0002:000033c0       ??_7?$CClassJobNoRef@V?$CryLobbyID@USCrySignInTaskID@CCrySignIn@@$03@@VCCrySignIn@@@CWorkQueue@@6B@ 0000000039aa83c0     CrySignIn.obj
 0002:000033d0       ??_7ICryStats@@6B@         0000000039aa83d0     CryStats.obj
 0002:00003450       ??_7CCryStats@@6BICryStats@@@ 0000000039aa8450     CryStats.obj
 0002:000034d0       ??_7CCryStats@@6BCMultiThreadRefCount@@@ 0000000039aa84d0     CryStats.obj
 0002:000034e8       ??_C@_0DN@FMGHHLEA@?$FLStats?$FN?5Encryption?5size?5mismatch@ 0000000039aa84e8     CryStats.obj
 0002:00003530       ??_C@_0EO@MFPDJMDG@?$FLStats?$FN?5Encrypted?5userdata?3?5Firs@ 0000000039aa8530     CryStats.obj
 0002:00003580       ??_C@_0FA@NAHOKDPF@?$FLStats?$FN?5Unencrypted?5userdata?3?5Fi@ 0000000039aa8580     CryStats.obj
 0002:000035d0       ??_C@_0DN@GAGPCDPM@?$FLStats?$FN?5Decryption?5size?5mismatch@ 0000000039aa85d0     CryStats.obj
 0002:00003610       ??_C@_0EO@CGHFNKDN@?$FLStats?$FN?5Decrypted?5userdata?3?5Firs@ 0000000039aa8610     CryStats.obj
 0002:00003660       ??_7ICryLobbyUI@@6B@       0000000039aa8660     CryLobbyUI.obj
 0002:00003660       ??_7ICryTCPService@@6B@    0000000039aa8660     CryTCPService.obj
 0002:000036c0       ??_7CCryTCPService@@6B@    0000000039aa86c0     CryTCPService.obj
 0002:00003750       ??_7CCryTCPServiceFactory@@6B@ 0000000039aa8750     CryTCPServiceFactory.obj
 0002:000037b0       ??_7ICryVoice@@6B@         0000000039aa87b0     CryVoice.obj
 0002:00003818       __real@47c35000            0000000039aa8818     CryVoice.obj
 0002:00003820       ??_7CCryVoice@@6BICryVoice@@@ 0000000039aa8820     CryVoice.obj
 0002:00003888       ??_7CCryVoice@@6BCMultiThreadRefCount@@@ 0000000039aa8888     CryVoice.obj
 0002:000038a8       ??_7CGameSpySBQR2AvailabilityCheck@@6B@ 0000000039aa88a8     GameSpySBQR2AvailabilityCheck.obj
 0002:000038c8       ??_7STask@CGameSpySBQR2Core@@6B@ 0000000039aa88c8     GameSpySBQR2Core.obj
 0002:000038d8       ??_7CGameSpySBQR2Core@@6B@ 0000000039aa88d8     GameSpySBQR2Core.obj
 0002:000038f8       ??_7STaskBase@CGameSpySBQR2NATNegotiation@@6B@ 0000000039aa88f8     GameSpySBQR2NatNegotiation.obj
 0002:00003910       ??_7SNegotiateTask@CGameSpySBQR2NATNegotiation@@6B@ 0000000039aa8910     GameSpySBQR2NatNegotiation.obj
 0002:00003928       ??_7SDetectTask@CGameSpySBQR2NATNegotiation@@6B@ 0000000039aa8928     GameSpySBQR2NatNegotiation.obj
 0002:00003940       ??_7CGameSpySBQR2NATNegotiation@@6B@ 0000000039aa8940     GameSpySBQR2NatNegotiation.obj
 0002:00003960       ??_7STaskBase@CGameSpySBQR2Sake@@6B@ 0000000039aa8960     GameSpySBQR2Sake.obj
 0002:00003988       ??_7CGameSpySBQR2Sake@@6B@ 0000000039aa8988     GameSpySBQR2Sake.obj
 0002:000039a8       ??_7?$STask@USAKEUpdateRecordInput@@@CGameSpySBQR2Sake@@6B@ 0000000039aa89a8     GameSpySBQR2Sake.obj
 0002:000039d0       ??_7?$STask@USAKECreateRecordInput@@@CGameSpySBQR2Sake@@6B@ 0000000039aa89d0     GameSpySBQR2Sake.obj
 0002:000039f8       ??_7?$STask@USAKEGetMyRecordsInput@@@CGameSpySBQR2Sake@@6B@ 0000000039aa89f8     GameSpySBQR2Sake.obj
 0002:00003a20       ??_7?$STask@USAKEGetRecordCountInput@@@CGameSpySBQR2Sake@@6B@ 0000000039aa8a20     GameSpySBQR2Sake.obj
 0002:00003a48       ??_7?$STask@USAKESearchForRecordsInput@@@CGameSpySBQR2Sake@@6B@ 0000000039aa8a48     GameSpySBQR2Sake.obj
 0002:00003a70       ??_7CGameSpySDK@@6B@       0000000039aa8a70     GameSpySDK.obj
 0002:00003a88       ??_7CGameSpyThinkerSDK@@6B@ 0000000039aa8a88     GameSpySDK.obj
 0002:00003aa8       ??_7?$CClassJobNoRef@IVCCryGameSpySBQR2DLCStore@@@CWorkQueue@@6B@ 0000000039aa8aa8     CryGameSpySBQR2DLCStore.obj
 0002:00003aa8       ??_7?$CClassJobNoRef@IVCCryDLCStore@@@CWorkQueue@@6B@ 0000000039aa8aa8     CryDLCStore.obj
 0002:00003ab8       ??_7?$CClassJob@XVCCryGameSpySBQR2DLCStore@@@CWorkQueue@@6B@ 0000000039aa8ab8     CryGameSpySBQR2DLCStore.obj
 0002:00003ac8       ??_7?$CClassJobNoRef6@P6AXIW4ECryLobbyError@@V?$_smart_ptr@USCryDLCDownloadableID@@@@_NIIPEBDPEAX@ZIV2@IIPEAXVCCryGameSpySBQR2DLCStore@@@CWorkQueue@@6B@ 0000000039aa8ac8     CryGameSpySBQR2DLCStore.obj
 0002:00003ad8       ??_7?$CClassJobNoRef3@PEAUSTaskLink@CCryGameSpySBQR2DLCStore@@IIV2@@CWorkQueue@@6B@ 0000000039aa8ad8     CryGameSpySBQR2DLCStore.obj
 0002:00003ae8       ??_7SCryGameSpySBQR2DLCDownloadableID@@6B@ 0000000039aa8ae8     CryGameSpySBQR2DLCStore.obj
 0002:00003ae8       ??_7SCryGameSpySBQR2DLCItemID@@6B@ 0000000039aa8ae8     CryGameSpySBQR2DLCStore.obj
 0002:00003ae8       ??_7SCryGameSpySBQR2DLCPaymentMethodID@@6B@ 0000000039aa8ae8     CryGameSpySBQR2DLCStore.obj
 0002:00003af8       ??_7SOrderLink@CCryGameSpySBQR2DLCStore@@6B@ 0000000039aa8af8     CryGameSpySBQR2DLCStore.obj
 0002:00003b00       ??_7SCryGameSpySBQR2DLCLicense@@6B@ 0000000039aa8b00     CryGameSpySBQR2DLCStore.obj
 0002:00003b10       ??_7SCryGameSpySBQR2DLCImageID@@6B@ 0000000039aa8b10     CryGameSpySBQR2DLCStore.obj
 0002:00003b10       ??_7SCryGameSpySBQR2DLCCategoryID@@6B@ 0000000039aa8b10     CryGameSpySBQR2DLCStore.obj
 0002:00003b20       ??_7?$CClassJobNoRef@USDispatchDownloadCompleteParam@CCryGameSpySBQR2DLCStore@@V2@@CWorkQueue@@6B@ 0000000039aa8b20     CryGameSpySBQR2DLCStore.obj
 0002:00003b30       ??_7?$CClassJobNoRef3@PEAUSTaskLink@CCryGameSpySBQR2DLCStore@@HV?$CryStringT@D@@V2@@CWorkQueue@@6B@ 0000000039aa8b30     CryGameSpySBQR2DLCStore.obj
 0002:00003b40       ??_7STaskLink@CCryGameSpySBQR2DLCStore@@6B@ 0000000039aa8b40     CryGameSpySBQR2DLCStore.obj
 0002:00003b48       ??_C@_15MAOEGKJF@?$AA?$CF?$AAS?$AA?$AA@ 0000000039aa8b48     CryGameSpySBQR2DLCStore.obj
 0002:00003b50       ??_C@_15KKKIBPM@?$AA0?$AA?4?$AA?$AA@ 0000000039aa8b50     CryGameSpySBQR2DLCStore.obj
 0002:00003b58       ??_C@_13JOFGPIOO@?$AA?4?$AA?$AA@ 0000000039aa8b58     CryGameSpySBQR2DLCStore.obj
 0002:00003b5c       ??_C@_11LOCGONAA@?$AA?$AA@ 0000000039aa8b5c     CryGameSpySBQR2DLCStore.obj
 0002:00003b60       ??_C@_13COJANIEC@?$AA0?$AA?$AA@ 0000000039aa8b60     CryGameSpySBQR2DLCStore.obj
 0002:00003b68       ??_C@_0DO@EEPJMONK@?$FLLobby?$FN?5CCryGameSpySBQR2DLCStore@ 0000000039aa8b68     CryGameSpySBQR2DLCStore.obj
 0002:00003ba8       __real@c8927c00            0000000039aa8ba8     CryGameSpySBQR2DLCStore.obj
 0002:00003bb0       ??_C@_0CD@MNPDEGJJ@?$FLLobby?$FN?5Start?5SessionJoin?5error?5@ 0000000039aa8bb0     CryGameSpySBQR2DLCStore.obj
 0002:00003bd8       ??_C@_0CD@NBCEJMGD@?$FLLobby?$FN?5Start?5ItemGetInfo?5error?5@ 0000000039aa8bd8     CryGameSpySBQR2DLCStore.obj
 0002:00003c00       ??_C@_0DA@BKPJDCDL@?$FLLobby?$FN?5Start?5DownloadableIsDown@ 0000000039aa8c00     CryGameSpySBQR2DLCStore.obj
 0002:00003c30       ??_C@_0CO@CJPPKLHO@?$FLLobby?$FN?5Start?5UserGetPurchaseHis@ 0000000039aa8c30     CryGameSpySBQR2DLCStore.obj
 0002:00003c60       ??_C@_0CG@DAHIAFBB@?$FLLobby?$FN?5Start?5UserStartOrder?5err@ 0000000039aa8c60     CryGameSpySBQR2DLCStore.obj
 0002:00003c88       ??_C@_0DB@PPLDILMG@?$FLLobby?$FN?5Start?5UserGetDownloadabl@ 0000000039aa8c88     CryGameSpySBQR2DLCStore.obj
 0002:00003cc0       ??_C@_0CI@CNJAFJJK@?$FLLobby?$FN?5Start?5UserDownloadItem?5e@ 0000000039aa8cc0     CryGameSpySBQR2DLCStore.obj
 0002:00003ce8       ??_C@_0DF@CKNCJOKH@?$FLLobby?$FN?5Start?5UserRedownloadAllM@ 0000000039aa8ce8     CryGameSpySBQR2DLCStore.obj
 0002:00003d20       ??_C@_0CE@ODJGNINH@?$FLLobby?$FN?5Start?5OrderAddItem?5error@ 0000000039aa8d20     CryGameSpySBQR2DLCStore.obj
 0002:00003d48       ??_C@_0CH@NEMEPEBJ@?$FLLobby?$FN?5Start?5OrderRemoveItem?5er@ 0000000039aa8d48     CryGameSpySBQR2DLCStore.obj
 0002:00003d70       ??_C@_0CM@JIDPCGF@?$FLLobby?$FN?5Start?5OrderAddItemQuanti@ 0000000039aa8d70     CryGameSpySBQR2DLCStore.obj
 0002:00003da0       ??_C@_0CP@DMPFDJOC@?$FLLobby?$FN?5Start?5OrderRemoveItemQua@ 0000000039aa8da0     CryGameSpySBQR2DLCStore.obj
 0002:00003dd0       ??_C@_0CG@PJFKCBFL@?$FLLobby?$FN?5Start?5OrderListItems?5err@ 0000000039aa8dd0     CryGameSpySBQR2DLCStore.obj
 0002:00003df8       ??_C@_0CE@PACMKMM@?$FLLobby?$FN?5Start?5OrderGetInfo?5error@ 0000000039aa8df8     CryGameSpySBQR2DLCStore.obj
 0002:00003e20       ??_C@_0CD@JMGHFIOF@?$FLLobby?$FN?5Start?5OrderCancel?5error?5@ 0000000039aa8e20     CryGameSpySBQR2DLCStore.obj
 0002:00003e48       ??_C@_0CB@IKJEPKNO@?$FLLobby?$FN?5Start?5OrderFree?5error?5?$CFd@ 0000000039aa8e48     CryGameSpySBQR2DLCStore.obj
 0002:00003e70       ??_C@_0CG@FFONAPJK@?$FLLobby?$FN?5Start?5ReleaseCatalog?5err@ 0000000039aa8e70     CryGameSpySBQR2DLCStore.obj
 0002:00003e98       ??_7CCryGameSpySBQR2DLCStore@@6B@ 0000000039aa8e98     CryGameSpySBQR2DLCStore.obj
 0002:00003eb0       ??_7CCryGameSpySBQR2DLCStore@@6BICryDLCStore@@@ 0000000039aa8eb0     CryGameSpySBQR2DLCStore.obj
 0002:00003fa0       ??_7CCryGameSpySBQR2DLCStore@@6BCMultiThreadRefCount@@@ 0000000039aa8fa0     CryGameSpySBQR2DLCStore.obj
 0002:00004010       __real@40a00000            0000000039aa9010     CryGameSpySBQR2DLCStore.obj
 0002:00004018       ??_7?$CClassJobNoRef@IVCCryGameSpySBQR2Friends@@@CWorkQueue@@6B@ 0000000039aa9018     CryGameSpySBQR2Friends.obj
 0002:00004028       ??_7?$CClassJobNoRef2@HW4EOnlineState@@VCCryGameSpySBQR2Friends@@@CWorkQueue@@6B@ 0000000039aa9028     CryGameSpySBQR2Friends.obj
 0002:00004028       ??_7?$CClassJobNoRef2@W4ECryLobbySystemEvent@@HVCCryGameSpySBQR2Friends@@@CWorkQueue@@6B@ 0000000039aa9028     CryGameSpySBQR2Friends.obj
 0002:00004038       ??_7SCryGameSpySBQR2UserID@@6B@ 0000000039aa9038     CryGameSpySBQR2Friends.obj
 0002:00004060       ??_C@_0GF@CKNOLMKL@?$FLLobby?$FN?5CCryGameSpySBQR2Friends?3@ 0000000039aa9060     CryGameSpySBQR2Friends.obj
 0002:000040c8       ??_C@_0M@ELPBDANP@sv_password?$AA@ 0000000039aa90c8     CryGameSpySBQR2Friends.obj
 0002:000040d4       ??_C@_04HCKDAFDF@?$CFllX?$AA@ 0000000039aa90d4     CryGameSpySBQR2Friends.obj
 0002:000040dc       ??_C@_01CLKCMJKC@?5?$AA@   0000000039aa90dc     CryGameSpySBQR2Friends.obj
 0002:000040e0       ??_C@_0HB@KCEFJEEE@?$FLLobby?$FN?5CCryGameSpySBQR2Friends?3@ 0000000039aa90e0     CryGameSpySBQR2Friends.obj
 0002:00004158       ??_C@_0L@CJDNELKH@?$CFd?5?$CFllX?5?$CFs?$AA@ 0000000039aa9158     CryGameSpySBQR2Friends.obj
 0002:00004164       ??_C@_03GACAABJG@?3?1?1?$AA@ 0000000039aa9164     CryGameSpySBQR2Friends.obj
 0002:00004168       ??_C@_04JIMNDDED@?$CF08X?$AA@ 0000000039aa9168     CryGameSpySBQR2Friends.obj
 0002:00004170       ??_C@_0EB@GKJNJAFI@?$FLLobby?$FN?5CCryGameSpySBQR2Friends?3@ 0000000039aa9170     CryGameSpySBQR2Friends.obj
 0002:000041c0       ??_C@_0EN@FIPFPNHE@?$FLLobby?$FN?5CCryGameSpySBQR2Friends?3@ 0000000039aa91c0     CryGameSpySBQR2Friends.obj
 0002:00004210       ??_C@_0GK@GCNLNLGB@?$FLLobby?$FN?5CCryGameSpySBQR2Friends?3@ 0000000039aa9210     CryGameSpySBQR2Friends.obj
 0002:00004280       ??_C@_0DE@KPNCJNHJ@?$FLGameSpy?$FN?5?3?5profile?5?$CFi?5friend?5au@ 0000000039aa9280     CryGameSpySBQR2Friends.obj
 0002:000042b8       ??_7CCryGameSpySBQR2Friends@@6BICryFriends@@@ 0000000039aa92b8     CryGameSpySBQR2Friends.obj
 0002:000042d0       ??_7CCryGameSpySBQR2Friends@@6BCMultiThreadRefCount@@@ 0000000039aa92d0     CryGameSpySBQR2Friends.obj
 0002:00004300       ??_C@_0IB@LJEGOGHF@?$FLLobby?$FN?5?3?5CCryGameSpySBQR2Friend@ 0000000039aa9300     CryGameSpySBQR2Friends.obj
 0002:00004390       ??_C@_0EG@EJLHLDOC@?$FLGameSpy?$FN?5?3?5status?5update?5for?5pr@ 0000000039aa9390     CryGameSpySBQR2Friends.obj
 0002:000043d8       ??_C@_0BF@CHNPFDFL@ReverseFriendRequest?$AA@ 0000000039aa93d8     CryGameSpySBQR2Friends.obj
 0002:000043f0       ??_C@_0DN@KLFIPFIO@?$FLLobby?$FN?5CCryGameSpySBQR2Friends?3@ 0000000039aa93f0     CryGameSpySBQR2Friends.obj
 0002:00004430       ??_C@_08LMOPGBBD@accepted?$AA@ 0000000039aa9430     CryGameSpySBQR2Friends.obj
 0002:00004440       ??_C@_0GP@IAHJKPNK@?$FLLobby?$FN?5CCryGameSpySBQR2Friends?3@ 0000000039aa9440     CryGameSpySBQR2Friends.obj
 0002:000044b0       ??_C@_0DF@IFDEOEIP@?$FLGameSpy?$FN?5?3?5profile?5?$CFi?5friend?5au@ 0000000039aa94b0     CryGameSpySBQR2Friends.obj
 0002:000044e8       ??_7?$CClassJobNoRef2@IV?$_smart_ptr@USCrySessionID@@@@VCCryGameSpySBQR2LobbyService@@@CWorkQueue@@6B@ 0000000039aa94e8     CryGameSpySBQR2FriendsManagement.obj
 0002:000044f8       ??_7SCryGameSpySBQR2SessionID@@6B@ 0000000039aa94f8     CryGameSpySBQR2FriendsManagement.obj
 0002:00004520       ??_C@_04BFAHMMK@?$CFlld?$AA@ 0000000039aa9520     CryGameSpySBQR2FriendsManagement.obj
 0002:00004528       ??_7CCryGameSpySBQR2SignIn@@6B@ 0000000039aa9528     CryGameSpySBQR2SignIn.obj
 0002:00004528       ??_7CCryGameSpySBQR2FriendsManagement@@6B@ 0000000039aa9528     CryGameSpySBQR2FriendsManagement.obj
 0002:00004528       ??_7CCryGameSpySBQR2Friends@@6B@ 0000000039aa9528     CryGameSpySBQR2Friends.obj
 0002:00004528       ??_7CCryGameSpySBQR2Stats@@6B@ 0000000039aa9528     CryGameSpySBQR2Stats.obj
 0002:00004528       ??_7CCryGameSpySBQR2Voice@@6B@ 0000000039aa9528     CryGameSpySBQR2Voice.obj
 0002:00004540       ??_7CCryGameSpySBQR2FriendsManagement@@6BICryFriendsManagement@@@ 0000000039aa9540     CryGameSpySBQR2FriendsManagement.obj
 0002:000045b0       ??_7CCryGameSpySBQR2FriendsManagement@@6BCMultiThreadRefCount@@@ 0000000039aa95b0     CryGameSpySBQR2FriendsManagement.obj
 0002:000045d0       ??_C@_0EH@KDBNKGKH@?$FLLobby?$FN?5CCryGameSpySBQR2FriendsM@ 0000000039aa95d0     CryGameSpySBQR2FriendsManagement.obj
 0002:00004620       ??_C@_0FC@LJGEHGIP@?$FLLobby?$FN?5CCryGameSpySBQR2FriendsM@ 0000000039aa9620     CryGameSpySBQR2FriendsManagement.obj
 0002:00004680       ??_C@_0IG@BCOIENLO@?$FLLobby?$FN?5CCryGameSpySBQR2FriendsM@ 0000000039aa9680     CryGameSpySBQR2FriendsManagement.obj
 0002:00004708       ??_C@_0BF@LIJAFHML@ForwardFriendRequest?$AA@ 0000000039aa9708     CryGameSpySBQR2FriendsManagement.obj
 0002:00004720       ??_C@_0IO@EJMKCCEJ@?$FLLobby?$FN?5CCryGameSpySBQR2FriendsM@ 0000000039aa9720     CryGameSpySBQR2FriendsManagement.obj
 0002:000047b0       ??_C@_0IO@KHDEGEED@?$FLLobby?$FN?5CCryGameSpySBQR2FriendsM@ 0000000039aa97b0     CryGameSpySBQR2FriendsManagement.obj
 0002:00004840       ??_C@_0IL@GMGCNJL@?$FLLobby?$FN?5CCryGameSpySBQR2FriendsM@ 0000000039aa9840     CryGameSpySBQR2FriendsManagement.obj
 0002:000048d0       ??_C@_0GP@LMCEMFKB@?$FLLobby?$FN?5CCryGameSpySBQR2FriendsM@ 0000000039aa98d0     CryGameSpySBQR2FriendsManagement.obj
 0002:00004940       ??_C@_0GL@JKCNBJEO@?$FLLobby?$FN?5CCryGameSpySBQR2FriendsM@ 0000000039aa9940     CryGameSpySBQR2FriendsManagement.obj
 0002:000049b0       ??_C@_0GP@NGAKKBJM@?$FLLobby?$FN?5CCryGameSpySBQR2FriendsM@ 0000000039aa99b0     CryGameSpySBQR2FriendsManagement.obj
 0002:00004a20       ??_C@_0HD@LMKBFJMC@?$FLLobby?$FN?5CCryGameSpySBQR2FriendsM@ 0000000039aa9a20     CryGameSpySBQR2FriendsManagement.obj
 0002:00004aa0       ??_C@_0GP@IDJEHMBK@?$FLLobby?$FN?5CCryGameSpySBQR2FriendsM@ 0000000039aa9aa0     CryGameSpySBQR2FriendsManagement.obj
 0002:00004b10       ??_C@_0GL@LEPGBJHH@?$FLLobby?$FN?5CCryGameSpySBQR2FriendsM@ 0000000039aa9b10     CryGameSpySBQR2FriendsManagement.obj
 0002:00004b80       ??_C@_0HE@BEBMAHPA@?$FLLobby?$FN?5CCryGameSpySBQR2FriendsM@ 0000000039aa9b80     CryGameSpySBQR2FriendsManagement.obj
 0002:00004c00       ??_C@_0FA@FCCFHNKB@?$FLLobby?$FN?5CCryGameSpySBQR2FriendsM@ 0000000039aa9c00     CryGameSpySBQR2FriendsManagement.obj
 0002:00004c50       ??_C@_0HC@JDBLKHJC@?$FLLobby?$FN?5CCryGameSpySBQR2FriendsM@ 0000000039aa9c50     CryGameSpySBQR2FriendsManagement.obj
 0002:00004cd0       ??_C@_0FD@JLIJJBHD@?$FLLobby?$FN?5CCryGameSpySBQR2FriendsM@ 0000000039aa9cd0     CryGameSpySBQR2FriendsManagement.obj
 0002:00004d30       ??_C@_0FL@CFOPDNBF@?$FLLobby?$FN?5CCryGameSpySBQR2FriendsM@ 0000000039aa9d30     CryGameSpySBQR2FriendsManagement.obj
 0002:00004d90       ??_C@_0FN@NPMALIOP@?$FLLobby?$FN?5CCryGameSpySBQR2FriendsM@ 0000000039aa9d90     CryGameSpySBQR2FriendsManagement.obj
 0002:00004df0       ??_C@_0FN@EOELFFEH@?$FLLobby?$FN?5CCryGameSpySBQR2FriendsM@ 0000000039aa9df0     CryGameSpySBQR2FriendsManagement.obj
 0002:00004e50       ??_C@_0FM@DGGLKHLE@?$FLLobby?$FN?5CCryGameSpySBQR2FriendsM@ 0000000039aa9e50     CryGameSpySBQR2FriendsManagement.obj
 0002:00004eb0       ??_C@_0FG@KMCJKPBF@?$FLLobby?$FN?5CCryGameSpySBQR2FriendsM@ 0000000039aa9eb0     CryGameSpySBQR2FriendsManagement.obj
 0002:00004f10       ??_C@_0FD@BGCBPNHE@?$FLLobby?$FN?5CCryGameSpySBQR2FriendsM@ 0000000039aa9f10     CryGameSpySBQR2FriendsManagement.obj
 0002:00004f70       ??_C@_0FF@IPDMMPMP@?$FLLobby?$FN?5CCryGameSpySBQR2FriendsM@ 0000000039aa9f70     CryGameSpySBQR2FriendsManagement.obj
 0002:00004fd0       ??_C@_0FH@COKGGLMF@?$FLLobby?$FN?5CCryGameSpySBQR2FriendsM@ 0000000039aa9fd0     CryGameSpySBQR2FriendsManagement.obj
 0002:00005030       ??_C@_0FG@BNDKOJG@?$FLLobby?$FN?5CCryGameSpySBQR2FriendsM@ 0000000039aaa030     CryGameSpySBQR2FriendsManagement.obj
 0002:00005090       ??_C@_0GE@DOCJCCMD@?$FLGameSpy?$FN?5CCryGameSpySBQR2LobbyS@ 0000000039aaa090     CryGameSpySBQR2Lobby.obj
 0002:000050f8       ??_C@_0O@NIPGCINC@Unknown?5error?$AA@ 0000000039aaa0f8     CryGameSpySBQR2Lobby.obj
 0002:00005108       ??_C@_0CJ@HLILIOMA@QR2?5failed?5to?5initialise?3?5error?5@ 0000000039aaa108     CryGameSpySBQR2Lobby.obj
 0002:00005138       ??_C@_0DL@BMOMHANC@?$FLLobby?$FN?5?5?5?5?5Request?5acknowledged@ 0000000039aaa138     CryGameSpySBQR2Lobby.obj
 0002:00005178       ??_C@_0DE@HBFDPIOP@?$FLLobby?$FN?5?5?5?5?5Direct?5negotiation?5w@ 0000000039aaa178     CryGameSpySBQR2Lobby.obj
 0002:000051b0       ??_C@_0CD@CFFGIFIG@?$FLLobby?$FN?5?5?5?5?5Cookie?3?5?5?5?5?5?5?5?5?5?5?5?5?5@ 0000000039aaa1b0     CryGameSpySBQR2Lobby.obj
 0002:000051d8       ??_C@_0CN@COEKCAHE@?$FLLobby?$FN?5Processing?5NAT?5negotiati@ 0000000039aaa1d8     CryGameSpySBQR2Lobby.obj
 0002:00005208       ??_C@_0CD@CGJHCINE@?$FLLobby?$FN?5?5?5?5?5Error?3?5?5?5?5?5?5?5?5?5?5?5?5?5?5@ 0000000039aaa208     CryGameSpySBQR2Lobby.obj
 0002:00005230       ??_C@_0CD@FLDPDGLO@?$FLLobby?$FN?5?5?5?5?5NAT?5negotiation?5fail@ 0000000039aaa230     CryGameSpySBQR2Lobby.obj
 0002:00005258       ??_C@_0CG@JJBBHJIK@?$FLLobby?$FN?5?5?5?5?5Negotiated?5address?3?5@ 0000000039aaa258     CryGameSpySBQR2Lobby.obj
 0002:00005280       ??_C@_0CG@GBDALEHF@?$FLLobby?$FN?5?5?5?5?5NAT?5negotiation?5succ@ 0000000039aaa280     CryGameSpySBQR2Lobby.obj
 0002:000052a8       ??_C@_0CM@PILNGGGL@?$FLLobby?$FN?5Finishing?5NAT?5negotiatio@ 0000000039aaa2a8     CryGameSpySBQR2Lobby.obj
 0002:000052e0       ??_C@_0FB@BNJNJNAC@?$CK?$CKWARNING?$CK?$CK?5CryGameSpyLobbyServi@ 0000000039aaa2e0     CryGameSpySBQR2Lobby.obj
 0002:00005338       ??_7?$CClassJobNoRef4@W4ECryLobbySystemEvent@@IW4EOnlineState@@W4ECryLobbyError@@VCCryGameSpySBQR2LobbyService@@@CWorkQueue@@6B@ 0000000039aaa338     CryGameSpySBQR2Lobby.obj
 0002:00005348       ??_7?$CClassJob@XVCCryLobbyService@@@CWorkQueue@@6B@ 0000000039aaa348     CryLobby.obj
 0002:00005348       ??_7?$CClassJob@XVCCryGameSpySBQR2LobbyService@@@CWorkQueue@@6B@ 0000000039aaa348     CryGameSpySBQR2Lobby.obj
 0002:00005358       ??_C@_0CL@JPAOJKLL@?$FLLobby?$FN?5Starting?5NAT?5negotiation@ 0000000039aaa358     CryGameSpySBQR2Lobby.obj
 0002:00005390       ??_C@_0GC@ELEAMLBK@?$FLGameSpy?$FN?5CCryGameSpySBQR2LobbyS@ 0000000039aaa390     CryGameSpySBQR2Lobby.obj
 0002:000053f8       ??_7CCryGameSpySBQR2LobbyService@@6B@ 0000000039aaa3f8     CryGameSpySBQR2Lobby.obj
 0002:00005410       ??_7CCryGameSpySBQR2LobbyService@@6BICryLobbyService@@@ 0000000039aaa410     CryGameSpySBQR2Lobby.obj
 0002:000054a0       ??_7CCryGameSpySBQR2LobbyService@@6BCMultiThreadRefCount@@@ 0000000039aaa4a0     CryGameSpySBQR2Lobby.obj
 0002:00005500       ??_C@_0CB@DFCOJKJE@net_gamespy_voip_playback_volume@ 0000000039aaa500     CryGameSpySBQR2Lobby.obj
 0002:00005528       ??_C@_0BN@KAKMPPCP@GameSpy?5VOIP?5playback?5volume?$AA@ 0000000039aaa528     CryGameSpySBQR2Lobby.obj
 0002:00005548       ??_C@_0BF@DDNJBDJJ@net_gamespy_voip_ptt?$AA@ 0000000039aaa548     CryGameSpySBQR2Lobby.obj
 0002:00005560       ??_C@_0CH@IDJNDCMB@Toggles?5GameSpy?5VOIP?5Push?9to?9tal@ 0000000039aaa560     CryGameSpySBQR2Lobby.obj
 0002:00005588       ??_C@_0BL@DLELEEII@net_gamespy_voip_threshold?$AA@ 0000000039aaa588     CryGameSpySBQR2Lobby.obj
 0002:000055a8       ??_C@_0CP@KDHBJHDO@Sets?5the?5GameSpy?5VOIP?5capture?5vo@ 0000000039aaa5a8     CryGameSpySBQR2Lobby.obj
 0002:000055d8       __real@3d4ccccd            0000000039aaa5d8     CryGameSpySBQR2Lobby.obj
 0002:000055e0       ??_C@_0BJ@PPEEDILM@net_gamespy_voip_logging?$AA@ 0000000039aaa5e0     CryGameSpySBQR2Lobby.obj
 0002:00005600       ??_C@_0CP@LELOFGAG@Toggles?5whether?5GameSpy?5VOIP?5log@ 0000000039aaa600     CryGameSpySBQR2Lobby.obj
 0002:00005630       ??_C@_0BK@EBKHPMCM@net_gamespy_voip_loopback?$AA@ 0000000039aaa630     CryGameSpySBQR2Lobby.obj
 0002:00005650       ??_C@_0EC@LJAGGB@Toggles?5whether?5GameSpy?5micropho@ 0000000039aaa650     CryGameSpySBQR2Lobby.obj
 0002:00005698       ??_C@_0BI@JLOBLAOG@net_gamespy_voip_enable?$AA@ 0000000039aaa698     CryGameSpySBQR2Lobby.obj
 0002:000056b0       ??_C@_0CM@NALODJPL@Toggles?5whether?5GameSpy?5VOIP?5ena@ 0000000039aaa6b0     CryGameSpySBQR2Lobby.obj
 0002:000056e0       ??_C@_0CK@MMLNEABG@?$FLLobby?$FN?5LobbyUI?5EndTask?5?$CFd?5?$CI?$CFd?$CJ?5@ 0000000039aaa6e0     CryGameSpySBQR2LobbyUI.obj
 0002:00005710       ??_7CCryGameSpySBQR2LobbyUI@@6BICryLobbyUI@@@ 0000000039aaa710     CryGameSpySBQR2LobbyUI.obj
 0002:00005770       ??_C@_02DPGMDCM@gc?$AA@    0000000039aaa770     CryGameSpySBQR2MatchMaking.obj
 0002:00005774       ??_C@_01PFHFFBPC@t?$AA@    0000000039aaa774     CryGameSpySBQR2MatchMaking.obj
 0002:00005778       ??_C@_02DGAFJLGB@dv?$AA@   0000000039aaa778     CryGameSpySBQR2MatchMaking.obj
 0002:0000577c       ??_C@_02ELHCGPCE@ds?$AA@   0000000039aaa77c     CryGameSpySBQR2MatchMaking.obj
 0002:00005780       ??_C@_01GOHFPIOK@m?$AA@    0000000039aaa780     CryGameSpySBQR2MatchMaking.obj
 0002:00005784       ??_C@_01INIBCBCB@f?$AA@    0000000039aaa784     CryGameSpySBQR2MatchMaking.obj
 0002:00005788       ??_C@_01KDCPPGHE@r?$AA@    0000000039aaa788     CryGameSpySBQR2MatchMaking.obj
 0002:0000578c       ??_C@_02FAFNGEII@ps?$AA@   0000000039aaa78c     CryGameSpySBQR2MatchMaking.obj
 0002:00005790       ??_C@_02EDKKPMHH@is?$AA@   0000000039aaa790     CryGameSpySBQR2MatchMaking.obj
 0002:00005794       ??_C@_02OCDGCAAK@si?$AA@   0000000039aaa794     CryGameSpySBQR2MatchMaking.obj
 0002:00005798       ??_C@_07NACDKLFL@exiting?$AA@ 0000000039aaa798     CryGameSpySBQR2MatchMaking.obj
 0002:000057a0       ??_C@_0O@LNGPCBFC@closedstaging?$AA@ 0000000039aaa7a0     CryGameSpySBQR2MatchMaking.obj
 0002:000057b0       ??_C@_0M@HPDILLDC@openstaging?$AA@ 0000000039aaa7b0     CryGameSpySBQR2MatchMaking.obj
 0002:000057c0       ??_C@_0M@HKFGEHJL@openplaying?$AA@ 0000000039aaa7c0     CryGameSpySBQR2MatchMaking.obj
 0002:000057d0       ??_C@_0O@LIABNNPL@closedplaying?$AA@ 0000000039aaa7d0     CryGameSpySBQR2MatchMaking.obj
 0002:000057e0       ??_C@_0O@MHNAPDPO@closedwaiting?$AA@ 0000000039aaa7e0     CryGameSpySBQR2MatchMaking.obj
 0002:000057f0       ??_C@_0M@FIHGJJO@openwaiting?$AA@ 0000000039aaa7f0     CryGameSpySBQR2MatchMaking.obj
 0002:00005800       ?k_gameModeNames@CCryGameSpySBQR2MatchMaking@@1QBQEBDB 0000000039aaa800     CryGameSpySBQR2MatchMaking.obj
 0002:00005838       ?k_sessionIDKeyName@CCryGameSpySBQR2MatchMaking@@1QEBDEB 0000000039aaa838     CryGameSpySBQR2MatchMaking.obj
 0002:00005840       ?k_numPrivateSlotsKeyName@CCryGameSpySBQR2MatchMaking@@1QEBDEB 0000000039aaa840     CryGameSpySBQR2MatchMaking.obj
 0002:00005848       ?k_numPublicSlotsKeyName@CCryGameSpySBQR2MatchMaking@@1QEBDEB 0000000039aaa848     CryGameSpySBQR2MatchMaking.obj
 0002:00005850       ?k_rankedKeyName@CCryGameSpySBQR2MatchMaking@@1QEBDEB 0000000039aaa850     CryGameSpySBQR2MatchMaking.obj
 0002:00005858       ?k_createFlagsKeyName@CCryGameSpySBQR2MatchMaking@@1QEBDEB 0000000039aaa858     CryGameSpySBQR2MatchMaking.obj
 0002:00005860       ?k_numMigrationsKeyName@CCryGameSpySBQR2MatchMaking@@1QEBDEB 0000000039aaa860     CryGameSpySBQR2MatchMaking.obj
 0002:00005868       ?k_dedicatedKeyName@CCryGameSpySBQR2MatchMaking@@1QEBDEB 0000000039aaa868     CryGameSpySBQR2MatchMaking.obj
 0002:00005870       ?k_dediVersionKeyName@CCryGameSpySBQR2MatchMaking@@1QEBDEB 0000000039aaa870     CryGameSpySBQR2MatchMaking.obj
 0002:00005878       ?k_dediUptimeKeyName@CCryGameSpySBQR2MatchMaking@@1QEBDEB 0000000039aaa878     CryGameSpySBQR2MatchMaking.obj
 0002:00005880       ?k_dediGameCountKeyName@CCryGameSpySBQR2MatchMaking@@1QEBDEB 0000000039aaa880     CryGameSpySBQR2MatchMaking.obj
 0002:00005888       ??_C@_0BD@CEDMBDHD@Validation?5Timeout?$AA@ 0000000039aaa888     CryGameSpySBQR2MatchMaking.obj
 0002:000058a0       ??_C@_0O@OOIFGDMN@CD?5Key?5in?5use?$AA@ 0000000039aaa8a0     CryGameSpySBQR2MatchMaking.obj
 0002:000058b0       ??_C@_0DD@JBKPDNJO@Your?5CD?5Key?5is?5disabled?4?5Contact@ 0000000039aaa8b0     CryGameSpySBQR2MatchMaking.obj
 0002:000058e8       ??_C@_0BH@ELNDJFPN@Invalid?5authentication?$AA@ 0000000039aaa8e8     CryGameSpySBQR2MatchMaking.obj
 0002:00005900       ??_C@_0P@CJNPEMPE@Invalid?5CD?5Key?$AA@ 0000000039aaa900     CryGameSpySBQR2MatchMaking.obj
 0002:00005910       ??_C@_0N@KNFGHCIP@Bad?5Response?$AA@ 0000000039aaa910     CryGameSpySBQR2MatchMaking.obj
 0002:00005920       __real@3c23d70a            0000000039aaa920     CryGameSpySBQR2MatchMaking.obj
 0002:00005928       ??_C@_0CD@HNLEIALF@Unhandled?5ECryLobbyUserDataType?5@ 0000000039aaa928     CryGameSpySBQR2MatchMaking.obj
 0002:00005950       ??_7SSession@CCryMatchMaking@@6B@ 0000000039aaa950     CryGameSpySBQR2MatchMaking.obj
 0002:00005950       ??_7IDatagramListener@@6B@ 0000000039aaa950     CryLobby.obj
 0002:00005950       ??_7ICryFriends@@6B@       0000000039aaa950     CryFriends.obj
 0002:00005968       ??_C@_0CN@DGMBJFGA@?$FLPassword?$FN?3?5received?5password?5up@ 0000000039aaa968     CryGameSpySBQR2MatchMaking.obj
 0002:00005998       ??_C@_0CN@GBAIPLPH@?$FLLobby?$FN?5Processing?5NAT?5negotiati@ 0000000039aaa998     CryGameSpySBQR2MatchMaking.obj
 0002:000059c8       ??_C@_0CJ@NANNAGOG@?$FLLobby?$FN?5?5?5?5?5Partner?3?5?5?5?5?5?5?5?5?5?5?5?5@ 0000000039aaa9c8     CryGameSpySBQR2MatchMaking.obj
 0002:000059f8       ??_C@_0N@FABGOMFN@other?5client?$AA@ 0000000039aaa9f8     CryGameSpySBQR2MatchMaking.obj
 0002:00005a08       ??_C@_06HJHJCKIO@server?$AA@ 0000000039aaaa08     CryGameSpySBQR2MatchMaking.obj
 0002:00005a10       ??_C@_0BM@BAGEGNHH@?$CF31?$FL?$FO?3?$FN?3?1?1?$CF21?$FL?40?99?3?$FN?1?$CF16llX?$AA@ 0000000039aaaa10     CryGameSpySBQR2MatchMaking.obj
 0002:00005a30       ??_C@_0GF@PJCNFHNK@CD?5key?5authentication?5timed?5out?5@ 0000000039aaaa30     CryGameSpySBQR2MatchMaking.obj
 0002:00005a98       ??_7?$CClassJobNoRef5@P6AXIW4ECryLobbyError@@PEAUSCrySessionSearchResult@@PEAX@ZIW41@PEAU2@PEAXVCCryGameSpySBQR2MatchMaking@@@CWorkQueue@@6B@ 0000000039aaaa98     CryGameSpySBQR2MatchMaking.obj
 0002:00005aa8       ??_7?$CClassJobNoRef4@IIIIVCCryGameSpySBQR2MatchMaking@@@CWorkQueue@@6B@ 0000000039aaaaa8     CryGameSpySBQR2MatchMaking.obj
 0002:00005ab8       ??_7SGameSpyKey@CCryGameSpySBQR2MatchMaking@@6B@ 0000000039aaaab8     CryGameSpySBQR2MatchMaking.obj
 0002:00005ac0       ??_7SRegisteredLobbyData@CCryGameSpySBQR2MatchMaking@@6B@ 0000000039aaaac0     CryGameSpySBQR2MatchMaking.obj
 0002:00005ac8       ??_C@_0CD@LEJJMDOD@?$FLLobby?$FN?5?5?5?5?5Result?3?5?5?5?5?5?5?5?5?5?5?5?5?5@ 0000000039aaaac8     CryGameSpySBQR2MatchMaking.obj
 0002:00005af0       ??_C@_0CM@LHPPLNOI@?$FLLobby?$FN?5Finishing?5NAT?5negotiatio@ 0000000039aaaaf0     CryGameSpySBQR2MatchMaking.obj
 0002:00005b20       ??_C@_0CL@MEICHIGD@?$FLLobby?$FN?5?5?5?5?5NAT?5negotiation?5alre@ 0000000039aaab20     CryGameSpySBQR2MatchMaking.obj
 0002:00005b50       ??_C@_0CO@DPELLPDD@?$FLLobby?$FN?5?5?5?5?5NAT?5negotiation?5alre@ 0000000039aaab50     CryGameSpySBQR2MatchMaking.obj
 0002:00005b80       ??_C@_0CM@OLHGBFM@?$FLLobby?$FN?5?5?5?5?5NAT?5negotiation?5alre@ 0000000039aaab80     CryGameSpySBQR2MatchMaking.obj
 0002:00005bb0       ??_C@_0DL@LCCFLPAP@?$FLLobby?$FN?5?5?5?5?5NAT?5negotiation?5fail@ 0000000039aaabb0     CryGameSpySBQR2MatchMaking.obj
 0002:00005bf0       ??_C@_0CC@LMAACEKA@?$FLLobby?$FN?5?5?5?5?5Sent?5cookie?5to?5serve@ 0000000039aaabf0     CryGameSpySBQR2MatchMaking.obj
 0002:00005c20       ??_C@_0FH@CKGDGMHL@?$FLLobby?$FN?5?5?5?5?5Partner?5behind?5same?5@ 0000000039aaac20     CryGameSpySBQR2MatchMaking.obj
 0002:00005c80       ??_C@_0FF@NGEHOIDF@?$FLLobby?$FN?5?5?5?5?5Partner?5behind?5same?5@ 0000000039aaac80     CryGameSpySBQR2MatchMaking.obj
 0002:00005cd8       ??_C@_0CL@NAEMEBDI@?$FLLobby?$FN?5Starting?5NAT?5negotiation@ 0000000039aaacd8     CryGameSpySBQR2MatchMaking.obj
 0002:00005d08       ??_C@_0M@BKHMLLGC@ban_timeout?$AA@ 0000000039aaad08     CryGameSpySBQR2MatchMaking.obj
 0002:00005d18       ??_C@_0CK@MCJKMNFP@?$CF31?$FL?$FO?3?$FN?3?1?1?$CF3hu?4?$CF3hu?4?$CF3hu?4?$CF3hu?3?$CF5@ 0000000039aaad18     CryGameSpySBQR2MatchMaking.obj
 0002:00005d48       ??_C@_0O@DNJPILDJ@cl_serveraddr?$AA@ 0000000039aaad48     CryGameSpySBQR2MatchMaking.obj
 0002:00005d58       ??_C@_0BJ@BOEHONPJ@?$CF3hu?4?$CF3hu?4?$CF3hu?4?$CF3hu?3?$CF5hu?$AA@ 0000000039aaad58     CryGameSpySBQR2MatchMaking.obj
 0002:00005d80       ??_C@_0HI@PNGEOHJI@?$FLLobby?$FN?5Send?5connection?5mmcid?5?$CFd@ 0000000039aaad80     CryGameSpySBQR2MatchMaking.obj
 0002:00005e00       ??_C@_0HM@DDBNIKEP@?$FLLobby?$FN?5Send?5new?5connection?5mmci@ 0000000039aaae00     CryGameSpySBQR2MatchMaking.obj
 0002:00005e80       ??_C@_0BC@FCFDBAEL@ed_lowercasepaths?$AA@ 0000000039aaae80     CryGameSpySBQR2MatchMaking.obj
 0002:00005e98       ??_C@_0BC@OJJABPH@?$HM?$CF?932s?$HM?$CF10s?$HM?$CF14s?$HM?$AA@ 0000000039aaae98     CryGameSpySBQR2MatchMaking.obj
 0002:00005eb0       ??_C@_0BE@LFCCKMGA@?$CF05d?3?$CF02d?3?$CF02d?3?$CF02d?$AA@ 0000000039aaaeb0     CryGameSpySBQR2MatchMaking.obj
 0002:00005ec8       ??_C@_0M@HPIECAAN@?$FLPERMANENT?$FN?$AA@ 0000000039aaaec8     CryGameSpySBQR2MatchMaking.obj
 0002:00005ed4       ??_C@_02GMHACPFF@?$CFu?$AA@ 0000000039aaaed4     CryGameSpySBQR2MatchMaking.obj
 0002:00005ed8       ??_C@_09NDGFAPBP@?$FLUNKNOWN?$FN?$AA@ 0000000039aaaed8     CryGameSpySBQR2MatchMaking.obj
 0002:00005ee8       ??_C@_07MJGJEDBB@expires?$AA@ 0000000039aaaee8     CryGameSpySBQR2MatchMaking.obj
 0002:00005ef0       ??_C@_0BC@PPEOHOLE@?$CFH?3?$CFM?3?$CFS?5?$CFd?1?$CFm?1?$CFY?$AA@ 0000000039aaaef0     CryGameSpySBQR2MatchMaking.obj
 0002:00005f04       ??_C@_02EGCJHIOB@id?$AA@   0000000039aaaf04     CryGameSpySBQR2MatchMaking.obj
 0002:00005f08       ??_C@_04MEMAJGDJ@name?$AA@ 0000000039aaaf08     CryGameSpySBQR2MatchMaking.obj
 0002:00005f10       ??_C@_0L@OFDOBKLE@BannedUser?$AA@ 0000000039aaaf10     CryGameSpySBQR2MatchMaking.obj
 0002:00005f20       ??_C@_0BO@KLMDEFIL@Cannot?5unban?5?$CFllu?3?5not?5banned?$AA@ 0000000039aaaf20     CryGameSpySBQR2MatchMaking.obj
 0002:00005f40       ??_C@_0O@PMEPLEJL@Unbanned?5?$CFllu?$AA@ 0000000039aaaf40     CryGameSpySBQR2MatchMaking.obj
 0002:00005f50       ??_C@_0BB@CEOGHOOH@Unbanned?5?$CFs?5?$CFllu?$AA@ 0000000039aaaf50     CryGameSpySBQR2MatchMaking.obj
 0002:00005f68       ??_C@_0BM@KNEMHOE@Cannot?5unban?5?$CFs?3?5not?5banned?$AA@ 0000000039aaaf68     CryGameSpySBQR2MatchMaking.obj
 0002:00005f88       ??_C@_0M@MJPCDEN@Unbanned?5?$CFs?$AA@ 0000000039aaaf88     CryGameSpySBQR2MatchMaking.obj
 0002:00005f98       ??_C@_0P@GKKHEBKN@Unbanned?5?$CFs?5?$CFu?$AA@ 0000000039aaaf98     CryGameSpySBQR2MatchMaking.obj
 0002:00005fa8       ??_C@_0DN@NLFMPHGD@?$HM?5?5?5?5?5?5?5?5?5?5?5?5?5?5Name?5?5?5?5?5?5?5?5?5?5?5?5?5@ 0000000039aaafa8     CryGameSpySBQR2MatchMaking.obj
 0002:00005fe8       ??_C@_0DN@CFJBNPFM@?$CL?9?9?9?9?9?9?9?9?9?9?9?9?9?9?9?9?9?9?9?9?9?9?9?9?9?9?9?9?9?9?9@ 0000000039aaafe8     CryGameSpySBQR2MatchMaking.obj
 0002:00006028       ??_C@_0BA@MMAIAPMA@?$CFs?3?1?1?$CFs?3?$CFd?1?$CFllX?$AA@ 0000000039aab028     CryGameSpySBQR2MatchMaking.obj
 0002:00006038       ??_C@_04HDOCAJNK@?$CFs?$CFs?$AA@ 0000000039aab038     CryGameSpySBQR2MatchMaking.obj
 0002:00006040       ??_C@_0L@OAPDKNNL@banned?4xml?$AA@ 0000000039aab040     CryGameSpySBQR2MatchMaking.obj
 0002:00006050       ??_C@_0P@NEMNJFNL@BannedUserList?$AA@ 0000000039aab050     CryGameSpySBQR2MatchMaking.obj
 0002:00006060       ??_C@_0CC@FPININNN@?$FLLobby?$FN?5Request?5join?5session?5?$CFll@ 0000000039aab060     CryGameSpySBQR2MatchMaking.obj
 0002:00006090       ??_C@_0GE@LHFOCNAC@Retrying?5CD?5key?5authentication?5f@ 0000000039aab090     CryGameSpySBQR2MatchMaking.obj
 0002:000060f8       ??_C@_0BN@EBODILIF@CD?5key?5authentication?5failed?$AA@ 0000000039aab0f8     CryGameSpySBQR2MatchMaking.obj
 0002:00006118       ??_C@_0BP@JHNBHKCB@Cannot?5ban?5?$CFu?3?5unknown?5profile?$AA@ 0000000039aab118     CryGameSpySBQR2MatchMaking.obj
 0002:00006140       ??_C@_0FJ@GFNFDKIA@Ban?5for?5?$CFs?5?$CFu?5expired?5before?5pro@ 0000000039aab140     CryGameSpySBQR2MatchMaking.obj
 0002:000061a0       ??_C@_0N@PLCGMPCN@Banned?5?$CFs?5?$CFu?$AA@ 0000000039aab1a0     CryGameSpySBQR2MatchMaking.obj
 0002:000061b0       ??_C@_0CD@OODHJHCF@Cannot?5ban?5?$CFs?3?5unknown?5unique?5ni@ 0000000039aab1b0     CryGameSpySBQR2MatchMaking.obj
 0002:000061e0       ??_C@_0FG@JHCFEMFN@Ban?5for?5?$CFs?5?$CFu?5expired?5before?5nam@ 0000000039aab1e0     CryGameSpySBQR2MatchMaking.obj
 0002:00006238       ??_C@_0CA@JJNJGBPJ@?$FLAndyC?$FN?3?5NAT?5neg?5timed?5out?5?$CFlld?$AA@ 0000000039aab238     CryGameSpySBQR2MatchMaking.obj
 0002:00006258       ??_C@_0BB@JAHKEOEL@?$CFs?$CFs?$CFs?$CFs?$CFs?$CFs?$CFs?$CFs?$AA@ 0000000039aab258     CryGameSpySBQR2MatchMaking.obj
 0002:0000626c       ??_C@_01GEODFPGF@?8?$AA@   0000000039aab26c     CryGameSpySBQR2MatchMaking.obj
 0002:00006270       ??_C@_05PAFDFGBB@?$CJ?$CB?$DN0?$CJ?$AA@ 0000000039aab270     CryGameSpySBQR2MatchMaking.obj
 0002:00006278       ??_C@_01HNPIGOCE@?$CG?$AA@ 0000000039aab278     CryGameSpySBQR2MatchMaking.obj
 0002:0000627c       ??_C@_02GLLNJPBP@?$CI?$CI?$AA@ 0000000039aab27c     CryGameSpySBQR2MatchMaking.obj
 0002:00006280       ??_C@_02EEKDKGMJ@?$DO?$DN?$AA@ 0000000039aab280     CryGameSpySBQR2MatchMaking.obj
 0002:00006284       ??_C@_01PPODPGHN@?$DO?$AA@ 0000000039aab284     CryGameSpySBQR2MatchMaking.obj
 0002:00006288       ??_C@_02EHCHHCKH@?$DM?$DN?$AA@ 0000000039aab288     CryGameSpySBQR2MatchMaking.obj
 0002:0000628c       ??_C@_01MNNFJEPP@?$DM?$AA@ 0000000039aab28c     CryGameSpySBQR2MatchMaking.obj
 0002:00006290       ??_C@_02FDNJECIE@?$CB?$DN?$AA@ 0000000039aab290     CryGameSpySBQR2MatchMaking.obj
 0002:00006294       ??_C@_01NEMOKFLO@?$DN?$AA@ 0000000039aab294     CryGameSpySBQR2MatchMaking.obj
 0002:00006298       ??_C@_0DH@DLEEBLMG@?$FLLobby?$FN?5Processed?5Session?5reques@ 0000000039aab298     CryGameSpySBQR2MatchMaking.obj
 0002:000062d0       ??_C@_0IE@MGHADJKB@?$FLLobby?$FN?5CCryGameSpySBQR2MatchMak@ 0000000039aab2d0     CryGameSpySBQR2MatchMaking.obj
 0002:00006360       ??_C@_0FD@MACCLLMO@?$FLLobby?$FN?5Add?5new?5connection?5sessi@ 0000000039aab360     CryGameSpySBQR2MatchMaking.obj
 0002:000063b8       ??_C@_0CN@NPPABOB@?$FLLobby?$FN?5Got?5new?5connections?5for?5@ 0000000039aab3b8     CryGameSpySBQR2MatchMaking.obj
 0002:000063e8       ??_C@_0DH@EHBKEOCL@?$FLLobby?$FN?5Processed?5session?5reques@ 0000000039aab3e8     CryGameSpySBQR2MatchMaking.obj
 0002:00006420       ??_C@_0FO@MIHCPOOH@?$FLLobby?$FN?5Created?5server?5connectio@ 0000000039aab420     CryGameSpySBQR2MatchMaking.obj
 0002:00006480       ??_C@_0EO@DOMCGNEK@?$FLLobby?$FN?5Created?5local?5connection@ 0000000039aab480     CryGameSpySBQR2MatchMaking.obj
 0002:000064d0       ??_C@_0DD@CCDNHLFH@?$FLLobby?$FN?5Received?5SessionRequestJ@ 0000000039aab4d0     CryGameSpySBQR2MatchMaking.obj
 0002:00006504       __real@42700000            0000000039aab504     CryGameSpySBQR2MatchMaking.obj
 0002:00006508       ??_C@_0P@BFGFNJAK@Banned?5?$CFs?5?$CFllu?$AA@ 0000000039aab508     CryGameSpySBQR2MatchMaking.obj
 0002:00006518       ??_C@_0DD@ECLGJMDC@Player?5?$CFllu?5not?5banned?5yet?0?5atte@ 0000000039aab518     CryGameSpySBQR2MatchMaking.obj
 0002:00006550       ??_C@_0DB@GOFPLLMJ@Player?5?$CFs?5not?5banned?5yet?0?5attemp@ 0000000039aab550     CryGameSpySBQR2MatchMaking.obj
 0002:00006588       ??_C@_0BC@PLBEOPGP@?$CFu?3?$CFu?3?$CFu?5?$CFu?1?$CFu?1?$CFu?$AA@ 0000000039aab588     CryGameSpySBQR2MatchMaking.obj
 0002:0000659c       ??_C@_02JDPG@rb?$AA@       0000000039aab59c     CryGameSpySBQR2MatchMaking.obj
 0002:000065a0       ??_7SSession@CCryGameSpySBQR2MatchMaking@@6B@ 0000000039aab5a0     CryGameSpySBQR2MatchMaking.obj
 0002:000065b8       ??_C@_0CP@IDEKGMPK@?$FLLobby?$FN?5Start?5SessionRegisterUse@ 0000000039aab5b8     CryGameSpySBQR2MatchMaking.obj
 0002:000065e8       ??_C@_0CF@KFHBMNGE@?$FLLobby?$FN?5Start?5SessionCreate?5erro@ 0000000039aab5e8     CryGameSpySBQR2MatchMaking.obj
 0002:00006610       ??_C@_0CI@JBNPKCOL@?$FLLobby?$FN?5Created?5local?5connection@ 0000000039aab610     CryGameSpySBQR2MatchMaking.obj
 0002:00006638       ??_C@_0CF@DPEAGPNE@?$FLLobby?$FN?5Start?5SessionSearch?5erro@ 0000000039aab638     CryGameSpySBQR2MatchMaking.obj
 0002:00006660       ??_C@_0CF@OJAEDAJC@?$FLLobby?$FN?5Start?5SessionDelete?5erro@ 0000000039aab660     CryGameSpySBQR2MatchMaking.obj
 0002:00006688       ??_C@_0CG@JAMKLKDC@?$FLLobby?$FN?5Start?5SessionMigrate?5err@ 0000000039aab688     CryGameSpySBQR2MatchMaking.obj
 0002:000066b0       ??_C@_0CF@CFEOMKPJ@?$FLLobby?$FN?5Start?5SessionUpdate?5erro@ 0000000039aab6b0     CryGameSpySBQR2MatchMaking.obj
 0002:000066d8       ??_C@_0CL@FCJBCPPN@?$FLLobby?$FN?5Start?5SessionUpdateSlots@ 0000000039aab6d8     CryGameSpySBQR2MatchMaking.obj
 0002:00006708       ??_C@_0CE@DLOBNHBN@?$FLLobby?$FN?5Start?5SessionQuery?5error@ 0000000039aab708     CryGameSpySBQR2MatchMaking.obj
 0002:00006730       ??_C@_0CH@OINHJPBO@?$FLLobby?$FN?5Start?5SessionGetUsers?5er@ 0000000039aab730     CryGameSpySBQR2MatchMaking.obj
 0002:00006758       ??_C@_0CE@FEFKAGL@?$FLLobby?$FN?5Start?5SessionStart?5error@ 0000000039aab758     CryGameSpySBQR2MatchMaking.obj
 0002:00006780       ??_C@_0CC@NCEDALHA@?$FLLobby?$FN?5Start?5SessionEnd?5error?5?$CF@ 0000000039aab780     CryGameSpySBQR2MatchMaking.obj
 0002:000067a8       ??_7CCryGameSpySBQR2MatchMaking@@6B@ 0000000039aab7a8     CryGameSpySBQR2MatchMaking.obj
 0002:000067c0       ??_7CCryGameSpySBQR2MatchMaking@@6BICryMatchMakingPrivate@@@ 0000000039aab7c0     CryGameSpySBQR2MatchMaking.obj
 0002:00006990       ??_7CCryGameSpySBQR2MatchMaking@@6BCMultiThreadRefCount@@@ 0000000039aab990     CryGameSpySBQR2MatchMaking.obj
 0002:000069e8       ??_C@_05LFNOAECD@?5AND?5?$AA@ 0000000039aab9e8     CryGameSpySBQR2MatchMaking.obj
 0002:000069f0       ??_C@_04MBNHLBPB@?5OR?5?$AA@ 0000000039aab9f0     CryGameSpySBQR2MatchMaking.obj
 0002:000069f8       ??_C@_06PPIPABNM@?5AND?5?$CI?$AA@ 0000000039aab9f8     CryGameSpySBQR2MatchMaking.obj
 0002:00006a00       ??_7SSessionLink@CCryGameSpySBQR2MatchMaking@@6B@ 0000000039aaba00     CryGameSpySBQR2MatchMaking.obj
 0002:00006a00       ??_7STaskLink@CCryGameSpySBQR2SignIn@@6B@ 0000000039aaba00     CryGameSpySBQR2SignIn.obj
 0002:00006a00       ??_7STaskLink@CCryGameSpySBQR2MatchMaking@@6B@ 0000000039aaba00     CryGameSpySBQR2MatchMaking.obj
 0002:00006a00       ??_7STaskLink@CCryGameSpySBQR2Friends@@6B@ 0000000039aaba00     CryGameSpySBQR2Friends.obj
 0002:00006a00       ??_7STaskLink@CCryGameSpySBQR2FriendsManagement@@6B@ 0000000039aaba00     CryGameSpySBQR2FriendsManagement.obj
 0002:00006a00       ??_7SThisLink@CCryGameSpySBQR2LobbyService@@6B@ 0000000039aaba00     CryGameSpySBQR2Lobby.obj
 0002:00006a00       ??_7CMultiThreadRefCount@@6B@ 0000000039aaba00     CryDLCStore.obj
 0002:00006a00       ??_7SThisLink@CCryGameSpySBQR2Friends@@6B@ 0000000039aaba00     CryGameSpySBQR2Friends.obj
 0002:00006a00       ??_7STaskLink@CCryGameSpySBQR2Stats@@6B@ 0000000039aaba00     CryGameSpySBQR2Stats.obj
 0002:00006a08       ??_7CCryGameSpySBQR2SignIn@@6BICrySignIn@@@ 0000000039aaba08     CryGameSpySBQR2SignIn.obj
 0002:00006a40       ??_7CCryGameSpySBQR2SignIn@@6BCMultiThreadRefCount@@@ 0000000039aaba40     CryGameSpySBQR2SignIn.obj
 0002:00006a98       ??_C@_0CC@MIAJONNO@?$FLLobby?$FN?5Start?5SignInUser?5error?5?$CF@ 0000000039aaba98     CryGameSpySBQR2SignIn.obj
 0002:00006ac0       ??_C@_0CD@DOPELBEG@?$FLLobby?$FN?5Start?5SignOutUser?5error?5@ 0000000039aabac0     CryGameSpySBQR2SignIn.obj
 0002:00006ae8       ??_C@_0CC@HEIKBPMP@?$FLLobby?$FN?5Start?5CreateUser?5error?5?$CF@ 0000000039aabae8     CryGameSpySBQR2SignIn.obj
 0002:00006b10       ??_C@_0CK@HKFNFDCF@?$FLLobby?$FN?5Start?5GetUserCredentials@ 0000000039aabb10     CryGameSpySBQR2SignIn.obj
 0002:00006b40       ??_C@_0N@CEFNBEOG@PROFILE?5?$DN?5?$CFd?$AA@ 0000000039aabb40     CryGameSpySBQR2Stats.obj
 0002:00006b50       ??_C@_0N@BDIGGIMF@ownerid?5?$DN?5?$CFd?$AA@ 0000000039aabb50     CryGameSpySBQR2Stats.obj
 0002:00006b60       ??_C@_0L@HPDDBGMB@SCORE?5desc?$AA@ 0000000039aabb60     CryGameSpySBQR2Stats.obj
 0002:00006b70       ??_C@_07ENELBAAD@FIELD?$CFd?$AA@ 0000000039aabb70     CryGameSpySBQR2Stats.obj
 0002:00006b78       ??_C@_04DFNBDBBL@DATA?$AA@ 0000000039aabb78     CryGameSpySBQR2Stats.obj
 0002:00006b80       ??_C@_05PKDFAPGJ@SCORE?$AA@ 0000000039aabb80     CryGameSpySBQR2Stats.obj
 0002:00006b88       ??_C@_08GNJFMINN@recordid?$AA@ 0000000039aabb88     CryGameSpySBQR2Stats.obj
 0002:00006b94       ??_C@_04IPKHEEB@NAME?$AA@  0000000039aabb94     CryGameSpySBQR2Stats.obj
 0002:00006ba0       ??_C@_07EAJOOGMN@PROFILE?$AA@ 0000000039aabba0     CryGameSpySBQR2Stats.obj
 0002:00006ba8       ??_C@_07FOFENMCI@ownerid?$AA@ 0000000039aabba8     CryGameSpySBQR2Stats.obj
 0002:00006bb0       ??_C@_03DMHICLNI@row?$AA@  0000000039aabbb0     CryGameSpySBQR2Stats.obj
 0002:00006bb8       ??_C@_0CI@DDBFHBAK@?$FLLobby?$FN?5Stats?5EndTask?5?$CFd?5?$CI?$CFd?$CJ?5Re@ 0000000039aabbb8     CryGameSpySBQR2Stats.obj
 0002:00006be0       ??_C@_07NBCGADJA@Unknown?$AA@ 0000000039aabbe0     CryGameSpySBQR2Stats.obj
 0002:00006be8       ??_C@_0DL@CMPAMOHE@?$FLLobby?$FN?5ReadUserDataCallback?5err@ 0000000039aabbe8     CryGameSpySBQR2Stats.obj
 0002:00006c28       ??_C@_0DJ@IEOJGCOC@?$FLLobby?$FN?5StartStatsReadLeaderBoar@ 0000000039aabc28     CryGameSpySBQR2Stats.obj
 0002:00006c68       ??_C@_0BM@ONMELLMO@Setting?5search?5filter?5to?5?$CFs?$AA@ 0000000039aabc68     CryGameSpySBQR2Stats.obj
 0002:00006c88       ??_C@_0DK@EMGMLIFN@?$FLLobby?$FN?5Start?5StatsReadLeaderBoa@ 0000000039aabc88     CryGameSpySBQR2Stats.obj
 0002:00006cc4       ??_C@_03ECMPIDPI@?$CFd?$CJ?$AA@ 0000000039aabcc4     CryGameSpySBQR2Stats.obj
 0002:00006cc8       ??_C@_04CAGLFDOE@?$CFd?0?5?$AA@ 0000000039aabcc8     CryGameSpySBQR2Stats.obj
 0002:00006cd0       ??_C@_07LKFPHOFI@?$CFs?5IN?5?$CI?$AA@ 0000000039aabcd0     CryGameSpySBQR2Stats.obj
 0002:00006cd8       ??_C@_0CO@NCECOAH@?$FLLobby?$FN?5Start?5StatsRegisterUserD@ 0000000039aabcd8     CryGameSpySBQR2Stats.obj
 0002:00006d08       ??_C@_0CL@JPEGAFLM@?$FLLobby?$FN?5Stats?5StatsWriteUserData@ 0000000039aabd08     CryGameSpySBQR2Stats.obj
 0002:00006d38       ??_C@_0CK@LNKAOLDD@?$FLLobby?$FN?5Start?5StatsReadUserData?5@ 0000000039aabd38     CryGameSpySBQR2Stats.obj
 0002:00006d70       ??_7CCryGameSpySBQR2Stats@@6BICryStats@@@ 0000000039aabd70     CryGameSpySBQR2Stats.obj
 0002:00006df0       ??_7CCryGameSpySBQR2Stats@@6BCMultiThreadRefCount@@@ 0000000039aabdf0     CryGameSpySBQR2Stats.obj
 0002:00006e08       ??_C@_0CK@DOILKBBO@?$FLLobby?$FN?5StartStatsWriteUserData?5@ 0000000039aabe08     CryGameSpySBQR2Stats.obj
 0002:00006e38       ??_C@_0CN@FMFHKPKD@?$FLLobby?$FN?5StartStatsWriteLeaderBoa@ 0000000039aabe38     CryGameSpySBQR2Stats.obj
 0002:00006e68       ??_C@_0DC@FDFLJIPN@?$FLLobby?$FN?5Start?5StatsRegisterLeade@ 0000000039aabe68     CryGameSpySBQR2Stats.obj
 0002:00006ea0       ??_C@_0CG@FCGKLCGM@?$FLVoice?$FN?3?5unregistering?5remote?5us@ 0000000039aabea0     CryGameSpySBQR2Voice.obj
 0002:00006ec8       ??_C@_0BM@ONLOAJAD@?$FLVoice?$FN?3?5created?$CFs?$CFs?5device?$AA@ 0000000039aabec8     CryGameSpySBQR2Voice.obj
 0002:00006ee8       ??_C@_08PMMMLBEH@?5capture?$AA@ 0000000039aabee8     CryGameSpySBQR2Voice.obj
 0002:00006ef8       ??_C@_09IJNDIKHO@?5playback?$AA@ 0000000039aabef8     CryGameSpySBQR2Voice.obj
 0002:00006f08       ??_C@_0DI@JEKLGBHJ@?$FLVoice?$FN?3?5captured?5?$CFi?5bytes?0?5fram@ 0000000039aabf08     CryGameSpySBQR2Voice.obj
 0002:00006f40       ??_C@_0DD@FPGACGOB@?$FLVoice?$FN?3?5playback?5from?5user?5?$CFi?0?5@ 0000000039aabf40     CryGameSpySBQR2Voice.obj
 0002:00006f74       ??_C@_02NFLNFON@NO?$AA@    0000000039aabf74     CryGameSpySBQR2Voice.obj
 0002:00006f78       ??_C@_03IPHJCBHH@YES?$AA@  0000000039aabf78     CryGameSpySBQR2Voice.obj
 0002:00006f80       ??_C@_0BM@LOLGKPKK@?$FLVoice?$FN?3?5gvStartup?$CI?$CJ?5failed?$AA@ 0000000039aabf80     CryGameSpySBQR2Voice.obj
 0002:00006fa0       ??_C@_0CE@KPJFELLK@?$FLVoice?$FN?3?5no?5default?5playback?5dev@ 0000000039aabfa0     CryGameSpySBQR2Voice.obj
 0002:00006fc8       ??_C@_0CD@PEAFNODE@?$FLVoice?$FN?3?5no?5default?5capture?5devi@ 0000000039aabfc8     CryGameSpySBQR2Voice.obj
 0002:00006ff0       ??_C@_0BN@ONFNALLM@?$FLVoice?$FN?3?5creating?5devices?4?4?4?$AA@ 0000000039aabff0     CryGameSpySBQR2Voice.obj
 0002:00007010       ??_C@_0CE@HFHDCBCJ@?$FLVoice?$FN?3?5received?5data?5from?5user@ 0000000039aac010     CryGameSpySBQR2Voice.obj
 0002:00007038       ??_C@_0CE@NCMEJLDB@?$FLVoice?$FN?3?5registering?5remote?5user@ 0000000039aac038     CryGameSpySBQR2Voice.obj
 0002:00007060       ??_7CCryGameSpySBQR2Voice@@6BICryVoice@@@ 0000000039aac060     CryGameSpySBQR2Voice.obj
 0002:000070c8       ??_7CCryGameSpySBQR2Voice@@6BCMultiThreadRefCount@@@ 0000000039aac0c8     CryGameSpySBQR2Voice.obj
 0002:000070e8       ??_C@_0CB@ODPMAKEP@?$FLVoice?$FN?3?5Sending?5data?5to?5user?5?$CFi@ 0000000039aac0e8     CryGameSpySBQR2Voice.obj
 0002:00007110       ??_C@_0DL@BFJLKBCH@?$FLVoice?$FN?3?5Remote?5user?5?$CFi?5?$CImuted?5g@ 0000000039aac110     CryGameSpySBQR2Voice.obj
 0002:0000714c       ??_C@_05MAJJAKPI@FALSE?$AA@ 0000000039aac14c     CryGameSpySBQR2Voice.obj
 0002:00007154       ??_C@_04HCDDPBNL@TRUE?$AA@ 0000000039aac154     CryGameSpySBQR2Voice.obj
 0002:00007160       ??_C@_0DC@PKPHOCKO@?$FLLobby?$FN?5eCLE_InternalError?3?5Game@ 0000000039aac160     GameSpySBQR2GPConnection.obj
 0002:00007198       ??_7?$SEventCallback@UGPRecvBuddyStatusArg@@@CGameSpySBQR2GPConnection@@6B@ 0000000039aac198     GameSpySBQR2GPConnection.obj
 0002:00007198       ??_7?$SEventCallback@UGPRecvBuddyRevokeArg@@@CGameSpySBQR2GPConnection@@6B@ 0000000039aac198     GameSpySBQR2GPConnection.obj
 0002:00007198       ??_7?$SEventCallback@UGPRecvBuddyAuthArg@@@CGameSpySBQR2GPConnection@@6B@ 0000000039aac198     GameSpySBQR2GPConnection.obj
 0002:00007198       ??_7?$SEventCallback@UGPRecvGameInviteArg@@@CGameSpySBQR2GPConnection@@6B@ 0000000039aac198     GameSpySBQR2GPConnection.obj
 0002:00007198       ??_7?$SEventCallback@UGPRecvBuddyMessageArg@@@CGameSpySBQR2GPConnection@@6B@ 0000000039aac198     GameSpySBQR2GPConnection.obj
 0002:00007198       ??_7?$SEventCallback@UGPErrorArg@@@CGameSpySBQR2GPConnection@@6B@ 0000000039aac198     GameSpySBQR2GPConnection.obj
 0002:00007198       ??_7?$SEventCallback@UGPRecvBuddyRequestArg@@@CGameSpySBQR2GPConnection@@6B@ 0000000039aac198     GameSpySBQR2GPConnection.obj
 0002:00007198       ??_7SCallbackBase@CGameSpySBQR2GPConnection@@6B@ 0000000039aac198     GameSpySBQR2GPConnection.obj
 0002:000071a0       ??_C@_07BMIEDOEC@Offline?$AA@ 0000000039aac1a0     GameSpySBQR2GPConnection.obj
 0002:000071a8       ??_7CGameSpySBQR2GPConnection@@6B@ 0000000039aac1a8     GameSpySBQR2GPConnection.obj
 0002:000071c8       ??_7STaskCallbackBase@CGameSpySBQR2GPConnection@@6B@ 0000000039aac1c8     GameSpySBQR2GPConnection.obj
 0002:000071e0       ??_7?$STaskCallbackMid@UGPGetReverseBuddiesResponseArg@@@CGameSpySBQR2GPConnection@@6B@ 0000000039aac1e0     GameSpySBQR2GPConnection.obj
 0002:000071e0       ??_7?$STaskCallbackMid@UGPCheckResponseArg@@@CGameSpySBQR2GPConnection@@6B@ 0000000039aac1e0     GameSpySBQR2GPConnection.obj
 0002:000071e0       ??_7?$STaskCallbackMid@UGPProfileSearchResponseArg@@@CGameSpySBQR2GPConnection@@6B@ 0000000039aac1e0     GameSpySBQR2GPConnection.obj
 0002:000071e0       ??_7?$STaskCallbackMid@UGPGetInfoResponseArg@@@CGameSpySBQR2GPConnection@@6B@ 0000000039aac1e0     GameSpySBQR2GPConnection.obj
 0002:000071e0       ??_7?$STaskCallbackMid@UGPRegisterUniqueNickResponseArg@@@CGameSpySBQR2GPConnection@@6B@ 0000000039aac1e0     GameSpySBQR2GPConnection.obj
 0002:000071e0       ??_7?$STaskCallbackMid@UGPConnectResponseArg@@@CGameSpySBQR2GPConnection@@6B@ 0000000039aac1e0     GameSpySBQR2GPConnection.obj
 0002:000071e0       ??_7?$STaskCallbackMid@UGPNewProfileResponseArg@@@CGameSpySBQR2GPConnection@@6B@ 0000000039aac1e0     GameSpySBQR2GPConnection.obj
 0002:000071e0       ??_7?$STaskCallbackMid@UGPNewUserResponseArg@@@CGameSpySBQR2GPConnection@@6B@ 0000000039aac1e0     GameSpySBQR2GPConnection.obj
 0002:000071f8       ??_7?$STaskCallback3@UGPCheckResponseArg@@V?$CryFixedStringT@$0BP@@@V?$CryFixedStringT@$0DD@@@V2@@CGameSpySBQR2GPConnection@@6B@ 0000000039aac1f8     GameSpySBQR2GPConnection.obj
 0002:00007210       ??_7?$STaskCallback4@UGPConnectResponseArg@@V?$CryFixedStringT@$0BP@@@V?$CryFixedStringT@$0DD@@@V2@W4GPEnum@@@CGameSpySBQR2GPConnection@@6B@ 0000000039aac210     GameSpySBQR2GPConnection.obj
 0002:00007228       ??_7?$STaskCallback3@UGPConnectResponseArg@@V?$CryFixedStringT@$0BF@@@V?$CryFixedStringT@$0BP@@@W4GPEnum@@@CGameSpySBQR2GPConnection@@6B@ 0000000039aac228     GameSpySBQR2GPConnection.obj
 0002:00007240       ??_7?$STaskCallback2@UGPGetInfoResponseArg@@HW4GPEnum@@@CGameSpySBQR2GPConnection@@6B@ 0000000039aac240     GameSpySBQR2GPConnection.obj
 0002:00007258       ??_7?$STaskCallback0@UGPGetReverseBuddiesResponseArg@@@CGameSpySBQR2GPConnection@@6B@ 0000000039aac258     GameSpySBQR2GPConnection.obj
 0002:00007270       ??_7?$STaskCallback2@UGPNewProfileResponseArg@@V?$CryFixedStringT@$0BP@@@W4GPEnum@@@CGameSpySBQR2GPConnection@@6B@ 0000000039aac270     GameSpySBQR2GPConnection.obj
 0002:00007288       ??_7?$STaskCallback5@UGPNewUserResponseArg@@V?$CryFixedStringT@$0BP@@@V?$CryFixedStringT@$0BF@@@V?$CryFixedStringT@$0DD@@@V2@PEBD@CGameSpySBQR2GPConnection@@6B@ 0000000039aac288     GameSpySBQR2GPConnection.obj
 0002:000072a0       ??_7?$STaskCallback6@UGPProfileSearchResponseArg@@V?$CryFixedStringT@$0BP@@@V?$CryFixedStringT@$0BF@@@V?$CryFixedStringT@$0DD@@@PEBDPEBDH@CGameSpySBQR2GPConnection@@6B@ 0000000039aac2a0     GameSpySBQR2GPConnection.obj
 0002:000072b8       ??_7?$STaskCallback3@UGPProfileSearchResponseArg@@V?$CryFixedStringT@$0BF@@@USIntPtrArg@CGameSpySBQR2GPConnection@@H@CGameSpySBQR2GPConnection@@6B@ 0000000039aac2b8     GameSpySBQR2GPConnection.obj
 0002:000072d0       ??_7?$STaskCallback2@UGPRegisterUniqueNickResponseArg@@V?$CryFixedStringT@$0BF@@@PEBD@CGameSpySBQR2GPConnection@@6B@ 0000000039aac2d0     GameSpySBQR2GPConnection.obj
 0002:000072f0       ??_C@_0EN@PAHNMBLI@?$CK?$CKWARNING?$CK?$CK?5CryLANLobbyService?3?3@ 0000000039aac2f0     CryLANLobby.obj
 0002:00007340       ??_7CCryLANLobbyService@@6BCMultiThreadRefCount@@@ 0000000039aac340     CryLANLobby.obj
 0002:000073a0       ??_7CCryLANLobbyService@@6BICryLobbyService@@@ 0000000039aac3a0     CryLANLobby.obj
 0002:00007430       ??_C@_0BA@CDJDKOOA@DedicatedServer?$AA@ 0000000039aac430     CryLANMatchMaking.obj
 0002:00007440       ??_7?$CClassJobNoRef@IVCCryGameSpySBQR2MatchMaking@@@CWorkQueue@@6B@ 0000000039aac440     CryGameSpySBQR2MatchMaking.obj
 0002:00007440       ??_7?$CClassJobNoRef@IVCCryMatchMaking@@@CWorkQueue@@6B@ 0000000039aac440     CryMatchMaking.obj
 0002:00007440       ??_7?$CClassJobNoRef@IVCCryLANMatchMaking@@@CWorkQueue@@6B@ 0000000039aac440     CryLANMatchMaking.obj
 0002:00007450       ??_7?$CClassJobNoRef5@IIGIIVCCryLANMatchMaking@@@CWorkQueue@@6B@ 0000000039aac450     CryLANMatchMaking.obj
 0002:00007460       ??_7SCryLANSessionID@@6B@  0000000039aac460     CryLANMatchMaking.obj
 0002:00007488       ??_C@_06NDDGGJP@?$CFd?5?3?$CFd?$AA@ 0000000039aac488     CryLANMatchMaking.obj
 0002:00007490       ??_7SCryLANUserID@@6B@     0000000039aac490     CryLANMatchMaking.obj
 0002:000074b0       ??_7SSession@CCryLANMatchMaking@@6B@ 0000000039aac4b0     CryLANMatchMaking.obj
 0002:000074c8       ??_C@_0CA@LJDICILL@Name?5resolution?5for?5?8?$CFs?8?5failed?$AA@ 0000000039aac4c8     CryLANMatchMaking.obj
 0002:000074e8       ??_C@_09JLECBOBH@?$DMsession?$DO?$AA@ 0000000039aac4e8     CryLANMatchMaking.obj
 0002:000074f8       ??_C@_0O@PJOPMKEO@cl_serverport?$AA@ 0000000039aac4f8     CryLANMatchMaking.obj
 0002:00007508       ??_C@_07LFLEPJNJ@?$CF016llx?$AA@ 0000000039aac508     CryLANMatchMaking.obj
 0002:00007510       ??_C@_0HC@DIDMAAOB@?$FLLobby?$FN?5Send?5connection?5mmcid?5?$CFd@ 0000000039aac510     CryLANMatchMaking.obj
 0002:00007588       ??_C@_0CA@OJHIHMPA@?$FLLobby?$FN?5Send?5new?5users?5to?5peers?$AA@ 0000000039aac588     CryLANMatchMaking.obj
 0002:000075b0       ??_C@_0HN@EDJJPLCH@?$FLLobby?$FN?5CCryLANMatchMaking?3?3Proc@ 0000000039aac5b0     CryLANMatchMaking.obj
 0002:00007630       ??_C@_0EH@LKGMDBMB@?$FLLobby?$FN?5Add?5new?5connection?5sessi@ 0000000039aac630     CryLANMatchMaking.obj
 0002:00007678       ??_C@_0CN@IEPLGEAJ@?$FLLobby?$FN?5Stop?5LAN?5search?5ticks?5?$CFd@ 0000000039aac678     CryLANMatchMaking.obj
 0002:000076b0       ??_C@_0EH@OAGGMCFE@?$FLLobby?$FN?5SessionJoin?5error?5sendin@ 0000000039aac6b0     CryLANMatchMaking.obj
 0002:00007700       ??_C@_0EK@PIEGKOKJ@?$FLLobby?$FN?5SessionJoin?5request?5sess@ 0000000039aac700     CryLANMatchMaking.obj
 0002:00007750       ??_C@_0EK@MEDKLOJD@?$FLLobby?$FN?5SessionJoin?5request?5sess@ 0000000039aac750     CryLANMatchMaking.obj
 0002:000077a0       ??_C@_0ED@BKKMIOKF@?$FLLobby?$FN?5Created?5server?5connectio@ 0000000039aac7a0     CryLANMatchMaking.obj
 0002:000077e8       ??_C@_0DM@DHBKKCLF@?$FLLobby?$FN?5Created?5local?5connection@ 0000000039aac7e8     CryLANMatchMaking.obj
 0002:00007828       ??_C@_0CF@DFLNAIPB@?$FLLobby?$FN?5Found?5Session?5?$CFd?4?$CFd?4?$CFd?4?$CF@ 0000000039aac828     CryLANMatchMaking.obj
 0002:00007850       ??_7CCryLANMatchMaking@@6BICryMatchMakingPrivate@@@ 0000000039aac850     CryLANMatchMaking.obj
 0002:00007a20       ??_7CCryLANMatchMaking@@6BCMultiThreadRefCount@@@ 0000000039aaca20     CryLANMatchMaking.obj
 0002:00007a78       ??_C@_0DK@MGELHDNF@?$FLGameSpy?$FN?5Invite?5to?5product?5?$CFd?0?5@ 0000000039aaca78     LobbyCVars.obj
 0002:00007ab8       ??_C@_07BIGACMLD@?$CFd?5?$CFllX?$AA@ 0000000039aacab8     LobbyCVars.obj
 0002:00007ac0       ??_C@_0BK@DBENICHM@?$FLGameSpy?$FN?5Friend?3?5?$CF?9?$CKs?5?$CFu?$AA@ 0000000039aacac0     LobbyCVars.obj
 0002:00007ae0       ??_C@_0CB@OFENOAPA@?$FLGameSpy?$FN?5Friend?5?$CFs?5from?5user?5?$CFd@ 0000000039aacae0     LobbyCVars.obj
 0002:00007b08       ??_C@_0BL@CEOOILDJ@?$FLGameSpy?$FN?5?$CFu?3?5is?$CFs?5blocked?$AA@ 0000000039aacb08     LobbyCVars.obj
 0002:00007b24       ??_C@_04CLDNJHDJ@?5not?$AA@ 0000000039aacb24     LobbyCVars.obj
 0002:00007b30       ??_C@_0BM@DDEKGBBM@?$FLGameSpy?$FN?5?$CFu?3?5is?$CFs?5a?5friend?$AA@ 0000000039aacb30     LobbyCVars.obj
 0002:00007b50       ??_C@_0BB@LLJJHLCO@?$FLGameSpy?$FN?5?$CFu?3?5?$CFs?$AA@ 0000000039aacb50     LobbyCVars.obj
 0002:00007b68       ??_C@_0BB@DLJKDPLF@?$FLGameSpy?$FN?5?$CFs?3?5?$CFu?$AA@ 0000000039aacb68     LobbyCVars.obj
 0002:00007b80       ??_C@_0CI@DEIEADPN@?$FLGameSpy?$FN?5Your?5GameSpy?5profile?5I@ 0000000039aacb80     LobbyCVars.obj
 0002:00007ba8       ??_C@_0CH@DJEPCICD@?$FLGameSpy?$FN?5Error?3?5no?5friends?5mana@ 0000000039aacba8     LobbyCVars.obj
 0002:00007bd0       ??_C@_0DH@OIJODKBN@?$FLGameSpy?$FN?5Error?3?5command?5require@ 0000000039aacbd0     LobbyCVars.obj
 0002:00007c08       ??_C@_0DH@KNFOBJFL@?$FLGameSpy?$FN?5Error?3?5argument?5must?5b@ 0000000039aacc08     LobbyCVars.obj
 0002:00007c40       ??_C@_0BP@HOPLJPCH@?$FLGameSpy?$FN?5Error?3?5out?5of?5memory?$AA@ 0000000039aacc40     LobbyCVars.obj
 0002:00007c60       ??_C@_0ED@KNPJOJFF@?$FLGameSpy?$FN?5Error?5accepting?5invite@ 0000000039aacc60     LobbyCVars.obj
 0002:00007ca8       ??_C@_0CN@LGIMFBKG@?$FLGameSpy?$FN?5Accepted?5invite?5from?5p@ 0000000039aacca8     LobbyCVars.obj
 0002:00007cd8       ??_C@_0CA@BEEHGDLA@?$FLGameSpy?$FN?5Error?3?5no?5matchmaking?$AA@ 0000000039aaccd8     LobbyCVars.obj
 0002:00007cf8       ??_C@_0BM@HAJBMHIK@?$FLGameSpy?$FN?5Error?3?5no?5friends?$AA@ 0000000039aaccf8     LobbyCVars.obj
 0002:00007d18       ??_C@_0CO@MGDNBDLI@?$FLGameSpy?$FN?5Error?3?5no?5current?5invi@ 0000000039aacd18     LobbyCVars.obj
 0002:00007d48       ??_C@_0DP@KEMGKDIP@?$FLGameSpy?$FN?5Error?5sending?5invite?5t@ 0000000039aacd48     LobbyCVars.obj
 0002:00007d88       ??_C@_0CH@EMHNHEHH@?$FLGameSpy?$FN?5Sent?5invite?5to?5profile@ 0000000039aacd88     LobbyCVars.obj
 0002:00007db0       ??_C@_0BO@GPLNALKA@?$FLGameSpy?$FN?5Now?5logging?5invites?$AA@ 0000000039aacdb0     LobbyCVars.obj
 0002:00007dd0       ??_C@_0CP@OMPPDEEL@?$FLGameSpy?$FN?5Error?5listing?5friends?3@ 0000000039aacdd0     LobbyCVars.obj
 0002:00007e00       ??_C@_0EH@IEFKHKO@?$FLGameSpy?$FN?5Error?5sending?5friend?5r@ 0000000039aace00     LobbyCVars.obj
 0002:00007e48       ??_C@_0CP@KBHDABBL@?$FLGameSpy?$FN?5Sent?5friend?5request?5to@ 0000000039aace48     LobbyCVars.obj
 0002:00007e80       ??_C@_0EL@OBPJIOKP@?$FLGameSpy?$FN?5Error?5accepting?5friend@ 0000000039aace80     LobbyCVars.obj
 0002:00007ed0       ??_C@_0DF@KIMKPIG@?$FLGameSpy?$FN?5Accepted?5friend?5reques@ 0000000039aaced0     LobbyCVars.obj
 0002:00007f10       ??_C@_0EI@PDJINCIM@?$FLGameSpy?$FN?5Error?5revoking?5friend?5@ 0000000039aacf10     LobbyCVars.obj
 0002:00007f58       ??_C@_0DC@LHCFBPHJ@?$FLGameSpy?$FN?5Revoked?5friend?5status?5@ 0000000039aacf58     LobbyCVars.obj
 0002:00007f90       ??_C@_0CE@OLIKJPFF@?$FLGameSpy?$FN?5Now?5logging?5friend?5eve@ 0000000039aacf90     LobbyCVars.obj
 0002:00007fb8       ??_C@_07MIJFAMBD@revoked?$AA@ 0000000039aacfb8     LobbyCVars.obj
 0002:00007fc0       ??_C@_0L@CCDCENAA@authorised?$AA@ 0000000039aacfc0     LobbyCVars.obj
 0002:00007fd0       ??_C@_07ENHGAJCI@request?$AA@ 0000000039aacfd0     LobbyCVars.obj
 0002:00007fd8       ??_C@_0DG@MBPNJLPN@?$FLGameSpy?$FN?5Error?5blocking?5profile@ 0000000039aacfd8     LobbyCVars.obj
 0002:00008010       ??_C@_0CA@LNJANDAJ@?$FLGameSpy?$FN?5Blocked?5profile?5ID?5?$CFu?$AA@ 0000000039aad010     LobbyCVars.obj
 0002:00008030       ??_C@_0DI@BJEDDADF@?$FLGameSpy?$FN?5Error?5unblocking?5profi@ 0000000039aad030     LobbyCVars.obj
 0002:00008068       ??_C@_0CC@OKIJOKJN@?$FLGameSpy?$FN?5Unblocked?5profile?5ID?5?$CF@ 0000000039aad068     LobbyCVars.obj
 0002:00008090       ??_C@_0DG@KDBGCOOF@?$FLGameSpy?$FN?5Error?5checking?5profile@ 0000000039aad090     LobbyCVars.obj
 0002:000080c8       ??_C@_0DH@HBAJPCK@?$FLGameSpy?$FN?5Error?3?5argument?5must?5b@ 0000000039aad0c8     LobbyCVars.obj
 0002:00008100       ??_C@_0EI@EBIAICFH@?$FLGameSpy?$FN?5Error?3?5argument?5must?5b@ 0000000039aad100     LobbyCVars.obj
 0002:00008148       ??_C@_0DA@FGHFCOOF@?$FLGameSpy?$FN?5Error?5checking?5name?5?$CFs@ 0000000039aad148     LobbyCVars.obj
 0002:00008178       ??_C@_0CC@HCJLCOAD@net_dedicatedServerArbitratorPor@ 0000000039aad178     LobbyCVars.obj
 0002:000081a0       ??_C@_0CA@LFKCMNGD@net_dedicatedServerArbitratorIP?$AA@ 0000000039aad1a0     LobbyCVars.obj
 0002:000081c0       ??_C@_0BC@CFHLHDAH@gamespy_find_user?$AA@ 0000000039aad1c0     LobbyCVars.obj
 0002:000081d8       ??_C@_0DE@BHBDICBL@Gets?5the?5ID?5of?5a?5profile?5with?5th@ 0000000039aad1d8     LobbyCVars.obj
 0002:00008210       ??_C@_0BB@BCOPFNME@gamespy_get_name?$AA@ 0000000039aad210     LobbyCVars.obj
 0002:00008228       ??_C@_0DE@LMPCPKLO@Gets?5the?5unique?5nick?5of?5a?5profil@ 0000000039aad228     LobbyCVars.obj
 0002:00008260       ??_C@_0BH@HAIFLNPK@gamespy_is_user_friend?$AA@ 0000000039aad260     LobbyCVars.obj
 0002:00008278       ??_C@_0CA@BCIDMDHC@Checks?5if?5a?5profile?5is?5a?5friend?$AA@ 0000000039aad278     LobbyCVars.obj
 0002:00008298       ??_C@_0BO@EAJFEKKJ@gamespy_is_profile_id_blocked?$AA@ 0000000039aad298     LobbyCVars.obj
 0002:000082b8       ??_C@_0BP@FJLIFAAN@Checks?5if?5a?5profile?5is?5blocked?$AA@ 0000000039aad2b8     LobbyCVars.obj
 0002:000082d8       ??_C@_0BL@NAPBKCBB@gamespy_unblock_profile_id?$AA@ 0000000039aad2d8     LobbyCVars.obj
 0002:000082f8       ??_C@_0BF@COJAEFOO@Unblock?5a?5profile?5id?$AA@ 0000000039aad2f8     LobbyCVars.obj
 0002:00008310       ??_C@_0BJ@EDPGHPLK@gamespy_block_profile_id?$AA@ 0000000039aad310     LobbyCVars.obj
 0002:00008330       ??_C@_0BD@JHMCFMFM@Block?5a?5profile?5id?$AA@ 0000000039aad330     LobbyCVars.obj
 0002:00008348       ??_C@_0BK@DCOLBCBA@gamespy_log_friend_events?$AA@ 0000000039aad348     LobbyCVars.obj
 0002:00008368       ??_C@_0BK@DCAEELAE@Log?5GameSpy?5friend?5events?$AA@ 0000000039aad368     LobbyCVars.obj
 0002:00008388       ??_C@_0BN@KHNGBDD@gamespy_revoke_friend_status?$AA@ 0000000039aad388     LobbyCVars.obj
 0002:000083a8       ??_C@_0BN@NNCLHPGA@Revoke?5GameSpy?5friend?5status?$AA@ 0000000039aad3a8     LobbyCVars.obj
 0002:000083c8       ??_C@_0BO@EENLEBE@gamespy_accept_friend_request?$AA@ 0000000039aad3c8     LobbyCVars.obj
 0002:000083e8       ??_C@_0CA@PMAOMBID@Accept?5a?5GameSpy?5friend?5request?$AA@ 0000000039aad3e8     LobbyCVars.obj
 0002:00008408       ??_C@_0BM@OGAMADCM@gamespy_send_friend_request?$AA@ 0000000039aad408     LobbyCVars.obj
 0002:00008428       ??_C@_0BO@KGAPNBGA@Send?5a?5GameSpy?5friend?5request?$AA@ 0000000039aad428     LobbyCVars.obj
 0002:00008448       ??_C@_0BF@NPGNIFEP@gamespy_list_friends?$AA@ 0000000039aad448     LobbyCVars.obj
 0002:00008460       ??_C@_0BF@CDOOMGKH@List?5GameSpy?5friends?$AA@ 0000000039aad460     LobbyCVars.obj
 0002:00008478       ??_C@_0BG@IDJCOJBJ@gamespy_accept_invite?$AA@ 0000000039aad478     LobbyCVars.obj
 0002:00008490       ??_C@_0BI@KDILNKIN@Accept?5a?5GameSpy?5invite?$AA@ 0000000039aad490     LobbyCVars.obj
 0002:000084a8       ??_C@_0BE@OMPABOEM@gamespy_send_invite?$AA@ 0000000039aad4a8     LobbyCVars.obj
 0002:000084c0       ??_C@_0BG@LFEEBBIA@Send?5a?5GameSpy?5invite?$AA@ 0000000039aad4c0     LobbyCVars.obj
 0002:000084d8       ??_C@_0BE@IJNFGID@gamespy_log_invites?$AA@ 0000000039aad4d8     LobbyCVars.obj
 0002:000084f0       ??_C@_0BE@NIEFJGAL@Log?5GameSpy?5invites?$AA@ 0000000039aad4f0     LobbyCVars.obj
 0002:00008508       ??_C@_0BH@KOBHPEDJ@gamespy_get_profile_id?$AA@ 0000000039aad508     LobbyCVars.obj
 0002:00008520       ??_C@_0CC@HBFJGPHJ@Get?5GameSpy?5profile?5ID?5for?5user?5@ 0000000039aad520     LobbyCVars.obj
 0002:00008548       ??_C@_0BM@MCGFPPBL@gamespy_search_ping_timeout?$AA@ 0000000039aad548     LobbyCVars.obj
 0002:00008568       ??_C@_0CM@MBBMMBNL@GameSpy?5search?5ping?5timeout?5in?5m@ 0000000039aad568     LobbyCVars.obj
 0002:00008598       ??_C@_0BK@KGJBAHFF@gamespy_search_ping_retry?$AA@ 0000000039aad598     LobbyCVars.obj
 0002:000085b8       ??_C@_0DD@DKFAAMPL@GameSpy?5search?5ping?5retry?5interv@ 0000000039aad5b8     LobbyCVars.obj
 0002:000085f0       ??_C@_0CM@DODLOFAE@net_lobby_gamespy_cdkey_timeout_@ 0000000039aad5f0     LobbyCVars.obj
 0002:00008620       ??_C@_0ED@HMOJOMGO@Whether?5if?5all?5CD?5key?5timeouts?5e@ 0000000039aad620     LobbyCVars.obj
 0002:00008668       ??_C@_0CG@FKGLHNDC@net_lobby_gamespy_retry_cdkey_ti@ 0000000039aad668     LobbyCVars.obj
 0002:00008690       ??_C@_0ED@IIIOCBHG@How?5long?5to?5wait?5before?5retrying@ 0000000039aad690     LobbyCVars.obj
 0002:000086d8       ??_C@_0CG@NHNIDINA@net_lobby_gamespy_allow_cdkey_ti@ 0000000039aad6d8     LobbyCVars.obj
 0002:00008700       ??_C@_0DF@LMHGDOJM@Can?5clients?5join?5if?5CD?5key?5authe@ 0000000039aad700     LobbyCVars.obj
 0002:00008738       ??_C@_0BP@FOKALAJ@net_lobby_gamespy_session_ping?$AA@ 0000000039aad738     LobbyCVars.obj
 0002:00008760       ??_C@_0EI@CNDPCKAF@Toggle?5whether?5a?5ping?5is?5sent?5to@ 0000000039aad760     LobbyCVars.obj
 0002:000087a8       ??_C@_0BP@JFMMPKNB@net_lobby_gamespy_client_cdkey?$AA@ 0000000039aad7a8     LobbyCVars.obj
 0002:000087c8       ??_C@_0DA@ILDLCMDM@Toggle?5whether?5the?5client?5authen@ 0000000039aad7c8     LobbyCVars.obj
 0002:000087f8       ??_C@_0BP@LJBGIIKE@net_lobby_gamespy_server_cdkey?$AA@ 0000000039aad7f8     LobbyCVars.obj
 0002:00008818       ??_C@_0DA@NPFFCFOE@Toggle?5whether?5the?5server?5authen@ 0000000039aad818     LobbyCVars.obj
 0002:00008848       ??_C@_0CB@FGBBEFAF@net_lobby_gamespy_search_timeout@ 0000000039aad848     LobbyCVars.obj
 0002:00008870       ??_C@_0DK@LBCBKODC@How?5long?5to?5wait?5without?5updates@ 0000000039aad870     LobbyCVars.obj
 0002:000088b0       ??_C@_0CD@HEGLLOKL@net_lobby_gamespy_server_ping_wa@ 0000000039aad8b0     LobbyCVars.obj
 0002:000088e0       ??_C@_0GI@GPNBBBAG@How?5long?5to?5wait?5for?5a?5server?5to@ 0000000039aad8e0     LobbyCVars.obj
 0002:00008948       ??_C@_0CG@DNMMIAFH@net_lobby_gamespy_symmetrical_fr@ 0000000039aad948     LobbyCVars.obj
 0002:00008970       ??_C@_0DO@NKNKIHEC@Toggle?5whether?5GameSpy?5friend?5re@ 0000000039aad970     LobbyCVars.obj
 0002:000089b0       ??_C@_0CK@MNJDHFPL@net_lobby_gamespy_connection_wai@ 0000000039aad9b0     LobbyCVars.obj
 0002:000089e0       ??_C@_0CP@HMOOJJK@Modify?5the?5connection?5wait?5timeo@ 0000000039aad9e0     LobbyCVars.obj
 0002:00008a10       ??_C@_0BO@HGNEBAIG@net_lobby_gamespy_online_port?$AA@ 0000000039aada10     LobbyCVars.obj
 0002:00008a30       ??_C@_0CD@OELNJJGK@Modify?5the?5online?5port?5for?5GameS@ 0000000039aada30     LobbyCVars.obj
 0002:00008a58       ??_C@_0BD@LGLPJJDC@cld_max_delay_time?$AA@ 0000000039aada58     LobbyCVars.obj
 0002:00008a70       ??_C@_0FE@CIJHBPME@The?5maximum?5time?5a?5cry?5lobby?5tas@ 0000000039aada70     LobbyCVars.obj
 0002:00008ac8       ??_C@_0BD@JBAEPOAD@cld_min_delay_time?$AA@ 0000000039aadac8     LobbyCVars.obj
 0002:00008ae0       ??_C@_0FE@KAFOIHIL@The?5minimum?5time?5a?5cry?5lobby?5tas@ 0000000039aadae0     LobbyCVars.obj
 0002:00008b38       ??_C@_0BF@PNGFDLKE@cld_error_percentage?$AA@ 0000000039aadb38     LobbyCVars.obj
 0002:00008b50       ??_C@_0DN@JMNMPKIH@How?5often?5a?5cry?5lobby?5task?5will?5@ 0000000039aadb50     LobbyCVars.obj
 0002:00008b90       ??_C@_0L@JMFGKKKN@cld_enable?$AA@ 0000000039aadb90     LobbyCVars.obj
 0002:00008ba0       ??_C@_0BN@PBCIOMPO@Enable?5cry?5lobby?5debug?5tests?$AA@ 0000000039aadba0     LobbyCVars.obj
 0002:00008bc0       ??_C@_0BL@LDKJGIAD@net_show_matchmaking_tasks?$AA@ 0000000039aadbc0     LobbyCVars.obj
 0002:00008be0       ??_C@_0EB@NBIGHMKD@Toggles?5whether?5active?5matchmaki@ 0000000039aadbe0     LobbyCVars.obj
 0002:00008c28       ??_C@_0CD@BIFFIPHB@net_serverpingnotificationinterv@ 0000000039aadc28     LobbyCVars.obj
 0002:00008c50       ??_C@_0DI@OELOEHAG@minimum?5interval?5between?5server?5@ 0000000039aadc50     LobbyCVars.obj
 0002:00008c88       ??_C@_0CG@CNMLGILB@net_minMicrophoneNotificationInt@ 0000000039aadc88     LobbyCVars.obj
 0002:00008cb0       ??_C@_0EG@BGAIHHJE@minimum?5interval?5between?5microph@ 0000000039aadcb0     LobbyCVars.obj
 0002:00008cf8       ??_C@_06HPGEIPLA@?$DMnull?$DO?$AA@ 0000000039aadcf8     StdAfx.obj
 0002:00008d00       ??_C@_07KAALEJHI@?$DMlocal?$DO?$AA@ 0000000039aadd00     StdAfx.obj
 0002:00008d08       _pRawDllMain               0000000039aadd08     MSVCRT:crtdll.obj
 0002:00008d08       _pDefaultRawDllMain        0000000039aadd08     MSVCRT:crtdll.obj
 0002:00008d10       ??_C@_05NNFHCGPF@?$CFs?4?$CFs?$AA@ 0000000039aadd10     GameSpy_2.11.00_VC10:natneg.obj
 0002:00008d18       ??_C@_0BE@FHOMNIIC@natneg3?4gamespy?4com?$AA@ 0000000039aadd18     GameSpy_2.11.00_VC10:natneg.obj
 0002:00008d30       ??_C@_0BE@MKODDJPE@natneg2?4gamespy?4com?$AA@ 0000000039aadd30     GameSpy_2.11.00_VC10:natneg.obj
 0002:00008d48       ??_C@_0BE@LGICBMCP@natneg1?4gamespy?4com?$AA@ 0000000039aadd48     GameSpy_2.11.00_VC10:natneg.obj
 0002:00008d60       ??_C@_0BJ@LCIEOOLF@?$CFs?4available?4gamespy?4com?$AA@ 0000000039aadd60     GameSpy_2.11.00_VC10:gsAvailable.obj
 0002:00008d7c       ??_C@_03NENMBKLN@?$PO?$PN?7?$AA@ 0000000039aadd7c     GameSpy_2.11.00_VC10:gsAvailable.obj
 0002:00008d80       ??_C@_01KICIPPFI@?2?$AA@   0000000039aadd80     GameSpy_2.11.00_VC10:ptMain.obj
 0002:00008d90       ??_C@_0EP@IHMDHNBL@?$CFs?$DPuserid?$DN?$CFd?$CGproductid?$DN?$CFd?$CGversio@ 0000000039aadd90     GameSpy_2.11.00_VC10:ptMain.obj
 0002:00008de0       ??_C@_0CG@MCNPLPOO@http?3?1?1motd?4gamespy?4com?1motd?1mot@ 0000000039aadde0     GameSpy_2.11.00_VC10:ptMain.obj
 0002:00008e20       ??_C@_0BB@IENBKNDD@InstalledContent?$AA@ 0000000039aade20     GameSpy_2.11.00_VC10:d2gMain.obj
 0002:00008e34       ??_C@_05DNKPJHDO@?2ka?2?$AA?$AA@ 0000000039aade34     GameSpy_2.11.00_VC10:gcdkeys.obj
 0002:00008e3c       ??_C@_04BDGLLBHF@?2?$CFs?2?$AA@ 0000000039aade3c     GameSpy_2.11.00_VC10:gcdkeys.obj
 0002:00008e48       ??_C@_0M@PCDKKIFJ@owatagusiam?$AA@ 0000000039aade48     GameSpy_2.11.00_VC10:gcdkeys.obj
 0002:00008e54       ??_C@_01LFCBOECM@?4?$AA@   0000000039aade54     GameSpy_2.11.00_VC10:gcdkeys.obj
 0002:00008e58       ??_C@_06PFFBCHML@?$CFs?$CFd?$CFs?$AA@ 0000000039aade58     GameSpy_2.11.00_VC10:gcdkeyc.obj
 0002:00008e60       ??_C@_04LNIPDHEN@?$CF?48x?$AA@ 0000000039aade60     GameSpy_2.11.00_VC10:gcdkeyc.obj
 0002:00008e68       ??_C@_0BN@GKKACOKD@CD?5Key?5or?5challenge?5too?5long?$AA@ 0000000039aade68     GameSpy_2.11.00_VC10:gcdkeyc.obj
 0002:00008e88       ??_C@_03GFPEDOMH@?2?$CFs?$AA@ 0000000039aade88     GameSpy_2.11.00_VC10:sb_serverbrowsing.obj
 0002:00008e90       ??_C@_0BA@FELBPFAN@255?4255?4255?4255?$AA@ 0000000039aade90     GameSpy_2.11.00_VC10:qr2.obj
 0002:00008ea0       ??_C@_08IHAGNMKK@?$CF08X?$CF04X?$AA@ 0000000039aadea0     GameSpy_2.11.00_VC10:qr2.obj
 0002:00008eb0       ??_C@_07CIFAGBMG@unknown?$AA@ 0000000039aadeb0     GameSpy_2.11.00_VC10:qr2.obj
 0002:00008eb8       ??_C@_08EKKHIELM@splitnum?$AA@ 0000000039aadeb8     GameSpy_2.11.00_VC10:qr2.obj
 0002:00008ec8       ??_C@_0BG@EGCNNADC@?$CFs?4master?4gamespy?4com?$AA@ 0000000039aadec8     GameSpy_2.11.00_VC10:qr2.obj
 0002:00008ee0       ??_C@_02DPKJAMEF@?$CFd?$AA@ 0000000039aadee0     GameSpy_2.11.00_VC10:qr2.obj
 0002:00008ee4       ??_C@_04NOJCDH@?$CF02x?$AA@ 0000000039aadee4     GameSpy_2.11.00_VC10:qr2.obj
 0002:00008ef0       ??_C@_0L@JJBEDNHO@publicport?$AA@ 0000000039aadef0     GameSpy_2.11.00_VC10:qr2.obj
 0002:00008f00       ??_C@_08LLHCOBBF@publicip?$AA@ 0000000039aadf00     GameSpy_2.11.00_VC10:qr2.obj
 0002:00008f10       ??_C@_08HCPAIKAO@gamename?$AA@ 0000000039aadf10     GameSpy_2.11.00_VC10:qr2.obj
 0002:00008f20       ??_C@_0N@ECBOGDJG@statechanged?$AA@ 0000000039aadf20     GameSpy_2.11.00_VC10:qr2.obj
 0002:00008f30       ??_C@_06MJLJPJFC@natneg?$AA@ 0000000039aadf30     GameSpy_2.11.00_VC10:qr2.obj
 0002:00008f38       ??_C@_09NOFGBFHM@localport?$AA@ 0000000039aadf38     GameSpy_2.11.00_VC10:qr2.obj
 0002:00008f48       ??_C@_09JIONINCC@localip?$CFd?$AA@ 0000000039aadf48     GameSpy_2.11.00_VC10:qr2.obj
 0002:00008f58       ??_C@_0DI@NMCMFPIB@No?5challenge?5value?5was?5received?5@ 0000000039aadf58     GameSpy_2.11.00_VC10:qr2.obj
 0002:00008f90       ??_C@_0O@LKGEAOMK@Invalid?5func?4?$AA@ 0000000039aadf90     GameSpy_2.11.00_VC10:gp.obj
 0002:00008fa0       ??_C@_0N@FGFIGEJF@No?5callback?4?$AA@ 0000000039aadfa0     GameSpy_2.11.00_VC10:gp.obj
 0002:00008fb0       ??_C@_0BD@MBOMGJAB@Password?5too?5long?4?$AA@ 0000000039aadfb0     GameSpy_2.11.00_VC10:gp.obj
 0002:00008fc8       ??_C@_0BA@IJBPCDAG@Email?5too?5long?4?$AA@ 0000000039aadfc8     GameSpy_2.11.00_VC10:gp.obj
 0002:00008fd8       ??_C@_0BF@FIEJEJLG@Uniquenick?5too?5long?4?$AA@ 0000000039aadfd8     GameSpy_2.11.00_VC10:gp.obj
 0002:00008ff0       ??_C@_0P@CHGIFCA@Nick?5too?5long?4?$AA@ 0000000039aadff0     GameSpy_2.11.00_VC10:gp.obj
 0002:00009000       ??_C@_0CO@FFBNBMHF@The?5connection?5has?5already?5been?5@ 0000000039aae000     GameSpy_2.11.00_VC10:gp.obj
 0002:00009030       ??_C@_0O@PFOHPEB@Invalid?5nick?4?$AA@ 0000000039aae030     GameSpy_2.11.00_VC10:gp.obj
 0002:00009040       ??_C@_0BB@LFPJPPAD@Invalid?5profile?4?$AA@ 0000000039aae040     GameSpy_2.11.00_VC10:gp.obj
 0002:00009058       ??_C@_0BA@LCNCPOLB@Invalid?5reason?4?$AA@ 0000000039aae058     GameSpy_2.11.00_VC10:gp.obj
 0002:00009068       ??_C@_0P@OILPNBEC@Invalid?5index?4?$AA@ 0000000039aae068     GameSpy_2.11.00_VC10:gp.obj
 0002:00009078       ??_C@_0BA@CGKLDCJN@Invalid?5status?4?$AA@ 0000000039aae078     GameSpy_2.11.00_VC10:gp.obj
 0002:00009088       ??_C@_07KNJCJIAE@?2final?2?$AA@ 0000000039aae088     GameSpy_2.11.00_VC10:gp.obj
 0002:00009090       ??_C@_0M@MKMIFMAO@?2locstring?2?$AA@ 0000000039aae090     GameSpy_2.11.00_VC10:gp.obj
 0002:000090a0       ??_C@_0N@IFKBCMGF@?2statstring?2?$AA@ 0000000039aae0a0     GameSpy_2.11.00_VC10:gp.obj
 0002:000090b0       ??_C@_09BBHKBFLD@?2sesskey?2?$AA@ 0000000039aae0b0     GameSpy_2.11.00_VC10:gp.obj
 0002:000090c0       ??_C@_08GEMKDFHH@?2status?2?$AA@ 0000000039aae0c0     GameSpy_2.11.00_VC10:gp.obj
 0002:000090d0       ??_C@_0BI@LCDLJEHJ@Invalid?5locationString?4?$AA@ 0000000039aae0d0     GameSpy_2.11.00_VC10:gp.obj
 0002:000090e8       ??_C@_0BG@LMGPNHBL@Invalid?5statusString?4?$AA@ 0000000039aae0e8     GameSpy_2.11.00_VC10:gp.obj
 0002:00009100       ??_C@_0BB@IKBMMLEF@Invalid?5message?4?$AA@ 0000000039aae100     GameSpy_2.11.00_VC10:gp.obj
 0002:00009118       ??_C@_0L@OOOLACLO@?2location?2?$AA@ 0000000039aae118     GameSpy_2.11.00_VC10:gp.obj
 0002:00009128       ??_C@_0M@EFCCMECF@?2productid?2?$AA@ 0000000039aae128     GameSpy_2.11.00_VC10:gp.obj
 0002:00009138       ??_C@_0M@LKPDJAF@?2profileid?2?$AA@ 0000000039aae138     GameSpy_2.11.00_VC10:gp.obj
 0002:00009148       ??_C@_09KOMFGJAK@?2pinvite?2?$AA@ 0000000039aae148     GameSpy_2.11.00_VC10:gp.obj
 0002:00009158       ??_C@_07FEIIEBCL@?2quiet?2?$AA@ 0000000039aae158     GameSpy_2.11.00_VC10:gp.obj
 0002:00009160       ??_C@_0CG@LMHCALKI@ns1?$DN?$CChttp?3?1?1gamespy?4net?1AuthServ@ 0000000039aae160     GameSpy_2.11.00_VC10:AuthService.obj
 0002:00009190       WS_AUTHSERVICE_SIGNATURE_KEY 0000000039aae190     GameSpy_2.11.00_VC10:AuthService.obj
 0002:00009294       WS_AUTHSERVICE_SIGNATURE_EXP 0000000039aae294     GameSpy_2.11.00_VC10:AuthService.obj
 0002:000092a0       ??_C@_0EA@NIIANJDJ@https?3?1?1?$CFs?4auth?4pubsvs?4gamespy?4c@ 0000000039aae2a0     GameSpy_2.11.00_VC10:AuthService.obj
 0002:000092e0       ??_C@_0N@ODBLELLB@responseCode?$AA@ 0000000039aae2e0     GameSpy_2.11.00_VC10:AuthService.obj
 0002:000092f0       ??_C@_05LPIJGKJ@Value?$AA@ 0000000039aae2f0     GameSpy_2.11.00_VC10:AuthService.obj
 0002:000092f8       ??_C@_0M@HPBMEKFC@namespaceid?$AA@ 0000000039aae2f8     GameSpy_2.11.00_VC10:AuthService.obj
 0002:00009308       ??_C@_0M@NOEPFNDH@partnercode?$AA@ 0000000039aae308     GameSpy_2.11.00_VC10:AuthService.obj
 0002:00009314       ??_C@_06MEOHGENE@gameid?$AA@ 0000000039aae314     GameSpy_2.11.00_VC10:AuthService.obj
 0002:00009320       ??_C@_07CPCPJPKL@version?$AA@ 0000000039aae320     GameSpy_2.11.00_VC10:AuthService.obj
 0002:00009328       ??_C@_03JFKIHBGI@ns1?$AA@  0000000039aae328     GameSpy_2.11.00_VC10:AuthService.obj
 0002:00009330       ??_C@_07PBILKAFL@Success?$AA@ 0000000039aae330     GameSpy_2.11.00_VC10:AuthService.obj
 0002:00009338       ??_C@_09CMIIOJHF@signature?$AA@ 0000000039aae338     GameSpy_2.11.00_VC10:AuthService.obj
 0002:00009348       ??_C@_0L@CPEONCJI@serverdata?$AA@ 0000000039aae348     GameSpy_2.11.00_VC10:AuthService.obj
 0002:00009358       ??_C@_0BA@ECDJDPNB@peerkeyexponent?$AA@ 0000000039aae358     GameSpy_2.11.00_VC10:AuthService.obj
 0002:00009368       ??_C@_0P@FGAHHJLA@peerkeymodulus?$AA@ 0000000039aae368     GameSpy_2.11.00_VC10:AuthService.obj
 0002:00009378       ??_C@_09IOEDOALI@cdkeyhash?$AA@ 0000000039aae378     GameSpy_2.11.00_VC10:AuthService.obj
 0002:00009388       ??_C@_0L@OMEPFEF@uniquenick?$AA@ 0000000039aae388     GameSpy_2.11.00_VC10:AuthService.obj
 0002:00009398       ??_C@_0M@HOIEEBNN@profilenick?$AA@ 0000000039aae398     GameSpy_2.11.00_VC10:AuthService.obj
 0002:000093a8       ??_C@_0L@FOFFKPLM@expiretime?$AA@ 0000000039aae3a8     GameSpy_2.11.00_VC10:AuthService.obj
 0002:000093b8       ??_C@_09OMJCKPGJ@profileid?$AA@ 0000000039aae3b8     GameSpy_2.11.00_VC10:AuthService.obj
 0002:000093c4       ??_C@_06IHAGGOEE@userid?$AA@ 0000000039aae3c4     GameSpy_2.11.00_VC10:AuthService.obj
 0002:000093cc       ??_C@_06IJDLPEM@length?$AA@ 0000000039aae3cc     GameSpy_2.11.00_VC10:AuthService.obj
 0002:000093d8       ??_C@_0P@KDLOMOHH@peerkeyprivate?$AA@ 0000000039aae3d8     GameSpy_2.11.00_VC10:AuthService.obj
 0002:000093e8       ??_C@_0M@LLNFCECG@certificate?$AA@ 0000000039aae3e8     GameSpy_2.11.00_VC10:AuthService.obj
 0002:000093f8       ??_C@_08NLHBPEGP@password?$AA@ 0000000039aae3f8     GameSpy_2.11.00_VC10:AuthService.obj
 0002:00009404       ??_C@_05HKHCDHCL@email?$AA@ 0000000039aae404     GameSpy_2.11.00_VC10:AuthService.obj
 0002:00009410       ??_C@_0BG@GEIODFNP@LoginUniqueNickResult?$AA@ 0000000039aae410     GameSpy_2.11.00_VC10:AuthService.obj
 0002:00009428       ??_C@_0DN@LIFPFPLL@SOAPAction?3?5?$CChttp?3?1?1gamespy?4net?1@ 0000000039aae428     GameSpy_2.11.00_VC10:AuthService.obj
 0002:00009468       ??_C@_0BA@PAFKEGCK@LoginUniqueNick?$AA@ 0000000039aae468     GameSpy_2.11.00_VC10:AuthService.obj
 0002:00009478       ??_C@_05FPBGKCKL@final?$AA@ 0000000039aae478     GameSpy_2.11.00_VC10:sb_server.obj
 0002:00009480       ??_C@_07MPPMNCEI@queryid?$AA@ 0000000039aae480     GameSpy_2.11.00_VC10:sb_server.obj
 0002:00009488       ??_C@_04HGGBINEM@?$CFs?$CFd?$AA@ 0000000039aae488     GameSpy_2.11.00_VC10:sb_server.obj
 0002:00009490       ??_C@_04OONEELOO@ping?$AA@ 0000000039aae490     GameSpy_2.11.00_VC10:sb_server.obj
 0002:00009498       ??_C@_06JEJEKGIK@region?$AA@ 0000000039aae498     GameSpy_2.11.00_VC10:qr2regkeys.obj
 0002:000094a0       ??_C@_07IJHPKHNG@country?$AA@ 0000000039aae4a0     GameSpy_2.11.00_VC10:qr2regkeys.obj
 0002:000094a8       ??_C@_0L@LAPOANEJ@nn_groupid?$AA@ 0000000039aae4a8     GameSpy_2.11.00_VC10:qr2regkeys.obj
 0002:000094b8       ??_C@_07FIKHDMPD@score_t?$AA@ 0000000039aae4b8     GameSpy_2.11.00_VC10:qr2regkeys.obj
 0002:000094c0       ??_C@_06GDCAOOAM@team_t?$AA@ 0000000039aae4c0     GameSpy_2.11.00_VC10:qr2regkeys.obj
 0002:000094c8       ??_C@_04PENMHCMD@pid_?$AA@ 0000000039aae4c8     GameSpy_2.11.00_VC10:qr2regkeys.obj
 0002:000094d0       ??_C@_07ENAODPBL@deaths_?$AA@ 0000000039aae4d0     GameSpy_2.11.00_VC10:qr2regkeys.obj
 0002:000094d8       ??_C@_05HBOKGADI@team_?$AA@ 0000000039aae4d8     GameSpy_2.11.00_VC10:qr2regkeys.obj
 0002:000094e0       ??_C@_05HKHPFKKP@ping_?$AA@ 0000000039aae4e0     GameSpy_2.11.00_VC10:qr2regkeys.obj
 0002:000094e8       ??_C@_06EEBMDLPG@skill_?$AA@ 0000000039aae4e8     GameSpy_2.11.00_VC10:qr2regkeys.obj
 0002:000094f0       ??_C@_06JIBIFHBI@score_?$AA@ 0000000039aae4f0     GameSpy_2.11.00_VC10:qr2regkeys.obj
 0002:000094f8       ??_C@_07CLFPDDEC@player_?$AA@ 0000000039aae4f8     GameSpy_2.11.00_VC10:qr2regkeys.obj
 0002:00009500       ??_C@_07NODMGEJG@groupid?$AA@ 0000000039aae500     GameSpy_2.11.00_VC10:qr2regkeys.obj
 0002:00009508       ??_C@_0N@OJFBIFHF@roundelapsed?$AA@ 0000000039aae508     GameSpy_2.11.00_VC10:qr2regkeys.obj
 0002:00009518       ??_C@_09NDLGFAEO@roundtime?$AA@ 0000000039aae518     GameSpy_2.11.00_VC10:qr2regkeys.obj
 0002:00009528       ??_C@_09KPHKOKCC@timelimit?$AA@ 0000000039aae528     GameSpy_2.11.00_VC10:qr2regkeys.obj
 0002:00009538       ??_C@_0M@GCHCHMOJ@timeelapsed?$AA@ 0000000039aae538     GameSpy_2.11.00_VC10:qr2regkeys.obj
 0002:00009548       ??_C@_0O@JIBNNMMH@teamfraglimit?$AA@ 0000000039aae548     GameSpy_2.11.00_VC10:qr2regkeys.obj
 0002:00009558       ??_C@_09GCIEGDDN@fraglimit?$AA@ 0000000039aae558     GameSpy_2.11.00_VC10:qr2regkeys.obj
 0002:00009568       ??_C@_08IKNDEHFO@teamplay?$AA@ 0000000039aae568     GameSpy_2.11.00_VC10:qr2regkeys.obj
 0002:00009578       ??_C@_08NKFOLMGC@gamemode?$AA@ 0000000039aae578     GameSpy_2.11.00_VC10:qr2regkeys.obj
 0002:00009588       ??_C@_0L@PCNFODNF@maxplayers?$AA@ 0000000039aae588     GameSpy_2.11.00_VC10:qr2regkeys.obj
 0002:00009598       ??_C@_08IFGAFGHM@numteams?$AA@ 0000000039aae598     GameSpy_2.11.00_VC10:qr2regkeys.obj
 0002:000095a8       ??_C@_0L@KDCFKDHI@numplayers?$AA@ 0000000039aae5a8     GameSpy_2.11.00_VC10:qr2regkeys.obj
 0002:000095b8       ??_C@_0M@GEOBBCMK@gamevariant?$AA@ 0000000039aae5b8     GameSpy_2.11.00_VC10:qr2regkeys.obj
 0002:000095c8       ??_C@_08NJPDEKHO@gametype?$AA@ 0000000039aae5c8     GameSpy_2.11.00_VC10:qr2regkeys.obj
 0002:000095d8       ??_C@_07KMNEBLH@mapname?$AA@ 0000000039aae5d8     GameSpy_2.11.00_VC10:qr2regkeys.obj
 0002:000095e0       ??_C@_08DMAEPIMN@hostport?$AA@ 0000000039aae5e0     GameSpy_2.11.00_VC10:qr2regkeys.obj
 0002:000095f0       ??_C@_07JFMLMHCD@gamever?$AA@ 0000000039aae5f0     GameSpy_2.11.00_VC10:qr2regkeys.obj
 0002:000095f8       ??_C@_08EHKIGBEA@hostname?$AA@ 0000000039aae5f8     GameSpy_2.11.00_VC10:qr2regkeys.obj
 0002:00009608       __real@3ff0000000000000    0000000039aae608     GameSpy_2.11.00_VC10:gvMain.obj
 0002:00009610       defaultEncoding            0000000039aae610     GameSpy_2.11.00_VC10:gsPlatformUtil.obj
 0002:00009614       alternateEncoding          0000000039aae614     GameSpy_2.11.00_VC10:gsPlatformUtil.obj
 0002:00009618       urlSafeEncodeing           0000000039aae618     GameSpy_2.11.00_VC10:gsPlatformUtil.obj
 0002:00009620       ??_C@_0DP@CCELEMID@0123456789abcdefghijklmnopqrstuv@ 0000000039aae620     GameSpy_2.11.00_VC10:gsPlatformUtil.obj
 0002:00009660       ??_C@_05ENHGKOIF@Crypt?$AA@ 0000000039aae660     GameSpy_2.11.00_VC10:gsPlatformUtil.obj
 0002:00009668       ??_C@_0CJ@NOGJADHF@Software?2GameSpy?2GameSpy?53D?2Regi@ 0000000039aae668     GameSpy_2.11.00_VC10:gsPlatformUtil.obj
 0002:00009694       ??_C@_03HODKBCIO@?3?$CFd?$AA@ 0000000039aae694     GameSpy_2.11.00_VC10:NATify.obj
 0002:00009698       ??_C@_02GMLFBBN@wb?$AA@    0000000039aae698     GameSpy_2.11.00_VC10:ghttpMain.obj
 0002:000096a0       ??_C@_0BO@KBMKMCOO@ns1?$DN?$CChttp?3?1?1gamespy?4net?1sake?$CC?$AA@ 0000000039aae6a0     GameSpy_2.11.00_VC10:sakeRequest.obj
 0002:000096c0       ??_C@_0BE@JOFEKFCK@TargetFilterInvalid?$AA@ 0000000039aae6c0     GameSpy_2.11.00_VC10:sakeRequest.obj
 0002:000096d8       ??_C@_0M@PAAFFMAG@SortInvalid?$AA@ 0000000039aae6d8     GameSpy_2.11.00_VC10:sakeRequest.obj
 0002:000096e8       ??_C@_0O@DHHEIGLO@FilterInvalid?$AA@ 0000000039aae6e8     GameSpy_2.11.00_VC10:sakeRequest.obj
 0002:000096f8       ??_C@_08DPMCNGNF@NotOwned?$AA@ 0000000039aae6f8     GameSpy_2.11.00_VC10:sakeRequest.obj
 0002:00009708       ??_C@_0M@NDHHFLF@NotRateable?$AA@ 0000000039aae708     GameSpy_2.11.00_VC10:sakeRequest.obj
 0002:00009718       ??_C@_0N@EMFDNCA@AlreadyRated?$AA@ 0000000039aae718     GameSpy_2.11.00_VC10:sakeRequest.obj
 0002:00009728       ??_C@_0BD@ELNOOFEG@RecordLimitReached?$AA@ 0000000039aae728     GameSpy_2.11.00_VC10:sakeRequest.obj
 0002:00009740       ??_C@_0N@OENMAFMN@NoPermission?$AA@ 0000000039aae740     GameSpy_2.11.00_VC10:sakeRequest.obj
 0002:00009750       ??_C@_0BB@MIDJAONN@FieldTypeInvalid?$AA@ 0000000039aae750     GameSpy_2.11.00_VC10:sakeRequest.obj
 0002:00009768       ??_C@_0O@PGIMNOFE@FieldNotFound?$AA@ 0000000039aae768     GameSpy_2.11.00_VC10:sakeRequest.obj
 0002:00009778       ??_C@_0P@ELBGMNFO@RecordNotFound?$AA@ 0000000039aae778     GameSpy_2.11.00_VC10:sakeRequest.obj
 0002:00009788       ??_C@_0O@LAAJHHEJ@TableNotFound?$AA@ 0000000039aae788     GameSpy_2.11.00_VC10:sakeRequest.obj
 0002:00009798       ??_C@_0BD@CPLKLAHD@LoginTicketExpired?$AA@ 0000000039aae798     GameSpy_2.11.00_VC10:sakeRequest.obj
 0002:000097b0       ??_C@_0BD@CDOOHNNM@LoginTicketInvalid?$AA@ 0000000039aae7b0     GameSpy_2.11.00_VC10:sakeRequest.obj
 0002:000097c8       ??_C@_0BE@MLKBMMLE@DatabaseUnavailable?$AA@ 0000000039aae7c8     GameSpy_2.11.00_VC10:sakeRequest.obj
 0002:000097e0       ??_C@_0BA@FGACLKFN@ServiceDisabled?$AA@ 0000000039aae7e0     GameSpy_2.11.00_VC10:sakeRequest.obj
 0002:000097f0       ??_C@_0BB@DNOFBOJD@SecretKeyInvalid?$AA@ 0000000039aae7f0     GameSpy_2.11.00_VC10:sakeRequest.obj
 0002:00009808       ??_C@_0M@KDFPLLAI@loginTicket?$AA@ 0000000039aae808     GameSpy_2.11.00_VC10:sakeRequest.obj
 0002:00009818       ??_C@_09JKPDMHAN@secretKey?$AA@ 0000000039aae818     GameSpy_2.11.00_VC10:sakeRequest.obj
 0002:00009830       ??_C@_0EA@BDGAFBPH@http?3?1?1?$CFs?4sake?4gamespy?4com?1SakeS@ 0000000039aae830     GameSpy_2.11.00_VC10:sakeRequest.obj
 0002:00009870       ??_C@_0BD@BNGKBOCM@DeleteRecordResult?$AA@ 0000000039aae870     GameSpy_2.11.00_VC10:sakeRequestModify.obj
 0002:00009888       ??_C@_0BF@KFMKFONE@DeleteRecordResponse?$AA@ 0000000039aae888     GameSpy_2.11.00_VC10:sakeRequestModify.obj
 0002:000098a0       ??_C@_0DD@IEABMPLL@SOAPAction?3?5?$CChttp?3?1?1gamespy?4net?1@ 0000000039aae8a0     GameSpy_2.11.00_VC10:sakeRequestModify.obj
 0002:000098d8       ??_C@_0N@GCEKDALH@DeleteRecord?$AA@ 0000000039aae8d8     GameSpy_2.11.00_VC10:sakeRequestModify.obj
 0002:000098e8       ??_C@_0BD@CBLCJLJI@UpdateRecordResult?$AA@ 0000000039aae8e8     GameSpy_2.11.00_VC10:sakeRequestModify.obj
 0002:00009900       ??_C@_0BF@LILBHOBP@UpdateRecordResponse?$AA@ 0000000039aae900     GameSpy_2.11.00_VC10:sakeRequestModify.obj
 0002:00009918       ??_C@_0DD@GAEBACBE@SOAPAction?3?5?$CChttp?3?1?1gamespy?4net?1@ 0000000039aae918     GameSpy_2.11.00_VC10:sakeRequestModify.obj
 0002:00009950       ??_C@_0N@CMEIJEDL@UpdateRecord?$AA@ 0000000039aae950     GameSpy_2.11.00_VC10:sakeRequestModify.obj
 0002:00009960       ??_C@_0BD@CNFOALEB@CreateRecordResult?$AA@ 0000000039aae960     GameSpy_2.11.00_VC10:sakeRequestModify.obj
 0002:00009978       ??_C@_0BF@BIEEJPOB@CreateRecordResponse?$AA@ 0000000039aae978     GameSpy_2.11.00_VC10:sakeRequestModify.obj
 0002:00009990       ??_C@_0DD@FMIIMOK@SOAPAction?3?5?$CChttp?3?1?1gamespy?4net?1@ 0000000039aae990     GameSpy_2.11.00_VC10:sakeRequestModify.obj
 0002:000099c8       ??_C@_0N@BFBPKMGD@CreateRecord?$AA@ 0000000039aae9c8     GameSpy_2.11.00_VC10:sakeRequestModify.obj
 0002:000099d8       ??_C@_0BA@NMIDMGFO@binaryDataValue?$AA@ 0000000039aae9d8     GameSpy_2.11.00_VC10:sakeRequestModify.obj
 0002:000099e8       ??_C@_0BB@PDGFCBIM@dateAndTimeValue?$AA@ 0000000039aae9e8     GameSpy_2.11.00_VC10:sakeRequestModify.obj
 0002:00009a00       ??_C@_0N@FIOMDIJC@booleanValue?$AA@ 0000000039aaea00     GameSpy_2.11.00_VC10:sakeRequestModify.obj
 0002:00009a10       ??_C@_0BD@MGEDAGKC@unicodeStringValue?$AA@ 0000000039aaea10     GameSpy_2.11.00_VC10:sakeRequestModify.obj
 0002:00009a28       ??_C@_0BB@FIENJGB@asciiStringValue?$AA@ 0000000039aaea28     GameSpy_2.11.00_VC10:sakeRequestModify.obj
 0002:00009a40       ??_C@_0L@CFLLCEAL@floatValue?$AA@ 0000000039aaea40     GameSpy_2.11.00_VC10:sakeRequestModify.obj
 0002:00009a50       ??_C@_0L@IHMLFDPK@int64Value?$AA@ 0000000039aaea50     GameSpy_2.11.00_VC10:sakeRequestModify.obj
 0002:00009a60       ??_C@_08HBLFFCOK@intValue?$AA@ 0000000039aaea60     GameSpy_2.11.00_VC10:sakeRequestModify.obj
 0002:00009a70       ??_C@_0L@BMFNKDA@shortValue?$AA@ 0000000039aaea70     GameSpy_2.11.00_VC10:sakeRequestModify.obj
 0002:00009a80       ??_C@_09CBDGACJH@byteValue?$AA@ 0000000039aaea80     GameSpy_2.11.00_VC10:sakeRequestModify.obj
 0002:00009a8c       ??_C@_05MFEJDJP@value?$AA@ 0000000039aaea8c     GameSpy_2.11.00_VC10:sakeRequestModify.obj
 0002:00009a98       ??_C@_0M@FMOIKPPP@RecordField?$AA@ 0000000039aaea98     GameSpy_2.11.00_VC10:sakeRequestModify.obj
 0002:00009aa4       ??_C@_06GEKOPAHD@values?$AA@ 0000000039aaeaa4     GameSpy_2.11.00_VC10:sakeRequestModify.obj
 0002:00009ab0       ??_C@_07MMJHJFIN@tableid?$AA@ 0000000039aaeab0     GameSpy_2.11.00_VC10:sakeRequestModify.obj
 0002:00009ab8       ??_C@_0BH@FIFPJHL@GetRandomRecordsResult?$AA@ 0000000039aaeab8     GameSpy_2.11.00_VC10:sakeRequestRead.obj
 0002:00009ad0       ??_C@_0BJ@GOFOPKHD@GetRandomRecordsResponse?$AA@ 0000000039aaead0     GameSpy_2.11.00_VC10:sakeRequestRead.obj
 0002:00009af0       ??_C@_0DH@JAMCNBMO@SOAPAction?3?5?$CChttp?3?1?1gamespy?4net?1@ 0000000039aaeaf0     GameSpy_2.11.00_VC10:sakeRequestRead.obj
 0002:00009b28       ??_C@_0BB@OMCHLMKF@GetRandomRecords?$AA@ 0000000039aaeb28     GameSpy_2.11.00_VC10:sakeRequestRead.obj
 0002:00009b40       ??_C@_0BJ@LJGMOHI@GetSpecificRecordsResult?$AA@ 0000000039aaeb40     GameSpy_2.11.00_VC10:sakeRequestRead.obj
 0002:00009b60       ??_C@_0BL@PNMOACKM@GetSpecificRecordsResponse?$AA@ 0000000039aaeb60     GameSpy_2.11.00_VC10:sakeRequestRead.obj
 0002:00009b80       ??_C@_0DJ@HGKBDGGG@SOAPAction?3?5?$CChttp?3?1?1gamespy?4net?1@ 0000000039aaeb80     GameSpy_2.11.00_VC10:sakeRequestRead.obj
 0002:00009bc0       ??_C@_0BD@PODFFDGA@GetSpecificRecords?$AA@ 0000000039aaebc0     GameSpy_2.11.00_VC10:sakeRequestRead.obj
 0002:00009bd8       ??_C@_0BD@PNJNODON@GetMyRecordsResult?$AA@ 0000000039aaebd8     GameSpy_2.11.00_VC10:sakeRequestRead.obj
 0002:00009bf0       ??_C@_0BF@LECHNGIN@GetMyRecordsResponse?$AA@ 0000000039aaebf0     GameSpy_2.11.00_VC10:sakeRequestRead.obj
 0002:00009c08       ??_C@_0DD@BOPEHIPL@SOAPAction?3?5?$CChttp?3?1?1gamespy?4net?1@ 0000000039aaec08     GameSpy_2.11.00_VC10:sakeRequestRead.obj
 0002:00009c40       ??_C@_0N@CIEOMGDG@GetMyRecords?$AA@ 0000000039aaec40     GameSpy_2.11.00_VC10:sakeRequestRead.obj
 0002:00009c50       ??_C@_0BH@EICNFPPN@SearchForRecordsResult?$AA@ 0000000039aaec50     GameSpy_2.11.00_VC10:sakeRequestRead.obj
 0002:00009c68       ??_C@_0BJ@DMDCIOML@SearchForRecordsResponse?$AA@ 0000000039aaec68     GameSpy_2.11.00_VC10:sakeRequestRead.obj
 0002:00009c88       ??_C@_0DH@MCFGADLE@SOAPAction?3?5?$CChttp?3?1?1gamespy?4net?1@ 0000000039aaec88     GameSpy_2.11.00_VC10:sakeRequestRead.obj
 0002:00009cc0       ??_C@_0BB@BABHPABG@SearchForRecords?$AA@ 0000000039aaecc0     GameSpy_2.11.00_VC10:sakeRequestRead.obj
 0002:00009cd4       ??_C@_06MOOAPOID@fields?$AA@ 0000000039aaecd4     GameSpy_2.11.00_VC10:sakeRequestRead.obj
 0002:00009ce0       ??_C@_09PMBNBBJE@recordids?$AA@ 0000000039aaece0     GameSpy_2.11.00_VC10:sakeRequestRead.obj
 0002:00009cf0       ??_C@_08DBPJNGBD@ownerids?$AA@ 0000000039aaecf0     GameSpy_2.11.00_VC10:sakeRequestRead.obj
 0002:00009d00       ??_C@_0M@BIKKAAJB@RecordValue?$AA@ 0000000039aaed00     GameSpy_2.11.00_VC10:sakeRequestRead.obj
 0002:00009d10       ??_C@_0BD@BJFFFMP@ArrayOfRecordValue?$AA@ 0000000039aaed10     GameSpy_2.11.00_VC10:sakeRequestRead.obj
 0002:00009d28       ??_C@_09BGFDDPAL@cacheFlag?$AA@ 0000000039aaed28     GameSpy_2.11.00_VC10:sakeRequestRead.obj
 0002:00009d38       ??_C@_0M@LDGOHLCM@surrounding?$AA@ 0000000039aaed38     GameSpy_2.11.00_VC10:sakeRequestRead.obj
 0002:00009d48       ??_C@_0N@LOLNLIMH@targetfilter?$AA@ 0000000039aaed48     GameSpy_2.11.00_VC10:sakeRequestRead.obj
 0002:00009d58       ??_C@_03LJAEFNNE@max?$AA@  0000000039aaed58     GameSpy_2.11.00_VC10:sakeRequestRead.obj
 0002:00009d5c       ??_C@_06KLHHMIGM@offset?$AA@ 0000000039aaed5c     GameSpy_2.11.00_VC10:sakeRequestRead.obj
 0002:00009d64       ??_C@_04PIMMHFGE@sort?$AA@ 0000000039aaed64     GameSpy_2.11.00_VC10:sakeRequestRead.obj
 0002:00009d6c       ??_C@_06EOIELIPE@filter?$AA@ 0000000039aaed6c     GameSpy_2.11.00_VC10:sakeRequestRead.obj
 0002:00009d78       ??_C@_0BF@EPGEFHFH@GetRecordCountResult?$AA@ 0000000039aaed78     GameSpy_2.11.00_VC10:sakeRequestMisc.obj
 0002:00009d90       ??_C@_0BH@GGABFFND@GetRecordCountResponse?$AA@ 0000000039aaed90     GameSpy_2.11.00_VC10:sakeRequestMisc.obj
 0002:00009da8       ??_C@_0DF@OFPPIIMD@SOAPAction?3?5?$CChttp?3?1?1gamespy?4net?1@ 0000000039aaeda8     GameSpy_2.11.00_VC10:sakeRequestMisc.obj
 0002:00009de0       ??_C@_0P@BFPFBMPF@GetRecordCount?$AA@ 0000000039aaede0     GameSpy_2.11.00_VC10:sakeRequestMisc.obj
 0002:00009df0       ??_C@_0BF@IFFNKOLA@GetRecordLimitResult?$AA@ 0000000039aaedf0     GameSpy_2.11.00_VC10:sakeRequestMisc.obj
 0002:00009e08       ??_C@_0BH@LDFPLAHJ@GetRecordLimitResponse?$AA@ 0000000039aaee08     GameSpy_2.11.00_VC10:sakeRequestMisc.obj
 0002:00009e20       ??_C@_0DF@IKJPPMN@SOAPAction?3?5?$CChttp?3?1?1gamespy?4net?1@ 0000000039aaee20     GameSpy_2.11.00_VC10:sakeRequestMisc.obj
 0002:00009e58       ??_C@_0P@PLABDCHF@GetRecordLimit?$AA@ 0000000039aaee58     GameSpy_2.11.00_VC10:sakeRequestMisc.obj
 0002:00009e68       ??_C@_0BB@FDLHBBF@RateRecordResult?$AA@ 0000000039aaee68     GameSpy_2.11.00_VC10:sakeRequestMisc.obj
 0002:00009e80       ??_C@_0BD@HGEDLHPG@RateRecordResponse?$AA@ 0000000039aaee80     GameSpy_2.11.00_VC10:sakeRequestMisc.obj
 0002:00009e98       ??_C@_0DB@JHJKHPOF@SOAPAction?3?5?$CChttp?3?1?1gamespy?4net?1@ 0000000039aaee98     GameSpy_2.11.00_VC10:sakeRequestMisc.obj
 0002:00009ed0       ??_C@_0L@LIILOHJM@RateRecord?$AA@ 0000000039aaeed0     GameSpy_2.11.00_VC10:sakeRequestMisc.obj
 0002:00009edc       ??_C@_06PIEFNILA@rating?$AA@ 0000000039aaeedc     GameSpy_2.11.00_VC10:sakeRequestMisc.obj
 0002:00009ee8       ??_C@_0O@PIHPFHEF@averageRating?$AA@ 0000000039aaeee8     GameSpy_2.11.00_VC10:sakeRequestMisc.obj
 0002:00009ef8       ??_C@_0L@IHLGEFKD@numRatings?$AA@ 0000000039aaeef8     GameSpy_2.11.00_VC10:sakeRequestMisc.obj
 0002:00009f08       ??_C@_08KCAOKAII@numOwned?$AA@ 0000000039aaef08     GameSpy_2.11.00_VC10:sakeRequestMisc.obj
 0002:00009f18       ??_C@_0O@MPHCJAHB@limitPerOwner?$AA@ 0000000039aaef18     GameSpy_2.11.00_VC10:sakeRequestMisc.obj
 0002:00009f28       ??_C@_05IOMEMJEC@count?$AA@ 0000000039aaef28     GameSpy_2.11.00_VC10:sakeRequestMisc.obj
 0002:00009f48       ??_C@_07FGAOOBMN@http?3?1?1?$AA@ 0000000039aaef48     GameSpy_2.11.00_VC10:d2gUtil.obj
 0002:00009f50       ??_C@_08MFLLBFBE@https?3?1?1?$AA@ 0000000039aaef50     GameSpy_2.11.00_VC10:d2gUtil.obj
 0002:00009f5c       ??_C@_06DIJPEION@?$CFs?$CFs?$CFs?$AA@ 0000000039aaef5c     GameSpy_2.11.00_VC10:d2gUtil.obj
 0002:00009f68       ??_C@_0CI@NLEIPHEE@?$CFs?4d2g?4pubsvs?4gamespy?4com?1commer@ 0000000039aaef68     GameSpy_2.11.00_VC10:d2gUtil.obj
 0002:00009f90       ??_C@_08OCNIHGPN@quantity?$AA@ 0000000039aaef90     GameSpy_2.11.00_VC10:d2gUtil.obj
 0002:00009f9c       ??_C@_05NCDILCCA@price?$AA@ 0000000039aaef9c     GameSpy_2.11.00_VC10:d2gUtil.obj
 0002:00009fa8       ??_C@_0L@LPBNGKGB@externalid?$AA@ 0000000039aaefa8     GameSpy_2.11.00_VC10:d2gUtil.obj
 0002:00009fb4       ??_C@_06DCAHOPIP@itemid?$AA@ 0000000039aaefb4     GameSpy_2.11.00_VC10:d2gUtil.obj
 0002:00009fc0       ??_C@_09MHDJHMDI@orderitem?$AA@ 0000000039aaefc0     GameSpy_2.11.00_VC10:d2gUtil.obj
 0002:00009fd0       ??_C@_0L@CMNHKLNH@orderitems?$AA@ 0000000039aaefd0     GameSpy_2.11.00_VC10:d2gUtil.obj
 0002:00009fdc       ??_C@_05KBOMEDGA@total?$AA@ 0000000039aaefdc     GameSpy_2.11.00_VC10:d2gUtil.obj
 0002:00009fe4       ??_C@_03JEBFEFMB@tax?$AA@  0000000039aaefe4     GameSpy_2.11.00_VC10:d2gUtil.obj
 0002:00009fe8       ??_C@_08MHJAMLEF@subtotal?$AA@ 0000000039aaefe8     GameSpy_2.11.00_VC10:d2gUtil.obj
 0002:00009ff8       ??_C@_0N@EMMCNFL@currencycode?$AA@ 0000000039aaeff8     GameSpy_2.11.00_VC10:d2gUtil.obj
 0002:0000a008       ??_C@_0M@BPPKNJDH@culturecode?$AA@ 0000000039aaf008     GameSpy_2.11.00_VC10:d2gUtil.obj
 0002:0000a018       ??_C@_09LLADOCGL@accountid?$AA@ 0000000039aaf018     GameSpy_2.11.00_VC10:d2gUtil.obj
 0002:0000a024       ??_C@_03GACNABDE@gsc?$AA@  0000000039aaf024     GameSpy_2.11.00_VC10:d2gUtil.obj
 0002:0000a028       ??_C@_05NDNMCCJH@order?$AA@ 0000000039aaf028     GameSpy_2.11.00_VC10:d2gUtil.obj
 0002:0000a030       ??_C@_04MMEBIPMJ@?4tmp?$AA@ 0000000039aaf030     GameSpy_2.11.00_VC10:d2gUtil.obj
 0002:0000a038       ??_C@_02CHHAKFFB@w?$CL?$AA@ 0000000039aaf038     GameSpy_2.11.00_VC10:d2gUtil.obj
 0002:0000a040       ??_C@_0O@EOFAHBG@downloadurlid?$AA@ 0000000039aaf040     GameSpy_2.11.00_VC10:d2gUtil.obj
 0002:0000a050       ??_C@_08HNIAHLMM@download?$AA@ 0000000039aaf050     GameSpy_2.11.00_VC10:d2gUtil.obj
 0002:0000a05c       ??_C@_01EEMJAFIK@?6?$AA@   0000000039aaf05c     GameSpy_2.11.00_VC10:d2gUtil.obj
 0002:0000a060       ??_C@_0CK@IIEBOJOK@gsc?$DN?$CChttp?3?1?1gamespy?4net?1commerce@ 0000000039aaf060     GameSpy_2.11.00_VC10:d2gServices.obj
 0002:0000a0a0       ??_C@_0FG@NBIEAAJF@SOAPAction?3?5?$CChttp?3?1?1gamespy?4net?1@ 0000000039aaf0a0     GameSpy_2.11.00_VC10:d2gServices.obj
 0002:0000a0f8       ??_C@_0M@PPAEFODI@accesstoken?$AA@ 0000000039aaf0f8     GameSpy_2.11.00_VC10:d2gServices.obj
 0002:0000a108       ??_C@_0BF@PLCHPOCM@GetStoreAvailability?$AA@ 0000000039aaf108     GameSpy_2.11.00_VC10:d2gServices.obj
 0002:0000a120       ??_C@_0BD@PMGFONNE@catalogservice?4svc?$AA@ 0000000039aaf120     GameSpy_2.11.00_VC10:d2gServices.obj
 0002:0000a140       ??_C@_0EN@HFFKMJOH@SOAPAction?3?5?$CChttp?3?1?1gamespy?4net?1@ 0000000039aaf140     GameSpy_2.11.00_VC10:d2gServices.obj
 0002:0000a190       ??_C@_0M@HAKLJEIK@GetAllItems?$AA@ 0000000039aaf190     GameSpy_2.11.00_VC10:d2gServices.obj
 0002:0000a1a0       ??_C@_08MBJIKOEN@category?$AA@ 0000000039aaf1a0     GameSpy_2.11.00_VC10:d2gServices.obj
 0002:0000a1b0       ??_C@_0FE@EPFGMGDN@SOAPAction?3?5?$CChttp?3?1?1gamespy?4net?1@ 0000000039aaf1b0     GameSpy_2.11.00_VC10:d2gServices.obj
 0002:0000a208       ??_C@_0BA@GBBLIJMF@returnvalidonly?$AA@ 0000000039aaf208     GameSpy_2.11.00_VC10:d2gServices.obj
 0002:0000a218       ??_C@_05NFGEEHFL@proof?$AA@ 0000000039aaf218     GameSpy_2.11.00_VC10:d2gServices.obj
 0002:0000a220       ??_C@_0BD@OGKOEFDD@GetUserCreditCards?$AA@ 0000000039aaf220     GameSpy_2.11.00_VC10:d2gServices.obj
 0002:0000a238       ??_C@_0BD@DMJGDAHJ@accountservice?4svc?$AA@ 0000000039aaf238     GameSpy_2.11.00_VC10:d2gServices.obj
 0002:0000a250       ??_C@_0FA@OLOLFJF@SOAPAction?3?5?$CChttp?3?1?1gamespy?4net?1@ 0000000039aaf250     GameSpy_2.11.00_VC10:d2gServices.obj
 0002:0000a2a0       ??_C@_0O@IDKCBHDM@GetOrderTotal?$AA@ 0000000039aaf2a0     GameSpy_2.11.00_VC10:d2gServices.obj
 0002:0000a2b0       ??_C@_0BE@JGGMNEID@purchaseservice?4svc?$AA@ 0000000039aaf2b0     GameSpy_2.11.00_VC10:d2gServices.obj
 0002:0000a2d0       ??_C@_0EN@BAMGIPDA@SOAPAction?3?5?$CChttp?3?1?1gamespy?4net?1@ 0000000039aaf2d0     GameSpy_2.11.00_VC10:d2gServices.obj
 0002:0000a320       ??_C@_0L@HBKCFPMJ@PlaceOrder?$AA@ 0000000039aaf320     GameSpy_2.11.00_VC10:d2gServices.obj
 0002:0000a330       ??_C@_0FB@KABCEGFI@SOAPAction?3?5?$CChttp?3?1?1gamespy?4net?1@ 0000000039aaf330     GameSpy_2.11.00_VC10:d2gServices.obj
 0002:0000a388       ??_C@_0M@DFPOHJFO@rootorderid?$AA@ 0000000039aaf388     GameSpy_2.11.00_VC10:d2gServices.obj
 0002:0000a398       ??_C@_0P@ELCEEMCB@GetPlacedOrder?$AA@ 0000000039aaf398     GameSpy_2.11.00_VC10:d2gServices.obj
 0002:0000a3a8       ??_C@_03BMGHOINI@url?$AA@  0000000039aaf3a8     GameSpy_2.11.00_VC10:d2gServices.obj
 0002:0000a3b0       ??_C@_07ONPBMBOP@message?$AA@ 0000000039aaf3b0     GameSpy_2.11.00_VC10:d2gServices.obj
 0002:0000a3b8       ??_C@_04NDFOBODE@code?$AA@ 0000000039aaf3b8     GameSpy_2.11.00_VC10:d2gServices.obj
 0002:0000a3c0       ??_C@_06DJIHEMFI@status?$AA@ 0000000039aaf3c0     GameSpy_2.11.00_VC10:d2gServices.obj
 0002:0000a3c8       ??_C@_0N@JAOMBGDD@downloadinfo?$AA@ 0000000039aaf3c8     GameSpy_2.11.00_VC10:d2gServices.obj
 0002:0000a3d8       ??_C@_0BG@BKABLAIH@GetDownloadInfoResult?$AA@ 0000000039aaf3d8     GameSpy_2.11.00_VC10:d2gServices.obj
 0002:0000a3f0       ??_C@_0FB@LEGNJNPM@SOAPAction?3?5?$CChttp?3?1?1gamespy?4net?1@ 0000000039aaf3f0     GameSpy_2.11.00_VC10:d2gServices.obj
 0002:0000a444       ??_C@_06LDKDMELN@fileid?$AA@ 0000000039aaf444     GameSpy_2.11.00_VC10:d2gServices.obj
 0002:0000a450       ??_C@_0BA@FAGBLGKM@GetDownloadInfo?$AA@ 0000000039aaf450     GameSpy_2.11.00_VC10:d2gServices.obj
 0002:0000a460       ??_C@_0FF@OLEOINIE@SOAPAction?3?5?$CChttp?3?1?1gamespy?4net?1@ 0000000039aaf460     GameSpy_2.11.00_VC10:d2gServices.obj
 0002:0000a4b8       ??_C@_0BD@GIAHKFGH@GetPurchaseHistory?$AA@ 0000000039aaf4b8     GameSpy_2.11.00_VC10:d2gServices.obj
 0002:0000a4e8       ??_C@_0O@HFPDPBLN@?2basic?2?2info?2?$AA@ 0000000039aaf4e8     GameSpy_2.11.00_VC10:sb_queryengine.obj
 0002:0000a4f8       ??_C@_0O@JHMFNCLB@Query?5Error?3?5?$AA@ 0000000039aaf4f8     GameSpy_2.11.00_VC10:sb_serverlist.obj
 0002:0000a508       ??_C@_0BE@HHKMJAKP@?$CFs?4ms?$CFd?4gamespy?4com?$AA@ 0000000039aaf508     GameSpy_2.11.00_VC10:sb_serverlist.obj
 0002:0000a51c       ??_C@_04A@?$PP?$PP?$PP?$PP?$AA@ 0000000039aaf51c     GameSpy_2.11.00_VC10:sb_serverlist.obj
 0002:0000a528       ??_C@_0CM@OHAIIBJP@There?5was?5an?5error?5reading?5from?5@ 0000000039aaf528     GameSpy_2.11.00_VC10:gpi.obj
 0002:0000a558       ??_C@_0M@FDKCFKNP@?2ka?2?2final?2?$AA@ 0000000039aaf558     GameSpy_2.11.00_VC10:gpi.obj
 0002:0000a568       ??_C@_0CG@PIKIKHCA@The?5server?5has?5closed?5the?5connec@ 0000000039aaf568     GameSpy_2.11.00_VC10:gpi.obj
 0002:0000a590       ??_C@_0P@ILLCNIIE@Out?5of?5memory?4?$AA@ 0000000039aaf590     GameSpy_2.11.00_VC10:gpi.obj
 0002:0000a5a0       ??_C@_0BD@EOLCCLGC@?2addbuddyresponse?2?$AA@ 0000000039aaf5a0     GameSpy_2.11.00_VC10:gpi.obj
 0002:0000a5b4       ??_C@_05HEICBLHP@?2rar?2?$AA@ 0000000039aaf5b4     GameSpy_2.11.00_VC10:gpi.obj
 0002:0000a5bc       ??_C@_05PFPPMMNP@?2blk?2?$AA@ 0000000039aaf5bc     GameSpy_2.11.00_VC10:gpi.obj
 0002:0000a5c4       ??_C@_05CPOJJDCO@?2bdy?2?$AA@ 0000000039aaf5c4     GameSpy_2.11.00_VC10:gpi.obj
 0002:0000a5cc       ??_C@_05POABFPHI@?2bsi?2?$AA@ 0000000039aaf5cc     GameSpy_2.11.00_VC10:gpi.obj
 0002:0000a5d4       ??_C@_04PADILAEH@?2lt?2?$AA@ 0000000039aaf5d4     GameSpy_2.11.00_VC10:gpi.obj
 0002:0000a5dc       ??_C@_04HHACOJGF@?2ka?2?$AA@ 0000000039aaf5dc     GameSpy_2.11.00_VC10:gpi.obj
 0002:0000a5e4       ??_C@_04DBAFPIL@?2bm?2?$AA@ 0000000039aaf5e4     GameSpy_2.11.00_VC10:gpi.obj
 0002:0000a5ec       ??_C@_04NLMAODAF@?2id?2?$AA@ 0000000039aaf5ec     GameSpy_2.11.00_VC10:gpi.obj
 0002:0000a5f4       ??_C@_02DHLFCEDM@CM?$AA@   0000000039aaf5f4     GameSpy_2.11.00_VC10:gpi.obj
 0002:0000a5f8       ??_C@_07GLJBJFEK@?2fatal?2?$AA@ 0000000039aaf5f8     GameSpy_2.11.00_VC10:gpiUtility.obj
 0002:0000a600       ??_C@_08GLDIOJFH@?2errmsg?2?$AA@ 0000000039aaf600     GameSpy_2.11.00_VC10:gpiUtility.obj
 0002:0000a60c       ??_C@_05OEOOKIJM@?2err?2?$AA@ 0000000039aaf60c     GameSpy_2.11.00_VC10:gpiUtility.obj
 0002:0000a618       ??_C@_07KGBMPDAL@?2error?2?$AA@ 0000000039aaf618     GameSpy_2.11.00_VC10:gpiUtility.obj
 0002:0000a620       ??_C@_0DI@PCKHBAKG@There?5was?5an?5error?5checking?5for?5@ 0000000039aaf620     GameSpy_2.11.00_VC10:gpiUtility.obj
 0002:0000a658       ??_C@_0N@PCLIMKID@Parse?5Error?4?$AA@ 0000000039aaf658     GameSpy_2.11.00_VC10:gpiUtility.obj
 0002:0000a668       ??_C@_0DP@EFDPGBGM@ABCDEFGHIJKLMNOPQRSTUVWXYZabcdef@ 0000000039aaf668     GameSpy_2.11.00_VC10:gpiConnect.obj
 0002:0000a6a8       ??_C@_0CI@IBKPDIGI@There?5was?5an?5error?5connecting?5a?5@ 0000000039aaf6a8     GameSpy_2.11.00_VC10:gpiConnect.obj
 0002:0000a6d0       ??_C@_0DA@JPNLJKDH@Could?5not?5resolve?5connection?5man@ 0000000039aaf6d0     GameSpy_2.11.00_VC10:gpiConnect.obj
 0002:0000a700       ??_C@_0DB@GBIIPCPG@There?5was?5an?5error?5making?5a?5sock@ 0000000039aaf700     GameSpy_2.11.00_VC10:gpiConnect.obj
 0002:0000a738       ??_C@_0CF@IKPHICDO@There?5was?5an?5error?5binding?5a?5soc@ 0000000039aaf738     GameSpy_2.11.00_VC10:gpiConnect.obj
 0002:0000a760       ??_C@_0CG@EFOKILB@There?5was?5an?5error?5creating?5a?5so@ 0000000039aaf760     GameSpy_2.11.00_VC10:gpiConnect.obj
 0002:0000a788       ??_C@_0CL@LKFGFBDA@There?5was?5an?5error?5starting?5the?5@ 0000000039aaf788     GameSpy_2.11.00_VC10:gpiConnect.obj
 0002:0000a7b8       ??_C@_0CI@CMJCJKOF@There?5was?5error?5starting?5the?5UDP@ 0000000039aaf7b8     GameSpy_2.11.00_VC10:gpiConnect.obj
 0002:0000a7e0       ??_C@_09PGMCBPKK@gamespygp?$AA@ 0000000039aaf7e0     GameSpy_2.11.00_VC10:gpiConnect.obj
 0002:0000a7ec       ??_C@_05LGOMDDNO@?2id?21?$AA@ 0000000039aaf7ec     GameSpy_2.11.00_VC10:gpiConnect.obj
 0002:0000a7f8       ??_C@_0O@MCOKPDNC@?2sdkrevision?2?$AA@ 0000000039aaf7f8     GameSpy_2.11.00_VC10:gpiConnect.obj
 0002:0000a808       ??_C@_0O@EACFFLDP@?2namespaceid?2?$AA@ 0000000039aaf808     GameSpy_2.11.00_VC10:gpiConnect.obj
 0002:0000a818       ??_C@_0L@LGNFJKM@?2gamename?2?$AA@ 0000000039aaf818     GameSpy_2.11.00_VC10:gpiConnect.obj
 0002:0000a824       ??_C@_06BCGGPENM@?2port?2?$AA@ 0000000039aaf824     GameSpy_2.11.00_VC10:gpiConnect.obj
 0002:0000a830       ??_C@_0M@KDICIJL@?2firewall?21?$AA@ 0000000039aaf830     GameSpy_2.11.00_VC10:gpiConnect.obj
 0002:0000a840       ??_C@_0L@DCBLLGKE@?2response?2?$AA@ 0000000039aaf840     GameSpy_2.11.00_VC10:gpiConnect.obj
 0002:0000a850       ??_C@_0M@JEEPLEEK@?2partnerid?2?$AA@ 0000000039aaf850     GameSpy_2.11.00_VC10:gpiConnect.obj
 0002:0000a860       ??_C@_08HAHFOIBK@?2userid?2?$AA@ 0000000039aaf860     GameSpy_2.11.00_VC10:gpiConnect.obj
 0002:0000a86c       ??_C@_01EOFPKCAF@?$EA?$AA@ 0000000039aaf86c     GameSpy_2.11.00_VC10:gpiConnect.obj
 0002:0000a870       ??_C@_06COPIAMHI@?2user?2?$AA@ 0000000039aaf870     GameSpy_2.11.00_VC10:gpiConnect.obj
 0002:0000a878       ??_C@_0N@PHCHGNNF@?2uniquenick?2?$AA@ 0000000039aaf878     GameSpy_2.11.00_VC10:gpiConnect.obj
 0002:0000a888       ??_C@_0M@MFPIPMEG@?2authtoken?2?$AA@ 0000000039aaf888     GameSpy_2.11.00_VC10:gpiConnect.obj
 0002:0000a898       ??_C@_0M@LGMPBPMO@?2challenge?2?$AA@ 0000000039aaf898     GameSpy_2.11.00_VC10:gpiConnect.obj
 0002:0000a8a8       ??_C@_07BEJLLKKH@?2login?2?$AA@ 0000000039aaf8a8     GameSpy_2.11.00_VC10:gpiConnect.obj
 0002:0000a8b0       ??_C@_0N@FHAODGGC@?$CFs?$CFs?$CFs?$CFs?$CFs?$CFs?$AA@ 0000000039aaf8b0     GameSpy_2.11.00_VC10:gpiConnect.obj
 0002:0000a8c0       ??_C@_0DB@NFMEPIDB@?5?5?5?5?5?5?5?5?5?5?5?5?5?5?5?5?5?5?5?5?5?5?5?5?5?5?5?5?5?5?5?5@ 0000000039aaf8c0     GameSpy_2.11.00_VC10:gpiConnect.obj
 0002:0000a8f8       ??_C@_07LOFIHOIL@?$CFs?$CFs?$EA?$CFs?$AA@ 0000000039aaf8f8     GameSpy_2.11.00_VC10:gpiConnect.obj
 0002:0000a900       ??_C@_03PGPAFDBG@?$CFd?$EA?$AA@ 0000000039aaf900     GameSpy_2.11.00_VC10:gpiConnect.obj
 0002:0000a908       ??_C@_0L@HDBFPCKB@?2cdkeyenc?2?$AA@ 0000000039aaf908     GameSpy_2.11.00_VC10:gpiConnect.obj
 0002:0000a918       ??_C@_0O@PDCIAFGL@?2passwordenc?2?$AA@ 0000000039aaf918     GameSpy_2.11.00_VC10:gpiConnect.obj
 0002:0000a928       ??_C@_06FLCFLGCA@?2nick?2?$AA@ 0000000039aaf928     GameSpy_2.11.00_VC10:gpiConnect.obj
 0002:0000a930       ??_C@_07EAAPHPLB@?2email?2?$AA@ 0000000039aaf930     GameSpy_2.11.00_VC10:gpiConnect.obj
 0002:0000a938       ??_C@_09DCCGEEDJ@?2newuser?2?$AA@ 0000000039aaf938     GameSpy_2.11.00_VC10:gpiConnect.obj
 0002:0000a948       ??_C@_0CO@EPAGKBK@Unexpected?5data?5was?5received?5fro@ 0000000039aaf948     GameSpy_2.11.00_VC10:gpiConnect.obj
 0002:0000a978       ??_C@_05ODNLIEBH@?2lc?21?$AA@ 0000000039aaf978     GameSpy_2.11.00_VC10:gpiConnect.obj
 0002:0000a980       ??_C@_0BP@JMECIFOB@Could?5not?5authenticate?5server?4?$AA@ 0000000039aaf980     GameSpy_2.11.00_VC10:gpiConnect.obj
 0002:0000a9a0       ??_C@_0CP@GLNHCNNG@Unexepected?5data?5was?5received?5fr@ 0000000039aaf9a0     GameSpy_2.11.00_VC10:gpiConnect.obj
 0002:0000a9d0       ??_C@_07BAKFBIPN@?2proof?2?$AA@ 0000000039aaf9d0     GameSpy_2.11.00_VC10:gpiConnect.obj
 0002:0000a9d8       ??_C@_05MIPGNHNE@?2lc?22?$AA@ 0000000039aaf9d8     GameSpy_2.11.00_VC10:gpiConnect.obj
 0002:0000a9e0       ??_C@_05OOJKBDE@?2nur?2?$AA@ 0000000039aaf9e0     GameSpy_2.11.00_VC10:gpiConnect.obj
 0002:0000a9e8       ??_C@_05NDFNLPDC@?2pid?2?$AA@ 0000000039aaf9e8     GameSpy_2.11.00_VC10:gpiConnect.obj
 0002:0000a9f0       ??_C@_0CH@JEMBONJN@The?5server?5has?5refused?5the?5conne@ 0000000039aaf9f0     GameSpy_2.11.00_VC10:gpiConnect.obj
 0002:0000aa18       ??_C@_0BC@LNCPHJMB@?2logout?2?2sesskey?2?$AA@ 0000000039aafa18     GameSpy_2.11.00_VC10:gpiConnect.obj
 0002:0000aa30       ??_C@_0BC@IPJCADHD@Invalid?5firewall?4?$AA@ 0000000039aafa30     GameSpy_2.11.00_VC10:gpiConnect.obj
 0002:0000aa48       ??_C@_0BE@LGEIEOFC@Invalid?5connection?4?$AA@ 0000000039aafa48     GameSpy_2.11.00_VC10:gpiConnect.obj
 0002:0000aa60       ??_C@_0CM@MDLGBANF@Could?5not?5resolve?5search?5manager@ 0000000039aafa60     GameSpy_2.11.00_VC10:gpiSearch.obj
 0002:0000aa90       ??_C@_0CH@DJCPMMFD@There?5was?5an?5error?5binding?5the?5s@ 0000000039aafa90     GameSpy_2.11.00_VC10:gpiSearch.obj
 0002:0000aab8       ??_C@_0BE@NKGHBCIJ@No?5search?5criteria?4?$AA@ 0000000039aafab8     GameSpy_2.11.00_VC10:gpiSearch.obj
 0002:0000aacc       ??_C@_04HEMFHPJH@more?$AA@ 0000000039aafacc     GameSpy_2.11.00_VC10:gpiSearch.obj
 0002:0000aad8       ??_C@_0CG@CONLIIKF@Error?5reading?5from?5the?5search?5se@ 0000000039aafad8     GameSpy_2.11.00_VC10:gpiSearch.obj
 0002:0000ab00       ??_C@_08PMOCCHO@lastname?$AA@ 0000000039aafb00     GameSpy_2.11.00_VC10:gpiSearch.obj
 0002:0000ab10       ??_C@_09GOBHFJBG@firstname?$AA@ 0000000039aafb10     GameSpy_2.11.00_VC10:gpiSearch.obj
 0002:0000ab1c       ??_C@_03ECKNCBG@bsr?$AA@   0000000039aafb1c     GameSpy_2.11.00_VC10:gpiSearch.obj
 0002:0000ab20       ??_C@_07MGENKODM@bsrdone?$AA@ 0000000039aafb20     GameSpy_2.11.00_VC10:gpiSearch.obj
 0002:0000ab28       ??_C@_06JIKFICKK@hidden?$AA@ 0000000039aafb28     GameSpy_2.11.00_VC10:gpiSearch.obj
 0002:0000ab30       ??_C@_06KEPJHAJL@pldone?$AA@ 0000000039aafb30     GameSpy_2.11.00_VC10:gpiSearch.obj
 0002:0000ab38       ??_C@_0M@NFDILPFD@profilelist?$AA@ 0000000039aafb38     GameSpy_2.11.00_VC10:gpiSearch.obj
 0002:0000ab44       ??_C@_06EEBOPHC@usdone?$AA@ 0000000039aafb44     GameSpy_2.11.00_VC10:gpiSearch.obj
 0002:0000ab4c       ??_C@_02FGJGKGGD@us?$AA@   0000000039aafb4c     GameSpy_2.11.00_VC10:gpiSearch.obj
 0002:0000ab50       ??_C@_06DFGPJMLM@oldone?$AA@ 0000000039aafb50     GameSpy_2.11.00_VC10:gpiSearch.obj
 0002:0000ab58       ??_C@_0L@CGAPHCDP@otherslist?$AA@ 0000000039aafb58     GameSpy_2.11.00_VC10:gpiSearch.obj
 0002:0000ab64       ??_C@_04PLGBGIDD@last?$AA@ 0000000039aafb64     GameSpy_2.11.00_VC10:gpiSearch.obj
 0002:0000ab6c       ??_C@_05NIGAKFML@first?$AA@ 0000000039aafb6c     GameSpy_2.11.00_VC10:gpiSearch.obj
 0002:0000ab74       ??_C@_01FMEDJKGI@o?$AA@    0000000039aafb74     GameSpy_2.11.00_VC10:gpiSearch.obj
 0002:0000ab78       ??_C@_05OCKLKMMD@odone?$AA@ 0000000039aafb78     GameSpy_2.11.00_VC10:gpiSearch.obj
 0002:0000ab80       ??_C@_06HJADPOOM@others?$AA@ 0000000039aafb80     GameSpy_2.11.00_VC10:gpiSearch.obj
 0002:0000ab88       ??_C@_03EKHBBBBM@nur?$AA@  0000000039aafb88     GameSpy_2.11.00_VC10:gpiSearch.obj
 0002:0000ab8c       ??_C@_03LIBLMJMB@cur?$AA@  0000000039aafb8c     GameSpy_2.11.00_VC10:gpiSearch.obj
 0002:0000ab90       ??_C@_0L@LGHNMDLL@statuscode?$AA@ 0000000039aafb90     GameSpy_2.11.00_VC10:gpiSearch.obj
 0002:0000ab9c       ??_C@_03PODKENAC@psr?$AA@  0000000039aafb9c     GameSpy_2.11.00_VC10:gpiSearch.obj
 0002:0000aba0       ??_C@_07PINDJIGK@psrdone?$AA@ 0000000039aafba0     GameSpy_2.11.00_VC10:gpiSearch.obj
 0002:0000aba8       ??_C@_05CJPHHPGG@ndone?$AA@ 0000000039aafba8     GameSpy_2.11.00_VC10:gpiSearch.obj
 0002:0000abb0       ??_C@_04JFGJLOFC@nick?$AA@ 0000000039aafbb0     GameSpy_2.11.00_VC10:gpiSearch.obj
 0002:0000abb8       ??_C@_02FPPONLLD@nr?$AA@   0000000039aafbb8     GameSpy_2.11.00_VC10:gpiSearch.obj
 0002:0000abbc       ??_C@_02ENMLCJHL@vr?$AA@   0000000039aafbbc     GameSpy_2.11.00_VC10:gpiSearch.obj
 0002:0000abc0       ??_C@_0CJ@POGGKJFB@Could?5not?5connect?5to?5the?5search?5@ 0000000039aafbc0     GameSpy_2.11.00_VC10:gpiSearch.obj
 0002:0000abf0       ??_C@_0N@JJJFKMBL@?2maxresults?2?$AA@ 0000000039aafbf0     GameSpy_2.11.00_VC10:gpiSearch.obj
 0002:0000ac00       ??_C@_0BC@LPFCPCDL@?2searchprofileid?2?$AA@ 0000000039aafc00     GameSpy_2.11.00_VC10:gpiSearch.obj
 0002:0000ac18       ??_C@_0O@DHIIEPFM@?2profilelist?2?$AA@ 0000000039aafc18     GameSpy_2.11.00_VC10:gpiSearch.obj
 0002:0000ac28       ??_C@_0BA@JCIKPFCA@?2preferrednick?2?$AA@ 0000000039aafc28     GameSpy_2.11.00_VC10:gpiSearch.obj
 0002:0000ac38       ??_C@_0P@DHOIKBNJ@?2uniquesearch?2?$AA@ 0000000039aafc38     GameSpy_2.11.00_VC10:gpiSearch.obj
 0002:0000ac48       ??_C@_01DNKMNLPK@?$HM?$AA@ 0000000039aafc48     GameSpy_2.11.00_VC10:gpiSearch.obj
 0002:0000ac50       ??_C@_07IOFHEGOL@?2opids?2?$AA@ 0000000039aafc50     GameSpy_2.11.00_VC10:gpiSearch.obj
 0002:0000ac58       ??_C@_0L@MOCLIGDH@?2numopids?2?$AA@ 0000000039aafc58     GameSpy_2.11.00_VC10:gpiSearch.obj
 0002:0000ac68       ??_C@_0N@EHNPDOHA@?2otherslist?2?$AA@ 0000000039aafc68     GameSpy_2.11.00_VC10:gpiSearch.obj
 0002:0000ac78       ??_C@_08KIIGMGFA@?2others?2?$AA@ 0000000039aafc78     GameSpy_2.11.00_VC10:gpiSearch.obj
 0002:0000ac88       ??_C@_07BOFLNNMB@?2cdkey?2?$AA@ 0000000039aafc88     GameSpy_2.11.00_VC10:gpiSearch.obj
 0002:0000ac90       ??_C@_0M@NNFNCNPL@?2productID?2?$AA@ 0000000039aafc90     GameSpy_2.11.00_VC10:gpiSearch.obj
 0002:0000aca0       ??_C@_07OMGAILBJ@?2check?2?$AA@ 0000000039aafca0     GameSpy_2.11.00_VC10:gpiSearch.obj
 0002:0000aca8       ??_C@_08HNACKPFL@?2pmatch?2?$AA@ 0000000039aafca8     GameSpy_2.11.00_VC10:gpiSearch.obj
 0002:0000acb8       ??_C@_09NFDNDIEK@?2passenc?2?$AA@ 0000000039aafcb8     GameSpy_2.11.00_VC10:gpiSearch.obj
 0002:0000acc8       ??_C@_07BOCKBGPL@?2nicks?2?$AA@ 0000000039aafcc8     GameSpy_2.11.00_VC10:gpiSearch.obj
 0002:0000acd0       ??_C@_07JHHIKMJA@?2valid?2?$AA@ 0000000039aafcd0     GameSpy_2.11.00_VC10:gpiSearch.obj
 0002:0000acd8       ??_C@_0N@JOKDNOGI@?2namespaces?2?$AA@ 0000000039aafcd8     GameSpy_2.11.00_VC10:gpiSearch.obj
 0002:0000ace8       ??_C@_0P@HOMDGNBL@?2searchunique?2?$AA@ 0000000039aafce8     GameSpy_2.11.00_VC10:gpiSearch.obj
 0002:0000acf8       ??_C@_06OBGDFIPA@?2skip?2?$AA@ 0000000039aafcf8     GameSpy_2.11.00_VC10:gpiSearch.obj
 0002:0000ad00       ??_C@_08BLEPEJPL@?2icquin?2?$AA@ 0000000039aafd00     GameSpy_2.11.00_VC10:gpiSearch.obj
 0002:0000ad10       ??_C@_0L@FLBFBGDI@?2lastname?2?$AA@ 0000000039aafd10     GameSpy_2.11.00_VC10:gpiSearch.obj
 0002:0000ad20       ??_C@_0M@MLJHNAFO@?2firstname?2?$AA@ 0000000039aafd20     GameSpy_2.11.00_VC10:gpiSearch.obj
 0002:0000ad30       ??_C@_08EPCCBDHP@?2search?2?$AA@ 0000000039aafd30     GameSpy_2.11.00_VC10:gpiSearch.obj
 0002:0000ad3c       ??_C@_02CLJDIHEM@SM?$AA@   0000000039aafd3c     GameSpy_2.11.00_VC10:gpiSearch.obj
 0002:0000ad40       ??_C@_0BF@IDBLLAJO@The?5search?5timed?5out?$AA@ 0000000039aafd40     GameSpy_2.11.00_VC10:gpiSearch.obj
 0002:0000ad58       ??_C@_0BI@FPCGDAHO@?2registernick?2?2sesskey?2?$AA@ 0000000039aafd58     GameSpy_2.11.00_VC10:gpiUnique.obj
 0002:0000ad70       ??_C@_04FBEPLGEN@?2rn?2?$AA@ 0000000039aafd70     GameSpy_2.11.00_VC10:gpiUnique.obj
 0002:0000ad78       ??_C@_04FJJHCFBO@?2rc?2?$AA@ 0000000039aafd78     GameSpy_2.11.00_VC10:gpiUnique.obj
 0002:0000ad80       ??_C@_05DJDHFBAG@?2npr?2?$AA@ 0000000039aafd80     GameSpy_2.11.00_VC10:gpiProfile.obj
 0002:0000ad88       ??_C@_09BJPJHHFK@?2oldnick?2?$AA@ 0000000039aafd88     GameSpy_2.11.00_VC10:gpiProfile.obj
 0002:0000ad98       ??_C@_09LPIOLGEK@?2replace?2?$AA@ 0000000039aafd98     GameSpy_2.11.00_VC10:gpiProfile.obj
 0002:0000ada8       ??_C@_0N@JHILOPBN@?2newprofile?2?$AA@ 0000000039aafda8     GameSpy_2.11.00_VC10:gpiProfile.obj
 0002:0000adb8       ??_C@_0BB@LFGPHLGB@Invalid?5replace?4?$AA@ 0000000039aafdb8     GameSpy_2.11.00_VC10:gpiProfile.obj
 0002:0000adcc       ??_C@_05HDIHEJKH@?2dpr?2?$AA@ 0000000039aafdcc     GameSpy_2.11.00_VC10:gpiProfile.obj
 0002:0000add8       ??_C@_0BH@KFFGNOMF@?2removeblock?2?2sesskey?2?$AA@ 0000000039aafdd8     GameSpy_2.11.00_VC10:gpiProfile.obj
 0002:0000adf0       ??_C@_0BE@FAPDOLCK@?2addblock?2?2sesskey?2?$AA@ 0000000039aafdf0     GameSpy_2.11.00_VC10:gpiProfile.obj
 0002:0000ae04       ??_C@_06FBIOKEPJ@?2list?2?$AA@ 0000000039aafe04     GameSpy_2.11.00_VC10:gpiProfile.obj
 0002:0000ae10       ??_C@_0O@FJOFFFMK@Invalid?5date?4?$AA@ 0000000039aafe10     GameSpy_2.11.00_VC10:gpiInfo.obj
 0002:0000ae20       ??_C@_0BE@HBPIMOF@?2updateui?2?2sesskey?2?$AA@ 0000000039aafe20     GameSpy_2.11.00_VC10:gpiInfo.obj
 0002:0000ae38       ??_C@_0BF@NNBHIBHC@?2updatepro?2?2sesskey?2?$AA@ 0000000039aafe38     GameSpy_2.11.00_VC10:gpiInfo.obj
 0002:0000ae50       ??_C@_04LBLHAPFO@?2i1?2?$AA@ 0000000039aafe50     GameSpy_2.11.00_VC10:gpiInfo.obj
 0002:0000ae58       ??_C@_05EJOOCDIA@?2chc?2?$AA@ 0000000039aafe58     GameSpy_2.11.00_VC10:gpiInfo.obj
 0002:0000ae60       ??_C@_05JGDCBLCM@?2mar?2?$AA@ 0000000039aafe60     GameSpy_2.11.00_VC10:gpiInfo.obj
 0002:0000ae68       ??_C@_05CGDFGEPN@?2inc?2?$AA@ 0000000039aafe68     GameSpy_2.11.00_VC10:gpiInfo.obj
 0002:0000ae70       ??_C@_05CDHKHCHI@?2ind?2?$AA@ 0000000039aafe70     GameSpy_2.11.00_VC10:gpiInfo.obj
 0002:0000ae78       ??_C@_05FLBPEJIA@?2occ?2?$AA@ 0000000039aafe78     GameSpy_2.11.00_VC10:gpiInfo.obj
 0002:0000ae80       ??_C@_05NGBCKJLH@?2pic?2?$AA@ 0000000039aafe80     GameSpy_2.11.00_VC10:gpiInfo.obj
 0002:0000ae88       ??_C@_05MLBHCAEO@?2sex?2?$AA@ 0000000039aafe88     GameSpy_2.11.00_VC10:gpiInfo.obj
 0002:0000ae90       ??_C@_09IAEIDFBA@?2zipcode?2?$AA@ 0000000039aafe90     GameSpy_2.11.00_VC10:gpiInfo.obj
 0002:0000ae9c       ??_C@_05IBAMDKIP@?2aim?2?$AA@ 0000000039aafe9c     GameSpy_2.11.00_VC10:gpiInfo.obj
 0002:0000aea8       ??_C@_0O@MJIACEHA@?2countrycode?2?$AA@ 0000000039aafea8     GameSpy_2.11.00_VC10:gpiInfo.obj
 0002:0000aeb8       ??_C@_0L@GEMFFKDM@?2homepage?2?$AA@ 0000000039aafeb8     GameSpy_2.11.00_VC10:gpiInfo.obj
 0002:0000aec8       ??_C@_0L@HDPNANMM@?2birthday?2?$AA@ 0000000039aafec8     GameSpy_2.11.00_VC10:gpiInfo.obj
 0002:0000aed8       ??_C@_0BG@JJHMIEGD@?2getprofile?2?2sesskey?2?$AA@ 0000000039aafed8     GameSpy_2.11.00_VC10:gpiInfo.obj
 0002:0000aef0       ??_C@_05JGLLHLLL@?2sig?2?$AA@ 0000000039aafef0     GameSpy_2.11.00_VC10:gpiInfo.obj
 0002:0000aef8       ??_C@_06JMFKEKGI@?2conn?2?$AA@ 0000000039aafef8     GameSpy_2.11.00_VC10:gpiInfo.obj
 0002:0000af00       ??_C@_04JENMFAIC@?2o1?2?$AA@ 0000000039aaff00     GameSpy_2.11.00_VC10:gpiInfo.obj
 0002:0000af08       ??_C@_07EPACGNKG@?2pmask?2?$AA@ 0000000039aaff08     GameSpy_2.11.00_VC10:gpiInfo.obj
 0002:0000af10       ??_C@_05FGGJIMOI@?2loc?2?$AA@ 0000000039aaff10     GameSpy_2.11.00_VC10:gpiInfo.obj
 0002:0000af18       ??_C@_05KPNPEOCO@?2lat?2?$AA@ 0000000039aaff18     GameSpy_2.11.00_VC10:gpiInfo.obj
 0002:0000af20       ??_C@_05FOLBBPLL@?2lon?2?$AA@ 0000000039aaff20     GameSpy_2.11.00_VC10:gpiInfo.obj
 0002:0000af28       ??_C@_04POAJGIED@?2pi?2?$AA@ 0000000039aaff28     GameSpy_2.11.00_VC10:gpiInfo.obj
 0002:0000af30       ??_C@_0L@MOJHFELE@?2autoSync?2?$AA@ 0000000039aaff30     GameSpy_2.11.00_VC10:gpiBuddy.obj
 0002:0000af40       ??_C@_0BA@DOHADMGK@?2fromprofileid?2?$AA@ 0000000039aaff40     GameSpy_2.11.00_VC10:gpiBuddy.obj
 0002:0000af50       ??_C@_09KFLDMNFO@?2authadd?2?$AA@ 0000000039aaff50     GameSpy_2.11.00_VC10:gpiBuddy.obj
 0002:0000af60       ??_C@_0BA@BLFEHLBD@?2syncrequested?2?$AA@ 0000000039aaff60     GameSpy_2.11.00_VC10:gpiBuddy.obj
 0002:0000af70       ??_C@_04LLKPOCGK@?$CFd?$CFd?$AA@ 0000000039aaff70     GameSpy_2.11.00_VC10:gpiBuddy.obj
 0002:0000af78       ??_C@_08PALDPJFL@?2reason?2?$AA@ 0000000039aaff78     GameSpy_2.11.00_VC10:gpiBuddy.obj
 0002:0000af88       ??_C@_0P@FBPMHNEJ@?2newprofileid?2?$AA@ 0000000039aaff88     GameSpy_2.11.00_VC10:gpiBuddy.obj
 0002:0000af98       ??_C@_0L@FPMJCBLH@?2addbuddy?2?$AA@ 0000000039aaff98     GameSpy_2.11.00_VC10:gpiBuddy.obj
 0002:0000afa8       ??_C@_0N@CLDGODDB@?2qmodeflags?2?$AA@ 0000000039aaffa8     GameSpy_2.11.00_VC10:gpiBuddy.obj
 0002:0000afb8       ??_C@_09BCEHDALB@?2product?2?$AA@ 0000000039aaffb8     GameSpy_2.11.00_VC10:gpiBuddy.obj
 0002:0000afc8       ??_C@_08KCPOCHOL@?2gameMn?2?$AA@ 0000000039aaffc8     GameSpy_2.11.00_VC10:gpiBuddy.obj
 0002:0000afd8       ??_C@_09BKGGEE@?2gameVnt?2?$AA@ 0000000039aaffd8     GameSpy_2.11.00_VC10:gpiBuddy.obj
 0002:0000afe8       ??_C@_0L@FMGPCOGG@?2gameType?2?$AA@ 0000000039aaffe8     GameSpy_2.11.00_VC10:gpiBuddy.obj
 0002:0000aff8       ??_C@_09IIFCHGFI@?2rstatus?2?$AA@ 0000000039aafff8     GameSpy_2.11.00_VC10:gpiBuddy.obj
 0002:0000b008       ??_C@_0M@NDOOFPFA@?2sessflags?2?$AA@ 0000000039ab0008     GameSpy_2.11.00_VC10:gpiBuddy.obj
 0002:0000b018       ??_C@_07LEINJDAD@?2hport?2?$AA@ 0000000039ab0018     GameSpy_2.11.00_VC10:gpiBuddy.obj
 0002:0000b020       ??_C@_07EGMLEKBO@?2qport?2?$AA@ 0000000039ab0020     GameSpy_2.11.00_VC10:gpiBuddy.obj
 0002:0000b028       ??_C@_09NCPJALBN@?2hprivip?2?$AA@ 0000000039ab0028     GameSpy_2.11.00_VC10:gpiBuddy.obj
 0002:0000b038       ??_C@_08HGFFCFNA@?2hostip?2?$AA@ 0000000039ab0038     GameSpy_2.11.00_VC10:gpiBuddy.obj
 0002:0000b048       ??_C@_07BAPNMMEN@?2bport?2?$AA@ 0000000039ab0048     GameSpy_2.11.00_VC10:gpiBuddy.obj
 0002:0000b050       ??_C@_05NCFCHAHM@?2bip?2?$AA@ 0000000039ab0050     GameSpy_2.11.00_VC10:gpiBuddy.obj
 0002:0000b058       ??_C@_07MNHKDBNL@?2state?2?$AA@ 0000000039ab0058     GameSpy_2.11.00_VC10:gpiBuddy.obj
 0002:0000b060       ??_C@_09LPBIDCCI@?2profile?2?$AA@ 0000000039ab0060     GameSpy_2.11.00_VC10:gpiBuddy.obj
 0002:0000b070       ??_C@_0P@OFGGIICE@?2confirmation?2?$AA@ 0000000039ab0070     GameSpy_2.11.00_VC10:gpiBuddy.obj
 0002:0000b080       ??_C@_0CK@MFDKMMHM@There?5was?5an?5error?5looking?5for?5a@ 0000000039ab0080     GameSpy_2.11.00_VC10:gpiBuddy.obj
 0002:0000b0ac       ??_C@_05HGMPOFKD@?2msg?2?$AA@ 0000000039ab00ac     GameSpy_2.11.00_VC10:gpiBuddy.obj
 0002:0000b0b4       ??_C@_03BKJGECCN@?2t?2?$AA@ 0000000039ab00b4     GameSpy_2.11.00_VC10:gpiBuddy.obj
 0002:0000b0b8       ??_C@_0CB@KLBEPEGP@Error?5reading?5keys?5reply?5message@ 0000000039ab00b8     GameSpy_2.11.00_VC10:gpiBuddy.obj
 0002:0000b0dc       ??_C@_04IEPFDAGF@keys?$AA@ 0000000039ab00dc     GameSpy_2.11.00_VC10:gpiBuddy.obj
 0002:0000b0e8       ??_C@_08MIEHMJEN@?2revoke?2?$AA@ 0000000039ab00e8     GameSpy_2.11.00_VC10:gpiBuddy.obj
 0002:0000b0f4       ??_C@_03DNBFDLHJ@?$HMl?$HM?$AA@ 0000000039ab00f4     GameSpy_2.11.00_VC10:gpiBuddy.obj
 0002:0000b0f8       ??_C@_04BFPJKMFM@?$HMqm?$HM?$AA@ 0000000039ab00f8     GameSpy_2.11.00_VC10:gpiBuddy.obj
 0002:0000b100       ??_C@_03CICJGBGN@?$HMp?$HM?$AA@ 0000000039ab0100     GameSpy_2.11.00_VC10:gpiBuddy.obj
 0002:0000b104       ??_C@_04JEKKODAP@?$HMip?$HM?$AA@ 0000000039ab0104     GameSpy_2.11.00_VC10:gpiBuddy.obj
 0002:0000b10c       ??_C@_04KBDCKNGE@?$HMls?$HM?$AA@ 0000000039ab010c     GameSpy_2.11.00_VC10:gpiBuddy.obj
 0002:0000b114       ??_C@_04KJEIOKKN@?$HMss?$HM?$AA@ 0000000039ab0114     GameSpy_2.11.00_VC10:gpiBuddy.obj
 0002:0000b11c       ??_C@_03CKGPNPDE@?$HMs?$HM?$AA@ 0000000039ab011c     GameSpy_2.11.00_VC10:gpiBuddy.obj
 0002:0000b120       ??_C@_08MAMPOACM@?$HMsigned?$HM?$AA@ 0000000039ab0120     GameSpy_2.11.00_VC10:gpiBuddy.obj
 0002:0000b12c       ??_C@_06NJOJMKL@?2date?2?$AA@ 0000000039ab012c     GameSpy_2.11.00_VC10:gpiBuddy.obj
 0002:0000b134       ??_C@_03FDEDFDD@?2f?2?$AA@ 0000000039ab0134     GameSpy_2.11.00_VC10:gpiBuddy.obj
 0002:0000b138       ??_C@_0P@POEBOOCA@?2delprofileid?2?$AA@ 0000000039ab0138     GameSpy_2.11.00_VC10:gpiBuddy.obj
 0002:0000b148       ??_C@_0L@HNHOOFAF@?2delbuddy?2?$AA@ 0000000039ab0148     GameSpy_2.11.00_VC10:gpiBuddy.obj
 0002:0000b154       ??_C@_06JKADEPDE@?2aack?2?$AA@ 0000000039ab0154     GameSpy_2.11.00_VC10:gpiPeer.obj
 0002:0000b160       ??_C@_07FICGNPON@?2anack?2?$AA@ 0000000039ab0160     GameSpy_2.11.00_VC10:gpiPeer.obj
 0002:0000b168       ??_C@_06PANCKDFN@?$CFs?$CFd?$CFd?$AA@ 0000000039ab0168     GameSpy_2.11.00_VC10:gpiPeer.obj
 0002:0000b170       ??_C@_06MAOLKPAJ@?2auth?2?$AA@ 0000000039ab0170     GameSpy_2.11.00_VC10:gpiPeer.obj
 0002:0000b178       ??_C@_0DH@BGCGBPNN@There?5was?5an?5error?5starting?5comm@ 0000000039ab0178     GameSpy_2.11.00_VC10:gpiPeer.obj
 0002:0000b1b0       ??_C@_0BM@HBBOFLCP@Error?5connecting?5to?5a?5peer?4?$AA@ 0000000039ab01b0     GameSpy_2.11.00_VC10:gpiPeer.obj
 0002:0000b1cc       ??_C@_06LFEGNFDN@?2msg?2?6?$AA@ 0000000039ab01cc     GameSpy_2.11.00_VC10:gpiPeer.obj
 0002:0000b1d4       ??_C@_05DBAMPPNP@?2len?2?$AA@ 0000000039ab01d4     GameSpy_2.11.00_VC10:gpiPeer.obj
 0002:0000b1dc       ??_C@_03JGBNKNC@?2m?2?$AA@ 0000000039ab01dc     GameSpy_2.11.00_VC10:gpiPeer.obj
 0002:0000b1e0       ??_C@_0BE@OFCBGMOK@?2m?2?$CFd?2xfer?2?$CFd?5?$CFu?5?$CFu?$AA@ 0000000039ab01e0     GameSpy_2.11.00_VC10:gpiPeer.obj
 0002:0000b1f8       ??_C@_0O@ONJKODNM@?2len?2?$CFd?2msg?2?6?$AA@ 0000000039ab01f8     GameSpy_2.11.00_VC10:gpiPeer.obj
 0002:0000b208       ??_C@_0BN@OKLGFAIB@Error?5parsing?5buddy?5message?4?$AA@ 0000000039ab0208     GameSpy_2.11.00_VC10:gpiPeer.obj
 0002:0000b228       ??_C@_0CD@ODDMLKOC@Error?5getting?5buddy?5authorizatio@ 0000000039ab0228     GameSpy_2.11.00_VC10:gpiPeer.obj
 0002:0000b250       ??_C@_0CI@OJEGHLKO@There?5was?5an?5error?5sending?5on?5a?5@ 0000000039ab0250     GameSpy_2.11.00_VC10:gpiBuffer.obj
 0002:0000b278       ??_C@_0CK@PHAHLLH@There?5was?5an?5error?5reading?5from?5@ 0000000039ab0278     GameSpy_2.11.00_VC10:gpiBuffer.obj
 0002:0000b2a8       ??_C@_0CH@MEEENENH@xsd?$DN?$CChttp?3?1?1www?4w3?4org?12001?1XMLS@ 0000000039ab02a8     GameSpy_2.11.00_VC10:gsXML.obj
 0002:0000b2d0       ??_C@_0DA@OOPIJLIO@xsi?$DN?$CChttp?3?1?1www?4w3?4org?12001?1XMLS@ 0000000039ab02d0     GameSpy_2.11.00_VC10:gsXML.obj
 0002:0000b300       ??_C@_0DF@GBBBDBDI@SOAP?9ENC?$DN?$CChttp?3?1?1schemas?4xmlsoap@ 0000000039ab0300     GameSpy_2.11.00_VC10:gsXML.obj
 0002:0000b338       ??_C@_0DF@EMCKDFHG@SOAP?9ENV?$DN?$CChttp?3?1?1schemas?4xmlsoap@ 0000000039ab0338     GameSpy_2.11.00_VC10:gsXML.obj
 0002:0000b370       ??_C@_04HHCDBDLF@?5?7?$AN?6?$AA@ 0000000039ab0370     GameSpy_2.11.00_VC10:gsXML.obj
 0002:0000b378       ??_C@_02ICNHGLNO@?$CG?$CD?$AA@ 0000000039ab0378     GameSpy_2.11.00_VC10:gsXML.obj
 0002:0000b37c       ??_C@_04NEJBHOB@?$CF08x?$AA@ 0000000039ab037c     GameSpy_2.11.00_VC10:gsXML.obj
 0002:0000b384       ??_C@_03IGAPNLEG@?$CG?$CDx?$AA@ 0000000039ab0384     GameSpy_2.11.00_VC10:gsXML.obj
 0002:0000b388       ??_C@_04LOOHDCEI@?$CGgt?$DL?$AA@ 0000000039ab0388     GameSpy_2.11.00_VC10:gsXML.obj
 0002:0000b390       ??_C@_04GJOGLFEJ@?$CGlt?$DL?$AA@ 0000000039ab0390     GameSpy_2.11.00_VC10:gsXML.obj
 0002:0000b398       ??_C@_06PNMEMOHD@?$CGapos?$DL?$AA@ 0000000039ab0398     GameSpy_2.11.00_VC10:gsXML.obj
 0002:0000b3a0       ??_C@_06DDLNFFBN@?$CGquot?$DL?$AA@ 0000000039ab03a0     GameSpy_2.11.00_VC10:gsXML.obj
 0002:0000b3a8       ??_C@_05JKJFEODM@?$CGamp?$DL?$AA@ 0000000039ab03a8     GameSpy_2.11.00_VC10:gsXML.obj
 0002:0000b3b0       ??_C@_08IKFBCBHI@?$CG?$CDx?$CF02x?$DL?$AA@ 0000000039ab03b0     GameSpy_2.11.00_VC10:gsXML.obj
 0002:0000b3bc       ??_C@_06MEJPMKDD@?$CG?$CDx20?$DL?$AA@ 0000000039ab03bc     GameSpy_2.11.00_VC10:gsXML.obj
 0002:0000b3c4       ??_C@_04CJICMGO@?$CF01x?$AA@ 0000000039ab03c4     GameSpy_2.11.00_VC10:gsXML.obj
 0002:0000b3d0       ??_C@_0BM@PGELMDGJ@?$CFi?9?$CF02d?9?$CF02dT?$CF02d?3?$CF02d?3?$CF02d?$AA@ 0000000039ab03d0     GameSpy_2.11.00_VC10:gsXML.obj
 0002:0000b3f0       ??_C@_0BA@NKBFEIBO@?$DMSOAP?9ENV?3Body?$DO?$AA@ 0000000039ab03f0     GameSpy_2.11.00_VC10:gsXML.obj
 0002:0000b400       ??_C@_06PNFLLAEF@xmlns?3?$AA@ 0000000039ab0400     GameSpy_2.11.00_VC10:gsXML.obj
 0002:0000b408       ??_C@_0DJ@KOAJJEOL@?$DM?$DPxml?5version?$DN?$CC1?40?$CC?5encoding?$DN?$CCUT@ 0000000039ab0408     GameSpy_2.11.00_VC10:gsXML.obj
 0002:0000b448       ??_C@_0CF@PEBFKDMP@?$DM?1SOAP?9ENV?3Body?$DO?$DM?1SOAP?9ENV?3Envel@ 0000000039ab0448     GameSpy_2.11.00_VC10:gsXML.obj
 0002:0000b470       ??_C@_02NJPGOMH@?$CFf?$AA@ 0000000039ab0470     GameSpy_2.11.00_VC10:gsXML.obj
 0002:0000b478       ??_C@_0BN@HOABMGGA@?$CFd?9?$CF02d?9?$CF02dT?$CF02d?3?$CF02d?3?$CF02dZ?$AA@ 0000000039ab0478     GameSpy_2.11.00_VC10:gsXML.obj
 0002:0000b498       ??_C@_02PCIJFNDE@?$AN?6?$AA@ 0000000039ab0498     GameSpy_2.11.00_VC10:gsLargeInt.obj
 0002:0000b4a0       GVDefaultPlaybackDeviceID  0000000039ab04a0     GameSpy_2.11.00_VC10:gvDirectSound.obj
 0002:0000b4b0       GVDefaultCaptureDeviceID   0000000039ab04b0     GameSpy_2.11.00_VC10:gvDirectSound.obj
 0002:0000b4c0       __real@409f400000000000    0000000039ab04c0     GameSpy_2.11.00_VC10:gvDirectSound.obj
 0002:0000b4c8       __real@0000000000000000    0000000039ab04c8     GameSpy_2.11.00_VC10:gvDirectSound.obj
 0002:0000b4d0       __real@477fff00            0000000039ab04d0     GameSpy_2.11.00_VC10:gvSource.obj
 0002:0000b4d8       __real@3fa0000000000000    0000000039ab04d8     GameSpy_2.11.00_VC10:gvSource.obj
 0002:0000b4e0       __real@3fef000000000000    0000000039ab04e0     GameSpy_2.11.00_VC10:gvSource.obj
 0002:0000b4e8       ??_C@_01KMDKNFGN@?1?$AA@   0000000039ab04e8     GameSpy_2.11.00_VC10:ghttpProcess.obj
 0002:0000b4ec       ??_C@_02DLFOHOMG@?3?1?$AA@ 0000000039ab04ec     GameSpy_2.11.00_VC10:ghttpProcess.obj
 0002:0000b4f0       ??_C@_0N@LAFFMKKA@Content?9Type?$AA@ 0000000039ab04f0     GameSpy_2.11.00_VC10:ghttpProcess.obj
 0002:0000b500       ??_C@_0P@HOJGPHBA@Content?9Length?$AA@ 0000000039ab0500     GameSpy_2.11.00_VC10:ghttpProcess.obj
 0002:0000b510       ??_C@_05LBOHBHFK@close?$AA@ 0000000039ab0510     GameSpy_2.11.00_VC10:ghttpProcess.obj
 0002:0000b518       ??_C@_0L@NEAPGCKH@Keep?9Alive?$AA@ 0000000039ab0518     GameSpy_2.11.00_VC10:ghttpProcess.obj
 0002:0000b528       ??_C@_0L@PJJKMLL@Connection?$AA@ 0000000039ab0528     GameSpy_2.11.00_VC10:ghttpProcess.obj
 0002:0000b538       ??_C@_0BA@CFMHCFDE@GameSpyHTTP?11?40?$AA@ 0000000039ab0538     GameSpy_2.11.00_VC10:ghttpProcess.obj
 0002:0000b548       ??_C@_0L@DMPACEMJ@User?9Agent?$AA@ 0000000039ab0548     GameSpy_2.11.00_VC10:ghttpProcess.obj
 0002:0000b554       ??_C@_06KICEPCA@Host?3?5?$AA@ 0000000039ab0554     GameSpy_2.11.00_VC10:ghttpProcess.obj
 0002:0000b55c       ??_C@_04CPPPJGME@Host?$AA@ 0000000039ab055c     GameSpy_2.11.00_VC10:ghttpProcess.obj
 0002:0000b568       ??_C@_0M@IHFDHEJ@?5HTTP?11?41?$AN?6?$AA@ 0000000039ab0568     GameSpy_2.11.00_VC10:ghttpProcess.obj
 0002:0000b574       ??_C@_04IBPFIGHK@GET?5?$AA@ 0000000039ab0574     GameSpy_2.11.00_VC10:ghttpProcess.obj
 0002:0000b57c       ??_C@_05PMJKDPIC@HEAD?5?$AA@ 0000000039ab057c     GameSpy_2.11.00_VC10:ghttpProcess.obj
 0002:0000b584       ??_C@_05LPJJJLLB@POST?5?$AA@ 0000000039ab0584     GameSpy_2.11.00_VC10:ghttpProcess.obj
 0002:0000b590       ??_C@_0BA@MDOOLGGO@HTTP?1?$CFd?4?$CFd?5?$CFd?$CFn?$AA@ 0000000039ab0590     GameSpy_2.11.00_VC10:ghttpProcess.obj
 0002:0000b5a0       ??_C@_02NJNOFBBI@?$CFx?$AA@ 0000000039ab05a0     GameSpy_2.11.00_VC10:ghttpProcess.obj
 0002:0000b5a8       ??_C@_0BL@CJMPBBIJ@Transfer?9Encoding?3?5chunked?$AA@ 0000000039ab05a8     GameSpy_2.11.00_VC10:ghttpProcess.obj
 0002:0000b5c8       ??_C@_0BE@EMNEAFKL@9223372036854775807?$AA@ 0000000039ab05c8     GameSpy_2.11.00_VC10:ghttpProcess.obj
 0002:0000b5e0       ??_C@_0BA@DIGAFIOK@Content?9Length?3?$AA@ 0000000039ab05e0     GameSpy_2.11.00_VC10:ghttpProcess.obj
 0002:0000b5f0       ??_C@_0P@GPICDECC@http?3?1?1?$CFs?3?$CFd?$CFs?$AA@ 0000000039ab05f0     GameSpy_2.11.00_VC10:ghttpProcess.obj
 0002:0000b600       ??_C@_09GILIFLDG@Location?3?$AA@ 0000000039ab0600     GameSpy_2.11.00_VC10:ghttpProcess.obj
 0002:0000b60c       ??_C@_04FMMHFHOO@?$AN?6?$AN?6?$AA@ 0000000039ab060c     GameSpy_2.11.00_VC10:ghttpProcess.obj
 0002:0000b614       ??_C@_02PHMGELLB@?6?6?$AA@ 0000000039ab0614     GameSpy_2.11.00_VC10:ghttpProcess.obj
 0002:0000b620       ??_C@_0EE@JPFGHMNM@abcdefghijklmnopqrstuvwxyzABCDEF@ 0000000039ab0620     GameSpy_2.11.00_VC10:ghttpPost.obj
 0002:0000b668       ??_C@_0CC@FLKANKNI@application?1x?9www?9form?9urlencode@ 0000000039ab0668     GameSpy_2.11.00_VC10:ghttpPost.obj
 0002:0000b690       ??_C@_08HNLEKLC@text?1xml?$AA@ 0000000039ab0690     GameSpy_2.11.00_VC10:ghttpPost.obj
 0002:0000b6a0       ??_C@_0EC@IAIKEPIM@multipart?1form?9data?$DL?5boundary?$DNQr@ 0000000039ab06a0     GameSpy_2.11.00_VC10:ghttpPost.obj
 0002:0000b6e8       ??_C@_0BB@KDHCEMMM@application?1dime?$AA@ 0000000039ab06e8     GameSpy_2.11.00_VC10:ghttpPost.obj
 0002:0000b700       ??_C@_0BB@JGGOGLEG@0123456789ABCDEF?$AA@ 0000000039ab0700     GameSpy_2.11.00_VC10:ghttpPost.obj
 0002:0000b720       ??_C@_0FB@LFLBBDBP@?$CFsContent?9Disposition?3?5form?9data@ 0000000039ab0720     GameSpy_2.11.00_VC10:ghttpPost.obj
 0002:0000b778       ??_C@_0CK@KLFMLHIL@http?3?1?1schemas?4xmlsoap?4org?1soap?1@ 0000000039ab0778     GameSpy_2.11.00_VC10:ghttpPost.obj
 0002:0000b7a8       ??_C@_07HENFIOBF@cid?3id0?$AA@ 0000000039ab07a8     GameSpy_2.11.00_VC10:ghttpPost.obj
 0002:0000b7b0       ??_C@_0DA@OGFACAAI@?$CFsContent?9Disposition?3?5form?9data@ 0000000039ab07b0     GameSpy_2.11.00_VC10:ghttpPost.obj
 0002:0000b7e0       ??_C@_0CK@LPMEGCKG@?$AN?6?9?9Qr4G823s23d?9?9?9?$DM?$DM?$DO?$DM?$DO?$DM?$DM?$DM?$DO?9?97d1@ 0000000039ab07e0     GameSpy_2.11.00_VC10:ghttpPost.obj
 0002:0000b810       ??_C@_0CI@NFLGGFMB@?9?9Qr4G823s23d?9?9?9?$DM?$DM?$DO?$DM?$DO?$DM?$DM?$DM?$DO?9?97d118@ 0000000039ab0810     GameSpy_2.11.00_VC10:ghttpPost.obj
 0002:0000b838       ??_C@_04NMOPBDPN@?$CG?$CFs?$DN?$AA@ 0000000039ab0838     GameSpy_2.11.00_VC10:ghttpPost.obj
 0002:0000b840       ??_C@_03HFAIOBFI@?$CFs?$DN?$AA@ 0000000039ab0840     GameSpy_2.11.00_VC10:ghttpPost.obj
 0002:0000b848       ??_C@_0CM@FFPCGHIF@?$AN?6?9?9Qr4G823s23d?9?9?9?$DM?$DM?$DO?$DM?$DO?$DM?$DM?$DM?$DO?9?97d1@ 0000000039ab0848     GameSpy_2.11.00_VC10:ghttpPost.obj
 0002:0000b874       ??_C@_02LMMGGCAJ@?3?5?$AA@ 0000000039ab0874     GameSpy_2.11.00_VC10:ghttpBuffer.obj
 0002:0000b890       ??_C@_07PJIIAIPG@summary?$AA@ 0000000039ab0890     GameSpy_2.11.00_VC10:d2gDeserialize.obj
 0002:0000b898       ??_C@_09DNECJBKD@developer?$AA@ 0000000039ab0898     GameSpy_2.11.00_VC10:d2gDeserialize.obj
 0002:0000b8a8       ??_C@_09LCNOBMAC@publisher?$AA@ 0000000039ab08a8     GameSpy_2.11.00_VC10:d2gDeserialize.obj
 0002:0000b8b8       ??_C@_0BB@FEMNIALK@filesizebytessum?$AA@ 0000000039ab08b8     GameSpy_2.11.00_VC10:d2gDeserialize.obj
 0002:0000b8d0       ??_C@_0M@INFFNGGL@releasedate?$AA@ 0000000039ab08d0     GameSpy_2.11.00_VC10:d2gDeserialize.obj
 0002:0000b8dc       ??_C@_05NGOMGBBD@image?$AA@ 0000000039ab08dc     GameSpy_2.11.00_VC10:d2gDeserialize.obj
 0002:0000b8e8       ??_C@_09JBMKNKFJ@imagelist?$AA@ 0000000039ab08e8     GameSpy_2.11.00_VC10:d2gDeserialize.obj
 0002:0000b8f8       ??_C@_0N@OIGLEKIA@categorylist?$AA@ 0000000039ab08f8     GameSpy_2.11.00_VC10:d2gDeserialize.obj
 0002:0000b908       ??_C@_0BE@NMIOJGPG@orderitemstatuscode?$AA@ 0000000039ab0908     GameSpy_2.11.00_VC10:d2gDeserialize.obj
 0002:0000b920       ??_C@_07MGLHPHCG@isvalid?$AA@ 0000000039ab0920     GameSpy_2.11.00_VC10:d2gDeserialize.obj
 0002:0000b928       ??_C@_0BE@ONBCKFDL@orderitemvalidation?$AA@ 0000000039ab0928     GameSpy_2.11.00_VC10:d2gDeserialize.obj
 0002:0000b940       ??_C@_0M@BDAKLDDB@licensename?$AA@ 0000000039ab0940     GameSpy_2.11.00_VC10:d2gDeserialize.obj
 0002:0000b950       ??_C@_0L@EFIKHNHE@licensekey?$AA@ 0000000039ab0950     GameSpy_2.11.00_VC10:d2gDeserialize.obj
 0002:0000b960       ??_C@_07EJMBNAEG@license?$AA@ 0000000039ab0960     GameSpy_2.11.00_VC10:d2gDeserialize.obj
 0002:0000b968       ??_C@_08JLOEAPEA@licenses?$AA@ 0000000039ab0968     GameSpy_2.11.00_VC10:d2gDeserialize.obj
 0002:0000b978       ??_C@_09NGICODJK@assettype?$AA@ 0000000039ab0978     GameSpy_2.11.00_VC10:d2gDeserialize.obj
 0002:0000b988       ??_C@_08IBBDGPOF@sequence?$AA@ 0000000039ab0988     GameSpy_2.11.00_VC10:d2gDeserialize.obj
 0002:0000b998       ??_C@_09JGLNCENF@downloads?$AA@ 0000000039ab0998     GameSpy_2.11.00_VC10:d2gDeserialize.obj
 0002:0000b9a8       ??_C@_0BC@IAMBJFOP@orderitempurchase?$AA@ 0000000039ab09a8     GameSpy_2.11.00_VC10:d2gDeserialize.obj
 0002:0000b9c0       ??_C@_0BD@DECHBEEJ@orderitempurchases?$AA@ 0000000039ab09c0     GameSpy_2.11.00_VC10:d2gDeserialize.obj
 0002:0000b9d8       ??_C@_0BA@GGOMMOJG@orderstatuscode?$AA@ 0000000039ab09d8     GameSpy_2.11.00_VC10:d2gDeserialize.obj
 0002:0000b9e8       ??_C@_0BA@FHHAPNFL@ordervalidation?$AA@ 0000000039ab09e8     GameSpy_2.11.00_VC10:d2gDeserialize.obj
 0002:0000b9f8       ??_C@_0P@PAGIGOMJ@orderitemtotal?$AA@ 0000000039ab09f8     GameSpy_2.11.00_VC10:d2gDeserialize.obj
 0002:0000ba08       ??_C@_0BA@OGFKDIEP@orderitemtotals?$AA@ 0000000039ab0a08     GameSpy_2.11.00_VC10:d2gDeserialize.obj
 0002:0000ba18       ??_C@_0L@NOFGMPDD@datequoted?$AA@ 0000000039ab0a18     GameSpy_2.11.00_VC10:d2gDeserialize.obj
 0002:0000ba28       ??_C@_0O@DLLNGH@datepurchased?$AA@ 0000000039ab0a28     GameSpy_2.11.00_VC10:d2gDeserialize.obj
 0002:0000ba38       ??_C@_01JLIPDDHJ@?3?$AA@   0000000039ab0a38     GameSpy_2.11.00_VC10:d2gDeserialize.obj
 0002:0000ba3c       ??_C@_03ICHNJLJF@key?$AA@  0000000039ab0a3c     GameSpy_2.11.00_VC10:d2gDeserialize.obj
 0002:0000ba40       ??_C@_0BB@KENJGEHM@urlrequestheader?$AA@ 0000000039ab0a40     GameSpy_2.11.00_VC10:d2gDeserialize.obj
 0002:0000ba58       ??_C@_0BF@OIHOCNEB@urlrequestheaderlist?$AA@ 0000000039ab0a58     GameSpy_2.11.00_VC10:d2gDeserialize.obj
 0002:0000ba70       ??_C@_0O@IGJALBIA@extensiondata?$AA@ 0000000039ab0a70     GameSpy_2.11.00_VC10:d2gDeserialize.obj
 0002:0000ba80       ??_C@_0BC@FLFHMGCN@extensiondatalist?$AA@ 0000000039ab0a80     GameSpy_2.11.00_VC10:d2gDeserialize.obj
 0002:0000ba98       ??_C@_0O@FLCIIHPG@storestatusid?$AA@ 0000000039ab0a98     GameSpy_2.11.00_VC10:d2gDeserialize.obj
 0002:0000baa8       ??_C@_0BL@HGAACLH@GetStoreAvailabilityResult?$AA@ 0000000039ab0aa8     GameSpy_2.11.00_VC10:d2gDeserialize.obj
 0002:0000bac8       ??_C@_09FJAGOGIC@isdefault?$AA@ 0000000039ab0ac8     GameSpy_2.11.00_VC10:d2gDeserialize.obj
 0002:0000bad8       ??_C@_0M@LOHFKBPI@accounttype?$AA@ 0000000039ab0ad8     GameSpy_2.11.00_VC10:d2gDeserialize.obj
 0002:0000bae8       ??_C@_0P@JOHGGBII@expirationdate?$AA@ 0000000039ab0ae8     GameSpy_2.11.00_VC10:d2gDeserialize.obj
 0002:0000baf8       ??_C@_0BA@CDOBBOGN@lastfournumbers?$AA@ 0000000039ab0af8     GameSpy_2.11.00_VC10:d2gDeserialize.obj
 0002:0000bb08       ??_C@_0L@GINGEIKC@creditcard?$AA@ 0000000039ab0b08     GameSpy_2.11.00_VC10:d2gDeserialize.obj
 0002:0000bb18       ??_C@_0P@KOIMODL@creditcardlist?$AA@ 0000000039ab0b18     GameSpy_2.11.00_VC10:d2gDeserialize.obj
 0002:0000bb28       ??_C@_0BJ@BGFIECGO@GetUserCreditCardsResult?$AA@ 0000000039ab0b28     GameSpy_2.11.00_VC10:d2gDeserialize.obj
 0002:0000bb48       ??_C@_0M@PPHNPGFJ@catalogitem?$AA@ 0000000039ab0b48     GameSpy_2.11.00_VC10:d2gDeserialize.obj
 0002:0000bb58       ??_C@_0BA@LHNHOPEC@catalogitemlist?$AA@ 0000000039ab0b58     GameSpy_2.11.00_VC10:d2gDeserialize.obj
 0002:0000bb68       ??_C@_0BC@FBEIGCEK@GetAllItemsResult?$AA@ 0000000039ab0b68     GameSpy_2.11.00_VC10:d2gDeserialize.obj
 0002:0000bb80       ??_C@_0L@KIEKNLAB@ordertotal?$AA@ 0000000039ab0b80     GameSpy_2.11.00_VC10:d2gDeserialize.obj
 0002:0000bb90       ??_C@_0BE@KBBHNKGD@GetOrderTotalResult?$AA@ 0000000039ab0b90     GameSpy_2.11.00_VC10:d2gDeserialize.obj
 0002:0000bba8       ??_C@_0O@FDKPEJFG@orderpurchase?$AA@ 0000000039ab0ba8     GameSpy_2.11.00_VC10:d2gDeserialize.obj
 0002:0000bbb8       ??_C@_0BB@DKILOGPP@PlaceOrderResult?$AA@ 0000000039ab0bb8     GameSpy_2.11.00_VC10:d2gDeserialize.obj
 0002:0000bbd0       ??_C@_0BF@GBCBLOD@GetPlacedOrderResult?$AA@ 0000000039ab0bd0     GameSpy_2.11.00_VC10:d2gDeserialize.obj
 0002:0000bbe8       ??_C@_0P@IGEJHBLN@orderpurchases?$AA@ 0000000039ab0be8     GameSpy_2.11.00_VC10:d2gDeserialize.obj
 0002:0000bbf8       ??_C@_0BJ@HCFLKPFF@GetPurchaseHistoryResult?$AA@ 0000000039ab0bf8     GameSpy_2.11.00_VC10:d2gDeserialize.obj
 0002:0000bd30       ??_C@_0BC@BMCHOAML@Invalid?5key?5value?$AA@ 0000000039ab0d30     GameSpy_2.11.00_VC10:gpiKeys.obj
 0002:0000bd48       ??_C@_0BB@GNMJJIKD@Invalid?5key?5name?$AA@ 0000000039ab0d48     GameSpy_2.11.00_VC10:gpiKeys.obj
 0002:0000bd60       ??_C@_08PFAMNKDI@?2keys?2?$CFd?$AA@ 0000000039ab0d60     GameSpy_2.11.00_VC10:gpiKeys.obj
 0002:0000bd70       ??_C@_0BG@GBOCBGGC@?2version?2?$CFd?2result?2?$CFd?$AA@ 0000000039ab0d70     GameSpy_2.11.00_VC10:gpiTransfer.obj
 0002:0000bd88       ??_C@_08OACDOGNM@?$CFd?5?$CFu?5?$CFu?$AA@ 0000000039ab0d88     GameSpy_2.11.00_VC10:gpiTransfer.obj
 0002:0000bd94       ??_C@_06DKGGAHFE@?2xfer?2?$AA@ 0000000039ab0d94     GameSpy_2.11.00_VC10:gpiTransfer.obj
 0002:0000bda0       __real@3f00000000000000    0000000039ab0da0     GameSpy_2.11.00_VC10:gvUtil.obj
 0002:0000bda8       __real@40dfffc000000000    0000000039ab0da8     GameSpy_2.11.00_VC10:gvUtil.obj
 0002:0000bdb0       ??_C@_04GDFOJGBM@DDDD?$AA@ 0000000039ab0db0     GameSpy_2.11.00_VC10:ghttpEncryption.obj
 0002:0000bdb8       ??_C@_03POJCPIGP@CCC?$AA@  0000000039ab0db8     GameSpy_2.11.00_VC10:ghttpEncryption.obj
 0002:0000bdbc       ??_C@_02LBOPFCME@BB?$AA@   0000000039ab0dbc     GameSpy_2.11.00_VC10:ghttpEncryption.obj
 0002:0000bdc0       ??_C@_0DB@EKDBJDAA@?2?2?2?2?2?2?2?2?2?2?2?2?2?2?2?2?2?2?2?2?2?2?2?2?2?2?2?2?2?2?2?2@ 0000000039ab0dc0     GameSpy_2.11.00_VC10:ghttpEncryption.obj
 0002:0000bdf4       ??_C@_01LLKFGJJG@?$BH?$AA@ 0000000039ab0df4     GameSpy_2.11.00_VC10:ghttpEncryption.obj
 0002:0000bdf8       ??_C@_0DB@IKGHIKMM@66666666666666666666666666666666@ 0000000039ab0df8     GameSpy_2.11.00_VC10:ghttpEncryption.obj
 0002:0000be2c       ??_C@_04FDJPPFGE@CLNT?$AA@ 0000000039ab0e2c     GameSpy_2.11.00_VC10:ghttpEncryption.obj
 0002:0000be38       gsSSLCipherSuites          0000000039ab0e38     GameSpy_2.11.00_VC10:gsSSL.obj
 0002:0000be48       gsSslRsaOid                0000000039ab0e48     GameSpy_2.11.00_VC10:gsSSL.obj
 0002:0000be54       ??_C@_04CLCEDBPF@time?$AA@ 0000000039ab0e54     GameSpy_2.11.00_VC10:gt2Message.obj
 0002:0000be5c       ??_C@_02DFNLLEAE@?$PO?$PO?$AA@ 0000000039ab0e5c     GameSpy_2.11.00_VC10:gt2Message.obj
 0002:0000be60       DSDEVID_DefaultVoicePlayback 0000000039ab0e60     dxguid:dxguid.obj
 0002:0000be70       DSDEVID_DefaultVoiceCapture 0000000039ab0e70     dxguid:dxguid.obj
 0002:0000bee8       __rtc_iaa                  0000000039ab0ee8     MSVCRT:_initsect_.obj
 0002:0000bef0       __rtc_izz                  0000000039ab0ef0     MSVCRT:_initsect_.obj
 0002:0000bef8       __rtc_taa                  0000000039ab0ef8     MSVCRT:_initsect_.obj
 0002:0000bf00       __rtc_tzz                  0000000039ab0f00     MSVCRT:_initsect_.obj
 0002:00018774       __IMPORT_DESCRIPTOR_WSOCK32 0000000039abd774     Wsock32:WSOCK32.dll
 0002:00018788       __IMPORT_DESCRIPTOR_WS2_32 0000000039abd788     Ws2_32:WS2_32.dll
 0002:0001879c       __IMPORT_DESCRIPTOR_KERNEL32 0000000039abd79c     kernel32:KERNEL32.dll
 0002:000187b0       __IMPORT_DESCRIPTOR_USER32 0000000039abd7b0     user32:USER32.dll
 0002:000187c4       __IMPORT_DESCRIPTOR_MSVCR100 0000000039abd7c4     MSVCRT:MSVCR100.dll
 0002:000187d8       __IMPORT_DESCRIPTOR_DSOUND 0000000039abd7d8     dsound:DSOUND.dll
 0002:000187ec       __IMPORT_DESCRIPTOR_ADVAPI32 0000000039abd7ec     advapi32:ADVAPI32.dll
 0002:00018800       __IMPORT_DESCRIPTOR_ole32  0000000039abd800     ole32:ole32.dll
 0002:00018814       __NULL_IMPORT_DESCRIPTOR   0000000039abd814     Wsock32:WSOCK32.dll
 0003:00000000       ?sEmptyStringBuffer@?1??_emptyHeader@?$CryStringT@_W@@KAPEAUStrHeader@2@XZ@4PAU32@A 0000000039abf000     CryDLCStore.obj
 0003:00000018       ?g_lobbyEncryptionKey@@3PEBDEB 0000000039abf018     CryLobby.obj
 0003:00000020       ?sEmptyStringBuffer@?1??_emptyHeader@?$CryStringT@D@@KAPEAUStrHeader@2@XZ@4PAU32@A 0000000039abf020     CryLobby.obj
 0003:00000040       ?type@?1???$GetVTableForType@USNullAddr@@@?$CConfigurableVariant@V?$CNode@USNullAddr@@V?$CNode@GV?$CNode@USIPv4Addr@@V?$CNode@ULobbyIdAddr@@VCEnd@NTypelist@@@NTypelist@@@NTypelist@@@NTypelist@@@NTypelist@@$07VCDefaultVariantConversion@NConfigurableVariantHelpers@@VCDefaultVariantConstruction@4@@@AEAAPEAUVTable@1@XZ@4U21@A 0000000039abf040     CryLobby.obj
 0003:00000080       ?type@?1???$GetVTableForType@USIPv4Addr@@@?$CConfigurableVariant@V?$CNode@USNullAddr@@V?$CNode@GV?$CNode@USIPv4Addr@@V?$CNode@ULobbyIdAddr@@VCEnd@NTypelist@@@NTypelist@@@NTypelist@@@NTypelist@@@NTypelist@@$07VCDefaultVariantConversion@NConfigurableVariantHelpers@@VCDefaultVariantConstruction@4@@@AEAAPEAUVTable@1@XZ@4U21@A 0000000039abf080     CryLobby.obj
 0003:000000c0       ?m_seed@CLCGRndGen@@0_KA   0000000039abf0c0     CryLobbyDLL.obj
 0003:000000e0       ?type@?1???$GetVTableForType@G@?$CConfigurableVariant@V?$CNode@USNullAddr@@V?$CNode@GV?$CNode@USIPv4Addr@@V?$CNode@ULobbyIdAddr@@VCEnd@NTypelist@@@NTypelist@@@NTypelist@@@NTypelist@@@NTypelist@@$07VCDefaultVariantConversion@NConfigurableVariantHelpers@@VCDefaultVariantConstruction@4@@@AEAAPEAUVTable@1@XZ@4U21@A 0000000039abf0e0     CryGameSpySBQR2MatchMaking.obj
 0003:00000120       ?pGameSpyFieldRowName@@3PEBDEB 0000000039abf120     CryGameSpySBQR2Stats.obj
 0003:00000128       ?pGameSpyFieldP2POwnerIDName@@3PEBDEB 0000000039abf128     CryGameSpySBQR2Stats.obj
 0003:00000130       ?pGameSpyFieldDedicatedOwnerIDName@@3PEBDEB 0000000039abf130     CryGameSpySBQR2Stats.obj
 0003:00000138       ?pGameSpyFieldOwnerNameName@@3PEBDEB 0000000039abf138     CryGameSpySBQR2Stats.obj
 0003:00000140       ?pGameSpyFieldRecordName@@3PEBDEB 0000000039abf140     CryGameSpySBQR2Stats.obj
 0003:00000148       ?pGameSpyFieldScoreName@@3PEBDEB 0000000039abf148     CryGameSpySBQR2Stats.obj
 0003:00000150       ?pGameSpyStatsFieldName@@3PEBDEB 0000000039abf150     CryGameSpySBQR2Stats.obj
 0003:00000158       ?pGameSpyStatsOrder@@3PEBDEB 0000000039abf158     CryGameSpySBQR2Stats.obj
 0003:00000160       ?pGameSpyFieldNameFormat@@3PEBDEB 0000000039abf160     CryGameSpySBQR2Stats.obj
 0003:00000168       ?pGameSpyTableOrder@@3PEBDEB 0000000039abf168     CryGameSpySBQR2Stats.obj
 0003:00000170       ?pGameSpySearchP2PFormat@@3PEBDEB 0000000039abf170     CryGameSpySBQR2Stats.obj
 0003:00000178       ?pGameSpySearchDedicatedFormat@@3PEBDEB 0000000039abf178     CryGameSpySBQR2Stats.obj
 0003:00000180       ?pGameSpyRecordFilter@@3PEBDEB 0000000039abf180     CryGameSpySBQR2Stats.obj
 0003:000001b8       ?fVec3_Zero@?$Vec3Constants@M@@2U?$Vec3_tpl@M@@B 0000000039abf1b8     StdAfx.obj
 0003:000001c8       ?fVec3_One@?$Vec3Constants@M@@2U?$Vec3_tpl@M@@B 0000000039abf1c8     StdAfx.obj
 0003:000001d8       ?fVec2_Zero@?$Vec2Constants@M@@2U?$Vec2_tpl@M@@A 0000000039abf1d8     StdAfx.obj
 0003:000001e0       ?fVec2_OneX@?$Vec2Constants@M@@2U?$Vec2_tpl@M@@A 0000000039abf1e0     StdAfx.obj
 0003:000001e8       ?fVec2_OneY@?$Vec2Constants@M@@2U?$Vec2_tpl@M@@A 0000000039abf1e8     StdAfx.obj
 0003:000001f0       ?fVec2_One@?$Vec2Constants@M@@2U?$Vec2_tpl@M@@A 0000000039abf1f0     StdAfx.obj
 0003:00000200       _fltused                   0000000039abf200     MSVCRT:dllsupp.obj
 0003:00000204       __native_dllmain_reason    0000000039abf204     MSVCRT:natstart.obj
 0003:00000208       __native_vcclrit_reason    0000000039abf208     MSVCRT:natstart.obj
 0003:00000210       __security_cookie          0000000039abf210     MSVCRT:gs_cookie.obj
 0003:00000218       __security_cookie_complement 0000000039abf218     MSVCRT:gs_cookie.obj
 0003:00000220       NNMagicData                0000000039abf220     GameSpy_2.11.00_VC10:natneg.obj
 0003:00000270       static_qr2_rec             0000000039abf270     GameSpy_2.11.00_VC10:qr2.obj
 0003:000016a0       WS_AUTHSERVICE_NAMESPACES  0000000039ac06a0     GameSpy_2.11.00_VC10:AuthService.obj
 0003:000016b0       qr2_registered_key_list    0000000039ac06b0     GameSpy_2.11.00_VC10:qr2regkeys.obj
 0003:00001ea8       GOAGetUniqueID             0000000039ac0ea8     GameSpy_2.11.00_VC10:gsPlatformUtil.obj
 0003:00001eb0       GSI_SAKE_SERVICE_NAMESPACES 0000000039ac0eb0     GameSpy_2.11.00_VC10:sakeRequest.obj
 0003:000021d8       GS_D2G_NAMESPACES          0000000039ac11d8     GameSpy_2.11.00_VC10:d2gServices.obj
 0003:00002230       GPConnectionManagerHostname 0000000039ac1230     GameSpy_2.11.00_VC10:gpiConnect.obj
 0003:00002270       GPSearchManagerHostname    0000000039ac1270     GameSpy_2.11.00_VC10:gpiSearch.obj
 0003:000023b8       GS_XML_SOAP_DEFAULT_NAMESPACES 0000000039ac13b8     GameSpy_2.11.00_VC10:gsXML.obj
 0003:000023d8       ghiThrottleBufferSize      0000000039ac13d8     GameSpy_2.11.00_VC10:ghttpCommon.obj
 0003:000023dc       ghiThrottleTimeDelay       0000000039ac13dc     GameSpy_2.11.00_VC10:ghttpCommon.obj
 0003:000023e0       GT2ChallengeKey            0000000039ac13e0     GameSpy_2.11.00_VC10:gt2Auth.obj
 0003:00002430       ?s_used_memory@?1??_usedMemory@?$CryStringT@_W@@SA_K_J@Z@4_KA 0000000039ac1430     CryDLCStore.obj
 0003:00002438       ?s_pMemReplay@?1??CryGetIMemReplay@@YAPEAUIMemReplay@@XZ@4PEAU2@EA 0000000039ac1438     CryDLCStore.obj
 0003:00002440       ?s_dummyMemReplay@?1??CryGetIMemReplay@@YAPEAUIMemReplay@@XZ@4UCDummyMemReplay@@A 0000000039ac1440     CryDLCStore.obj
 0003:00002448       ??_B?1??CryGetIMemReplay@@YAPEAUIMemReplay@@XZ@51 0000000039ac1448     CryDLCStore.obj
 0003:00002468       ?g_pObjcnt@@3PEAUSObjectCounters@@EA 0000000039ac1468     CryLobby.obj
 0003:00002470       ?m_pLobby@CCryLobby@@0PEAUICryLobby@@EA 0000000039ac1470     CryLobby.obj
 0003:00002480       ?g_time@@3VCTimeValue@@A   0000000039ac1480     CryLobby.obj
 0003:00002488       ?s_used_memory@?1??_usedMemory@?$CryStringT@D@@SA_K_J@Z@4_KA 0000000039ac1488     CryLobby.obj
 0003:00002490       ?s_used_memory@?1??_usedMemory@?$CryStackStringT@D$0IA@@@SA_K_K@Z@4_KA 0000000039ac1490     CryLobby.obj
 0003:000024a0       ?numAllocations@_CryMemoryManagerPoolHelper@@2HC 0000000039ac14a0     CryLobbyDLL.obj
 0003:000024a4       ?requestedMemory@_CryMemoryManagerPoolHelper@@2JC 0000000039ac14a4     CryLobbyDLL.obj
 0003:000024a8       ?freedMemory@_CryMemoryManagerPoolHelper@@2JC 0000000039ac14a8     CryLobbyDLL.obj
 0003:000024ac       ?allocatedMemory@_CryMemoryManagerPoolHelper@@2JC 0000000039ac14ac     CryLobbyDLL.obj
 0003:000024b0       ?gEnv@@3PEAUSSystemGlobalEnvironment@@EA 0000000039ac14b0     CryLobbyDLL.obj
 0003:000024b8       ?m_pFirst@Test@CryUnitTest@@2PEAU12@EA 0000000039ac14b8     CryLobbyDLL.obj
 0003:000024c0       ?m_pLast@Test@CryUnitTest@@2PEAU12@EA 0000000039ac14c0     CryLobbyDLL.obj
 0003:000024c8       ?g_pHeadToRegFactories@@3PEAUSRegFactoryNode@@EA 0000000039ac14c8     CryLobbyDLL.obj
 0003:000024d0       ?g_bProfilerEnabled@@3_NA  0000000039ac14d0     CryLobbyDLL.obj
 0003:000024d4       ?g_iTraceAllocations@@3HA  0000000039ac14d4     CryLobbyDLL.obj
 0003:000024d8       ?_CryMalloc@_CryMemoryManagerPoolHelper@@2P6APEAX_KAEA_K0@ZEA 0000000039ac14d8     CryLobbyDLL.obj
 0003:000024e0       ?_CryGetMemSize@_CryMemoryManagerPoolHelper@@2P6A_KPEAX_K@ZEA 0000000039ac14e0     CryLobbyDLL.obj
 0003:000024e8       ?_CryRealloc@_CryMemoryManagerPoolHelper@@2P6APEAXPEAX_KAEA_K21@ZEA 0000000039ac14e8     CryLobbyDLL.obj
 0003:000024f0       ?_CryFree@_CryMemoryManagerPoolHelper@@2P6A_KPEAX_K@ZEA 0000000039ac14f0     CryLobbyDLL.obj
 0003:000024f8       ?_CryCrtMalloc@_CryMemoryManagerPoolHelper@@2P6APEAX_K@ZEA 0000000039ac14f8     CryLobbyDLL.obj
 0003:00002500       ?_CryCrtRealloc@_CryMemoryManagerPoolHelper@@2P6APEAXPEAX_K@ZEA 0000000039ac1500     CryLobbyDLL.obj
 0003:00002508       ?_CryCrtFree@_CryMemoryManagerPoolHelper@@2P6A_KPEAX@ZEA 0000000039ac1508     CryLobbyDLL.obj
 0003:00002510       ?_CryCrtSize@_CryMemoryManagerPoolHelper@@2P6A_KPEAX@ZEA 0000000039ac1510     CryLobbyDLL.obj
 0003:00002518       ?_CryGetIMemoryManagerInterface@_CryMemoryManagerPoolHelper@@2P6AXPEAPEAX@ZEA 0000000039ac1518     CryLobbyDLL.obj
 0003:00002520       ?m_bInitialized@_CryMemoryManagerPoolHelper@@2HA 0000000039ac1520     CryLobbyDLL.obj
 0003:00002524       ?g_random_generator@@3VCLCGRndGen@@A 0000000039ac1524     CryLobbyDLL.obj
 0003:00002530       ?s_factory@CFactory@CEngineModule_CryLobby@@0V12@A 0000000039ac1530     CryLobbyDLL.obj
 0003:00002588       ?s_used_memory@?1??_usedMemory@?$CryStackStringT@D$0BAA@@@SA_K_K@Z@4_KA 0000000039ac1588     CryLobbyDLL.obj
 0003:00002590       ?supportedIIDs@?1???0CFactory@CEngineModule_CryLobby@@AEAA@XZ@4PAUCryGUID@@A 0000000039ac1590     CryLobbyDLL.obj
 0003:000025b0       ?p@?1??CreateClassInstance@CFactory@CEngineModule_CryLobby@@UEBA?AV?$shared_ptr@UICryUnknown@@@boost@@XZ@4V?$shared_ptr@VCEngineModule_CryLobby@@@5@A 0000000039ac15b0     CryLobbyDLL.obj
 0003:000025c0       ??_B?1??CreateClassInstance@CFactory@CEngineModule_CryLobby@@UEBA?AV?$shared_ptr@UICryUnknown@@@boost@@XZ@51 0000000039ac15c0     CryLobbyDLL.obj
 0003:00002620       ?s_pDetectTask@CGameSpySBQR2NATNegotiation@@0V?$_smart_ptr@USDetectTask@CGameSpySBQR2NATNegotiation@@@@A 0000000039ac1620     GameSpySBQR2NatNegotiation.obj
 0003:00002638       ?s_used_memory@?1??_usedMemory@?$CryStackStringT@D$0BAE@@@SA_K_K@Z@4_KA 0000000039ac1638     CryGameSpySBQR2DLCStore.obj
 0003:00002640       ?s_EmptyElems@?1??set_null@?$SmallDynStorage@V?$_smart_ptr@USCryDLCCategoryID@@@@HUStandardAlloc@NAlloc@@@NArray@@IEAAXXZ@4PEAV?$_smart_ptr@USCryDLCCategoryID@@@@EA 0000000039ac1640     CryGameSpySBQR2DLCStore.obj
 0003:00002648       ?s_EmptyHeader@?1??set_null@?$SmallDynStorage@V?$_smart_ptr@USCryDLCCategoryID@@@@HUStandardAlloc@NAlloc@@@NArray@@IEAAXXZ@4UEmptyHeader@23@A 0000000039ac1648     CryGameSpySBQR2DLCStore.obj
 0003:00002654       ??_B?1??set_null@?$SmallDynStorage@V?$_smart_ptr@USCryDLCCategoryID@@@@HUStandardAlloc@NAlloc@@@NArray@@IEAAXXZ@51 0000000039ac1654     CryGameSpySBQR2DLCStore.obj
 0003:00002658       ?s_EmptyElems@?1??set_null@?$SmallDynStorage@V?$_smart_ptr@USCryDLCImageID@@@@HUStandardAlloc@NAlloc@@@NArray@@IEAAXXZ@4PEAV?$_smart_ptr@USCryDLCImageID@@@@EA 0000000039ac1658     CryGameSpySBQR2DLCStore.obj
 0003:00002660       ?s_EmptyHeader@?1??set_null@?$SmallDynStorage@V?$_smart_ptr@USCryDLCImageID@@@@HUStandardAlloc@NAlloc@@@NArray@@IEAAXXZ@4UEmptyHeader@23@A 0000000039ac1660     CryGameSpySBQR2DLCStore.obj
 0003:0000266c       ??_B?1??set_null@?$SmallDynStorage@V?$_smart_ptr@USCryDLCImageID@@@@HUStandardAlloc@NAlloc@@@NArray@@IEAAXXZ@51 0000000039ac166c     CryGameSpySBQR2DLCStore.obj
 0003:00002678       ?s_used_memory@?1??_usedMemory@?$CryStackStringT@D$0CA@@@SA_K_K@Z@4_KA 0000000039ac1678     CryGameSpySBQR2Friends.obj
 0003:00002680       ?s_used_memory@?1??_usedMemory@?$CryStackStringT@D$0CI@@@SA_K_K@Z@4_KA 0000000039ac1680     CryGameSpySBQR2Friends.obj
 0003:000026a0       ?s_used_memory@?1??_usedMemory@?$CryStackStringT@D$0BF@@@SA_K_K@Z@4_KA 0000000039ac16a0     CryGameSpySBQR2Lobby.obj
 0003:000026a8       ?s_used_memory@?1??_usedMemory@?$CryStackStringT@D$0BP@@@SA_K_K@Z@4_KA 0000000039ac16a8     CryGameSpySBQR2Lobby.obj
 0003:000026b0       ?s_used_memory@?1??_usedMemory@?$CryStackStringT@D$0DD@@@SA_K_K@Z@4_KA 0000000039ac16b0     CryGameSpySBQR2Lobby.obj
 0003:000026b8       ?s_used_memory@?1??_usedMemory@?$CryStackStringT@D$0EB@@@SA_K_K@Z@4_KA 0000000039ac16b8     CryGameSpySBQR2Lobby.obj
 0003:000026c0       ?s_used_memory@?1??_usedMemory@?$CryStackStringT@D$0EA@@@SA_K_K@Z@4_KA 0000000039ac16c0     CryGameSpySBQR2Lobby.obj
 0003:000026e0       ?s_used_memory@?1??_usedMemory@?$CryStackStringT@D$0EJ@@@SA_K_K@Z@4_KA 0000000039ac16e0     CryGameSpySBQR2MatchMaking.obj
 0003:000026e8       ?s_used_memory@?1??_usedMemory@?$CryStackStringT@D$0BPP@@@SA_K_K@Z@4_KA 0000000039ac16e8     CryGameSpySBQR2MatchMaking.obj
 0003:00002710       ?s_EmptyElems@?1??set_null@?$SmallDynStorage@USUserCredential@@HUStandardAlloc@NAlloc@@@NArray@@IEAAXXZ@4PEAUSUserCredential@@EA 0000000039ac1710     CryGameSpySBQR2SignIn.obj
 0003:00002718       ?s_EmptyHeader@?1??set_null@?$SmallDynStorage@USUserCredential@@HUStandardAlloc@NAlloc@@@NArray@@IEAAXXZ@4UEmptyHeader@23@A 0000000039ac1718     CryGameSpySBQR2SignIn.obj
 0003:00002724       ??_B?1??set_null@?$SmallDynStorage@USUserCredential@@HUStandardAlloc@NAlloc@@@NArray@@IEAAXXZ@51 0000000039ac1724     CryGameSpySBQR2SignIn.obj
 0003:00002730       ?s_used_memory@?1??_usedMemory@?$CryStackStringT@D$07@@SA_K_K@Z@4_KA 0000000039ac1730     CryGameSpySBQR2Stats.obj
 0003:00002738       ?s_EmptyElems@?1??set_null@?$SmallDynStorage@USRegisterLeaderBoardDataGroup@CCryGameSpySBQR2Stats@@HUStandardAlloc@NAlloc@@@NArray@@IEAAXXZ@4PEAUSRegisterLeaderBoardDataGroup@CCryGameSpySBQR2Stats@@EA 0000000039ac1738     CryGameSpySBQR2Stats.obj
 0003:00002740       ?s_EmptyHeader@?1??set_null@?$SmallDynStorage@USRegisterLeaderBoardDataGroup@CCryGameSpySBQR2Stats@@HUStandardAlloc@NAlloc@@@NArray@@IEAAXXZ@4UEmptyHeader@23@A 0000000039ac1740     CryGameSpySBQR2Stats.obj
 0003:0000274c       ??_B?1??set_null@?$SmallDynStorage@USRegisterLeaderBoardDataGroup@CCryGameSpySBQR2Stats@@HUStandardAlloc@NAlloc@@@NArray@@IEAAXXZ@51 0000000039ac174c     CryGameSpySBQR2Stats.obj
 0003:00002750       ?s_EmptyElems@?1??set_null@?$SmallDynStorage@USRegisterUserData@CCryGameSpySBQR2Stats@@HUStandardAlloc@NAlloc@@@NArray@@IEAAXXZ@4PEAUSRegisterUserData@CCryGameSpySBQR2Stats@@EA 0000000039ac1750     CryGameSpySBQR2Stats.obj
 0003:00002758       ?s_EmptyHeader@?1??set_null@?$SmallDynStorage@USRegisterUserData@CCryGameSpySBQR2Stats@@HUStandardAlloc@NAlloc@@@NArray@@IEAAXXZ@4UEmptyHeader@23@A 0000000039ac1758     CryGameSpySBQR2Stats.obj
 0003:00002760       ??_B?1??set_null@?$SmallDynStorage@USRegisterUserData@CCryGameSpySBQR2Stats@@HUStandardAlloc@NAlloc@@@NArray@@IEAAXXZ@51 0000000039ac1760     CryGameSpySBQR2Stats.obj
 0003:000027b0       ?m_pThis@CLobbyCVars@@0PEAV1@EA 0000000039ac17b0     LobbyCVars.obj
 0003:000027e0       ?g_globalSections@?$Node_Alloc_Lock@$00$00@@2PAUInternalCriticalSectionDummy@@A 0000000039ac17e0     StdAfx.obj
 0003:00003860       ?m_bInitialized@?$Node_Alloc_Lock@$00$00@@2_NA 0000000039ac2860     StdAfx.obj
 0003:00003898       ?__type_info_root_node@@3U__type_info_node@@A 0000000039ac2898     MSVCRT:tncleanup.obj
 0003:00003ac0       g_forceGameSpyToBindToThisAddress 0000000039ac2ac0     GameSpy_2.11.00_VC10:natneg.obj
 0003:00003ac4       matchup1ip                 0000000039ac2ac4     GameSpy_2.11.00_VC10:natneg.obj
 0003:00003ac8       negotiateList              0000000039ac2ac8     GameSpy_2.11.00_VC10:natneg.obj
 0003:00003ad0       matchup2ip                 0000000039ac2ad0     GameSpy_2.11.00_VC10:natneg.obj
 0003:00003ad4       matchup3ip                 0000000039ac2ad4     GameSpy_2.11.00_VC10:natneg.obj
 0003:00003b48       __GSIACResult              0000000039ac2b48     GameSpy_2.11.00_VC10:gsAvailable.obj
 0003:00003b50       __GSIACGamename            0000000039ac2b50     GameSpy_2.11.00_VC10:gsAvailable.obj
 0003:00003b90       GSIACHostname              0000000039ac2b90     GameSpy_2.11.00_VC10:gsAvailable.obj
 0003:00005230       gcd_hostname               0000000039ac4230     GameSpy_2.11.00_VC10:gcdkeys.obj
 0003:000053b0       wsAuthServiceURL           0000000039ac43b0     GameSpy_2.11.00_VC10:AuthService.obj
 0003:00005438       g_SBRefStrList             0000000039ac4438     GameSpy_2.11.00_VC10:sb_server.obj
 0003:00005440       SBNullServer               0000000039ac4440     GameSpy_2.11.00_VC10:sb_server.obj
 0003:000057b0       sakeiSoapUrl               0000000039ac47b0     GameSpy_2.11.00_VC10:sakeRequest.obj
 0003:00005838       SBOverrideMasterServer     0000000039ac4838     GameSpy_2.11.00_VC10:sb_serverlist.obj
 0003:00015f80       __native_startup_state     0000000039ad4f80     <common>
 0003:00015f88       __native_startup_lock      0000000039ad4f88     <common>
 0003:00015f90       __dyn_tls_init_callback    0000000039ad4f90     <common>
 0003:00015f98       __onexitend                0000000039ad4f98     <common>
 0003:00015fa0       __onexitbegin              0000000039ad4fa0     <common>
 0003:00015fa8       ghiProxyPort               0000000039ad4fa8     <common>
 0003:00015fb0       ghiProxyAddress            0000000039ad4fb0     <common>
 0003:00015fb8       GVIBytesPerFrame           0000000039ad4fb8     <common>
 0003:00015fbc       GVIEncodedFrameSize        0000000039ad4fbc     <common>
 0003:00015fc0       GVIBytesPerSecond          0000000039ad4fc0     <common>
 0003:00015fc4       GVISampleRate              0000000039ad4fc4     <common>
 0003:00015fc8       GVISamplesPerFrame         0000000039ad4fc8     <common>
 0003:00015fcc       GVIGlobalMute              0000000039ad4fcc     <common>
 0003:00015fd0       gotERT1                    0000000039ad4fd0     <common>
 0003:00015fd4       gotADDRESS1b               0000000039ad4fd4     <common>
 0003:00015fd8       gotADDRESS2                0000000039ad4fd8     <common>
 0003:00015fdc       gotERT2                    0000000039ad4fdc     <common>
 0003:00015fe0       gotADDRESS1a               0000000039ad4fe0     <common>
 0003:00015fe4       gotADDRESS3                0000000039ad4fe4     <common>
 0003:00015fe8       gotERT3                    0000000039ad4fe8     <common>
 0003:00016000       qr2_hostname               0000000039ad5000     <common>
 0003:00016040       products                   0000000039ad5040     <common>
 0003:000160c0       gPTAMOTDURL                0000000039ad50c0     <common>
 0003:000168c0       Matchup1Hostname           0000000039ad58c0     <common>
 0003:000168e0       nat                        0000000039ad58e0     <common>
 0003:000169b8       Matchup2Hostname           0000000039ad59b8     <common>
 0003:000169c0       Matchup3Hostname           0000000039ad59c0     <common>
 0003:000169c8       natifyCallback             0000000039ad59c8     <common>
 0005:00000000       ?m_Self@CrySimpleThreadSelf@@1PEAV1@EA 0000000039ae3000     CryLobbyDLL.obj

 entry point at        0001:0006a548

 Static symbols

 0001:000005f0       gsiXmlUtilElementFree      0000000039a015f0 f i CryDLCStore.obj
 0001:000005f0       NatNegProgressCallback     0000000039a015f0 f i CryDLCStore.obj
 0001:000005f0       gsiXmlUtilAttributeFree    0000000039a015f0 f i CryDLCStore.obj
 0001:0006a150       pre_c_init                 0000000039a6b150 f   MSVCRT:crtdll.obj
 0001:0006a40c       __DllMainCRTStartup        0000000039a6b40c f   MSVCRT:crtdll.obj
 0001:0006a7e0       FindNegotiatorForCookie    0000000039a6b7e0 f   GameSpy_2.11.00_VC10:natneg.obj
 0001:0006a850       AddNegotiator              0000000039a6b850 f   GameSpy_2.11.00_VC10:natneg.obj
 0001:0006a8e0       RemoveNegotiator           0000000039a6b8e0 f   GameSpy_2.11.00_VC10:natneg.obj
 0001:0006a990       SendPacket                 0000000039a6b990 f   GameSpy_2.11.00_VC10:natneg.obj
 0001:0006aa10       SendReportPacket           0000000039a6ba10 f   GameSpy_2.11.00_VC10:natneg.obj
 0001:0006ab70       SendPreinitPacket          0000000039a6bb70 f   GameSpy_2.11.00_VC10:natneg.obj
 0001:0006acb0       SendInitPackets            0000000039a6bcb0 f   GameSpy_2.11.00_VC10:natneg.obj
 0001:0006aec0       SendPingPacket             0000000039a6bec0 f   GameSpy_2.11.00_VC10:natneg.obj
 0001:0006afe0       CheckNatifyStatus          0000000039a6bfe0 f   GameSpy_2.11.00_VC10:natneg.obj
 0001:0006b0e0       ResolveServers             0000000039a6c0e0 f   GameSpy_2.11.00_VC10:natneg.obj
 0001:0006b680       SendConnectAck             0000000039a6c680 f   GameSpy_2.11.00_VC10:natneg.obj
 0001:0006b750       ProcessInitPacket          0000000039a6c750 f   GameSpy_2.11.00_VC10:natneg.obj
 0001:0006b840       StartReport                0000000039a6c840 f   GameSpy_2.11.00_VC10:natneg.obj
 0001:0006b920       ProcessConnectPacket       0000000039a6c920 f   GameSpy_2.11.00_VC10:natneg.obj
 0001:0006b9f0       ProcessPingPacket          0000000039a6c9f0 f   GameSpy_2.11.00_VC10:natneg.obj
 0001:0006bcb0       NegotiateThink             0000000039a6ccb0 f   GameSpy_2.11.00_VC10:natneg.obj
 0001:0006c020       SendPacket                 0000000039a6d020 f   GameSpy_2.11.00_VC10:gsAvailable.obj
 0001:0006c4d0       gsiCoreAtExitShutdown      0000000039a6d4d0 f   GameSpy_2.11.00_VC10:gsCore.obj
 0001:0006ced0       d2giCatalogCacheFreeItem   0000000039a6ded0 f   GameSpy_2.11.00_VC10:d2gMain.obj
 0001:0006cef0       d2giExtraInfoCacheFree     0000000039a6def0 f   GameSpy_2.11.00_VC10:d2gMain.obj
 0001:0006d620       _gsi_malloc                0000000039a6e620 f   GameSpy_2.11.00_VC10:gsMemory.obj
 0001:0006d630       _gsi_free                  0000000039a6e630 f   GameSpy_2.11.00_VC10:gsMemory.obj
 0001:0006d640       _gsi_realloc               0000000039a6e640 f   GameSpy_2.11.00_VC10:gsMemory.obj
 0001:0006d650       _gsi_memalign              0000000039a6e650 f   GameSpy_2.11.00_VC10:gsMemory.obj
 0001:0006d6a0       value_for_key              0000000039a6e6a0 f   GameSpy_2.11.00_VC10:gcdkeys.obj
 0001:0006d780       free_client_node           0000000039a6e780 f   GameSpy_2.11.00_VC10:gcdkeys.obj
 0001:0006d820       init_incoming_socket       0000000039a6e820 f   GameSpy_2.11.00_VC10:gcdkeys.obj
 0001:0006d900       process_oks                0000000039a6e900 f   GameSpy_2.11.00_VC10:gcdkeys.obj
 0001:0006da70       process_ucount             0000000039a6ea70 f   GameSpy_2.11.00_VC10:gcdkeys.obj
 0001:0006dbd0       send_uon                   0000000039a6ebd0 f   GameSpy_2.11.00_VC10:gcdkeys.obj
 0001:0006dce0       send_uoff                  0000000039a6ece0 f   GameSpy_2.11.00_VC10:gcdkeys.obj
 0001:0006ddb0       process_ison               0000000039a6edb0 f   GameSpy_2.11.00_VC10:gcdkeys.obj
 0001:0006dfe0       send_disconnect_req        0000000039a6efe0 f   GameSpy_2.11.00_VC10:gcdkeys.obj
 0001:0006e0e0       send_auth_req              0000000039a6f0e0 f   GameSpy_2.11.00_VC10:gcdkeys.obj
 0001:0006e2a0       send_keep_alive            0000000039a6f2a0 f   GameSpy_2.11.00_VC10:gcdkeys.obj
 0001:0006e970       cdkey_process_buf          0000000039a6f970 f   GameSpy_2.11.00_VC10:gcdkeys.obj
 0001:0006f0b0       ListCallback               0000000039a700b0 f   GameSpy_2.11.00_VC10:sb_serverbrowsing.obj
 0001:0006f2a0       EngineCallback             0000000039a702a0 f   GameSpy_2.11.00_VC10:sb_serverbrowsing.obj
 0001:0006f700       WaitForTriggerUpdate       0000000039a70700 f   GameSpy_2.11.00_VC10:sb_serverbrowsing.obj
 0001:0006f970       gs_encode                  0000000039a70970 f   GameSpy_2.11.00_VC10:qr2.obj
 0001:0006fa60       gs_encrypt                 0000000039a70a60 f   GameSpy_2.11.00_VC10:qr2.obj
 0001:0006fbe0       NatNegCompletedCallback    0000000039a70be0 f   GameSpy_2.11.00_VC10:qr2.obj
 0001:0006fc10       compute_challenge_response 0000000039a70c10 f   GameSpy_2.11.00_VC10:qr2.obj
 0001:0006fce0       handle_public_address      0000000039a70ce0 f   GameSpy_2.11.00_VC10:qr2.obj
 0001:0006fd60       qr_build_partial_query_reply 0000000039a70d60 f   GameSpy_2.11.00_VC10:qr2.obj
 0001:00070020       qr_build_query_reply       0000000039a71020 f   GameSpy_2.11.00_VC10:qr2.obj
 0001:00070090       qr_build_split_query_reply 0000000039a71090 f   GameSpy_2.11.00_VC10:qr2.obj
 0001:00070360       qr_process_query           0000000039a71360 f   GameSpy_2.11.00_VC10:qr2.obj
 0001:00070530       qr_process_client_message  0000000039a71530 f   GameSpy_2.11.00_VC10:qr2.obj
 0001:00070670       qr2_check_ip_verify        0000000039a71670 f   GameSpy_2.11.00_VC10:qr2.obj
 0001:000706f0       send_keepalive             0000000039a716f0 f   GameSpy_2.11.00_VC10:qr2.obj
 0001:00070b70       qr2_process_ip_verify      0000000039a71b70 f   GameSpy_2.11.00_VC10:qr2.obj
 0001:00071070       send_heartbeat             0000000039a72070 f   GameSpy_2.11.00_VC10:qr2.obj
 0001:00071750       qr2_check_queries          0000000039a72750 f   GameSpy_2.11.00_VC10:qr2.obj
 0001:00071820       qr2_check_send_heartbeat   0000000039a72820 f   GameSpy_2.11.00_VC10:qr2.obj
 0001:00073100       wsiLoginEncryptPassword    0000000039a74100 f   GameSpy_2.11.00_VC10:AuthService.obj
 0001:000737e0       wsLoginUniqueCallback      0000000039a747e0 f   GameSpy_2.11.00_VC10:AuthService.obj
 0001:00073c70       RefStringCompare           0000000039a74c70 f   GameSpy_2.11.00_VC10:sb_server.obj
 0001:00073c80       RefStringFree              0000000039a74c80 f   GameSpy_2.11.00_VC10:sb_server.obj
 0001:000745e0       KeyValFree                 0000000039a755e0 f   GameSpy_2.11.00_VC10:sb_server.obj
 0001:00074610       KeyValCompareKey           0000000039a75610 f   GameSpy_2.11.00_VC10:sb_server.obj
 0001:00074740       KeyValHashKey              0000000039a75740 f   GameSpy_2.11.00_VC10:sb_server.obj
 0001:00074740       RefStringHash              0000000039a75740 f   GameSpy_2.11.00_VC10:sb_server.obj
 0001:00074dd0       TripToQuart                0000000039a75dd0 f   GameSpy_2.11.00_VC10:gsPlatformUtil.obj
 0001:000753e0       GenerateID                 0000000039a763e0 f   GameSpy_2.11.00_VC10:gsPlatformUtil.obj
 0001:00075aa0       mylsearch                  0000000039a76aa0 f   GameSpy_2.11.00_VC10:darray.obj
 0001:00075b30       mybsearch                  0000000039a76b30 f   GameSpy_2.11.00_VC10:darray.obj
 0001:00076440       GetLocalIP                 0000000039a77440 f   GameSpy_2.11.00_VC10:NATify.obj
 0001:00076440       GetLocalIP                 0000000039a77440 f   GameSpy_2.11.00_VC10:NATify.obj
 0001:000766a0       Think                      0000000039a776a0 f   GameSpy_2.11.00_VC10:NATify.obj
 0001:00077090       ghiHandleStatus            0000000039a78090 f   GameSpy_2.11.00_VC10:ghttpMain.obj
 0001:00077100       ghiProcessConnection       0000000039a78100 f   GameSpy_2.11.00_VC10:ghttpMain.obj
 0001:000774f0       _ghttpSaveEx               0000000039a784f0 f   GameSpy_2.11.00_VC10:ghttpMain.obj
 0001:00077a20       sakeiCheckSakeResult       0000000039a78a20 f   GameSpy_2.11.00_VC10:sakeRequest.obj
 0001:00077cb0       sakeiSoapCallback          0000000039a78cb0 f   GameSpy_2.11.00_VC10:sakeRequest.obj
 0001:00077e20       sakeiSetupRequest          0000000039a78e20 f   GameSpy_2.11.00_VC10:sakeRequest.obj
 0001:00077fd0       sakeiValidateRequestFields 0000000039a78fd0 f   GameSpy_2.11.00_VC10:sakeRequestModify.obj
 0001:00078050       sakeiFillSoapRequestFieldValues 0000000039a79050 f   GameSpy_2.11.00_VC10:sakeRequestModify.obj
 0001:00078410       sakeiCreateRecordValidateInput 0000000039a79410 f   GameSpy_2.11.00_VC10:sakeRequestModify.obj
 0001:00078450       sakeiCreateRecordFillSoapRequest 0000000039a79450 f   GameSpy_2.11.00_VC10:sakeRequestModify.obj
 0001:000784a0       sakeiCreateRecordProcessSoapResponse 0000000039a794a0 f   GameSpy_2.11.00_VC10:sakeRequestModify.obj
 0001:000784e0       sakeiUpdateRecordValidateInput 0000000039a794e0 f   GameSpy_2.11.00_VC10:sakeRequestModify.obj
 0001:00078510       sakeiUpdateRecordFillSoapRequest 0000000039a79510 f   GameSpy_2.11.00_VC10:sakeRequestModify.obj
 0001:00078590       sakeiDeleteRecordFillSoapRequest 0000000039a79590 f   GameSpy_2.11.00_VC10:sakeRequestModify.obj
 0001:000785f0       sakeiFillSoapRequestFieldNames 0000000039a795f0 f   GameSpy_2.11.00_VC10:sakeRequestRead.obj
 0001:00078680       sakeiFillSoapRequestRecordIds 0000000039a79680 f   GameSpy_2.11.00_VC10:sakeRequestRead.obj
 0001:00078710       sakeiFillSoapRequestOwnerIds 0000000039a79710 f   GameSpy_2.11.00_VC10:sakeRequestRead.obj
 0001:000787a0       sakeiReadOutputRecords     0000000039a797a0 f   GameSpy_2.11.00_VC10:sakeRequestRead.obj
 0001:00078ce0       sakeiFreeOutputRecords     0000000039a79ce0 f   GameSpy_2.11.00_VC10:sakeRequestRead.obj
 0001:00078db0       sakeiSearchForRecordsValidateInput 0000000039a79db0 f   GameSpy_2.11.00_VC10:sakeRequestRead.obj
 0001:00078e30       sakeiSearchForRecordsFillSoapRequest 0000000039a79e30 f   GameSpy_2.11.00_VC10:sakeRequestRead.obj
 0001:00078f60       sakeiSearchForRecordsFreeData 0000000039a79f60 f   GameSpy_2.11.00_VC10:sakeRequestRead.obj
 0001:00078f60       sakeiGetMyRecordsFreeData  0000000039a79f60 f   GameSpy_2.11.00_VC10:sakeRequestRead.obj
 0001:00078fa0       sakeiGetMyRecordsFillSoapRequest 0000000039a79fa0 f   GameSpy_2.11.00_VC10:sakeRequestRead.obj
 0001:00078ff0       sakeiSearchForRecordsProcessSoapResponse 0000000039a79ff0 f   GameSpy_2.11.00_VC10:sakeRequestRead.obj
 0001:00078ff0       sakeiGetMyRecordsProcessSoapResponse 0000000039a79ff0 f   GameSpy_2.11.00_VC10:sakeRequestRead.obj
 0001:00079030       sakeiGetSpecificRecordsValidateInput 0000000039a7a030 f   GameSpy_2.11.00_VC10:sakeRequestRead.obj
 0001:000790b0       sakeiGetSpecificRecordsFillSoapRequest 0000000039a7a0b0 f   GameSpy_2.11.00_VC10:sakeRequestRead.obj
 0001:00079110       sakeiGetSpecificRecordsProcessSoapResponse 0000000039a7a110 f   GameSpy_2.11.00_VC10:sakeRequestRead.obj
 0001:00079140       sakeiGetSpecificRecordsFreeData 0000000039a7a140 f   GameSpy_2.11.00_VC10:sakeRequestRead.obj
 0001:00079170       sakeiGetMyRecordsValidateInput 0000000039a7a170 f   GameSpy_2.11.00_VC10:sakeRequestRead.obj
 0001:00079170       sakeiGetRandomRecordValidateInput 0000000039a7a170 f   GameSpy_2.11.00_VC10:sakeRequestRead.obj
 0001:000791e0       sakeiGetRandomRecordFillSoapRequest 0000000039a7a1e0 f   GameSpy_2.11.00_VC10:sakeRequestRead.obj
 0001:00079270       sakeiGetRandomRecordProcessSoapResponse 0000000039a7a270 f   GameSpy_2.11.00_VC10:sakeRequestRead.obj
 0001:000792e0       sakeiGetRandomRecordFreeData 0000000039a7a2e0 f   GameSpy_2.11.00_VC10:sakeRequestRead.obj
 0001:00079360       sakeiRateRecordFillSoapRequest 0000000039a7a360 f   GameSpy_2.11.00_VC10:sakeRequestMisc.obj
 0001:000793d0       sakeiRateRecordProcessSoapResponse 0000000039a7a3d0 f   GameSpy_2.11.00_VC10:sakeRequestMisc.obj
 0001:00079430       sakeiGetRecordLimitFillSoapRequest 0000000039a7a430 f   GameSpy_2.11.00_VC10:sakeRequestMisc.obj
 0001:00079460       sakeiGetRecordLimitProcessSoapResponse 0000000039a7a460 f   GameSpy_2.11.00_VC10:sakeRequestMisc.obj
 0001:000794c0       sakeiDeleteRecordValidateInput 0000000039a7a4c0 f   GameSpy_2.11.00_VC10:sakeRequestMisc.obj
 0001:000794c0       sakeiGetRecordLimitValidateInput 0000000039a7a4c0 f   GameSpy_2.11.00_VC10:sakeRequestMisc.obj
 0001:000794c0       sakeiRateRecordValidateInput 0000000039a7a4c0 f   GameSpy_2.11.00_VC10:sakeRequestMisc.obj
 0001:000794c0       sakeiGetRecordCountValidateInput 0000000039a7a4c0 f   GameSpy_2.11.00_VC10:sakeRequestMisc.obj
 0001:000794e0       sakeiGetRecordCountFillSoapRequest 0000000039a7a4e0 f   GameSpy_2.11.00_VC10:sakeRequestMisc.obj
 0001:00079560       sakeiGetRecordCountProcessSoapResponse 0000000039a7a560 f   GameSpy_2.11.00_VC10:sakeRequestMisc.obj
 0001:0007b2e0       d2giGetStoreAvailCallback  0000000039a7c2e0 f   GameSpy_2.11.00_VC10:d2gServices.obj
 0001:0007b540       d2giServiceLoadCatalogItemsCallback 0000000039a7c540 f   GameSpy_2.11.00_VC10:d2gServices.obj
 0001:0007b7b0       d2giServiceGetUserCreditCardsCallback 0000000039a7c7b0 f   GameSpy_2.11.00_VC10:d2gServices.obj
 0001:0007ba80       d2giGetOrderTotalCallback  0000000039a7ca80 f   GameSpy_2.11.00_VC10:d2gServices.obj
 0001:0007c280       d2giServiceDownloadFileByIdCallback 0000000039a7d280 f   GameSpy_2.11.00_VC10:d2gServices.obj
 0001:0007c6c0       d2giServiceGetPurchaseHistoryCallback 0000000039a7d6c0 f   GameSpy_2.11.00_VC10:d2gServices.obj
 0001:0007caa0       GSMD5Transform             0000000039a7daa0 f   GameSpy_2.11.00_VC10:md5c.obj
 0001:0007d580       FIFORemove                 0000000039a7e580 f   GameSpy_2.11.00_VC10:sb_queryengine.obj
 0001:0007d5e0       QEStartQuery               0000000039a7e5e0 f   GameSpy_2.11.00_VC10:sb_queryengine.obj
 0001:0007da20       ParseSingleQR2Reply        0000000039a7ea20 f   GameSpy_2.11.00_VC10:sb_queryengine.obj
 0001:0007dbf0       ParseSingleGOAReply        0000000039a7ebf0 f   GameSpy_2.11.00_VC10:sb_queryengine.obj
 0001:0007dce0       TimeoutOldQueries          0000000039a7ece0 f   GameSpy_2.11.00_VC10:sb_queryengine.obj
 0001:0007e430       ServerListConnect          0000000039a7f430 f   GameSpy_2.11.00_VC10:sb_serverlist.obj
 0001:0007e5e0       SetupListChallenge         0000000039a7f5e0 f   GameSpy_2.11.00_VC10:sb_serverlist.obj
 0001:0007e6d0       FreePopularValues          0000000039a7f6d0 f   GameSpy_2.11.00_VC10:sb_serverlist.obj
 0001:0007e780       FreeKeyList                0000000039a7f780 f   GameSpy_2.11.00_VC10:sb_serverlist.obj
 0001:0007e890       InitCryptKey               0000000039a7f890 f   GameSpy_2.11.00_VC10:sb_serverlist.obj
 0001:0007e940       FullRulesPresent           0000000039a7f940 f   GameSpy_2.11.00_VC10:sb_serverlist.obj
 0001:0007e9d0       AllKeysPresent             0000000039a7f9d0 f   GameSpy_2.11.00_VC10:sb_serverlist.obj
 0001:0007eaa0       ParseServer                0000000039a7faa0 f   GameSpy_2.11.00_VC10:sb_serverlist.obj
 0001:0007ecf0       IncomingListParseServer    0000000039a7fcf0 f   GameSpy_2.11.00_VC10:sb_serverlist.obj
 0001:0007ee30       ProcessMainListData        0000000039a7fe30 f   GameSpy_2.11.00_VC10:sb_serverlist.obj
 0001:0007f2b0       ProcessPushKeyList         0000000039a802b0 f   GameSpy_2.11.00_VC10:sb_serverlist.obj
 0001:0007f3a0       ProcessPlayerSearch        0000000039a803a0 f   GameSpy_2.11.00_VC10:sb_serverlist.obj
 0001:0007f540       ProcessMaploop             0000000039a80540 f   GameSpy_2.11.00_VC10:sb_serverlist.obj
 0001:0007f660       ProcessPushServer          0000000039a80660 f   GameSpy_2.11.00_VC10:sb_serverlist.obj
 0001:0007f790       ProcessLanData             0000000039a80790 f   GameSpy_2.11.00_VC10:sb_serverlist.obj
 0001:0007fab0       ErrorDisconnect            0000000039a80ab0 f   GameSpy_2.11.00_VC10:sb_serverlist.obj
 0001:0007fe50       ProcessAdHocData           0000000039a80e50 f   GameSpy_2.11.00_VC10:sb_serverlist.obj
 0001:00080000       ProcessIncomingData        0000000039a81000 f   GameSpy_2.11.00_VC10:sb_serverlist.obj
 0001:00080190       SendWithRetry              0000000039a81190 f   GameSpy_2.11.00_VC10:sb_serverlist.obj
 0001:000804c0       gpiResetProfile            0000000039a814c0 f   GameSpy_2.11.00_VC10:gpi.obj
 0001:000815c0       randomString               0000000039a825c0 f   GameSpy_2.11.00_VC10:gpiConnect.obj
 0001:00081670       gpiStartConnect            0000000039a82670 f   GameSpy_2.11.00_VC10:gpiConnect.obj
 0001:00081980       gpiSendLogin               0000000039a82980 f   GameSpy_2.11.00_VC10:gpiConnect.obj
 0001:00081e80       gpiSendNewuser             0000000039a82e80 f   GameSpy_2.11.00_VC10:gpiConnect.obj
 0001:00082740       gpiDisconnectCleanupProfile 0000000039a83740 f   GameSpy_2.11.00_VC10:gpiConnect.obj
 0001:00082e10       gpiStartProfileSearch      0000000039a83e10 f   GameSpy_2.11.00_VC10:gpiSearch.obj
 0001:00082fc0       gpiInitSearchData          0000000039a83fc0 f   GameSpy_2.11.00_VC10:gpiSearch.obj
 0001:00083070       gpiStartSearch             0000000039a84070 f   GameSpy_2.11.00_VC10:gpiSearch.obj
 0001:00083740       gpiProcessSearch           0000000039a84740 f   GameSpy_2.11.00_VC10:gpiSearch.obj
 0001:00085730       gpiSendRegisterUniqueNick  0000000039a86730 f   GameSpy_2.11.00_VC10:gpiUnique.obj
 0001:00085b60       gpiProfilesTableHash       0000000039a86b60 f   GameSpy_2.11.00_VC10:gpiProfile.obj
 0001:00085b70       gpiProfilesTableCompare    0000000039a86b70 f   GameSpy_2.11.00_VC10:gpiProfile.obj
 0001:00085b80       gpiProfilesTableFree       0000000039a86b80 f   GameSpy_2.11.00_VC10:gpiProfile.obj
 0001:000861f0       gpiCheckProfileForUser     0000000039a871f0 f   GameSpy_2.11.00_VC10:gpiProfile.obj
 0001:00086280       gpiProfileMapCallback      0000000039a87280 f   GameSpy_2.11.00_VC10:gpiProfile.obj
 0001:000862e0       gpiCheckForBuddy           0000000039a872e0 f   GameSpy_2.11.00_VC10:gpiProfile.obj
 0001:00086460       gpiFixBlockIndices         0000000039a87460 f   GameSpy_2.11.00_VC10:gpiProfile.obj
 0001:00086bb0       gpiIsValidDate             0000000039a87bb0 f   GameSpy_2.11.00_VC10:gpiInfo.obj
 0001:00089f90       gpiProcessPeerAcceptingConnection 0000000039a8af90 f   GameSpy_2.11.00_VC10:gpiPeer.obj
 0001:0008a290       gpiProcessPeerConnected    0000000039a8b290 f   GameSpy_2.11.00_VC10:gpiPeer.obj
 0001:0008a810       gpiFreeMessage             0000000039a8b810 f   GameSpy_2.11.00_VC10:gpiPeer.obj
 0001:0008afe0       gpiProcessPeerInitiatingConnection 0000000039a8bfe0 f   GameSpy_2.11.00_VC10:gpiPeer.obj
 0001:0008bd70       gsiXmlUtilSkipWhiteSpace   0000000039a8cd70 f   GameSpy_2.11.00_VC10:gsXML.obj
 0001:0008bde0       gsiXmlUtilParseName        0000000039a8cde0 f   GameSpy_2.11.00_VC10:gsXML.obj
 0001:0008bf00       gsiXmlUtilDecodeString     0000000039a8cf00 f   GameSpy_2.11.00_VC10:gsXML.obj
 0001:0008c240       gsiXmlUtilTagMatches       0000000039a8d240 f   GameSpy_2.11.00_VC10:gsXML.obj
 0001:0008c510       gsiXmlUtilParseString      0000000039a8d510 f   GameSpy_2.11.00_VC10:gsXML.obj
 0001:0008c600       gsiXmlUtilWriteChar        0000000039a8d600 f   GameSpy_2.11.00_VC10:gsXML.obj
 0001:0008c680       gsiXmlUtilWriteString      0000000039a8d680 f   GameSpy_2.11.00_VC10:gsXML.obj
 0001:0008c730       gsiXmlUtilWriteXmlSafeString 0000000039a8d730 f   GameSpy_2.11.00_VC10:gsXML.obj
 0001:0008dc40       gsiXmlUtilParseElement     0000000039a8ec40 f   GameSpy_2.11.00_VC10:gsXML.obj
 0001:0008ec20       gsiXmlUtilWriteUnicodeString 0000000039a8fc20 f   GameSpy_2.11.00_VC10:gsXML.obj
 0001:0008ef10       gsiSoapTaskHttpCompletedCallback 0000000039a8ff10 f   GameSpy_2.11.00_VC10:gsSoap.obj
 0001:0008ef90       gsiSoapTaskThink           0000000039a8ff90 f   GameSpy_2.11.00_VC10:gsSoap.obj
 0001:0008efc0       gsiSoapTaskExecute         0000000039a8ffc0 f   GameSpy_2.11.00_VC10:gsSoap.obj
 0001:0008f060       gsiSoapTaskCancel          0000000039a90060 f   GameSpy_2.11.00_VC10:gsSoap.obj
 0001:0008f090       gsiSoapTaskCallback        0000000039a90090 f   GameSpy_2.11.00_VC10:gsSoap.obj
 0001:0008f0b0       gsiSoapTaskCleanup         0000000039a900b0 f   GameSpy_2.11.00_VC10:gsSoap.obj
 0001:0008f210       gsCryptRSAPKCS1EncryptBuffer 0000000039a90210 f   GameSpy_2.11.00_VC10:gsCrypt.obj
 0001:0008f5a0       gsiLargeIntTimerExit       0000000039a905a0 f   GameSpy_2.11.00_VC10:gsLargeInt.obj
 0001:0008f5e0       gsiLargeIntCompare         0000000039a905e0 f   GameSpy_2.11.00_VC10:gsLargeInt.obj
 0001:0008f680       gsiLargeIntSub             0000000039a90680 f   GameSpy_2.11.00_VC10:gsLargeInt.obj
 0001:0008f800       gsiLargeIntMult            0000000039a90800 f   GameSpy_2.11.00_VC10:gsLargeInt.obj
 0001:0008fa20       gsiLargeIntSubDivide       0000000039a90a20 f   GameSpy_2.11.00_VC10:gsLargeInt.obj
 0001:00090140       gsiLargeIntDiv             0000000039a91140 f   GameSpy_2.11.00_VC10:gsLargeInt.obj
 0001:00091210       gviFreeArrayDevice         0000000039a92210 f   GameSpy_2.11.00_VC10:gvDirectSound.obj
 0001:00091670       gviEnumDevicesCallback     0000000039a92670 f   GameSpy_2.11.00_VC10:gvDirectSound.obj
 0001:000918c0       gviHardwareFreeDevice      0000000039a928c0 f   GameSpy_2.11.00_VC10:gvDirectSound.obj
 0001:000918d0       gviStartPlaybackDevice     0000000039a928d0 f   GameSpy_2.11.00_VC10:gvDirectSound.obj
 0001:000919b0       gviHardwareStartDevice     0000000039a929b0 f   GameSpy_2.11.00_VC10:gvDirectSound.obj
 0001:000919e0       gviHardwareStopDevice      0000000039a929e0 f   GameSpy_2.11.00_VC10:gvDirectSound.obj
 0001:00091a30       gviHardwareIsDeviceStarted 0000000039a92a30 f   GameSpy_2.11.00_VC10:gvDirectSound.obj
 0001:00091a70       gviHardwareSetDeviceVolume 0000000039a92a70 f   GameSpy_2.11.00_VC10:gvDirectSound.obj
 0001:00091ae0       gviHardwareGetDeviceVolume 0000000039a92ae0 f   GameSpy_2.11.00_VC10:gvDirectSound.obj
 0001:00091b40       gviHardwareSetCaptureThreshold 0000000039a92b40 f   GameSpy_2.11.00_VC10:gvDirectSound.obj
 0001:00091b50       gviHardwareGetCaptureThreshold 0000000039a92b50 f   GameSpy_2.11.00_VC10:gvDirectSound.obj
 0001:00091b60       gviHardwareGetAvailableCaptureBytes 0000000039a92b60 f   GameSpy_2.11.00_VC10:gvDirectSound.obj
 0001:00091bd0       gviHardwareCapturePacket   0000000039a92bd0 f   GameSpy_2.11.00_VC10:gvDirectSound.obj
 0001:00091f30       gviHardwarePlayPacket      0000000039a92f30 f   GameSpy_2.11.00_VC10:gvDirectSound.obj
 0001:00091f70       gviHardwareIsSourceTalking 0000000039a92f70 f   GameSpy_2.11.00_VC10:gvDirectSound.obj
 0001:00091f90       gviHardwareListTalkingSources 0000000039a92f90 f   GameSpy_2.11.00_VC10:gvDirectSound.obj
 0001:00091fb0       gviInitPlaybackDevice      0000000039a92fb0 f   GameSpy_2.11.00_VC10:gvDirectSound.obj
 0001:00092090       gviInitCaptureDevice       0000000039a93090 f   GameSpy_2.11.00_VC10:gvDirectSound.obj
 0001:000924c0       gviAddSourceToList         0000000039a934c0 f   GameSpy_2.11.00_VC10:gvSource.obj
 0001:000925a0       gviAddPacketToSource       0000000039a935a0 f   GameSpy_2.11.00_VC10:gvSource.obj
 0001:00092c40       ghiFindFreeSlot            0000000039a93c40 f   GameSpy_2.11.00_VC10:ghttpConnection.obj
 0001:00093440       ghiParseURL                0000000039a94440 f   GameSpy_2.11.00_VC10:ghttpProcess.obj
 0001:00093f40       ghiParseStatus             0000000039a94f40 f   GameSpy_2.11.00_VC10:ghttpProcess.obj
 0001:000941d0       ghiDeliverIncomingFileData 0000000039a951d0 f   GameSpy_2.11.00_VC10:ghttpProcess.obj
 0001:000942b0       ghiAppendToChunkHeaderBuffer 0000000039a952b0 f   GameSpy_2.11.00_VC10:ghttpProcess.obj
 0001:00094320       ghiProcessIncomingFileData 0000000039a95320 f   GameSpy_2.11.00_VC10:ghttpProcess.obj
 0001:00095170       ghiPostDataFree            0000000039a96170 f   GameSpy_2.11.00_VC10:ghttpPost.obj
 0001:00095330       ghiPostGetNoFilesContentLength 0000000039a96330 f   GameSpy_2.11.00_VC10:ghttpPost.obj
 0001:000953f0       ghiPostGetHasFilesContentLength 0000000039a963f0 f   GameSpy_2.11.00_VC10:ghttpPost.obj
 0001:00095980       ghiPostStringStateDoPosting 0000000039a96980 f   GameSpy_2.11.00_VC10:ghttpPost.obj
 0001:00095b40       ghiPostXmlStateDoPosting   0000000039a96b40 f   GameSpy_2.11.00_VC10:ghttpPost.obj
 0001:00095ca0       ghiPostFileDiskStateDoPosting 0000000039a96ca0 f   GameSpy_2.11.00_VC10:ghttpPost.obj
 0001:00095dc0       ghiPostFileMemoryStateDoPosting 0000000039a96dc0 f   GameSpy_2.11.00_VC10:ghttpPost.obj
 0001:00095f80       ghiPostStateDoPosting      0000000039a96f80 f   GameSpy_2.11.00_VC10:ghttpPost.obj
 0001:0009a6f0       gpiCallCallback            0000000039a9b6f0 f   GameSpy_2.11.00_VC10:gpiCallback.obj
 0001:0009c3e0       ghiEncryptorParseASN1Sequence 0000000039a9d3e0 f   GameSpy_2.11.00_VC10:ghttpEncryption.obj
 0001:0009c4c0       ghiEncryptorGenerateEncryptionKeys 0000000039a9d4c0 f   GameSpy_2.11.00_VC10:ghttpEncryption.obj
 0001:0009cf80       ghiEncryptorProcessSSLHandshake 0000000039a9df80 f   GameSpy_2.11.00_VC10:ghttpEncryption.obj
 0001:0009e500       gti2CloseAllConnectionsHardMap 0000000039a9f500 f   GameSpy_2.11.00_VC10:gt2Main.obj
 0001:0009ee50       gti2ConnectionHash         0000000039a9fe50 f   GameSpy_2.11.00_VC10:gt2Socket.obj
 0001:0009ee70       gti2ConnectionCompare      0000000039a9fe70 f   GameSpy_2.11.00_VC10:gt2Socket.obj
 0001:0009ee90       gti2ConnectionFree         0000000039a9fe90 f   GameSpy_2.11.00_VC10:gt2Socket.obj
 0001:0009f490       gti2SocketConnectionsThinkMap 0000000039aa0490 f   GameSpy_2.11.00_VC10:gt2Socket.obj
 0001:0009f7e0       gti2ConnectionError        0000000039aa07e0 f   GameSpy_2.11.00_VC10:gt2Message.obj
 0001:0009f880       gti2HandleESN              0000000039aa0880 f   GameSpy_2.11.00_VC10:gt2Message.obj
 0001:0009f980       gti2HandleAppUnreliable    0000000039aa0980 f   GameSpy_2.11.00_VC10:gt2Message.obj
 0001:0009fa20       gti2HandleAppReliable      0000000039aa0a20 f   GameSpy_2.11.00_VC10:gt2Message.obj
 0001:0009faf0       gti2IncomingBufferMessageCompare 0000000039aa0af0 f   GameSpy_2.11.00_VC10:gt2Message.obj
 0001:0009fb00       gti2RemoveHoldMessage      0000000039aa0b00 f   GameSpy_2.11.00_VC10:gt2Message.obj
 0001:0009fd10       gti2StoreOutgoingReliableMessageInfo 0000000039aa0d10 f   GameSpy_2.11.00_VC10:gt2Message.obj
 0001:0009fdb0       gti2EndReliableMessage     0000000039aa0db0 f   GameSpy_2.11.00_VC10:gt2Message.obj
 0001:000a01c0       gti2BufferIncomingMessage  0000000039aa11c0 f   GameSpy_2.11.00_VC10:gt2Message.obj
 0001:000a0340       gti2HandleNack             0000000039aa1340 f   GameSpy_2.11.00_VC10:gt2Message.obj
 0001:000a0430       gti2HandleUnreliableMessage 0000000039aa1430 f   GameSpy_2.11.00_VC10:gt2Message.obj
 0001:000a0580       gti2ConnectionMemoryError  0000000039aa1580 f   GameSpy_2.11.00_VC10:gt2Message.obj
 0001:000a05c0       gti2HandleClientResponse   0000000039aa15c0 f   GameSpy_2.11.00_VC10:gt2Message.obj
 0001:000a06c0       gti2HandleReject           0000000039aa16c0 f   GameSpy_2.11.00_VC10:gt2Message.obj
 0001:000a0750       gti2BeginReliableMessage   0000000039aa1750 f   GameSpy_2.11.00_VC10:gt2Message.obj
 0001:000a0c00       gti2HandleClientChallenge  0000000039aa1c00 f   GameSpy_2.11.00_VC10:gt2Message.obj
 0001:000a0d20       gti2HandleServerChallenge  0000000039aa1d20 f   GameSpy_2.11.00_VC10:gt2Message.obj
 0001:000a0df0       gti2DeliverReliableMessage 0000000039aa1df0 f   GameSpy_2.11.00_VC10:gt2Message.obj
 0001:000a0f20       gti2DeliverHoldMessages    0000000039aa1f20 f   GameSpy_2.11.00_VC10:gt2Message.obj
 0001:000a0fc0       gti2HandleReliableMessage  0000000039aa1fc0 f   GameSpy_2.11.00_VC10:gt2Message.obj
 0001:000a1170       gti2HandleMessage          0000000039aa2170 f   GameSpy_2.11.00_VC10:gt2Message.obj
 0001:000a1740       gti2SendRetries            0000000039aa2740 f   GameSpy_2.11.00_VC10:gt2Connection.obj
 0001:000a18a0       gti2CheckTimeout           0000000039aa28a0 f   GameSpy_2.11.00_VC10:gt2Connection.obj
 0001:000a2610       _onexit$fin$0              0000000039aa3610 f   MSVCRT:atonexit.obj
 0001:000a262b       __DllMainCRTStartup$filt$0 0000000039aa362b f   MSVCRT:crtdll.obj
 0001:000a265b       __DllMainCRTStartup$fin$1  0000000039aa365b f   MSVCRT:crtdll.obj
 0001:000a2680       _IsNonwritableInCurrentImage$filt$0 0000000039aa3680 f   MSVCRT:pesect.obj
 0001:000a26b0       ??__ECryUserInvalidID@@YAXXZ 0000000039aa36b0 f   CryDedicatedServer.obj
 0001:000a26c0       ??__ECryUserInvalidID@@YAXXZ 0000000039aa36c0 f   CryDedicatedServerArbitrator.obj
 0001:000a26d0       ??__ECryUserInvalidID@@YAXXZ 0000000039aa36d0 f   CryFriends.obj
 0001:000a26e0       ??__ECryUserInvalidID@@YAXXZ 0000000039aa36e0 f   CryFriendsManagement.obj
 0001:000a26f0       ??__ECryUserInvalidID@@YAXXZ 0000000039aa36f0 f   CryHostMigration.obj
 0001:000a2700       ??__ECryUserInvalidID@@YAXXZ 0000000039aa3700 f   CryLobby.obj
 0001:000a2710       ??__Eg_time@@YAXXZ         0000000039aa3710 f   CryLobby.obj
 0001:000a2720       ??__Eg_random_generator@@YAXXZ 0000000039aa3720 f   CryLobbyDLL.obj
 0001:000a2730       ??__Eg_system_event_listener_crylobby@@YAXXZ 0000000039aa3730 f   CryLobbyDLL.obj
 0001:000a2740       ??__E?s_factory@CFactory@CEngineModule_CryLobby@@0V12@A@@YAXXZ 0000000039aa3740 f   CryLobbyDLL.obj
 0001:000a2760       ??__ECryUserInvalidID@@YAXXZ 0000000039aa3760 f   CryLobbyUI.obj
 0001:000a2770       ??__ECryUserInvalidID@@YAXXZ 0000000039aa3770 f   CryMatchMaking.obj
 0001:000a2780       ??__ECrySessionInvalidID@@YAXXZ 0000000039aa3780 f   CryMatchMaking.obj
 0001:000a2790       ??__ECryUserInvalidID@@YAXXZ 0000000039aa3790 f   CryRebroadcaster.obj
 0001:000a27a0       ??__ECryUserInvalidID@@YAXXZ 0000000039aa37a0 f   CryStats.obj
 0001:000a27b0       ??__ECryUserInvalidID@@YAXXZ 0000000039aa37b0 f   CryVoice.obj
 0001:000a27c0       ??__ECryUserInvalidID@@YAXXZ 0000000039aa37c0 f   GameSpySBQR2AvailabilityCheck.obj
 0001:000a27d0       ??__ECryUserInvalidID@@YAXXZ 0000000039aa37d0 f   GameSpySBQR2Core.obj
 0001:000a27e0       ??__ECryUserInvalidID@@YAXXZ 0000000039aa37e0 f   GameSpySBQR2NatNegotiation.obj
 0001:000a27f0       ??__E?s_pDetectTask@CGameSpySBQR2NATNegotiation@@0V?$_smart_ptr@USDetectTask@CGameSpySBQR2NATNegotiation@@@@A@@YAXXZ 0000000039aa37f0 f   GameSpySBQR2NatNegotiation.obj
 0001:000a2800       ??__ECryUserInvalidID@@YAXXZ 0000000039aa3800 f   GameSpySBQR2Sake.obj
 0001:000a2810       ??__ECryUserInvalidID@@YAXXZ 0000000039aa3810 f   GameSpySDK.obj
 0001:000a2820       ??__ECryUserInvalidID@@YAXXZ 0000000039aa3820 f   CryGameSpySBQR2DLCStore.obj
 0001:000a2830       ??__ECryUserInvalidID@@YAXXZ 0000000039aa3830 f   CryGameSpySBQR2Friends.obj
 0001:000a2840       ??__ECrySessionInvalidID@@YAXXZ 0000000039aa3840 f   CryGameSpySBQR2Friends.obj
 0001:000a2850       ??__ECryUserInvalidID@@YAXXZ 0000000039aa3850 f   CryGameSpySBQR2FriendsManagement.obj
 0001:000a2860       ??__ECryUserInvalidID@@YAXXZ 0000000039aa3860 f   CryGameSpySBQR2Lobby.obj
 0001:000a2870       ??__ECryUserInvalidID@@YAXXZ 0000000039aa3870 f   CryGameSpySBQR2LobbyUI.obj
 0001:000a2880       ??__ECrySessionInvalidID@@YAXXZ 0000000039aa3880 f   CryGameSpySBQR2LobbyUI.obj
 0001:000a2890       ??__ECryUserInvalidID@@YAXXZ 0000000039aa3890 f   CryGameSpySBQR2MatchMaking.obj
 0001:000a28a0       ??__ECrySessionInvalidID@@YAXXZ 0000000039aa38a0 f   CryGameSpySBQR2MatchMaking.obj
 0001:000a28b0       ??__ECryUserInvalidID@@YAXXZ 0000000039aa38b0 f   CryGameSpySBQR2SignIn.obj
 0001:000a28c0       ??__ECryUserInvalidID@@YAXXZ 0000000039aa38c0 f   CryGameSpySBQR2Stats.obj
 0001:000a28d0       ??__ECryUserInvalidID@@YAXXZ 0000000039aa38d0 f   CryGameSpySBQR2Voice.obj
 0001:000a28e0       ??__ECryUserInvalidID@@YAXXZ 0000000039aa38e0 f   GameSpySBQR2GPConnection.obj
 0001:000a28f0       ??__ECryUserInvalidID@@YAXXZ 0000000039aa38f0 f   CryGameSpyMatchMaking.obj
 0001:000a2900       ??__ECryUserInvalidID@@YAXXZ 0000000039aa3900 f   CryGameSpyStats.obj
 0001:000a2910       ??__ECryUserInvalidID@@YAXXZ 0000000039aa3910 f   CryGameSpyVoice.obj
 0001:000a2920       ??__ECryUserInvalidID@@YAXXZ 0000000039aa3920 f   CryLANLobby.obj
 0001:000a2930       ??__ECryUserInvalidID@@YAXXZ 0000000039aa3930 f   CryLANMatchMaking.obj
 0001:000a2940       ??__ECrySessionInvalidID@@YAXXZ 0000000039aa3940 f   CryLANMatchMaking.obj
 0001:000a2950       ??__ECryUserInvalidID@@YAXXZ 0000000039aa3950 f   LobbyCVars.obj
 0001:000a2960       ??__ECryUserInvalidID@@YAXXZ 0000000039aa3960 f   CryPSNMatchMaking.obj
 0001:000a2970       ??__ECryUserInvalidID@@YAXXZ 0000000039aa3970 f   CryPSNStats.obj
 0001:000a2980       ??__EautoInitializer@@YAXXZ 0000000039aa3980 f   StdAfx.obj
 0001:000a29e0       ??__ECryUserInvalidID@@YAXXZ 0000000039aa39e0 f   StdAfx.obj
 0001:000a29f0       ??__ECrySessionInvalidID@@YAXXZ 0000000039aa39f0 f   StdAfx.obj
 0001:000a2a00       ??__FCryUserInvalidID@@YAXXZ 0000000039aa3a00 f   CryDedicatedServer.obj
 0001:000a2a50       ??__FCryUserInvalidID@@YAXXZ 0000000039aa3a50 f   CryDedicatedServerArbitrator.obj
 0001:000a2ab0       ??__FCryUserInvalidID@@YAXXZ 0000000039aa3ab0 f   CryFriends.obj
 0001:000a2b00       ??__FCryUserInvalidID@@YAXXZ 0000000039aa3b00 f   CryFriendsManagement.obj
 0001:000a2b50       ??__FCryUserInvalidID@@YAXXZ 0000000039aa3b50 f   CryHostMigration.obj
 0001:000a2ba0       ??__Fg_time@@YAXXZ         0000000039aa3ba0 f   CryLobby.obj
 0001:000a2bb0       ??__FCryUserInvalidID@@YAXXZ 0000000039aa3bb0 f   CryLobby.obj
 0001:000a2c00       ??__F?s_factory@CFactory@CEngineModule_CryLobby@@0V12@A@@YAXXZ 0000000039aa3c00 f   CryLobbyDLL.obj
 0001:000a2c30       ??__Fg_system_event_listener_crylobby@@YAXXZ 0000000039aa3c30 f   CryLobbyDLL.obj
 0001:000a2c80       ??__FCryUserInvalidID@@YAXXZ 0000000039aa3c80 f   CryLobbyUI.obj
 0001:000a2cd0       ??__FCrySessionInvalidID@@YAXXZ 0000000039aa3cd0 f   CryMatchMaking.obj
 0001:000a2d20       ??__FCryUserInvalidID@@YAXXZ 0000000039aa3d20 f   CryMatchMaking.obj
 0001:000a2d70       ??__FCryUserInvalidID@@YAXXZ 0000000039aa3d70 f   CryRebroadcaster.obj
 0001:000a2dc0       ??__FCryUserInvalidID@@YAXXZ 0000000039aa3dc0 f   CryStats.obj
 0001:000a2e10       ??__FCryUserInvalidID@@YAXXZ 0000000039aa3e10 f   CryVoice.obj
 0001:000a2e60       ??__FCryUserInvalidID@@YAXXZ 0000000039aa3e60 f   GameSpySBQR2AvailabilityCheck.obj
 0001:000a2eb0       ??__FCryUserInvalidID@@YAXXZ 0000000039aa3eb0 f   GameSpySBQR2Core.obj
 0001:000a2f00       ??__F?s_pDetectTask@CGameSpySBQR2NATNegotiation@@0V?$_smart_ptr@USDetectTask@CGameSpySBQR2NATNegotiation@@@@A@@YAXXZ 0000000039aa3f00 f   GameSpySBQR2NatNegotiation.obj
 0001:000a2f50       ??__FCryUserInvalidID@@YAXXZ 0000000039aa3f50 f   GameSpySBQR2NatNegotiation.obj
 0001:000a2fa0       ??__FCryUserInvalidID@@YAXXZ 0000000039aa3fa0 f   GameSpySBQR2Sake.obj
 0001:000a2ff0       ??__FCryUserInvalidID@@YAXXZ 0000000039aa3ff0 f   GameSpySDK.obj
 0001:000a3040       ??__FCryUserInvalidID@@YAXXZ 0000000039aa4040 f   CryGameSpySBQR2DLCStore.obj
 0001:000a3090       ??__FCrySessionInvalidID@@YAXXZ 0000000039aa4090 f   CryGameSpySBQR2Friends.obj
 0001:000a30e0       ??__FCryUserInvalidID@@YAXXZ 0000000039aa40e0 f   CryGameSpySBQR2Friends.obj
 0001:000a3130       ??__FCryUserInvalidID@@YAXXZ 0000000039aa4130 f   CryGameSpySBQR2FriendsManagement.obj
 0001:000a3180       ??__FCryUserInvalidID@@YAXXZ 0000000039aa4180 f   CryGameSpySBQR2Lobby.obj
 0001:000a31d0       ??__FCrySessionInvalidID@@YAXXZ 0000000039aa41d0 f   CryGameSpySBQR2LobbyUI.obj
 0001:000a3220       ??__FCryUserInvalidID@@YAXXZ 0000000039aa4220 f   CryGameSpySBQR2LobbyUI.obj
 0001:000a3270       ??__FCrySessionInvalidID@@YAXXZ 0000000039aa4270 f   CryGameSpySBQR2MatchMaking.obj
 0001:000a32c0       ??__FCryUserInvalidID@@YAXXZ 0000000039aa42c0 f   CryGameSpySBQR2MatchMaking.obj
 0001:000a3310       ??__FCryUserInvalidID@@YAXXZ 0000000039aa4310 f   CryGameSpySBQR2SignIn.obj
 0001:000a3360       ??__FCryUserInvalidID@@YAXXZ 0000000039aa4360 f   CryGameSpySBQR2Stats.obj
 0001:000a33b0       ??__FCryUserInvalidID@@YAXXZ 0000000039aa43b0 f   CryGameSpySBQR2Voice.obj
 0001:000a3400       ??__FCryUserInvalidID@@YAXXZ 0000000039aa4400 f   GameSpySBQR2GPConnection.obj
 0001:000a3450       ??__FCryUserInvalidID@@YAXXZ 0000000039aa4450 f   CryGameSpyMatchMaking.obj
 0001:000a34a0       ??__FCryUserInvalidID@@YAXXZ 0000000039aa44a0 f   CryGameSpyStats.obj
 0001:000a34f0       ??__FCryUserInvalidID@@YAXXZ 0000000039aa44f0 f   CryGameSpyVoice.obj
 0001:000a3540       ??__FCryUserInvalidID@@YAXXZ 0000000039aa4540 f   CryLANLobby.obj
 0001:000a3590       ??__FCrySessionInvalidID@@YAXXZ 0000000039aa4590 f   CryLANMatchMaking.obj
 0001:000a35e0       ??__FCryUserInvalidID@@YAXXZ 0000000039aa45e0 f   CryLANMatchMaking.obj
 0001:000a3630       ??__FCryUserInvalidID@@YAXXZ 0000000039aa4630 f   LobbyCVars.obj
 0001:000a3680       ??__FCryUserInvalidID@@YAXXZ 0000000039aa4680 f   CryPSNMatchMaking.obj
 0001:000a36d0       ??__FCryUserInvalidID@@YAXXZ 0000000039aa46d0 f   CryPSNStats.obj
 0001:000a3720       ??__FautoInitializer@@YAXXZ 0000000039aa4720 f   StdAfx.obj
 0001:000a3730       ??__FCrySessionInvalidID@@YAXXZ 0000000039aa4730 f   StdAfx.obj
 0001:000a3780       ??__FCryUserInvalidID@@YAXXZ 0000000039aa4780 f   StdAfx.obj
